 luafar3

 Timestamp is 5b66fa50 (Sun Aug  5 16:23:28 2018)

 Preferred load address is 0000000180000000

 Start         Length     Name                   Class
 0001:00000000 00000008H .CRT$XCA                CODE
 0001:00000008 00000008H .CRT$XCZ                CODE
 0001:00000010 00000008H .CRT$XIA                CODE
 0001:00000018 00000018H .CRT$XIC                CODE
 0001:00000030 00000008H .CRT$XIZ                CODE
 0001:00000038 00000008H .CRT$XPA                CODE
 0001:00000040 00000018H .CRT$XPX                CODE
 0001:00000058 00000008H .CRT$XPXA               CODE
 0001:00000060 00000008H .CRT$XPZ                CODE
 0001:00000068 00000008H .CRT$XTA                CODE
 0001:00000070 00000010H .CRT$XTZ                CODE
 0001:00000078 00000000H .gfids$y                CODE
 0001:00000080 00019340H .rdata                  CODE
 0001:000193c0 00000000H .rdata$r                CODE
 0001:000193c0 00000280H .rdata$zzzdbg           CODE
 0001:00019640 00000008H .rtc$IAA                CODE
 0001:00019648 00000008H .rtc$IZZ                CODE
 0001:00019650 00000008H .rtc$TAA                CODE
 0001:00019658 00000008H .rtc$TZZ                CODE
 0001:00019660 00040490H .text$mn                CODE
 0001:00059af0 00000020H .text$mn$00             CODE
 0001:00059b10 00000490H .text$x                 CODE
 0001:00059fa0 000033d0H .xdata                  CODE
 0001:0005d368 00000000H .xdata$x                CODE
 0001:0005d370 00000482H .edata                  CODE
 0002:00000000 00005f40H .data                   DATA
 0002:00005f40 00000000H .data$r                 DATA
 0002:00005f40 00001230H .bss                    DATA
 0003:00000000 00003b1cH .pdata                  DATA
 0004:00000000 000006f0H .idata$5                DATA
 0004:000006f0 00000010H .00cfg                  DATA
 0004:00000700 00000078H .idata$2                DATA
 0004:00000778 00000018H .idata$3                DATA
 0004:00000790 000006f0H .idata$4                DATA
 0004:00000e80 00000f50H .idata$6                DATA
 0005:00000000 00000060H .rsrc$01                DATA
 0005:00000060 00000358H .rsrc$02                DATA

  Address         Publics by Value              Rva+Base               Lib:Object

 0000:00000000       __guard_longjmp_count      0000000000000000     <absolute>
 0000:00000000       __dynamic_value_reloc_table 0000000000000000     <absolute>
 0000:00000000       __guard_longjmp_table      0000000000000000     <absolute>
 0000:00000000       __guard_iat_table          0000000000000000     <absolute>
 0000:00000000       __hybrid_auxiliary_iat     0000000000000000     <absolute>
 0000:00000000       __guard_iat_count          0000000000000000     <absolute>
 0000:00000000       __guard_fids_count         0000000000000000     <absolute>
 0000:00000000       __enclave_config           0000000000000000     <absolute>
 0000:00000000       ___safe_se_handler_table   0000000000000000     <absolute>
 0000:00000000       ___safe_se_handler_count   0000000000000000     <absolute>
 0000:00000000       __hybrid_code_map          0000000000000000     <absolute>
 0000:00000000       __hybrid_code_map_count    0000000000000000     <absolute>
 0000:00000000       __guard_fids_table         0000000000000000     <absolute>
 0000:00000100       __guard_flags              0000000000000100     <absolute>
 0000:00000000       __ImageBase                0000000180000000     <linker-defined>
 0001:00000000       __xc_a                     0000000180001000     LIBCMT:initializers.obj
 0001:00000008       __xc_z                     0000000180001008     LIBCMT:initializers.obj
 0001:00000010       __xi_a                     0000000180001010     LIBCMT:initializers.obj
 0001:00000018       __acrt_stdio_initializer   0000000180001018     libucrt:stdio_initializer.obj
 0001:00000020       __acrt_multibyte_initializer 0000000180001020     libucrt:multibyte_initializer.obj
 0001:00000028       __acrt_tran_fma3_initializer 0000000180001028     libucrt:fma3_initializer.obj
 0001:00000030       __xi_z                     0000000180001030     LIBCMT:initializers.obj
 0001:00000038       __xp_a                     0000000180001038     LIBCMT:initializers.obj
 0001:00000040       __acrt_locale_terminator   0000000180001040     libucrt:locale_initializer.obj
 0001:00000048       __acrt_tmpfile_terminator  0000000180001048     libucrt:tmpfile_initializer.obj
 0001:00000050       __dcrt_console_output_terminator 0000000180001050     libucrt:console_output_initializer.obj
 0001:00000058       __acrt_stdio_terminator    0000000180001058     libucrt:stdio_initializer.obj
 0001:00000060       __xp_z                     0000000180001060     LIBCMT:initializers.obj
 0001:00000068       __xt_a                     0000000180001068     LIBCMT:initializers.obj
 0001:00000070       __xt_z                     0000000180001070     LIBCMT:initializers.obj
 0001:00000250       metatable_name             0000000180001250     bit64.obj
 0001:00000260       ??_C@_04JAOJMBA@bnot?$AA@  0000000180001260     bit64.obj
 0001:00000268       ??_C@_04BKGNPECA@band?$AA@ 0000000180001268     bit64.obj
 0001:00000270       ??_C@_03BBBGIIAC@bor?$AA@  0000000180001270     bit64.obj
 0001:00000274       ??_C@_04CKCGDDNF@bxor?$AA@ 0000000180001274     bit64.obj
 0001:0000027c       ??_C@_06ELFGPGBK@lshift?$AA@ 000000018000127c     bit64.obj
 0001:00000284       ??_C@_06HMLHBBIJ@rshift?$AA@ 0000000180001284     bit64.obj
 0001:00000290       ??_C@_07JILILBLL@arshift?$AA@ 0000000180001290     bit64.obj
 0001:00000298       ??_C@_03CLCAEGCJ@new?$AA@  0000000180001298     bit64.obj
 0001:0000029c       ??_C@_03BDGOHNNK@add?$AA@  000000018000129c     bit64.obj
 0001:000002a0       ??_C@_03KCMAIMAP@sub?$AA@  00000001800012a0     bit64.obj
 0001:000002a4       ??_C@_03IMIFIBCN@mul?$AA@  00000001800012a4     bit64.obj
 0001:000002a8       ??_C@_03FEJMGOGI@div?$AA@  00000001800012a8     bit64.obj
 0001:000002ac       ??_C@_03FFONCNID@mod?$AA@  00000001800012ac     bit64.obj
 0001:000002b0       ??_C@_02HIIGGHJB@eq?$AA@   00000001800012b0     bit64.obj
 0001:000002b4       ??_C@_02KCAKIFL@lt?$AA@    00000001800012b4     bit64.obj
 0001:000002b8       ??_C@_02FJPJILEL@le?$AA@   00000001800012b8     bit64.obj
 0001:000002bc       ??_C@_04GPMDFGEJ@type?$AA@ 00000001800012bc     bit64.obj
 0001:000002c4       ??_C@_05MEHDOBFN@__add?$AA@ 00000001800012c4     bit64.obj
 0001:000002cc       ??_C@_05HFNNBAII@__sub?$AA@ 00000001800012cc     bit64.obj
 0001:000002d4       ??_C@_05FLJIBNKK@__mul?$AA@ 00000001800012d4     bit64.obj
 0001:000002dc       ??_C@_05IDIBPCOP@__div?$AA@ 00000001800012dc     bit64.obj
 0001:000002e4       ??_C@_05ICPALBAE@__mod?$AA@ 00000001800012e4     bit64.obj
 0001:000002ec       ??_C@_05MHFNBPAK@__unm?$AA@ 00000001800012ec     bit64.obj
 0001:000002f4       ??_C@_04GIMIAOHA@__eq?$AA@ 00000001800012f4     bit64.obj
 0001:000002fc       ??_C@_04BKGOMBLK@__lt?$AA@ 00000001800012fc     bit64.obj
 0001:00000304       ??_C@_04EJLHOCKK@__le?$AA@ 0000000180001304     bit64.obj
 0001:00000310       ??_C@_0L@HDFPAPPH@__tostring?$AA@ 0000000180001310     bit64.obj
 0001:00000320       ??_C@_09GPALILFO@bad?5int64?$AA@ 0000000180001320     bit64.obj
 0001:0000032c       ??_C@_05LLAMLEHD@?$CFI64d?$AA@ 000000018000132c     bit64.obj
 0001:00000334       ??_C@_05OALCLICP@bit64?$AA@ 0000000180001334     bit64.obj
 0001:00000340       __real@433fffffffffffff    0000000180001340     bit64.obj
 0001:00000350       __xmm@80000000000000008000000000000000 0000000180001350     bit64.obj
 0001:00000bf0       COLLECTOR_FD               0000000180001bf0     exported.obj
 0001:00000c08       COLLECTOR_OPI              0000000180001c08     exported.obj
 0001:00000c20       COLLECTOR_PI               0000000180001c20     exported.obj
 0001:00000c38       KEY_OBJECT                 0000000180001c38     exported.obj
 0001:00000c40       ??_C@_05GFCDIDHO@debug?$AA@ 0000000180001c40     exported.obj
 0001:00000c48       ??_C@_09GPFEECNC@traceback?$AA@ 0000000180001c48     exported.obj
 0001:00000c54       ??_C@_06NKNNMLDJ@export?$AA@ 0000000180001c54     exported.obj
 0001:00000c60       ??_C@_07PCNKBAGB@OnError?$AA@ 0000000180001c60     exported.obj
 0001:00000c68       ??_C@_0N@NJMIGDDL@CreationTime?$AA@ 0000000180001c68     exported.obj
 0001:00000c78       ??_C@_0P@MFHPCDDH@LastAccessTime?$AA@ 0000000180001c78     exported.obj
 0001:00000c88       ??_C@_0O@FCFNCAHK@LastWriteTime?$AA@ 0000000180001c88     exported.obj
 0001:00000c98       ??_C@_0L@FCILKIIG@ChangeTime?$AA@ 0000000180001c98     exported.obj
 0001:00000ca8       ??_C@_08BHIEONMC@FileSize?$AA@ 0000000180001ca8     exported.obj
 0001:00000cb8       ??_C@_0P@JBACEJLL@AllocationSize?$AA@ 0000000180001cb8     exported.obj
 0001:00000cc8       ??_C@_05BOOEKJH@Flags?$AA@ 0000000180001cc8     exported.obj
 0001:00000cd0       ??_C@_0O@DLGJHFNH@NumberOfLinks?$AA@ 0000000180001cd0     exported.obj
 0001:00000ce0       ??_C@_05MHNOECFO@CRC32?$AA@ 0000000180001ce0     exported.obj
 0001:00000ce8       ??_C@_08FDCJCDOL@FileName?$AA@ 0000000180001ce8     exported.obj
 0001:00000cf8       ??_C@_0BC@COCBGKAE@AlternateFileName?$AA@ 0000000180001cf8     exported.obj
 0001:00000d10       ??_C@_0M@OHKMKKDH@Description?$AA@ 0000000180001d10     exported.obj
 0001:00000d1c       ??_C@_05HDCNEILF@Owner?$AA@ 0000000180001d1c     exported.obj
 0001:00000d28       ??_C@_0BB@OKGMKOG@CustomColumnData?$AA@ 0000000180001d28     exported.obj
 0001:00000d3c       ??_C@_11LOCGONAA@?$AA?$AA@ 0000000180001d3c     exported.obj
 0001:00000d40       ??_C@_08JNHPECBG@UserData?$AA@ 0000000180001d40     exported.obj
 0001:00000d50       ??_C@_0M@DFMHDHBL@GetFindData?$AA@ 0000000180001d50     exported.obj
 0001:00000d60       ??_C@_08FFPEEIHA@GetFiles?$AA@ 0000000180001d60     exported.obj
 0001:00000d70       ??_C@_0BC@IECOKJFL@GetFiles?4DestPath?$AA@ 0000000180001d70     exported.obj
 0001:00000d84       ??_C@_05LFOKGKBN@?$DMboot?$AA@ 0000000180001d84     exported.obj
 0001:00000d8c       ??_C@_15CBMDENPJ@?$AA?4?$AA?9?$AA?$AA@ 0000000180001d8c     exported.obj
 0001:00000d98       ??_C@_07KNEGBPNO@package?$AA@ 0000000180001d98     exported.obj
 0001:00000da0       ??_C@_07GCEAJMEA@preload?$AA@ 0000000180001da0     exported.obj
 0001:00000da8       ??_C@_19BCNABNAK@?$AA?4?$AAl?$AAu?$AAa?$AA?$AA@ 0000000180001da8     exported.obj
 0001:00000db4       ??_C@_13BPINEIPE@?$AAr?$AA?$AA@ 0000000180001db4     exported.obj
 0001:00000db8       ??_C@_1DC@PABHCCON@?$AAD?$AAe?$AAf?$AAa?$AAu?$AAl?$AAt?$AA?5?$AAs?$AAc?$AAr?$AAi?$AAp?$AAt?$AA?5?$AAn?$AAo?$AAt?$AA?5?$AAf?$AAo?$AAu?$AAn?$AAd?$AA?$AA@ 0000000180001db8     exported.obj
 0001:00000dec       ??_C@_03JEOKDCFP@far?$AA@  0000000180001dec     exported.obj
 0001:00000df0       ??_C@_0BE@HCPAIELH@ReloadDefaultScript?$AA@ 0000000180001df0     exported.obj
 0001:00000e08       ??_C@_0L@OCPPMCCK@StructSize?$AA@ 0000000180001e08     exported.obj
 0001:00000e14       ??_C@_06LBMCOACO@Buffer?$AA@ 0000000180001e14     exported.obj
 0001:00000e1c       ??_C@_06EPIAKPGD@OpMode?$AA@ 0000000180001e1c     exported.obj
 0001:00000e28       ??_C@_07GDADDFBD@Analyse?$AA@ 0000000180001e28     exported.obj
 0001:00000e30       ??_C@_0BB@CKIGBGLB@GetOpenPanelInfo?$AA@ 0000000180001e30     exported.obj
 0001:00000e48       ??_C@_08KDMNIFGM@FreeSize?$AA@ 0000000180001e48     exported.obj
 0001:00000e58       ??_C@_08PAJOMFPO@HostFile?$AA@ 0000000180001e58     exported.obj
 0001:00000e64       ??_C@_06IBPEEEAJ@CurDir?$AA@ 0000000180001e64     exported.obj
 0001:00000e6c       ??_C@_06PEPCFMNJ@Format?$AA@ 0000000180001e6c     exported.obj
 0001:00000e78       ??_C@_0L@CMHIOLLB@PanelTitle?$AA@ 0000000180001e78     exported.obj
 0001:00000e88       ??_C@_09PMEOAIAA@InfoLines?$AA@ 0000000180001e88     exported.obj
 0001:00000e98       ??_C@_0BA@BLCGOCOG@InfoLinesNumber?$AA@ 0000000180001e98     exported.obj
 0001:00000ea8       ??_C@_04OJAHODMC@Text?$AA@ 0000000180001ea8     exported.obj
 0001:00000eb0       ??_C@_04DICKPMGH@Data?$AA@ 0000000180001eb0     exported.obj
 0001:00000eb8       ??_C@_0L@FPEHOFAI@DescrFiles?$AA@ 0000000180001eb8     exported.obj
 0001:00000ec8       ??_C@_0BA@BBOGKOKF@PanelModesArray?$AA@ 0000000180001ec8     exported.obj
 0001:00000ed8       ??_C@_0BB@LFNABPEF@PanelModesNumber?$AA@ 0000000180001ed8     exported.obj
 0001:00000ef0       ??_C@_0M@KDJPJFOF@ColumnTypes?$AA@ 0000000180001ef0     exported.obj
 0001:00000f00       ??_C@_0N@ILFJPGHI@ColumnWidths?$AA@ 0000000180001f00     exported.obj
 0001:00000f10       ??_C@_0BC@KELOOKNK@StatusColumnTypes?$AA@ 0000000180001f10     exported.obj
 0001:00000f28       ??_C@_0BD@DNDIPKDK@StatusColumnWidths?$AA@ 0000000180001f28     exported.obj
 0001:00000f40       ??_C@_0N@EHCEJHEE@ColumnTitles?$AA@ 0000000180001f40     exported.obj
 0001:00000f50       ??_C@_0P@BEEDPJDK@StartPanelMode?$AA@ 0000000180001f50     exported.obj
 0001:00000f60       ??_C@_0O@NIFKFGBJ@StartSortMode?$AA@ 0000000180001f60     exported.obj
 0001:00000f70       ??_C@_0P@KMACBLNK@StartSortOrder?$AA@ 0000000180001f70     exported.obj
 0001:00000f80       ??_C@_06ONGFDHIA@KeyBar?$AA@ 0000000180001f80     exported.obj
 0001:00000f88       ??_C@_0P@PKDBPEJI@VirtualKeyCode?$AA@ 0000000180001f88     exported.obj
 0001:00000f98       ??_C@_0BA@MFFHAKP@ControlKeyState?$AA@ 0000000180001f98     exported.obj
 0001:00000fa8       ??_C@_08DGDJEKCP@LongText?$AA@ 0000000180001fa8     exported.obj
 0001:00000fb8       ??_C@_0N@IHDKLODA@ShortcutData?$AA@ 0000000180001fb8     exported.obj
 0001:00000fc8       ??_C@_05HIFJDKLD@array?$AA@ 0000000180001fc8     exported.obj
 0001:00000fd0       ??_C@_01EFFIKLCJ@n?$AA@    0000000180001fd0     exported.obj
 0001:00000fd2       ??_C@_00CNPNBAHC@?$AA@     0000000180001fd2     exported.obj
 0001:00000fd4       ??_C@_04DNCDCIAE@Open?$AA@ 0000000180001fd4     exported.obj
 0001:00000fdc       ??_C@_04OPJIDECA@hDlg?$AA@ 0000000180001fdc     exported.obj
 0001:00000fe4       ??_C@_06BNNOMDLO@Handle?$AA@ 0000000180001fe4     exported.obj
 0001:00000fec       ??_C@_05LNOAKADA@panel?$AA@ 0000000180001fec     exported.obj
 0001:00000ff8       ??_C@_0L@JMPDJFBN@ClosePanel?$AA@ 0000000180001ff8     exported.obj
 0001:00001008       ??_C@_07MBOMJGGF@Compare?$AA@ 0000000180002008     exported.obj
 0001:00001010       ??_C@_09NANCCILE@Configure?$AA@ 0000000180002010     exported.obj
 0001:00001020       ??_C@_0M@MMKKMEFA@DeleteFiles?$AA@ 0000000180002020     exported.obj
 0001:00001030       ??_C@_0O@GLLEDHJA@MakeDirectory?$AA@ 0000000180002030     exported.obj
 0001:00001040       ??_C@_0BD@PJNONGDB@MakeDirectory?4Name?$AA@ 0000000180002040     exported.obj
 0001:00001058       ??_C@_0BC@COPMJGBI@ProcessPanelEvent?$AA@ 0000000180002058     exported.obj
 0001:00001070       ??_C@_0BA@DPJAKFGC@ProcessHostFile?$AA@ 0000000180002070     exported.obj
 0001:00001080       ??_C@_0BC@HOBKGBBM@ProcessPanelInput?$AA@ 0000000180002080     exported.obj
 0001:00001098       ??_C@_08OBOOFGOD@PutFiles?$AA@ 0000000180002098     exported.obj
 0001:000010a8       ??_C@_0N@KCFEBPAO@SetDirectory?$AA@ 00000001800020a8     exported.obj
 0001:000010b8       ??_C@_0M@PNOHHCCH@SetFindList?$AA@ 00000001800020b8     exported.obj
 0001:000010c8       ??_C@_07EACELFAO@ExitFAR?$AA@ 00000001800020c8     exported.obj
 0001:000010d0       ??_C@_0O@OBCKADMD@GetPluginInfo?$AA@ 00000001800020d0     exported.obj
 0001:000010e0       ??_C@_0O@GDMHGAFH@CommandPrefix?$AA@ 00000001800020e0     exported.obj
 0001:000010f0       ??_C@_0O@PHBKMNMJ@DiskMenuGuids?$AA@ 00000001800020f0     exported.obj
 0001:00001100       ??_C@_0BA@NLBDFPEO@DiskMenuStrings?$AA@ 0000000180002100     exported.obj
 0001:00001110       ??_C@_0BA@FOMPNLJF@PluginMenuGuids?$AA@ 0000000180002110     exported.obj
 0001:00001120       ??_C@_0BC@DJMJFBJC@PluginMenuStrings?$AA@ 0000000180002120     exported.obj
 0001:00001138       ??_C@_0BC@ILBHAHCH@PluginConfigGuids?$AA@ 0000000180002138     exported.obj
 0001:00001150       ??_C@_0BE@GAFPNGIP@PluginConfigStrings?$AA@ 0000000180002150     exported.obj
 0001:00001168       ??_C@_0BD@DECJPBBK@ProcessEditorInput?$AA@ 0000000180002168     exported.obj
 0001:00001180       ??_C@_0BD@GEMPAGBO@ProcessEditorEvent?$AA@ 0000000180002180     exported.obj
 0001:00001194       ??_C@_04KOACHJEN@Type?$AA@ 0000000180002194     exported.obj
 0001:000011a0       ??_C@_0N@EKPHGDMI@StringNumber?$AA@ 00000001800021a0     exported.obj
 0001:000011b0       ??_C@_07MOCFLHCN@FileEOL?$AA@ 00000001800021b0     exported.obj
 0001:000011b8       ??_C@_08DOHJINHB@CodePage?$AA@ 00000001800021b8     exported.obj
 0001:000011c8       ??_C@_0BD@GGKMLEJG@ProcessViewerEvent?$AA@ 00000001800021c8     exported.obj
 0001:000011e0       ??_C@_0BD@FNHBEIC@ProcessDialogEvent?$AA@ 00000001800021e0     exported.obj
 0001:000011f4       ??_C@_06CPBJDKAC@Param2?$AA@ 00000001800021f4     exported.obj
 0001:000011fc       ??_C@_06EDEGJMB@Param1?$AA@ 00000001800021fc     exported.obj
 0001:00001204       ??_C@_03MLMOILGK@Msg?$AA@  0000000180002204     exported.obj
 0001:00001208       ??_C@_0BE@LHJGGGHN@ProcessSynchroEvent?$AA@ 0000000180002208     exported.obj
 0001:00001220       ??_C@_0BB@PHIEFGHD@GetContentFields?$AA@ 0000000180002220     exported.obj
 0001:00001238       ??_C@_0P@DPJDPMPI@GetContentData?$AA@ 0000000180002238     exported.obj
 0001:00001248       ??_C@_0N@DDJEHLKE@?$DM_globalinfo?$AA@ 0000000180002248     exported.obj
 0001:00001258       ??_C@_1CA@IBKDMBNJ@?$AA_?$AAg?$AAl?$AAo?$AAb?$AAa?$AAl?$AAi?$AAn?$AAf?$AAo?$AA?4?$AAl?$AAu?$AAa?$AA?$AA@ 0000000180002258     exported.obj
 0001:00001278       ??_C@_0O@GJMOPLGM@GetGlobalInfo?$AA@ 0000000180002278     exported.obj
 0001:00001288       ??_C@_0O@CALOEOI@MinFarVersion?$AA@ 0000000180002288     exported.obj
 0001:00001298       ??_C@_07NGFJPNPN@Version?$AA@ 0000000180002298     exported.obj
 0001:000012a0       ??_C@_04MJHIICBJ@Guid?$AA@ 00000001800022a0     exported.obj
 0001:000012a8       ??_C@_05PABKJLOM@Title?$AA@ 00000001800022a8     exported.obj
 0001:000012b0       ??_C@_06HHECMMLE@Author?$AA@ 00000001800022b0     exported.obj
 0001:000012b8       ??_C@_0BE@DONMOPMJ@ProcessConsoleInput?$AA@ 00000001800022b8     exported.obj
 0001:000012d0       __real@43e0000000000000    00000001800022d0     exported.obj
 0001:000012d8       __real@bff0000000000000    00000001800022d8     exported.obj
 0001:00001b60       Vals                       0000000180002b60     flags.obj
 0001:000031a8       ??_C@_0BI@IDKIJMME@FARMANAGERVERSION_MAJOR?$AA@ 00000001800041a8     flags.obj
 0001:000031c0       ??_C@_0BI@DMLKEAFC@FARMANAGERVERSION_MINOR?$AA@ 00000001800041c0     flags.obj
 0001:000031d8       ??_C@_0BL@NMALNAFP@FARMANAGERVERSION_REVISION?$AA@ 00000001800041d8     flags.obj
 0001:000031f8       ??_C@_0BI@OLPFLLDD@FARMANAGERVERSION_BUILD?$AA@ 00000001800041f8     flags.obj
 0001:00003210       ??_C@_0BI@MOOFLFPC@FARMANAGERVERSION_STAGE?$AA@ 0000000180004210     flags.obj
 0001:00003228       ??_C@_0L@MIDBGFJO@CP_UNICODE?$AA@ 0000000180004228     flags.obj
 0001:00003238       ??_C@_0O@MNMCMEJH@CP_REVERSEBOM?$AA@ 0000000180004238     flags.obj
 0001:00003248       ??_C@_0L@JDNPCEDH@CP_DEFAULT?$AA@ 0000000180004248     flags.obj
 0001:00003258       ??_C@_0M@OMCMFJHA@CP_REDETECT?$AA@ 0000000180004258     flags.obj
 0001:00003268       ??_C@_09MNAPNKKC@INDEXMASK?$AA@ 0000000180004268     flags.obj
 0001:00003278       ??_C@_09BLFIDJLF@COLORMASK?$AA@ 0000000180004278     flags.obj
 0001:00003288       ??_C@_09ENNBLPJC@ALPHAMASK?$AA@ 0000000180004288     flags.obj
 0001:00003298       ??_C@_0L@EHFOPLFD@PANEL_NONE?$AA@ 0000000180004298     flags.obj
 0001:000032a8       ??_C@_0N@LPMKALBG@PANEL_ACTIVE?$AA@ 00000001800042a8     flags.obj
 0001:000032b8       ??_C@_0O@HPKEABPN@PANEL_PASSIVE?$AA@ 00000001800042b8     flags.obj
 0001:000032c8       ??_C@_0L@GOEBPENN@PANEL_STOP?$AA@ 00000001800042c8     flags.obj
 0001:000032d8       ??_C@_0N@HLIFAAPJ@EEREDRAW_ALL?$AA@ 00000001800042d8     flags.obj
 0001:000032e8       ??_C@_0P@NHNDIKJ@CURRENT_EDITOR?$AA@ 00000001800042e8     flags.obj
 0001:000032f8       ??_C@_0BN@PPNDCHHA@EDITOR_COLOR_NORMAL_PRIORITY?$AA@ 00000001800042f8     flags.obj
 0001:00003318       ??_C@_07MGGAEAFF@DI_TEXT?$AA@ 0000000180004318     flags.obj
 0001:00003320       ??_C@_08HODBDEHE@DI_VTEXT?$AA@ 0000000180004320     flags.obj
 0001:00003330       ??_C@_0N@IGKKGFMF@DI_SINGLEBOX?$AA@ 0000000180004330     flags.obj
 0001:00003340       ??_C@_0N@EDCLIEAE@DI_DOUBLEBOX?$AA@ 0000000180004340     flags.obj
 0001:00003350       ??_C@_07DOLIFAEF@DI_EDIT?$AA@ 0000000180004350     flags.obj
 0001:00003358       ??_C@_0L@EOMEIIFM@DI_PSWEDIT?$AA@ 0000000180004358     flags.obj
 0001:00003368       ??_C@_0L@MGOIMBKF@DI_FIXEDIT?$AA@ 0000000180004368     flags.obj
 0001:00003378       ??_C@_09GGAEMAPJ@DI_BUTTON?$AA@ 0000000180004378     flags.obj
 0001:00003388       ??_C@_0M@MHFHGPHJ@DI_CHECKBOX?$AA@ 0000000180004388     flags.obj
 0001:00003398       ??_C@_0P@GIPCGMBE@DI_RADIOBUTTON?$AA@ 0000000180004398     flags.obj
 0001:000033a8       ??_C@_0M@MAKBFNGC@DI_COMBOBOX?$AA@ 00000001800043a8     flags.obj
 0001:000033b8       ??_C@_0L@ONDMPPPO@DI_LISTBOX?$AA@ 00000001800043b8     flags.obj
 0001:000033c8       ??_C@_0P@GDJDPEIK@DI_USERCONTROL?$AA@ 00000001800043c8     flags.obj
 0001:000033d8       ??_C@_08KAEGOLOB@DM_FIRST?$AA@ 00000001800043d8     flags.obj
 0001:000033e8       ??_C@_08MJMBFJHA@DM_CLOSE?$AA@ 00000001800043e8     flags.obj
 0001:000033f8       ??_C@_09KLJOCKAA@DM_ENABLE?$AA@ 00000001800043f8     flags.obj
 0001:00003408       ??_C@_0BA@KAMJGFDG@DM_ENABLEREDRAW?$AA@ 0000000180004408     flags.obj
 0001:00003418       ??_C@_0O@FKGMMKLP@DM_GETDLGDATA?$AA@ 0000000180004418     flags.obj
 0001:00003428       ??_C@_0O@HEGKCPOI@DM_GETDLGITEM?$AA@ 0000000180004428     flags.obj
 0001:00003438       ??_C@_0O@BEHCGMCL@DM_GETDLGRECT?$AA@ 0000000180004438     flags.obj
 0001:00003448       ??_C@_0L@ELBDNLFO@DM_GETTEXT?$AA@ 0000000180004448     flags.obj
 0001:00003454       ??_C@_06IKGPEGEJ@DM_KEY?$AA@ 0000000180004454     flags.obj
 0001:00003460       ??_C@_0O@DIPLLJEH@DM_MOVEDIALOG?$AA@ 0000000180004460     flags.obj
 0001:00003470       ??_C@_0O@EEEDHNPG@DM_SETDLGDATA?$AA@ 0000000180004470     flags.obj
 0001:00003480       ??_C@_0O@GKEFJIKB@DM_SETDLGITEM?$AA@ 0000000180004480     flags.obj
 0001:00003490       ??_C@_0M@GOFGHDFK@DM_SETFOCUS?$AA@ 0000000180004490     flags.obj
 0001:000034a0       ??_C@_09ILPFEDOM@DM_REDRAW?$AA@ 00000001800044a0     flags.obj
 0001:000034b0       ??_C@_0L@LDOCOEIP@DM_SETTEXT?$AA@ 00000001800044b0     flags.obj
 0001:000034c0       ??_C@_0BE@LABEAIPD@DM_SETMAXTEXTLENGTH?$AA@ 00000001800044c0     flags.obj
 0001:000034d8       ??_C@_0O@BIFKIPIP@DM_SHOWDIALOG?$AA@ 00000001800044d8     flags.obj
 0001:000034e8       ??_C@_0M@JPHKGACH@DM_GETFOCUS?$AA@ 00000001800044e8     flags.obj
 0001:000034f8       ??_C@_0BA@NLMONBKJ@DM_GETCURSORPOS?$AA@ 00000001800044f8     flags.obj
 0001:00003508       ??_C@_0BA@KPHABNOF@DM_SETCURSORPOS?$AA@ 0000000180004508     flags.obj
 0001:00003518       ??_C@_0O@LGEKFPKK@DM_SETTEXTPTR?$AA@ 0000000180004518     flags.obj
 0001:00003528       ??_C@_0M@NCOJHJKI@DM_SHOWITEM?$AA@ 0000000180004528     flags.obj
 0001:00003538       ??_C@_0O@GKKCFHIM@DM_ADDHISTORY?$AA@ 0000000180004538     flags.obj
 0001:00003548       ??_C@_0M@MCEMDFMD@DM_GETCHECK?$AA@ 0000000180004548     flags.obj
 0001:00003558       ??_C@_0M@DDGACGLO@DM_SETCHECK?$AA@ 0000000180004558     flags.obj
 0001:00003568       ??_C@_0N@MEGOPFGK@DM_SET3STATE?$AA@ 0000000180004568     flags.obj
 0001:00003578       ??_C@_0M@GEPBDDNC@DM_LISTSORT?$AA@ 0000000180004578     flags.obj
 0001:00003588       ??_C@_0P@NFJNHAKH@DM_LISTGETITEM?$AA@ 0000000180004588     flags.obj
 0001:00003598       ??_C@_0BB@EEIMACNO@DM_LISTGETCURPOS?$AA@ 0000000180004598     flags.obj
 0001:000035b0       ??_C@_0BB@GKMJCDEM@DM_LISTSETCURPOS?$AA@ 00000001800045b0     flags.obj
 0001:000035c8       ??_C@_0O@NOPCAHGJ@DM_LISTDELETE?$AA@ 00000001800045c8     flags.obj
 0001:000035d8       ??_C@_0L@BMEAECNG@DM_LISTADD?$AA@ 00000001800045d8     flags.obj
 0001:000035e8       ??_C@_0O@HBHDMHP@DM_LISTADDSTR?$AA@ 00000001800045e8     flags.obj
 0001:000035f8       ??_C@_0O@PDFCNPKN@DM_LISTUPDATE?$AA@ 00000001800045f8     flags.obj
 0001:00003608       ??_C@_0O@GAAGMJJL@DM_LISTINSERT?$AA@ 0000000180004608     flags.obj
 0001:00003618       ??_C@_0BC@MIFCLOBD@DM_LISTFINDSTRING?$AA@ 0000000180004618     flags.obj
 0001:00003630       ??_C@_0M@EEAEBLKC@DM_LISTINFO?$AA@ 0000000180004630     flags.obj
 0001:00003640       ??_C@_0P@PLJLJFPA@DM_LISTGETDATA?$AA@ 0000000180004640     flags.obj
 0001:00003650       ??_C@_0P@DGKKKCB@DM_LISTSETDATA?$AA@ 0000000180004650     flags.obj
 0001:00003660       ??_C@_0BB@CELMNLLN@DM_LISTSETTITLES?$AA@ 0000000180004660     flags.obj
 0001:00003678       ??_C@_0BB@KPJPKCP@DM_LISTGETTITLES?$AA@ 0000000180004678     flags.obj
 0001:00003690       ??_C@_0BA@ICDJCFLE@DM_RESIZEDIALOG?$AA@ 0000000180004690     flags.obj
 0001:000036a0       ??_C@_0BD@CNGGHGJF@DM_SETITEMPOSITION?$AA@ 00000001800046a0     flags.obj
 0001:000036b8       ??_C@_0BF@JMINBGBA@DM_GETDROPDOWNOPENED?$AA@ 00000001800046b8     flags.obj
 0001:000036d0       ??_C@_0BF@LJIGJNAO@DM_SETDROPDOWNOPENED?$AA@ 00000001800046d0     flags.obj
 0001:000036e8       ??_C@_0O@NPDKADMJ@DM_SETHISTORY?$AA@ 00000001800046e8     flags.obj
 0001:000036f8       ??_C@_0BD@BPHAAEIM@DM_GETITEMPOSITION?$AA@ 00000001800046f8     flags.obj
 0001:00003710       ??_C@_0BC@BENFKLNH@DM_SETINPUTNOTIFY?$AA@ 0000000180004710     flags.obj
 0001:00003728       ??_C@_0BH@CFMLLNNM@DM_SETMOUSEEVENTNOTIFY?$AA@ 0000000180004728     flags.obj
 0001:00003740       ??_C@_0BF@IAGIACOD@DM_EDITUNCHANGEDFLAG?$AA@ 0000000180004740     flags.obj
 0001:00003758       ??_C@_0P@OJKNHIPN@DM_GETITEMDATA?$AA@ 0000000180004758     flags.obj
 0001:00003768       ??_C@_0P@OGLDKOHO@DM_SETITEMDATA?$AA@ 0000000180004768     flags.obj
 0001:00003778       ??_C@_0L@KNFAKFKE@DM_LISTSET?$AA@ 0000000180004778     flags.obj
 0001:00003788       ??_C@_0BB@EPMFHAFO@DM_GETCURSORSIZE?$AA@ 0000000180004788     flags.obj
 0001:000037a0       ??_C@_0BB@DANLMDCJ@DM_SETCURSORSIZE?$AA@ 00000001800047a0     flags.obj
 0001:000037b8       ??_C@_0BD@LAOOKGHD@DM_LISTGETDATASIZE?$AA@ 00000001800047b8     flags.obj
 0001:000037d0       ??_C@_0BA@BHGANJAP@DM_GETSELECTION?$AA@ 00000001800047d0     flags.obj
 0001:000037e0       ??_C@_0BA@GDNOBFED@DM_SETSELECTION?$AA@ 00000001800047e0     flags.obj
 0001:000037f0       ??_C@_0BD@FIHDGIGO@DM_GETEDITPOSITION?$AA@ 00000001800047f0     flags.obj
 0001:00003808       ??_C@_0BD@GKGFBKHH@DM_SETEDITPOSITION?$AA@ 0000000180004808     flags.obj
 0001:00003820       ??_C@_0BE@MCECGHBC@DM_SETCOMBOBOXEVENT?$AA@ 0000000180004820     flags.obj
 0001:00003838       ??_C@_0BE@KGBLNJKA@DM_GETCOMBOBOXEVENT?$AA@ 0000000180004838     flags.obj
 0001:00003850       ??_C@_0BD@CJEPBACF@DM_GETCONSTTEXTPTR?$AA@ 0000000180004850     flags.obj
 0001:00003868       ??_C@_0BD@HOOHICEG@DM_GETDLGITEMSHORT?$AA@ 0000000180004868     flags.obj
 0001:00003880       ??_C@_0BD@EMPBPAFP@DM_SETDLGITEMSHORT?$AA@ 0000000180004880     flags.obj
 0001:00003898       ??_C@_0BB@GAPFMPKE@DM_GETDIALOGINFO?$AA@ 0000000180004898     flags.obj
 0001:000038b0       ??_C@_0BC@KJOLMFGG@DM_GETDIALOGTITLE?$AA@ 00000001800048b0     flags.obj
 0001:000038c8       ??_C@_08COMJOMAC@DN_FIRST?$AA@ 00000001800048c8     flags.obj
 0001:000038d8       ??_C@_0M@NNNAPNMA@DN_BTNCLICK?$AA@ 00000001800048d8     flags.obj
 0001:000038e8       ??_C@_0BC@MJFJAANN@DN_CTLCOLORDIALOG?$AA@ 00000001800048e8     flags.obj
 0001:00003900       ??_C@_0BD@HFGBIBBL@DN_CTLCOLORDLGITEM?$AA@ 0000000180004900     flags.obj
 0001:00003918       ??_C@_0BD@JMFJPHPD@DN_CTLCOLORDLGLIST?$AA@ 0000000180004918     flags.obj
 0001:00003930       ??_C@_0O@NKBDPILK@DN_DRAWDIALOG?$AA@ 0000000180004930     flags.obj
 0001:00003940       ??_C@_0P@KGKEDPBI@DN_DRAWDLGITEM?$AA@ 0000000180004940     flags.obj
 0001:00003950       ??_C@_0O@JMKNGFLE@DN_EDITCHANGE?$AA@ 0000000180004950     flags.obj
 0001:00003960       ??_C@_0N@OCGKCPJF@DN_ENTERIDLE?$AA@ 0000000180004960     flags.obj
 0001:00003970       ??_C@_0M@JHFIBKOO@DN_GOTFOCUS?$AA@ 0000000180004970     flags.obj
 0001:00003980       ??_C@_07NJJEMKPA@DN_HELP?$AA@ 0000000180004980     flags.obj
 0001:00003988       ??_C@_09EDGJFAK@DN_HOTKEY?$AA@ 0000000180004988     flags.obj
 0001:00003998       ??_C@_0O@BJECHBCA@DN_INITDIALOG?$AA@ 0000000180004998     flags.obj
 0001:000039a8       ??_C@_0N@CHLLLNBO@DN_KILLFOCUS?$AA@ 00000001800049a8     flags.obj
 0001:000039b8       ??_C@_0O@CLPABIGO@DN_LISTCHANGE?$AA@ 00000001800049b8     flags.obj
 0001:000039c8       ??_C@_0L@MLMFBHN@DN_DRAGGED?$AA@ 00000001800049c8     flags.obj
 0001:000039d8       ??_C@_0BB@BOOOCAEG@DN_RESIZECONSOLE?$AA@ 00000001800049d8     flags.obj
 0001:000039f0       ??_C@_0BC@FHPPFLKG@DN_DRAWDIALOGDONE?$AA@ 00000001800049f0     flags.obj
 0001:00003a08       ??_C@_0O@EONPBNNP@DN_LISTHOTKEY?$AA@ 0000000180004a08     flags.obj
 0001:00003a18       ??_C@_08MDDLDGPO@DN_INPUT?$AA@ 0000000180004a18     flags.obj
 0001:00003a28       ??_C@_0BA@FGOGLDBC@DN_CONTROLINPUT?$AA@ 0000000180004a28     flags.obj
 0001:00003a38       ??_C@_08EHEOFOJD@DN_CLOSE?$AA@ 0000000180004a38     flags.obj
 0001:00003a48       ??_C@_0M@POIFBPFN@DN_GETVALUE?$AA@ 0000000180004a48     flags.obj
 0001:00003a58       ??_C@_0BC@MHCBFAAO@DN_DROPDOWNOPENED?$AA@ 0000000180004a58     flags.obj
 0001:00003a70       ??_C@_0BD@NGEKAPIF@DN_DRAWDLGITEMDONE?$AA@ 0000000180004a70     flags.obj
 0001:00003a88       ??_C@_07DIJJNCBA@DM_USER?$AA@ 0000000180004a88     flags.obj
 0001:00003a90       ??_C@_0BB@HLBBGMAN@BSTATE_UNCHECKED?$AA@ 0000000180004a90     flags.obj
 0001:00003aa8       ??_C@_0P@FALAMPGP@BSTATE_CHECKED?$AA@ 0000000180004aa8     flags.obj
 0001:00003ab8       ??_C@_0O@KBIFGGHO@BSTATE_3STATE?$AA@ 0000000180004ab8     flags.obj
 0001:00003ac8       ??_C@_0O@ILJOJGLD@BSTATE_TOGGLE?$AA@ 0000000180004ac8     flags.obj
 0001:00003ad8       ??_C@_08PPADCPCM@CBET_KEY?$AA@ 0000000180004ad8     flags.obj
 0001:00003ae8       ??_C@_0L@KHCLMGFJ@CBET_MOUSE?$AA@ 0000000180004ae8     flags.obj
 0001:00003af8       ??_C@_0BA@KNHGEBNE@PTYPE_FILEPANEL?$AA@ 0000000180004af8     flags.obj
 0001:00003b08       ??_C@_0BA@LPPHNHIG@PTYPE_TREEPANEL?$AA@ 0000000180004b08     flags.obj
 0001:00003b18       ??_C@_0BB@JBINOKAI@PTYPE_QVIEWPANEL?$AA@ 0000000180004b18     flags.obj
 0001:00003b30       ??_C@_0BA@NKMDEBG@PTYPE_INFOPANEL?$AA@ 0000000180004b30     flags.obj
 0001:00003b40       ??_C@_0L@OPHJOKKE@SM_DEFAULT?$AA@ 0000000180004b40     flags.obj
 0001:00003b50       ??_C@_0M@JGBFGGEA@SM_UNSORTED?$AA@ 0000000180004b50     flags.obj
 0001:00003b60       ??_C@_07KIFHAGIL@SM_NAME?$AA@ 0000000180004b60     flags.obj
 0001:00003b68       ??_C@_06GJJJNNFE@SM_EXT?$AA@ 0000000180004b68     flags.obj
 0001:00003b70       ??_C@_08FICJBKFN@SM_MTIME?$AA@ 0000000180004b70     flags.obj
 0001:00003b80       ??_C@_08GCCDHLCN@SM_CTIME?$AA@ 0000000180004b80     flags.obj
 0001:00003b90       ??_C@_08CPOLNKCG@SM_ATIME?$AA@ 0000000180004b90     flags.obj
 0001:00003ba0       ??_C@_07OMPKMIKC@SM_SIZE?$AA@ 0000000180004ba0     flags.obj
 0001:00003ba8       ??_C@_08BCBPOLMA@SM_DESCR?$AA@ 0000000180004ba8     flags.obj
 0001:00003bb8       ??_C@_08MEAGCMBB@SM_OWNER?$AA@ 0000000180004bb8     flags.obj
 0001:00003bc8       ??_C@_0BC@NKDBNAHD@SM_COMPRESSEDSIZE?$AA@ 0000000180004bc8     flags.obj
 0001:00003be0       ??_C@_0M@PKNLKFI@SM_NUMLINKS?$AA@ 0000000180004be0     flags.obj
 0001:00003bf0       ??_C@_0O@CCKEKPHL@SM_NUMSTREAMS?$AA@ 0000000180004bf0     flags.obj
 0001:00003c00       ??_C@_0P@PKGMDPMD@SM_STREAMSSIZE?$AA@ 0000000180004c00     flags.obj
 0001:00003c10       ??_C@_0M@OAFEBGNH@SM_FULLNAME?$AA@ 0000000180004c10     flags.obj
 0001:00003c20       ??_C@_09KFKGJDHC@SM_CHTIME?$AA@ 0000000180004c20     flags.obj
 0001:00003c30       ??_C@_08DOEDKINA@SM_COUNT?$AA@ 0000000180004c30     flags.obj
 0001:00003c40       ??_C@_0P@FEMAMJLE@EEC_OPEN_ERROR?$AA@ 0000000180004c40     flags.obj
 0001:00003c50       ??_C@_0N@GLMELIKF@EEC_MODIFIED?$AA@ 0000000180004c50     flags.obj
 0001:00003c60       ??_C@_0BB@HALKEFOL@EEC_NOT_MODIFIED?$AA@ 0000000180004c60     flags.obj
 0001:00003c78       ??_C@_0BI@CNPFKHKO@EEC_LOADING_INTERRUPTED?$AA@ 0000000180004c78     flags.obj
 0001:00003c90       ??_C@_0BK@PHBCABMB@ACTL_GETFARMANAGERVERSION?$AA@ 0000000180004c90     flags.obj
 0001:00003cb0       ??_C@_0N@DPABJDML@ACTL_WAITKEY?$AA@ 0000000180004cb0     flags.obj
 0001:00003cc0       ??_C@_0O@CEHHJAFD@ACTL_GETCOLOR?$AA@ 0000000180004cc0     flags.obj
 0001:00003cd0       ??_C@_0BD@OKPAACIK@ACTL_GETARRAYCOLOR?$AA@ 0000000180004cd0     flags.obj
 0001:00003ce8       ??_C@_0BD@DIFEEKNN@ACTL_GETWINDOWINFO?$AA@ 0000000180004ce8     flags.obj
 0001:00003d00       ??_C@_0BE@PJBIPKOD@ACTL_GETWINDOWCOUNT?$AA@ 0000000180004d00     flags.obj
 0001:00003d18       ??_C@_0BG@MNKPOEEN@ACTL_SETCURRENTWINDOW?$AA@ 0000000180004d18     flags.obj
 0001:00003d30       ??_C@_0M@IHHFGPPA@ACTL_COMMIT?$AA@ 0000000180004d30     flags.obj
 0001:00003d40       ??_C@_0BA@CLHFKJJP@ACTL_GETFARHWND?$AA@ 0000000180004d40     flags.obj
 0001:00003d50       ??_C@_0BD@JFOOLBPN@ACTL_SETARRAYCOLOR?$AA@ 0000000180004d50     flags.obj
 0001:00003d68       ??_C@_0P@JECKFIA@ACTL_REDRAWALL?$AA@ 0000000180004d68     flags.obj
 0001:00003d78       ??_C@_0N@DHPLJLHO@ACTL_SYNCHRO?$AA@ 0000000180004d78     flags.obj
 0001:00003d88       ??_C@_0BG@IJPADENB@ACTL_SETPROGRESSSTATE?$AA@ 0000000180004d88     flags.obj
 0001:00003da0       ??_C@_0BG@ICJFAPHK@ACTL_SETPROGRESSVALUE?$AA@ 0000000180004da0     flags.obj
 0001:00003db8       ??_C@_09HNDBKLDC@ACTL_QUIT?$AA@ 0000000180004db8     flags.obj
 0001:00003dc8       ??_C@_0BA@LJCPDIKK@ACTL_GETFARRECT?$AA@ 0000000180004dc8     flags.obj
 0001:00003dd8       ??_C@_0BC@FELBEIDG@ACTL_GETCURSORPOS?$AA@ 0000000180004dd8     flags.obj
 0001:00003df0       ??_C@_0BC@CAAPIEHK@ACTL_SETCURSORPOS?$AA@ 0000000180004df0     flags.obj
 0001:00003e08       ??_C@_0BE@NPJGMDBM@ACTL_PROGRESSNOTIFY?$AA@ 0000000180004e08     flags.obj
 0001:00003e20       ??_C@_0BD@IPKOEBIA@ACTL_GETWINDOWTYPE?$AA@ 0000000180004e20     flags.obj
 0001:00003e38       ??_C@_09CEDFMINA@MSSC_POST?$AA@ 0000000180004e38     flags.obj
 0001:00003e48       ??_C@_0L@MOADGAEB@MSSC_CHECK?$AA@ 0000000180004e48     flags.obj
 0001:00003e58       ??_C@_0BA@MMOAIEKP@MACROAREA_OTHER?$AA@ 0000000180004e58     flags.obj
 0001:00003e68       ??_C@_0BA@DEBOOAEB@MACROAREA_SHELL?$AA@ 0000000180004e68     flags.obj
 0001:00003e78       ??_C@_0BB@JIMPEHCD@MACROAREA_VIEWER?$AA@ 0000000180004e78     flags.obj
 0001:00003e90       ??_C@_0BB@KILFBFJH@MACROAREA_EDITOR?$AA@ 0000000180004e90     flags.obj
 0001:00003ea8       ??_C@_0BB@CADENPFI@MACROAREA_DIALOG?$AA@ 0000000180004ea8     flags.obj
 0001:00003ec0       ??_C@_0BB@MLMLHIGE@MACROAREA_SEARCH?$AA@ 0000000180004ec0     flags.obj
 0001:00003ed8       ??_C@_0BA@KKMKOLIK@MACROAREA_DISKS?$AA@ 0000000180004ed8     flags.obj
 0001:00003ee8       ??_C@_0BD@IGOOIJP@MACROAREA_MAINMENU?$AA@ 0000000180004ee8     flags.obj
 0001:00003f00       ??_C@_0P@LFLMAHBF@MACROAREA_MENU?$AA@ 0000000180004f00     flags.obj
 0001:00003f10       ??_C@_0P@DKPKIEO@MACROAREA_HELP?$AA@ 0000000180004f10     flags.obj
 0001:00003f20       ??_C@_0BE@MDJPICHC@MACROAREA_INFOPANEL?$AA@ 0000000180004f20     flags.obj
 0001:00003f38       ??_C@_0BF@NLJMHMPP@MACROAREA_QVIEWPANEL?$AA@ 0000000180004f38     flags.obj
 0001:00003f50       ??_C@_0BE@HBMEGBOC@MACROAREA_TREEPANEL?$AA@ 0000000180004f50     flags.obj
 0001:00003f68       ??_C@_0BF@FCHKCGLL@MACROAREA_FINDFOLDER?$AA@ 0000000180004f68     flags.obj
 0001:00003f80       ??_C@_0BD@JCFMJGDE@MACROAREA_USERMENU?$AA@ 0000000180004f80     flags.obj
 0001:00003f98       ??_C@_0BO@OMLEPJPM@MACROAREA_SHELLAUTOCOMPLETION?$AA@ 0000000180004f98     flags.obj
 0001:00003fb8       ??_C@_0BP@OIHAIGBK@MACROAREA_DIALOGAUTOCOMPLETION?$AA@ 0000000180004fb8     flags.obj
 0001:00003fd8       ??_C@_0BC@EIJFKPMK@MACROAREA_GRABBER?$AA@ 0000000180004fd8     flags.obj
 0001:00003ff0       ??_C@_0BC@GNLOCEJP@MACROAREA_DESKTOP?$AA@ 0000000180004ff0     flags.obj
 0001:00004008       ??_C@_0BB@JPEEDDOG@MACROAREA_COMMON?$AA@ 0000000180005008     flags.obj
 0001:00004020       ??_C@_0BD@DIKEKAIJ@MACROSTATE_NOMACRO?$AA@ 0000000180005020     flags.obj
 0001:00004038       ??_C@_0BF@PCDEFEGP@MACROSTATE_EXECUTING?$AA@ 0000000180005038     flags.obj
 0001:00004050       ??_C@_0BM@EJOFDENO@MACROSTATE_EXECUTING_COMMON?$AA@ 0000000180005050     flags.obj
 0001:00004070       ??_C@_0BF@BGODKPBB@MACROSTATE_RECORDING?$AA@ 0000000180005070     flags.obj
 0001:00004088       ??_C@_0BM@OICPADFE@MACROSTATE_RECORDING_COMMON?$AA@ 0000000180005088     flags.obj
 0001:000040a8       ??_C@_0N@CGFFMLBC@MPEC_SUCCESS?$AA@ 00000001800050a8     flags.obj
 0001:000040b8       ??_C@_0L@FJDDLDNN@MPEC_ERROR?$AA@ 00000001800050b8     flags.obj
 0001:000040c8       ??_C@_0N@IBOAADDD@FMVT_UNKNOWN?$AA@ 00000001800050c8     flags.obj
 0001:000040d8       ??_C@_0N@BDMFKEKE@FMVT_INTEGER?$AA@ 00000001800050d8     flags.obj
 0001:000040e8       ??_C@_0M@LFMLDDKI@FMVT_STRING?$AA@ 00000001800050e8     flags.obj
 0001:000040f8       ??_C@_0M@CKDAIOEN@FMVT_DOUBLE?$AA@ 00000001800050f8     flags.obj
 0001:00004108       ??_C@_0N@MHKOBOGF@FMVT_BOOLEAN?$AA@ 0000000180005108     flags.obj
 0001:00004118       ??_C@_0M@GKPDICDA@FMVT_BINARY?$AA@ 0000000180005118     flags.obj
 0001:00004128       ??_C@_0N@FMHCFNDF@FMVT_POINTER?$AA@ 0000000180005128     flags.obj
 0001:00004138       ??_C@_08DDPDBBNO@FMVT_NIL?$AA@ 0000000180005138     flags.obj
 0001:00004148       ??_C@_0L@DJIKMOJA@FMVT_ARRAY?$AA@ 0000000180005148     flags.obj
 0001:00004158       ??_C@_0L@PMDDFEBD@FMVT_PANEL?$AA@ 0000000180005158     flags.obj
 0001:00004168       ??_C@_0O@DCGKMPOM@WTYPE_DESKTOP?$AA@ 0000000180005168     flags.obj
 0001:00004178       ??_C@_0N@FNCFCPIG@WTYPE_PANELS?$AA@ 0000000180005178     flags.obj
 0001:00004188       ??_C@_0N@EJKMDMBK@WTYPE_VIEWER?$AA@ 0000000180005188     flags.obj
 0001:00004198       ??_C@_0N@HJNGGOKO@WTYPE_EDITOR?$AA@ 0000000180005198     flags.obj
 0001:000041a8       ??_C@_0N@PBFHKEGB@WTYPE_DIALOG?$AA@ 00000001800051a8     flags.obj
 0001:000041b8       ??_C@_0M@OMKLELFA@WTYPE_VMENU?$AA@ 00000001800051b8     flags.obj
 0001:000041c8       ??_C@_0L@BCEMNGOG@WTYPE_HELP?$AA@ 00000001800051c8     flags.obj
 0001:000041d8       ??_C@_0P@MMIDEOJJ@WTYPE_COMBOBOX?$AA@ 00000001800051d8     flags.obj
 0001:000041e8       ??_C@_0O@BHEBEELJ@WTYPE_GRABBER?$AA@ 00000001800051e8     flags.obj
 0001:000041f8       ??_C@_0M@NFHHCILL@WTYPE_HMENU?$AA@ 00000001800051f8     flags.obj
 0001:00004208       ??_C@_0BA@IPEAOBGN@TBPS_NOPROGRESS?$AA@ 0000000180005208     flags.obj
 0001:00004218       ??_C@_0BD@HMEHMDAL@TBPS_INDETERMINATE?$AA@ 0000000180005218     flags.obj
 0001:00004230       ??_C@_0M@KHLNKPHE@TBPS_NORMAL?$AA@ 0000000180005230     flags.obj
 0001:00004240       ??_C@_0L@DFDPCOFD@TBPS_ERROR?$AA@ 0000000180005240     flags.obj
 0001:00004250       ??_C@_0M@GHGAPHPP@TBPS_PAUSED?$AA@ 0000000180005250     flags.obj
 0001:00004260       ??_C@_0O@MCNCFBLF@VSMT_VIEWMODE?$AA@ 0000000180005260     flags.obj
 0001:00004270       ??_C@_09FLKONCNO@VSMT_WRAP?$AA@ 0000000180005270     flags.obj
 0001:00004280       ??_C@_0O@INKALKJK@VSMT_WORDWRAP?$AA@ 0000000180005280     flags.obj
 0001:00004290       ??_C@_08FNEFFFEL@VMT_TEXT?$AA@ 0000000180005290     flags.obj
 0001:000042a0       ??_C@_07FLIHDEDA@VMT_HEX?$AA@ 00000001800052a0     flags.obj
 0001:000042a8       ??_C@_08BDDNDBMJ@VMT_DUMP?$AA@ 00000001800052a8     flags.obj
 0001:000042b8       ??_C@_07OJCLGDHJ@VE_READ?$AA@ 00000001800052b8     flags.obj
 0001:000042c0       ??_C@_08JIBCCIDC@VE_CLOSE?$AA@ 00000001800052c0     flags.obj
 0001:000042d0       ??_C@_0M@FEFKOOMJ@VE_GOTFOCUS?$AA@ 00000001800052d0     flags.obj
 0001:000042e0       ??_C@_0N@ICHCAKIB@VE_KILLFOCUS?$AA@ 00000001800052e0     flags.obj
 0001:000042f0       ??_C@_07BLBPFFLB@EE_READ?$AA@ 00000001800052f0     flags.obj
 0001:000042f8       ??_C@_07KJGPGPOC@EE_SAVE?$AA@ 00000001800052f8     flags.obj
 0001:00004300       ??_C@_09NPOPIKMK@EE_REDRAW?$AA@ 0000000180005300     flags.obj
 0001:00004310       ??_C@_08NFPFGIG@EE_CLOSE?$AA@ 0000000180005310     flags.obj
 0001:00004320       ??_C@_0M@CPNMNBMF@EE_GOTFOCUS?$AA@ 0000000180005320     flags.obj
 0001:00004330       ??_C@_0N@ILLPMAJF@EE_KILLFOCUS?$AA@ 0000000180005330     flags.obj
 0001:00004340       ??_C@_09MIOGFFI@EE_CHANGE?$AA@ 0000000180005340     flags.obj
 0001:00004350       ??_C@_0P@MBHAHBBG@DE_DLGPROCINIT?$AA@ 0000000180005350     flags.obj
 0001:00004360       ??_C@_0BC@BMFEJAMO@DE_DEFDLGPROCINIT?$AA@ 0000000180005360     flags.obj
 0001:00004378       ??_C@_0O@ICBCOJCG@DE_DLGPROCEND?$AA@ 0000000180005378     flags.obj
 0001:00004388       ??_C@_0BB@MNODJNPE@SE_COMMONSYNCHRO?$AA@ 0000000180005388     flags.obj
 0001:000043a0       ??_C@_0N@HKGMPMJE@ESPT_TABSIZE?$AA@ 00000001800053a0     flags.obj
 0001:000043b0       ??_C@_0BA@GOKHPFCK@ESPT_EXPANDTABS?$AA@ 00000001800053b0     flags.obj
 0001:000043c0       ??_C@_0BA@KOADDMLI@ESPT_AUTOINDENT?$AA@ 00000001800053c0     flags.obj
 0001:000043d0       ??_C@_0BF@LPNONOMF@ESPT_CURSORBEYONDEOL?$AA@ 00000001800053d0     flags.obj
 0001:000043e8       ??_C@_0BC@OECOCGLJ@ESPT_CHARCODEBASE?$AA@ 00000001800053e8     flags.obj
 0001:00004400       ??_C@_0O@PIAOJINE@ESPT_CODEPAGE?$AA@ 0000000180005400     flags.obj
 0001:00004410       ??_C@_0BG@HAPABMJH@ESPT_SAVEFILEPOSITION?$AA@ 0000000180005410     flags.obj
 0001:00004428       ??_C@_0O@KCPDJCKC@ESPT_LOCKMODE?$AA@ 0000000180005428     flags.obj
 0001:00004438       ??_C@_0BA@EIGIAOHM@ESPT_SETWORDDIV?$AA@ 0000000180005438     flags.obj
 0001:00004448       ??_C@_0BA@FGEHLJDF@ESPT_GETWORDDIV?$AA@ 0000000180005448     flags.obj
 0001:00004458       ??_C@_0BE@MACJBCFP@ESPT_SHOWWHITESPACE?$AA@ 0000000180005458     flags.obj
 0001:00004470       ??_C@_0M@FICNFPPA@ESPT_SETBOM?$AA@ 0000000180005470     flags.obj
 0001:00004480       ??_C@_09FLEMPKKP@EUR_BEGIN?$AA@ 0000000180005480     flags.obj
 0001:00004490       ??_C@_07DDJDFJCN@EUR_END?$AA@ 0000000180005490     flags.obj
 0001:00004498       ??_C@_08FCONALGE@EUR_UNDO?$AA@ 0000000180005498     flags.obj
 0001:000044a8       ??_C@_08DHMMFAHF@EUR_REDO?$AA@ 00000001800054a8     flags.obj
 0001:000044b8       ??_C@_0O@PKOIFEBO@EXPAND_NOTABS?$AA@ 00000001800054b8     flags.obj
 0001:000044c8       ??_C@_0P@MLHPCNDM@EXPAND_ALLTABS?$AA@ 00000001800054c8     flags.obj
 0001:000044d8       ??_C@_0P@OONGIIBL@EXPAND_NEWTABS?$AA@ 00000001800054d8     flags.obj
 0001:000044e8       ??_C@_0BD@DKHPEOHH@EOPT_EXPANDALLTABS?$AA@ 00000001800054e8     flags.obj
 0001:00004500       ??_C@_0BG@BOINMDEK@EOPT_PERSISTENTBLOCKS?$AA@ 0000000180005500     flags.obj
 0001:00004518       ??_C@_0BG@PIIHHCAN@EOPT_DELREMOVESBLOCKS?$AA@ 0000000180005518     flags.obj
 0001:00004530       ??_C@_0BA@KPJEAKBD@EOPT_AUTOINDENT?$AA@ 0000000180005530     flags.obj
 0001:00004540       ??_C@_0BG@MBPADLG@EOPT_SAVEFILEPOSITION?$AA@ 0000000180005540     flags.obj
 0001:00004558       ??_C@_0BI@PFHCGCAI@EOPT_AUTODETECTCODEPAGE?$AA@ 0000000180005558     flags.obj
 0001:00004570       ??_C@_0BF@IMCOEIAL@EOPT_CURSORBEYONDEOL?$AA@ 0000000180005570     flags.obj
 0001:00004588       ??_C@_0BH@CJPAGGLC@EOPT_EXPANDONLYNEWTABS?$AA@ 0000000180005588     flags.obj
 0001:000045a0       ??_C@_0BE@DDKCDJDC@EOPT_SHOWWHITESPACE?$AA@ 00000001800055a0     flags.obj
 0001:000045b8       ??_C@_08HMMLONBH@EOPT_BOM?$AA@ 00000001800055b8     flags.obj
 0001:000045c8       ??_C@_0BD@CLLAKGOA@EOPT_SHOWLINEBREAK?$AA@ 00000001800055c8     flags.obj
 0001:000045e0       ??_C@_0BC@JCJEPKEC@EOPT_SHOWTITLEBAR?$AA@ 00000001800055e0     flags.obj
 0001:000045f8       ??_C@_0BA@KPGMOBKI@EOPT_SHOWKEYBAR?$AA@ 00000001800055f8     flags.obj
 0001:00004608       ??_C@_0BD@EFCFEAD@EOPT_SHOWSCROLLBAR?$AA@ 0000000180005608     flags.obj
 0001:00004620       ??_C@_0L@BJCBJJNB@BTYPE_NONE?$AA@ 0000000180005620     flags.obj
 0001:00004630       ??_C@_0N@OPHHGFPF@BTYPE_STREAM?$AA@ 0000000180005630     flags.obj
 0001:00004640       ??_C@_0N@EMEGNPLI@BTYPE_COLUMN?$AA@ 0000000180005640     flags.obj
 0001:00004650       ??_C@_0BB@BNPDAPGB@ECSTATE_MODIFIED?$AA@ 0000000180005650     flags.obj
 0001:00004668       ??_C@_0O@GBBGHDFM@ECSTATE_SAVED?$AA@ 0000000180005668     flags.obj
 0001:00004678       ??_C@_0P@BECIAJAM@ECSTATE_LOCKED?$AA@ 0000000180005678     flags.obj
 0001:00004688       ??_C@_0P@DOBJCNIG@ECTYPE_CHANGED?$AA@ 0000000180005688     flags.obj
 0001:00004698       ??_C@_0N@MDEFMEEA@ECTYPE_ADDED?$AA@ 0000000180005698     flags.obj
 0001:000046a8       ??_C@_0P@NMOJJPOB@ECTYPE_DELETED?$AA@ 00000001800056a8     flags.obj
 0001:000046b8       ??_C@_08HHHKLJPB@PLT_PATH?$AA@ 00000001800056b8     flags.obj
 0001:000046c8       ??_C@_08KBAMIIFB@PFM_GUID?$AA@ 00000001800056c8     flags.obj
 0001:000046d8       ??_C@_0P@KKEMMPNI@PFM_MODULENAME?$AA@ 00000001800056d8     flags.obj
 0001:000046e8       ??_C@_09BOODOHKD@FFT_PANEL?$AA@ 00000001800056e8     flags.obj
 0001:000046f8       ??_C@_0N@GMEDAGNH@FFT_FINDFILE?$AA@ 00000001800056f8     flags.obj
 0001:00004708       ??_C@_08KKCPIPGP@FFT_COPY?$AA@ 0000000180005708     flags.obj
 0001:00004718       ??_C@_0L@EKPDMFDD@FFT_SELECT?$AA@ 0000000180005718     flags.obj
 0001:00004728       ??_C@_0L@LGPEDLLD@FFT_CUSTOM?$AA@ 0000000180005728     flags.obj
 0001:00004738       ??_C@_0M@OIOMMFOE@FST_UNKNOWN?$AA@ 0000000180005738     flags.obj
 0001:00004748       ??_C@_0L@GGGOEGKJ@FST_SUBKEY?$AA@ 0000000180005748     flags.obj
 0001:00004758       ??_C@_09LFEEAJIC@FST_QWORD?$AA@ 0000000180005758     flags.obj
 0001:00004768       ??_C@_0L@LPMPBKDL@FST_STRING?$AA@ 0000000180005768     flags.obj
 0001:00004778       ??_C@_08EJJJCLIG@FST_DATA?$AA@ 0000000180005778     flags.obj
 0001:00004788       ??_C@_09OBBBBFPE@FSSF_ROOT?$AA@ 0000000180005788     flags.obj
 0001:00004798       ??_C@_0BB@HDKCPBIO@FSSF_HISTORY_CMD?$AA@ 0000000180005798     flags.obj
 0001:000047b0       ??_C@_0BE@BLPOFODL@FSSF_HISTORY_FOLDER?$AA@ 00000001800057b0     flags.obj
 0001:000047c8       ??_C@_0BC@NJCJCCNH@FSSF_HISTORY_VIEW?$AA@ 00000001800057c8     flags.obj
 0001:000047e0       ??_C@_0BC@CODELNPP@FSSF_HISTORY_EDIT?$AA@ 00000001800057e0     flags.obj
 0001:000047f8       ??_C@_0BG@IFGEMJIF@FSSF_HISTORY_EXTERNAL?$AA@ 00000001800057f8     flags.obj
 0001:00004810       ??_C@_0BG@DGAKDKFK@FSSF_FOLDERSHORTCUT_0?$AA@ 0000000180005810     flags.obj
 0001:00004828       ??_C@_0BG@CPBBALBL@FSSF_FOLDERSHORTCUT_1?$AA@ 0000000180005828     flags.obj
 0001:00004840       ??_C@_0BG@EDMFINI@FSSF_FOLDERSHORTCUT_2?$AA@ 0000000180005840     flags.obj
 0001:00004858       ??_C@_0BG@BNCHGJJJ@FSSF_FOLDERSHORTCUT_3?$AA@ 0000000180005858     flags.obj
 0001:00004870       ??_C@_0BG@FCGGPPFO@FSSF_FOLDERSHORTCUT_4?$AA@ 0000000180005870     flags.obj
 0001:00004888       ??_C@_0BG@ELHNMOBP@FSSF_FOLDERSHORTCUT_5?$AA@ 0000000180005888     flags.obj
 0001:000048a0       ??_C@_0BG@GAFAJNNM@FSSF_FOLDERSHORTCUT_6?$AA@ 00000001800058a0     flags.obj
 0001:000048b8       ??_C@_0BG@HJELKMJN@FSSF_FOLDERSHORTCUT_7?$AA@ 00000001800058b8     flags.obj
 0001:000048d0       ??_C@_0BG@PONDLAFC@FSSF_FOLDERSHORTCUT_8?$AA@ 00000001800058d0     flags.obj
 0001:000048e8       ??_C@_0BG@OHMIIBBD@FSSF_FOLDERSHORTCUT_9?$AA@ 00000001800058e8     flags.obj
 0001:00004900       ??_C@_0BD@PBIEGEHP@FSSF_CONFIRMATIONS?$AA@ 0000000180005900     flags.obj
 0001:00004918       ??_C@_0M@PIGDMPJB@FSSF_SYSTEM?$AA@ 0000000180005918     flags.obj
 0001:00004928       ??_C@_0L@LBFNJGFB@FSSF_PANEL?$AA@ 0000000180005928     flags.obj
 0001:00004938       ??_C@_0M@KJLIHDEL@FSSF_EDITOR?$AA@ 0000000180005938     flags.obj
 0001:00004948       ??_C@_0M@KEMGKEOF@FSSF_SCREEN?$AA@ 0000000180005948     flags.obj
 0001:00004958       ??_C@_0M@CBDJLJIE@FSSF_DIALOG?$AA@ 0000000180005958     flags.obj
 0001:00004968       ??_C@_0P@OCDADNBF@FSSF_INTERFACE?$AA@ 0000000180005968     flags.obj
 0001:00004978       ??_C@_0BB@GBBEBNKE@FSSF_PANELLAYOUT?$AA@ 0000000180005978     flags.obj
 0001:00004990       ??_C@_0M@JCGHGLJF@PSL_ROAMING?$AA@ 0000000180005990     flags.obj
 0001:000049a0       ??_C@_09EDBNDHCM@PSL_LOCAL?$AA@ 00000001800059a0     flags.obj
 0001:000049b0       ??_C@_07BPEFOPGM@FCT_ANY?$AA@ 00000001800059b0     flags.obj
 0001:000049b8       ??_C@_0L@CDAEILNM@FCT_STREAM?$AA@ 00000001800059b8     flags.obj
 0001:000049c8       ??_C@_0L@IADFDBJB@FCT_COLUMN?$AA@ 00000001800059c8     flags.obj
 0001:000049d8       ??_C@_0O@KJFMBLFE@LINK_HARDLINK?$AA@ 00000001800059d8     flags.obj
 0001:000049e8       ??_C@_0O@OOAFIIDA@LINK_JUNCTION?$AA@ 00000001800059e8     flags.obj
 0001:000049f8       ??_C@_0O@FIAPLKLH@LINK_VOLMOUNT?$AA@ 00000001800059f8     flags.obj
 0001:00004a08       ??_C@_0BB@JDBEPJDK@LINK_SYMLINKFILE?$AA@ 0000000180005a08     flags.obj
 0001:00004a20       ??_C@_0BA@GFPIOFMG@LINK_SYMLINKDIR?$AA@ 0000000180005a20     flags.obj
 0001:00004a30       ??_C@_0N@PJENIJFN@LINK_SYMLINK?$AA@ 0000000180005a30     flags.obj
 0001:00004a40       ??_C@_08HNOHKPBK@CPM_FULL?$AA@ 0000000180005a40     flags.obj
 0001:00004a50       ??_C@_08LAEGFKJE@CPM_REAL?$AA@ 0000000180005a50     flags.obj
 0001:00004a60       ??_C@_0L@NPJNPCJM@CPM_NATIVE?$AA@ 0000000180005a60     flags.obj
 0001:00004a70       ??_C@_0L@NCFOENCC@VS_RELEASE?$AA@ 0000000180005a70     flags.obj
 0001:00004a80       ??_C@_08BDGLHPMJ@VS_ALPHA?$AA@ 0000000180005a80     flags.obj
 0001:00004a90       ??_C@_07OKFPMINB@VS_BETA?$AA@ 0000000180005a90     flags.obj
 0001:00004a98       ??_C@_05MMFLPJEB@VS_RC?$AA@ 0000000180005a98     flags.obj
 0001:00004aa0       ??_C@_0BC@OOKLINPG@OPEN_LEFTDISKMENU?$AA@ 0000000180005aa0     flags.obj
 0001:00004ab8       ??_C@_0BB@CEFDHHLF@OPEN_PLUGINSMENU?$AA@ 0000000180005ab8     flags.obj
 0001:00004ad0       ??_C@_0O@IEJHJCNB@OPEN_FINDLIST?$AA@ 0000000180005ad0     flags.obj
 0001:00004ae0       ??_C@_0O@OGDCDPNG@OPEN_SHORTCUT?$AA@ 0000000180005ae0     flags.obj
 0001:00004af0       ??_C@_0BB@JHCCMIPF@OPEN_COMMANDLINE?$AA@ 0000000180005af0     flags.obj
 0001:00004b08       ??_C@_0M@DMJLHMGM@OPEN_EDITOR?$AA@ 0000000180005b08     flags.obj
 0001:00004b18       ??_C@_0M@MOBCONI@OPEN_VIEWER?$AA@ 0000000180005b18     flags.obj
 0001:00004b28       ??_C@_0P@LCDNLGDE@OPEN_FILEPANEL?$AA@ 0000000180005b28     flags.obj
 0001:00004b38       ??_C@_0M@LEBKLGKD@OPEN_DIALOG?$AA@ 0000000180005b38     flags.obj
 0001:00004b48       ??_C@_0N@CBHPGAKB@OPEN_ANALYSE?$AA@ 0000000180005b48     flags.obj
 0001:00004b58       ??_C@_0BD@NFNGGFHI@OPEN_RIGHTDISKMENU?$AA@ 0000000180005b58     flags.obj
 0001:00004b70       ??_C@_0P@FOKOAMLC@OPEN_FROMMACRO?$AA@ 0000000180005b70     flags.obj
 0001:00004b80       ??_C@_0O@NEDDJIHC@OPEN_LUAMACRO?$AA@ 0000000180005b80     flags.obj
 0001:00004b90       ??_C@_0P@GBMLNMMI@MCT_MACROPARSE?$AA@ 0000000180005b90     flags.obj
 0001:00004ba0       ??_C@_0P@GNPFPCF@MCT_LOADMACROS?$AA@ 0000000180005ba0     flags.obj
 0001:00004bb0       ??_C@_0P@HMDDACMI@MCT_ENUMMACROS?$AA@ 0000000180005bb0     flags.obj
 0001:00004bc0       ??_C@_0BA@MOCJHMJK@MCT_WRITEMACROS?$AA@ 0000000180005bc0     flags.obj
 0001:00004bd0       ??_C@_0N@IGJGAHKE@MCT_GETMACRO?$AA@ 0000000180005bd0     flags.obj
 0001:00004be0       ??_C@_0BC@NFGGBILF@MCT_RECORDEDMACRO?$AA@ 0000000180005be0     flags.obj
 0001:00004bf8       ??_C@_0N@OLCKOJMI@MCT_DELMACRO?$AA@ 0000000180005bf8     flags.obj
 0001:00004c08       ??_C@_0BC@NALHIHJ@MCT_RUNSTARTMACRO?$AA@ 0000000180005c08     flags.obj
 0001:00004c20       ??_C@_0P@HOMHAEFB@MCT_EXECSTRING?$AA@ 0000000180005c20     flags.obj
 0001:00004c30       ??_C@_0O@CDBDPKIC@MCT_PANELSORT?$AA@ 0000000180005c30     flags.obj
 0001:00004c40       ??_C@_0BH@PKKJIOHM@MCT_GETCUSTOMSORTMODES?$AA@ 0000000180005c40     flags.obj
 0001:00004c58       ??_C@_0N@FOPIOCHO@MCT_ADDMACRO?$AA@ 0000000180005c58     flags.obj
 0001:00004c68       ??_C@_0N@BHFJFHA@MCT_KEYMACRO?$AA@ 0000000180005c68     flags.obj
 0001:00004c78       ??_C@_0BB@LPDAOGB@MCT_CANPANELSORT?$AA@ 0000000180005c78     flags.obj
 0001:00004c90       ??_C@_0BC@IOECJI@MPRT_NORMALFINISH?$AA@ 0000000180005c90     flags.obj
 0001:00004ca8       ??_C@_0BB@PMCBIGCA@MPRT_ERRORFINISH?$AA@ 0000000180005ca8     flags.obj
 0001:00004cc0       ??_C@_0BA@BCBAEEOI@MPRT_ERRORPARSE?$AA@ 0000000180005cc0     flags.obj
 0001:00004cd0       ??_C@_09EJDAADCN@MPRT_KEYS?$AA@ 0000000180005cd0     flags.obj
 0001:00004ce0       ??_C@_0L@GEHHCKFA@MPRT_PRINT?$AA@ 0000000180005ce0     flags.obj
 0001:00004cf0       ??_C@_0BA@OBIDLEIM@MPRT_PLUGINCALL?$AA@ 0000000180005cf0     flags.obj
 0001:00004d00       ??_C@_0BA@EJFFOAMM@MPRT_PLUGINMENU?$AA@ 0000000180005d00     flags.obj
 0001:00004d10       ??_C@_0BC@LEDOPMKI@MPRT_PLUGINCONFIG?$AA@ 0000000180005d10     flags.obj
 0001:00004d28       ??_C@_0BD@HHINMPPI@MPRT_PLUGINCOMMAND?$AA@ 0000000180005d28     flags.obj
 0001:00004d40       ??_C@_0O@IEMNLPAB@MPRT_USERMENU?$AA@ 0000000180005d40     flags.obj
 0001:00004d50       ??_C@_0BA@GEAFHJNF@MPRT_HASNOMACRO?$AA@ 0000000180005d50     flags.obj
 0001:00004d60       ??_C@_0BC@PNCKAHJO@FE_CHANGEVIEWMODE?$AA@ 0000000180005d60     flags.obj
 0001:00004d78       ??_C@_09DENIDBMJ@FE_REDRAW?$AA@ 0000000180005d78     flags.obj
 0001:00004d88       ??_C@_07CLNPDBLG@FE_IDLE?$AA@ 0000000180005d88     flags.obj
 0001:00004d90       ??_C@_08DENCGKED@FE_CLOSE?$AA@ 0000000180005d90     flags.obj
 0001:00004da0       ??_C@_08MOMCCKPB@FE_BREAK?$AA@ 0000000180005da0     flags.obj
 0001:00004db0       ??_C@_0L@LELAIPLL@FE_COMMAND?$AA@ 0000000180005db0     flags.obj
 0001:00004dc0       ??_C@_0M@FIECADDF@FE_GOTFOCUS?$AA@ 0000000180005dc0     flags.obj
 0001:00004dd0       ??_C@_0N@DGHFKMFL@FE_KILLFOCUS?$AA@ 0000000180005dd0     flags.obj
 0001:00004de0       ??_C@_0BE@PONEECEM@FE_CHANGESORTPARAMS?$AA@ 0000000180005de0     flags.obj
 0001:00004df8       ??_C@_0M@HNDHDHHO@FCF_FG_4BIT?$AA@ 0000000180005df8     flags.obj
 0001:00004e08       ??_C@_0M@PJHNDJIE@FCF_BG_4BIT?$AA@ 0000000180005e08     flags.obj
 0001:00004e18       ??_C@_0N@HMKJBHOA@FCF_4BITMASK?$AA@ 0000000180005e18     flags.obj
 0001:00004e28       ??_C@_0BB@PJFLJJLD@FCF_RAWATTR_MASK?$AA@ 0000000180005e28     flags.obj
 0001:00004e40       ??_C@_0BC@NKBLNNIA@FCF_EXTENDEDFLAGS?$AA@ 0000000180005e40     flags.obj
 0001:00004e58       ??_C@_0M@LFMGCKHG@FCF_FG_BOLD?$AA@ 0000000180005e58     flags.obj
 0001:00004e68       ??_C@_0O@FAPDECBF@FCF_FG_ITALIC?$AA@ 0000000180005e68     flags.obj
 0001:00004e78       ??_C@_0BB@NPEFGEGA@FCF_FG_UNDERLINE?$AA@ 0000000180005e78     flags.obj
 0001:00004e90       ??_C@_0O@LGBGBIGB@FCF_STYLEMASK?$AA@ 0000000180005e90     flags.obj
 0001:00004ea0       ??_C@_08BKNBBLHK@FCF_NONE?$AA@ 0000000180005ea0     flags.obj
 0001:00004eb0       ??_C@_08FKIDFHCM@CDF_NONE?$AA@ 0000000180005eb0     flags.obj
 0001:00004ec0       ??_C@_0N@ELMEMNDH@FMSG_WARNING?$AA@ 0000000180005ec0     flags.obj
 0001:00004ed0       ??_C@_0P@HHIGLJAP@FMSG_ERRORTYPE?$AA@ 0000000180005ed0     flags.obj
 0001:00004ee0       ??_C@_0BE@FHOOILPH@FMSG_KEEPBACKGROUND?$AA@ 0000000180005ee0     flags.obj
 0001:00004ef8       ??_C@_0P@KBEMNNEP@FMSG_LEFTALIGN?$AA@ 0000000180005ef8     flags.obj
 0001:00004f08       ??_C@_0O@FOIOKDHJ@FMSG_ALLINONE?$AA@ 0000000180005f08     flags.obj
 0001:00004f18       ??_C@_0L@BGALGPOK@FMSG_MB_OK?$AA@ 0000000180005f18     flags.obj
 0001:00004f28       ??_C@_0BB@JGAPGIEP@FMSG_MB_OKCANCEL?$AA@ 0000000180005f28     flags.obj
 0001:00004f40       ??_C@_0BJ@BKJADAHA@FMSG_MB_ABORTRETRYIGNORE?$AA@ 0000000180005f40     flags.obj
 0001:00004f60       ??_C@_0O@GPCAPHCL@FMSG_MB_YESNO?$AA@ 0000000180005f60     flags.obj
 0001:00004f70       ??_C@_0BE@IBNOLCGP@FMSG_MB_YESNOCANCEL?$AA@ 0000000180005f70     flags.obj
 0001:00004f88       ??_C@_0BE@OCLAIENB@FMSG_MB_RETRYCANCEL?$AA@ 0000000180005f88     flags.obj
 0001:00004fa0       ??_C@_09NEGPLEAH@FMSG_NONE?$AA@ 0000000180005fa0     flags.obj
 0001:00004fb0       ??_C@_0N@DHJCDIKM@DIF_BOXCOLOR?$AA@ 0000000180005fb0     flags.obj
 0001:00004fc0       ??_C@_09IAEPIICA@DIF_GROUP?$AA@ 0000000180005fc0     flags.obj
 0001:00004fd0       ??_C@_0N@GCKJNBCM@DIF_LEFTTEXT?$AA@ 0000000180005fd0     flags.obj
 0001:00004fe0       ??_C@_0P@BGPBEDHH@DIF_MOVESELECT?$AA@ 0000000180005fe0     flags.obj
 0001:00004ff0       ??_C@_0BC@PDKFKKEI@DIF_SHOWAMPERSAND?$AA@ 0000000180005ff0     flags.obj
 0001:00005008       ??_C@_0BA@BLCOKAAO@DIF_CENTERGROUP?$AA@ 0000000180006008     flags.obj
 0001:00005018       ??_C@_0P@MKFBJPOB@DIF_NOBRACKETS?$AA@ 0000000180006018     flags.obj
 0001:00005028       ??_C@_0BF@JBCDBJCL@DIF_MANUALADDHISTORY?$AA@ 0000000180006028     flags.obj
 0001:00005040       ??_C@_0O@JKNMBNLA@DIF_SEPARATOR?$AA@ 0000000180006040     flags.obj
 0001:00005050       ??_C@_0P@CGILDLOA@DIF_SEPARATOR2?$AA@ 0000000180006050     flags.obj
 0001:00005060       ??_C@_0L@NBPFNGLB@DIF_EDITOR?$AA@ 0000000180006060     flags.obj
 0001:00005070       ??_C@_0BE@PFICAGJF@DIF_LISTNOAMPERSAND?$AA@ 0000000180006070     flags.obj
 0001:00005088       ??_C@_0O@FFJNBMAD@DIF_LISTNOBOX?$AA@ 0000000180006088     flags.obj
 0001:00005098       ??_C@_0M@IPFBMFDN@DIF_HISTORY?$AA@ 0000000180006098     flags.obj
 0001:000050a8       ??_C@_0P@EGFAEEDC@DIF_BTNNOCLOSE?$AA@ 00000001800060a8     flags.obj
 0001:000050b8       ??_C@_0P@KOJCCCGB@DIF_CENTERTEXT?$AA@ 00000001800060b8     flags.obj
 0001:000050c8       ??_C@_0BC@ODEMBOPK@DIF_SEPARATORUSER?$AA@ 00000001800060c8     flags.obj
 0001:000050e0       ??_C@_0O@IKJBMPOF@DIF_SETSHIELD?$AA@ 00000001800060e0     flags.obj
 0001:000050f0       ??_C@_0P@EEJEDBLH@DIF_EDITEXPAND?$AA@ 00000001800060f0     flags.obj
 0001:00005100       ??_C@_0BB@EIMEKEFP@DIF_DROPDOWNLIST?$AA@ 0000000180006100     flags.obj
 0001:00005118       ??_C@_0BD@MNGIOLFF@DIF_USELASTHISTORY?$AA@ 0000000180006118     flags.obj
 0001:00005130       ??_C@_0N@MOCGNIKC@DIF_MASKEDIT?$AA@ 0000000180006130     flags.obj
 0001:00005140       ??_C@_0BD@LPDHCLJI@DIF_LISTTRACKMOUSE?$AA@ 0000000180006140     flags.obj
 0001:00005158       ??_C@_0BK@LEFIBDOA@DIF_LISTTRACKMOUSEINFOCUS?$AA@ 0000000180006158     flags.obj
 0001:00005178       ??_C@_0BC@JNLDMGBD@DIF_SELECTONENTRY?$AA@ 0000000180006178     flags.obj
 0001:00005190       ??_C@_0L@KKNJDNBK@DIF_3STATE?$AA@ 0000000180006190     flags.obj
 0001:000051a0       ??_C@_0N@GBGHICKO@DIF_EDITPATH?$AA@ 00000001800061a0     flags.obj
 0001:000051b0       ??_C@_0BB@NPNALIGO@DIF_LISTWRAPMODE?$AA@ 00000001800061b0     flags.obj
 0001:000051c8       ??_C@_0BD@MFOKKGGF@DIF_NOAUTOCOMPLETE?$AA@ 00000001800061c8     flags.obj
 0001:000051e0       ??_C@_0BG@MONEJILE@DIF_LISTAUTOHIGHLIGHT?$AA@ 00000001800061e0     flags.obj
 0001:000051f8       ??_C@_0BA@JNOKLHOL@DIF_LISTNOCLOSE?$AA@ 00000001800061f8     flags.obj
 0001:00005208       ??_C@_0BB@GMKDKOOP@DIF_EDITPATHEXEC?$AA@ 0000000180006208     flags.obj
 0001:00005220       ??_C@_0L@EPNFOPAK@DIF_HIDDEN?$AA@ 0000000180006220     flags.obj
 0001:00005230       ??_C@_0N@KOGKCAKJ@DIF_READONLY?$AA@ 0000000180006230     flags.obj
 0001:00005240       ??_C@_0M@NLLDINIM@DIF_NOFOCUS?$AA@ 0000000180006240     flags.obj
 0001:00005250       ??_C@_0M@HCFLMDHK@DIF_DISABLE?$AA@ 0000000180006250     flags.obj
 0001:00005260       ??_C@_0BC@CHAAKEJO@DIF_DEFAULTBUTTON?$AA@ 0000000180006260     flags.obj
 0001:00005278       ??_C@_09LCJIOEMN@DIF_FOCUS?$AA@ 0000000180006278     flags.obj
 0001:00005288       ??_C@_0O@KJADCBBN@DIF_RIGHTTEXT?$AA@ 0000000180006288     flags.obj
 0001:00005298       ??_C@_0N@LAEOODAD@DIF_WORDWRAP?$AA@ 0000000180006298     flags.obj
 0001:000052a8       ??_C@_08KFOHCPDE@DIF_NONE?$AA@ 00000001800062a8     flags.obj
 0001:000052b8       ??_C@_0N@EDHAFIIL@LIF_SELECTED?$AA@ 00000001800062b8     flags.obj
 0001:000052c8       ??_C@_0M@BMGIEAIL@LIF_CHECKED?$AA@ 00000001800062c8     flags.obj
 0001:000052d8       ??_C@_0O@KJIFADIG@LIF_SEPARATOR?$AA@ 00000001800062d8     flags.obj
 0001:000052e8       ??_C@_0M@HEFHLFIE@LIF_DISABLE?$AA@ 00000001800062e8     flags.obj
 0001:000052f8       ??_C@_0L@PKDDGEEG@LIF_GRAYED?$AA@ 00000001800062f8     flags.obj
 0001:00005308       ??_C@_0L@PFBGAOEP@LIF_HIDDEN?$AA@ 0000000180006308     flags.obj
 0001:00005318       ??_C@_0BD@HEPCOIEH@LIF_DELETEUSERDATA?$AA@ 0000000180006318     flags.obj
 0001:00005330       ??_C@_08BODPINCM@LIF_NONE?$AA@ 0000000180006330     flags.obj
 0001:00005340       ??_C@_0BC@BGAENNBJ@LIFIND_EXACTMATCH?$AA@ 0000000180006340     flags.obj
 0001:00005358       ??_C@_0M@FPOGKIGO@LIFIND_NONE?$AA@ 0000000180006358     flags.obj
 0001:00005368       ??_C@_0BA@OOIEKCFB@LINFO_SHOWNOBOX?$AA@ 0000000180006368     flags.obj
 0001:00005378       ??_C@_0BE@DECCEGNO@LINFO_AUTOHIGHLIGHT?$AA@ 0000000180006378     flags.obj
 0001:00005390       ??_C@_0BH@BADLEILJ@LINFO_REVERSEHIGHLIGHT?$AA@ 0000000180006390     flags.obj
 0001:000053a8       ??_C@_0P@KLBMHNCG@LINFO_WRAPMODE?$AA@ 00000001800063a8     flags.obj
 0001:000053b8       ??_C@_0BE@OHJCOKAE@LINFO_SHOWAMPERSAND?$AA@ 00000001800063b8     flags.obj
 0001:000053d0       ??_C@_0L@EPACPANF@LINFO_NONE?$AA@ 00000001800063d0     flags.obj
 0001:000053e0       ??_C@_0N@OLGDMHKL@FDLG_WARNING?$AA@ 00000001800063e0     flags.obj
 0001:000053f0       ??_C@_0BB@DKMEBDJJ@FDLG_SMALLDIALOG?$AA@ 00000001800063f0     flags.obj
 0001:00005408       ??_C@_0BC@ONGLDAJN@FDLG_NODRAWSHADOW?$AA@ 0000000180006408     flags.obj
 0001:00005420       ??_C@_0BB@NPLEEAKK@FDLG_NODRAWPANEL?$AA@ 0000000180006420     flags.obj
 0001:00005438       ??_C@_0BG@GHNOOENB@FDLG_KEEPCONSOLETITLE?$AA@ 0000000180006438     flags.obj
 0001:00005450       ??_C@_0O@MKFABCNE@FDLG_NONMODAL?$AA@ 0000000180006450     flags.obj
 0001:00005460       ??_C@_09NNFHCBNL@FDLG_NONE?$AA@ 0000000180006460     flags.obj
 0001:00005470       ??_C@_0N@JOOGIBAO@MIF_SELECTED?$AA@ 0000000180006470     flags.obj
 0001:00005480       ??_C@_0M@IHMNAMOE@MIF_CHECKED?$AA@ 0000000180006480     flags.obj
 0001:00005490       ??_C@_0O@DEIKOCPA@MIF_SEPARATOR?$AA@ 0000000180006490     flags.obj
 0001:000054a0       ??_C@_0M@OPPCPJOL@MIF_DISABLE?$AA@ 00000001800064a0     flags.obj
 0001:000054b0       ??_C@_0L@DLLNLLIG@MIF_GRAYED?$AA@ 00000001800064b0     flags.obj
 0001:000054c0       ??_C@_0L@DEJINBIP@MIF_HIDDEN?$AA@ 00000001800064c0     flags.obj
 0001:000054d0       ??_C@_08JEEJJGP@MIF_NONE?$AA@ 00000001800064d0     flags.obj
 0001:000054e0       ??_C@_0BE@FALMPPJK@FMENU_SHOWAMPERSAND?$AA@ 00000001800064e0     flags.obj
 0001:000054f8       ??_C@_0P@HICDNKDJ@FMENU_WRAPMODE?$AA@ 00000001800064f8     flags.obj
 0001:00005508       ??_C@_0BE@IDAMFDEA@FMENU_AUTOHIGHLIGHT?$AA@ 0000000180006508     flags.obj
 0001:00005520       ??_C@_0BL@OKAIKPMN@FMENU_REVERSEAUTOHIGHLIGHT?$AA@ 0000000180006520     flags.obj
 0001:00005540       ??_C@_0BJ@FCEONOJC@FMENU_CHANGECONSOLETITLE?$AA@ 0000000180006540     flags.obj
 0001:00005560       ??_C@_0L@DGFIEOMD@FMENU_NONE?$AA@ 0000000180006560     flags.obj
 0001:00005570       ??_C@_0O@JEAJLDHC@PPIF_SELECTED?$AA@ 0000000180006570     flags.obj
 0001:00005580       ??_C@_0BC@LPBDBIOM@PPIF_PROCESSDESCR?$AA@ 0000000180006580     flags.obj
 0001:00005598       ??_C@_09OIFMMGNJ@PPIF_NONE?$AA@ 0000000180006598     flags.obj
 0001:000055a8       ??_C@_0BC@BONLDOOD@PFLAGS_SHOWHIDDEN?$AA@ 00000001800065a8     flags.obj
 0001:000055c0       ??_C@_0BB@BCAJEJEH@PFLAGS_HIGHLIGHT?$AA@ 00000001800065c0     flags.obj
 0001:000055d8       ??_C@_0BI@BFAFODJ@PFLAGS_REVERSESORTORDER?$AA@ 00000001800065d8     flags.obj
 0001:000055f0       ??_C@_0BF@KJNCJPKN@PFLAGS_USESORTGROUPS?$AA@ 00000001800065f0     flags.obj
 0001:00005608       ??_C@_0BF@LBBAIOCD@PFLAGS_SELECTEDFIRST?$AA@ 0000000180006608     flags.obj
 0001:00005620       ??_C@_0BB@KDANIJNM@PFLAGS_REALNAMES?$AA@ 0000000180006620     flags.obj
 0001:00005638       ??_C@_0BB@ILEHDKFJ@PFLAGS_PANELLEFT?$AA@ 0000000180006638     flags.obj
 0001:00005650       ??_C@_0BI@EHHAJLOH@PFLAGS_DIRECTORIESFIRST?$AA@ 0000000180006650     flags.obj
 0001:00005668       ??_C@_0BA@KJEPHDOM@PFLAGS_USECRC32?$AA@ 0000000180006668     flags.obj
 0001:00005678       ??_C@_0O@DBPJGING@PFLAGS_PLUGIN?$AA@ 0000000180006678     flags.obj
 0001:00005688       ??_C@_0P@MLDEBNPK@PFLAGS_VISIBLE?$AA@ 0000000180006688     flags.obj
 0001:00005698       ??_C@_0N@EOFAELOJ@PFLAGS_FOCUS?$AA@ 0000000180006698     flags.obj
 0001:000056a8       ??_C@_0BI@EOCCAHFA@PFLAGS_ALTERNATIVENAMES?$AA@ 00000001800066a8     flags.obj
 0001:000056c0       ??_C@_0BA@GHMDCHHI@PFLAGS_SHORTCUT?$AA@ 00000001800066c0     flags.obj
 0001:000056d0       ??_C@_0M@NEMAHHGP@PFLAGS_NONE?$AA@ 00000001800066d0     flags.obj
 0001:000056e0       ??_C@_0M@IDNADAFL@VF_NONMODAL?$AA@ 00000001800066e0     flags.obj
 0001:000056f0       ??_C@_0BB@OCDDPIKL@VF_DELETEONCLOSE?$AA@ 00000001800066f0     flags.obj
 0001:00005708       ??_C@_0N@LDHALKKM@VF_ENABLE_F6?$AA@ 0000000180006708     flags.obj
 0001:00005718       ??_C@_0BC@DLGKMECC@VF_DISABLEHISTORY?$AA@ 0000000180006718     flags.obj
 0001:00005730       ??_C@_0BD@DHJCMLFI@VF_IMMEDIATERETURN?$AA@ 0000000180006730     flags.obj
 0001:00005748       ??_C@_0BJ@OGNFHEJG@VF_DELETEONLYFILEONCLOSE?$AA@ 0000000180006748     flags.obj
 0001:00005768       ??_C@_07CJJFHP@VF_NONE?$AA@ 0000000180006768     flags.obj
 0001:00005770       ??_C@_0M@PIFGAPFH@EF_NONMODAL?$AA@ 0000000180006770     flags.obj
 0001:00005780       ??_C@_0N@DBHFPBEO@EF_CREATENEW?$AA@ 0000000180006780     flags.obj
 0001:00005790       ??_C@_0N@LKLNHALI@EF_ENABLE_F6?$AA@ 0000000180006790     flags.obj
 0001:000057a0       ??_C@_0BC@PPEPEFFI@EF_DISABLEHISTORY?$AA@ 00000001800067a0     flags.obj
 0001:000057b8       ??_C@_0BB@KGPIDKFC@EF_DELETEONCLOSE?$AA@ 00000001800067b8     flags.obj
 0001:000057d0       ??_C@_0BD@IHIGHGPL@EF_IMMEDIATERETURN?$AA@ 00000001800067d0     flags.obj
 0001:000057e8       ??_C@_0BJ@ILCPOFKL@EF_DELETEONLYFILEONCLOSE?$AA@ 00000001800067e8     flags.obj
 0001:00005808       ??_C@_09IJMPFPLB@EF_LOCKED?$AA@ 0000000180006808     flags.obj
 0001:00005818       ??_C@_0BC@GFHJGKD@EF_DISABLESAVEPOS?$AA@ 0000000180006818     flags.obj
 0001:00005830       ??_C@_0BB@NILAHAFO@EF_OPENMODE_MASK?$AA@ 0000000180006830     flags.obj
 0001:00005848       ??_C@_0BC@GAIDEJIA@EF_OPENMODE_QUERY?$AA@ 0000000180006848     flags.obj
 0001:00005860       ??_C@_0BG@BFKJJBAG@EF_OPENMODE_NEWIFOPEN?$AA@ 0000000180006860     flags.obj
 0001:00005878       ??_C@_0BI@KGOKGPEI@EF_OPENMODE_USEEXISTING?$AA@ 0000000180006878     flags.obj
 0001:00005890       ??_C@_0BI@EJBKKDJ@EF_OPENMODE_BREAKIFOPEN?$AA@ 0000000180006890     flags.obj
 0001:000058a8       ??_C@_0BJ@MOLGCBMH@EF_OPENMODE_RELOADIFOPEN?$AA@ 00000001800068a8     flags.obj
 0001:000058c8       ??_C@_07MBPCONNA@EN_NONE?$AA@ 00000001800068c8     flags.obj
 0001:000058d0       ??_C@_0BC@HHNGCBAM@FHELP_NOSHOWERROR?$AA@ 00000001800068d0     flags.obj
 0001:000058e8       ??_C@_0P@GANNLHEJ@FHELP_SELFHELP?$AA@ 00000001800068e8     flags.obj
 0001:000058f8       ??_C@_0O@FLGGLFLC@FHELP_FARHELP?$AA@ 00000001800068f8     flags.obj
 0001:00005908       ??_C@_0BB@KNKDPNI@FHELP_CUSTOMFILE?$AA@ 0000000180006908     flags.obj
 0001:00005920       ??_C@_0BB@IHFFPJJA@FHELP_CUSTOMPATH?$AA@ 0000000180006920     flags.obj
 0001:00005938       ??_C@_0L@OOIMFPBD@FHELP_GUID?$AA@ 0000000180006938     flags.obj
 0001:00005948       ??_C@_0BC@PNPOIHMG@FHELP_USECONTENTS?$AA@ 0000000180006948     flags.obj
 0001:00005960       ??_C@_0L@MAGMKNFN@FHELP_NONE?$AA@ 0000000180006960     flags.obj
 0001:00005970       ??_C@_0BE@GEGKIINM@KMFLAGS_SILENTCHECK?$AA@ 0000000180006970     flags.obj
 0001:00005988       ??_C@_0BM@BBOPLPKC@KMFLAGS_NOSENDKEYSTOPLUGINS?$AA@ 0000000180006988     flags.obj
 0001:000059a8       ??_C@_0BF@PHHPAAOK@KMFLAGS_ENABLEOUTPUT?$AA@ 00000001800069a8     flags.obj
 0001:000059c0       ??_C@_0BB@NCECNBPK@KMFLAGS_LANGMASK?$AA@ 00000001800069c0     flags.obj
 0001:000059d8       ??_C@_0M@HFBACHCP@KMFLAGS_LUA?$AA@ 00000001800069d8     flags.obj
 0001:000059e8       ??_C@_0BD@JHNPMIGP@KMFLAGS_MOONSCRIPT?$AA@ 00000001800069e8     flags.obj
 0001:00005a00       ??_C@_0N@GIJCDFJI@KMFLAGS_NONE?$AA@ 0000000180006a00     flags.obj
 0001:00005a10       ??_C@_0O@GKOLBMFK@AKMFLAGS_NONE?$AA@ 0000000180006a10     flags.obj
 0001:00005a20       ??_C@_0P@LMBMJIMF@FSETCLR_REDRAW?$AA@ 0000000180006a20     flags.obj
 0001:00005a30       ??_C@_0N@LCOHPDHN@FSETCLR_NONE?$AA@ 0000000180006a30     flags.obj
 0001:00005a40       ??_C@_0N@MLMCEKPH@WIF_MODIFIED?$AA@ 0000000180006a40     flags.obj
 0001:00005a50       ??_C@_0M@ICPAPCOF@WIF_CURRENT?$AA@ 0000000180006a50     flags.obj
 0001:00005a60       ??_C@_09FPGEBDGO@WIF_MODAL?$AA@ 0000000180006a60     flags.obj
 0001:00005a70       ??_C@_08DAKKFBIA@WIF_NONE?$AA@ 0000000180006a70     flags.obj
 0001:00005a80       ??_C@_0BG@JMJAOELH@VOPT_SAVEFILEPOSITION?$AA@ 0000000180006a80     flags.obj
 0001:00005a98       ??_C@_0BI@NCAHLEBN@VOPT_AUTODETECTCODEPAGE?$AA@ 0000000180006a98     flags.obj
 0001:00005ab0       ??_C@_0BC@FGLBHLDI@VOPT_SHOWTITLEBAR?$AA@ 0000000180006ab0     flags.obj
 0001:00005ac8       ??_C@_0BA@GAIDGLME@VOPT_SHOWKEYBAR?$AA@ 0000000180006ac8     flags.obj
 0001:00005ad8       ??_C@_0BD@LEEGOJKA@VOPT_SHOWSCROLLBAR?$AA@ 0000000180006ad8     flags.obj
 0001:00005af0       ??_C@_0P@NEIKPMJJ@VOPT_QUICKVIEW?$AA@ 0000000180006af0     flags.obj
 0001:00005b00       ??_C@_09FIOJMNJ@VOPT_NONE?$AA@ 0000000180006b00     flags.obj
 0001:00005b10       ??_C@_0N@ILNDJNNO@VSMFL_REDRAW?$AA@ 0000000180006b10     flags.obj
 0001:00005b20       ??_C@_0L@DLLCFLOD@VSMFL_NONE?$AA@ 0000000180006b20     flags.obj
 0001:00005b30       ??_C@_0N@GHEHKHJN@VSP_NOREDRAW?$AA@ 0000000180006b30     flags.obj
 0001:00005b40       ??_C@_0M@LHNGMHFO@VSP_PERCENT?$AA@ 0000000180006b40     flags.obj
 0001:00005b50       ??_C@_0N@JGGGCNIP@VSP_RELATIVE?$AA@ 0000000180006b50     flags.obj
 0001:00005b60       ??_C@_0BA@JKDMJLJG@VSP_NORETNEWPOS?$AA@ 0000000180006b60     flags.obj
 0001:00005b70       ??_C@_08MOKEMBNE@VSP_NONE?$AA@ 0000000180006b70     flags.obj
 0001:00005b80       ??_C@_08FAPBJAKB@VMF_WRAP?$AA@ 0000000180006b80     flags.obj
 0001:00005b90       ??_C@_0N@GHBDMLON@VMF_WORDWRAP?$AA@ 0000000180006b90     flags.obj
 0001:00005ba0       ??_C@_08KDJLELDJ@VMF_NONE?$AA@ 0000000180006ba0     flags.obj
 0001:00005bb0       ??_C@_0BB@EDGIEBDF@ECF_TABMARKFIRST?$AA@ 0000000180006bb0     flags.obj
 0001:00005bc8       ??_C@_0BD@DKGCCJNG@ECF_TABMARKCURRENT?$AA@ 0000000180006bc8     flags.obj
 0001:00005be0       ??_C@_0P@BAFEMBAJ@ECF_AUTODELETE?$AA@ 0000000180006be0     flags.obj
 0001:00005bf0       ??_C@_08CDFMCHLP@ECF_NONE?$AA@ 0000000180006bf0     flags.obj
 0001:00005c00       ??_C@_0BA@KNNLMGCA@FIB_ENABLEEMPTY?$AA@ 0000000180006c00     flags.obj
 0001:00005c10       ??_C@_0N@DLDJCGJI@FIB_PASSWORD?$AA@ 0000000180006c10     flags.obj
 0001:00005c20       ??_C@_0O@DOHEGELC@FIB_EXPANDENV?$AA@ 0000000180006c20     flags.obj
 0001:00005c30       ??_C@_0BF@CEMIHIOK@FIB_NOUSELASTHISTORY?$AA@ 0000000180006c30     flags.obj
 0001:00005c48       ??_C@_0M@KJOJJDIM@FIB_BUTTONS?$AA@ 0000000180006c48     flags.obj
 0001:00005c58       ??_C@_0BA@COBBDHNL@FIB_NOAMPERSAND?$AA@ 0000000180006c58     flags.obj
 0001:00005c68       ??_C@_0N@LBOCEEGH@FIB_EDITPATH?$AA@ 0000000180006c68     flags.obj
 0001:00005c78       ??_C@_0BB@DCODFLEL@FIB_EDITPATHEXEC?$AA@ 0000000180006c78     flags.obj
 0001:00005c90       ??_C@_08HPFOCDKB@FIB_NONE?$AA@ 0000000180006c90     flags.obj
 0001:00005ca0       ??_C@_0L@NMBLFMBN@FPF_LOADED?$AA@ 0000000180006ca0     flags.obj
 0001:00005cb0       ??_C@_08GKECKCCJ@FPF_ANSI?$AA@ 0000000180006cb0     flags.obj
 0001:00005cc0       ??_C@_08OIOFCNLC@FPF_NONE?$AA@ 0000000180006cc0     flags.obj
 0001:00005cd0       ??_C@_0L@HODJIPGA@PN_CMPNAME?$AA@ 0000000180006cd0     flags.obj
 0001:00005ce0       ??_C@_0P@KDEENAHJ@PN_CMPNAMELIST?$AA@ 0000000180006ce0     flags.obj
 0001:00005cf0       ??_C@_0BA@BJCCEIOI@PN_GENERATENAME?$AA@ 0000000180006cf0     flags.obj
 0001:00005d00       ??_C@_0N@FEGPCCPJ@PN_CHECKMASK?$AA@ 0000000180006d00     flags.obj
 0001:00005d10       ??_C@_0M@NOOLKEBH@PN_SKIPPATH?$AA@ 0000000180006d10     flags.obj
 0001:00005d20       ??_C@_0BE@OPDBOAAE@PN_SHOWERRORMESSAGE?$AA@ 0000000180006d20     flags.obj
 0001:00005d38       ??_C@_07PFKJNCJP@PN_NONE?$AA@ 0000000180006d38     flags.obj
 0001:00005d40       ??_C@_0BG@GOMJDMCK@XLAT_SWITCHKEYBLAYOUT?$AA@ 0000000180006d40     flags.obj
 0001:00005d58       ??_C@_0BE@KOIJDNLA@XLAT_SWITCHKEYBBEEP?$AA@ 0000000180006d58     flags.obj
 0001:00005d70       ??_C@_0BH@KBFAFPNA@XLAT_USEKEYBLAYOUTNAME?$AA@ 0000000180006d70     flags.obj
 0001:00005d88       ??_C@_0BH@IANKLOAC@XLAT_CONVERTALLCMDLINE?$AA@ 0000000180006d88     flags.obj
 0001:00005da0       ??_C@_09JCNLKBBK@XLAT_NONE?$AA@ 0000000180006da0     flags.obj
 0001:00005db0       ??_C@_0N@PJEDCNNJ@FRS_RETUPDIR?$AA@ 0000000180006db0     flags.obj
 0001:00005dc0       ??_C@_09GHEPLOHO@FRS_RECUR?$AA@ 0000000180006dc0     flags.obj
 0001:00005dd0       ??_C@_0BA@JCPHOEAE@FRS_SCANSYMLINK?$AA@ 0000000180006dd0     flags.obj
 0001:00005de0       ??_C@_08JPCGJJKG@FRS_NONE?$AA@ 0000000180006de0     flags.obj
 0001:00005df0       ??_C@_0P@LJPBHEIE@MLF_SHOWERRMSG?$AA@ 0000000180006df0     flags.obj
 0001:00005e00       ??_C@_0BF@LMAGFLHF@MLF_DONOTUPDATEPANEL?$AA@ 0000000180006e00     flags.obj
 0001:00005e18       ??_C@_0P@EPFBLPAE@MLF_HOLDTARGET?$AA@ 0000000180006e18     flags.obj
 0001:00005e28       ??_C@_08EBKEJHAL@MLF_NONE?$AA@ 0000000180006e28     flags.obj
 0001:00005e38       ??_C@_0M@JDMKDBDH@FFFS_COMMAS?$AA@ 0000000180006e38     flags.obj
 0001:00005e48       ??_C@_0P@JPMLNBKL@FFFS_FLOATSIZE?$AA@ 0000000180006e48     flags.obj
 0001:00005e58       ??_C@_0BE@NPKCCEJ@FFFS_SHOWBYTESINDEX?$AA@ 0000000180006e58     flags.obj
 0001:00005e70       ??_C@_0O@FPIOAIMC@FFFS_ECONOMIC?$AA@ 0000000180006e70     flags.obj
 0001:00005e80       ??_C@_0O@HFIGPFIH@FFFS_THOUSAND?$AA@ 0000000180006e80     flags.obj
 0001:00005e90       ??_C@_0BC@LLLANJJO@FFFS_MINSIZEINDEX?$AA@ 0000000180006e90     flags.obj
 0001:00005ea8       ??_C@_0BH@PEGBPJKE@FFFS_MINSIZEINDEX_MASK?$AA@ 0000000180006ea8     flags.obj
 0001:00005ec0       ??_C@_09PBPAKNEI@FFFS_NONE?$AA@ 0000000180006ec0     flags.obj
 0001:00005ed0       ??_C@_0L@NHEJGKCF@PF_PRELOAD?$AA@ 0000000180006ed0     flags.obj
 0001:00005ee0       ??_C@_0BB@GCINAIGN@PF_DISABLEPANELS?$AA@ 0000000180006ee0     flags.obj
 0001:00005ef8       ??_C@_09OENCMPGE@PF_EDITOR?$AA@ 0000000180006ef8     flags.obj
 0001:00005f08       ??_C@_09NEKIJNNA@PF_VIEWER?$AA@ 0000000180006f08     flags.obj
 0001:00005f18       ??_C@_0P@MBLBBCNK@PF_FULLCMDLINE?$AA@ 0000000180006f18     flags.obj
 0001:00005f28       ??_C@_09GMFDAFKL@PF_DIALOG?$AA@ 0000000180006f28     flags.obj
 0001:00005f38       ??_C@_07MGEGJMPI@PF_NONE?$AA@ 0000000180006f38     flags.obj
 0001:00005f40       ??_C@_0BD@EGELEIIG@IPLFLAGS_SEPARATOR?$AA@ 0000000180006f40     flags.obj
 0001:00005f58       ??_C@_0O@JBNJFHHK@IPLFLAGS_NONE?$AA@ 0000000180006f58     flags.obj
 0001:00005f68       ??_C@_0BD@KGHJOBGM@PMFLAGS_FULLSCREEN?$AA@ 0000000180006f68     flags.obj
 0001:00005f80       ??_C@_0BH@GDAAKEMH@PMFLAGS_DETAILEDSTATUS?$AA@ 0000000180006f80     flags.obj
 0001:00005f98       ??_C@_0BI@BMHIBDMH@PMFLAGS_ALIGNEXTENSIONS?$AA@ 0000000180006f98     flags.obj
 0001:00005fb0       ??_C@_0BH@KOFCBJBO@PMFLAGS_CASECONVERSION?$AA@ 0000000180006fb0     flags.obj
 0001:00005fc8       ??_C@_0N@DLFMCMOB@PMFLAGS_NONE?$AA@ 0000000180006fc8     flags.obj
 0001:00005fd8       ??_C@_0BD@PBMGDJEM@OPIF_DISABLEFILTER?$AA@ 0000000180006fd8     flags.obj
 0001:00005ff0       ??_C@_0BH@FHBKALPD@OPIF_DISABLESORTGROUPS?$AA@ 0000000180006ff0     flags.obj
 0001:00006008       ??_C@_0BJ@NGLIANCL@OPIF_DISABLEHIGHLIGHTING?$AA@ 0000000180007008     flags.obj
 0001:00006028       ??_C@_0N@JANKJMLP@OPIF_ADDDOTS?$AA@ 0000000180007028     flags.obj
 0001:00006038       ??_C@_0BC@HOFHNJIG@OPIF_RAWSELECTION?$AA@ 0000000180007038     flags.obj
 0001:00006050       ??_C@_0P@OFEDJCO@OPIF_REALNAMES?$AA@ 0000000180007050     flags.obj
 0001:00006060       ??_C@_0BD@FPGMNAPD@OPIF_SHOWNAMESONLY?$AA@ 0000000180007060     flags.obj
 0001:00006078       ??_C@_0BJ@NMIFAPJD@OPIF_SHOWRIGHTALIGNNAMES?$AA@ 0000000180007078     flags.obj
 0001:00006098       ??_C@_0BG@HGPMKHIE@OPIF_SHOWPRESERVECASE?$AA@ 0000000180007098     flags.obj
 0001:000060b0       ??_C@_0BE@GJEJHNKJ@OPIF_COMPAREFATTIME?$AA@ 00000001800070b0     flags.obj
 0001:000060c8       ??_C@_0BB@PELHBPAM@OPIF_EXTERNALGET?$AA@ 00000001800070c8     flags.obj
 0001:000060e0       ??_C@_0BB@CFFPNDFK@OPIF_EXTERNALPUT?$AA@ 00000001800070e0     flags.obj
 0001:000060f8       ??_C@_0BE@LKEMICNM@OPIF_EXTERNALDELETE?$AA@ 00000001800070f8     flags.obj
 0001:00006110       ??_C@_0BD@JIMJPFEP@OPIF_EXTERNALMKDIR?$AA@ 0000000180007110     flags.obj
 0001:00006128       ??_C@_0BJ@CALDMPLF@OPIF_USEATTRHIGHLIGHTING?$AA@ 0000000180007128     flags.obj
 0001:00006148       ??_C@_0O@JHHHMHIG@OPIF_USECRC32?$AA@ 0000000180007148     flags.obj
 0001:00006158       ??_C@_0BB@PFDFAFHG@OPIF_USEFREESIZE?$AA@ 0000000180007158     flags.obj
 0001:00006170       ??_C@_0O@FJPLJDBC@OPIF_SHORTCUT?$AA@ 0000000180007170     flags.obj
 0001:00006180       ??_C@_09DOPJBMLM@OPIF_NONE?$AA@ 0000000180007180     flags.obj
 0001:00006190       ??_C@_0L@GEHHKNBL@OPM_SILENT?$AA@ 0000000180007190     flags.obj
 0001:000061a0       ??_C@_08EKEBOKEP@OPM_FIND?$AA@ 00000001800071a0     flags.obj
 0001:000061b0       ??_C@_08EHBLNDLO@OPM_VIEW?$AA@ 00000001800071b0     flags.obj
 0001:000061c0       ??_C@_08LAAGEMJG@OPM_EDIT?$AA@ 00000001800071c0     flags.obj
 0001:000061d0       ??_C@_0N@NDGKAFDM@OPM_TOPLEVEL?$AA@ 00000001800071d0     flags.obj
 0001:000061e0       ??_C@_09EBKAPHPA@OPM_DESCR?$AA@ 00000001800071e0     flags.obj
 0001:000061f0       ??_C@_0O@OPDAGBBE@OPM_QUICKVIEW?$AA@ 00000001800071f0     flags.obj
 0001:00006200       ??_C@_08LCEGJCAC@OPM_PGDN?$AA@ 0000000180007200     flags.obj
 0001:00006210       ??_C@_0N@HKCLLJDG@OPM_COMMANDS?$AA@ 0000000180007210     flags.obj
 0001:00006220       ??_C@_08EGEBMPBD@OPM_NONE?$AA@ 0000000180007220     flags.obj
 0001:00006230       ??_C@_0M@MIGJPBPE@FOSF_ACTIVE?$AA@ 0000000180007230     flags.obj
 0001:00006240       ??_C@_09FMOOJHDF@FOSF_NONE?$AA@ 0000000180007240     flags.obj
 0001:00006250       ??_C@_09HNBBLIGN@PCIF_NONE?$AA@ 0000000180007250     flags.obj
 0001:00006260       ??_C@_0BA@MAEBFMHC@FOREGROUND_BLUE?$AA@ 0000000180007260     flags.obj
 0001:00006270       ??_C@_0BB@PDFNMAI@FOREGROUND_GREEN?$AA@ 0000000180007270     flags.obj
 0001:00006288       ??_C@_0P@PBJHCFGA@FOREGROUND_RED?$AA@ 0000000180007288     flags.obj
 0001:00006298       ??_C@_0BF@OOGEJCC@FOREGROUND_INTENSITY?$AA@ 0000000180007298     flags.obj
 0001:000062b0       ??_C@_0BA@PIFINJCK@BACKGROUND_BLUE?$AA@ 00000001800072b0     flags.obj
 0001:000062c0       ??_C@_0BB@GKLNBMEL@BACKGROUND_GREEN?$AA@ 00000001800072c0     flags.obj
 0001:000062d8       ??_C@_0P@DANALJMC@BACKGROUND_RED?$AA@ 00000001800072d8     flags.obj
 0001:000062e8       ??_C@_0BF@NIGKKPCF@BACKGROUND_INTENSITY?$AA@ 00000001800072e8     flags.obj
 0001:00006300       ??_C@_0N@FEFOEFHG@CTRL_C_EVENT?$AA@ 0000000180007300     flags.obj
 0001:00006310       ??_C@_0BB@ELEIIFAE@CTRL_BREAK_EVENT?$AA@ 0000000180007310     flags.obj
 0001:00006328       ??_C@_0BB@KMPDMOKK@CTRL_CLOSE_EVENT?$AA@ 0000000180007328     flags.obj
 0001:00006340       ??_C@_0BC@MCKCEPAL@CTRL_LOGOFF_EVENT?$AA@ 0000000180007340     flags.obj
 0001:00006358       ??_C@_0BE@BCNEFGKM@CTRL_SHUTDOWN_EVENT?$AA@ 0000000180007358     flags.obj
 0001:00006370       ??_C@_0BC@BBOPHMOM@ENABLE_LINE_INPUT?$AA@ 0000000180007370     flags.obj
 0001:00006388       ??_C@_0BC@JPFKLHOC@ENABLE_ECHO_INPUT?$AA@ 0000000180007388     flags.obj
 0001:000063a0       ??_C@_0BH@EHINFMOF@ENABLE_PROCESSED_INPUT?$AA@ 00000001800073a0     flags.obj
 0001:000063b8       ??_C@_0BE@BLAHACNB@ENABLE_WINDOW_INPUT?$AA@ 00000001800073b8     flags.obj
 0001:000063d0       ??_C@_0BD@BJECBJPO@ENABLE_MOUSE_INPUT?$AA@ 00000001800073d0     flags.obj
 0001:000063e8       ??_C@_0BD@KJBPOMPN@ENABLE_INSERT_MODE?$AA@ 00000001800073e8     flags.obj
 0001:00006400       ??_C@_0BH@BJKMFKAO@ENABLE_QUICK_EDIT_MODE?$AA@ 0000000180007400     flags.obj
 0001:00006418       ??_C@_0BG@CBCHHIEH@ENABLE_EXTENDED_FLAGS?$AA@ 0000000180007418     flags.obj
 0001:00006430       ??_C@_0BF@PEBFEBKN@ENABLE_AUTO_POSITION?$AA@ 0000000180007430     flags.obj
 0001:00006448       ??_C@_0BI@MHKNPIFM@ENABLE_PROCESSED_OUTPUT?$AA@ 0000000180007448     flags.obj
 0001:00006460       ??_C@_0BK@CDKLKCHJ@ENABLE_WRAP_AT_EOL_OUTPUT?$AA@ 0000000180007460     flags.obj
 0001:00006480       ??_C@_09JBABGNAE@KEY_EVENT?$AA@ 0000000180007480     flags.obj
 0001:00006490       ??_C@_0M@CPILDGOO@MOUSE_EVENT?$AA@ 0000000180007490     flags.obj
 0001:000064a0       ??_C@_0BJ@OHDOHJKG@WINDOW_BUFFER_SIZE_EVENT?$AA@ 00000001800074a0     flags.obj
 0001:000064c0       ??_C@_0L@MPODFLFH@MENU_EVENT?$AA@ 00000001800074c0     flags.obj
 0001:000064d0       ??_C@_0M@LNGHCCGJ@FOCUS_EVENT?$AA@ 00000001800074d0     flags.obj
 0001:000064e0       ??_C@_0M@MKBGBFGO@CAPSLOCK_ON?$AA@ 00000001800074e0     flags.obj
 0001:000064f0       ??_C@_0N@EMEOEKDA@ENHANCED_KEY?$AA@ 00000001800074f0     flags.obj
 0001:00006500       ??_C@_0BC@GDHABBAP@RIGHT_ALT_PRESSED?$AA@ 0000000180007500     flags.obj
 0001:00006518       ??_C@_0BB@MCADLJJO@LEFT_ALT_PRESSED?$AA@ 0000000180007518     flags.obj
 0001:00006530       ??_C@_0BD@NEHHNAHO@RIGHT_CTRL_PRESSED?$AA@ 0000000180007530     flags.obj
 0001:00006548       ??_C@_0BC@FDNOAAAE@LEFT_CTRL_PRESSED?$AA@ 0000000180007548     flags.obj
 0001:00006560       ??_C@_0O@OGDFJMBK@SHIFT_PRESSED?$AA@ 0000000180007560     flags.obj
 0001:00006570       ??_C@_0L@IMGKKBIM@NUMLOCK_ON?$AA@ 0000000180007570     flags.obj
 0001:00006580       ??_C@_0O@LAHFNPLG@SCROLLLOCK_ON?$AA@ 0000000180007580     flags.obj
 0001:00006590       ??_C@_0BN@HACKHGAB@FROM_LEFT_1ST_BUTTON_PRESSED?$AA@ 0000000180007590     flags.obj
 0001:000065b0       ??_C@_0BJ@JECFAJNJ@RIGHTMOST_BUTTON_PRESSED?$AA@ 00000001800075b0     flags.obj
 0001:000065d0       ??_C@_0BN@BJCFPKCG@FROM_LEFT_2ND_BUTTON_PRESSED?$AA@ 00000001800075d0     flags.obj
 0001:000065f0       ??_C@_0BN@PMJNFPGM@FROM_LEFT_3RD_BUTTON_PRESSED?$AA@ 00000001800075f0     flags.obj
 0001:00006610       ??_C@_0BN@CNMHAAPD@FROM_LEFT_4TH_BUTTON_PRESSED?$AA@ 0000000180007610     flags.obj
 0001:00006630       ??_C@_0M@KKBDEELB@MOUSE_MOVED?$AA@ 0000000180007630     flags.obj
 0001:00006640       ??_C@_0N@EDCKBGJE@DOUBLE_CLICK?$AA@ 0000000180007640     flags.obj
 0001:00006650       ??_C@_0O@GABDOPO@MOUSE_WHEELED?$AA@ 0000000180007650     flags.obj
 0001:00006660       ??_C@_0BA@OOKCCMHH@KEY_WOW64_32KEY?$AA@ 0000000180007660     flags.obj
 0001:00006670       ??_C@_0BA@DBCPEIGE@KEY_WOW64_64KEY?$AA@ 0000000180007670     flags.obj
 0001:0000894c       ??_C@_06ICDCBJPI@Colors?$AA@ 000000018000994c     keysandcolors.obj
 0001:00008954       ??_C@_05GALAPKHH@Guids?$AA@ 0000000180009954     keysandcolors.obj
 0001:000091f0       ??_C@_01EEMJAFIK@?6?$AA@   000000018000a1f0     lflua.obj
 0001:000091f8       ??_C@_0BB@BJDGDOHH@cannot?5?$CFs?5?$CFs?3?5?$CFs?$AA@ 000000018000a1f8     lflua.obj
 0001:0000920c       ??_C@_03PKPBNCAL@?o?$LL?$LP?$AA@ 000000018000a20c     lflua.obj
 0001:00009210       ??_C@_06CCPPALKB@?$DNstdin?$AA@ 000000018000a210     lflua.obj
 0001:00009218       ??_C@_01EOFPKCAF@?$EA?$AA@ 000000018000a218     lflua.obj
 0001:0000921c       ??_C@_04PMOCAHAA@open?$AA@ 000000018000a21c     lflua.obj
 0001:00009224       ??_C@_15JJPIMNBO@?$AAr?$AAb?$AA?$AA@ 000000018000a224     lflua.obj
 0001:0000922c       ??_C@_06IEGCHAII@reopen?$AA@ 000000018000a22c     lflua.obj
 0001:00009234       ??_C@_04POLDLDMI@read?$AA@ 000000018000a234     lflua.obj
 0001:0000923c       ??_C@_02LOCGON@?$AA?$AA?$AA@ 000000018000a23c     lflua.obj
 0001:00009ad0       regex_methods              000000018000aad0     lregex.obj
 0001:00009b70       regex_functions            000000018000ab70     lregex.obj
 0001:00009c10       ??_C@_04CKFJHKAP@find?$AA@ 000000018000ac10     lregex.obj
 0001:00009c18       ??_C@_04GOLEAPFD@gsub?$AA@ 000000018000ac18     lregex.obj
 0001:00009c20       ??_C@_05FNONLPDI@match?$AA@ 000000018000ac20     lregex.obj
 0001:00009c28       ??_C@_05GFGPIPHI@findW?$AA@ 000000018000ac28     lregex.obj
 0001:00009c30       ??_C@_05HPGHPNC@gsubW?$AA@ 000000018000ac30     lregex.obj
 0001:00009c38       ??_C@_06NNKFJOLC@matchW?$AA@ 000000018000ac38     lregex.obj
 0001:00009c40       ??_C@_0O@OJAOCNID@bracketscount?$AA@ 000000018000ac40     lregex.obj
 0001:00009c50       ??_C@_04BDLIKKMN@__gc?$AA@ 000000018000ac50     lregex.obj
 0001:00009c58       ??_C@_06DPFCLDIO@gmatch?$AA@ 000000018000ac58     lregex.obj
 0001:00009c60       ??_C@_07PPMFDHAH@gmatchW?$AA@ 000000018000ac60     lregex.obj
 0001:00009c68       ??_C@_09KIEPBIJC@far_regex?$AA@ 000000018000ac68     lregex.obj
 0001:00009c78       ??_C@_0BO@PBOFMCLL@attempt?5to?5access?5freed?5regex?$AA@ 000000018000ac78     lregex.obj
 0001:00009c98       ??_C@_07IHINEPFG@?$CFs?5?$CI?$CFp?$CJ?$AA@ 000000018000ac98     lregex.obj
 0001:00009ca0       ??_C@_01KMDKNFGN@?1?$AA@   000000018000aca0     lregex.obj
 0001:00009ca8       ??_C@_0BE@BBBEAHLK@RECTL_CREATE?5failed?$AA@ 000000018000aca8     lregex.obj
 0001:00009cc0       ??_C@_0BL@HEFMPIBG@invalid?5regular?5expression?$AA@ 000000018000acc0     lregex.obj
 0001:00009ce0       ??_C@_0BK@JCLHPPNA@cannot?5add?5?$CFd?5stack?5slots?$AA@ 000000018000ace0     lregex.obj
 0001:00009d00       ??_C@_0BM@MOHHGMBK@string?5or?5table?5or?5function?$AA@ 000000018000ad00     lregex.obj
 0001:00009d20       ??_C@_0CG@IDFLGMFM@replace?5string?3?5invalid?5capture?5@ 000000018000ad20     lregex.obj
 0001:00009d48       ??_C@_0BJ@IMAIDFKH@invalid?5replacement?5type?$AA@ 000000018000ad48     lregex.obj
 0001:00009d68       ??_C@_0BE@KPDOHKBE@invalid?5return?5type?$AA@ 000000018000ad68     lregex.obj
 0001:00009d80       ??_C@_07NHABFFHN@__index?$AA@ 000000018000ad80     lregex.obj
 0001:00009d88       ??_C@_05FGAODPCE@regex?$AA@ 000000018000ad88     lregex.obj
 0001:0000a630       ??_C@_0BC@PMGNICBE@MacroPluginReturn?$AA@ 000000018000b630     luamacro.obj
 0001:0000a644       ??_C@_02JIEIHMJD@wl?$AA@   000000018000b644     luamacro.obj
 0001:0000a648       ??_C@_15PMCGDJNJ@?$AAO?$AAK?$AA?$AA@ 000000018000b648     luamacro.obj
 0001:0000a650       ??_C@_1BC@GBFPAMBP@?$AAL?$AAu?$AAa?$AAM?$AAa?$AAc?$AAr?$AAo?$AA?$AA@ 000000018000b650     luamacro.obj
 0001:0000a670       ??_C@_1FA@DAFHIDEP@?$AAt?$AAo?$AAo?$AA?5?$AAm?$AAa?$AAn?$AAy?$AA?5?$AAv?$AAa?$AAl?$AAu?$AAe?$AAs?$AA?5?$AAt?$AAo?$AA?5?$AAp?$AAl?$AAa?$AAc?$AAe?$AA?5?$AAo?$AAn?$AAt?$AAo?$AA?5?$AAL?$AAu@ 000000018000b670     luamacro.obj
 0001:0000a6c0       ??_C@_0BN@ICDOMFBB@invalid?5argument?5?$CD?$CFd?5to?5?8?$CFs?8?$AA@ 000000018000b6c0     luamacro.obj
 0001:0000a6e0       ??_C@_0BB@FCMFBGOM@invalid?5argument?$AA@ 000000018000b6e0     luamacro.obj
 0001:0000af80       usercontrol_methods        000000018000bf80     lusercontrol.obj
 0001:0000afd0       usercontrol_functions      000000018000bfd0     lusercontrol.obj
 0001:0000aff0       ??_C@_05MNDELLDN@__len?$AA@ 000000018000bff0     lusercontrol.obj
 0001:0000aff8       ??_C@_0L@GADKNKH@__newindex?$AA@ 000000018000bff8     lusercontrol.obj
 0001:0000b008       ??_C@_0BC@KFJDHEIC@CreateUserControl?$AA@ 000000018000c008     lusercontrol.obj
 0001:0000b020       ??_C@_0BA@MDNLMOMP@far_usercontrol?$AA@ 000000018000c020     lusercontrol.obj
 0001:0000b030       ??_C@_0BH@DOPNHMGD@bounds?5checking?5failed?$AA@ 000000018000c030     lusercontrol.obj
 0001:0000b048       ??_C@_09LDLEBFOB@rawhandle?$AA@ 000000018000c048     lusercontrol.obj
 0001:0000b054       ??_C@_04IMAAEPPE@Char?$AA@ 000000018000c054     lusercontrol.obj
 0001:0000b060       ??_C@_0L@PLFFHFAH@Attributes?$AA@ 000000018000c060     lusercontrol.obj
 0001:0000b070       ??_C@_0BD@BPIMECDH@X?5must?5be?5positive?$AA@ 000000018000c070     lusercontrol.obj
 0001:0000b088       ??_C@_0BD@MIGOMCGP@Y?5must?5be?5positive?$AA@ 000000018000c088     lusercontrol.obj
 0001:0000b0a0       FarFileFilterType          000000018000c0a0     service.obj
 0001:0000b0b0       FarTimerType               000000018000c0b0     service.obj
 0001:0000b0c0       FarTimerQueueKey           000000018000c0c0     service.obj
 0001:0000b0d0       FarDialogType              000000018000c0d0     service.obj
 0001:0000b0e0       SettingsType               000000018000c0e0     service.obj
 0001:0000b0f0       SettingsHandles            000000018000c0f0     service.obj
 0001:0000b108       PluginHandleType           000000018000c108     service.obj
 0001:0000b118       AddMacroDataType           000000018000c118     service.obj
 0001:0000b128       SavedScreenType            000000018000c128     service.obj
 0001:0000b138       FAR_VIRTUALKEYS            000000018000c138     service.obj
 0001:0000b148       FAR_FLAGSTABLE             000000018000c148     service.obj
 0001:0000b158       FAR_DN_STORAGE             000000018000c158     service.obj
 0001:0000ba20       timer_methods              000000018000ca20     service.obj
 0001:0000ba70       filefilter_methods         000000018000ca70     service.obj
 0001:0000bae0       dialog_methods             000000018000cae0     service.obj
 0001:0000bb30       Settings_methods           000000018000cb30     service.obj
 0001:0000bbd0       editor_funcs               000000018000cbd0     service.obj
 0001:0000be60       viewer_funcs               000000018000ce60     service.obj
 0001:0000bf00       panel_funcs                000000018000cf00     service.obj
 0001:0000c110       far_funcs                  000000018000d110     service.obj
 0001:0000c5a0       far_Dialog                 000000018000d5a0     service.obj
 0001:0000c890       api_functions              000000018000d890     service.obj
 0001:0000c958       ??_C@_07PHPIFDKI@LBUTTON?$AA@ 000000018000d958     service.obj
 0001:0000c960       ??_C@_07JOMJHALB@RBUTTON?$AA@ 000000018000d960     service.obj
 0001:0000c968       ??_C@_06JHILMIHF@CANCEL?$AA@ 000000018000d968     service.obj
 0001:0000c970       ??_C@_07DLFCFDDG@MBUTTON?$AA@ 000000018000d970     service.obj
 0001:0000c978       ??_C@_08OPILMHEG@XBUTTON1?$AA@ 000000018000d978     service.obj
 0001:0000c988       ??_C@_08MEKGJEIF@XBUTTON2?$AA@ 000000018000d988     service.obj
 0001:0000c994       ??_C@_04FJBHJJME@BACK?$AA@ 000000018000d994     service.obj
 0001:0000c99c       ??_C@_03CJMDHCGG@TAB?$AA@  000000018000d99c     service.obj
 0001:0000c9a0       ??_C@_05PONODPI@CLEAR?$AA@ 000000018000d9a0     service.obj
 0001:0000c9a8       ??_C@_06LJMOENAO@RETURN?$AA@ 000000018000d9a8     service.obj
 0001:0000c9b0       ??_C@_05OAHIEJBI@SHIFT?$AA@ 000000018000d9b0     service.obj
 0001:0000c9b8       ??_C@_07DBEDOPMC@CONTROL?$AA@ 000000018000d9b8     service.obj
 0001:0000c9c0       ??_C@_04IILMDFMO@MENU?$AA@ 000000018000d9c0     service.obj
 0001:0000c9c8       ??_C@_05DIAHPDGL@PAUSE?$AA@ 000000018000d9c8     service.obj
 0001:0000c9d0       ??_C@_07OPCFNGJB@CAPITAL?$AA@ 000000018000d9d0     service.obj
 0001:0000c9d8       ??_C@_04KGDAIAGM@KANA?$AA@ 000000018000d9d8     service.obj
 0001:0000c9e0       ??_C@_05PPKJGOLB@JUNJA?$AA@ 000000018000d9e0     service.obj
 0001:0000c9e8       ??_C@_05JEIAEFOF@FINAL?$AA@ 000000018000d9e8     service.obj
 0001:0000c9f0       ??_C@_05CHABPOPI@HANJA?$AA@ 000000018000d9f0     service.obj
 0001:0000c9f8       ??_C@_06CDPDIIDH@ESCAPE?$AA@ 000000018000d9f8     service.obj
 0001:0000ca00       ??_C@_0L@ODNCKDCK@NONCONVERT?$AA@ 000000018000da00     service.obj
 0001:0000ca0c       ??_C@_06INBBKPI@ACCEPT?$AA@ 000000018000da0c     service.obj
 0001:0000ca18       ??_C@_0L@HEHNEBED@MODECHANGE?$AA@ 000000018000da18     service.obj
 0001:0000ca24       ??_C@_05CAEOFMEP@SPACE?$AA@ 000000018000da24     service.obj
 0001:0000ca2c       ??_C@_05BFDHCIJM@PRIOR?$AA@ 000000018000da2c     service.obj
 0001:0000ca34       ??_C@_04MOKMKBJN@NEXT?$AA@ 000000018000da34     service.obj
 0001:0000ca3c       ??_C@_03JMGAKCCH@END?$AA@  000000018000da3c     service.obj
 0001:0000ca40       ??_C@_04GHGFPGNC@HOME?$AA@ 000000018000da40     service.obj
 0001:0000ca48       ??_C@_04KCNEHMIH@LEFT?$AA@ 000000018000da48     service.obj
 0001:0000ca50       ??_C@_02NAHCJHOC@UP?$AA@   000000018000da50     service.obj
 0001:0000ca54       ??_C@_05PMAFOJDE@RIGHT?$AA@ 000000018000da54     service.obj
 0001:0000ca5c       ??_C@_04FANAOELO@DOWN?$AA@ 000000018000da5c     service.obj
 0001:0000ca64       ??_C@_06LCPJPOPK@SELECT?$AA@ 000000018000da64     service.obj
 0001:0000ca6c       ??_C@_05ECKPOFCN@PRINT?$AA@ 000000018000da6c     service.obj
 0001:0000ca78       ??_C@_07LBDEDADF@EXECUTE?$AA@ 000000018000da78     service.obj
 0001:0000ca80       ??_C@_08EMOKHGD@SNAPSHOT?$AA@ 000000018000da80     service.obj
 0001:0000ca8c       ??_C@_06OEMEAEKN@INSERT?$AA@ 000000018000da8c     service.obj
 0001:0000ca94       ??_C@_06FKDAMKFP@DELETE?$AA@ 000000018000da94     service.obj
 0001:0000ca9c       ??_C@_04DOKPJKJF@HELP?$AA@ 000000018000da9c     service.obj
 0001:0000caa4       ??_C@_01GBGANLPD@0?$AA@    000000018000daa4     service.obj
 0001:0000caa8       ??_C@_01HIHLOKLC@1?$AA@    000000018000daa8     service.obj
 0001:0000caac       ??_C@_01FDFGLJHB@2?$AA@    000000018000daac     service.obj
 0001:0000cab0       ??_C@_01EKENIIDA@3?$AA@    000000018000dab0     service.obj
 0001:0000cab4       ??_C@_01FAMBOPH@4?$AA@     000000018000dab4     service.obj
 0001:0000cab8       ??_C@_01BMBHCPLG@5?$AA@    000000018000dab8     service.obj
 0001:0000cabc       ??_C@_01DHDKHMHF@6?$AA@    000000018000dabc     service.obj
 0001:0000cac0       ??_C@_01COCBENDE@7?$AA@    000000018000dac0     service.obj
 0001:0000cac4       ??_C@_01KJLJFBPL@8?$AA@    000000018000dac4     service.obj
 0001:0000cac8       ??_C@_01LAKCGALK@9?$AA@    000000018000dac8     service.obj
 0001:0000cacc       ??_C@_01FHEEJDEE@A?$AA@    000000018000dacc     service.obj
 0001:0000cad0       ??_C@_01HMGJMAIH@B?$AA@    000000018000dad0     service.obj
 0001:0000cad4       ??_C@_01GFHCPBMG@C?$AA@    000000018000dad4     service.obj
 0001:0000cad8       ??_C@_01CKDDGHAB@D?$AA@    000000018000dad8     service.obj
 0001:0000cadc       ??_C@_01DDCIFGEA@E?$AA@    000000018000dadc     service.obj
 0001:0000cae0       ??_C@_01BIAFAFID@F?$AA@    000000018000dae0     service.obj
 0001:0000cae4       ??_C@_01BBODEMC@G?$AA@     000000018000dae4     service.obj
 0001:0000cae8       ??_C@_01IGIGCIAN@H?$AA@    000000018000dae8     service.obj
 0001:0000caec       ??_C@_01JPJNBJEM@I?$AA@    000000018000daec     service.obj
 0001:0000caf0       ??_C@_01LELAEKIP@J?$AA@    000000018000daf0     service.obj
 0001:0000caf4       ??_C@_01KNKLHLMO@K?$AA@    000000018000daf4     service.obj
 0001:0000caf8       ??_C@_01OCOKONAJ@L?$AA@    000000018000daf8     service.obj
 0001:0000cafc       ??_C@_01PLPBNMEI@M?$AA@    000000018000dafc     service.obj
 0001:0000cb00       ??_C@_01NANMIPIL@N?$AA@    000000018000db00     service.obj
 0001:0000cb04       ??_C@_01MJMHLOMK@O?$AA@    000000018000db04     service.obj
 0001:0000cb08       ??_C@_01EJNLAFE@P?$AA@     000000018000db08     service.obj
 0001:0000cb0c       ??_C@_01BNIGIBBF@Q?$AA@    000000018000db0c     service.obj
 0001:0000cb10       ??_C@_01DGKLNCNG@R?$AA@    000000018000db10     service.obj
 0001:0000cb14       ??_C@_01CPLAODJH@S?$AA@    000000018000db14     service.obj
 0001:0000cb18       ??_C@_01GAPBHFFA@T?$AA@    000000018000db18     service.obj
 0001:0000cb1c       ??_C@_01HJOKEEBB@U?$AA@    000000018000db1c     service.obj
 0001:0000cb20       ??_C@_01FCMHBHNC@V?$AA@    000000018000db20     service.obj
 0001:0000cb24       ??_C@_01ELNMCGJD@W?$AA@    000000018000db24     service.obj
 0001:0000cb28       ??_C@_01MMEEDKFM@X?$AA@    000000018000db28     service.obj
 0001:0000cb2c       ??_C@_01NFFPALBN@Y?$AA@    000000018000db2c     service.obj
 0001:0000cb30       ??_C@_01POHCFINO@Z?$AA@    000000018000db30     service.obj
 0001:0000cb34       ??_C@_04ODLFFOHF@LWIN?$AA@ 000000018000db34     service.obj
 0001:0000cb3c       ??_C@_04DMGFHHJG@RWIN?$AA@ 000000018000db3c     service.obj
 0001:0000cb44       ??_C@_04GKGJFGJO@APPS?$AA@ 000000018000db44     service.obj
 0001:0000cb4c       ??_C@_05DJAECLDN@SLEEP?$AA@ 000000018000db4c     service.obj
 0001:0000cb58       ??_C@_07NHIPMMJH@NUMPAD0?$AA@ 000000018000db58     service.obj
 0001:0000cb60       ??_C@_07MOJEPNNG@NUMPAD1?$AA@ 000000018000db60     service.obj
 0001:0000cb68       ??_C@_07OFLJKOBF@NUMPAD2?$AA@ 000000018000db68     service.obj
 0001:0000cb70       ??_C@_07PMKCJPFE@NUMPAD3?$AA@ 000000018000db70     service.obj
 0001:0000cb78       ??_C@_07LDODAJJD@NUMPAD4?$AA@ 000000018000db78     service.obj
 0001:0000cb80       ??_C@_07KKPIDINC@NUMPAD5?$AA@ 000000018000db80     service.obj
 0001:0000cb88       ??_C@_07IBNFGLBB@NUMPAD6?$AA@ 000000018000db88     service.obj
 0001:0000cb90       ??_C@_07JIMOFKFA@NUMPAD7?$AA@ 000000018000db90     service.obj
 0001:0000cb98       ??_C@_07BPFGEGJP@NUMPAD8?$AA@ 000000018000db98     service.obj
 0001:0000cba0       ??_C@_07GENHHNO@NUMPAD9?$AA@ 000000018000dba0     service.obj
 0001:0000cba8       ??_C@_08LDEOAAGM@MULTIPLY?$AA@ 000000018000dba8     service.obj
 0001:0000cbb4       ??_C@_03BOJFLAKG@ADD?$AA@  000000018000dbb4     service.obj
 0001:0000cbb8       ??_C@_09POPINEFK@SEPARATOR?$AA@ 000000018000dbb8     service.obj
 0001:0000cbc8       ??_C@_08MGBEENML@SUBTRACT?$AA@ 000000018000dbc8     service.obj
 0001:0000cbd8       ??_C@_07LJPMJDLL@DECIMAL?$AA@ 000000018000dbd8     service.obj
 0001:0000cbe0       ??_C@_06FBFCJJMP@DIVIDE?$AA@ 000000018000dbe0     service.obj
 0001:0000cbe8       ??_C@_02LCPENACN@F1?$AA@   000000018000dbe8     service.obj
 0001:0000cbec       ??_C@_02JJNJIDOO@F2?$AA@   000000018000dbec     service.obj
 0001:0000cbf0       ??_C@_02IAMCLCKP@F3?$AA@   000000018000dbf0     service.obj
 0001:0000cbf4       ??_C@_02MPIDCEGI@F4?$AA@   000000018000dbf4     service.obj
 0001:0000cbf8       ??_C@_02NGJIBFCJ@F5?$AA@   000000018000dbf8     service.obj
 0001:0000cbfc       ??_C@_02PNLFEGOK@F6?$AA@   000000018000dbfc     service.obj
 0001:0000cc00       ??_C@_02OEKOHHKL@F7?$AA@   000000018000dc00     service.obj
 0001:0000cc04       ??_C@_02GDDGGLGE@F8?$AA@   000000018000dc04     service.obj
 0001:0000cc08       ??_C@_02HKCNFKCF@F9?$AA@   000000018000dc08     service.obj
 0001:0000cc0c       ??_C@_03JKCLJOFG@F10?$AA@  000000018000dc0c     service.obj
 0001:0000cc10       ??_C@_03IDDAKPBH@F11?$AA@  000000018000dc10     service.obj
 0001:0000cc14       ??_C@_03KIBNPMNE@F12?$AA@  000000018000dc14     service.obj
 0001:0000cc18       ??_C@_03LBAGMNJF@F13?$AA@  000000018000dc18     service.obj
 0001:0000cc1c       ??_C@_03POEHFLFC@F14?$AA@  000000018000dc1c     service.obj
 0001:0000cc20       ??_C@_03OHFMGKBD@F15?$AA@  000000018000dc20     service.obj
 0001:0000cc24       ??_C@_03MMHBDJNA@F16?$AA@  000000018000dc24     service.obj
 0001:0000cc28       ??_C@_03NFGKAIJB@F17?$AA@  000000018000dc28     service.obj
 0001:0000cc2c       ??_C@_03FCPCBEFO@F18?$AA@  000000018000dc2c     service.obj
 0001:0000cc30       ??_C@_03ELOJCFBP@F19?$AA@  000000018000dc30     service.obj
 0001:0000cc34       ??_C@_03JIGNCAAP@F20?$AA@  000000018000dc34     service.obj
 0001:0000cc38       ??_C@_03IBHGBBEO@F21?$AA@  000000018000dc38     service.obj
 0001:0000cc3c       ??_C@_03KKFLECIN@F22?$AA@  000000018000dc3c     service.obj
 0001:0000cc40       ??_C@_03LDEAHDMM@F23?$AA@  000000018000dc40     service.obj
 0001:0000cc44       ??_C@_03PMABOFAL@F24?$AA@  000000018000dc44     service.obj
 0001:0000cc48       ??_C@_07FLMEHHJP@NUMLOCK?$AA@ 000000018000dc48     service.obj
 0001:0000cc50       ??_C@_06FNIKALAE@SCROLL?$AA@ 000000018000dc50     service.obj
 0001:0000cc58       ??_C@_0O@DBBJDALK@OEM_NEC_EQUAL?$AA@ 000000018000dc58     service.obj
 0001:0000cc68       ??_C@_0P@JKGCFGCD@OEM_FJ_MASSHOU?$AA@ 000000018000dc68     service.obj
 0001:0000cc78       ??_C@_0P@NIEOFNLG@OEM_FJ_TOUROKU?$AA@ 000000018000dc78     service.obj
 0001:0000cc88       ??_C@_0M@IBEHGLCM@OEM_FJ_LOYA?$AA@ 000000018000dc88     service.obj
 0001:0000cc98       ??_C@_0M@FOJHECMP@OEM_FJ_ROYA?$AA@ 000000018000dc98     service.obj
 0001:0000cca4       ??_C@_06EPHNCIMI@LSHIFT?$AA@ 000000018000dca4     service.obj
 0001:0000ccac       ??_C@_06HIJMMPFL@RSHIFT?$AA@ 000000018000dcac     service.obj
 0001:0000ccb8       ??_C@_08IKMONEBG@LCONTROL?$AA@ 000000018000dcb8     service.obj
 0001:0000ccc8       ??_C@_08OOMMENPF@RCONTROL?$AA@ 000000018000dcc8     service.obj
 0001:0000ccd4       ??_C@_05IHMGKJGH@LMENU?$AA@ 000000018000dcd4     service.obj
 0001:0000ccdc       ??_C@_05LOBKMKIM@RMENU?$AA@ 000000018000dcdc     service.obj
 0001:0000cce8       ??_C@_0N@OAJIELLG@BROWSER_BACK?$AA@ 000000018000dce8     service.obj
 0001:0000ccf8       ??_C@_0BA@ENOAJOGH@BROWSER_FORWARD?$AA@ 000000018000dcf8     service.obj
 0001:0000cd08       ??_C@_0BA@GDNDIDGJ@BROWSER_REFRESH?$AA@ 000000018000dd08     service.obj
 0001:0000cd18       ??_C@_0N@HKPDGANH@BROWSER_STOP?$AA@ 000000018000dd18     service.obj
 0001:0000cd28       ??_C@_0P@BEAEBJDD@BROWSER_SEARCH?$AA@ 000000018000dd28     service.obj
 0001:0000cd38       ??_C@_0BC@BOMJIH@BROWSER_FAVORITES?$AA@ 000000018000dd38     service.obj
 0001:0000cd50       ??_C@_0N@NOOKCEKA@BROWSER_HOME?$AA@ 000000018000dd50     service.obj
 0001:0000cd60       ??_C@_0M@ENOHKBMG@VOLUME_MUTE?$AA@ 000000018000dd60     service.obj
 0001:0000cd70       ??_C@_0M@JOOBBDNO@VOLUME_DOWN?$AA@ 000000018000dd70     service.obj
 0001:0000cd80       ??_C@_09MGPMNMJC@VOLUME_UP?$AA@ 000000018000dd80     service.obj
 0001:0000cd90       ??_C@_0BB@KLAENPA@MEDIA_NEXT_TRACK?$AA@ 000000018000dd90     service.obj
 0001:0000cda8       ??_C@_0BB@CMOIJKPH@MEDIA_PREV_TRACK?$AA@ 000000018000dda8     service.obj
 0001:0000cdc0       ??_C@_0L@KBJOCDHK@MEDIA_STOP?$AA@ 000000018000ddc0     service.obj
 0001:0000cdd0       ??_C@_0BB@HAEMIJHO@MEDIA_PLAY_PAUSE?$AA@ 000000018000ddd0     service.obj
 0001:0000cde8       ??_C@_0M@GCIKMBID@LAUNCH_MAIL?$AA@ 000000018000dde8     service.obj
 0001:0000cdf8       ??_C@_0BE@FADJJAPM@LAUNCH_MEDIA_SELECT?$AA@ 000000018000ddf8     service.obj
 0001:0000ce10       ??_C@_0M@MGLJIDDM@LAUNCH_APP1?$AA@ 000000018000de10     service.obj
 0001:0000ce20       ??_C@_0M@ONJENAPP@LAUNCH_APP2?$AA@ 000000018000de20     service.obj
 0001:0000ce2c       ??_C@_05OIODNPAD@OEM_1?$AA@ 000000018000de2c     service.obj
 0001:0000ce38       ??_C@_08LDJEIPBH@OEM_PLUS?$AA@ 000000018000de38     service.obj
 0001:0000ce48       ??_C@_09CLPFJEOD@OEM_COMMA?$AA@ 000000018000de48     service.obj
 0001:0000ce58       ??_C@_09OGMLCNMG@OEM_MINUS?$AA@ 000000018000de58     service.obj
 0001:0000ce68       ??_C@_0L@DNNMNDGM@OEM_PERIOD?$AA@ 000000018000de68     service.obj
 0001:0000ce74       ??_C@_05MDMOIMMA@OEM_2?$AA@ 000000018000de74     service.obj
 0001:0000ce7c       ??_C@_05NKNFLNIB@OEM_3?$AA@ 000000018000de7c     service.obj
 0001:0000ce84       ??_C@_05JFJECLEG@OEM_4?$AA@ 000000018000de84     service.obj
 0001:0000ce8c       ??_C@_05IMIPBKAH@OEM_5?$AA@ 000000018000de8c     service.obj
 0001:0000ce94       ??_C@_05KHKCEJME@OEM_6?$AA@ 000000018000de94     service.obj
 0001:0000ce9c       ??_C@_05LOLJHIIF@OEM_7?$AA@ 000000018000de9c     service.obj
 0001:0000cea4       ??_C@_05DJCBGEEK@OEM_8?$AA@ 000000018000dea4     service.obj
 0001:0000ceb0       ??_C@_07PEFKMFIE@OEM_102?$AA@ 000000018000deb0     service.obj
 0001:0000ceb8       ??_C@_0L@EFLJCPAM@PROCESSKEY?$AA@ 000000018000deb8     service.obj
 0001:0000cec4       ??_C@_06HOICDKCB@PACKET?$AA@ 000000018000dec4     service.obj
 0001:0000ced0       ??_C@_09CAKPMKHM@OEM_RESET?$AA@ 000000018000ded0     service.obj
 0001:0000cee0       ??_C@_08INMNLJCK@OEM_JUMP?$AA@ 000000018000dee0     service.obj
 0001:0000cef0       ??_C@_07JNOAEEG@OEM_PA1?$AA@ 000000018000def0     service.obj
 0001:0000cef8       ??_C@_07CCPDFHIF@OEM_PA2?$AA@ 000000018000def8     service.obj
 0001:0000cf00       ??_C@_07DLOIGGME@OEM_PA3?$AA@ 000000018000df00     service.obj
 0001:0000cf08       ??_C@_0L@OCAIHDP@OEM_WSCTRL?$AA@ 000000018000df08     service.obj
 0001:0000cf14       ??_C@_04BNGOAFAJ@ATTN?$AA@ 000000018000df14     service.obj
 0001:0000cf1c       ??_C@_05HGAHFFFL@CRSEL?$AA@ 000000018000df1c     service.obj
 0001:0000cf24       ??_C@_05OKOOKOOH@EXSEL?$AA@ 000000018000df24     service.obj
 0001:0000cf2c       ??_C@_05CCFENDFJ@EREOF?$AA@ 000000018000df2c     service.obj
 0001:0000cf34       ??_C@_04MKCNCBEG@PLAY?$AA@ 000000018000df34     service.obj
 0001:0000cf3c       ??_C@_04LGBIGMFG@ZOOM?$AA@ 000000018000df3c     service.obj
 0001:0000cf44       ??_C@_06LJIOOKLP@NONAME?$AA@ 000000018000df44     service.obj
 0001:0000cf4c       ??_C@_03KCLDMPAE@PA1?$AA@  000000018000df4c     service.obj
 0001:0000cf50       ??_C@_09MBBEHOCK@OEM_CLEAR?$AA@ 000000018000df50     service.obj
 0001:0000cf5c       ??_C@_05LCLENNFI@table?$AA@ 000000018000df5c     service.obj
 0001:0000cf64       ??_C@_06ICGJLFIM@string?$AA@ 000000018000df64     service.obj
 0001:0000cf70       ??_C@_0P@LKPINHLK@FreeFileFilter?$AA@ 000000018000df70     service.obj
 0001:0000cf80       ??_C@_0BA@JGEOEAE@OpenFiltersMenu?$AA@ 000000018000df80     service.obj
 0001:0000cf90       ??_C@_0BB@OPPOFOAK@StartingToFilter?$AA@ 000000018000df90     service.obj
 0001:0000cfa8       ??_C@_0P@JDMCHDIM@IsFileInFilter?$AA@ 000000018000dfa8     service.obj
 0001:0000cfb8       ??_C@_04MIIPNNEF@send?$AA@ 000000018000dfb8     service.obj
 0001:0000cfc0       ??_C@_06JBKGCNBB@Delete?$AA@ 000000018000dfc0     service.obj
 0001:0000cfc8       ??_C@_04PAFOOALK@Enum?$AA@ 000000018000dfc8     service.obj
 0001:0000cfd0       ??_C@_04HJMOFLDF@Free?$AA@ 000000018000dfd0     service.obj
 0001:0000cfd8       ??_C@_03NNDHPFFO@Get?$AA@  000000018000dfd8     service.obj
 0001:0000cfdc       ??_C@_03CEMDFJG@Set?$AA@   000000018000dfdc     service.obj
 0001:0000cfe0       ??_C@_0N@OELJMCEC@CreateSubkey?$AA@ 000000018000dfe0     service.obj
 0001:0000cff0       ??_C@_0L@CPCKAMD@OpenSubkey?$AA@ 000000018000dff0     service.obj
 0001:0000d000       ??_C@_08EGJLHNCO@AddColor?$AA@ 000000018000e000     service.obj
 0001:0000d010       ??_C@_0BD@DOFEEDDC@AddSessionBookmark?$AA@ 000000018000e010     service.obj
 0001:0000d028       ??_C@_0BG@IGFHDIIN@ClearSessionBookmarks?$AA@ 000000018000e028     service.obj
 0001:0000d040       ??_C@_08PDEJHGJI@DelColor?$AA@ 000000018000e040     service.obj
 0001:0000d050       ??_C@_0M@LPIECDD@DeleteBlock?$AA@ 000000018000e050     service.obj
 0001:0000d060       ??_C@_0L@BCLIBKOC@DeleteChar?$AA@ 000000018000e060     service.obj
 0001:0000d070       ??_C@_0BG@KOELEFCN@DeleteSessionBookmark?$AA@ 000000018000e070     service.obj
 0001:0000d088       ??_C@_0N@EKENACAE@DeleteString?$AA@ 000000018000e088     service.obj
 0001:0000d098       ??_C@_06MJDIICIN@Editor?$AA@ 000000018000e098     service.obj
 0001:0000d0a0       ??_C@_0L@HDLPOLMA@ExpandTabs?$AA@ 000000018000e0a0     service.obj
 0001:0000d0b0       ??_C@_0N@MGAOADJN@GetBookmarks?$AA@ 000000018000e0b0     service.obj
 0001:0000d0c0       ??_C@_08JOPFJIPE@GetColor?$AA@ 000000018000e0c0     service.obj
 0001:0000d0d0       ??_C@_0M@FECPLAMN@GetFileName?$AA@ 000000018000e0d0     service.obj
 0001:0000d0e0       ??_C@_07NAJNLNAF@GetInfo?$AA@ 000000018000e0e0     service.obj
 0001:0000d0e8       ??_C@_0N@KIILHCLH@GetSelection?$AA@ 000000018000e0e8     service.obj
 0001:0000d0f8       ??_C@_0BE@LBJJGOGD@GetSessionBookmarks?$AA@ 000000018000e0f8     service.obj
 0001:0000d110       ??_C@_09HBLKHMEA@GetString?$AA@ 000000018000e110     service.obj
 0001:0000d120       ??_C@_0L@IDFHDAHP@GetStringW?$AA@ 000000018000e120     service.obj
 0001:0000d130       ??_C@_0N@ICPGLOEG@InsertString?$AA@ 000000018000e130     service.obj
 0001:0000d140       ??_C@_0L@JMOIGJIA@InsertText?$AA@ 000000018000e140     service.obj
 0001:0000d150       ??_C@_0M@BINOKANK@InsertTextW?$AA@ 000000018000e150     service.obj
 0001:0000d160       ??_C@_0BE@CNGODNDI@NextSessionBookmark?$AA@ 000000018000e160     service.obj
 0001:0000d178       ??_C@_0BE@IEBIGOAP@PrevSessionBookmark?$AA@ 000000018000e178     service.obj
 0001:0000d190       ??_C@_0N@FNCEPAJJ@ProcessInput?$AA@ 000000018000e190     service.obj
 0001:0000d1a0       ??_C@_04GMBKPCGK@Quit?$AA@ 000000018000e1a0     service.obj
 0001:0000d1a8       ??_C@_09KINLOJJJ@ReadInput?$AA@ 000000018000e1a8     service.obj
 0001:0000d1b8       ??_C@_09DBPLBJBJ@RealToTab?$AA@ 000000018000e1b8     service.obj
 0001:0000d1c4       ??_C@_06KAPLBEK@Redraw?$AA@ 000000018000e1c4     service.obj
 0001:0000d1d0       ??_C@_08FBDDPFPJ@SaveFile?$AA@ 000000018000e1d0     service.obj
 0001:0000d1dc       ??_C@_06HJGPBJLE@Select?$AA@ 000000018000e1dc     service.obj
 0001:0000d1e8       ??_C@_09PPEOOGEC@SetKeyBar?$AA@ 000000018000e1e8     service.obj
 0001:0000d1f8       ??_C@_08CCKJEGOF@SetParam?$AA@ 000000018000e1f8     service.obj
 0001:0000d208       ??_C@_0M@GKIFPNAD@SetPosition?$AA@ 000000018000e208     service.obj
 0001:0000d218       ??_C@_09FPPPFNNC@SetString?$AA@ 000000018000e218     service.obj
 0001:0000d228       ??_C@_0L@JNHIIHDG@SetStringW?$AA@ 000000018000e228     service.obj
 0001:0000d238       ??_C@_08GMCCAJLF@SetTitle?$AA@ 000000018000e238     service.obj
 0001:0000d248       ??_C@_08JNAOBKMI@GetTitle?$AA@ 000000018000e248     service.obj
 0001:0000d258       ??_C@_0BF@LIMPGNED@SubscribeChangeEvent?$AA@ 000000018000e258     service.obj
 0001:0000d270       ??_C@_09JFBCONJH@TabToReal?$AA@ 000000018000e270     service.obj
 0001:0000d280       ??_C@_08IBJJAHJG@UndoRedo?$AA@ 000000018000e280     service.obj
 0001:0000d290       ??_C@_07JMDLHPJF@SetMode?$AA@ 000000018000e290     service.obj
 0001:0000d298       ??_C@_06PJECNADJ@Viewer?$AA@ 000000018000e298     service.obj
 0001:0000d2a0       ??_C@_0BB@PJGDGIKA@CheckPanelsExist?$AA@ 000000018000e2a0     service.obj
 0001:0000d2b8       ??_C@_0P@DFBDDHFA@ClearSelection?$AA@ 000000018000e2b8     service.obj
 0001:0000d2c8       ??_C@_0L@KOHCMOPM@GetCmdLine?$AA@ 000000018000e2c8     service.obj
 0001:0000d2d8       ??_C@_0O@NLDIMJEA@GetCmdLinePos?$AA@ 000000018000e2d8     service.obj
 0001:0000d2e8       ??_C@_0BE@CBPLLCEH@GetCmdLineSelection?$AA@ 000000018000e2e8     service.obj
 0001:0000d300       ??_C@_0P@CMFANDFM@GetColumnTypes?$AA@ 000000018000e300     service.obj
 0001:0000d310       ??_C@_0BA@DJGLDCBG@GetColumnWidths?$AA@ 000000018000e310     service.obj
 0001:0000d320       ??_C@_0BE@JPAIJBCI@GetCurrentPanelItem?$AA@ 000000018000e320     service.obj
 0001:0000d338       ??_C@_0BC@NGKPIKGL@GetPanelDirectory?$AA@ 000000018000e338     service.obj
 0001:0000d350       ??_C@_0P@GODLFFFJ@GetPanelFormat?$AA@ 000000018000e350     service.obj
 0001:0000d360       ??_C@_0BB@LCMBHPNI@GetPanelHostFile?$AA@ 000000018000e360     service.obj
 0001:0000d378       ??_C@_0N@HPIPGDFA@GetPanelInfo?$AA@ 000000018000e378     service.obj
 0001:0000d388       ??_C@_0N@HAFLAIHA@GetPanelItem?$AA@ 000000018000e388     service.obj
 0001:0000d398       ??_C@_0P@HCBKDPMP@GetPanelPrefix?$AA@ 000000018000e398     service.obj
 0001:0000d3a8       ??_C@_0BF@MEMFMMGB@GetSelectedPanelItem?$AA@ 000000018000e3a8     service.obj
 0001:0000d3c0       ??_C@_0O@HEGDGAJG@GetUserScreen?$AA@ 000000018000e3c0     service.obj
 0001:0000d3d0       ??_C@_0O@EHOCCHAL@InsertCmdLine?$AA@ 000000018000e3d0     service.obj
 0001:0000d3e0       ??_C@_0O@OMMHIHHH@IsActivePanel?$AA@ 000000018000e3e0     service.obj
 0001:0000d3f0       ??_C@_0M@LCEPDNPK@RedrawPanel?$AA@ 000000018000e3f0     service.obj
 0001:0000d400       ??_C@_0P@OPKJJMLB@SetActivePanel?$AA@ 000000018000e400     service.obj
 0001:0000d410       ??_C@_0L@LAFNHJLF@SetCmdLine?$AA@ 000000018000e410     service.obj
 0001:0000d420       ??_C@_0O@KECGHKDH@SetCmdLinePos?$AA@ 000000018000e420     service.obj
 0001:0000d430       ??_C@_0BE@IPNAPCDL@SetCmdLineSelection?$AA@ 000000018000e430     service.obj
 0001:0000d448       ??_C@_0BE@PAPEKLCP@SetDirectoriesFirst?$AA@ 000000018000e448     service.obj
 0001:0000d460       ??_C@_0BC@PDKEABHF@SetPanelDirectory?$AA@ 000000018000e460     service.obj
 0001:0000d478       ??_C@_0N@NMDFLOPL@SetSelection?$AA@ 000000018000e478     service.obj
 0001:0000d488       ??_C@_0M@CMMMGIDG@SetSortMode?$AA@ 000000018000e488     service.obj
 0001:0000d498       ??_C@_0N@HCHLALN@SetSortOrder?$AA@ 000000018000e498     service.obj
 0001:0000d4a8       ??_C@_0O@LHNNDOB@SetUserScreen?$AA@ 000000018000e4a8     service.obj
 0001:0000d4b8       ??_C@_0M@IENJPEBA@SetViewMode?$AA@ 000000018000e4b8     service.obj
 0001:0000d4c8       ??_C@_0M@EICBHAOA@UpdatePanel?$AA@ 000000018000e4c8     service.obj
 0001:0000d4d8       ??_C@_0BC@BIIKJLKB@PluginStartupInfo?$AA@ 000000018000e4d8     service.obj
 0001:0000d4f0       ??_C@_0L@PJAHNOGM@DialogInit?$AA@ 000000018000e4f0     service.obj
 0001:0000d500       ??_C@_09DBEDLMHB@DialogRun?$AA@ 000000018000e500     service.obj
 0001:0000d510       ??_C@_0L@DLFLHLOO@DialogFree?$AA@ 000000018000e510     service.obj
 0001:0000d520       ??_C@_0P@HLOFPDFP@SendDlgMessage?$AA@ 000000018000e520     service.obj
 0001:0000d530       ??_C@_0L@CKELNLCE@GetDlgItem?$AA@ 000000018000e530     service.obj
 0001:0000d540       ??_C@_0L@DEGEGMGN@SetDlgItem?$AA@ 000000018000e540     service.obj
 0001:0000d550       ??_C@_0BK@EBIPEKDH@SubscribeDialogDrawEvents?$AA@ 000000018000e550     service.obj
 0001:0000d570       ??_C@_0L@MCFABBED@GetDirList?$AA@ 000000018000e570     service.obj
 0001:0000d57c       ??_C@_06KCCBBIBJ@GetMsg?$AA@ 000000018000e57c     service.obj
 0001:0000d588       ??_C@_0BB@HIDBFOJJ@GetPluginDirList?$AA@ 000000018000e588     service.obj
 0001:0000d59c       ??_C@_04IFEHPILC@Menu?$AA@ 000000018000e59c     service.obj
 0001:0000d5a8       ??_C@_07BEIHKDLJ@Message?$AA@ 000000018000e5a8     service.obj
 0001:0000d5b0       ??_C@_0O@CGLFPNOD@RestoreScreen?$AA@ 000000018000e5b0     service.obj
 0001:0000d5c0       ??_C@_0L@PGGGPLFK@SaveScreen?$AA@ 000000018000e5c0     service.obj
 0001:0000d5d0       ??_C@_08DAHHHDJC@ShowHelp?$AA@ 000000018000e5d0     service.obj
 0001:0000d5e0       ??_C@_08IAADAJIH@InputBox?$AA@ 000000018000e5e0     service.obj
 0001:0000d5f0       ??_C@_0L@HHLOIHOP@AdvControl?$AA@ 000000018000e5f0     service.obj
 0001:0000d600       ??_C@_0N@GHGEMEN@MacroLoadAll?$AA@ 000000018000e600     service.obj
 0001:0000d610       ??_C@_0N@NAGBAPAE@MacroSaveAll?$AA@ 000000018000e610     service.obj
 0001:0000d620       ??_C@_0O@KGHDMPAJ@MacroGetState?$AA@ 000000018000e620     service.obj
 0001:0000d630       ??_C@_0N@PNLHCOIE@MacroGetArea?$AA@ 000000018000e630     service.obj
 0001:0000d640       ??_C@_09KGKKBHMO@MacroPost?$AA@ 000000018000e640     service.obj
 0001:0000d650       ??_C@_0L@KBAKOGFP@MacroCheck?$AA@ 000000018000e650     service.obj
 0001:0000d660       ??_C@_08KAFLEHAN@MacroAdd?$AA@ 000000018000e660     service.obj
 0001:0000d670       ??_C@_0M@KFMHCNNB@MacroDelete?$AA@ 000000018000e670     service.obj
 0001:0000d680       ??_C@_0BC@MJDKBAPF@MacroGetLastError?$AA@ 000000018000e680     service.obj
 0001:0000d698       ??_C@_0N@COEPENFH@MacroExecute?$AA@ 000000018000e698     service.obj
 0001:0000d6a8       ??_C@_0BB@BICELPOF@CreateFileFilter?$AA@ 000000018000e6a8     service.obj
 0001:0000d6c0       ??_C@_0L@CHJBHF@LoadPlugin?$AA@ 000000018000e6c0     service.obj
 0001:0000d6d0       ??_C@_0N@DHIONCLI@UnloadPlugin?$AA@ 000000018000e6d0     service.obj
 0001:0000d6e0       ??_C@_0BB@IJHIBGJA@ForcedLoadPlugin?$AA@ 000000018000e6e0     service.obj
 0001:0000d6f8       ??_C@_0L@DACPHGGH@FindPlugin?$AA@ 000000018000e6f8     service.obj
 0001:0000d708       ??_C@_0BF@KLOGLFMF@GetPluginInformation?$AA@ 000000018000e708     service.obj
 0001:0000d720       ??_C@_0L@JIDCIJHM@GetPlugins?$AA@ 000000018000e720     service.obj
 0001:0000d730       ??_C@_0P@IKAEEPOB@IsPluginLoaded?$AA@ 000000018000e730     service.obj
 0001:0000d740       ??_C@_0P@HMKEDHIE@CreateSettings?$AA@ 000000018000e740     service.obj
 0001:0000d750       ??_C@_0N@GOMOBHDB@FreeSettings?$AA@ 000000018000e750     service.obj
 0001:0000d760       ??_C@_0M@IFKFGKML@ColorDialog?$AA@ 000000018000e760     service.obj
 0001:0000d770       ??_C@_0BA@EOCNNPOG@CopyToClipboard?$AA@ 000000018000e770     service.obj
 0001:0000d780       ??_C@_0BD@PLIHDKFC@PasteFromClipboard?$AA@ 000000018000e780     service.obj
 0001:0000d798       ??_C@_0BC@FJDIKOMH@InputRecordToName?$AA@ 000000018000e798     service.obj
 0001:0000d7b0       ??_C@_0BC@FFNOIDFI@NameToInputRecord?$AA@ 000000018000e7b0     service.obj
 0001:0000d7c8       ??_C@_08HGLFNLMB@LStricmp?$AA@ 000000018000e7c8     service.obj
 0001:0000d7d8       ??_C@_09GALOFBAC@LStrnicmp?$AA@ 000000018000e7d8     service.obj
 0001:0000d7e8       ??_C@_0M@KPPMMAOL@ProcessName?$AA@ 000000018000e7e8     service.obj
 0001:0000d7f8       ??_C@_0M@KFCNKLDK@GetPathRoot?$AA@ 000000018000e7f8     service.obj
 0001:0000d808       ??_C@_0BE@EPGHGPJC@GetReparsePointInfo?$AA@ 000000018000e808     service.obj
 0001:0000d820       ??_C@_08DNJCLFF@LIsAlpha?$AA@ 000000018000e820     service.obj
 0001:0000d830       ??_C@_0M@LKJIEECA@LIsAlphanum?$AA@ 000000018000e830     service.obj
 0001:0000d840       ??_C@_08MAHKICD@LIsLower?$AA@ 000000018000e840     service.obj
 0001:0000d850       ??_C@_08FHLJMDJK@LIsUpper?$AA@ 000000018000e850     service.obj
 0001:0000d860       ??_C@_09LPKAHGM@LLowerBuf?$AA@ 000000018000e860     service.obj
 0001:0000d870       ??_C@_09GLKFOOEP@LUpperBuf?$AA@ 000000018000e870     service.obj
 0001:0000d87c       ??_C@_06ILCHIEBO@MkTemp?$AA@ 000000018000e87c     service.obj
 0001:0000d884       ??_C@_06DKBBJCCG@MkLink?$AA@ 000000018000e884     service.obj
 0001:0000d890       ??_C@_0N@CCDDAJK@TruncPathStr?$AA@ 000000018000e890     service.obj
 0001:0000d8a0       ??_C@_08BNEIIKEJ@TruncStr?$AA@ 000000018000e8a0     service.obj
 0001:0000d8b0       ??_C@_0BA@CLEHBIPM@RecursiveSearch?$AA@ 000000018000e8b0     service.obj
 0001:0000d8c0       ??_C@_0M@HKHGOOHG@ConvertPath?$AA@ 000000018000e8c0     service.obj
 0001:0000d8cc       ??_C@_04OCDKHGII@XLat?$AA@ 000000018000e8cc     service.obj
 0001:0000d8d8       ??_C@_0P@BGLLKGOI@FormatFileSize?$AA@ 000000018000e8d8     service.obj
 0001:0000d8e8       ??_C@_08KJBLDCDF@FarClock?$AA@ 000000018000e8e8     service.obj
 0001:0000d8f8       ??_C@_0BD@ELMHPHAC@CPluginStartupInfo?$AA@ 000000018000e8f8     service.obj
 0001:0000d910       ??_C@_0BE@DJLJEKBK@GetCurrentDirectory?$AA@ 000000018000e910     service.obj
 0001:0000d928       ??_C@_0N@MOMBJEKA@GetFileOwner?$AA@ 000000018000e928     service.obj
 0001:0000d938       ??_C@_0BB@JBNBALEM@GetNumberOfLinks?$AA@ 000000018000e938     service.obj
 0001:0000d950       ??_C@_0O@BJEAJNBH@MakeMenuItems?$AA@ 000000018000e950     service.obj
 0001:0000d960       ??_C@_0BB@HLFLDCHO@RunDefaultScript?$AA@ 000000018000e960     service.obj
 0001:0000d974       ??_C@_04JLAJABDJ@Show?$AA@ 000000018000e974     service.obj
 0001:0000d97c       ??_C@_05NHFJDMOA@Timer?$AA@ 000000018000e97c     service.obj
 0001:0000d984       ??_C@_02KFNNKBCK@io?$AA@   000000018000e984     service.obj
 0001:0000d988       ??_C@_02EHCHIAMF@os?$AA@   000000018000e988     service.obj
 0001:0000d98c       ??_C@_04CFDJAKFL@math?$AA@ 000000018000e98c     service.obj
 0001:0000d998       ??_C@_07GAJMMAJO@unicode?$AA@ 000000018000e998     service.obj
 0001:0000d9a0       ??_C@_03JECLAOEA@win?$AA@  000000018000e9a0     service.obj
 0001:0000d9a8       ??_C@_09GJGOMOL@lua51?4dll?$AA@ 000000018000e9a8     service.obj
 0001:0000d9b8       ??_C@_0M@PLOBHAKE@luaopen_bit?$AA@ 000000018000e9b8     service.obj
 0001:0000d9c8       ??_C@_0M@IALDMMNC@luaopen_ffi?$AA@ 000000018000e9c8     service.obj
 0001:0000d9d8       ??_C@_0M@DOFFFIEL@luaopen_jit?$AA@ 000000018000e9d8     service.obj
 0001:0000d9e8       ??_C@_0BE@OEPKKAAB@integer?5or?5userdata?$AA@ 000000018000e9e8     service.obj
 0001:0000da00       ??_C@_0BD@PNJHLBDA@invalid?5flag?3?5?$CC?$CFs?$CC?$AA@ 000000018000ea00     service.obj
 0001:0000da18       ??_C@_0N@JJLBBDOC@invalid?5flag?$AA@ 000000018000ea18     service.obj
 0001:0000da28       ??_C@_0BJ@MIKGPOKL@invalid?5flag?5combination?$AA@ 000000018000ea28     service.obj
 0001:0000da48       ??_C@_0P@EANMLDOP@MousePositionX?$AA@ 000000018000ea48     service.obj
 0001:0000da58       ??_C@_0P@FJMHICKO@MousePositionY?$AA@ 000000018000ea58     service.obj
 0001:0000da68       ??_C@_0M@BJAICPIE@ButtonState?$AA@ 000000018000ea68     service.obj
 0001:0000da78       ??_C@_0L@EMFBJIPA@EventFlags?$AA@ 000000018000ea78     service.obj
 0001:0000da88       ??_C@_07EEJLMCNH@CurLine?$AA@ 000000018000ea88     service.obj
 0001:0000da90       ??_C@_06EDBJMJDC@CurPos?$AA@ 000000018000ea90     service.obj
 0001:0000da98       ??_C@_09EGONKHKB@CurTabPos?$AA@ 000000018000ea98     service.obj
 0001:0000daa8       ??_C@_0O@OKGGHEJK@TopScreenLine?$AA@ 000000018000eaa8     service.obj
 0001:0000dab8       ??_C@_07GDAKJHLE@LeftPos?$AA@ 000000018000eab8     service.obj
 0001:0000dac0       ??_C@_08LLJICOLD@Overtype?$AA@ 000000018000eac0     service.obj
 0001:0000dad0       ??_C@_0L@GEIEADPN@ModuleName?$AA@ 000000018000ead0     service.obj
 0001:0000dae0       ??_C@_09HOIHBHIM@ModuleDir?$AA@ 000000018000eae0     service.obj
 0001:0000daf0       ??_C@_0L@JLHCLFBG@PluginGuid?$AA@ 000000018000eaf0     service.obj
 0001:0000db00       ??_C@_08GGMFPBHM@EditorID?$AA@ 000000018000eb00     service.obj
 0001:0000db10       ??_C@_0M@CPDBGLHN@WindowSizeX?$AA@ 000000018000eb10     service.obj
 0001:0000db20       ??_C@_0M@DGCKFKDM@WindowSizeY?$AA@ 000000018000eb20     service.obj
 0001:0000db30       ??_C@_0L@PMKENHMA@TotalLines?$AA@ 000000018000eb30     service.obj
 0001:0000db40       ??_C@_09HKBEFIPN@BlockType?$AA@ 000000018000eb40     service.obj
 0001:0000db50       ??_C@_0P@GAEEHNHE@BlockStartLine?$AA@ 000000018000eb50     service.obj
 0001:0000db60       ??_C@_07KHIHFBFN@Options?$AA@ 000000018000eb60     service.obj
 0001:0000db68       ??_C@_07FLDNELFM@TabSize?$AA@ 000000018000eb68     service.obj
 0001:0000db70       ??_C@_0O@EBLDFOPH@BookmarkCount?$AA@ 000000018000eb70     service.obj
 0001:0000db80       ??_C@_0BF@ODFKBFAK@SessionBookmarkCount?$AA@ 000000018000eb80     service.obj
 0001:0000db98       ??_C@_08CPAOHJDL@CurState?$AA@ 000000018000eb98     service.obj
 0001:0000dba8       ??_C@_0N@DAJMJAE@StringLength?$AA@ 000000018000eba8     service.obj
 0001:0000dbb8       ??_C@_08JPMALCFA@SelStart?$AA@ 000000018000ebb8     service.obj
 0001:0000dbc4       ??_C@_06JLEHDHII@SelEnd?$AA@ 000000018000ebc4     service.obj
 0001:0000dbd0       ??_C@_0L@IFNFGDGN@StringText?$AA@ 000000018000ebd0     service.obj
 0001:0000dbe0       ??_C@_09IBGOAAEM@StringEOL?$AA@ 000000018000ebe0     service.obj
 0001:0000dbec       ??_C@_01LOCGONAA@?$AA?$AA@ 000000018000ebec     service.obj
 0001:0000dbf0       ??_C@_06MFLCIING@redraw?$AA@ 000000018000ebf0     service.obj
 0001:0000dbf8       ??_C@_07HICINA@restore?$AA@ 000000018000ebf8     service.obj
 0001:0000dc00       ??_C@_0CG@LAKEGANL@must?5be?5?8redraw?8?0?5?8restore?8?0?5or?5@ 000000018000ec00     service.obj
 0001:0000dc28       ??_C@_04LIDDHMOL@Line?$AA@ 000000018000ec28     service.obj
 0001:0000dc30       ??_C@_06OIIFPIKD@Cursor?$AA@ 000000018000ec30     service.obj
 0001:0000dc38       ??_C@_0L@GDDEHGKI@ScreenLine?$AA@ 000000018000ec38     service.obj
 0001:0000dc48       ??_C@_0O@CIAFMMMB@BlockStartPos?$AA@ 000000018000ec48     service.obj
 0001:0000dc58       ??_C@_0L@EKLJJHPF@BlockWidth?$AA@ 000000018000ec58     service.obj
 0001:0000dc68       ??_C@_0M@NKKGBDGK@BlockHeight?$AA@ 000000018000ec68     service.obj
 0001:0000dc78       ??_C@_09JFPCGCOC@StartLine?$AA@ 000000018000ec78     service.obj
 0001:0000dc88       ??_C@_08JBNOANJG@StartPos?$AA@ 000000018000ec88     service.obj
 0001:0000dc98       ??_C@_07DCKCOCOC@EndLine?$AA@ 000000018000ec98     service.obj
 0001:0000dca0       ??_C@_06KGHIGMHC@EndPos?$AA@ 000000018000eca0     service.obj
 0001:0000dca8       ??_C@_0BA@HNIJJEO@ForegroundColor?$AA@ 000000018000eca8     service.obj
 0001:0000dcb8       ??_C@_0BA@DPMBBMBG@BackgroundColor?$AA@ 000000018000ecb8     service.obj
 0001:0000dcc8       ??_C@_0O@NHKEGDJF@GUID?5required?$AA@ 000000018000ecc8     service.obj
 0001:0000dcd8       ??_C@_0BJ@BMOGHFAN@table?5or?5number?5expected?$AA@ 000000018000ecd8     service.obj
 0001:0000dcf8       ??_C@_08KGEIBGG@Priority?$AA@ 000000018000ecf8     service.obj
 0001:0000dd04       ??_C@_05PDOBBJNA@Color?$AA@ 000000018000ed04     service.obj
 0001:0000dd10       ??_C@_09KDLBEGCN@EventType?$AA@ 000000018000ed10     service.obj
 0001:0000dd20       ??_C@_07HPHPOAEG@KeyDown?$AA@ 000000018000ed20     service.obj
 0001:0000dd28       ??_C@_0M@FGGHEADP@RepeatCount?$AA@ 000000018000ed28     service.obj
 0001:0000dd38       ??_C@_0BA@KCCLHPM@VirtualScanCode?$AA@ 000000018000ed38     service.obj
 0001:0000dd48       ??_C@_0M@PBJKDIHH@UnicodeChar?$AA@ 000000018000ed48     service.obj
 0001:0000dd54       ??_C@_05GIPJKPFG@SizeX?$AA@ 000000018000ed54     service.obj
 0001:0000dd5c       ??_C@_05HBOCJOBH@SizeY?$AA@ 000000018000ed5c     service.obj
 0001:0000dd68       ??_C@_09GEJJJAHL@CommandId?$AA@ 000000018000ed68     service.obj
 0001:0000dd78       ??_C@_08GPNNBNIL@SetFocus?$AA@ 000000018000ed78     service.obj
 0001:0000dd88       ??_C@_0M@BEDENHPD@invalid?5key?$AA@ 000000018000ed88     service.obj
 0001:0000dd98       ??_C@_19IBCFILMC@?$AAM?$AAe?$AAn?$AAu?$AA?$AA@ 000000018000ed98     service.obj
 0001:0000dda8       ??_C@_0BN@JBAMKCCJ@must?5be?5table?0?5string?5or?5nil?$AA@ 000000018000eda8     service.obj
 0001:0000ddc8       ??_C@_09FDAFFNEA@MaxHeight?$AA@ 000000018000edc8     service.obj
 0001:0000ddd4       ??_C@_06DDHCBBGN@Bottom?$AA@ 000000018000edd4     service.obj
 0001:0000dde0       ??_C@_09CFELDMD@HelpTopic?$AA@ 000000018000ede0     service.obj
 0001:0000ddf0       ??_C@_0M@GGMLPAIK@SelectIndex?$AA@ 000000018000edf0     service.obj
 0001:0000ddfc       ??_C@_02HOGEDOAB@Id?$AA@   000000018000edfc     service.obj
 0001:0000de00       ??_C@_07FJOBMBFC@checked?$AA@ 000000018000ee00     service.obj
 0001:0000de08       ??_C@_09MOAJOJKN@separator?$AA@ 000000018000ee08     service.obj
 0001:0000de18       ??_C@_07DBNODEFN@disable?$AA@ 000000018000ee18     service.obj
 0001:0000de20       ??_C@_06JHIAOIKD@grayed?$AA@ 000000018000ee20     service.obj
 0001:0000de28       ??_C@_06JIKFICKK@hidden?$AA@ 000000018000ee28     service.obj
 0001:0000de30       ??_C@_08CJLOJPNI@selected?$AA@ 000000018000ee30     service.obj
 0001:0000de40       ??_C@_08MMCKBNNI@AccelKey?$AA@ 000000018000ee40     service.obj
 0001:0000de50       ??_C@_08PNHLLJE@BreakKey?$AA@ 000000018000ee50     service.obj
 0001:0000de5c       ??_C@_15FMBEJGOH@?$AAO?$AAk?$AA?$AA@ 000000018000ee5c     service.obj
 0001:0000de68       ??_C@_1BC@IBCAPFAE@?$AAO?$AAk?$AAC?$AAa?$AAn?$AAc?$AAe?$AAl?$AA?$AA@ 000000018000ee68     service.obj
 0001:0000de80       ??_C@_1CC@HODOHOHB@?$AAA?$AAb?$AAo?$AAr?$AAt?$AAR?$AAe?$AAt?$AAr?$AAy?$AAI?$AAg?$AAn?$AAo?$AAr?$AAe?$AA?$AA@ 000000018000ee80     service.obj
 0001:0000dea8       ??_C@_1M@GGPOIMAD@?$AAY?$AAe?$AAs?$AAN?$AAo?$AA?$AA@ 000000018000eea8     service.obj
 0001:0000deb8       ??_C@_1BI@BNDFIGCI@?$AAY?$AAe?$AAs?$AAN?$AAo?$AAC?$AAa?$AAn?$AAc?$AAe?$AAl?$AA?$AA@ 000000018000eeb8     service.obj
 0001:0000ded0       ??_C@_1BI@KMMIHPHF@?$AAR?$AAe?$AAt?$AAr?$AAy?$AAC?$AAa?$AAn?$AAc?$AAe?$AAl?$AA?$AA@ 000000018000eed0     service.obj
 0001:0000dee8       ??_C@_1DG@LMKDDADI@?$AA?$DM?$AAn?$AAo?$AAn?$AA?9?$AAs?$AAt?$AAr?$AAi?$AAn?$AAg?$AA?5?$AAe?$AAr?$AAr?$AAo?$AAr?$AA?5?$AAm?$AAe?$AAs?$AAs?$AAa?$AAg?$AAe?$AA?$DO?$AA?$AA@ 000000018000eee8     service.obj
 0001:0000df20       ??_C@_15IEGBJKPD@?$AA?3?$AA?6?$AA?$AA@ 000000018000ef20     service.obj
 0001:0000df28       ??_C@_19FFLPMPBO@?$AA?6?$AA?5?$AA?5?$AA?5?$AA?$AA@ 000000018000ef28     service.obj
 0001:0000df34       ??_C@_15JCKODCLA@?$AA?6?$AA?7?$AA?$AA@ 000000018000ef34     service.obj
 0001:0000df40       ??_C@_1M@ILHOPKA@?$AAE?$AAr?$AAr?$AAo?$AAr?$AA?$AA@ 000000018000ef40     service.obj
 0001:0000df50       ??_C@_08FNIIFOJC@tostring?$AA@ 000000018000ef50     service.obj
 0001:0000df60       ??_C@_0BJ@JOELOGM@cannot?5convert?5to?5string?$AA@ 000000018000ef60     service.obj
 0001:0000df80       ??_C@_1BA@HHOMBECE@?$AAM?$AAe?$AAs?$AAs?$AAa?$AAg?$AAe?$AA?$AA@ 000000018000ef80     service.obj
 0001:0000df90       ??_C@_17PAGBAIDI@?$AA?$DL?$AAO?$AAK?$AA?$AA@ 000000018000ef90     service.obj
 0001:0000df98       ??_C@_09ENKGJCEC@OwnerGuid?$AA@ 000000018000ef98     service.obj
 0001:0000dfa8       ??_C@_0N@CCPLCIHE@PluginHandle?$AA@ 000000018000efa8     service.obj
 0001:0000dfb8       ??_C@_0N@HEHBMBNM@PluginObject?$AA@ 000000018000efb8     service.obj
 0001:0000dfc8       ??_C@_09BKHPOLGD@PanelType?$AA@ 000000018000efc8     service.obj
 0001:0000dfd4       ??_C@_04GOOOJOPP@left?$AA@ 000000018000efd4     service.obj
 0001:0000dfdc       ??_C@_03FGFCOCMD@top?$AA@  000000018000efdc     service.obj
 0001:0000dfe0       ??_C@_05DHJDAOHK@right?$AA@ 000000018000efe0     service.obj
 0001:0000dfe8       ??_C@_06PMMPCIPB@bottom?$AA@ 000000018000efe8     service.obj
 0001:0000dff0       ??_C@_09MCEJMINN@PanelRect?$AA@ 000000018000eff0     service.obj
 0001:0000e000       ??_C@_0M@DDGFKGKJ@ItemsNumber?$AA@ 000000018000f000     service.obj
 0001:0000e010       ??_C@_0BE@EOBAHHNK@SelectedItemsNumber?$AA@ 000000018000f010     service.obj
 0001:0000e028       ??_C@_0M@JMILNLLF@CurrentItem?$AA@ 000000018000f028     service.obj
 0001:0000e038       ??_C@_0N@CDHIFJIH@TopPanelItem?$AA@ 000000018000f038     service.obj
 0001:0000e048       ??_C@_08IMMBLBLF@ViewMode?$AA@ 000000018000f048     service.obj
 0001:0000e058       ??_C@_08CENECNJD@SortMode?$AA@ 000000018000f058     service.obj
 0001:0000e064       ??_C@_04FABLJDN@Name?$AA@  000000018000f064     service.obj
 0001:0000e06c       ??_C@_05LOJBNELM@Param?$AA@ 000000018000f06c     service.obj
 0001:0000e074       ??_C@_04PBAHLACE@File?$AA@ 000000018000f074     service.obj
 0001:0000e080       ??_C@_08HGEAFCFN@PluginId?$AA@ 000000018000f080     service.obj
 0001:0000e090       ??_C@_0BA@MLHECKCE@table?5or?5string?$AA@ 000000018000f090     service.obj
 0001:0000e0a0       ??_C@_0BD@CKJHMJBG@non?9positive?5index?$AA@ 000000018000f0a0     service.obj
 0001:0000e0b8       ??_C@_0BA@GNKNKKDM@number?5or?5table?$AA@ 000000018000f0b8     service.obj
 0001:0000e0c8       ??_C@_0CI@DDAJHJKO@?$CFs?5?9?5unsupported?5type?5in?5dialog?5@ 000000018000f0c8     service.obj
 0001:0000e0f0       ??_C@_0CD@JIANOKII@unsupported?5flag?5in?5dialog?5item?5@ 000000018000f0f0     service.obj
 0001:0000e118       ??_C@_0CB@EOGFCCCC@value?5at?5index?5?$CFd?5is?5not?5a?5table@ 000000018000f118     service.obj
 0001:0000e140       ??_C@_0O@FEBHKEHB@closed?5dialog?$AA@ 000000018000f140     service.obj
 0001:0000e150       ??_C@_0BK@NEMPGLFN@operation?5not?5implemented?$AA@ 000000018000f150     service.obj
 0001:0000e16c       ??_C@_04KPCPLBPL@Left?$AA@ 000000018000f16c     service.obj
 0001:0000e174       ??_C@_03PGGAENPN@Top?$AA@  000000018000f174     service.obj
 0001:0000e178       ??_C@_05DADPALEM@Right?$AA@ 000000018000f178     service.obj
 0001:0000e180       ??_C@_0CK@JHNDGJBB@element?5?$CD?$CFd?5in?5argument?5?$CD4?5is?5no@ 000000018000f180     service.obj
 0001:0000e1b0       ??_C@_0L@CECHCPAP@StartIndex?$AA@ 000000018000f1b0     service.obj
 0001:0000e1bc       ??_C@_05IJGIMMHE@Count?$AA@ 000000018000f1bc     service.obj
 0001:0000e1c8       ??_C@_07NOCIGAPP@Pattern?$AA@ 000000018000f1c8     service.obj
 0001:0000e1d0       ??_C@_09IMOCKOO@SelectPos?$AA@ 000000018000f1d0     service.obj
 0001:0000e1dc       ??_C@_06DJONBJOP@TopPos?$AA@ 000000018000f1dc     service.obj
 0001:0000e1e8       ??_C@_09OGCBKCAK@MaxLength?$AA@ 000000018000f1e8     service.obj
 0001:0000e1f4       ??_C@_05FNNGFGLF@Index?$AA@ 000000018000f1f4     service.obj
 0001:0000e200       ??_C@_07GHGHLGFI@GetType?$AA@ 000000018000f200     service.obj
 0001:0000e208       ??_C@_07MMLMCDAI@ValType?$AA@ 000000018000f208     service.obj
 0001:0000e210       ??_C@_05LPIJGKJ@Value?$AA@ 000000018000f210     service.obj
 0001:0000e218       ??_C@_0L@LPFMIAHH@helpstring?$AA@ 000000018000f218     service.obj
 0001:0000e228       ??_C@_0P@NABDHFON@getvaluestring?$AA@ 000000018000f228     service.obj
 0001:0000e238       ??_C@_0BJ@IINAPFDG@Items?$FL?$CFd?$FN?5is?5not?5a?5table?$AA@ 000000018000f238     service.obj
 0001:0000e258       ??_C@_0CC@GBOJFNBI@error?5occured?5in?5dialog?5procedur@ 000000018000f258     service.obj
 0001:0000e280       ??_C@_0M@EHMONPJO@?$CFs?5?$CIclosed?$CJ?$AA@ 000000018000f280     service.obj
 0001:0000e290       ??_C@_08GDAJJKGC@ViewerID?$AA@ 000000018000f290     service.obj
 0001:0000e2a0       ??_C@_07MJHBHMFM@FilePos?$AA@ 000000018000f2a0     service.obj
 0001:0000e2a8       ??_C@_07FBAHDBGN@CurMode?$AA@ 000000018000f2a8     service.obj
 0001:0000e2b0       ??_C@_06IMBBKDFH@iParam?$AA@ 000000018000f2b0     service.obj
 0001:0000e2b8       ??_C@_1BE@CGKCNEEP@?$AAI?$AAn?$AAp?$AAu?$AAt?$AA?5?$AAB?$AAo?$AAx?$AA?$AA@ 000000018000f2b8     service.obj
 0001:0000e2d0       ??_C@_1CA@PCDNIBFH@?$AAE?$AAn?$AAt?$AAe?$AAr?$AA?5?$AAt?$AAh?$AAe?$AA?5?$AAt?$AAe?$AAx?$AAt?$AA?3?$AA?$AA@ 000000018000f2d0     service.obj
 0001:0000e2f0       ??_C@_0BG@GAFLOAPP@command?5not?5supported?$AA@ 000000018000f2f0     service.obj
 0001:0000e308       ??_C@_09MIJAKHKB@Completed?$AA@ 000000018000f308     service.obj
 0001:0000e314       ??_C@_05KGEAEGFG@Total?$AA@ 000000018000f314     service.obj
 0001:0000e320       ??_C@_0P@DJOANNIK@?$CFd?4?$CFd?4?$CFd?4?$CFd?4?$CFd?$AA@ 000000018000f320     service.obj
 0001:0000e330       ??_C@_03FCCPIJGJ@Pos?$AA@  000000018000f330     service.obj
 0001:0000e338       ??_C@_08NNKIOIN@TypeName?$AA@ 000000018000f338     service.obj
 0001:0000e348       ??_C@_07ONPPLIAF@ErrCode?$AA@ 000000018000f348     service.obj
 0001:0000e350       ??_C@_07LJDOKIBM@ErrPosX?$AA@ 000000018000f350     service.obj
 0001:0000e358       ??_C@_07KACFJJFN@ErrPosY?$AA@ 000000018000f358     service.obj
 0001:0000e360       ??_C@_06HBEFEBCM@ErrSrc?$AA@ 000000018000f360     service.obj
 0001:0000e368       ??_C@_06LDIMCHFC@?$CF?$CKs?$CFs?5?$AA@ 000000018000f368     service.obj
 0001:0000e370       ??_C@_09HNJDNMKK@?$CF?$CF?$CFdd?$CF?$CFs?5?$AA@ 000000018000f370     service.obj
 0001:0000e380       ??_C@_0CC@JIGPFMKG@global?5?$GAtostring?8?5is?5not?5functio@ 000000018000f380     service.obj
 0001:0000e3a8       ??_C@_0CH@OINAPBOJ@tostring?$CI?$CJ?5returned?5a?5non?9string@ 000000018000f3a8     service.obj
 0001:0000e3d0       ??_C@_04CIMGMMMG@text?$AA@ 000000018000f3d0     service.obj
 0001:0000e3d8       ??_C@_03CAOIPBNL@arg?$AA@  000000018000f3d8     service.obj
 0001:0000e3e0       ??_C@_0ME@JDKAEDFJ@local?5items?0n?$DN?4?4?4?6local?5bottom?$DNn@ 000000018000f3e0     service.obj
 0001:0000e4a8       ??_C@_0CG@FGNNCNLL@attempt?5to?5access?5invalid?5file?5f@ 000000018000f4a8     service.obj
 0001:0000e4d0       ??_C@_07BJOIOONN@Strings?$AA@ 000000018000f4d0     service.obj
 0001:0000e4d8       ??_C@_08FGAFMHLF@DiskMenu?$AA@ 000000018000f4d8     service.obj
 0001:0000e4e8       ??_C@_0L@NHENMPLN@PluginMenu?$AA@ 000000018000f4e8     service.obj
 0001:0000e4f8       ??_C@_0N@IEACHFBM@PluginConfig?$AA@ 000000018000f4f8     service.obj
 0001:0000e508       ??_C@_05GCJGCMFJ@PInfo?$AA@ 000000018000f508     service.obj
 0001:0000e510       ??_C@_05HMEFBOHK@GInfo?$AA@ 000000018000f510     service.obj
 0001:0000e518       ??_C@_0N@GAMEMCEE@invalid?5GUID?$AA@ 000000018000f518     service.obj
 0001:0000e528       ??_C@_0BP@NJEEOHDB@attempt?5to?5access?5closed?5timer?$AA@ 000000018000f528     service.obj
 0001:0000e548       ??_C@_05LGELBCGM@Close?$AA@ 000000018000f548     service.obj
 0001:0000e550       ??_C@_07DOAOMMKG@Enabled?$AA@ 000000018000f550     service.obj
 0001:0000e558       ??_C@_08KDKDEPAG@Interval?$AA@ 000000018000f558     service.obj
 0001:0000e568       ??_C@_07CIINKFND@OnTimer?$AA@ 000000018000f568     service.obj
 0001:0000e570       ??_C@_06EFCDMIMC@Closed?$AA@ 000000018000f570     service.obj
 0001:0000e578       ??_C@_0CE@LHJCBGGH@attempt?5to?5call?5non?9existent?5met@ 000000018000f578     service.obj
 0001:0000e5a0       ??_C@_0BO@PNFLEJKN@attempt?5to?5access?5a?5closed?5?$CFs?$AA@ 000000018000f5a0     service.obj
 0001:0000e5c0       ??_C@_04OKOFBOPB@Time?$AA@ 000000018000f5c0     service.obj
 0001:0000e5c8       ??_C@_04LADJNOK@Lock?$AA@  000000018000f5c8     service.obj
 0001:0000e5d0       ??_C@_0N@ECMJOJJG@MacroCallFar?$AA@ 000000018000f5d0     service.obj
 0001:0000e5e0       ??_C@_0BC@JJHHFNMP@FarMacroCallToLua?$AA@ 000000018000f5e0     service.obj
 0001:0000e5f4       ??_C@_06GIFLLBB@editor?$AA@ 000000018000f5f4     service.obj
 0001:0000e5fc       ??_C@_06DGPPOJKF@viewer?$AA@ 000000018000f5fc     service.obj
 0001:0000e604       ??_C@_01DICPFPGM@k?$AA@    000000018000f604     service.obj
 0001:0000e608       ??_C@_06BPGFKLEK@__mode?$AA@ 000000018000f608     service.obj
 0001:0000e610       ??_C@_1CC@OPOAGCKN@?$AA?2?$AAl?$AAu?$AAa?$AAf?$AAa?$AAr?$AA_?$AAi?$AAn?$AAi?$AAt?$AA?4?$AAl?$AAu?$AAa?$AA?$AA@ 000000018000f610     service.obj
 0001:0000e638       ??_C@_1BG@BDOBMIBP@?$AAF?$AAA?$AAR?$AAP?$AAR?$AAO?$AAF?$AAI?$AAL?$AAE?$AA?$AA@ 000000018000f638     service.obj
 0001:0000e650       ??_C@_04LHHHFLPP@utf8?$AA@ 000000018000f650     service.obj
 0001:0000e658       ??_C@_03EDMBFDDG@bit?$AA@  000000018000f658     service.obj
 0001:0000e65c       ??_C@_03IGHFHLNJ@jit?$AA@  000000018000f65c     service.obj
 0001:0000e660       ??_C@_08LBNNGFKE@_PRELOAD?$AA@ 000000018000f660     service.obj
 0001:0000e66c       ??_C@_03DIJDOPEA@ffi?$AA@  000000018000f66c     service.obj
 0001:0000e670       ??_C@_06ONNDGCDK@dofile?$AA@ 000000018000f670     service.obj
 0001:0000e678       ??_C@_08BNNFLGCJ@loadfile?$AA@ 000000018000f678     service.obj
 0001:0000e684       ??_C@_03OFAPEBGM@?$CFs?6?$AA@ 000000018000f684     service.obj
 0001:0000e688       __real@3ff0000000000000    000000018000f688     service.obj
 0001:0000e690       __real@4059000000000000    000000018000f690     service.obj
 0001:0000e698       __real@41e0000000000000    000000018000f698     service.obj
 0001:0000e6a0       __real@43f0000000000000    000000018000f6a0     service.obj
 0001:0000e6b0       __xmm@ffffffffffffffffffffffffffffffff 000000018000f6b0     service.obj
 0001:0000e7d0       ??_C@_04IHGKJMLH@byte?$AA@ 000000018000f7d0     slnunico.obj
 0001:0000e7d8       ??_C@_04ENMBGAPA@char?$AA@ 000000018000f7d8     slnunico.obj
 0001:0000e7e0       ??_C@_04GGLOKIEE@dump?$AA@ 000000018000f7e0     slnunico.obj
 0001:0000e7e8       ??_C@_06DLEPGFEF@format?$AA@ 000000018000f7e8     slnunico.obj
 0001:0000e7f0       ??_C@_05EIEIBDFD@gfind?$AA@ 000000018000f7f0     slnunico.obj
 0001:0000e7f8       ??_C@_03BKCJCHLK@len?$AA@  000000018000f7f8     slnunico.obj
 0001:0000e7fc       ??_C@_05IPJEPLHL@lower?$AA@ 000000018000f7fc     slnunico.obj
 0001:0000e804       ??_C@_03HOKODIMJ@rep?$AA@  000000018000f804     slnunico.obj
 0001:0000e808       ??_C@_07KOIEOCCE@reverse?$AA@ 000000018000f808     slnunico.obj
 0001:0000e810       ??_C@_05NECKJAMC@upper?$AA@ 000000018000f810     slnunico.obj
 0001:0000e818       ??_C@_09GCBMKPBD@utf8valid?$AA@ 000000018000f818     slnunico.obj
 0001:0000e824       ??_C@_04GMGOKAFF@mode?$AA@ 000000018000f824     slnunico.obj
 0001:0000e830       ??_C@_0BG@DFAIEAEC@string?5slice?5too?5long?$AA@ 000000018000f830     slnunico.obj
 0001:0000e848       ??_C@_0O@EAJJMEEM@invalid?5value?$AA@ 000000018000f848     slnunico.obj
 0001:0000e858       ??_C@_0BO@BNLBHKJN@unable?5to?5dump?5given?5function?$AA@ 000000018000f858     slnunico.obj
 0001:0000e878       ??_C@_0BG@LEHNKOGD@invalid?5capture?5index?$AA@ 000000018000f878     slnunico.obj
 0001:0000e890       ??_C@_0BI@ECNPHIBF@invalid?5pattern?5capture?$AA@ 000000018000f890     slnunico.obj
 0001:0000e8a8       ??_C@_0CD@PLJBIEHA@malformed?5pattern?5?$CIends?5with?5?8?$CF?$CF@ 000000018000f8a8     slnunico.obj
 0001:0000e8d0       ??_C@_0CA@CFGACOGB@malformed?5pattern?5?$CImissing?5?8?$FN?8?$CJ?$AA@ 000000018000f8d0     slnunico.obj
 0001:0000e8f0       ??_C@_0BD@NGJIMPLI@unbalanced?5pattern?$AA@ 000000018000f8f0     slnunico.obj
 0001:0000e908       ??_C@_0BC@IMEAEJPD@too?5many?5captures?$AA@ 000000018000f908     slnunico.obj
 0001:0000e920       ??_C@_0BD@BFKNEALP@unfinished?5capture?$AA@ 000000018000f920     slnunico.obj
 0001:0000e938       ??_C@_0L@NLFJOONJ@?$FO$?$CK?$CL?$DP?4?$CI?$FL?$CF?9?$AA@ 000000018000f938     slnunico.obj
 0001:0000e948       ??_C@_0CO@MAGJPEI@?8string?4gfind?8?5was?5renamed?5to?5?8s@ 000000018000f948     slnunico.obj
 0001:0000e978       ??_C@_0BP@PPPOBACA@string?1function?1table?5expected?$AA@ 000000018000f978     slnunico.obj
 0001:0000e998       ??_C@_0CB@LPDIHGGA@invalid?5replacement?5value?5?$CIa?5?$CFs?$CJ@ 000000018000f998     slnunico.obj
 0001:0000e9bc       ??_C@_02HIBBOKEN@?2r?$AA@  000000018000f9bc     slnunico.obj
 0001:0000e9c0       ??_C@_04MPDIABOK@?2000?$AA@ 000000018000f9c0     slnunico.obj
 0001:0000e9c8       ??_C@_05GGBDHNF@?9?$CL?5?$CD0?$AA@ 000000018000f9c8     slnunico.obj
 0001:0000e9d0       ??_C@_0CA@COOMGCAO@invalid?5format?5?$CIrepeated?5flags?$CJ?$AA@ 000000018000f9d0     slnunico.obj
 0001:0000e9f0       ??_C@_0CN@KALFEKPN@invalid?5format?5?$CIwidth?5or?5precisi@ 000000018000f9f0     slnunico.obj
 0001:0000ea20       ??_C@_0CC@KIPBEOBI@invalid?5option?5?8?$CF?$CF?$CFc?8?5to?5?8format@ 000000018000fa20     slnunico.obj
 0001:0000ea48       ??_C@_0O@EJMKHGFJ@unicode?4ascii?$AA@ 000000018000fa48     slnunico.obj
 0001:0000ea58       ??_C@_0P@CMOFLLND@unicode?4latin1?$AA@ 000000018000fa58     slnunico.obj
 0001:0000ea68       ??_C@_0BB@EFCDCNG@unicode?4grapheme?$AA@ 000000018000fa68     slnunico.obj
 0001:0000ea80       ??_C@_0N@DKIDGKBP@unicode?4utf8?$AA@ 000000018000fa80     slnunico.obj
 0001:0000ec70       ??_C@_05DFJCHPDH@input?$AA@ 000000018000fc70     uliolib51.obj
 0001:0000ec78       ??_C@_06DKIGHACF@output?$AA@ 000000018000fc78     uliolib51.obj
 0001:0000ec80       ??_C@_03KCHOJKKI@set?$AA@  000000018000fc80     uliolib51.obj
 0001:0000ec84       ??_C@_03LIBLMJMB@cur?$AA@  000000018000fc84     uliolib51.obj
 0001:0000ec88       ??_C@_03JBJLGPFL@end?$AA@  000000018000fc88     uliolib51.obj
 0001:0000ec8c       ??_C@_02KAJCLHKP@no?$AA@   000000018000fc8c     uliolib51.obj
 0001:0000ec90       ??_C@_04PLMLMMEO@full?$AA@ 000000018000fc90     uliolib51.obj
 0001:0000ec98       ??_C@_04HJPCFDOP@line?$AA@ 000000018000fc98     uliolib51.obj
 0001:0000eca0       ??_C@_05LBOHBHFK@close?$AA@ 000000018000fca0     uliolib51.obj
 0001:0000eca8       ??_C@_05GLCAEPFP@flush?$AA@ 000000018000fca8     uliolib51.obj
 0001:0000ecb0       ??_C@_05DENOCHIP@lines?$AA@ 000000018000fcb0     uliolib51.obj
 0001:0000ecb8       ??_C@_05IACAFMHP@popen?$AA@ 000000018000fcb8     uliolib51.obj
 0001:0000ecc0       ??_C@_07FKJPAINK@tmpfile?$AA@ 000000018000fcc0     uliolib51.obj
 0001:0000ecc8       ??_C@_05NGFEDHGN@write?$AA@ 000000018000fcc8     uliolib51.obj
 0001:0000ecd0       ??_C@_04EDECCOGL@seek?$AA@ 000000018000fcd0     uliolib51.obj
 0001:0000ecd8       ??_C@_07HHBPNGAN@setvbuf?$AA@ 000000018000fcd8     uliolib51.obj
 0001:0000ece0       ??_C@_06DJHOIPC@?$CFs?3?5?$CFs?$AA@ 000000018000fce0     uliolib51.obj
 0001:0000ece8       ??_C@_02DKCKIIND@?$CFs?$AA@ 000000018000fce8     uliolib51.obj
 0001:0000ecec       ??_C@_05KCHOJJD@FILE?$CK?$AA@ 000000018000fcec     uliolib51.obj
 0001:0000ecf8       ??_C@_0M@IBKPHHKH@closed?5file?$AA@ 000000018000fcf8     uliolib51.obj
 0001:0000ed04       ??_C@_04DAMGJPCA@file?$AA@ 000000018000fd04     uliolib51.obj
 0001:0000ed10       ??_C@_0BN@LPOOHAOM@attempt?5to?5use?5a?5closed?5file?$AA@ 000000018000fd10     uliolib51.obj
 0001:0000ed30       ??_C@_0BL@PEFGCPAG@cannot?5close?5standard?5file?$AA@ 000000018000fd30     uliolib51.obj
 0001:0000ed50       ??_C@_07DMJMBBKE@__close?$AA@ 000000018000fd50     uliolib51.obj
 0001:0000ed58       ??_C@_0O@PLFAPHPG@file?5?$CIclosed?$CJ?$AA@ 000000018000fd58     uliolib51.obj
 0001:0000ed68       ??_C@_09BPMAMLLD@file?5?$CI?$CFp?$CJ?$AA@ 000000018000fd68     uliolib51.obj
 0001:0000ed78       ??_C@_17OBBFBLGE@?$AAr?$AAw?$AAa?$AA?$AA@ 000000018000fd78     uliolib51.obj
 0001:0000ed80       ??_C@_0CP@DHGANCPP@invalid?5mode?5?8?$CFs?8?5?$CIshould?5match?5@ 000000018000fd80     uliolib51.obj
 0001:0000edb0       ??_C@_0BL@JMNLNGCA@standard?5?$CFs?5file?5is?5closed?$AA@ 000000018000fdb0     uliolib51.obj
 0001:0000edcc       ??_C@_13CIFDLIMG@?$AAw?$AA?$AA@ 000000018000fdcc     uliolib51.obj
 0001:0000edd0       ??_C@_03DLDNIBIK@?$CFlf?$AA@ 000000018000fdd0     uliolib51.obj
 0001:0000edd8       ??_C@_0BD@IOJAAODF@too?5many?5arguments?$AA@ 000000018000fdd8     uliolib51.obj
 0001:0000edf0       ??_C@_0P@PJFAGLMH@invalid?5option?$AA@ 000000018000fdf0     uliolib51.obj
 0001:0000ee00       ??_C@_0P@CENJCLHM@invalid?5format?$AA@ 000000018000fe00     uliolib51.obj
 0001:0000ee10       ??_C@_0BH@PBGIDLEF@file?5is?5already?5closed?$AA@ 000000018000fe10     uliolib51.obj
 0001:0000ee28       ??_C@_05CGOEHEFE@?$CF?414g?$AA@ 000000018000fe28     uliolib51.obj
 0001:0000ee30       ??_C@_05MHOFLBOO@stdin?$AA@ 000000018000fe30     uliolib51.obj
 0001:0000ee38       ??_C@_06DJDOIFHB@stdout?$AA@ 000000018000fe38     uliolib51.obj
 0001:0000ee40       ??_C@_06FJGNEBG@stderr?$AA@ 000000018000fe40     uliolib51.obj
 0001:0000eed8       ??_C@_07KOEABFCN@loadlib?$AA@ 000000018000fed8     uloadlib51.obj
 0001:0000eee0       ??_C@_06LNOHAKGK@seeall?$AA@ 000000018000fee0     uloadlib51.obj
 0001:0000eee8       ??_C@_06BIEEJMKO@module?$AA@ 000000018000fee8     uloadlib51.obj
 0001:0000eef0       ??_C@_07FFLLPPLH@require?$AA@ 000000018000fef0     uloadlib51.obj
 0001:0000eef8       ??_C@_0BN@GMPFCLAN@unable?5to?5get?5ModuleFileName?$AA@ 000000018000fef8     uloadlib51.obj
 0001:0000ef18       ??_C@_13MGDFOILI@?$AA?$CB?$AA?$AA@ 000000018000ff18     uloadlib51.obj
 0001:0000ef20       ??_C@_09GMLHALBF@LOADLIB?3?5?$AA@ 000000018000ff20     uloadlib51.obj
 0001:0000ef2c       ??_C@_04HDOCAJNK@?$CFs?$CFs?$AA@ 000000018000ff2c     uloadlib51.obj
 0001:0000ef38       ??_C@_08HNNNOMMJ@_LOADLIB?$AA@ 000000018000ff38     uloadlib51.obj
 0001:0000ef44       ??_C@_04HKFDNBLD@init?$AA@ 000000018000ff44     uloadlib51.obj
 0001:0000ef4c       ??_C@_13FPGAJAPJ@?$AA?2?$AA?$AA@ 000000018000ff4c     uloadlib51.obj
 0001:0000ef50       ??_C@_13JOFGPIOO@?$AA?4?$AA?$AA@ 000000018000ff50     uloadlib51.obj
 0001:0000ef58       ??_C@_0BO@COFCKCAL@?8package?4?$CFs?8?5must?5be?5a?5string?$AA@ 000000018000ff58     uloadlib51.obj
 0001:0000ef78       ??_C@_0CE@EPEHLLIH@?8package?4?$CFs?8?5contains?5invalid?5UT@ 000000018000ff78     uloadlib51.obj
 0001:0000ef9c       ??_C@_13HGPDMIBE@?$AA?$DP?$AA?$AA@ 000000018000ff9c     uloadlib51.obj
 0001:0000efa0       ??_C@_0P@NEBKIMDC@?6?7no?5file?5?8?$CFs?8?$AA@ 000000018000ffa0     uloadlib51.obj
 0001:0000efb0       ??_C@_0CO@KHMIPLKM@error?5loading?5module?5?8?$CFs?8?5from?5f@ 000000018000ffb0     uloadlib51.obj
 0001:0000efe0       ??_C@_04LNEJFJGI@path?$AA@ 000000018000ffe0     uloadlib51.obj
 0001:0000efe8       ??_C@_01IDAFKMJL@_?$AA@    000000018000ffe8     uloadlib51.obj
 0001:0000efec       ??_C@_01LFCBOECM@?4?$AA@   000000018000ffec     uloadlib51.obj
 0001:0000eff0       ??_C@_0L@KHKMBFOE@luaopen_?$CFs?$AA@ 000000018000fff0     uloadlib51.obj
 0001:0000effc       ??_C@_05EEMJHCCC@cpath?$AA@ 000000018000fffc     uloadlib51.obj
 0001:0000f008       ??_C@_0BO@KOILFIGK@?6?7no?5module?5?8?$CFs?8?5in?5file?5?8?$CFs?8?$AA@ 0000000180010008     uloadlib51.obj
 0001:0000f028       ??_C@_0CC@CCJHFBLH@?8package?4preload?8?5must?5be?5a?5tabl@ 0000000180010028     uloadlib51.obj
 0001:0000f050       ??_C@_0CB@NPNABMBF@?6?7no?5field?5package?4preload?$FL?8?$CFs?8?$FN@ 0000000180010050     uloadlib51.obj
 0001:0000f078       ??_C@_07PINPBNPB@_LOADED?$AA@ 0000000180010078     uloadlib51.obj
 0001:0000f080       ??_C@_0CL@DIEJCPFH@loop?5or?5previous?5error?5loading?5m@ 0000000180010080     uloadlib51.obj
 0001:0000f0b0       ??_C@_07JAOCDFCG@loaders?$AA@ 00000001800100b0     uloadlib51.obj
 0001:0000f0b8       ??_C@_0CC@IGEJMOFI@?8package?4loaders?8?5must?5be?5a?5tabl@ 00000001800100b8     uloadlib51.obj
 0001:0000f0e0       ??_C@_0BJ@HFHHABH@module?5?8?$CFs?8?5not?5found?3?$CFs?$AA@ 00000001800100e0     uloadlib51.obj
 0001:0000f0fc       ??_C@_01INIBCBCB@f?$AA@    00000001800100fc     uloadlib51.obj
 0001:0000f100       ??_C@_0CI@GKOMOAFD@?8module?8?5not?5called?5from?5a?5Lua?5f@ 0000000180010100     uloadlib51.obj
 0001:0000f128       ??_C@_02CCIJHOCI@_M?$AA@   0000000180010128     uloadlib51.obj
 0001:0000f12c       ??_C@_05ICMCJINN@_NAME?$AA@ 000000018001012c     uloadlib51.obj
 0001:0000f138       ??_C@_08HONLOGDK@_PACKAGE?$AA@ 0000000180010138     uloadlib51.obj
 0001:0000f148       ??_C@_0BO@CBJIAGLF@name?5conflict?5for?5module?5?8?$CFs?8?$AA@ 0000000180010148     uloadlib51.obj
 0001:0000f168       ??_C@_17KOAMMDLI@?$AA?$DL?$AA?$AB?$AA?$DL?$AA?$AA@ 0000000180010168     uloadlib51.obj
 0001:0000f170       ??_C@_15HKKNGJC@?$AA?$DL?$AA?$DL?$AA?$AA@ 0000000180010170     uloadlib51.obj
 0001:0000f178       ??_C@_13GGAHEHIG@?$AA?$AB?$AA?$AA@ 0000000180010178     uloadlib51.obj
 0001:0000f180       ??_C@_1HE@JLDBNBHO@?$AA?4?$AA?2?$AA?$DP?$AA?4?$AAl?$AAu?$AAa?$AA?$DL?$AA?$CB?$AA?2?$AAl?$AAu?$AAa?$AA?2?$AA?$DP?$AA?4?$AAl?$AAu?$AAa?$AA?$DL?$AA?$CB?$AA?2?$AAl?$AAu?$AAa?$AA?2?$AA?$DP?$AA?2?$AAi?$AAn?$AAi?$AAt@ 0000000180010180     uloadlib51.obj
 0001:0000f1f8       ??_C@_1BC@ILFFIBFI@?$AAL?$AAU?$AAA?$AA_?$AAP?$AAA?$AAT?$AAH?$AA?$AA@ 00000001800101f8     uloadlib51.obj
 0001:0000f210       ??_C@_1DM@FGPGEDD@?$AA?4?$AA?2?$AA?$DP?$AA?4?$AAd?$AAl?$AAl?$AA?$DL?$AA?$CB?$AA?2?$AA?$DP?$AA?4?$AAd?$AAl?$AAl?$AA?$DL?$AA?$CB?$AA?2?$AAl?$AAo?$AAa?$AAd?$AAa?$AAl?$AAl?$AA?4?$AAd?$AAl?$AAl?$AA?$AA@ 0000000180010210     uloadlib51.obj
 0001:0000f250       ??_C@_1BE@EFNILHBI@?$AAL?$AAU?$AAA?$AA_?$AAC?$AAP?$AAA?$AAT?$AAH?$AA?$AA@ 0000000180010250     uloadlib51.obj
 0001:0000f268       ??_C@_1BE@CKNDCMBB@?$AA?2?$AA?6?$AA?$DL?$AA?6?$AA?$DP?$AA?6?$AA?$CB?$AA?6?$AA?9?$AA?$AA@ 0000000180010268     uloadlib51.obj
 0001:0000f27c       ??_C@_06HEJKKHEK@config?$AA@ 000000018001027c     uloadlib51.obj
 0001:0000f284       ??_C@_06IILMCCFO@loaded?$AA@ 0000000180010284     uloadlib51.obj
 0001:0000f290       ustring_funcs              0000000180010290     ustring.obj
 0001:0000f440       ??_C@_0BE@DEHGONAH@EnumSystemCodePages?$AA@ 0000000180010440     ustring.obj
 0001:0000f454       ??_C@_06FMJLOCAF@GetACP?$AA@ 0000000180010454     ustring.obj
 0001:0000f460       ??_C@_09HLFMNDA@GetCPInfo?$AA@ 0000000180010460     ustring.obj
 0001:0000f470       ??_C@_0O@PIBBCLJF@GetCurrentDir?$AA@ 0000000180010470     ustring.obj
 0001:0000f480       ??_C@_0N@IIBOJKJ@GetDriveType?$AA@ 0000000180010480     ustring.obj
 0001:0000f490       ??_C@_0M@KHMMJMNI@GetFileAttr?$AA@ 0000000180010490     ustring.obj
 0001:0000f4a0       ??_C@_0M@ONGMCNNE@GetKeyState?$AA@ 00000001800104a0     ustring.obj
 0001:0000f4b0       ??_C@_0BH@KKAFOIJJ@GetLogicalDriveStrings?$AA@ 00000001800104b0     ustring.obj
 0001:0000f4c8       ??_C@_08OMCNFONF@GetOEMCP?$AA@ 00000001800104c8     ustring.obj
 0001:0000f4d8       ??_C@_0BD@IHIHPGDL@GlobalMemoryStatus?$AA@ 00000001800104d8     ustring.obj
 0001:0000f4f0       ??_C@_0BE@HCIKGJGE@MultiByteToWideChar?$AA@ 00000001800104f0     ustring.obj
 0001:0000f508       ??_C@_09EPINLGBH@OemToUtf8?$AA@ 0000000180010508     ustring.obj
 0001:0000f518       ??_C@_0BC@NFCPMJFM@OutputDebugString?$AA@ 0000000180010518     ustring.obj
 0001:0000f530       ??_C@_0BA@MNJFBAJH@SHGetFolderPath?$AA@ 0000000180010530     ustring.obj
 0001:0000f540       ??_C@_0L@PMCLJMMJ@SearchPath?$AA@ 0000000180010540     ustring.obj
 0001:0000f550       ??_C@_0O@IHAPJIOC@SetCurrentDir?$AA@ 0000000180010550     ustring.obj
 0001:0000f560       ??_C@_0M@KINCEKFL@SetFileAttr?$AA@ 0000000180010560     ustring.obj
 0001:0000f56c       ??_C@_05PFDOMJEF@Sleep?$AA@ 000000018001056c     ustring.obj
 0001:0000f578       ??_C@_0M@KJELMDJD@Utf16ToUtf8?$AA@ 0000000180010578     ustring.obj
 0001:0000f588       ??_C@_09LCEKPEGC@Utf8ToOem?$AA@ 0000000180010588     ustring.obj
 0001:0000f598       ??_C@_0M@GJGCILHG@Utf8ToUtf16?$AA@ 0000000180010598     ustring.obj
 0001:0000f5a4       ??_C@_04NDFIEGPL@Uuid?$AA@ 00000001800105a4     ustring.obj
 0001:0000f5b0       ??_C@_0BE@LJADKLBD@WideCharToMultiByte?$AA@ 00000001800105b0     ustring.obj
 0001:0000f5c4       ??_C@_04GFOHBGIO@subW?$AA@ 00000001800105c4     ustring.obj
 0001:0000f5cc       ??_C@_06FHFOAHML@system?$AA@ 00000001800105cc     ustring.obj
 0001:0000f5d4       ??_C@_04NOFELICG@lenW?$AA@ 00000001800105d4     ustring.obj
 0001:0000f5e0       ??_C@_0BB@BLJKPILH@system?5error?5?$CFd?6?$AA@ 00000001800105e0     ustring.obj
 0001:0000f5f8       ??_C@_0BJ@MEAJDMDL@invalid?5multibyte?5string?$AA@ 00000001800105f8     ustring.obj
 0001:0000f618       ??_C@_0BG@ELIKBHAO@invalid?5UTF?916?5string?$AA@ 0000000180010618     ustring.obj
 0001:0000f630       ??_C@_0M@KJGJBDLL@MaxCharSize?$AA@ 0000000180010630     ustring.obj
 0001:0000f640       ??_C@_0M@IMOFNPBB@DefaultChar?$AA@ 0000000180010640     ustring.obj
 0001:0000f650       ??_C@_08HIIJAENB@LeadByte?$AA@ 0000000180010650     ustring.obj
 0001:0000f660       ??_C@_0BD@CBNPFFPH@UnicodeDefaultChar?$AA@ 0000000180010660     ustring.obj
 0001:0000f678       ??_C@_0N@DJCOCBOB@CodePageName?$AA@ 0000000180010678     ustring.obj
 0001:0000f688       ??_C@_0N@IFJMFGJK@unknown?5type?$AA@ 0000000180010688     ustring.obj
 0001:0000f698       ??_C@_0BC@GPFCFLGN@no?5root?5directory?$AA@ 0000000180010698     ustring.obj
 0001:0000f6b0       ??_C@_09HPGMKNKO@removable?$AA@ 00000001800106b0     ustring.obj
 0001:0000f6bc       ??_C@_05OFLEIIDM@fixed?$AA@ 00000001800106bc     ustring.obj
 0001:0000f6c4       ??_C@_06IMIHEKN@remote?$AA@ 00000001800106c4     ustring.obj
 0001:0000f6cc       ??_C@_05POABADMF@cdrom?$AA@ 00000001800106cc     ustring.obj
 0001:0000f6d8       ??_C@_07BHCBOAMP@ramdisk?$AA@ 00000001800106d8     ustring.obj
 0001:0000f6e0       ??_C@_0L@PLJFMBIJ@MemoryLoad?$AA@ 00000001800106e0     ustring.obj
 0001:0000f6f0       ??_C@_09MMAOIBBJ@TotalPhys?$AA@ 00000001800106f0     ustring.obj
 0001:0000f700       ??_C@_09KFOEOLH@AvailPhys?$AA@ 0000000180010700     ustring.obj
 0001:0000f710       ??_C@_0O@PEEMGPEP@TotalPageFile?$AA@ 0000000180010710     ustring.obj
 0001:0000f720       ??_C@_0O@LLHOKNF@AvailPageFile?$AA@ 0000000180010720     ustring.obj
 0001:0000f730       ??_C@_0N@LCJEOHMM@TotalVirtual?$AA@ 0000000180010730     ustring.obj
 0001:0000f740       ??_C@_0N@EGHLANBF@AvailVirtual?$AA@ 0000000180010740     ustring.obj
 0001:0000f750       ??_C@_0BF@KKNLCGDE@AvailExtendedVirtual?$AA@ 0000000180010750     ustring.obj
 0001:0000f768       ??_C@_0P@KJDDGAFH@FileAttributes?$AA@ 0000000180010768     ustring.obj
 0001:0000f778       ??_C@_07JOJHCKGP@ustring?$AA@ 0000000180010778     ustring.obj
 0001:00010000       ??_C@_0DJ@KKHMCMAP@bad?5field?5?$FL?$CFd?$FN?5in?5table?5stackpos@ 0000000180011000     util.obj
 0001:00010040       ??_C@_0DJ@PFHHGAMM@bad?5field?5?8?$CFs?8?5in?5table?5stackpos@ 0000000180011040     util.obj
 0001:0001007c       ??_C@_06EBGNBFIA@number?$AA@ 000000018001107c     util.obj
 0001:00010910       win_funcs                  0000000180011910     win.obj
 0001:00010ad0       ??_C@_0O@CFPMOCDP@CompareString?$AA@ 0000000180011ad0     win.obj
 0001:00010ae0       ??_C@_08PPLNFCGA@CopyFile?$AA@ 0000000180011ae0     win.obj
 0001:00010af0       ??_C@_09INHPLKKM@CreateDir?$AA@ 0000000180011af0     win.obj
 0001:00010b00       ??_C@_0L@GPLPOFDC@DeleteFile?$AA@ 0000000180011b00     win.obj
 0001:00010b10       ??_C@_0N@FOJPHHPH@DeleteRegKey?$AA@ 0000000180011b10     win.obj
 0001:00010b20       ??_C@_0P@PCCDOIAL@DeleteRegValue?$AA@ 0000000180011b20     win.obj
 0001:00010b30       ??_C@_0L@DGAGCFOP@EnumRegKey?$AA@ 0000000180011b30     win.obj
 0001:00010b40       ??_C@_0N@PFFNCIBD@EnumRegValue?$AA@ 0000000180011b40     win.obj
 0001:00010b50       ??_C@_0L@MGMEFCAE@ExtractKey?$AA@ 0000000180011b50     win.obj
 0001:00010b60       ??_C@_0N@HALOIPMN@ExtractKeyEx?$AA@ 0000000180011b60     win.obj
 0001:00010b70       ??_C@_0BI@EKFDIGHI@FileTimeToLocalFileTime?$AA@ 0000000180011b70     win.obj
 0001:00010b88       ??_C@_0BF@KPJNHALE@FileTimeToSystemTime?$AA@ 0000000180011b88     win.obj
 0001:00010ba0       ??_C@_0BL@NAIJNMLL@GetConsoleScreenBufferInfo?$AA@ 0000000180011ba0     win.obj
 0001:00010bbc       ??_C@_06CALCCDMF@GetEnv?$AA@ 0000000180011bbc     win.obj
 0001:00010bc8       ??_C@_0M@EINGHLOA@GetFileInfo?$AA@ 0000000180011bc8     win.obj
 0001:00010bd8       ??_C@_09GFGIAJLD@GetRegKey?$AA@ 0000000180011bd8     win.obj
 0001:00010be8       ??_C@_0BI@ENMDHCMK@GetSystemTimeAsFileTime?$AA@ 0000000180011be8     win.obj
 0001:00010c00       ??_C@_0P@GGGHOPAD@GetVirtualKeys?$AA@ 0000000180011c00     win.obj
 0001:00010c10       ??_C@_0P@MIPPOCAO@IsProcess64bit?$AA@ 0000000180011c10     win.obj
 0001:00010c20       ??_C@_08CALLHOCI@MoveFile?$AA@ 0000000180011c20     win.obj
 0001:00010c30       ??_C@_09EDKALOCB@RemoveDir?$AA@ 0000000180011c30     win.obj
 0001:00010c40       ??_C@_0L@HBAGBENL@RenameFile?$AA@ 0000000180011c40     win.obj
 0001:00010c4c       ??_C@_06LDCDJLBI@SetEnv?$AA@ 0000000180011c4c     win.obj
 0001:00010c58       ??_C@_09ELCNCICB@SetRegKey?$AA@ 0000000180011c58     win.obj
 0001:00010c68       ??_C@_0N@BFFIJKHB@ShellExecute?$AA@ 0000000180011c68     win.obj
 0001:00010c78       ??_C@_0BF@HBHGIPOG@SystemTimeToFileTime?$AA@ 0000000180011c78     win.obj
 0001:00010c90       ??_C@_06DNONFAKH@wcscmp?$AA@ 0000000180011c90     win.obj
 0001:00010c98       ??_C@_04CBBMIBLK@HKLM?$AA@ 0000000180011c98     win.obj
 0001:00010ca0       ??_C@_04LEMDOLAJ@HKCC?$AA@ 0000000180011ca0     win.obj
 0001:00010ca8       ??_C@_04OHBKMIBJ@HKCR?$AA@ 0000000180011ca8     win.obj
 0001:00010cb0       ??_C@_04KIFLFONO@HKCU?$AA@ 0000000180011cb0     win.obj
 0001:00010cb8       ??_C@_03DLBIJLAB@HKU?$AA@  0000000180011cb8     win.obj
 0001:00010cc0       ??_C@_0DA@DKALLFDI@must?5be?5?8HKLM?8?0?5?8HKCC?8?0?5?8HKCR?8?0?5@ 0000000180011cc0     win.obj
 0001:00010cf0       ??_C@_05KDALNKAH@dword?$AA@ 0000000180011cf0     win.obj
 0001:00010cf8       ??_C@_06FNFBAEBE@binary?$AA@ 0000000180011cf8     win.obj
 0001:00010d00       ??_C@_0N@CBOMHLPN@expandstring?$AA@ 0000000180011d00     win.obj
 0001:00010d10       ??_C@_0M@PEGIPCHN@multistring?$AA@ 0000000180011d10     win.obj
 0001:00010d20       ??_C@_0BH@NOJOGNJM@unsupported?5value?5type?$AA@ 0000000180011d20     win.obj
 0001:00010d38       ??_C@_0BD@MJODDCFG@OpenRegKey?5failed?4?$AA@ 0000000180011d38     win.obj
 0001:00010d50       ??_C@_0BI@COLHBIIE@RegQueryValueEx?5failed?4?$AA@ 0000000180011d50     win.obj
 0001:00010d68       ??_C@_1BK@BIGILECK@?$AAA?$AAd?$AAv?$AAa?$AAp?$AAi?$AA3?$AA2?$AA?4?$AAd?$AAl?$AAl?$AA?$AA@ 0000000180011d68     win.obj
 0001:00010d88       ??_C@_0BA@LILAPHGE@RegDeleteKeyExW?$AA@ 0000000180011d88     win.obj
 0001:00010d98       ??_C@_0BG@HHFHBIKG@RegOpenKeyExW?5failed?4?$AA@ 0000000180011d98     win.obj
 0001:00010db0       ??_C@_05DFPNHDMN@wYear?$AA@ 0000000180011db0     win.obj
 0001:00010db8       ??_C@_06MGNNJGBJ@wMonth?$AA@ 0000000180011db8     win.obj
 0001:00010dc0       ??_C@_0L@OAHPHHP@wDayOfWeek?$AA@ 0000000180011dc0     win.obj
 0001:00010dcc       ??_C@_04NBLBJIPP@wDay?$AA@ 0000000180011dcc     win.obj
 0001:00010dd4       ??_C@_05BMOPCGDH@wHour?$AA@ 0000000180011dd4     win.obj
 0001:00010de0       ??_C@_07HPODENI@wMinute?$AA@ 0000000180011de0     win.obj
 0001:00010de8       ??_C@_07IIEDHHJN@wSecond?$AA@ 0000000180011de8     win.obj
 0001:00010df0       ??_C@_0O@HBAPEOKP@wMilliseconds?$AA@ 0000000180011df0     win.obj
 0001:00010e00       ??_C@_01LKDEMHDF@s?$AA@    0000000180011e00     win.obj
 0001:00010e08       ??_C@_0BA@IAFODGNM@CursorPositionX?$AA@ 0000000180011e08     win.obj
 0001:00010e18       ??_C@_0BA@JJEFAHJN@CursorPositionY?$AA@ 0000000180011e18     win.obj
 0001:00010e28       ??_C@_0L@NFCEOFBF@WindowLeft?$AA@ 0000000180011e28     win.obj
 0001:00010e38       ??_C@_09JHGOALHG@WindowTop?$AA@ 0000000180011e38     win.obj
 0001:00010e48       ??_C@_0M@HHPHMPGH@WindowRight?$AA@ 0000000180011e48     win.obj
 0001:00010e58       ??_C@_0N@JPIJCAOJ@WindowBottom?$AA@ 0000000180011e58     win.obj
 0001:00010e68       ??_C@_0BD@DOLDEII@MaximumWindowSizeX?$AA@ 0000000180011e68     win.obj
 0001:00010e80       ??_C@_0BD@BKPAAFMJ@MaximumWindowSizeY?$AA@ 0000000180011e80     win.obj
 0001:00010e94       ??_C@_01PFHFFBPC@t?$AA@    0000000180011e94     win.obj
 0001:00010e98       ??_C@_0BJ@LPJMBJJL@directory?5already?5exists?$AA@ 0000000180011e98     win.obj
 0001:00010eb8       __real@41f0000000000000    0000000180011eb8     win.obj
 0001:00010ec0       _pRawDllMain               0000000180011ec0     LIBCMT:dll_dllmain.obj
 0001:00010ec0       _pDefaultRawDllMain        0000000180011ec0     LIBCMT:dll_dllmain.obj
 0001:00011200       ??_C@_08EHJDFFNH@__based?$CI?$AA@ 0000000180012200     libvcruntime:undname.obj
 0001:00011210       ??_C@_07KOLFKCDI@__cdecl?$AA@ 0000000180012210     libvcruntime:undname.obj
 0001:00011218       ??_C@_08GHMPAG@__pascal?$AA@ 0000000180012218     libvcruntime:undname.obj
 0001:00011228       ??_C@_09IFJBGAPI@__stdcall?$AA@ 0000000180012228     libvcruntime:undname.obj
 0001:00011238       ??_C@_0L@NPHFGOKO@__thiscall?$AA@ 0000000180012238     libvcruntime:undname.obj
 0001:00011248       ??_C@_0L@JMKHOMEK@__fastcall?$AA@ 0000000180012248     libvcruntime:undname.obj
 0001:00011258       ??_C@_0N@BCKKPABJ@__vectorcall?$AA@ 0000000180012258     libvcruntime:undname.obj
 0001:00011268       ??_C@_09HIJEGCPM@__clrcall?$AA@ 0000000180012268     libvcruntime:undname.obj
 0001:00011274       ??_C@_06GHPCKEAG@__eabi?$AA@ 0000000180012274     libvcruntime:undname.obj
 0001:00011280       ??_C@_07EECFKIPL@__swift?$AA@ 0000000180012280     libvcruntime:undname.obj
 0001:00011288       ??_C@_07JOMMBBKO@__ptr64?$AA@ 0000000180012288     libvcruntime:undname.obj
 0001:00011290       ??_C@_0L@PILCLIHE@__restrict?$AA@ 0000000180012290     libvcruntime:undname.obj
 0001:000112a0       ??_C@_0M@GFIIJFMG@__unaligned?$AA@ 00000001800122a0     libvcruntime:undname.obj
 0001:000112b0       ??_C@_09DHDLOLLB@restrict?$CI?$AA@ 00000001800122b0     libvcruntime:undname.obj
 0001:000112bc       ??_C@_04NIHEBCM@?5new?$AA@ 00000001800122bc     libvcruntime:undname.obj
 0001:000112c8       ??_C@_07FPCDHGMM@?5delete?$AA@ 00000001800122c8     libvcruntime:undname.obj
 0001:000112d0       ??_C@_01NEMOKFLO@?$DN?$AA@ 00000001800122d0     libvcruntime:undname.obj
 0001:000112d4       ??_C@_02GPIOPFAK@?$DO?$DO?$AA@ 00000001800122d4     libvcruntime:undname.obj
 0001:000112d8       ??_C@_02FODMEDOG@?$DM?$DM?$AA@ 00000001800122d8     libvcruntime:undname.obj
 0001:000112dc       ??_C@_01DCLJPIOD@?$CB?$AA@ 00000001800122dc     libvcruntime:undname.obj
 0001:000112e0       ??_C@_02EGOFBIJA@?$DN?$DN?$AA@ 00000001800122e0     libvcruntime:undname.obj
 0001:000112e4       ??_C@_02FDNJECIE@?$CB?$DN?$AA@ 00000001800122e4     libvcruntime:undname.obj
 0001:000112e8       ??_C@_02GPECMEKF@?$FL?$FN?$AA@ 00000001800122e8     libvcruntime:undname.obj
 0001:000112f0       ??_C@_08LHJFAFGD@operator?$AA@ 00000001800122f0     libvcruntime:undname.obj
 0001:000112fc       ??_C@_02HBOOOICD@?9?$DO?$AA@ 00000001800122fc     libvcruntime:undname.obj
 0001:00011300       ??_C@_01NBENCBCI@?$CK?$AA@ 0000000180012300     libvcruntime:undname.obj
 0001:00011304       ??_C@_02ECNGHCIF@?$CL?$CL?$AA@ 0000000180012304     libvcruntime:undname.obj
 0001:00011308       ??_C@_02BAABKJLB@?9?9?$AA@ 0000000180012308     libvcruntime:undname.obj
 0001:0001130c       ??_C@_01JOAMLHOP@?9?$AA@   000000018001230c     libvcruntime:undname.obj
 0001:00011310       ??_C@_01MIFGBAGJ@?$CL?$AA@ 0000000180012310     libvcruntime:undname.obj
 0001:00011314       ??_C@_01HNPIGOCE@?$CG?$AA@ 0000000180012314     libvcruntime:undname.obj
 0001:00011318       ??_C@_03MNHNFDLC@?9?$DO?$CK?$AA@ 0000000180012318     libvcruntime:undname.obj
 0001:0001131c       ??_C@_01FGNFDNOH@?$CF?$AA@ 000000018001231c     libvcruntime:undname.obj
 0001:00011320       ??_C@_01MNNFJEPP@?$DM?$AA@ 0000000180012320     libvcruntime:undname.obj
 0001:00011324       ??_C@_02EHCHHCKH@?$DM?$DN?$AA@ 0000000180012324     libvcruntime:undname.obj
 0001:00011328       ??_C@_01PPODPGHN@?$DO?$AA@ 0000000180012328     libvcruntime:undname.obj
 0001:0001132c       ??_C@_02EEKDKGMJ@?$DO?$DN?$AA@ 000000018001232c     libvcruntime:undname.obj
 0001:00011330       ??_C@_01IHBHIGKO@?0?$AA@   0000000180012330     libvcruntime:undname.obj
 0001:00011334       ??_C@_02HCKGKOFO@?$CI?$CJ?$AA@ 0000000180012334     libvcruntime:undname.obj
 0001:00011338       ??_C@_01PJKLJHI@?$HO?$AA@  0000000180012338     libvcruntime:undname.obj
 0001:0001133c       ??_C@_01JKBOJNNK@?$FO?$AA@ 000000018001233c     libvcruntime:undname.obj
 0001:00011340       ??_C@_01DNKMNLPK@?$HM?$AA@ 0000000180012340     libvcruntime:undname.obj
 0001:00011344       ??_C@_02PPKAJPJL@?$CG?$CG?$AA@ 0000000180012344     libvcruntime:undname.obj
 0001:00011348       ??_C@_02NONPIBCD@?$HM?$HM?$AA@ 0000000180012348     libvcruntime:undname.obj
 0001:0001134c       ??_C@_02FPIMKNGF@?$CK?$DN?$AA@ 000000018001234c     libvcruntime:undname.obj
 0001:00011350       ??_C@_02FOEOMHFC@?$CL?$DN?$AA@ 0000000180012350     libvcruntime:undname.obj
 0001:00011354       ??_C@_02FKMDLLOA@?9?$DN?$AA@ 0000000180012354     libvcruntime:undname.obj
 0001:00011358       ??_C@_02FJEHGPIO@?1?$DN?$AA@ 0000000180012358     libvcruntime:undname.obj
 0001:0001135c       ??_C@_02FENAOKFI@?$CF?$DN?$AA@ 000000018001235c     libvcruntime:undname.obj
 0001:00011360       ??_C@_03IKFCCPFF@?$DO?$DO?$DN?$AA@ 0000000180012360     libvcruntime:undname.obj
 0001:00011364       ??_C@_03CDNPDDLA@?$DM?$DM?$DN?$AA@ 0000000180012364     libvcruntime:undname.obj
 0001:00011368       ??_C@_02FGJGFEAB@?$CG?$DN?$AA@ 0000000180012368     libvcruntime:undname.obj
 0001:0001136c       ??_C@_02DHLNPPGH@?$HM?$DN?$AA@ 000000018001236c     libvcruntime:undname.obj
 0001:00011370       ??_C@_02MHEGNOJ@?$FO?$DN?$AA@ 0000000180012370     libvcruntime:undname.obj
 0001:00011378       ??_C@_09IFPLHPGF@?$GAvftable?8?$AA@ 0000000180012378     libvcruntime:undname.obj
 0001:00011388       ??_C@_09BLBHBJP@?$GAvbtable?8?$AA@ 0000000180012388     libvcruntime:undname.obj
 0001:00011398       ??_C@_07FEEIOKP@?$GAvcall?8?$AA@ 0000000180012398     libvcruntime:undname.obj
 0001:000113a0       ??_C@_08LLFFHHDJ@?$GAtypeof?8?$AA@ 00000001800123a0     libvcruntime:undname.obj
 0001:000113b0       ??_C@_0BF@KDPPACIK@?$GAlocal?5static?5guard?8?$AA@ 00000001800123b0     libvcruntime:undname.obj
 0001:000113c8       ??_C@_08OBABFOLI@?$GAstring?8?$AA@ 00000001800123c8     libvcruntime:undname.obj
 0001:000113d8       ??_C@_0BD@JDLKDPAB@?$GAvbase?5destructor?8?$AA@ 00000001800123d8     libvcruntime:undname.obj
 0001:000113f0       ??_C@_0BN@DEGPLNFK@?$GAvector?5deleting?5destructor?8?$AA@ 00000001800123f0     libvcruntime:undname.obj
 0001:00011410       ??_C@_0BO@OBMKPJIG@?$GAdefault?5constructor?5closure?8?$AA@ 0000000180012410     libvcruntime:undname.obj
 0001:00011430       ??_C@_0BN@IMDCHIKM@?$GAscalar?5deleting?5destructor?8?$AA@ 0000000180012430     libvcruntime:undname.obj
 0001:00011450       ??_C@_0BO@PFGOCPJJ@?$GAvector?5constructor?5iterator?8?$AA@ 0000000180012450     libvcruntime:undname.obj
 0001:00011470       ??_C@_0BN@LFPFMEDL@?$GAvector?5destructor?5iterator?8?$AA@ 0000000180012470     libvcruntime:undname.obj
 0001:00011490       ??_C@_0CE@IKBNEHA@?$GAvector?5vbase?5constructor?5iterat@ 0000000180012490     libvcruntime:undname.obj
 0001:000114b8       ??_C@_0BL@NILFHHPC@?$GAvirtual?5displacement?5map?8?$AA@ 00000001800124b8     libvcruntime:undname.obj
 0001:000114d8       ??_C@_0CB@JONCMFFK@?$GAeh?5vector?5constructor?5iterator?8@ 00000001800124d8     libvcruntime:undname.obj
 0001:00011500       ??_C@_0CA@GCEOPDGL@?$GAeh?5vector?5destructor?5iterator?8?$AA@ 0000000180012500     libvcruntime:undname.obj
 0001:00011520       ??_C@_0CH@OOJPLCPH@?$GAeh?5vector?5vbase?5constructor?5ite@ 0000000180012520     libvcruntime:undname.obj
 0001:00011548       ??_C@_0BL@LLKPOHJI@?$GAcopy?5constructor?5closure?8?$AA@ 0000000180012548     libvcruntime:undname.obj
 0001:00011568       ??_C@_0BA@KBCDOMBN@?$GAudt?5returning?8?$AA@ 0000000180012568     libvcruntime:undname.obj
 0001:00011578       ??_C@_03KLGMFNMG@?$GAEH?$AA@ 0000000180012578     libvcruntime:undname.obj
 0001:0001157c       ??_C@_05KHLCHHI@?$GARTTI?$AA@ 000000018001257c     libvcruntime:undname.obj
 0001:00011588       ??_C@_0BA@KKLDJDLB@?$GAlocal?5vftable?8?$AA@ 0000000180012588     libvcruntime:undname.obj
 0001:00011598       ??_C@_0CE@IIHCMGGL@?$GAlocal?5vftable?5constructor?5closu@ 0000000180012598     libvcruntime:undname.obj
 0001:000115bc       ??_C@_06FHBGPFGH@?5new?$FL?$FN?$AA@ 00000001800125bc     libvcruntime:undname.obj
 0001:000115c8       ??_C@_09LBNFPBCA@?5delete?$FL?$FN?$AA@ 00000001800125c8     libvcruntime:undname.obj
 0001:000115d8       ??_C@_0P@HJKNJFNN@?$GAomni?5callsig?8?$AA@ 00000001800125d8     libvcruntime:undname.obj
 0001:000115e8       ??_C@_0BL@CNOONJFP@?$GAplacement?5delete?5closure?8?$AA@ 00000001800125e8     libvcruntime:undname.obj
 0001:00011608       ??_C@_0BN@CKNJLHMB@?$GAplacement?5delete?$FL?$FN?5closure?8?$AA@ 0000000180012608     libvcruntime:undname.obj
 0001:00011628       ??_C@_0CG@CFDHKGGD@?$GAmanaged?5vector?5constructor?5iter@ 0000000180012628     libvcruntime:undname.obj
 0001:00011650       ??_C@_0CF@IMGKMJNO@?$GAmanaged?5vector?5destructor?5itera@ 0000000180012650     libvcruntime:undname.obj
 0001:00011678       ??_C@_0CG@HLDDJMAG@?$GAeh?5vector?5copy?5constructor?5iter@ 0000000180012678     libvcruntime:undname.obj
 0001:000116a0       ??_C@_0CM@FCBBDIGB@?$GAeh?5vector?5vbase?5copy?5constructo@ 00000001800126a0     libvcruntime:undname.obj
 0001:000116d0       ??_C@_0BL@CLIPGLGB@?$GAdynamic?5initializer?5for?5?8?$AA@ 00000001800126d0     libvcruntime:undname.obj
 0001:000116f0       ??_C@_0CB@PDBIFEP@?$GAdynamic?5atexit?5destructor?5for?5?8@ 00000001800126f0     libvcruntime:undname.obj
 0001:00011718       ??_C@_0CD@CGAJBKEJ@?$GAvector?5copy?5constructor?5iterato@ 0000000180012718     libvcruntime:undname.obj
 0001:00011740       ??_C@_0CJ@GJELGAMM@?$GAvector?5vbase?5copy?5constructor?5i@ 0000000180012740     libvcruntime:undname.obj
 0001:00011770       ??_C@_0CL@FGIJHLCE@?$GAmanaged?5vector?5copy?5constructor@ 0000000180012770     libvcruntime:undname.obj
 0001:000117a0       ??_C@_0BM@PMGGMLDN@?$GAlocal?5static?5thread?5guard?8?$AA@ 00000001800127a0     libvcruntime:undname.obj
 0001:000117c0       ??_C@_0N@BDNMDMOL@operator?5?$CC?$CC?5?$AA@ 00000001800127c0     libvcruntime:undname.obj
 0001:000117d0       ??_C@_0BC@GGEBGALA@operator?5co_await?$AA@ 00000001800127d0     libvcruntime:undname.obj
 0001:000117e8       ??_C@_0BC@DAFEJGAK@?5Type?5Descriptor?8?$AA@ 00000001800127e8     libvcruntime:undname.obj
 0001:00011800       ??_C@_0BM@LDKODKLH@?5Base?5Class?5Descriptor?5at?5?$CI?$AA@ 0000000180012800     libvcruntime:undname.obj
 0001:00011820       ??_C@_0BD@LGICGFMM@?5Base?5Class?5Array?8?$AA@ 0000000180012820     libvcruntime:undname.obj
 0001:00011838       ??_C@_0BN@MECKDCOJ@?5Class?5Hierarchy?5Descriptor?8?$AA@ 0000000180012838     libvcruntime:undname.obj
 0001:00011858       ??_C@_0BK@CFCOFLF@?5Complete?5Object?5Locator?8?$AA@ 0000000180012858     libvcruntime:undname.obj
 0001:00011890       ??_C@_1DM@KHCHBNEB@?$AAa?$AAp?$AAi?$AA?9?$AAm?$AAs?$AA?9?$AAw?$AAi?$AAn?$AA?9?$AAc?$AAo?$AAr?$AAe?$AA?9?$AAf?$AAi?$AAb?$AAe?$AAr?$AAs?$AA?9?$AAl?$AA1?$AA?9?$AA1?$AA?9?$AA1?$AA?$AA@ 0000000180012890     libvcruntime:winapi_downlevel.obj
 0001:000118d0       ??_C@_1DK@LPPGFMPP@?$AAa?$AAp?$AAi?$AA?9?$AAm?$AAs?$AA?9?$AAw?$AAi?$AAn?$AA?9?$AAc?$AAo?$AAr?$AAe?$AA?9?$AAs?$AAy?$AAn?$AAc?$AAh?$AA?9?$AAl?$AA1?$AA?9?$AA2?$AA?9?$AA0?$AA?$AA@ 00000001800128d0     libvcruntime:winapi_downlevel.obj
 0001:00011910       ??_C@_1BC@GDMECMAK@?$AAk?$AAe?$AAr?$AAn?$AAe?$AAl?$AA3?$AA2?$AA?$AA@ 0000000180012910     libvcruntime:winapi_downlevel.obj
 0001:00011928       ??_C@_1BA@PFFKHIOG@?$AAa?$AAp?$AAi?$AA?9?$AAm?$AAs?$AA?9?$AA?$AA@ 0000000180012928     libvcruntime:winapi_downlevel.obj
 0001:00011938       ??_C@_1BA@IAIFMGEF@?$AAe?$AAx?$AAt?$AA?9?$AAm?$AAs?$AA?9?$AA?$AA@ 0000000180012938     libvcruntime:winapi_downlevel.obj
 0001:00011950       ??_C@_08KNHFBNJ@FlsAlloc?$AA@ 0000000180012950     libvcruntime:winapi_downlevel.obj
 0001:00011968       ??_C@_07PEJMOBNF@FlsFree?$AA@ 0000000180012968     libvcruntime:winapi_downlevel.obj
 0001:00011978       ??_C@_0M@GDNOONDI@FlsGetValue?$AA@ 0000000180012978     libvcruntime:winapi_downlevel.obj
 0001:00011990       ??_C@_0M@JCPCPOEF@FlsSetValue?$AA@ 0000000180012990     libvcruntime:winapi_downlevel.obj
 0001:000119a8       ??_C@_0BM@HCFOFFN@InitializeCriticalSectionEx?$AA@ 00000001800129a8     libvcruntime:winapi_downlevel.obj
 0001:000119c8       _pDestructExceptionObject  00000001800129c8     libvcruntime:ehhelpers.obj
 0001:000119d0       standard_lookup_table      00000001800129d0     libucrt:output.obj
 0001:00011a30       ??_C@_1O@CEDCILHN@?$AA?$CI?$AAn?$AAu?$AAl?$AAl?$AA?$CJ?$AA?$AA@ 0000000180012a30     libucrt:output.obj
 0001:00011a40       ??_C@_06OJHGLDPL@?$CInull?$CJ?$AA@ 0000000180012a40     libucrt:output.obj
 0001:00011bb0       ??_C@_0EA@FCLIIPNN@Visual?5C?$CL?$CL?5CRT?3?5Not?5enough?5memor@ 0000000180012bb0     libucrt:strerror.obj
 0001:00011c40       ?large_power_data@?1??multiply_by_power_of_ten@__crt_strtox@@YA_NAEAUbig_integer@2@I@Z@4QBIB 0000000180012c40     libucrt:input.obj
 0001:00012550       ?large_power_indices@?1??multiply_by_power_of_ten@__crt_strtox@@YA_NAEAUbig_integer@2@I@Z@4QBUunpack_index@?1??12@YA_N0I@Z@B 0000000180013550     libucrt:input.obj
 0001:000125e8       ?small_powers_of_ten@?1??multiply_by_power_of_ten@__crt_strtox@@YA_NAEAUbig_integer@2@I@Z@4QBIB 00000001800135e8     libucrt:input.obj
 0001:00012610       ??_C@_1GE@DPGDJKLM@?$AAm?$AAi?$AAn?$AAk?$AAe?$AAr?$AAn?$AAe?$AAl?$AA?2?$AAc?$AAr?$AAt?$AAs?$AA?2?$AAu?$AAc?$AAr?$AAt?$AA?2?$AAi?$AAn?$AAc?$AA?2?$AAc?$AAo?$AAr?$AAe?$AAc?$AAr?$AAt?$AA_@ 0000000180013610     libucrt:input.obj
 0001:00012680       ??_C@_1FM@FELNCOBF@?$AA_?$AA_?$AAc?$AAr?$AAt?$AA_?$AAs?$AAt?$AAr?$AAt?$AAo?$AAx?$AA?3?$AA?3?$AAf?$AAl?$AAo?$AAa?$AAt?$AAi?$AAn?$AAg?$AA_?$AAp?$AAo?$AAi?$AAn?$AAt?$AA_?$AAv?$AAa?$AAl@ 0000000180013680     libucrt:input.obj
 0001:000126e0       ??_C@_1BG@GEMHBGAF@?$AA_?$AAi?$AAs?$AA_?$AAd?$AAo?$AAu?$AAb?$AAl?$AAe?$AA?$AA@ 00000001800136e0     libucrt:input.obj
 0001:00012700       ??_C@_1FK@JOJELFFO@?$AA_?$AA_?$AAc?$AAr?$AAt?$AA_?$AAs?$AAt?$AAr?$AAt?$AAo?$AAx?$AA?3?$AA?3?$AAf?$AAl?$AAo?$AAa?$AAt?$AAi?$AAn?$AAg?$AA_?$AAp?$AAo?$AAi?$AAn?$AAt?$AA_?$AAv?$AAa?$AAl@ 0000000180013700     libucrt:input.obj
 0001:00012760       ??_C@_1BI@BANMPGJI@?$AA?$CB?$AA_?$AAi?$AAs?$AA_?$AAd?$AAo?$AAu?$AAb?$AAl?$AAe?$AA?$AA@ 0000000180013760     libucrt:input.obj
 0001:00012780       ?constraints@?1??is_length_valid@__crt_stdio_input@@YA_NW4conversion_mode@2@W4length_modifier@2@@Z@4QAY0M@$$CBEA 0000000180013780     libucrt:input.obj
 0001:000127f8       ?inf_uppercase@?1???$parse_floating_point_possible_infinity@DV?$input_adapter_character_source@V?$stream_input_adapter@D@__crt_stdio_input@@@__crt_strtox@@_K@__crt_strtox@@YA?AW4floating_point_parse_result@1@AEADAEAV?$input_adapter_character_source@V?$stream_input_adapter@D@__crt_stdio_input@@@1@_K@Z@4QBDB 00000001800137f8     libucrt:input.obj
 0001:000127fc       ?inf_lowercase@?1???$parse_floating_point_possible_infinity@DV?$input_adapter_character_source@V?$stream_input_adapter@D@__crt_stdio_input@@@__crt_strtox@@_K@__crt_strtox@@YA?AW4floating_point_parse_result@1@AEADAEAV?$input_adapter_character_source@V?$stream_input_adapter@D@__crt_stdio_input@@@1@_K@Z@4QBDB 00000001800137fc     libucrt:input.obj
 0001:00012800       ?inity_uppercase@?1???$parse_floating_point_possible_infinity@DV?$input_adapter_character_source@V?$stream_input_adapter@D@__crt_stdio_input@@@__crt_strtox@@_K@__crt_strtox@@YA?AW4floating_point_parse_result@1@AEADAEAV?$input_adapter_character_source@V?$stream_input_adapter@D@__crt_stdio_input@@@1@_K@Z@4QBDB 0000000180013800     libucrt:input.obj
 0001:00012808       ?inity_lowercase@?1???$parse_floating_point_possible_infinity@DV?$input_adapter_character_source@V?$stream_input_adapter@D@__crt_stdio_input@@@__crt_strtox@@_K@__crt_strtox@@YA?AW4floating_point_parse_result@1@AEADAEAV?$input_adapter_character_source@V?$stream_input_adapter@D@__crt_stdio_input@@@1@_K@Z@4QBDB 0000000180013808     libucrt:input.obj
 0001:00012810       ?uppercase@?1???$parse_floating_point_possible_nan@DV?$input_adapter_character_source@V?$stream_input_adapter@D@__crt_stdio_input@@@__crt_strtox@@_K@__crt_strtox@@YA?AW4floating_point_parse_result@1@AEADAEAV?$input_adapter_character_source@V?$stream_input_adapter@D@__crt_stdio_input@@@1@_K@Z@4QBDB 0000000180013810     libucrt:input.obj
 0001:00012814       ?lowercase@?1???$parse_floating_point_possible_nan@DV?$input_adapter_character_source@V?$stream_input_adapter@D@__crt_stdio_input@@@__crt_strtox@@_K@__crt_strtox@@YA?AW4floating_point_parse_result@1@AEADAEAV?$input_adapter_character_source@V?$stream_input_adapter@D@__crt_stdio_input@@@1@_K@Z@4QBDB 0000000180013814     libucrt:input.obj
 0001:00012818       ?uppercase@?1???$parse_floating_point_possible_nan_is_snan@DV?$input_adapter_character_source@V?$stream_input_adapter@D@__crt_stdio_input@@@__crt_strtox@@@__crt_strtox@@YA_NAEADAEAV?$input_adapter_character_source@V?$stream_input_adapter@D@__crt_stdio_input@@@1@@Z@4QBDB 0000000180013818     libucrt:input.obj
 0001:00012820       ?lowercase@?1???$parse_floating_point_possible_nan_is_snan@DV?$input_adapter_character_source@V?$stream_input_adapter@D@__crt_stdio_input@@@__crt_strtox@@@__crt_strtox@@YA_NAEADAEAV?$input_adapter_character_source@V?$stream_input_adapter@D@__crt_stdio_input@@@1@@Z@4QBDB 0000000180013820     libucrt:input.obj
 0001:00012828       ?uppercase@?1???$parse_floating_point_possible_nan_is_ind@DV?$input_adapter_character_source@V?$stream_input_adapter@D@__crt_stdio_input@@@__crt_strtox@@@__crt_strtox@@YA_NAEADAEAV?$input_adapter_character_source@V?$stream_input_adapter@D@__crt_stdio_input@@@1@@Z@4QBDB 0000000180013828     libucrt:input.obj
 0001:0001282c       ?lowercase@?1???$parse_floating_point_possible_nan_is_ind@DV?$input_adapter_character_source@V?$stream_input_adapter@D@__crt_stdio_input@@@__crt_strtox@@@__crt_strtox@@YA_NAEADAEAV?$input_adapter_character_source@V?$stream_input_adapter@D@__crt_stdio_input@@@1@@Z@4QBDB 000000018001382c     libucrt:input.obj
 0001:00012860       __acrt_exception_action_table 0000000180013860     libucrt:exception_filter.obj
 0001:00012920       __acrt_signal_action_table_count 0000000180013920     libucrt:exception_filter.obj
 0001:00012928       __acrt_signal_action_first_fpe_index 0000000180013928     libucrt:exception_filter.obj
 0001:00012930       __acrt_signal_action_fpe_count 0000000180013930     libucrt:exception_filter.obj
 0001:00012938       ??_C@_1BI@BGOHAHKC@?$AAm?$AAs?$AAc?$AAo?$AAr?$AAe?$AAe?$AA?4?$AAd?$AAl?$AAl?$AA?$AA@ 0000000180013938     libucrt:exit.obj
 0001:00012950       ??_C@_0P@MIGLKIOC@CorExitProcess?$AA@ 0000000180013950     libucrt:exit.obj
 0001:00012a60       ??_C@_03OEIAHPBN@INF?$AA@  0000000180013a60     libucrt:cvt.obj
 0001:00012a64       ??_C@_03OJHLLCGB@inf?$AA@  0000000180013a64     libucrt:cvt.obj
 0001:00012a68       ??_C@_03LKNCIKJB@NAN?$AA@  0000000180013a68     libucrt:cvt.obj
 0001:00012a6c       ??_C@_03LHCJEHON@nan?$AA@  0000000180013a6c     libucrt:cvt.obj
 0001:00012a70       ??_C@_09OFJJIMPC@NAN?$CISNAN?$CJ?$AA@ 0000000180013a70     libucrt:cvt.obj
 0001:00012a80       ??_C@_09IPFBKMDL@nan?$CIsnan?$CJ?$AA@ 0000000180013a80     libucrt:cvt.obj
 0001:00012a90       ??_C@_08IKHNHAJ@NAN?$CIIND?$CJ?$AA@ 0000000180013a90     libucrt:cvt.obj
 0001:00012aa0       ??_C@_08OFCDMILK@nan?$CIind?$CJ?$AA@ 0000000180013aa0     libucrt:cvt.obj
 0001:00012aac       ??_C@_05KLBDPFGC@e?$CL000?$AA@ 0000000180013aac     libucrt:cvt.obj
 0001:00012ac0       __lc_time_c                0000000180013ac0     libucrt:nlsdata.obj
 0001:00012d80       ??_C@_03KOEHGMDN@Sun?$AA@  0000000180013d80     libucrt:nlsdata.obj
 0001:00012d84       ??_C@_03PDAGKDH@Mon?$AA@   0000000180013d84     libucrt:nlsdata.obj
 0001:00012d88       ??_C@_03NAGEINEP@Tue?$AA@  0000000180013d88     libucrt:nlsdata.obj
 0001:00012d8c       ??_C@_03MHOMLAJA@Wed?$AA@  0000000180013d8c     libucrt:nlsdata.obj
 0001:00012d90       ??_C@_03IOFIKPDN@Thu?$AA@  0000000180013d90     libucrt:nlsdata.obj
 0001:00012d94       ??_C@_03IDIOELNC@Fri?$AA@  0000000180013d94     libucrt:nlsdata.obj
 0001:00012d98       ??_C@_03FEFJNEK@Sat?$AA@   0000000180013d98     libucrt:nlsdata.obj
 0001:00012d9c       ??_C@_06OOPIFAJ@Sunday?$AA@ 0000000180013d9c     libucrt:nlsdata.obj
 0001:00012da4       ??_C@_06JLEDEDGH@Monday?$AA@ 0000000180013da4     libucrt:nlsdata.obj
 0001:00012db0       ??_C@_07BAAGCFCM@Tuesday?$AA@ 0000000180013db0     libucrt:nlsdata.obj
 0001:00012db8       ??_C@_09DLIGFAKA@Wednesday?$AA@ 0000000180013db8     libucrt:nlsdata.obj
 0001:00012dc8       ??_C@_08HACCIKIA@Thursday?$AA@ 0000000180013dc8     libucrt:nlsdata.obj
 0001:00012dd4       ??_C@_06JECMNKMI@Friday?$AA@ 0000000180013dd4     libucrt:nlsdata.obj
 0001:00012de0       ??_C@_08INBOOONO@Saturday?$AA@ 0000000180013de0     libucrt:nlsdata.obj
 0001:00012dec       ??_C@_03JIHJHPIE@Jan?$AA@  0000000180013dec     libucrt:nlsdata.obj
 0001:00012df0       ??_C@_03HJBDCHOM@Feb?$AA@  0000000180013df0     libucrt:nlsdata.obj
 0001:00012df4       ??_C@_03ODNJBKGA@Mar?$AA@  0000000180013df4     libucrt:nlsdata.obj
 0001:00012df8       ??_C@_03LEOLGMJP@Apr?$AA@  0000000180013df8     libucrt:nlsdata.obj
 0001:00012dfc       ??_C@_03CNMDKL@May?$AA@    0000000180013dfc     libucrt:nlsdata.obj
 0001:00012e00       ??_C@_03IDFGHECI@Jun?$AA@  0000000180013e00     libucrt:nlsdata.obj
 0001:00012e04       ??_C@_03LBGABGKK@Jul?$AA@  0000000180013e04     libucrt:nlsdata.obj
 0001:00012e08       ??_C@_03IFJFEIGA@Aug?$AA@  0000000180013e08     libucrt:nlsdata.obj
 0001:00012e0c       ??_C@_03GGCAPAJC@Sep?$AA@  0000000180013e0c     libucrt:nlsdata.obj
 0001:00012e10       ??_C@_03BMAOKBAD@Oct?$AA@  0000000180013e10     libucrt:nlsdata.obj
 0001:00012e14       ??_C@_03JPJOFNIA@Nov?$AA@  0000000180013e14     libucrt:nlsdata.obj
 0001:00012e18       ??_C@_03MKABNOCG@Dec?$AA@  0000000180013e18     libucrt:nlsdata.obj
 0001:00012e20       ??_C@_07CGJPFGJA@January?$AA@ 0000000180013e20     libucrt:nlsdata.obj
 0001:00012e28       ??_C@_08GNJGEPFN@February?$AA@ 0000000180013e28     libucrt:nlsdata.obj
 0001:00012e34       ??_C@_05HPCKOFNC@March?$AA@ 0000000180013e34     libucrt:nlsdata.obj
 0001:00012e3c       ??_C@_05DMJDNLEJ@April?$AA@ 0000000180013e3c     libucrt:nlsdata.obj
 0001:00012e44       ??_C@_04CNLMGBGM@June?$AA@ 0000000180013e44     libucrt:nlsdata.obj
 0001:00012e4c       ??_C@_04MIEPOIFP@July?$AA@ 0000000180013e4c     libucrt:nlsdata.obj
 0001:00012e54       ??_C@_06LBBHFDDG@August?$AA@ 0000000180013e54     libucrt:nlsdata.obj
 0001:00012e60       ??_C@_09BHHEALKD@September?$AA@ 0000000180013e60     libucrt:nlsdata.obj
 0001:00012e70       ??_C@_07JJNFCEND@October?$AA@ 0000000180013e70     libucrt:nlsdata.obj
 0001:00012e78       ??_C@_08HCHEGEOA@November?$AA@ 0000000180013e78     libucrt:nlsdata.obj
 0001:00012e88       ??_C@_08EDHMEBNP@December?$AA@ 0000000180013e88     libucrt:nlsdata.obj
 0001:00012e94       ??_C@_02DEDBPAFC@AM?$AA@   0000000180013e94     libucrt:nlsdata.obj
 0001:00012e98       ??_C@_02CJNFDJBF@PM?$AA@   0000000180013e98     libucrt:nlsdata.obj
 0001:00012ea0       ??_C@_08BPBNCDIB@MM?1dd?1yy?$AA@ 0000000180013ea0     libucrt:nlsdata.obj
 0001:00012eb0       ??_C@_0BE@CKGJFCPC@dddd?0?5MMMM?5dd?0?5yyyy?$AA@ 0000000180013eb0     libucrt:nlsdata.obj
 0001:00012ec8       ??_C@_08JCCMCCIL@HH?3mm?3ss?$AA@ 0000000180013ec8     libucrt:nlsdata.obj
 0001:00012ed8       ??_C@_17MBGCMIPB@?$AAS?$AAu?$AAn?$AA?$AA@ 0000000180013ed8     libucrt:nlsdata.obj
 0001:00012ee0       ??_C@_17KBOMKBF@?$AAM?$AAo?$AAn?$AA?$AA@ 0000000180013ee0     libucrt:nlsdata.obj
 0001:00012ee8       ??_C@_17BMKGEGOJ@?$AAT?$AAu?$AAe?$AA?$AA@ 0000000180013ee8     libucrt:nlsdata.obj
 0001:00012ef0       ??_C@_17CJEDCEPE@?$AAW?$AAe?$AAd?$AA?$AA@ 0000000180013ef0     libucrt:nlsdata.obj
 0001:00012ef8       ??_C@_17PDPHAADD@?$AAT?$AAh?$AAu?$AA?$AA@ 0000000180013ef8     libucrt:nlsdata.obj
 0001:00012f00       ??_C@_17HFOLPPLP@?$AAF?$AAr?$AAi?$AA?$AA@ 0000000180013f00     libucrt:nlsdata.obj
 0001:00012f08       ??_C@_17GGIBDPIH@?$AAS?$AAa?$AAt?$AA?$AA@ 0000000180013f08     libucrt:nlsdata.obj
 0001:00012f10       ??_C@_1O@IHNHDHPB@?$AAS?$AAu?$AAn?$AAd?$AAa?$AAy?$AA?$AA@ 0000000180013f10     libucrt:nlsdata.obj
 0001:00012f20       ??_C@_1O@MMNBFLIA@?$AAM?$AAo?$AAn?$AAd?$AAa?$AAy?$AA?$AA@ 0000000180013f20     libucrt:nlsdata.obj
 0001:00012f30       ??_C@_1BA@ENFBFFEK@?$AAT?$AAu?$AAe?$AAs?$AAd?$AAa?$AAy?$AA?$AA@ 0000000180013f30     libucrt:nlsdata.obj
 0001:00012f40       ??_C@_1BE@EBOGMDOH@?$AAW?$AAe?$AAd?$AAn?$AAe?$AAs?$AAd?$AAa?$AAy?$AA?$AA@ 0000000180013f40     libucrt:nlsdata.obj
 0001:00012f58       ??_C@_1BC@HHMNLIHE@?$AAT?$AAh?$AAu?$AAr?$AAs?$AAd?$AAa?$AAy?$AA?$AA@ 0000000180013f58     libucrt:nlsdata.obj
 0001:00012f70       ??_C@_1O@PDICJHAG@?$AAF?$AAr?$AAi?$AAd?$AAa?$AAy?$AA?$AA@ 0000000180013f70     libucrt:nlsdata.obj
 0001:00012f80       ??_C@_1BC@ENMNNPAJ@?$AAS?$AAa?$AAt?$AAu?$AAr?$AAd?$AAa?$AAy?$AA?$AA@ 0000000180013f80     libucrt:nlsdata.obj
 0001:00012f98       ??_C@_17DKNBKCHM@?$AAJ?$AAa?$AAn?$AA?$AA@ 0000000180013f98     libucrt:nlsdata.obj
 0001:00012fa0       ??_C@_17LMDJEKJN@?$AAF?$AAe?$AAb?$AA?$AA@ 0000000180013fa0     libucrt:nlsdata.obj
 0001:00012fa8       ??_C@_17CKNLEDEC@?$AAM?$AAa?$AAr?$AA?$AA@ 0000000180013fa8     libucrt:nlsdata.obj
 0001:00012fb0       ??_C@_17LFPOIHDD@?$AAA?$AAp?$AAr?$AA?$AA@ 0000000180013fb0     libucrt:nlsdata.obj
 0001:00012fb8       ??_C@_17PNNKMEED@?$AAM?$AAa?$AAy?$AA?$AA@ 0000000180013fb8     libucrt:nlsdata.obj
 0001:00012fc0       ??_C@_17KCJGOCPB@?$AAJ?$AAu?$AAn?$AA?$AA@ 0000000180013fc0     libucrt:nlsdata.obj
 0001:00012fc8       ??_C@_17IJPCKHK@?$AAJ?$AAu?$AAl?$AA?$AA@ 0000000180013fc8     libucrt:nlsdata.obj
 0001:00012fd0       ??_C@_17ICPELBCN@?$AAA?$AAu?$AAg?$AA?$AA@ 0000000180013fd0     libucrt:nlsdata.obj
 0001:00012fd8       ??_C@_17HCHCOKMG@?$AAS?$AAe?$AAp?$AA?$AA@ 0000000180013fd8     libucrt:nlsdata.obj
 0001:00012fe0       ??_C@_17FNLKOI@?$AAO?$AAc?$AAt?$AA?$AA@ 0000000180013fe0     libucrt:nlsdata.obj
 0001:00012fe8       ??_C@_17BBDMLCIG@?$AAN?$AAo?$AAv?$AA?$AA@ 0000000180013fe8     libucrt:nlsdata.obj
 0001:00012ff0       ??_C@_17EGKACKIF@?$AAD?$AAe?$AAc?$AA?$AA@ 0000000180013ff0     libucrt:nlsdata.obj
 0001:00012ff8       ??_C@_1BA@EFMEIEBA@?$AAJ?$AAa?$AAn?$AAu?$AAa?$AAr?$AAy?$AA?$AA@ 0000000180013ff8     libucrt:nlsdata.obj
 0001:00013008       ??_C@_1BC@JGDDFFAM@?$AAF?$AAe?$AAb?$AAr?$AAu?$AAa?$AAr?$AAy?$AA?$AA@ 0000000180014008     libucrt:nlsdata.obj
 0001:00013020       ??_C@_1M@IKEENEDF@?$AAM?$AAa?$AAr?$AAc?$AAh?$AA?$AA@ 0000000180014020     libucrt:nlsdata.obj
 0001:00013030       ??_C@_1M@GJNLMHFD@?$AAA?$AAp?$AAr?$AAi?$AAl?$AA?$AA@ 0000000180014030     libucrt:nlsdata.obj
 0001:00013040       ??_C@_19EPFLPGAP@?$AAJ?$AAu?$AAn?$AAe?$AA?$AA@ 0000000180014040     libucrt:nlsdata.obj
 0001:00013050       ??_C@_19BIFMLPCD@?$AAJ?$AAu?$AAl?$AAy?$AA?$AA@ 0000000180014050     libucrt:nlsdata.obj
 0001:00013060       ??_C@_1O@PAHLKOAC@?$AAA?$AAu?$AAg?$AAu?$AAs?$AAt?$AA?$AA@ 0000000180014060     libucrt:nlsdata.obj
 0001:00013070       ??_C@_1BE@DKAAMBJL@?$AAS?$AAe?$AAp?$AAt?$AAe?$AAm?$AAb?$AAe?$AAr?$AA?$AA@ 0000000180014070     libucrt:nlsdata.obj
 0001:00013088       ??_C@_1BA@EPANDLNG@?$AAO?$AAc?$AAt?$AAo?$AAb?$AAe?$AAr?$AA?$AA@ 0000000180014088     libucrt:nlsdata.obj
 0001:00013098       ??_C@_1BC@BGLIFPF@?$AAN?$AAo?$AAv?$AAe?$AAm?$AAb?$AAe?$AAr?$AA?$AA@ 0000000180014098     libucrt:nlsdata.obj
 0001:000130b0       ??_C@_1BC@FEMKIFH@?$AAD?$AAe?$AAc?$AAe?$AAm?$AAb?$AAe?$AAr?$AA?$AA@ 00000001800140b0     libucrt:nlsdata.obj
 0001:000130c4       ??_C@_15ODEHAHHF@?$AAA?$AAM?$AA?$AA@ 00000001800140c4     libucrt:nlsdata.obj
 0001:000130cc       ??_C@_15CLMNNGEL@?$AAP?$AAM?$AA?$AA@ 00000001800140cc     libucrt:nlsdata.obj
 0001:000130d8       ??_C@_1BC@IEBCMHCM@?$AAM?$AAM?$AA?1?$AAd?$AAd?$AA?1?$AAy?$AAy?$AA?$AA@ 00000001800140d8     libucrt:nlsdata.obj
 0001:000130f0       ??_C@_1CI@KNAKOEBC@?$AAd?$AAd?$AAd?$AAd?$AA?0?$AA?5?$AAM?$AAM?$AAM?$AAM?$AA?5?$AAd?$AAd?$AA?0?$AA?5?$AAy?$AAy?$AAy?$AAy?$AA?$AA@ 00000001800140f0     libucrt:nlsdata.obj
 0001:00013118       ??_C@_1BC@GDGBMEMK@?$AAH?$AAH?$AA?3?$AAm?$AAm?$AA?3?$AAs?$AAs?$AA?$AA@ 0000000180014118     libucrt:nlsdata.obj
 0001:00013130       ??_C@_1M@BMHNFIME@?$AAe?$AAn?$AA?9?$AAU?$AAS?$AA?$AA@ 0000000180014130     libucrt:nlsdata.obj
 0001:0001313c       ?ccs@?1???$__acrt_stdio_parse_mode@_W@@YA?AU__acrt_stdio_stream_mode@@QEB_W@Z@4QB_WB 000000018001413c     libucrt:openfile.obj
 0001:00013148       ?utf8_encoding@?1???$__acrt_stdio_parse_mode@_W@@YA?AU__acrt_stdio_stream_mode@@QEB_W@Z@4QB_WB 0000000180014148     libucrt:openfile.obj
 0001:00013158       ?utf16_encoding@?1???$__acrt_stdio_parse_mode@_W@@YA?AU__acrt_stdio_stream_mode@@QEB_W@Z@4QB_WB 0000000180014158     libucrt:openfile.obj
 0001:00013168       ?unicode_encoding@?1???$__acrt_stdio_parse_mode@_W@@YA?AU__acrt_stdio_stream_mode@@QEB_W@Z@4QB_WB 0000000180014168     libucrt:openfile.obj
 0001:00013190       _sys_errlist               0000000180014190     libucrt:syserr.obj
 0001:000132f0       ??_C@_08INEPGKHH@No?5error?$AA@ 00000001800142f0     libucrt:syserr.obj
 0001:00013300       ??_C@_0BI@BJFCGOHL@Operation?5not?5permitted?$AA@ 0000000180014300     libucrt:syserr.obj
 0001:00013318       ??_C@_0BK@FMDHKPNF@No?5such?5file?5or?5directory?$AA@ 0000000180014318     libucrt:syserr.obj
 0001:00013338       ??_C@_0BA@FKIAIBGA@No?5such?5process?$AA@ 0000000180014338     libucrt:syserr.obj
 0001:00013348       ??_C@_0BK@FJBOAFDK@Interrupted?5function?5call?$AA@ 0000000180014348     libucrt:syserr.obj
 0001:00013368       ??_C@_0BD@KKNFOBBD@Input?1output?5error?$AA@ 0000000180014368     libucrt:syserr.obj
 0001:00013380       ??_C@_0BK@DPKMCKJ@No?5such?5device?5or?5address?$AA@ 0000000180014380     libucrt:syserr.obj
 0001:000133a0       ??_C@_0BC@MFFGCDFL@Arg?5list?5too?5long?$AA@ 00000001800143a0     libucrt:syserr.obj
 0001:000133b8       ??_C@_0BC@HKPNECK@Exec?5format?5error?$AA@ 00000001800143b8     libucrt:syserr.obj
 0001:000133d0       ??_C@_0BE@NFGDDCEF@Bad?5file?5descriptor?$AA@ 00000001800143d0     libucrt:syserr.obj
 0001:000133e8       ??_C@_0BD@LOHELEP@No?5child?5processes?$AA@ 00000001800143e8     libucrt:syserr.obj
 0001:00013400       ??_C@_0CB@EPFKGNAK@Resource?5temporarily?5unavailable@ 0000000180014400     libucrt:syserr.obj
 0001:00013428       ??_C@_0BB@IMDKMPFB@Not?5enough?5space?$AA@ 0000000180014428     libucrt:syserr.obj
 0001:00013440       ??_C@_0BC@HFNFNKAI@Permission?5denied?$AA@ 0000000180014440     libucrt:syserr.obj
 0001:00013458       ??_C@_0M@LOEHLCJD@Bad?5address?$AA@ 0000000180014458     libucrt:syserr.obj
 0001:00013468       ??_C@_0O@NIPGCINC@Unknown?5error?$AA@ 0000000180014468     libucrt:syserr.obj
 0001:00013478       ??_C@_0BA@BIBLIOEK@Resource?5device?$AA@ 0000000180014478     libucrt:syserr.obj
 0001:00013488       ??_C@_0M@NAAJNNGH@File?5exists?$AA@ 0000000180014488     libucrt:syserr.obj
 0001:00013498       ??_C@_0O@OAMDNOCP@Improper?5link?$AA@ 0000000180014498     libucrt:syserr.obj
 0001:000134a8       ??_C@_0P@NLEIANHE@No?5such?5device?$AA@ 00000001800144a8     libucrt:syserr.obj
 0001:000134b8       ??_C@_0BA@CJBACOOL@Not?5a?5directory?$AA@ 00000001800144b8     libucrt:syserr.obj
 0001:000134c8       ??_C@_0P@NDHGCGKE@Is?5a?5directory?$AA@ 00000001800144c8     libucrt:syserr.obj
 0001:000134d8       ??_C@_0BB@HMGGCEBG@Invalid?5argument?$AA@ 00000001800144d8     libucrt:syserr.obj
 0001:000134f0       ??_C@_0BO@IIFBODJE@Too?5many?5open?5files?5in?5system?$AA@ 00000001800144f0     libucrt:syserr.obj
 0001:00013510       ??_C@_0BE@INBJMKGG@Too?5many?5open?5files?$AA@ 0000000180014510     libucrt:syserr.obj
 0001:00013528       ??_C@_0CE@ONOKNLPF@Inappropriate?5I?1O?5control?5operat@ 0000000180014528     libucrt:syserr.obj
 0001:00013550       ??_C@_0P@LFMMIPAE@File?5too?5large?$AA@ 0000000180014550     libucrt:syserr.obj
 0001:00013560       ??_C@_0BI@FEALHKLD@No?5space?5left?5on?5device?$AA@ 0000000180014560     libucrt:syserr.obj
 0001:00013578       ??_C@_0N@FEHLOILP@Invalid?5seek?$AA@ 0000000180014578     libucrt:syserr.obj
 0001:00013588       ??_C@_0BG@DDBFNKBH@Read?9only?5file?5system?$AA@ 0000000180014588     libucrt:syserr.obj
 0001:000135a0       ??_C@_0P@PKCJJLLM@Too?5many?5links?$AA@ 00000001800145a0     libucrt:syserr.obj
 0001:000135b0       ??_C@_0M@LHEPIIOM@Broken?5pipe?$AA@ 00000001800145b0     libucrt:syserr.obj
 0001:000135c0       ??_C@_0N@MMJPGLJK@Domain?5error?$AA@ 00000001800145c0     libucrt:syserr.obj
 0001:000135d0       ??_C@_0BB@FCBJFCAJ@Result?5too?5large?$AA@ 00000001800145d0     libucrt:syserr.obj
 0001:000135e8       ??_C@_0BK@JAEBMJJM@Resource?5deadlock?5avoided?$AA@ 00000001800145e8     libucrt:syserr.obj
 0001:00013608       ??_C@_0BC@BEDIHIDK@Filename?5too?5long?$AA@ 0000000180014608     libucrt:syserr.obj
 0001:00013620       ??_C@_0BD@CLHBCGPB@No?5locks?5available?$AA@ 0000000180014620     libucrt:syserr.obj
 0001:00013638       ??_C@_0BJ@IHEHINLI@Function?5not?5implemented?$AA@ 0000000180014638     libucrt:syserr.obj
 0001:00013658       ??_C@_0BE@ICMCHPHH@Directory?5not?5empty?$AA@ 0000000180014658     libucrt:syserr.obj
 0001:00013670       ??_C@_0BG@KLEAJEFJ@Illegal?5byte?5sequence?$AA@ 0000000180014670     libucrt:syserr.obj
 0001:00013688       _sys_nerr                  0000000180014688     libucrt:syserr.obj
 0001:00013730       ??_C@_1EA@JGEFHKEI@?$AAa?$AAp?$AAi?$AA?9?$AAm?$AAs?$AA?9?$AAw?$AAi?$AAn?$AA?9?$AAc?$AAo?$AAr?$AAe?$AA?9?$AAd?$AAa?$AAt?$AAe?$AAt?$AAi?$AAm?$AAe?$AA?9?$AAl?$AA1?$AA?9?$AA1?$AA?9?$AA1?$AA?$AA@ 0000000180014730     libucrt:winapi_thunks.obj
 0001:00013770       ??_C@_1DI@IJCEHOCB@?$AAa?$AAp?$AAi?$AA?9?$AAm?$AAs?$AA?9?$AAw?$AAi?$AAn?$AA?9?$AAc?$AAo?$AAr?$AAe?$AA?9?$AAf?$AAi?$AAl?$AAe?$AA?9?$AAl?$AA1?$AA?9?$AA2?$AA?9?$AA2?$AA?$AA@ 0000000180014770     libucrt:winapi_thunks.obj
 0001:000137b0       ??_C@_1EI@MPIAOHOC@?$AAa?$AAp?$AAi?$AA?9?$AAm?$AAs?$AA?9?$AAw?$AAi?$AAn?$AA?9?$AAc?$AAo?$AAr?$AAe?$AA?9?$AAl?$AAo?$AAc?$AAa?$AAl?$AAi?$AAz?$AAa?$AAt?$AAi?$AAo?$AAn?$AA?9?$AAl?$AA1?$AA?9@ 00000001800147b0     libucrt:winapi_thunks.obj
 0001:00013800       ??_C@_1FK@FPHCKFIE@?$AAa?$AAp?$AAi?$AA?9?$AAm?$AAs?$AA?9?$AAw?$AAi?$AAn?$AA?9?$AAc?$AAo?$AAr?$AAe?$AA?9?$AAl?$AAo?$AAc?$AAa?$AAl?$AAi?$AAz?$AAa?$AAt?$AAi?$AAo?$AAn?$AA?9?$AAo?$AAb?$AAs@ 0000000180014800     libucrt:winapi_thunks.obj
 0001:00013860       ??_C@_1EM@DILCGIIO@?$AAa?$AAp?$AAi?$AA?9?$AAm?$AAs?$AA?9?$AAw?$AAi?$AAn?$AA?9?$AAc?$AAo?$AAr?$AAe?$AA?9?$AAp?$AAr?$AAo?$AAc?$AAe?$AAs?$AAs?$AAt?$AAh?$AAr?$AAe?$AAa?$AAd?$AAs?$AA?9?$AAl@ 0000000180014860     libucrt:winapi_thunks.obj
 0001:000138b0       ??_C@_1DM@LNCGDDPN@?$AAa?$AAp?$AAi?$AA?9?$AAm?$AAs?$AA?9?$AAw?$AAi?$AAn?$AA?9?$AAc?$AAo?$AAr?$AAe?$AA?9?$AAs?$AAt?$AAr?$AAi?$AAn?$AAg?$AA?9?$AAl?$AA1?$AA?9?$AA1?$AA?9?$AA0?$AA?$AA@ 00000001800148b0     libucrt:winapi_thunks.obj
 0001:000138f0       ??_C@_1DO@FPAPJEMD@?$AAa?$AAp?$AAi?$AA?9?$AAm?$AAs?$AA?9?$AAw?$AAi?$AAn?$AA?9?$AAc?$AAo?$AAr?$AAe?$AA?9?$AAs?$AAy?$AAs?$AAi?$AAn?$AAf?$AAo?$AA?9?$AAl?$AA1?$AA?9?$AA2?$AA?9?$AA1?$AA?$AA@ 00000001800148f0     libucrt:winapi_thunks.obj
 0001:00013930       ??_C@_1DK@NDHNAHIO@?$AAa?$AAp?$AAi?$AA?9?$AAm?$AAs?$AA?9?$AAw?$AAi?$AAn?$AA?9?$AAc?$AAo?$AAr?$AAe?$AA?9?$AAw?$AAi?$AAn?$AAr?$AAt?$AA?9?$AAl?$AA1?$AA?9?$AA1?$AA?9?$AA0?$AA?$AA@ 0000000180014930     libucrt:winapi_thunks.obj
 0001:00013970       ??_C@_1DM@KGHDGBCM@?$AAa?$AAp?$AAi?$AA?9?$AAm?$AAs?$AA?9?$AAw?$AAi?$AAn?$AA?9?$AAc?$AAo?$AAr?$AAe?$AA?9?$AAx?$AAs?$AAt?$AAa?$AAt?$AAe?$AA?9?$AAl?$AA2?$AA?9?$AA1?$AA?9?$AA0?$AA?$AA@ 0000000180014970     libucrt:winapi_thunks.obj
 0001:000139b0       ??_C@_1EO@IJIOEFOH@?$AAa?$AAp?$AAi?$AA?9?$AAm?$AAs?$AA?9?$AAw?$AAi?$AAn?$AA?9?$AAr?$AAt?$AAc?$AAo?$AAr?$AAe?$AA?9?$AAn?$AAt?$AAu?$AAs?$AAe?$AAr?$AA?9?$AAw?$AAi?$AAn?$AAd?$AAo?$AAw?$AA?9@ 00000001800149b0     libucrt:winapi_thunks.obj
 0001:00013a00       ??_C@_1FG@HHGEKANL@?$AAa?$AAp?$AAi?$AA?9?$AAm?$AAs?$AA?9?$AAw?$AAi?$AAn?$AA?9?$AAs?$AAe?$AAc?$AAu?$AAr?$AAi?$AAt?$AAy?$AA?9?$AAs?$AAy?$AAs?$AAt?$AAe?$AAm?$AAf?$AAu?$AAn?$AAc?$AAt?$AAi@ 0000000180014a00     libucrt:winapi_thunks.obj
 0001:00013a60       ??_C@_1EG@DBIOJECG@?$AAe?$AAx?$AAt?$AA?9?$AAm?$AAs?$AA?9?$AAw?$AAi?$AAn?$AA?9?$AAn?$AAt?$AAu?$AAs?$AAe?$AAr?$AA?9?$AAd?$AAi?$AAa?$AAl?$AAo?$AAg?$AAb?$AAo?$AAx?$AA?9?$AAl?$AA1?$AA?9?$AA1@ 0000000180014a60     libucrt:winapi_thunks.obj
 0001:00013ab0       ??_C@_1EO@FIHMJCLF@?$AAe?$AAx?$AAt?$AA?9?$AAm?$AAs?$AA?9?$AAw?$AAi?$AAn?$AA?9?$AAn?$AAt?$AAu?$AAs?$AAe?$AAr?$AA?9?$AAw?$AAi?$AAn?$AAd?$AAo?$AAw?$AAs?$AAt?$AAa?$AAt?$AAi?$AAo?$AAn?$AA?9@ 0000000180014ab0     libucrt:winapi_thunks.obj
 0001:00013b00       ??_C@_1BC@DNHGCMLG@?$AAa?$AAd?$AAv?$AAa?$AAp?$AAi?$AA3?$AA2?$AA?$AA@ 0000000180014b00     libucrt:winapi_thunks.obj
 0001:00013b18       ??_C@_1M@OAIMIKLP@?$AAn?$AAt?$AAd?$AAl?$AAl?$AA?$AA@ 0000000180014b18     libucrt:winapi_thunks.obj
 0001:00013b30       ??_C@_1EG@DPGNFKGC@?$AAa?$AAp?$AAi?$AA?9?$AAm?$AAs?$AA?9?$AAw?$AAi?$AAn?$AA?9?$AAa?$AAp?$AAp?$AAm?$AAo?$AAd?$AAe?$AAl?$AA?9?$AAr?$AAu?$AAn?$AAt?$AAi?$AAm?$AAe?$AA?9?$AAl?$AA1?$AA?9?$AA1@ 0000000180014b30     libucrt:winapi_thunks.obj
 0001:00013b78       ??_C@_1O@BCCLBEOE@?$AAu?$AAs?$AAe?$AAr?$AA3?$AA2?$AA?$AA@ 0000000180014b78     libucrt:winapi_thunks.obj
 0001:00013b90       ??_C@_0BA@FHFNEAED@AreFileApisANSI?$AA@ 0000000180014b90     libucrt:winapi_thunks.obj
 0001:00013ba8       ??_C@_0BA@IHGNDAEB@CompareStringEx?$AA@ 0000000180014ba8     libucrt:winapi_thunks.obj
 0001:00013be8       ??_C@_0O@KKBNKAPF@LCMapStringEx?$AA@ 0000000180014be8     libucrt:winapi_thunks.obj
 0001:00013c00       ??_C@_0BB@HBDEELFH@LocaleNameToLCID?$AA@ 0000000180014c00     libucrt:winapi_thunks.obj
 0001:00013c18       ??_C@_0CF@OJOFEIGO@AppPolicyGetProcessTerminationMe@ 0000000180014c18     libucrt:winapi_thunks.obj
 0001:00013c40       __newctype                 0000000180014c40     libucrt:ctype.obj
 0001:00013f40       __newclmap                 0000000180014f40     libucrt:ctype.obj
 0001:000140c0       __newcumap                 00000001800150c0     libucrt:ctype.obj
 0001:00014240       _wctype                    0000000180015240     libucrt:ctype.obj
 0001:00014498       ??_C@_1M@HPNHIDJI@?$AAj?$AAa?$AA?9?$AAJ?$AAP?$AA?$AA@ 0000000180015498     libucrt:mbctype.obj
 0001:000144a8       ??_C@_1M@BIBDDEMK@?$AAz?$AAh?$AA?9?$AAC?$AAN?$AA?$AA@ 00000001800154a8     libucrt:mbctype.obj
 0001:000144b8       ??_C@_1M@JLOOOEGK@?$AAk?$AAo?$AA?9?$AAK?$AAR?$AA?$AA@ 00000001800154b8     libucrt:mbctype.obj
 0001:000144c8       ??_C@_1M@CLNBBOPM@?$AAz?$AAh?$AA?9?$AAT?$AAW?$AA?$AA@ 00000001800154c8     libucrt:mbctype.obj
 0001:000144d4       ??_C@_05DNEBIAHO@1?$CDINF?$AA@ 00000001800154d4     libucrt:cfout.obj
 0001:000144dc       ??_C@_06IMKFLFPG@1?$CDQNAN?$AA@ 00000001800154dc     libucrt:cfout.obj
 0001:000144e4       ??_C@_06PGGFOGJG@1?$CDSNAN?$AA@ 00000001800154e4     libucrt:cfout.obj
 0001:000144ec       ??_C@_05PHHOCPM@1?$CDIND?$AA@ 00000001800154ec     libucrt:cfout.obj
 0001:000144f4       ??_C@_15PJPFLCCM@?$AAu?$AAk?$AA?$AA@ 00000001800154f4     libucrt:get_qualified_locale.obj
 0001:00014500       ??_C@_1M@BJNKEDC@?$AAc?$AAa?$AA?9?$AAE?$AAS?$AA?$AA@ 0000000180015500     libucrt:lcidtoname_downlevel.obj
 0001:00014510       ??_C@_1M@IJJHFJHA@?$AAc?$AAs?$AA?9?$AAC?$AAZ?$AA?$AA@ 0000000180015510     libucrt:lcidtoname_downlevel.obj
 0001:00014520       ??_C@_1M@CLPEOBGI@?$AAd?$AAa?$AA?9?$AAD?$AAK?$AA?$AA@ 0000000180015520     libucrt:lcidtoname_downlevel.obj
 0001:00014530       ??_C@_1M@MCMADGCB@?$AAd?$AAe?$AA?9?$AAD?$AAE?$AA?$AA@ 0000000180015530     libucrt:lcidtoname_downlevel.obj
 0001:00014540       ??_C@_1M@OOCKEMAM@?$AAe?$AAl?$AA?9?$AAG?$AAR?$AA?$AA@ 0000000180015540     libucrt:lcidtoname_downlevel.obj
 0001:00014550       ??_C@_1M@DDNJFGID@?$AAf?$AAi?$AA?9?$AAF?$AAI?$AA?$AA@ 0000000180015550     libucrt:lcidtoname_downlevel.obj
 0001:00014560       ??_C@_1M@GLIPPMAC@?$AAf?$AAr?$AA?9?$AAF?$AAR?$AA?$AA@ 0000000180015560     libucrt:lcidtoname_downlevel.obj
 0001:00014570       ??_C@_1M@GFMCHPE@?$AAh?$AAe?$AA?9?$AAI?$AAL?$AA?$AA@ 0000000180015570     libucrt:lcidtoname_downlevel.obj
 0001:00014580       ??_C@_1M@MHLPGNKM@?$AAh?$AAu?$AA?9?$AAH?$AAU?$AA?$AA@ 0000000180015580     libucrt:lcidtoname_downlevel.obj
 0001:00014590       ??_C@_1M@LPDDNNPN@?$AAi?$AAs?$AA?9?$AAI?$AAS?$AA?$AA@ 0000000180015590     libucrt:lcidtoname_downlevel.obj
 0001:000145a0       ??_C@_1M@MADIPODN@?$AAi?$AAt?$AA?9?$AAI?$AAT?$AA?$AA@ 00000001800155a0     libucrt:lcidtoname_downlevel.obj
 0001:000145b0       ??_C@_1M@IHBJJGG@?$AAn?$AAl?$AA?9?$AAN?$AAL?$AA?$AA@ 00000001800155b0     libucrt:lcidtoname_downlevel.obj
 0001:000145c0       ??_C@_1M@EANAGDL@?$AAn?$AAb?$AA?9?$AAN?$AAO?$AA?$AA@ 00000001800155c0     libucrt:lcidtoname_downlevel.obj
 0001:000145d0       ??_C@_1M@NEIEMEGP@?$AAp?$AAl?$AA?9?$AAP?$AAL?$AA?$AA@ 00000001800155d0     libucrt:lcidtoname_downlevel.obj
 0001:000145e0       ??_C@_1M@BOCFIGEP@?$AAp?$AAt?$AA?9?$AAB?$AAR?$AA?$AA@ 00000001800155e0     libucrt:lcidtoname_downlevel.obj
 0001:000145f0       ??_C@_1M@IMPFOPBG@?$AAr?$AAo?$AA?9?$AAR?$AAO?$AA?$AA@ 00000001800155f0     libucrt:lcidtoname_downlevel.obj
 0001:00014600       ??_C@_1M@IDNNEJMM@?$AAr?$AAu?$AA?9?$AAR?$AAU?$AA?$AA@ 0000000180015600     libucrt:lcidtoname_downlevel.obj
 0001:00014610       ??_C@_1M@LILEEOGM@?$AAh?$AAr?$AA?9?$AAH?$AAR?$AA?$AA@ 0000000180015610     libucrt:lcidtoname_downlevel.obj
 0001:00014620       ??_C@_1M@FKIFEHPB@?$AAs?$AAk?$AA?9?$AAS?$AAK?$AA?$AA@ 0000000180015620     libucrt:lcidtoname_downlevel.obj
 0001:00014630       ??_C@_1M@LJMAMNPJ@?$AAs?$AAq?$AA?9?$AAA?$AAL?$AA?$AA@ 0000000180015630     libucrt:lcidtoname_downlevel.obj
 0001:00014640       ??_C@_1M@GIAKDKJK@?$AAs?$AAv?$AA?9?$AAS?$AAE?$AA?$AA@ 0000000180015640     libucrt:lcidtoname_downlevel.obj
 0001:00014650       ??_C@_1M@MKJKIKCL@?$AAt?$AAh?$AA?9?$AAT?$AAH?$AA?$AA@ 0000000180015650     libucrt:lcidtoname_downlevel.obj
 0001:00014660       ??_C@_1M@MFLCCMPB@?$AAt?$AAr?$AA?9?$AAT?$AAR?$AA?$AA@ 0000000180015660     libucrt:lcidtoname_downlevel.obj
 0001:00014670       ??_C@_1M@OIJHDKJN@?$AAu?$AAr?$AA?9?$AAP?$AAK?$AA?$AA@ 0000000180015670     libucrt:lcidtoname_downlevel.obj
 0001:00014680       ??_C@_1M@LHIPCIEK@?$AAi?$AAd?$AA?9?$AAI?$AAD?$AA?$AA@ 0000000180015680     libucrt:lcidtoname_downlevel.obj
 0001:00014690       ??_C@_1M@MFMOBGI@?$AAu?$AAk?$AA?9?$AAU?$AAA?$AA?$AA@ 0000000180015690     libucrt:lcidtoname_downlevel.obj
 0001:000146a0       ??_C@_1M@OBGLJIPL@?$AAb?$AAe?$AA?9?$AAB?$AAY?$AA?$AA@ 00000001800156a0     libucrt:lcidtoname_downlevel.obj
 0001:000146b0       ??_C@_1M@BCFAJEAD@?$AAs?$AAl?$AA?9?$AAS?$AAI?$AA?$AA@ 00000001800156b0     libucrt:lcidtoname_downlevel.obj
 0001:000146c0       ??_C@_1M@FKFFEDDN@?$AAe?$AAt?$AA?9?$AAE?$AAE?$AA?$AA@ 00000001800156c0     libucrt:lcidtoname_downlevel.obj
 0001:000146d0       ??_C@_1M@KGKKAACI@?$AAl?$AAv?$AA?9?$AAL?$AAV?$AA?$AA@ 00000001800156d0     libucrt:lcidtoname_downlevel.obj
 0001:000146e0       ??_C@_1M@IFGBIJO@?$AAl?$AAt?$AA?9?$AAL?$AAT?$AA?$AA@ 00000001800156e0     libucrt:lcidtoname_downlevel.obj
 0001:000146f0       ??_C@_1M@FGEAHEDM@?$AAf?$AAa?$AA?9?$AAI?$AAR?$AA?$AA@ 00000001800156f0     libucrt:lcidtoname_downlevel.obj
 0001:00014700       ??_C@_1M@KBMAIBFN@?$AAv?$AAi?$AA?9?$AAV?$AAN?$AA?$AA@ 0000000180015700     libucrt:lcidtoname_downlevel.obj
 0001:00014710       ??_C@_1M@GPCBKDJK@?$AAh?$AAy?$AA?9?$AAA?$AAM?$AA?$AA@ 0000000180015710     libucrt:lcidtoname_downlevel.obj
 0001:00014720       ??_C@_1BG@BECMDDJB@?$AAa?$AAz?$AA?9?$AAA?$AAZ?$AA?9?$AAL?$AAa?$AAt?$AAn?$AA?$AA@ 0000000180015720     libucrt:lcidtoname_downlevel.obj
 0001:00014738       ??_C@_1M@MAOFCAEA@?$AAe?$AAu?$AA?9?$AAE?$AAS?$AA?$AA@ 0000000180015738     libucrt:lcidtoname_downlevel.obj
 0001:00014748       ??_C@_1M@IGHABKPI@?$AAm?$AAk?$AA?9?$AAM?$AAK?$AA?$AA@ 0000000180015748     libucrt:lcidtoname_downlevel.obj
 0001:00014758       ??_C@_1M@IAIGNEJG@?$AAt?$AAn?$AA?9?$AAZ?$AAA?$AA?$AA@ 0000000180015758     libucrt:lcidtoname_downlevel.obj
 0001:00014768       ??_C@_1M@IIJCOJFA@?$AAx?$AAh?$AA?9?$AAZ?$AAA?$AA?$AA@ 0000000180015768     libucrt:lcidtoname_downlevel.obj
 0001:00014778       ??_C@_1M@LGPJHNJH@?$AAz?$AAu?$AA?9?$AAZ?$AAA?$AA?$AA@ 0000000180015778     libucrt:lcidtoname_downlevel.obj
 0001:00014788       ??_C@_1M@HOKAOIO@?$AAa?$AAf?$AA?9?$AAZ?$AAA?$AA?$AA@ 0000000180015788     libucrt:lcidtoname_downlevel.obj
 0001:00014798       ??_C@_1M@DPCLHLIE@?$AAk?$AAa?$AA?9?$AAG?$AAE?$AA?$AA@ 0000000180015798     libucrt:lcidtoname_downlevel.obj
 0001:000147a8       ??_C@_1M@BLKMHJBI@?$AAf?$AAo?$AA?9?$AAF?$AAO?$AA?$AA@ 00000001800157a8     libucrt:lcidtoname_downlevel.obj
 0001:000147b8       ??_C@_1M@LGGJAPPB@?$AAh?$AAi?$AA?9?$AAI?$AAN?$AA?$AA@ 00000001800157b8     libucrt:lcidtoname_downlevel.obj
 0001:000147c8       ??_C@_1M@FIKPIHFE@?$AAm?$AAt?$AA?9?$AAM?$AAT?$AA?$AA@ 00000001800157c8     libucrt:lcidtoname_downlevel.obj
 0001:000147d8       ??_C@_1M@HEGGPBFA@?$AAs?$AAe?$AA?9?$AAN?$AAO?$AA?$AA@ 00000001800157d8     libucrt:lcidtoname_downlevel.obj
 0001:000147e8       ??_C@_1M@EIBJEEPA@?$AAm?$AAs?$AA?9?$AAM?$AAY?$AA?$AA@ 00000001800157e8     libucrt:lcidtoname_downlevel.obj
 0001:000147f8       ??_C@_1M@FHLBGMPP@?$AAk?$AAk?$AA?9?$AAK?$AAZ?$AA?$AA@ 00000001800157f8     libucrt:lcidtoname_downlevel.obj
 0001:00014808       ??_C@_1M@NGJJLCGI@?$AAk?$AAy?$AA?9?$AAK?$AAG?$AA?$AA@ 0000000180015808     libucrt:lcidtoname_downlevel.obj
 0001:00014818       ??_C@_1M@GIENNBFC@?$AAs?$AAw?$AA?9?$AAK?$AAE?$AA?$AA@ 0000000180015818     libucrt:lcidtoname_downlevel.obj
 0001:00014828       ??_C@_1BG@NDGMJIMJ@?$AAu?$AAz?$AA?9?$AAU?$AAZ?$AA?9?$AAL?$AAa?$AAt?$AAn?$AA?$AA@ 0000000180015828     libucrt:lcidtoname_downlevel.obj
 0001:00014840       ??_C@_1M@IDCCIHBC@?$AAt?$AAt?$AA?9?$AAR?$AAU?$AA?$AA@ 0000000180015840     libucrt:lcidtoname_downlevel.obj
 0001:00014850       ??_C@_1M@LOICPMOJ@?$AAb?$AAn?$AA?9?$AAI?$AAN?$AA?$AA@ 0000000180015850     libucrt:lcidtoname_downlevel.obj
 0001:00014860       ??_C@_1M@KPKKNEAH@?$AAp?$AAa?$AA?9?$AAI?$AAN?$AA?$AA@ 0000000180015860     libucrt:lcidtoname_downlevel.obj
 0001:00014870       ??_C@_1M@PJGPPBOG@?$AAg?$AAu?$AA?9?$AAI?$AAN?$AA?$AA@ 0000000180015870     libucrt:lcidtoname_downlevel.obj
 0001:00014880       ??_C@_1M@KMKMOPHI@?$AAt?$AAa?$AA?9?$AAI?$AAN?$AA?$AA@ 0000000180015880     libucrt:lcidtoname_downlevel.obj
 0001:00014890       ??_C@_1M@KFEHEPAC@?$AAt?$AAe?$AA?9?$AAI?$AAN?$AA?$AA@ 0000000180015890     libucrt:lcidtoname_downlevel.obj
 0001:000148a0       ??_C@_1M@CDCLMGHI@?$AAk?$AAn?$AA?9?$AAI?$AAN?$AA?$AA@ 00000001800158a0     libucrt:lcidtoname_downlevel.obj
 0001:000148b0       ??_C@_1M@MIODLDKF@?$AAm?$AAl?$AA?9?$AAI?$AAN?$AA?$AA@ 00000001800158b0     libucrt:lcidtoname_downlevel.obj
 0001:000148c0       ??_C@_1M@PBIEACPO@?$AAm?$AAr?$AA?9?$AAI?$AAN?$AA?$AA@ 00000001800158c0     libucrt:lcidtoname_downlevel.obj
 0001:000148d0       ??_C@_1M@NIDEAGPH@?$AAs?$AAa?$AA?9?$AAI?$AAN?$AA?$AA@ 00000001800158d0     libucrt:lcidtoname_downlevel.obj
 0001:000148e0       ??_C@_1M@FHIHCBIO@?$AAm?$AAn?$AA?9?$AAM?$AAN?$AA?$AA@ 00000001800158e0     libucrt:lcidtoname_downlevel.obj
 0001:000148f0       ??_C@_1M@JAIJPENP@?$AAc?$AAy?$AA?9?$AAG?$AAB?$AA?$AA@ 00000001800158f0     libucrt:lcidtoname_downlevel.obj
 0001:00014900       ??_C@_1M@PHGFBEPN@?$AAg?$AAl?$AA?9?$AAE?$AAS?$AA?$AA@ 0000000180015900     libucrt:lcidtoname_downlevel.obj
 0001:00014910       ??_C@_1O@KPIPDNCP@?$AAk?$AAo?$AAk?$AA?9?$AAI?$AAN?$AA?$AA@ 0000000180015910     libucrt:lcidtoname_downlevel.obj
 0001:00014920       ??_C@_1O@KNHJLDJA@?$AAs?$AAy?$AAr?$AA?9?$AAS?$AAY?$AA?$AA@ 0000000180015920     libucrt:lcidtoname_downlevel.obj
 0001:00014930       ??_C@_1O@MKEKBLAH@?$AAd?$AAi?$AAv?$AA?9?$AAM?$AAV?$AA?$AA@ 0000000180015930     libucrt:lcidtoname_downlevel.obj
 0001:00014940       ??_C@_1O@OHDCKDDF@?$AAq?$AAu?$AAz?$AA?9?$AAB?$AAO?$AA?$AA@ 0000000180015940     libucrt:lcidtoname_downlevel.obj
 0001:00014950       ??_C@_1M@LEPJNLFD@?$AAn?$AAs?$AA?9?$AAZ?$AAA?$AA?$AA@ 0000000180015950     libucrt:lcidtoname_downlevel.obj
 0001:00014960       ??_C@_1M@OMLEIIJB@?$AAm?$AAi?$AA?9?$AAN?$AAZ?$AA?$AA@ 0000000180015960     libucrt:lcidtoname_downlevel.obj
 0001:00014970       ??_C@_1M@PMPEAILG@?$AAa?$AAr?$AA?9?$AAI?$AAQ?$AA?$AA@ 0000000180015970     libucrt:lcidtoname_downlevel.obj
 0001:00014980       ??_C@_1M@CNKPNOEE@?$AAd?$AAe?$AA?9?$AAC?$AAH?$AA?$AA@ 0000000180015980     libucrt:lcidtoname_downlevel.obj
 0001:00014990       ??_C@_1M@LKMGMLKO@?$AAe?$AAn?$AA?9?$AAG?$AAB?$AA?$AA@ 0000000180015990     libucrt:lcidtoname_downlevel.obj
 0001:000149a0       ??_C@_1M@PGKJFFGL@?$AAe?$AAs?$AA?9?$AAM?$AAX?$AA?$AA@ 00000001800159a0     libucrt:lcidtoname_downlevel.obj
 0001:000149b0       ??_C@_1M@DNNANBDC@?$AAf?$AAr?$AA?9?$AAB?$AAE?$AA?$AA@ 00000001800159b0     libucrt:lcidtoname_downlevel.obj
 0001:000149c0       ??_C@_1M@HLGMDFHM@?$AAi?$AAt?$AA?9?$AAC?$AAH?$AA?$AA@ 00000001800159c0     libucrt:lcidtoname_downlevel.obj
 0001:000149d0       ??_C@_1M@CLLBGJH@?$AAn?$AAl?$AA?9?$AAB?$AAE?$AA?$AA@ 00000001800159d0     libucrt:lcidtoname_downlevel.obj
 0001:000149e0       ??_C@_1M@BODBOGLF@?$AAn?$AAn?$AA?9?$AAN?$AAO?$AA?$AA@ 00000001800159e0     libucrt:lcidtoname_downlevel.obj
 0001:000149f0       ??_C@_1M@HFFAHKAD@?$AAp?$AAt?$AA?9?$AAP?$AAT?$AA?$AA@ 00000001800159f0     libucrt:lcidtoname_downlevel.obj
 0001:00014a00       ??_C@_1BG@LNOAKHIE@?$AAs?$AAr?$AA?9?$AAS?$AAP?$AA?9?$AAL?$AAa?$AAt?$AAn?$AA?$AA@ 0000000180015a00     libucrt:lcidtoname_downlevel.obj
 0001:00014a18       ??_C@_1M@HBMHBGAK@?$AAs?$AAv?$AA?9?$AAF?$AAI?$AA?$AA@ 0000000180015a18     libucrt:lcidtoname_downlevel.obj
 0001:00014a28       ??_C@_1BG@DGCJGJBE@?$AAa?$AAz?$AA?9?$AAA?$AAZ?$AA?9?$AAC?$AAy?$AAr?$AAl?$AA?$AA@ 0000000180015a28     libucrt:lcidtoname_downlevel.obj
 0001:00014a40       ??_C@_1M@KEJDAAHB@?$AAs?$AAe?$AA?9?$AAS?$AAE?$AA?$AA@ 0000000180015a40     libucrt:lcidtoname_downlevel.obj
 0001:00014a50       ??_C@_1M@HEIBJJAD@?$AAm?$AAs?$AA?9?$AAB?$AAN?$AA?$AA@ 0000000180015a50     libucrt:lcidtoname_downlevel.obj
 0001:00014a60       ??_C@_1BG@PBGJMCEM@?$AAu?$AAz?$AA?9?$AAU?$AAZ?$AA?9?$AAC?$AAy?$AAr?$AAl?$AA?$AA@ 0000000180015a60     libucrt:lcidtoname_downlevel.obj
 0001:00014a78       ??_C@_1O@LAOBCMDF@?$AAq?$AAu?$AAz?$AA?9?$AAE?$AAC?$AA?$AA@ 0000000180015a78     libucrt:lcidtoname_downlevel.obj
 0001:00014a88       ??_C@_1M@POEEMAIO@?$AAa?$AAr?$AA?9?$AAE?$AAG?$AA?$AA@ 0000000180015a88     libucrt:lcidtoname_downlevel.obj
 0001:00014a98       ??_C@_1M@EFAKDEDL@?$AAz?$AAh?$AA?9?$AAH?$AAK?$AA?$AA@ 0000000180015a98     libucrt:lcidtoname_downlevel.obj
 0001:00014aa8       ??_C@_1M@HKKIJHGI@?$AAd?$AAe?$AA?9?$AAA?$AAT?$AA?$AA@ 0000000180015aa8     libucrt:lcidtoname_downlevel.obj
 0001:00014ab8       ??_C@_1M@KBFBEHJF@?$AAe?$AAn?$AA?9?$AAA?$AAU?$AA?$AA@ 0000000180015ab8     libucrt:lcidtoname_downlevel.obj
 0001:00014ac8       ??_C@_1M@MNPLFAAH@?$AAe?$AAs?$AA?9?$AAE?$AAS?$AA?$AA@ 0000000180015ac8     libucrt:lcidtoname_downlevel.obj
 0001:00014ad8       ??_C@_1M@HJOOJFMA@?$AAf?$AAr?$AA?9?$AAC?$AAA?$AA?$AA@ 0000000180015ad8     libucrt:lcidtoname_downlevel.obj
 0001:00014ae8       ??_C@_1BG@JPOFPNAB@?$AAs?$AAr?$AA?9?$AAS?$AAP?$AA?9?$AAC?$AAy?$AAr?$AAl?$AA?$AA@ 0000000180015ae8     libucrt:lcidtoname_downlevel.obj
 0001:00014b00       ??_C@_1M@LNFOCMOB@?$AAs?$AAe?$AA?9?$AAF?$AAI?$AA?$AA@ 0000000180015b00     libucrt:lcidtoname_downlevel.obj
 0001:00014b10       ??_C@_1O@MGJBOAMB@?$AAq?$AAu?$AAz?$AA?9?$AAP?$AAE?$AA?$AA@ 0000000180015b10     libucrt:lcidtoname_downlevel.obj
 0001:00014b20       ??_C@_1M@GJINLBOK@?$AAa?$AAr?$AA?9?$AAL?$AAY?$AA?$AA@ 0000000180015b20     libucrt:lcidtoname_downlevel.obj
 0001:00014b30       ??_C@_1M@GGMNHJNL@?$AAz?$AAh?$AA?9?$AAS?$AAG?$AA?$AA@ 0000000180015b30     libucrt:lcidtoname_downlevel.obj
 0001:00014b40       ??_C@_1M@HOIKODND@?$AAd?$AAe?$AA?9?$AAL?$AAU?$AA?$AA@ 0000000180015b40     libucrt:lcidtoname_downlevel.obj
 0001:00014b50       ??_C@_1M@DDOCCGFG@?$AAe?$AAn?$AA?9?$AAC?$AAA?$AA?$AA@ 0000000180015b50     libucrt:lcidtoname_downlevel.obj
 0001:00014b60       ??_C@_1M@BNOEMJLF@?$AAe?$AAs?$AA?9?$AAG?$AAT?$AA?$AA@ 0000000180015b60     libucrt:lcidtoname_downlevel.obj
 0001:00014b70       ??_C@_1M@EOGNKEK@?$AAf?$AAr?$AA?9?$AAC?$AAH?$AA?$AA@ 0000000180015b70     libucrt:lcidtoname_downlevel.obj
 0001:00014b80       ??_C@_1M@FLIDJFHL@?$AAh?$AAr?$AA?9?$AAB?$AAA?$AA?$AA@ 0000000180015b80     libucrt:lcidtoname_downlevel.obj
 0001:00014b90       ??_C@_1O@FMCELNAJ@?$AAs?$AAm?$AAj?$AA?9?$AAN?$AAO?$AA?$AA@ 0000000180015b90     libucrt:lcidtoname_downlevel.obj
 0001:00014ba0       ??_C@_1M@JHGLJMGJ@?$AAa?$AAr?$AA?9?$AAD?$AAZ?$AA?$AA@ 0000000180015ba0     libucrt:lcidtoname_downlevel.obj
 0001:00014bb0       ??_C@_1M@JKKFDCNP@?$AAz?$AAh?$AA?9?$AAM?$AAO?$AA?$AA@ 0000000180015bb0     libucrt:lcidtoname_downlevel.obj
 0001:00014bc0       ??_C@_1M@GEEFALPE@?$AAd?$AAe?$AA?9?$AAL?$AAI?$AA?$AA@ 0000000180015bc0     libucrt:lcidtoname_downlevel.obj
 0001:00014bd0       ??_C@_1M@IGEOFBG@?$AAe?$AAn?$AA?9?$AAN?$AAZ?$AA?$AA@ 0000000180015bd0     libucrt:lcidtoname_downlevel.obj
 0001:00014be0       ??_C@_1M@KDBONEHP@?$AAe?$AAs?$AA?9?$AAC?$AAR?$AA?$AA@ 0000000180015be0     libucrt:lcidtoname_downlevel.obj
 0001:00014bf0       ??_C@_1M@FHMDOHNN@?$AAf?$AAr?$AA?9?$AAL?$AAU?$AA?$AA@ 0000000180015bf0     libucrt:lcidtoname_downlevel.obj
 0001:00014c00       ??_C@_1BG@NFKKMAFG@?$AAb?$AAs?$AA?9?$AAB?$AAA?$AA?9?$AAL?$AAa?$AAt?$AAn?$AA?$AA@ 0000000180015c00     libucrt:lcidtoname_downlevel.obj
 0001:00014c18       ??_C@_1O@IMNBEMCI@?$AAs?$AAm?$AAj?$AA?9?$AAS?$AAE?$AA?$AA@ 0000000180015c18     libucrt:lcidtoname_downlevel.obj
 0001:00014c28       ??_C@_1M@DHHMBNDP@?$AAa?$AAr?$AA?9?$AAM?$AAA?$AA?$AA@ 0000000180015c28     libucrt:lcidtoname_downlevel.obj
 0001:00014c38       ??_C@_1M@BNBLJCGH@?$AAe?$AAn?$AA?9?$AAI?$AAE?$AA?$AA@ 0000000180015c38     libucrt:lcidtoname_downlevel.obj
 0001:00014c48       ??_C@_1M@GEPAFMDL@?$AAe?$AAs?$AA?9?$AAP?$AAA?$AA?$AA@ 0000000180015c48     libucrt:lcidtoname_downlevel.obj
 0001:00014c58       ??_C@_1M@OJONDMDL@?$AAf?$AAr?$AA?9?$AAM?$AAC?$AA?$AA@ 0000000180015c58     libucrt:lcidtoname_downlevel.obj
 0001:00014c68       ??_C@_1BG@OBCNFJB@?$AAs?$AAr?$AA?9?$AAB?$AAA?$AA?9?$AAL?$AAa?$AAt?$AAn?$AA?$AA@ 0000000180015c68     libucrt:lcidtoname_downlevel.obj
 0001:00014c80       ??_C@_1O@KEMEEGPO@?$AAs?$AAm?$AAa?$AA?9?$AAN?$AAO?$AA?$AA@ 0000000180015c80     libucrt:lcidtoname_downlevel.obj
 0001:00014c90       ??_C@_1M@ELMGFODK@?$AAa?$AAr?$AA?9?$AAT?$AAN?$AA?$AA@ 0000000180015c90     libucrt:lcidtoname_downlevel.obj
 0001:00014ca0       ??_C@_1M@BHDLHFAF@?$AAe?$AAn?$AA?9?$AAZ?$AAA?$AA?$AA@ 0000000180015ca0     libucrt:lcidtoname_downlevel.obj
 0001:00014cb0       ??_C@_1M@BMGIGLIF@?$AAe?$AAs?$AA?9?$AAD?$AAO?$AA?$AA@ 0000000180015cb0     libucrt:lcidtoname_downlevel.obj
 0001:00014cc0       ??_C@_1BG@CMBHIPBE@?$AAs?$AAr?$AA?9?$AAB?$AAA?$AA?9?$AAC?$AAy?$AAr?$AAl?$AA?$AA@ 0000000180015cc0     libucrt:lcidtoname_downlevel.obj
 0001:00014cd8       ??_C@_1O@HEDBLHNP@?$AAs?$AAm?$AAa?$AA?9?$AAS?$AAE?$AA?$AA@ 0000000180015cd8     libucrt:lcidtoname_downlevel.obj
 0001:00014ce8       ??_C@_1M@DAGCADIM@?$AAa?$AAr?$AA?9?$AAO?$AAM?$AA?$AA@ 0000000180015ce8     libucrt:lcidtoname_downlevel.obj
 0001:00014cf8       ??_C@_1M@FODLMICG@?$AAe?$AAn?$AA?9?$AAJ?$AAM?$AA?$AA@ 0000000180015cf8     libucrt:lcidtoname_downlevel.obj
 0001:00014d08       ??_C@_1M@DNMLCIHB@?$AAe?$AAs?$AA?9?$AAV?$AAE?$AA?$AA@ 0000000180015d08     libucrt:lcidtoname_downlevel.obj
 0001:00014d18       ??_C@_1O@EOKHMKJK@?$AAs?$AAm?$AAs?$AA?9?$AAF?$AAI?$AA?$AA@ 0000000180015d18     libucrt:lcidtoname_downlevel.obj
 0001:00014d28       ??_C@_1M@CAFJMKOF@?$AAa?$AAr?$AA?9?$AAY?$AAE?$AA?$AA@ 0000000180015d28     libucrt:lcidtoname_downlevel.obj
 0001:00014d38       ??_C@_1M@CBFHIJLI@?$AAe?$AAn?$AA?9?$AAC?$AAB?$AA?$AA@ 0000000180015d38     libucrt:lcidtoname_downlevel.obj
 0001:00014d48       ??_C@_1M@BGNFLDN@?$AAe?$AAs?$AA?9?$AAC?$AAO?$AA?$AA@ 0000000180015d48     libucrt:lcidtoname_downlevel.obj
 0001:00014d58       ??_C@_1O@JMPHMAMC@?$AAs?$AAm?$AAn?$AA?9?$AAF?$AAI?$AA?$AA@ 0000000180015d58     libucrt:lcidtoname_downlevel.obj
 0001:00014d68       ??_C@_1M@JLANABKE@?$AAa?$AAr?$AA?9?$AAS?$AAY?$AA?$AA@ 0000000180015d68     libucrt:lcidtoname_downlevel.obj
 0001:00014d78       ??_C@_1M@HPKGCFGN@?$AAe?$AAn?$AA?9?$AAB?$AAZ?$AA?$AA@ 0000000180015d78     libucrt:lcidtoname_downlevel.obj
 0001:00014d88       ??_C@_1M@OLJCMLGM@?$AAe?$AAs?$AA?9?$AAP?$AAE?$AA?$AA@ 0000000180015d88     libucrt:lcidtoname_downlevel.obj
 0001:00014d98       ??_C@_1M@MKKGFKLE@?$AAa?$AAr?$AA?9?$AAJ?$AAO?$AA?$AA@ 0000000180015d98     libucrt:lcidtoname_downlevel.obj
 0001:00014da8       ??_C@_1M@EKPGLDNI@?$AAe?$AAn?$AA?9?$AAT?$AAT?$AA?$AA@ 0000000180015da8     libucrt:lcidtoname_downlevel.obj
 0001:00014db8       ??_C@_1M@OONGHFHE@?$AAe?$AAs?$AA?9?$AAA?$AAR?$AA?$AA@ 0000000180015db8     libucrt:lcidtoname_downlevel.obj
 0001:00014dc8       ??_C@_1M@OOJFGBHE@?$AAa?$AAr?$AA?9?$AAL?$AAB?$AA?$AA@ 0000000180015dc8     libucrt:lcidtoname_downlevel.obj
 0001:00014dd8       ??_C@_1M@GCEJHNEG@?$AAe?$AAn?$AA?9?$AAZ?$AAW?$AA?$AA@ 0000000180015dd8     libucrt:lcidtoname_downlevel.obj
 0001:00014de8       ??_C@_1M@JNOCAHJI@?$AAe?$AAs?$AA?9?$AAE?$AAC?$AA?$AA@ 0000000180015de8     libucrt:lcidtoname_downlevel.obj
 0001:00014df8       ??_C@_1M@JEFHPGGB@?$AAa?$AAr?$AA?9?$AAK?$AAW?$AA?$AA@ 0000000180015df8     libucrt:lcidtoname_downlevel.obj
 0001:00014e08       ??_C@_1M@MLKIBJOJ@?$AAe?$AAn?$AA?9?$AAP?$AAH?$AA?$AA@ 0000000180015e08     libucrt:lcidtoname_downlevel.obj
 0001:00014e18       ??_C@_1M@BDNIPEND@?$AAe?$AAs?$AA?9?$AAC?$AAL?$AA?$AA@ 0000000180015e18     libucrt:lcidtoname_downlevel.obj
 0001:00014e28       ??_C@_1M@MPNMEKBD@?$AAa?$AAr?$AA?9?$AAA?$AAE?$AA?$AA@ 0000000180015e28     libucrt:lcidtoname_downlevel.obj
 0001:00014e38       ??_C@_1M@KBJALCPI@?$AAe?$AAs?$AA?9?$AAU?$AAY?$AA?$AA@ 0000000180015e38     libucrt:lcidtoname_downlevel.obj
 0001:00014e48       ??_C@_1M@LLCCOAGA@?$AAa?$AAr?$AA?9?$AAB?$AAH?$AA?$AA@ 0000000180015e48     libucrt:lcidtoname_downlevel.obj
 0001:00014e58       ??_C@_1M@PBFNCDEL@?$AAe?$AAs?$AA?9?$AAP?$AAY?$AA?$AA@ 0000000180015e58     libucrt:lcidtoname_downlevel.obj
 0001:00014e68       ??_C@_1M@EDGINPNP@?$AAa?$AAr?$AA?9?$AAQ?$AAA?$AA?$AA@ 0000000180015e68     libucrt:lcidtoname_downlevel.obj
 0001:00014e78       ??_C@_1M@MKDBIIJI@?$AAe?$AAs?$AA?9?$AAB?$AAO?$AA?$AA@ 0000000180015e78     libucrt:lcidtoname_downlevel.obj
 0001:00014e88       ??_C@_1M@CPKKEBLD@?$AAe?$AAs?$AA?9?$AAS?$AAV?$AA?$AA@ 0000000180015e88     libucrt:lcidtoname_downlevel.obj
 0001:00014e98       ??_C@_1M@NDBGMMJL@?$AAe?$AAs?$AA?9?$AAH?$AAN?$AA?$AA@ 0000000180015e98     libucrt:lcidtoname_downlevel.obj
 0001:00014ea8       ??_C@_1M@JIJIBHDP@?$AAe?$AAs?$AA?9?$AAN?$AAI?$AA?$AA@ 0000000180015ea8     libucrt:lcidtoname_downlevel.obj
 0001:00014eb8       ??_C@_1M@CGFMKEEK@?$AAe?$AAs?$AA?9?$AAP?$AAR?$AA?$AA@ 0000000180015eb8     libucrt:lcidtoname_downlevel.obj
 0001:00014ec8       ??_C@_1O@ICJHKIIK@?$AAz?$AAh?$AA?9?$AAC?$AAH?$AAT?$AA?$AA@ 0000000180015ec8     libucrt:lcidtoname_downlevel.obj
 0001:00014ed8       ??_C@_15CLNEJCE@?$AAs?$AAr?$AA?$AA@ 0000000180015ed8     libucrt:lcidtoname_downlevel.obj
 0001:00015d20       ??_C@_1M@KAHEKEIG@?$AAa?$AAf?$AA?9?$AAz?$AAa?$AA?$AA@ 0000000180016d20     libucrt:lcidtoname_downlevel.obj
 0001:00015d30       ??_C@_1M@GIECOABL@?$AAa?$AAr?$AA?9?$AAa?$AAe?$AA?$AA@ 0000000180016d30     libucrt:lcidtoname_downlevel.obj
 0001:00015d40       ??_C@_1M@BMLMEKGI@?$AAa?$AAr?$AA?9?$AAb?$AAh?$AA?$AA@ 0000000180016d40     libucrt:lcidtoname_downlevel.obj
 0001:00015d50       ??_C@_1M@DAPFDGGB@?$AAa?$AAr?$AA?9?$AAd?$AAz?$AA?$AA@ 0000000180016d50     libucrt:lcidtoname_downlevel.obj
 0001:00015d60       ??_C@_1M@FJNKGKIG@?$AAa?$AAr?$AA?9?$AAe?$AAg?$AA?$AA@ 0000000180016d60     libucrt:lcidtoname_downlevel.obj
 0001:00015d70       ??_C@_1M@FLGKKCLO@?$AAa?$AAr?$AA?9?$AAi?$AAq?$AA?$AA@ 0000000180016d70     libucrt:lcidtoname_downlevel.obj
 0001:00015d80       ??_C@_1M@GNDIPALM@?$AAa?$AAr?$AA?9?$AAj?$AAo?$AA?$AA@ 0000000180016d80     libucrt:lcidtoname_downlevel.obj
 0001:00015d90       ??_C@_1M@DDMJFMGJ@?$AAa?$AAr?$AA?9?$AAk?$AAw?$AA?$AA@ 0000000180016d90     libucrt:lcidtoname_downlevel.obj
 0001:00015da0       ??_C@_1M@EJALMLHM@?$AAa?$AAr?$AA?9?$AAl?$AAb?$AA?$AA@ 0000000180016da0     libucrt:lcidtoname_downlevel.obj
 0001:00015db0       ??_C@_1M@MOBDBLOC@?$AAa?$AAr?$AA?9?$AAl?$AAy?$AA?$AA@ 0000000180016db0     libucrt:lcidtoname_downlevel.obj
 0001:00015dc0       ??_C@_1M@JAOCLHDH@?$AAa?$AAr?$AA?9?$AAm?$AAa?$AA?$AA@ 0000000180016dc0     libucrt:lcidtoname_downlevel.obj
 0001:00015dd0       ??_C@_1M@JHPMKJIE@?$AAa?$AAr?$AA?9?$AAo?$AAm?$AA?$AA@ 0000000180016dd0     libucrt:lcidtoname_downlevel.obj
 0001:00015de0       ??_C@_1M@OEPGHFNH@?$AAa?$AAr?$AA?9?$AAq?$AAa?$AA?$AA@ 0000000180016de0     libucrt:lcidtoname_downlevel.obj
 0001:00015df0       ??_C@_1M@KJDONENM@?$AAa?$AAr?$AA?9?$AAs?$AAa?$AA?$AA@ 0000000180016df0     libucrt:lcidtoname_downlevel.obj
 0001:00015e00       ??_C@_1M@DMJDKLKM@?$AAa?$AAr?$AA?9?$AAs?$AAy?$AA?$AA@ 0000000180016e00     libucrt:lcidtoname_downlevel.obj
 0001:00015e10       ??_C@_1M@OMFIPEDC@?$AAa?$AAr?$AA?9?$AAt?$AAn?$AA?$AA@ 0000000180016e10     libucrt:lcidtoname_downlevel.obj
 0001:00015e20       ??_C@_1M@IHMHGAON@?$AAa?$AAr?$AA?9?$AAy?$AAe?$AA?$AA@ 0000000180016e20     libucrt:lcidtoname_downlevel.obj
 0001:00015e30       ??_C@_1BG@KDCPGJGB@?$AAa?$AAz?$AA?9?$AAa?$AAz?$AA?9?$AAc?$AAy?$AAr?$AAl?$AA?$AA@ 0000000180016e30     libucrt:lcidtoname_downlevel.obj
 0001:00015e48       ??_C@_1BG@IBCKDDOE@?$AAa?$AAz?$AA?9?$AAa?$AAz?$AA?9?$AAl?$AAa?$AAt?$AAn?$AA?$AA@ 0000000180016e48     libucrt:lcidtoname_downlevel.obj
 0001:00015e60       ??_C@_1M@EGPFDCPD@?$AAb?$AAe?$AA?9?$AAb?$AAy?$AA?$AA@ 0000000180016e60     libucrt:lcidtoname_downlevel.obj
 0001:00015e70       ??_C@_1M@PCMGMCGC@?$AAb?$AAg?$AA?9?$AAb?$AAg?$AA?$AA@ 0000000180016e70     libucrt:lcidtoname_downlevel.obj
 0001:00015e80       ??_C@_1M@BJBMFGOB@?$AAb?$AAn?$AA?9?$AAi?$AAn?$AA?$AA@ 0000000180016e80     libucrt:lcidtoname_downlevel.obj
 0001:00015e90       ??_C@_1BG@EAKMMACD@?$AAb?$AAs?$AA?9?$AAb?$AAa?$AA?9?$AAl?$AAa?$AAt?$AAn?$AA?$AA@ 0000000180016e90     libucrt:lcidtoname_downlevel.obj
 0001:00015ea8       ??_C@_1M@KGADAODK@?$AAc?$AAa?$AA?9?$AAe?$AAs?$AA?$AA@ 0000000180016ea8     libucrt:lcidtoname_downlevel.obj
 0001:00015eb8       ??_C@_1M@COAJPDHI@?$AAc?$AAs?$AA?9?$AAc?$AAz?$AA?$AA@ 0000000180016eb8     libucrt:lcidtoname_downlevel.obj
 0001:00015ec8       ??_C@_1M@DHBHFONH@?$AAc?$AAy?$AA?9?$AAg?$AAb?$AA?$AA@ 0000000180016ec8     libucrt:lcidtoname_downlevel.obj
 0001:00015ed8       ??_C@_1M@IMGKELGA@?$AAd?$AAa?$AA?9?$AAd?$AAk?$AA?$AA@ 0000000180016ed8     libucrt:lcidtoname_downlevel.obj
 0001:00015ee8       ??_C@_1M@NNDGDNGA@?$AAd?$AAe?$AA?9?$AAa?$AAt?$AA?$AA@ 0000000180016ee8     libucrt:lcidtoname_downlevel.obj
 0001:00015ef8       ??_C@_1M@IKDBHEEM@?$AAd?$AAe?$AA?9?$AAc?$AAh?$AA?$AA@ 0000000180016ef8     libucrt:lcidtoname_downlevel.obj
 0001:00015f08       ??_C@_1M@GFFOJMCJ@?$AAd?$AAe?$AA?9?$AAd?$AAe?$AA?$AA@ 0000000180016f08     libucrt:lcidtoname_downlevel.obj
 0001:00015f18       ??_C@_1M@MDNLKBPM@?$AAd?$AAe?$AA?9?$AAl?$AAi?$AA?$AA@ 0000000180016f18     libucrt:lcidtoname_downlevel.obj
 0001:00015f28       ??_C@_1M@NJBEEJNL@?$AAd?$AAe?$AA?9?$AAl?$AAu?$AA?$AA@ 0000000180016f28     libucrt:lcidtoname_downlevel.obj
 0001:00015f38       ??_C@_1O@GNNELBAP@?$AAd?$AAi?$AAv?$AA?9?$AAm?$AAv?$AA?$AA@ 0000000180016f38     libucrt:lcidtoname_downlevel.obj
 0001:00015f48       ??_C@_1M@EJLEOGAE@?$AAe?$AAl?$AA?9?$AAg?$AAr?$AA?$AA@ 0000000180016f48     libucrt:lcidtoname_downlevel.obj
 0001:00015f58       ??_C@_1M@GMPONJN@?$AAe?$AAn?$AA?9?$AAa?$AAu?$AA?$AA@ 0000000180016f58     libucrt:lcidtoname_downlevel.obj
 0001:00015f68       ??_C@_1M@NIDIIPGF@?$AAe?$AAn?$AA?9?$AAb?$AAz?$AA?$AA@ 0000000180016f68     libucrt:lcidtoname_downlevel.obj
 0001:00015f78       ??_C@_1M@JEHMIMFO@?$AAe?$AAn?$AA?9?$AAc?$AAa?$AA?$AA@ 0000000180016f78     libucrt:lcidtoname_downlevel.obj
 0001:00015f88       ??_C@_1M@IGMJCDLA@?$AAe?$AAn?$AA?9?$AAc?$AAb?$AA?$AA@ 0000000180016f88     libucrt:lcidtoname_downlevel.obj
 0001:00015f98       ??_C@_1M@BNFIGBKG@?$AAe?$AAn?$AA?9?$AAg?$AAb?$AA?$AA@ 0000000180016f98     libucrt:lcidtoname_downlevel.obj
 0001:00015fa8       ??_C@_1M@LKIFDIGP@?$AAe?$AAn?$AA?9?$AAi?$AAe?$AA?$AA@ 0000000180016fa8     libucrt:lcidtoname_downlevel.obj
 0001:00015fb8       ??_C@_1M@PJKFGCCO@?$AAe?$AAn?$AA?9?$AAj?$AAm?$AA?$AA@ 0000000180016fb8     libucrt:lcidtoname_downlevel.obj
 0001:00015fc8       ??_C@_1M@KPPKEPBO@?$AAe?$AAn?$AA?9?$AAn?$AAz?$AA?$AA@ 0000000180016fc8     libucrt:lcidtoname_downlevel.obj
 0001:00015fd8       ??_C@_1M@GMDGLDOB@?$AAe?$AAn?$AA?9?$AAp?$AAh?$AA?$AA@ 0000000180016fd8     libucrt:lcidtoname_downlevel.obj
 0001:00015fe8       ??_C@_1M@ONGIBJNA@?$AAe?$AAn?$AA?9?$AAt?$AAt?$AA?$AA@ 0000000180016fe8     libucrt:lcidtoname_downlevel.obj
 0001:00015ff8       ??_C@_1M@LLODPCMM@?$AAe?$AAn?$AA?9?$AAu?$AAs?$AA?$AA@ 0000000180016ff8     libucrt:lcidtoname_downlevel.obj
 0001:00016008       ??_C@_1M@LAKFNPAN@?$AAe?$AAn?$AA?9?$AAz?$AAa?$AA?$AA@ 0000000180017008     libucrt:lcidtoname_downlevel.obj
 0001:00016018       ??_C@_1M@MFNHNHEO@?$AAe?$AAn?$AA?9?$AAz?$AAw?$AA?$AA@ 0000000180017018     libucrt:lcidtoname_downlevel.obj
 0001:00016028       ??_C@_1M@EJEINPHM@?$AAe?$AAs?$AA?9?$AAa?$AAr?$AA?$AA@ 0000000180017028     libucrt:lcidtoname_downlevel.obj
 0001:00016038       ??_C@_1M@GNKPCCJA@?$AAe?$AAs?$AA?9?$AAb?$AAo?$AA?$AA@ 0000000180017038     libucrt:lcidtoname_downlevel.obj
 0001:00016048       ??_C@_1M@LEEGFONL@?$AAe?$AAs?$AA?9?$AAc?$AAl?$AA?$AA@ 0000000180017048     libucrt:lcidtoname_downlevel.obj
 0001:00016058       ??_C@_1M@KGPDPBDF@?$AAe?$AAs?$AA?9?$AAc?$AAo?$AA?$AA@ 0000000180017058     libucrt:lcidtoname_downlevel.obj
 0001:00016068       ??_C@_1M@EIAHOHH@?$AAe?$AAs?$AA?9?$AAc?$AAr?$AA?$AA@ 0000000180017068     libucrt:lcidtoname_downlevel.obj
 0001:00016078       ??_C@_1M@LLPGMBIN@?$AAe?$AAs?$AA?9?$AAd?$AAo?$AA?$AA@ 0000000180017078     libucrt:lcidtoname_downlevel.obj
 0001:00016088       ??_C@_1M@DKHMKNJA@?$AAe?$AAs?$AA?9?$AAe?$AAc?$AA?$AA@ 0000000180017088     libucrt:lcidtoname_downlevel.obj
 0001:00016098       ??_C@_1M@GKGFPKAP@?$AAe?$AAs?$AA?9?$AAe?$AAs?$AA?$AA@ 0000000180017098     libucrt:lcidtoname_downlevel.obj
 0001:000160a8       ??_C@_1M@LKHKGDLN@?$AAe?$AAs?$AA?9?$AAg?$AAt?$AA?$AA@ 00000001800170a8     libucrt:lcidtoname_downlevel.obj
 0001:000160b8       ??_C@_1M@HEIIGGJD@?$AAe?$AAs?$AA?9?$AAh?$AAn?$AA?$AA@ 00000001800170b8     libucrt:lcidtoname_downlevel.obj
 0001:000160c8       ??_C@_1M@FBDHPPGD@?$AAe?$AAs?$AA?9?$AAm?$AAx?$AA?$AA@ 00000001800170c8     libucrt:lcidtoname_downlevel.obj
 0001:000160d8       ??_C@_1M@DPAGLNDH@?$AAe?$AAs?$AA?9?$AAn?$AAi?$AA?$AA@ 00000001800170d8     libucrt:lcidtoname_downlevel.obj
 0001:000160e8       ??_C@_1M@MDGOPGDD@?$AAe?$AAs?$AA?9?$AAp?$AAa?$AA?$AA@ 00000001800170e8     libucrt:lcidtoname_downlevel.obj
 0001:000160f8       ??_C@_1M@EMAMGBGE@?$AAe?$AAs?$AA?9?$AAp?$AAe?$AA?$AA@ 00000001800170f8     libucrt:lcidtoname_downlevel.obj
 0001:00016108       ??_C@_1M@IBMCAOEC@?$AAe?$AAs?$AA?9?$AAp?$AAr?$AA?$AA@ 0000000180017108     libucrt:lcidtoname_downlevel.obj
 0001:00016118       ??_C@_1M@FGMDIJED@?$AAe?$AAs?$AA?9?$AAp?$AAy?$AA?$AA@ 0000000180017118     libucrt:lcidtoname_downlevel.obj
 0001:00016128       ??_C@_1M@IIDEOLLL@?$AAe?$AAs?$AA?9?$AAs?$AAv?$AA?$AA@ 0000000180017128     libucrt:lcidtoname_downlevel.obj
 0001:00016138       ??_C@_1M@GAOBIPA@?$AAe?$AAs?$AA?9?$AAu?$AAy?$AA?$AA@ 0000000180017138     libucrt:lcidtoname_downlevel.obj
 0001:00016148       ??_C@_1M@JKFFICHJ@?$AAe?$AAs?$AA?9?$AAv?$AAe?$AA?$AA@ 0000000180017148     libucrt:lcidtoname_downlevel.obj
 0001:00016158       ??_C@_1M@PNMLOJDF@?$AAe?$AAt?$AA?9?$AAe?$AAe?$AA?$AA@ 0000000180017158     libucrt:lcidtoname_downlevel.obj
 0001:00016168       ??_C@_1M@GHHLIKEI@?$AAe?$AAu?$AA?9?$AAe?$AAs?$AA?$AA@ 0000000180017168     libucrt:lcidtoname_downlevel.obj
 0001:00016178       ??_C@_1M@PBNONODE@?$AAf?$AAa?$AA?9?$AAi?$AAr?$AA?$AA@ 0000000180017178     libucrt:lcidtoname_downlevel.obj
 0001:00016188       ??_C@_1M@JEEHPMIL@?$AAf?$AAi?$AA?9?$AAf?$AAi?$AA?$AA@ 0000000180017188     libucrt:lcidtoname_downlevel.obj
 0001:00016198       ??_C@_1M@LMDCNDBA@?$AAf?$AAo?$AA?9?$AAf?$AAo?$AA?$AA@ 0000000180017198     libucrt:lcidtoname_downlevel.obj
 0001:000161a8       ??_C@_1M@JKEOHLDK@?$AAf?$AAr?$AA?9?$AAb?$AAe?$AA?$AA@ 00000001800171a8     libucrt:lcidtoname_downlevel.obj
 0001:000161b8       ??_C@_1M@NOHADPMI@?$AAf?$AAr?$AA?9?$AAc?$AAa?$AA?$AA@ 00000001800171b8     libucrt:lcidtoname_downlevel.obj
 0001:000161c8       ??_C@_1M@KDHIHAEC@?$AAf?$AAr?$AA?9?$AAc?$AAh?$AA?$AA@ 00000001800171c8     libucrt:lcidtoname_downlevel.obj
 0001:000161d8       ??_C@_1M@MMBBFGAK@?$AAf?$AAr?$AA?9?$AAf?$AAr?$AA?$AA@ 00000001800171d8     libucrt:lcidtoname_downlevel.obj
 0001:000161e8       ??_C@_1M@PAFNENNF@?$AAf?$AAr?$AA?9?$AAl?$AAu?$AA?$AA@ 00000001800171e8     libucrt:lcidtoname_downlevel.obj
 0001:000161f8       ??_C@_1M@EOHDJGDD@?$AAf?$AAr?$AA?9?$AAm?$AAc?$AA?$AA@ 00000001800171f8     libucrt:lcidtoname_downlevel.obj
 0001:00016208       ??_C@_1M@FAPLLOPF@?$AAg?$AAl?$AA?9?$AAe?$AAs?$AA?$AA@ 0000000180017208     libucrt:lcidtoname_downlevel.obj
 0001:00016218       ??_C@_1M@FOPBFLOO@?$AAg?$AAu?$AA?9?$AAi?$AAn?$AA?$AA@ 0000000180017218     libucrt:lcidtoname_downlevel.obj
 0001:00016228       ??_C@_1M@KBMCINPM@?$AAh?$AAe?$AA?9?$AAi?$AAl?$AA?$AA@ 0000000180017228     libucrt:lcidtoname_downlevel.obj
 0001:00016238       ??_C@_1M@BBPHKFPJ@?$AAh?$AAi?$AA?9?$AAi?$AAn?$AA?$AA@ 0000000180017238     libucrt:lcidtoname_downlevel.obj
 0001:00016248       ??_C@_1M@PMBNDPHD@?$AAh?$AAr?$AA?9?$AAb?$AAa?$AA?$AA@ 0000000180017248     libucrt:lcidtoname_downlevel.obj
 0001:00016258       ??_C@_1M@BPCKOEGE@?$AAh?$AAr?$AA?9?$AAh?$AAr?$AA?$AA@ 0000000180017258     libucrt:lcidtoname_downlevel.obj
 0001:00016268       ??_C@_1M@GACBMHKE@?$AAh?$AAu?$AA?9?$AAh?$AAu?$AA?$AA@ 0000000180017268     libucrt:lcidtoname_downlevel.obj
 0001:00016278       ??_C@_1M@MILPAJJC@?$AAh?$AAy?$AA?9?$AAa?$AAm?$AA?$AA@ 0000000180017278     libucrt:lcidtoname_downlevel.obj
 0001:00016288       ??_C@_1M@BABBICEC@?$AAi?$AAd?$AA?9?$AAi?$AAd?$AA?$AA@ 0000000180017288     libucrt:lcidtoname_downlevel.obj
 0001:00016298       ??_C@_1M@BIKNHHPF@?$AAi?$AAs?$AA?9?$AAi?$AAs?$AA?$AA@ 0000000180017298     libucrt:lcidtoname_downlevel.obj
 0001:000162a8       ??_C@_1M@NMPCJPHE@?$AAi?$AAt?$AA?9?$AAc?$AAh?$AA?$AA@ 00000001800172a8     libucrt:lcidtoname_downlevel.obj
 0001:000162b8       ??_C@_1M@GHKGFEDF@?$AAi?$AAt?$AA?9?$AAi?$AAt?$AA?$AA@ 00000001800172b8     libucrt:lcidtoname_downlevel.obj
 0001:000162c8       ??_C@_1M@NIEJCJJA@?$AAj?$AAa?$AA?9?$AAj?$AAp?$AA?$AA@ 00000001800172c8     libucrt:lcidtoname_downlevel.obj
 0001:000162d8       ??_C@_1M@JILFNBIM@?$AAk?$AAa?$AA?9?$AAg?$AAe?$AA?$AA@ 00000001800172d8     libucrt:lcidtoname_downlevel.obj
 0001:000162e8       ??_C@_1M@PACPMGPH@?$AAk?$AAk?$AA?9?$AAk?$AAz?$AA?$AA@ 00000001800172e8     libucrt:lcidtoname_downlevel.obj
 0001:000162f8       ??_C@_1M@IELFGMHA@?$AAk?$AAn?$AA?9?$AAi?$AAn?$AA?$AA@ 00000001800172f8     libucrt:lcidtoname_downlevel.obj
 0001:00016308       ??_C@_1O@IBBJHCH@?$AAk?$AAo?$AAk?$AA?9?$AAi?$AAn?$AA?$AA@ 0000000180017308     libucrt:lcidtoname_downlevel.obj
 0001:00016318       ??_C@_1M@DMHAEOGC@?$AAk?$AAo?$AA?9?$AAk?$AAr?$AA?$AA@ 0000000180017318     libucrt:lcidtoname_downlevel.obj
 0001:00016328       ??_C@_1M@HBAHBIGA@?$AAk?$AAy?$AA?9?$AAk?$AAg?$AA?$AA@ 0000000180017328     libucrt:lcidtoname_downlevel.obj
 0001:00016338       ??_C@_1M@KPMILCJG@?$AAl?$AAt?$AA?9?$AAl?$AAt?$AA?$AA@ 0000000180017338     libucrt:lcidtoname_downlevel.obj
 0001:00016348       ??_C@_1M@BDEKKCA@?$AAl?$AAv?$AA?9?$AAl?$AAv?$AA?$AA@ 0000000180017348     libucrt:lcidtoname_downlevel.obj
 0001:00016358       ??_C@_1M@ELCKCCJJ@?$AAm?$AAi?$AA?9?$AAn?$AAz?$AA?$AA@ 0000000180017358     libucrt:lcidtoname_downlevel.obj
 0001:00016368       ??_C@_1M@CBOOLAPA@?$AAm?$AAk?$AA?9?$AAm?$AAk?$AA?$AA@ 0000000180017368     libucrt:lcidtoname_downlevel.obj
 0001:00016378       ??_C@_1M@GPHNBJKN@?$AAm?$AAl?$AA?9?$AAi?$AAn?$AA?$AA@ 0000000180017378     libucrt:lcidtoname_downlevel.obj
 0001:00016388       ??_C@_1M@PABJILIG@?$AAm?$AAn?$AA?9?$AAm?$AAn?$AA?$AA@ 0000000180017388     libucrt:lcidtoname_downlevel.obj
 0001:00016398       ??_C@_1M@FGBKKIPG@?$AAm?$AAr?$AA?9?$AAi?$AAn?$AA?$AA@ 0000000180017398     libucrt:lcidtoname_downlevel.obj
 0001:000163a8       ??_C@_1M@NDBPDDAL@?$AAm?$AAs?$AA?9?$AAb?$AAn?$AA?$AA@ 00000001800173a8     libucrt:lcidtoname_downlevel.obj
 0001:000163b8       ??_C@_1M@OPIHOOPI@?$AAm?$AAs?$AA?9?$AAm?$AAy?$AA?$AA@ 00000001800173b8     libucrt:lcidtoname_downlevel.obj
 0001:000163c8       ??_C@_1M@PPDBCNFM@?$AAm?$AAt?$AA?9?$AAm?$AAt?$AA?$AA@ 00000001800173c8     libucrt:lcidtoname_downlevel.obj
 0001:000163d8       ??_C@_1M@KDJDKMDD@?$AAn?$AAb?$AA?9?$AAn?$AAo?$AA?$AA@ 00000001800173d8     libucrt:lcidtoname_downlevel.obj
 0001:000163e8       ??_C@_1M@KFCFLMJP@?$AAn?$AAl?$AA?9?$AAb?$AAe?$AA?$AA@ 00000001800173e8     libucrt:lcidtoname_downlevel.obj
 0001:000163f8       ??_C@_1M@KPOPDDGO@?$AAn?$AAl?$AA?9?$AAn?$AAl?$AA?$AA@ 00000001800173f8     libucrt:lcidtoname_downlevel.obj
 0001:00016408       ??_C@_1M@LJKPEMLN@?$AAn?$AAn?$AA?9?$AAn?$AAo?$AA?$AA@ 0000000180017408     libucrt:lcidtoname_downlevel.obj
 0001:00016418       ??_C@_1M@BDGHHBFL@?$AAn?$AAs?$AA?9?$AAz?$AAa?$AA?$AA@ 0000000180017418     libucrt:lcidtoname_downlevel.obj
 0001:00016428       ??_C@_1M@IDEHOAP@?$AAp?$AAa?$AA?9?$AAi?$AAn?$AA?$AA@ 0000000180017428     libucrt:lcidtoname_downlevel.obj
 0001:00016438       ??_C@_1M@HDBKGOGH@?$AAp?$AAl?$AA?9?$AAp?$AAl?$AA?$AA@ 0000000180017438     libucrt:lcidtoname_downlevel.obj
 0001:00016448       ??_C@_1M@LJLLCMEH@?$AAp?$AAt?$AA?9?$AAb?$AAr?$AA?$AA@ 0000000180017448     libucrt:lcidtoname_downlevel.obj
 0001:00016458       ??_C@_1M@NCMONAAL@?$AAp?$AAt?$AA?9?$AAp?$AAt?$AA?$AA@ 0000000180017458     libucrt:lcidtoname_downlevel.obj
 0001:00016468       ??_C@_1O@EAKMAJDN@?$AAq?$AAu?$AAz?$AA?9?$AAb?$AAo?$AA?$AA@ 0000000180017468     libucrt:lcidtoname_downlevel.obj
 0001:00016478       ??_C@_1O@BHHPIGDN@?$AAq?$AAu?$AAz?$AA?9?$AAe?$AAc?$AA?$AA@ 0000000180017478     libucrt:lcidtoname_downlevel.obj
 0001:00016488       ??_C@_1O@GBAPEKMJ@?$AAq?$AAu?$AAz?$AA?9?$AAp?$AAe?$AA?$AA@ 0000000180017488     libucrt:lcidtoname_downlevel.obj
 0001:00016498       ??_C@_1M@CLGLEFBO@?$AAr?$AAo?$AA?9?$AAr?$AAo?$AA?$AA@ 0000000180017498     libucrt:lcidtoname_downlevel.obj
 0001:000164a8       ??_C@_1M@CEEDODME@?$AAr?$AAu?$AA?9?$AAr?$AAu?$AA?$AA@ 00000001800174a8     libucrt:lcidtoname_downlevel.obj
 0001:000164b8       ??_C@_1M@HPKKKMPP@?$AAs?$AAa?$AA?9?$AAi?$AAn?$AA?$AA@ 00000001800174b8     libucrt:lcidtoname_downlevel.obj
 0001:000164c8       ??_C@_1M@BKMAIGOJ@?$AAs?$AAe?$AA?9?$AAf?$AAi?$AA?$AA@ 00000001800174c8     libucrt:lcidtoname_downlevel.obj
 0001:000164d8       ??_C@_1M@NDPIFLFI@?$AAs?$AAe?$AA?9?$AAn?$AAo?$AA?$AA@ 00000001800174d8     libucrt:lcidtoname_downlevel.obj
 0001:000164e8       ??_C@_1M@DANKKHJ@?$AAs?$AAe?$AA?9?$AAs?$AAe?$AA?$AA@ 00000001800174e8     libucrt:lcidtoname_downlevel.obj
 0001:000164f8       ??_C@_1M@PNBLONPJ@?$AAs?$AAk?$AA?9?$AAs?$AAk?$AA?$AA@ 00000001800174f8     libucrt:lcidtoname_downlevel.obj
 0001:00016508       ??_C@_1M@LFMODOAL@?$AAs?$AAl?$AA?9?$AAs?$AAi?$AA?$AA@ 0000000180017508     libucrt:lcidtoname_downlevel.obj
 0001:00016518       ??_C@_1O@DFKOMPG@?$AAs?$AAm?$AAa?$AA?9?$AAn?$AAo?$AA?$AA@ 0000000180017518     libucrt:lcidtoname_downlevel.obj
 0001:00016528       ??_C@_1O@NDKPBNNH@?$AAs?$AAm?$AAa?$AA?9?$AAs?$AAe?$AA?$AA@ 0000000180017528     libucrt:lcidtoname_downlevel.obj
 0001:00016538       ??_C@_1O@PLLKBHAB@?$AAs?$AAm?$AAj?$AA?9?$AAn?$AAo?$AA?$AA@ 0000000180017538     libucrt:lcidtoname_downlevel.obj
 0001:00016548       ??_C@_1O@CLEPOGCA@?$AAs?$AAm?$AAj?$AA?9?$AAs?$AAe?$AA?$AA@ 0000000180017548     libucrt:lcidtoname_downlevel.obj
 0001:00016558       ??_C@_1O@DLGJGKMK@?$AAs?$AAm?$AAn?$AA?9?$AAf?$AAi?$AA?$AA@ 0000000180017558     libucrt:lcidtoname_downlevel.obj
 0001:00016568       ??_C@_1O@OJDJGAJC@?$AAs?$AAm?$AAs?$AA?9?$AAf?$AAi?$AA?$AA@ 0000000180017568     libucrt:lcidtoname_downlevel.obj
 0001:00016578       ??_C@_1M@BOFOGHPB@?$AAs?$AAq?$AA?9?$AAa?$AAl?$AA?$AA@ 0000000180017578     libucrt:lcidtoname_downlevel.obj
 0001:00016588       ??_C@_1BG@LJBBIPGB@?$AAs?$AAr?$AA?9?$AAb?$AAa?$AA?9?$AAc?$AAy?$AAr?$AAl?$AA?$AA@ 0000000180017588     libucrt:lcidtoname_downlevel.obj
 0001:000165a0       ??_C@_1BG@JLBENFOE@?$AAs?$AAr?$AA?9?$AAb?$AAa?$AA?9?$AAl?$AAa?$AAt?$AAn?$AA?$AA@ 00000001800175a0     libucrt:lcidtoname_downlevel.obj
 0001:000165b8       ??_C@_1BG@KODPNHE@?$AAs?$AAr?$AA?9?$AAs?$AAp?$AA?9?$AAc?$AAy?$AAr?$AAl?$AA?$AA@ 00000001800175b8     libucrt:lcidtoname_downlevel.obj
 0001:000165d0       ??_C@_1BG@CIOGKHPB@?$AAs?$AAr?$AA?9?$AAs?$AAp?$AA?9?$AAl?$AAa?$AAt?$AAn?$AA?$AA@ 00000001800175d0     libucrt:lcidtoname_downlevel.obj
 0001:000165e8       ??_C@_1M@NGFJLMAC@?$AAs?$AAv?$AA?9?$AAf?$AAi?$AA?$AA@ 00000001800175e8     libucrt:lcidtoname_downlevel.obj
 0001:000165f8       ??_C@_1M@MPJEJAJC@?$AAs?$AAv?$AA?9?$AAs?$AAe?$AA?$AA@ 00000001800175f8     libucrt:lcidtoname_downlevel.obj
 0001:00016608       ??_C@_1M@MPNDHLFK@?$AAs?$AAw?$AA?9?$AAk?$AAe?$AA?$AA@ 0000000180017608     libucrt:lcidtoname_downlevel.obj
 0001:00016618       ??_C@_1O@KOHBJJI@?$AAs?$AAy?$AAr?$AA?9?$AAs?$AAy?$AA?$AA@ 0000000180017618     libucrt:lcidtoname_downlevel.obj
 0001:00016628       ??_C@_1M@LDCEFHA@?$AAt?$AAa?$AA?9?$AAi?$AAn?$AA?$AA@ 0000000180017628     libucrt:lcidtoname_downlevel.obj
 0001:00016638       ??_C@_1M@CNJOFAK@?$AAt?$AAe?$AA?9?$AAi?$AAn?$AA?$AA@ 0000000180017638     libucrt:lcidtoname_downlevel.obj
 0001:00016648       ??_C@_1M@GNAECACD@?$AAt?$AAh?$AA?9?$AAt?$AAh?$AA?$AA@ 0000000180017648     libucrt:lcidtoname_downlevel.obj
 0001:00016658       ??_C@_1M@CHBIHOJO@?$AAt?$AAn?$AA?9?$AAz?$AAa?$AA?$AA@ 0000000180017658     libucrt:lcidtoname_downlevel.obj
 0001:00016668       ??_C@_1M@GCCMIGPJ@?$AAt?$AAr?$AA?9?$AAt?$AAr?$AA?$AA@ 0000000180017668     libucrt:lcidtoname_downlevel.obj
 0001:00016678       ??_C@_1M@CELMCNBK@?$AAt?$AAt?$AA?9?$AAr?$AAu?$AA?$AA@ 0000000180017678     libucrt:lcidtoname_downlevel.obj
 0001:00016688       ??_C@_1M@KLMCELGA@?$AAu?$AAk?$AA?9?$AAu?$AAa?$AA?$AA@ 0000000180017688     libucrt:lcidtoname_downlevel.obj
 0001:00016698       ??_C@_1M@EPAJJAJF@?$AAu?$AAr?$AA?9?$AAp?$AAk?$AA?$AA@ 0000000180017698     libucrt:lcidtoname_downlevel.obj
 0001:000166a8       ??_C@_1BG@GEGPMCDJ@?$AAu?$AAz?$AA?9?$AAu?$AAz?$AA?9?$AAc?$AAy?$AAr?$AAl?$AA?$AA@ 00000001800176a8     libucrt:lcidtoname_downlevel.obj
 0001:000166c0       ??_C@_1BG@EGGKJILM@?$AAu?$AAz?$AA?9?$AAu?$AAz?$AA?9?$AAl?$AAa?$AAt?$AAn?$AA?$AA@ 00000001800176c0     libucrt:lcidtoname_downlevel.obj
 0001:000166d8       ??_C@_1M@GFOCLFF@?$AAv?$AAi?$AA?9?$AAv?$AAn?$AA?$AA@ 00000001800176d8     libucrt:lcidtoname_downlevel.obj
 0001:000166e8       ??_C@_1M@CPAMEDFI@?$AAx?$AAh?$AA?9?$AAz?$AAa?$AA?$AA@ 00000001800176e8     libucrt:lcidtoname_downlevel.obj
 0001:000166f8       ??_C@_1O@EBKIFIGN@?$AAz?$AAh?$AA?9?$AAc?$AAh?$AAs?$AA?$AA@ 00000001800176f8     libucrt:lcidtoname_downlevel.obj
 0001:00016708       ??_C@_1O@NMHPGANE@?$AAz?$AAh?$AA?9?$AAc?$AAh?$AAt?$AA?$AA@ 0000000180017708     libucrt:lcidtoname_downlevel.obj
 0001:00016718       ??_C@_1M@LPINJOMC@?$AAz?$AAh?$AA?9?$AAc?$AAn?$AA?$AA@ 0000000180017718     libucrt:lcidtoname_downlevel.obj
 0001:00016728       ??_C@_1M@OCJEJODD@?$AAz?$AAh?$AA?9?$AAh?$AAk?$AA?$AA@ 0000000180017728     libucrt:lcidtoname_downlevel.obj
 0001:00016738       ??_C@_1M@DNDLJINH@?$AAz?$AAh?$AA?9?$AAm?$AAo?$AA?$AA@ 0000000180017738     libucrt:lcidtoname_downlevel.obj
 0001:00016748       ??_C@_1M@MBFDNDND@?$AAz?$AAh?$AA?9?$AAs?$AAg?$AA?$AA@ 0000000180017748     libucrt:lcidtoname_downlevel.obj
 0001:00016758       ??_C@_1M@IMEPLEPE@?$AAz?$AAh?$AA?9?$AAt?$AAw?$AA?$AA@ 0000000180017758     libucrt:lcidtoname_downlevel.obj
 0001:00016768       ??_C@_1M@BBGHNHJP@?$AAz?$AAu?$AA?9?$AAz?$AAa?$AA?$AA@ 0000000180017768     libucrt:lcidtoname_downlevel.obj
 0001:000175c0       ??_C@_15EMKDOKLE@?$AAa?$AAr?$AA?$AA@ 00000001800185c0     libucrt:lcidtoname_downlevel.obj
 0001:000175c8       ??_C@_15KNPADPLH@?$AAb?$AAg?$AA?$AA@ 00000001800185c8     libucrt:lcidtoname_downlevel.obj
 0001:000175d0       ??_C@_15EDMHLDMO@?$AAc?$AAa?$AA?$AA@ 00000001800185d0     libucrt:lcidtoname_downlevel.obj
 0001:000175d8       ??_C@_1O@BPEAJADD@?$AAz?$AAh?$AA?9?$AAC?$AAH?$AAS?$AA?$AA@ 00000001800185d8     libucrt:lcidtoname_downlevel.obj
 0001:000175e8       ??_C@_15LJNHCMNK@?$AAc?$AAs?$AA?$AA@ 00000001800185e8     libucrt:lcidtoname_downlevel.obj
 0001:000175f0       ??_C@_15FOMCIDHG@?$AAd?$AAa?$AA?$AA@ 00000001800185f0     libucrt:lcidtoname_downlevel.obj
 0001:000175f8       ??_C@_15NBKABECB@?$AAd?$AAe?$AA?$AA@ 00000001800185f8     libucrt:lcidtoname_downlevel.obj
 0001:00017600       ??_C@_15GHPEIIAO@?$AAe?$AAl?$AA?$AA@ 0000000180018600     libucrt:lcidtoname_downlevel.obj
 0001:00017608       ??_C@_15MNPNEAIF@?$AAe?$AAn?$AA?$AA@ 0000000180018608     libucrt:lcidtoname_downlevel.obj
 0001:00017610       ??_C@_15GPIOMPMH@?$AAe?$AAs?$AA?$AA@ 0000000180018610     libucrt:lcidtoname_downlevel.obj
 0001:00017618       ??_C@_15NGLOAKJC@?$AAf?$AAi?$AA?$AA@ 0000000180018618     libucrt:lcidtoname_downlevel.obj
 0001:00017620       ??_C@_15FBKGNKAM@?$AAf?$AAr?$AA?$AA@ 0000000180018620     libucrt:lcidtoname_downlevel.obj
 0001:00017628       ??_C@_15KGGCNEFK@?$AAh?$AAe?$AA?$AA@ 0000000180018628     libucrt:lcidtoname_downlevel.obj
 0001:00017630       ??_C@_15PGHLIDMF@?$AAh?$AAu?$AA?$AA@ 0000000180018630     libucrt:lcidtoname_downlevel.obj
 0001:00017638       ??_C@_15BIEMAPLM@?$AAi?$AAs?$AA?$AA@ 0000000180018638     libucrt:lcidtoname_downlevel.obj
 0001:00017640       ??_C@_15IFJLDHAF@?$AAi?$AAt?$AA?$AA@ 0000000180018640     libucrt:lcidtoname_downlevel.obj
 0001:00017648       ??_C@_15GEMIOCAG@?$AAj?$AAa?$AA?$AA@ 0000000180018648     libucrt:lcidtoname_downlevel.obj
 0001:00017650       ??_C@_15EPELEGJA@?$AAk?$AAo?$AA?$AA@ 0000000180018650     libucrt:lcidtoname_downlevel.obj
 0001:00017658       ??_C@_15NDDHIMN@?$AAn?$AAl?$AA?$AA@ 0000000180018658     libucrt:lcidtoname_downlevel.obj
 0001:00017660       ??_C@_15BPIGNHCD@?$AAn?$AAo?$AA?$AA@ 0000000180018660     libucrt:lcidtoname_downlevel.obj
 0001:00017668       ??_C@_15DEOPBLCG@?$AAp?$AAl?$AA?$AA@ 0000000180018668     libucrt:lcidtoname_downlevel.obj
 0001:00017670       ??_C@_15KBECGEFG@?$AAp?$AAt?$AA?$AA@ 0000000180018670     libucrt:lcidtoname_downlevel.obj
 0001:00017678       ??_C@_15GLJCBFMD@?$AAr?$AAo?$AA?$AA@ 0000000180018678     libucrt:lcidtoname_downlevel.obj
 0001:00017680       ??_C@_15FEDGKCDI@?$AAr?$AAu?$AA?$AA@ 0000000180018680     libucrt:lcidtoname_downlevel.obj
 0001:00017688       ??_C@_15GLKMLLHM@?$AAh?$AAr?$AA?$AA@ 0000000180018688     libucrt:lcidtoname_downlevel.obj
 0001:00017690       ??_C@_15CPKMFBDB@?$AAs?$AAk?$AA?$AA@ 0000000180018690     libucrt:lcidtoname_downlevel.obj
 0001:00017698       ??_C@_15BAAIOGMK@?$AAs?$AAq?$AA?$AA@ 0000000180018698     libucrt:lcidtoname_downlevel.obj
 0001:000176a0       ??_C@_15INNPNOHD@?$AAs?$AAv?$AA?$AA@ 00000001800186a0     libucrt:lcidtoname_downlevel.obj
 0001:000176a8       ??_C@_15CABMMOGH@?$AAt?$AAh?$AA?$AA@ 00000001800186a8     libucrt:lcidtoname_downlevel.obj
 0001:000176b0       ??_C@_15BPLIHJJM@?$AAt?$AAr?$AA?$AA@ 00000001800186b0     libucrt:lcidtoname_downlevel.obj
 0001:000176b8       ??_C@_15NEOEKKDJ@?$AAu?$AAr?$AA?$AA@ 00000001800186b8     libucrt:lcidtoname_downlevel.obj
 0001:000176c0       ??_C@_15NFICGAJK@?$AAi?$AAd?$AA?$AA@ 00000001800186c0     libucrt:lcidtoname_downlevel.obj
 0001:000176c8       ??_C@_15HPJPHDM@?$AAb?$AAe?$AA?$AA@ 00000001800186c8     libucrt:lcidtoname_downlevel.obj
 0001:000176d0       ??_C@_15LCHLGJII@?$AAs?$AAl?$AA?$AA@ 00000001800186d0     libucrt:lcidtoname_downlevel.obj
 0001:000176d8       ??_C@_15PCFJPHHO@?$AAe?$AAt?$AA?$AA@ 00000001800186d8     libucrt:lcidtoname_downlevel.obj
 0001:000176e0       ??_C@_15HPFPGODN@?$AAl?$AAv?$AA?$AA@ 00000001800186e0     libucrt:lcidtoname_downlevel.obj
 0001:000176e8       ??_C@_15NFFGKGLG@?$AAl?$AAt?$AA?$AA@ 00000001800186e8     libucrt:lcidtoname_downlevel.obj
 0001:000176f0       ??_C@_15BDAKCCHN@?$AAf?$AAa?$AA?$AA@ 00000001800186f0     libucrt:lcidtoname_downlevel.obj
 0001:000176f8       ??_C@_15NFGIAIAJ@?$AAv?$AAi?$AA?$AA@ 00000001800186f8     libucrt:lcidtoname_downlevel.obj
 0001:00017700       ??_C@_15LMKNDMHN@?$AAh?$AAy?$AA?$AA@ 0000000180018700     libucrt:lcidtoname_downlevel.obj
 0001:00017708       ??_C@_15IJBHMCFL@?$AAa?$AAz?$AA?$AA@ 0000000180018708     libucrt:lcidtoname_downlevel.obj
 0001:00017710       ??_C@_15EKOFJABL@?$AAe?$AAu?$AA?$AA@ 0000000180018710     libucrt:lcidtoname_downlevel.obj
 0001:00017718       ??_C@_15BGHADCNK@?$AAm?$AAk?$AA?$AA@ 0000000180018718     libucrt:lcidtoname_downlevel.obj
 0001:00017720       ??_C@_15JDNICKHM@?$AAa?$AAf?$AA?$AA@ 0000000180018720     libucrt:lcidtoname_downlevel.obj
 0001:00017728       ??_C@_15KPJEDBKD@?$AAk?$AAa?$AA?$AA@ 0000000180018728     libucrt:lcidtoname_downlevel.obj
 0001:00017730       ??_C@_15PDNFFFEO@?$AAf?$AAo?$AA?$AA@ 0000000180018730     libucrt:lcidtoname_downlevel.obj
 0001:00017738       ??_C@_15OMLEGLOC@?$AAh?$AAi?$AA?$AA@ 0000000180018738     libucrt:lcidtoname_downlevel.obj
 0001:00017740       ??_C@_15IDNNENKK@?$AAm?$AAs?$AA?$AA@ 0000000180018740     libucrt:lcidtoname_downlevel.obj
 0001:00017748       ??_C@_15MACJNBMH@?$AAk?$AAk?$AA?$AA@ 0000000180018748     libucrt:lcidtoname_downlevel.obj
 0001:00017750       ??_C@_15DKDJEOND@?$AAk?$AAy?$AA?$AA@ 0000000180018750     libucrt:lcidtoname_downlevel.obj
 0001:00017758       ??_C@_15DFGDLJBG@?$AAs?$AAw?$AA?$AA@ 0000000180018758     libucrt:lcidtoname_downlevel.obj
 0001:00017760       ??_C@_15BBFAICNG@?$AAu?$AAz?$AA?$AA@ 0000000180018760     libucrt:lcidtoname_downlevel.obj
 0001:00017768       ??_C@_15DKNDCGEA@?$AAt?$AAt?$AA?$AA@ 0000000180018768     libucrt:lcidtoname_downlevel.obj
 0001:00017770       ??_C@_15MGIFMDPL@?$AAp?$AAa?$AA?$AA@ 0000000180018770     libucrt:lcidtoname_downlevel.obj
 0001:00017778       ??_C@_15HCNDBBA@?$AAg?$AAu?$AA?$AA@ 0000000180018778     libucrt:lcidtoname_downlevel.obj
 0001:00017780       ??_C@_15FNBEIBON@?$AAt?$AAa?$AA?$AA@ 0000000180018780     libucrt:lcidtoname_downlevel.obj
 0001:00017788       ??_C@_15NCHGBGLK@?$AAt?$AAe?$AA?$AA@ 0000000180018788     libucrt:lcidtoname_downlevel.obj
 0001:00017790       ??_C@_15PHPHCBPF@?$AAk?$AAn?$AA?$AA@ 0000000180018790     libucrt:lcidtoname_downlevel.obj
 0001:00017798       ??_C@_15DLGBCKMP@?$AAm?$AAr?$AA?$AA@ 0000000180018798     libucrt:lcidtoname_downlevel.obj
 0001:000177a0       ??_C@_15EABBLBFF@?$AAs?$AAa?$AA?$AA@ 00000001800187a0     libucrt:lcidtoname_downlevel.obj
 0001:000177a8       ??_C@_15CBKOMCOI@?$AAm?$AAn?$AA?$AA@ 00000001800187a8     libucrt:lcidtoname_downlevel.obj
 0001:000177b0       ??_C@_15CKDMCJAF@?$AAg?$AAl?$AA?$AA@ 00000001800187b0     libucrt:lcidtoname_downlevel.obj
 0001:000177b8       ??_C@_17CNJFBPG@?$AAk?$AAo?$AAk?$AA?$AA@ 00000001800187b8     libucrt:lcidtoname_downlevel.obj
 0001:000177c0       ??_C@_17FFBJICPL@?$AAs?$AAy?$AAr?$AA?$AA@ 00000001800187c0     libucrt:lcidtoname_downlevel.obj
 0001:000177c8       ??_C@_17KPNDCPAF@?$AAd?$AAi?$AAv?$AA?$AA@ 00000001800187c8     libucrt:lcidtoname_downlevel.obj
 0001:000177d0       ??_C@_1M@OKAHONE@?$AAa?$AAr?$AA?9?$AAS?$AAA?$AA?$AA@ 00000001800187d0     libucrt:lcidtoname_downlevel.obj
 0001:000177e0       ??_C@_1M@FFFIGIGK@?$AAb?$AAg?$AA?9?$AAB?$AAG?$AA?$AA@ 00000001800187e0     libucrt:lcidtoname_downlevel.obj
 0001:00017a40       ??_C@_1BA@BALFACEM@?$AAC?$AAO?$AAN?$AAO?$AAU?$AAT?$AA$?$AA?$AA@ 0000000180018a40     libucrt:initcon.obj
 0001:00017a50       __log10_256_lead           0000000180018a50     libucrt:log10_256_lead_tail_table.obj
 0001:00018260       __log10_256_tail           0000000180019260     libucrt:log10_256_lead_tail_table.obj
 0001:00018a70       __log_F_inv_qword          0000000180019a70     libucrt:log_f_inv_qword_table.obj
 0001:00019280       ??_C@_05HGHHAHAP@log10?$AA@ 000000018001a280     libucrt:log_special.obj
 0001:000192c0       _load_config_used          000000018001a2c0     LIBCMT:loadcfg.obj
 0001:00019640       __rtc_iaa                  000000018001a640     LIBCMT:_initsect_.obj
 0001:00019648       __rtc_izz                  000000018001a648     LIBCMT:_initsect_.obj
 0001:00019650       __rtc_taa                  000000018001a650     LIBCMT:_initsect_.obj
 0001:00019658       __rtc_tzz                  000000018001a658     LIBCMT:_initsect_.obj
 0001:00019670       _alloca_probe              000000018001a670 f   chkstk.obj
 0001:00019670       __chkstk                   000000018001a670 f   chkstk.obj
 0001:0001a1c0       __local_stdio_printf_options 000000018001b1c0 f i bit64.obj
 0001:0001a1d0       bit64_getvalue             000000018001b1d0 f   bit64.obj
 0001:0001a280       bit64_push                 000000018001b280 f   bit64.obj
 0001:0001a310       bit64_pushuserdata         000000018001b310 f   bit64.obj
 0001:0001a4a0       luaopen_bit64              000000018001b4a0 f   bit64.obj
 0001:0001a4f0       sprintf                    000000018001b4f0 f i bit64.obj
 0001:0001a550       AddBufToCollector          000000018001b550 f   exported.obj
 0001:0001a5c0       CreateStringsArray         000000018001b5c0 f   exported.obj
 0001:0001a6b0       FarPanelItemFreeCallback   000000018001b6b0 f   exported.obj
 0001:0001a990       FillFindData               000000018001b990 f   exported.obj
 0001:0001adb0       FillPluginPanelItem        000000018001bdb0 f   exported.obj
 0001:0001b080       GetExportFunction          000000018001c080 f   exported.obj
 0001:0001b130       LF_Analyse                 000000018001c130 f   exported.obj
 0001:0001b1f0       LF_CloseAnalyse            000000018001c1f0 f   exported.obj
 0001:0001b200       LF_ClosePanel              000000018001c200 f   exported.obj
 0001:0001b2e0       LF_Compare                 000000018001c2e0 f   exported.obj
 0001:0001b3e0       LF_Configure               000000018001c3e0 f   exported.obj
 0001:0001b470       LF_DeleteFiles             000000018001c470 f   exported.obj
 0001:0001b560       LF_ExitFAR                 000000018001c560 f   exported.obj
 0001:0001b5c0       LF_FreeContentData         000000018001c5c0 f   exported.obj
 0001:0001b610       LF_FreeFindData            000000018001c610 f   exported.obj
 0001:0001b670       LF_GetContentData          000000018001c670 f   exported.obj
 0001:0001b7d0       LF_GetContentFields        000000018001c7d0 f   exported.obj
 0001:0001b8a0       LF_GetFiles                000000018001c8a0 f   exported.obj
 0001:0001ba40       LF_GetFindData             000000018001ca40 f   exported.obj
 0001:0001bb50       LF_GetGlobalInfo           000000018001cb50 f   exported.obj
 0001:0001bf90       LF_GetOpenPanelInfo        000000018001cf90 f   exported.obj
 0001:0001c890       LF_GetPluginInfo           000000018001d890 f   exported.obj
 0001:0001c9d0       LF_MakeDirectory           000000018001d9d0 f   exported.obj
 0001:0001cb20       LF_Open                    000000018001db20 f   exported.obj
 0001:0001cf30       LF_ProcessConsoleInput     000000018001df30 f   exported.obj
 0001:0001d020       LF_ProcessDialogEvent      000000018001e020 f   exported.obj
 0001:0001d240       LF_ProcessEditorEvent      000000018001e240 f   exported.obj
 0001:0001d3b0       LF_ProcessEditorInput      000000018001e3b0 f   exported.obj
 0001:0001d430       LF_ProcessHostFile         000000018001e430 f   exported.obj
 0001:0001d550       LF_ProcessPanelEvent       000000018001e550 f   exported.obj
 0001:0001d670       LF_ProcessPanelInput       000000018001e670 f   exported.obj
 0001:0001d740       LF_ProcessSynchroEvent     000000018001e740 f   exported.obj
 0001:0001d930       LF_ProcessViewerEvent      000000018001e930 f   exported.obj
 0001:0001d9e0       LF_PutFiles                000000018001e9e0 f   exported.obj
 0001:0001db20       LF_RunDefaultScript        000000018001eb20 f   exported.obj
 0001:0001db30       LF_SetDirectory            000000018001eb30 f   exported.obj
 0001:0001dc10       LF_SetFindList             000000018001ec10 f   exported.obj
 0001:0001dcf0       PackMacroValues            000000018001ecf0 f   exported.obj
 0001:0001def0       PushFarMacroValue          000000018001eef0 f   exported.obj
 0001:0001e020       PushPluginObject           000000018001f020 f   exported.obj
 0001:0001e0d0       ReplacePluginInfoCollector 000000018001f0d0 f   exported.obj
 0001:0001e110       RunDefaultScript           000000018001f110 f   exported.obj
 0001:0001e350       UpdateFileSelection        000000018001f350 f   exported.obj
 0001:0001e430       _AddStringToCollector      000000018001f430 f   exported.obj
 0001:0001e4b0       getPluginMenuItems         000000018001f4b0 f   exported.obj
 0001:0001e580       pcall_msg                  000000018001f580 f   exported.obj
 0001:0001e680       traceback                  000000018001f680 f   exported.obj
 0001:0001e740       push_flags_table           000000018001f740 f   flags.obj
 0001:0001e7c0       SetFarColors               000000018001f7c0 f   keysandcolors.obj
 0001:0001e830       LF_Gsub                    000000018001f830 f   lflua.obj
 0001:0001e970       LF_LoadFile                000000018001f970 f   lflua.obj
 0001:0001ecd0       luaB_dofileW               000000018001fcd0 f   lflua.obj
 0001:0001ed40       luaB_loadfileW             000000018001fd40 f   lflua.obj
 0001:0001ed90       method_gc                  000000018001fd90 f   lregex.obj
 0001:0001ee10       method_tostring            000000018001fe10 f   lregex.obj
 0001:0001ee80       func_Gmatch                000000018001fe80 f   lregex.obj
 0001:0001ee90       func_GmatchW               000000018001fe90 f   lregex.obj
 0001:0001eea0       method_bracketscount       000000018001fea0 f   lregex.obj
 0001:0001ef20       func_New                   000000018001ff20 f   lregex.obj
 0001:0001ef70       method_find                000000018001ff70 f   lregex.obj
 0001:0001ef80       func_find                  000000018001ff80 f   lregex.obj
 0001:0001ef90       method_findW               000000018001ff90 f   lregex.obj
 0001:0001efb0       func_findW                 000000018001ffb0 f   lregex.obj
 0001:0001efc0       method_match               000000018001ffc0 f   lregex.obj
 0001:0001efd0       func_match                 000000018001ffd0 f   lregex.obj
 0001:0001efe0       method_matchW              000000018001ffe0 f   lregex.obj
 0001:0001eff0       func_matchW                000000018001fff0 f   lregex.obj
 0001:0001f000       method_gsub                0000000180020000 f   lregex.obj
 0001:0001f010       func_gsub                  0000000180020010 f   lregex.obj
 0001:0001f020       method_gsubW               0000000180020020 f   lregex.obj
 0001:0001f030       func_gsubW                 0000000180020030 f   lregex.obj
 0001:0001f040       _Gmatch                    0000000180020040 f   lregex.obj
 0001:0001f160       _regex_gmatch_closure      0000000180020160 f   lregex.obj
 0001:0001f2a0       check_regex_pattern        00000001800202a0 f   lregex.obj
 0001:0001f380       luaopen_regex              0000000180020380 f   lregex.obj
 0001:0001f410       push_far_regex             0000000180020410 f   lregex.obj
 0001:0001f4c0       regex_gmatch_closure       00000001800204c0 f   lregex.obj
 0001:0001f4d0       regex_gmatch_closureW      00000001800204d0 f   lregex.obj
 0001:0001f4e0       rx_find_match              00000001800204e0 f   lregex.obj
 0001:0001f770       rx_gsub                    0000000180020770 f   lregex.obj
 0001:00020070       Open_Luamacro              0000000180021070 f   luamacro.obj
 0001:00020470       far_FarMacroCallToLua      0000000180021470 f   luamacro.obj
 0001:00020510       far_MacroCallFar           0000000180021510 f   luamacro.obj
 0001:00020760       uc_len                     0000000180021760 f   lusercontrol.obj
 0001:00020a80       CheckFarUserControl        0000000180021a80 f   lusercontrol.obj
 0001:00020a90       luaopen_usercontrol        0000000180021a90 f   lusercontrol.obj
 0001:00020ae0       CreateRegKey               0000000180021ae0 f   reg.obj
 0001:00020b30       OpenRegKey                 0000000180021b30 f   reg.obj
 0001:00020b70       SetRegKeyArr               0000000180021b70 f   reg.obj
 0001:00020c00       SetRegKeyDword             0000000180021c00 f   reg.obj
 0001:00020c90       SetRegKeyStr               0000000180021c90 f   reg.obj
 0001:0002bd30       ConvertLuaValue            000000018002cd30 f   service.obj
 0001:0002be70       CreateList                 000000018002ce70 f   service.obj
 0001:0002c060       DeleteLuaStateTimerQueue   000000018002d060 f   service.obj
 0001:0002c090       DialogHandleEqual          000000018002d090 f   service.obj
 0001:0002c0f0       DllMain                    000000018002d0f0 f   service.obj
 0001:0002c340       FillInputRecord            000000018002d340 f   service.obj
 0001:0002c880       GetFarColor                000000018002d880 f   service.obj
 0001:0002c9c0       GetFlagCombination         000000018002d9c0 f   service.obj
 0001:0002cbe0       GetFlagsFromTable          000000018002dbe0 f   service.obj
 0001:0002cc20       GetLuaStateTimerQueue      000000018002dc20 f   service.obj
 0001:0002cc70       GetPluginData              000000018002dc70 f   service.obj
 0001:0002cc90       IsLuaJIT                   000000018002dc90 f   service.obj
 0001:0002cca0       LF_DlgProc                 000000018002dca0 f   service.obj
 0001:0002ce90       LF_DoFile                  000000018002de90 f   service.obj
 0001:0002cf60       LF_Error                   000000018002df60 f   service.obj
 0001:0002d060       LF_GetLuafarAPI            000000018002e060 f   service.obj
 0001:0002d0a0       LF_InitLuaState1           000000018002e0a0 f   service.obj
 0001:0002d2b0       LF_InitLuaState2           000000018002e2b0 f   service.obj
 0001:0002d380       LF_MacroCallback           000000018002e380 f   service.obj
 0001:0002d390       LF_Message                 000000018002e390 f   service.obj
 0001:0002d880       LF_ProcessEnvVars          000000018002e880 f   service.obj
 0001:0002d880       _guard_check_icall_nop     000000018002e880 f   LIBCMT:guard_support.obj
 0001:0002d890       LF_RunLuafarInit           000000018002e890 f   service.obj
 0001:0002d970       MacroAddCallback           000000018002e970 f   service.obj
 0001:0002dbb0       NewDialogData              000000018002ebb0 f   service.obj
 0001:0002dc70       NewVirtualKeyTable         000000018002ec70 f   service.obj
 0001:0002dd30       OptFlags                   000000018002ed30 f   service.obj
 0001:0002dda0       OptHandle                  000000018002eda0 f   service.obj
 0001:0002dee0       ProcessDNResult            000000018002eee0 f   service.obj
 0001:0002e350       PushDMParams               000000018002f350 f   service.obj
 0001:0002e450       PushDNParams               000000018002f450 f   service.obj
 0001:0002ea60       PushFarColor               000000018002fa60 f   service.obj
 0001:0002eae0       PushInputRecord            000000018002fae0 f   service.obj
 0001:0002ecc0       PushPanelItem              000000018002fcc0 f   service.obj
 0001:0002ef30       PushPanelItems             000000018002ff30 f   service.obj
 0001:0002f260       PutFlagsToTable            0000000180030260 f   service.obj
 0001:0002fb70       TimerCallback              0000000180030b70 f   service.obj
 0001:00030210       dir_exist                  0000000180031210 f   service.obj
 0001:00030240       fprintf                    0000000180031240 f i service.obj
 0001:00030ac0       pushFileTime               0000000180031ac0 f   service.obj
 0001:00032290       _snwprintf                 0000000180033290 f i slnunico.obj
 0001:000327b0       luaopen_unicode            00000001800337b0 f   slnunico.obj
 0001:00034cb0       __local_stdio_scanf_options 0000000180035cb0 f i uliolib51.obj
 0001:00034d80       fscanf                     0000000180035d80 f i uliolib51.obj
 0001:00035450       luaopen_uio                0000000180036450 f   uliolib51.obj
 0001:00036660       luaopen_upackage           0000000180037660 f   uloadlib51.obj
 0001:00036a20       ustring_WideCharToMultiByte 0000000180037a20 f   ustring.obj
 0001:00036bb0       ustring_MultiByteToWideChar 0000000180037bb0 f   ustring.obj
 0001:00036d40       ustring_OemToUtf8          0000000180037d40 f   ustring.obj
 0001:00036e40       ustring_Utf8ToOem          0000000180037e40 f   ustring.obj
 0001:00036f30       ustring_Utf16ToUtf8        0000000180037f30 f   ustring.obj
 0001:00036f80       ustring_Utf8ToUtf16        0000000180037f80 f   ustring.obj
 0001:00037060       ustring_GetACP             0000000180038060 f   ustring.obj
 0001:00037090       ustring_GetOEMCP           0000000180038090 f   ustring.obj
 0001:000370c0       ustring_EnumSystemCodePages 00000001800380c0 f   ustring.obj
 0001:00037150       ustring_GetCPInfo          0000000180038150 f   ustring.obj
 0001:000373f0       ustring_GetLogicalDriveStrings 00000001800383f0 f   ustring.obj
 0001:00037510       ustring_GetDriveType       0000000180038510 f   ustring.obj
 0001:00037620       ustring_Uuid               0000000180038620 f   ustring.obj
 0001:000376f0       ustring_SearchPath         00000001800386f0 f   ustring.obj
 0001:00037900       ustring_GlobalMemoryStatus 0000000180038900 f   ustring.obj
 0001:00037b10       ustring_Sleep              0000000180038b10 f   ustring.obj
 0001:00037b30       ustring_SetFileAttr        0000000180038b30 f   ustring.obj
 0001:00037d10       ustring_GetFileAttr        0000000180038d10 f   ustring.obj
 0001:00037e30       ustring_SHGetFolderPath    0000000180038e30 f   ustring.obj
 0001:00037f70       ustring_sub                0000000180038f70 f   ustring.obj
 0001:00038030       ustring_len                0000000180039030 f   ustring.obj
 0001:000382e0       ustring_GetCurrentDir      00000001800392e0 f   ustring.obj
 0001:00038470       ustring_SetCurrentDir      0000000180039470 f   ustring.obj
 0001:00038590       ustring_GetKeyState        0000000180039590 f   ustring.obj
 0001:000385e0       DecodeAttributes           00000001800395e0 f   ustring.obj
 0001:00038690       EnumCodePagesProc          0000000180039690 f   ustring.obj
 0001:00038700       GetBoolFromTable           0000000180039700 f   ustring.obj
 0001:00038750       GetOptBoolFromTable        0000000180039750 f   ustring.obj
 0001:000387b0       GetOptIntFromArray         00000001800397b0 f   ustring.obj
 0001:00038810       GetOptIntFromTable         0000000180039810 f   ustring.obj
 0001:00038870       GetOptNumFromTable         0000000180039870 f   ustring.obj
 0001:000388d0       PushAttrString             00000001800398d0 f   ustring.obj
 0001:00038990       PutAttrToTable             0000000180039990 f   ustring.obj
 0001:000389c0       PutBoolToTable             00000001800399c0 f   ustring.obj
 0001:00038a00       PutIntToArray              0000000180039a00 f   ustring.obj
 0001:00038a40       PutIntToTable              0000000180039a40 f   ustring.obj
 0001:00038a80       PutLStrToTable             0000000180039a80 f   ustring.obj
 0001:00038ac0       PutNumToTable              0000000180039ac0 f   ustring.obj
 0001:00038b00       PutStrToArray              0000000180039b00 f   ustring.obj
 0001:00038b40       PutStrToTable              0000000180039b40 f   ustring.obj
 0001:00038b80       PutWStrToArray             0000000180039b80 f   ustring.obj
 0001:00038be0       PutWStrToTable             0000000180039be0 f   ustring.obj
 0001:00038c20       SysErrorReturn             0000000180039c20 f   ustring.obj
 0001:00038c60       check_utf16_string         0000000180039c60 f   ustring.obj
 0001:00038c90       check_utf8_string          0000000180039c90 f   ustring.obj
 0001:00038cc0       convert_multibyte_string   0000000180039cc0 f   ustring.obj
 0001:00038df0       luaopen_ustring            0000000180039df0 f   ustring.obj
 0001:00038e50       opt_utf16_string           0000000180039e50 f   ustring.obj
 0001:00038e60       opt_utf8_string            0000000180039e60 f   ustring.obj
 0001:00038f70       push_multibyte_string      0000000180039f70 f   ustring.obj
 0001:00039080       push_utf16_string          000000018003a080 f   ustring.obj
 0001:000390b0       push_utf8_string           000000018003a0b0 f   ustring.obj
 0001:000390e0       pusherror                  000000018003a0e0 f   ustring.obj
 0001:00039100       pusherrorcode              000000018003a100 f   ustring.obj
 0001:000391a0       utf8_to_utf16              000000018003a1a0 f   ustring.obj
 0001:000391d0       GetAttrFromTable           000000018003a1d0 f   util.obj
 0001:00039230       GetFileSizeFromTable       000000018003a230 f   util.obj
 0001:000392c0       GetFileTimeFromTable       000000018003a2c0 f   util.obj
 0001:00039350       GetIntFromArray            000000018003a350 f   util.obj
 0001:00039410       PutFileTimeToTable         000000018003a410 f   util.obj
 0001:00039450       luaLF_FieldError           000000018003a450 f   util.obj
 0001:000394d0       luaLF_SlotError            000000018003a4d0 f   util.obj
 0001:0003acd0       luaopen_win                000000018003bcd0 f   win.obj
 0001:0003af6c       lua_gettop                 000000018003bf6c f   lua51:lua51.dll
 0001:0003af72       lua_settop                 000000018003bf72 f   lua51:lua51.dll
 0001:0003af78       lua_type                   000000018003bf78 f   lua51:lua51.dll
 0001:0003af7e       lua_rawequal               000000018003bf7e f   lua51:lua51.dll
 0001:0003af84       lua_tonumber               000000018003bf84 f   lua51:lua51.dll
 0001:0003af8a       lua_tolstring              000000018003bf8a f   lua51:lua51.dll
 0001:0003af90       lua_touserdata             000000018003bf90 f   lua51:lua51.dll
 0001:0003af96       lua_pushnil                000000018003bf96 f   lua51:lua51.dll
 0001:0003af9c       lua_pushnumber             000000018003bf9c f   lua51:lua51.dll
 0001:0003afa2       lua_pushstring             000000018003bfa2 f   lua51:lua51.dll
 0001:0003afa8       lua_pushboolean            000000018003bfa8 f   lua51:lua51.dll
 0001:0003afae       lua_getfield               000000018003bfae f   lua51:lua51.dll
 0001:0003afb4       lua_newuserdata            000000018003bfb4 f   lua51:lua51.dll
 0001:0003afba       lua_getmetatable           000000018003bfba f   lua51:lua51.dll
 0001:0003afc0       lua_setmetatable           000000018003bfc0 f   lua51:lua51.dll
 0001:0003afc6       luaL_register              000000018003bfc6 f   lua51:lua51.dll
 0001:0003afcc       luaL_argerror              000000018003bfcc f   lua51:lua51.dll
 0001:0003afd2       luaL_checkinteger          000000018003bfd2 f   lua51:lua51.dll
 0001:0003afd8       luaL_newmetatable          000000018003bfd8 f   lua51:lua51.dll
 0001:0003afde       lua_pushvalue              000000018003bfde f   lua51:lua51.dll
 0001:0003afe4       lua_remove                 000000018003bfe4 f   lua51:lua51.dll
 0001:0003afea       lua_insert                 000000018003bfea f   lua51:lua51.dll
 0001:0003aff0       lua_isnumber               000000018003bff0 f   lua51:lua51.dll
 0001:0003aff6       lua_isstring               000000018003bff6 f   lua51:lua51.dll
 0001:0003affc       lua_tointeger              000000018003bffc f   lua51:lua51.dll
 0001:0003b002       lua_toboolean              000000018003c002 f   lua51:lua51.dll
 0001:0003b008       lua_objlen                 000000018003c008 f   lua51:lua51.dll
 0001:0003b00e       lua_pushinteger            000000018003c00e f   lua51:lua51.dll
 0001:0003b014       lua_pushlstring            000000018003c014 f   lua51:lua51.dll
 0001:0003b01a       lua_pushcclosure           000000018003c01a f   lua51:lua51.dll
 0001:0003b020       lua_pushlightuserdata      000000018003c020 f   lua51:lua51.dll
 0001:0003b026       lua_gettable               000000018003c026 f   lua51:lua51.dll
 0001:0003b02c       lua_rawgeti                000000018003c02c f   lua51:lua51.dll
 0001:0003b032       lua_createtable            000000018003c032 f   lua51:lua51.dll
 0001:0003b038       lua_setfield               000000018003c038 f   lua51:lua51.dll
 0001:0003b03e       lua_rawseti                000000018003c03e f   lua51:lua51.dll
 0001:0003b044       lua_call                   000000018003c044 f   lua51:lua51.dll
 0001:0003b04a       lua_pcall                  000000018003c04a f   lua51:lua51.dll
 0001:0003b050       lua_gc                     000000018003c050 f   lua51:lua51.dll
 0001:0003b056       luaL_ref                   000000018003c056 f   lua51:lua51.dll
 0001:0003b05c       luaL_unref                 000000018003c05c f   lua51:lua51.dll
 0001:0003b062       luaL_loadstring            000000018003c062 f   lua51:lua51.dll
 0001:0003b068       lua_pushfstring            000000018003c068 f   lua51:lua51.dll
 0001:0003b06e       lua_load                   000000018003c06e f   lua51:lua51.dll
 0001:0003b074       lua_error                  000000018003c074 f   lua51:lua51.dll
 0001:0003b07a       lua_concat                 000000018003c07a f   lua51:lua51.dll
 0001:0003b080       luaL_buffinit              000000018003c080 f   lua51:lua51.dll
 0001:0003b086       luaL_addlstring            000000018003c086 f   lua51:lua51.dll
 0001:0003b08c       luaL_pushresult            000000018003c08c f   lua51:lua51.dll
 0001:0003b092       lua_replace                000000018003c092 f   lua51:lua51.dll
 0001:0003b098       lua_checkstack             000000018003c098 f   lua51:lua51.dll
 0001:0003b09e       luaL_checklstring          000000018003c09e f   lua51:lua51.dll
 0001:0003b0a4       luaL_optlstring            000000018003c0a4 f   lua51:lua51.dll
 0001:0003b0aa       luaL_optinteger            000000018003c0aa f   lua51:lua51.dll
 0001:0003b0b0       luaL_checkudata            000000018003c0b0 f   lua51:lua51.dll
 0001:0003b0b6       luaL_error                 000000018003c0b6 f   lua51:lua51.dll
 0001:0003b0bc       luaL_addvalue              000000018003c0bc f   lua51:lua51.dll
 0001:0003b0c2       lua_getstack               000000018003c0c2 f   lua51:lua51.dll
 0001:0003b0c8       lua_getinfo                000000018003c0c8 f   lua51:lua51.dll
 0001:0003b0ce       luaL_checktype             000000018003c0ce f   lua51:lua51.dll
 0001:0003b0d4       luaopen_base               000000018003c0d4 f   lua51:lua51.dll
 0001:0003b0da       luaopen_table              000000018003c0da f   lua51:lua51.dll
 0001:0003b0e0       luaopen_os                 000000018003c0e0 f   lua51:lua51.dll
 0001:0003b0e6       luaopen_string             000000018003c0e6 f   lua51:lua51.dll
 0001:0003b0ec       luaopen_math               000000018003c0ec f   lua51:lua51.dll
 0001:0003b0f2       luaopen_debug              000000018003c0f2 f   lua51:lua51.dll
 0001:0003b0f8       lua_rawget                 000000018003c0f8 f   lua51:lua51.dll
 0001:0003b0fe       lua_getfenv                000000018003c0fe f   lua51:lua51.dll
 0001:0003b104       lua_settable               000000018003c104 f   lua51:lua51.dll
 0001:0003b10a       lua_rawset                 000000018003c10a f   lua51:lua51.dll
 0001:0003b110       lua_setfenv                000000018003c110 f   lua51:lua51.dll
 0001:0003b116       lua_next                   000000018003c116 f   lua51:lua51.dll
 0001:0003b11c       lua_getallocf              000000018003c11c f   lua51:lua51.dll
 0001:0003b122       lua_setallocf              000000018003c122 f   lua51:lua51.dll
 0001:0003b128       luaL_typerror              000000018003c128 f   lua51:lua51.dll
 0001:0003b12e       luaL_checknumber           000000018003c12e f   lua51:lua51.dll
 0001:0003b134       luaL_optnumber             000000018003c134 f   lua51:lua51.dll
 0001:0003b13a       luaL_checkany              000000018003c13a f   lua51:lua51.dll
 0001:0003b140       luaL_findtable             000000018003c140 f   lua51:lua51.dll
 0001:0003b146       lua_typename               000000018003c146 f   lua51:lua51.dll
 0001:0003b14c       lua_dump                   000000018003c14c f   lua51:lua51.dll
 0001:0003b152       luaL_checkstack            000000018003c152 f   lua51:lua51.dll
 0001:0003b158       luaL_prepbuffer            000000018003c158 f   lua51:lua51.dll
 0001:0003b15e       lua_tocfunction            000000018003c15e f   lua51:lua51.dll
 0001:0003b164       luaL_checkoption           000000018003c164 f   lua51:lua51.dll
 0001:0003b16a       lua_iscfunction            000000018003c16a f   lua51:lua51.dll
 0001:0003b170       luaL_gsub                  000000018003c170 f   lua51:lua51.dll
 0001:0003b176       lua_isuserdata             000000018003c176 f   lua51:lua51.dll
 0001:0003b49c       _DllMainCRTStartup         000000018003c49c f   LIBCMT:dll_dllmain.obj
 0001:0003b4dc       __security_init_cookie     000000018003c4dc f   LIBCMT:gs_support.obj
 0001:0003b58c       ?__scrt_initialize_type_info@@YAXXZ 000000018003c58c f   LIBCMT:tncleanup.obj
 0001:0003b59c       ?__scrt_uninitialize_type_info@@YAXXZ 000000018003c59c f   LIBCMT:tncleanup.obj
 0001:0003b5a8       __scrt_initialize_default_local_stdio_options 000000018003c5a8 f   LIBCMT:default_local_stdio_options.obj
 0001:0003b5c4       __scrt_acquire_startup_lock 000000018003c5c4 f   LIBCMT:utility.obj
 0001:0003b600       __scrt_dllmain_after_initialize_c 000000018003c600 f   LIBCMT:utility.obj
 0001:0003b634       __scrt_dllmain_before_initialize_c 000000018003c634 f   LIBCMT:utility.obj
 0001:0003b64c       __scrt_dllmain_crt_thread_attach 000000018003c64c f   LIBCMT:utility.obj
 0001:0003b674       __scrt_dllmain_crt_thread_detach 000000018003c674 f   LIBCMT:utility.obj
 0001:0003b68c       __scrt_dllmain_exception_filter 000000018003c68c f   LIBCMT:utility.obj
 0001:0003b6ec       __scrt_dllmain_uninitialize_c 000000018003c6ec f   LIBCMT:utility.obj
 0001:0003b71c       __scrt_dllmain_uninitialize_critical 000000018003c71c f   LIBCMT:utility.obj
 0001:0003b730       __scrt_initialize_crt      000000018003c730 f   LIBCMT:utility.obj
 0001:0003b77c       __scrt_initialize_onexit_tables 000000018003c77c f   LIBCMT:utility.obj
 0001:0003b858       __scrt_is_nonwritable_in_current_image 000000018003c858 f   LIBCMT:utility.obj
 0001:0003b8f4       __scrt_release_startup_lock 000000018003c8f4 f   LIBCMT:utility.obj
 0001:0003b918       __scrt_uninitialize_crt    000000018003c918 f   LIBCMT:utility.obj
 0001:0003b944       __scrt_get_dyn_tls_init_callback 000000018003c944 f   LIBCMT:dyn_tls_init.obj
 0001:0003b94c       __crt_debugger_hook        000000018003c94c f   LIBCMT:utility_desktop.obj
 0001:0003b954       __scrt_fastfail            000000018003c954 f   LIBCMT:utility_desktop.obj
 0001:0003baa0       _RTC_Initialize            000000018003caa0 f   LIBCMT:_initsect_.obj
 0001:0003badc       _RTC_Terminate             000000018003cadc f   LIBCMT:_initsect_.obj
 0001:0003bb18       __isa_available_init       000000018003cb18 f   LIBCMT:_cpu_disp_.obj
 0001:0003bcd4       _get_startup_argv_mode     000000018003ccd4 f   LIBCMT:argv_mode.obj
 0001:0003bcdc       __scrt_is_ucrt_dll_in_use  000000018003ccdc f   LIBCMT:ucrt_detection.obj
 0001:0003bcf0       wcsrchr                    000000018003ccf0 f   libvcruntime:wcsrchr.obj
 0001:0003bdc0       memmove                    000000018003cdc0 f   libvcruntime:memcpy.obj
 0001:0003bdc0       memcpy                     000000018003cdc0 f   libvcruntime:memcpy.obj
 0001:0003c220       memset                     000000018003d220 f   libvcruntime:memset.obj
 0001:0003c3d0       wcsstr                     000000018003d3d0 f   libvcruntime:wcsstr.obj
 0001:0003c5ec       strchr                     000000018003d5ec f   libvcruntime:strchr.obj
 0001:0003c678       wcschr                     000000018003d678 f   libvcruntime:wcschr.obj
 0001:0003c720       memchr                     000000018003d720 f   libvcruntime:memchr.obj
 0001:0003c7a0       memcmp                     000000018003d7a0 f   libvcruntime:memcmp.obj
 0001:0003c868       strrchr                    000000018003d868 f   libvcruntime:strrchr.obj
 0001:0003c9b4       __C_specific_handler       000000018003d9b4 f   libvcruntime:_riscchandler_.obj
 0001:0003cbc0       __std_type_info_destroy_list 000000018003dbc0 f   libvcruntime:std_type_info.obj
 0001:0003cbec       __vcrt_initialize          000000018003dbec f   libvcruntime:initialization.obj
 0001:0003cc20       __vcrt_thread_attach       000000018003dc20 f   libvcruntime:initialization.obj
 0001:0003cc34       __vcrt_thread_detach       000000018003dc34 f   libvcruntime:initialization.obj
 0001:0003cc48       __vcrt_uninitialize        000000018003dc48 f   libvcruntime:initialization.obj
 0001:0003cc68       __vcrt_uninitialize_critical 000000018003dc68 f   libvcruntime:initialization.obj
 0001:0003cc90       _local_unwind              000000018003dc90 f   libvcruntime:_jmpuwind_.obj
 0001:0003ccc0       _NLG_Notify                000000018003dcc0 f   libvcruntime:_jmpuwind_.obj
 0001:0003cce0       __NLG_Dispatch2            000000018003dce0 f   libvcruntime:_jmpuwind_.obj
 0001:0003ccf0       __NLG_Return2              000000018003dcf0 f   libvcruntime:_jmpuwind_.obj
 0001:0003ccf4       __except_validate_context_record 000000018003dcf4 f   libvcruntime:jbcxrval.obj
 0001:0003cd2c       __vcrt_freefls             000000018003dd2c f   libvcruntime:per_thread_data.obj
 0001:0003cd4c       __vcrt_freeptd             000000018003dd4c f   libvcruntime:per_thread_data.obj
 0001:0003cd9c       __vcrt_getptd_noexit       000000018003dd9c f   libvcruntime:per_thread_data.obj
 0001:0003ce54       __vcrt_initialize_ptd      000000018003de54 f   libvcruntime:per_thread_data.obj
 0001:0003cea4       __vcrt_uninitialize_ptd    000000018003dea4 f   libvcruntime:per_thread_data.obj
 0001:0003cec8       __vcrt_initialize_locks    000000018003dec8 f   libvcruntime:locks.obj
 0001:0003cf10       __vcrt_uninitialize_locks  000000018003df10 f   libvcruntime:locks.obj
 0001:0003d120       __vcrt_FlsAlloc            000000018003e120 f   libvcruntime:winapi_downlevel.obj
 0001:0003d168       __vcrt_FlsFree             000000018003e168 f   libvcruntime:winapi_downlevel.obj
 0001:0003d1b0       __vcrt_FlsGetValue         000000018003e1b0 f   libvcruntime:winapi_downlevel.obj
 0001:0003d1f8       __vcrt_FlsSetValue         000000018003e1f8 f   libvcruntime:winapi_downlevel.obj
 0001:0003d24c       __vcrt_InitializeCriticalSectionEx 000000018003e24c f   libvcruntime:winapi_downlevel.obj
 0001:0003d2b0       __vcrt_initialize_winapi_thunks 000000018003e2b0 f   libvcruntime:winapi_downlevel.obj
 0001:0003d2e0       __vcrt_uninitialize_winapi_thunks 000000018003e2e0 f   libvcruntime:winapi_downlevel.obj
 0001:0003d320       __vcrt_initialize_pure_virtual_call_handler 000000018003e320 f   libvcruntime:purevirt_data.obj
 0001:0003d340       _CallSettingFrame          000000018003e340 f   libvcruntime:handlers.obj
 0001:0003d380       __DestructExceptionObject  000000018003e380 f   libvcruntime:ehhelpers.obj
 0001:0003d3f4       ?_CallMemberFunction0@@YAXQEAX0@Z 000000018003e3f4 f i libvcruntime:ehhelpers.obj
 0001:0003d7d8       ??$ensure_buffer_is_big_enough@D@formatting_buffer@__crt_stdio_output@@QEAA_N_K@Z 000000018003e7d8 f i libucrt:output.obj
 0001:0003d880       ??$ensure_buffer_is_big_enough@_W@formatting_buffer@__crt_stdio_output@@QEAA_N_K@Z 000000018003e880 f i libucrt:output.obj
 0001:0003d92c       ??$is_wide_character_specifier@_W@__crt_stdio_output@@YA_N_K_WW4length_modifier@0@@Z 000000018003e92c f i libucrt:output.obj
 0001:0003d96c       ??$type_case_integer_parse_into_buffer@I@?$output_processor@DV?$stream_output_adapter@D@__crt_stdio_output@@V?$standard_base@DV?$stream_output_adapter@D@__crt_stdio_output@@@2@@__crt_stdio_output@@AEAAXII_N@Z 000000018003e96c f i libucrt:output.obj
 0001:0003d96c       ??$type_case_integer_parse_into_buffer@I@?$output_processor@DV?$string_output_adapter@D@__crt_stdio_output@@V?$standard_base@DV?$string_output_adapter@D@__crt_stdio_output@@@2@@__crt_stdio_output@@AEAAXII_N@Z 000000018003e96c f i libucrt:output.obj
 0001:0003d9f4       ??$type_case_integer_parse_into_buffer@I@?$output_processor@_WV?$string_output_adapter@_W@__crt_stdio_output@@V?$standard_base@_WV?$string_output_adapter@_W@__crt_stdio_output@@@2@@__crt_stdio_output@@AEAAXII_N@Z 000000018003e9f4 f i libucrt:output.obj
 0001:0003da90       ??$type_case_integer_parse_into_buffer@_K@?$output_processor@DV?$stream_output_adapter@D@__crt_stdio_output@@V?$standard_base@DV?$stream_output_adapter@D@__crt_stdio_output@@@2@@__crt_stdio_output@@AEAAX_KI_N@Z 000000018003ea90 f i libucrt:output.obj
 0001:0003da90       ??$type_case_integer_parse_into_buffer@_K@?$output_processor@DV?$string_output_adapter@D@__crt_stdio_output@@V?$standard_base@DV?$string_output_adapter@D@__crt_stdio_output@@@2@@__crt_stdio_output@@AEAAX_KI_N@Z 000000018003ea90 f i libucrt:output.obj
 0001:0003db20       ??$type_case_integer_parse_into_buffer@_K@?$output_processor@_WV?$string_output_adapter@_W@__crt_stdio_output@@V?$standard_base@_WV?$string_output_adapter@_W@__crt_stdio_output@@@2@@__crt_stdio_output@@AEAAX_KI_N@Z 000000018003eb20 f i libucrt:output.obj
 0001:0003dbc0       ??$write_multiple_characters@V?$stream_output_adapter@D@__crt_stdio_output@@D@__crt_stdio_output@@YAXAEBV?$stream_output_adapter@D@0@DHQEAH@Z 000000018003ebc0 f i libucrt:output.obj
 0001:0003dc44       ??$write_multiple_characters@V?$string_output_adapter@D@__crt_stdio_output@@D@__crt_stdio_output@@YAXAEBV?$string_output_adapter@D@0@DHQEAH@Z 000000018003ec44 f i libucrt:output.obj
 0001:0003dca0       ??$write_multiple_characters@V?$string_output_adapter@_W@__crt_stdio_output@@D@__crt_stdio_output@@YAXAEBV?$string_output_adapter@_W@0@DHQEAH@Z 000000018003eca0 f i libucrt:output.obj
 0001:0003dd10       ??0_LocaleUpdate@@QEAA@QEAU__crt_locale_pointers@@@Z 000000018003ed10 f i libucrt:output.obj
 0001:0003ded0       ?force_decimal_point@__crt_stdio_output@@YAXPEADQEAU__crt_locale_pointers@@@Z 000000018003eed0 f i libucrt:output.obj
 0001:0003df40       ?parse_int_from_format_string@?$output_processor@DV?$string_output_adapter@D@__crt_stdio_output@@V?$standard_base@DV?$string_output_adapter@D@__crt_stdio_output@@@2@@__crt_stdio_output@@AEAA_NQEAH@Z 000000018003ef40 f i libucrt:output.obj
 0001:0003df40       ?parse_int_from_format_string@?$output_processor@DV?$stream_output_adapter@D@__crt_stdio_output@@V?$standard_base@DV?$stream_output_adapter@D@__crt_stdio_output@@@2@@__crt_stdio_output@@AEAA_NQEAH@Z 000000018003ef40 f i libucrt:output.obj
 0001:0003dfe4       ?parse_int_from_format_string@?$output_processor@_WV?$string_output_adapter@_W@__crt_stdio_output@@V?$standard_base@_WV?$string_output_adapter@_W@__crt_stdio_output@@@2@@__crt_stdio_output@@AEAA_NQEAH@Z 000000018003efe4 f i libucrt:output.obj
 0001:0003e088       ?process@?$output_processor@DV?$stream_output_adapter@D@__crt_stdio_output@@V?$standard_base@DV?$stream_output_adapter@D@__crt_stdio_output@@@2@@__crt_stdio_output@@QEAAHXZ 000000018003f088 f i libucrt:output.obj
 0001:0003e29c       ?process@?$output_processor@DV?$string_output_adapter@D@__crt_stdio_output@@V?$standard_base@DV?$string_output_adapter@D@__crt_stdio_output@@@2@@__crt_stdio_output@@QEAAHXZ 000000018003f29c f i libucrt:output.obj
 0001:0003e4a4       ?process@?$output_processor@_WV?$string_output_adapter@_W@__crt_stdio_output@@V?$standard_base@_WV?$string_output_adapter@_W@__crt_stdio_output@@@2@@__crt_stdio_output@@QEAAHXZ 000000018003f4a4 f i libucrt:output.obj
 0001:0003e70c       ?state_case_normal@?$output_processor@DV?$stream_output_adapter@D@__crt_stdio_output@@V?$standard_base@DV?$stream_output_adapter@D@__crt_stdio_output@@@2@@__crt_stdio_output@@AEAA_NXZ 000000018003f70c f i libucrt:output.obj
 0001:0003e77c       ?state_case_normal@?$output_processor@DV?$string_output_adapter@D@__crt_stdio_output@@V?$standard_base@DV?$string_output_adapter@D@__crt_stdio_output@@@2@@__crt_stdio_output@@AEAA_NXZ 000000018003f77c f i libucrt:output.obj
 0001:0003e7f0       ?state_case_normal_tchar@?$output_processor@DV?$stream_output_adapter@D@__crt_stdio_output@@V?$standard_base@DV?$stream_output_adapter@D@__crt_stdio_output@@@2@@__crt_stdio_output@@AEAA_ND@Z 000000018003f7f0 f i libucrt:output.obj
 0001:0003e88c       ?state_case_normal_tchar@?$output_processor@DV?$string_output_adapter@D@__crt_stdio_output@@V?$standard_base@DV?$string_output_adapter@D@__crt_stdio_output@@@2@@__crt_stdio_output@@AEAA_ND@Z 000000018003f88c f i libucrt:output.obj
 0001:0003e924       ?state_case_size@?$output_processor@DV?$stream_output_adapter@D@__crt_stdio_output@@V?$standard_base@DV?$stream_output_adapter@D@__crt_stdio_output@@@2@@__crt_stdio_output@@AEAA_NXZ 000000018003f924 f i libucrt:output.obj
 0001:0003eaa0       ?state_case_size@?$output_processor@DV?$string_output_adapter@D@__crt_stdio_output@@V?$standard_base@DV?$string_output_adapter@D@__crt_stdio_output@@@2@@__crt_stdio_output@@AEAA_NXZ 000000018003faa0 f i libucrt:output.obj
 0001:0003ec1c       ?state_case_size@?$output_processor@_WV?$string_output_adapter@_W@__crt_stdio_output@@V?$standard_base@_WV?$string_output_adapter@_W@__crt_stdio_output@@@2@@__crt_stdio_output@@AEAA_NXZ 000000018003fc1c f i libucrt:output.obj
 0001:0003edc0       ?state_case_type@?$output_processor@DV?$stream_output_adapter@D@__crt_stdio_output@@V?$standard_base@DV?$stream_output_adapter@D@__crt_stdio_output@@@2@@__crt_stdio_output@@AEAA_NXZ 000000018003fdc0 f i libucrt:output.obj
 0001:0003f058       ?state_case_type@?$output_processor@DV?$string_output_adapter@D@__crt_stdio_output@@V?$standard_base@DV?$string_output_adapter@D@__crt_stdio_output@@@2@@__crt_stdio_output@@AEAA_NXZ 0000000180040058 f i libucrt:output.obj
 0001:0003f2cc       ?state_case_type@?$output_processor@_WV?$string_output_adapter@_W@__crt_stdio_output@@V?$standard_base@_WV?$string_output_adapter@_W@__crt_stdio_output@@@2@@__crt_stdio_output@@AEAA_NXZ 00000001800402cc f i libucrt:output.obj
 0001:0003f5a8       ?type_case_Z@?$output_processor@DV?$string_output_adapter@D@__crt_stdio_output@@V?$standard_base@DV?$string_output_adapter@D@__crt_stdio_output@@@2@@__crt_stdio_output@@AEAA_NXZ 00000001800405a8 f i libucrt:output.obj
 0001:0003f5a8       ?type_case_Z@?$output_processor@DV?$stream_output_adapter@D@__crt_stdio_output@@V?$standard_base@DV?$stream_output_adapter@D@__crt_stdio_output@@@2@@__crt_stdio_output@@AEAA_NXZ 00000001800405a8 f i libucrt:output.obj
 0001:0003f628       ?type_case_Z@?$output_processor@_WV?$string_output_adapter@_W@__crt_stdio_output@@V?$standard_base@_WV?$string_output_adapter@_W@__crt_stdio_output@@@2@@__crt_stdio_output@@AEAA_NXZ 0000000180040628 f i libucrt:output.obj
 0001:0003f6a8       ?type_case_a@?$output_processor@DV?$stream_output_adapter@D@__crt_stdio_output@@V?$standard_base@DV?$stream_output_adapter@D@__crt_stdio_output@@@2@@__crt_stdio_output@@AEAA_NXZ 00000001800406a8 f i libucrt:output.obj
 0001:0003f6a8       ?type_case_a@?$output_processor@DV?$string_output_adapter@D@__crt_stdio_output@@V?$standard_base@DV?$string_output_adapter@D@__crt_stdio_output@@@2@@__crt_stdio_output@@AEAA_NXZ 00000001800406a8 f i libucrt:output.obj
 0001:0003f8c0       ?type_case_a@?$output_processor@_WV?$string_output_adapter@_W@__crt_stdio_output@@V?$standard_base@_WV?$string_output_adapter@_W@__crt_stdio_output@@@2@@__crt_stdio_output@@AEAA_NXZ 00000001800408c0 f i libucrt:output.obj
 0001:0003fb00       ?type_case_c_tchar@?$output_processor@DV?$stream_output_adapter@D@__crt_stdio_output@@V?$standard_base@DV?$stream_output_adapter@D@__crt_stdio_output@@@2@@__crt_stdio_output@@AEAA_ND@Z 0000000180040b00 f i libucrt:output.obj
 0001:0003fb00       ?type_case_c_tchar@?$output_processor@DV?$string_output_adapter@D@__crt_stdio_output@@V?$standard_base@DV?$string_output_adapter@D@__crt_stdio_output@@@2@@__crt_stdio_output@@AEAA_ND@Z 0000000180040b00 f i libucrt:output.obj
 0001:0003fbcc       ?type_case_c_tchar@?$output_processor@_WV?$string_output_adapter@_W@__crt_stdio_output@@V?$standard_base@_WV?$string_output_adapter@_W@__crt_stdio_output@@@2@@__crt_stdio_output@@AEAA_N_W@Z 0000000180040bcc f i libucrt:output.obj
 0001:0003fc74       ?type_case_integer@?$output_processor@DV?$string_output_adapter@D@__crt_stdio_output@@V?$standard_base@DV?$string_output_adapter@D@__crt_stdio_output@@@2@@__crt_stdio_output@@AEAA_NI_N@Z 0000000180040c74 f i libucrt:output.obj
 0001:0003fc74       ?type_case_integer@?$output_processor@DV?$stream_output_adapter@D@__crt_stdio_output@@V?$standard_base@DV?$stream_output_adapter@D@__crt_stdio_output@@@2@@__crt_stdio_output@@AEAA_NI_N@Z 0000000180040c74 f i libucrt:output.obj
 0001:0003fe38       ?type_case_integer@?$output_processor@_WV?$string_output_adapter@_W@__crt_stdio_output@@V?$standard_base@_WV?$string_output_adapter@_W@__crt_stdio_output@@@2@@__crt_stdio_output@@AEAA_NI_N@Z 0000000180040e38 f i libucrt:output.obj
 0001:00040004       ?type_case_n@?$output_processor@DV?$stream_output_adapter@D@__crt_stdio_output@@V?$standard_base@DV?$stream_output_adapter@D@__crt_stdio_output@@@2@@__crt_stdio_output@@AEAA_NXZ 0000000180041004 f i libucrt:output.obj
 0001:00040004       ?type_case_n@?$output_processor@_WV?$string_output_adapter@_W@__crt_stdio_output@@V?$standard_base@_WV?$string_output_adapter@_W@__crt_stdio_output@@@2@@__crt_stdio_output@@AEAA_NXZ 0000000180041004 f i libucrt:output.obj
 0001:00040004       ?type_case_n@?$output_processor@DV?$string_output_adapter@D@__crt_stdio_output@@V?$standard_base@DV?$string_output_adapter@D@__crt_stdio_output@@@2@@__crt_stdio_output@@AEAA_NXZ 0000000180041004 f i libucrt:output.obj
 0001:000400e0       ?type_case_s@?$output_processor@DV?$string_output_adapter@D@__crt_stdio_output@@V?$standard_base@DV?$string_output_adapter@D@__crt_stdio_output@@@2@@__crt_stdio_output@@AEAA_NXZ 00000001800410e0 f i libucrt:output.obj
 0001:000400e0       ?type_case_s@?$output_processor@DV?$stream_output_adapter@D@__crt_stdio_output@@V?$standard_base@DV?$stream_output_adapter@D@__crt_stdio_output@@@2@@__crt_stdio_output@@AEAA_NXZ 00000001800410e0 f i libucrt:output.obj
 0001:0004017c       ?type_case_s@?$output_processor@_WV?$string_output_adapter@_W@__crt_stdio_output@@V?$standard_base@_WV?$string_output_adapter@_W@__crt_stdio_output@@@2@@__crt_stdio_output@@AEAA_NXZ 000000018004117c f i libucrt:output.obj
 0001:00040244       ?validate_stream_is_ansi_if_required@?$__acrt_stdio_char_traits@D@@SA_NQEAU_iobuf@@@Z 0000000180041244 f i libucrt:output.obj
 0001:000402d0       ?write_stored_string_tchar@?$output_processor@DV?$stream_output_adapter@D@__crt_stdio_output@@V?$standard_base@DV?$stream_output_adapter@D@__crt_stdio_output@@@2@@__crt_stdio_output@@AEAA_ND@Z 00000001800412d0 f i libucrt:output.obj
 0001:000403f4       ?write_stored_string_tchar@?$output_processor@DV?$string_output_adapter@D@__crt_stdio_output@@V?$standard_base@DV?$string_output_adapter@D@__crt_stdio_output@@@2@@__crt_stdio_output@@AEAA_ND@Z 00000001800413f4 f i libucrt:output.obj
 0001:000404cc       ?write_stored_string_tchar@?$output_processor@_WV?$string_output_adapter@_W@__crt_stdio_output@@V?$standard_base@_WV?$string_output_adapter@_W@__crt_stdio_output@@@2@@__crt_stdio_output@@AEAA_N_W@Z 00000001800414cc f i libucrt:output.obj
 0001:000405bc       ?write_string@?$string_output_adapter@D@__crt_stdio_output@@QEBAXQEBDHQEAHAEAV__crt_deferred_errno_cache@@@Z 00000001800415bc f i libucrt:output.obj
 0001:00040660       ?write_string@?$string_output_adapter@_W@__crt_stdio_output@@QEBAXQEB_WHQEAHAEAV__crt_deferred_errno_cache@@@Z 0000000180041660 f i libucrt:output.obj
 0001:00040708       ?write_string_impl@?$output_adapter_common@DV?$stream_output_adapter@D@__crt_stdio_output@@@__crt_stdio_output@@IEBAXQEBDHQEAHAEAV__crt_deferred_errno_cache@@@Z 0000000180041708 f i libucrt:output.obj
 0001:00040800       __stdio_common_vfprintf    0000000180041800 f   libucrt:output.obj
 0001:0004088c       __stdio_common_vsprintf    000000018004188c f   libucrt:output.obj
 0001:00040894       __stdio_common_vswprintf   0000000180041894 f   libucrt:output.obj
 0001:0004089c       _wcsdup                    000000018004189c f   libucrt:wcsdup.obj
 0001:0004089c       wcsdup                     000000018004189c f   libucrt:wcsdup.obj
 0001:00040920       free                       0000000180041920 f   libucrt:free.obj
 0001:00040934       malloc                     0000000180041934 f   libucrt:malloc.obj
 0001:00040a04       _wfopen                    0000000180041a04 f   libucrt:fopen.obj
 0001:00040a10       _fclose_nolock             0000000180041a10 f   libucrt:fclose.obj
 0001:00040a94       fclose                     0000000180041a94 f   libucrt:fclose.obj
 0001:00040af8       _clearfp                   0000000180041af8 f   libucrt:ieee.obj
 0001:00040b68       _control87                 0000000180041b68 f   libucrt:ieee.obj
 0001:00040e30       __acrt_errno_from_os_error 0000000180041e30 f   libucrt:errno.obj
 0001:00040e78       __acrt_errno_map_os_error  0000000180041e78 f   libucrt:errno.obj
 0001:00040ec8       __doserrno                 0000000180041ec8 f   libucrt:errno.obj
 0001:00040ee8       _errno                     0000000180041ee8 f   libucrt:errno.obj
 0001:00040f08       strerror                   0000000180041f08 f   libucrt:strerror.obj
 0001:00040fac       __acrt_initialize_stdio    0000000180041fac f   libucrt:_file.obj
 0001:000410cc       __acrt_iob_func            00000001800420cc f   libucrt:_file.obj
 0001:000410e0       __acrt_uninitialize_stdio  00000001800420e0 f   libucrt:_file.obj
 0001:0004113c       _lock_file                 000000018004213c f   libucrt:_file.obj
 0001:00041148       _unlock_file               0000000180042148 f   libucrt:_file.obj
 0001:00041258       _wfreopen                  0000000180042258 f   libucrt:freopen.obj
 0001:00041288       feof                       0000000180042288 f   libucrt:feoferr.obj
 0001:000412b4       ferror                     00000001800422b4 f   libucrt:feoferr.obj
 0001:000412e0       _fread_nolock_s            00000001800422e0 f   libucrt:fread.obj
 0001:00041574       fread                      0000000180042574 f   libucrt:fread.obj
 0001:00041594       fread_s                    0000000180042594 f   libucrt:fread.obj
 0001:0004163c       _fgetc_nolock              000000018004263c f   libucrt:fgetc.obj
 0001:00041680       _getc_nolock               0000000180042680 f   libucrt:fgetc.obj
 0001:00041688       fgetc                      0000000180042688 f   libucrt:fgetc.obj
 0001:00041784       getc                       0000000180042784 f   libucrt:fgetc.obj
 0001:0004178c       rewind                     000000018004278c f   libucrt:rewind.obj
 0001:0004184c       _ungetc_nolock             000000018004284c f   libucrt:ungetc.obj
 0001:0004195c       ungetc                     000000018004295c f   libucrt:ungetc.obj
 0001:000419d0       strcmp                     00000001800429d0 f   libucrt:strcmp.obj
 0001:00041a38       iswctype                   0000000180042a38 f   libucrt:iswctype.obj
 0001:00041aa8       isdigit                    0000000180042aa8 f i libucrt:_ctype.obj
 0001:00041b1c       isspace                    0000000180042b1c f i libucrt:_ctype.obj
 0001:00041b90       wcsncpy                    0000000180042b90 f   libucrt:wcsncpy.obj
 0001:00041bd8       _wcsicmp                   0000000180042bd8 f   libucrt:wcsicmp.obj
 0001:00041c5c       _wcsicmp_l                 0000000180042c5c f   libucrt:wcsicmp.obj
 0001:00041d60       strncmp                    0000000180042d60 f   libucrt:strncmp.obj
 0001:00041df0       strncpy                    0000000180042df0 f   libucrt:strncpy.obj
 0001:00042000       strpbrk                    0000000180043000 f   libucrt:strpbrk.obj
 0001:00042b30       _pclose                    0000000180043b30 f   libucrt:popen.obj
 0001:00042c08       _wpopen                    0000000180043c08 f   libucrt:popen.obj
 0001:00042c10       clearerr                   0000000180043c10 f   libucrt:clearerr.obj
 0001:00042c18       clearerr_s                 0000000180043c18 f   libucrt:clearerr.obj
 0001:00042ee4       __acrt_stdio_flush_nolock  0000000180043ee4 f   libucrt:fflush.obj
 0001:00042f60       _fflush_nolock             0000000180043f60 f   libucrt:fflush.obj
 0001:00042fac       _flushall                  0000000180043fac f   libucrt:fflush.obj
 0001:00042fb4       fflush                     0000000180043fb4 f   libucrt:fflush.obj
 0001:000430ec       fgets                      00000001800440ec f   libucrt:fgets.obj
 0001:0004330c       fseek                      000000018004430c f   libucrt:fseek.obj
 0001:00043814       _ftelli64_nolock           0000000180044814 f   libucrt:ftell.obj
 0001:0004381c       ftell                      000000018004481c f   libucrt:ftell.obj
 0001:000438c8       _fwrite_nolock             00000001800448c8 f   libucrt:fwrite.obj
 0001:00043a60       fwrite                     0000000180044a60 f   libucrt:fwrite.obj
 0001:00043c14       setvbuf                    0000000180044c14 f   libucrt:setvbuf.obj
 0001:00044040       __acrt_stdio_free_tmpfile_name_buffers_nolock 0000000180045040 f   libucrt:tmpfile.obj
 0001:000440c8       tmpfile                    00000001800450c8 f   libucrt:tmpfile.obj
 0001:0004412c       ??$is_overflow_condition@_K@__crt_strtox@@YA_NI_K@Z 000000018004512c f i libucrt:input.obj
 0001:0004415c       ??$parse_floating_point@V?$input_adapter_character_source@V?$stream_input_adapter@D@__crt_stdio_input@@@__crt_strtox@@M@__crt_strtox@@YA?AW4SLD_STATUS@@QEAU__crt_locale_pointers@@V?$input_adapter_character_source@V?$stream_input_adapter@D@__crt_stdio_input@@@0@QEAM@Z 000000018004515c f i libucrt:input.obj
 0001:00044204       ??$parse_floating_point@V?$input_adapter_character_source@V?$stream_input_adapter@D@__crt_stdio_input@@@__crt_strtox@@N@__crt_strtox@@YA?AW4SLD_STATUS@@QEAU__crt_locale_pointers@@V?$input_adapter_character_source@V?$stream_input_adapter@D@__crt_stdio_input@@@0@QEAN@Z 0000000180045204 f i libucrt:input.obj
 0001:000442ac       ??$parse_floating_point_from_source@V?$input_adapter_character_source@V?$stream_input_adapter@D@__crt_stdio_input@@@__crt_strtox@@@__crt_strtox@@YA?AW4floating_point_parse_result@0@QEAU__crt_locale_pointers@@AEAV?$input_adapter_character_source@V?$stream_input_adapter@D@__crt_stdio_input@@@0@AEAUfloating_point_string@0@@Z 00000001800452ac f i libucrt:input.obj
 0001:00044ac8       ??$parse_floating_point_possible_infinity@DV?$input_adapter_character_source@V?$stream_input_adapter@D@__crt_stdio_input@@@__crt_strtox@@_K@__crt_strtox@@YA?AW4floating_point_parse_result@0@AEADAEAV?$input_adapter_character_source@V?$stream_input_adapter@D@__crt_stdio_input@@@0@_K@Z 0000000180045ac8 f i libucrt:input.obj
 0001:00044d0c       ??$parse_floating_point_possible_nan@DV?$input_adapter_character_source@V?$stream_input_adapter@D@__crt_stdio_input@@@__crt_strtox@@_K@__crt_strtox@@YA?AW4floating_point_parse_result@0@AEADAEAV?$input_adapter_character_source@V?$stream_input_adapter@D@__crt_stdio_input@@@0@_K@Z 0000000180045d0c f i libucrt:input.obj
 0001:00044f84       ??$parse_floating_point_possible_nan_is_ind@DV?$input_adapter_character_source@V?$stream_input_adapter@D@__crt_stdio_input@@@__crt_strtox@@@__crt_strtox@@YA_NAEADAEAV?$input_adapter_character_source@V?$stream_input_adapter@D@__crt_stdio_input@@@0@@Z 0000000180045f84 f i libucrt:input.obj
 0001:00045018       ??$parse_floating_point_possible_nan_is_snan@DV?$input_adapter_character_source@V?$stream_input_adapter@D@__crt_stdio_input@@@__crt_strtox@@@__crt_strtox@@YA_NAEADAEAV?$input_adapter_character_source@V?$stream_input_adapter@D@__crt_stdio_input@@@0@@Z 0000000180046018 f i libucrt:input.obj
 0001:000450ac       ??$parse_floating_point_write_result@M@__crt_strtox@@YA?AW4SLD_STATUS@@W4floating_point_parse_result@0@AEBUfloating_point_string@0@QEAM@Z 00000001800460ac f i libucrt:input.obj
 0001:000451c4       ??$parse_floating_point_write_result@N@__crt_strtox@@YA?AW4SLD_STATUS@@W4floating_point_parse_result@0@AEBUfloating_point_string@0@QEAN@Z 00000001800461c4 f i libucrt:input.obj
 0001:000452ec       ??$parse_integer@_KV?$input_adapter_character_source@V?$stream_input_adapter@D@__crt_stdio_input@@@__crt_strtox@@@__crt_strtox@@YA_KQEAU__crt_locale_pointers@@V?$input_adapter_character_source@V?$stream_input_adapter@D@__crt_stdio_input@@@0@H_N@Z 00000001800462ec f i libucrt:input.obj
 0001:00045764       ??$process_floating_point_specifier_t@M@?$input_processor@DV?$stream_input_adapter@D@__crt_stdio_input@@@__crt_stdio_input@@AEAA_NXZ 0000000180046764 f i libucrt:input.obj
 0001:00045804       ??$process_floating_point_specifier_t@N@?$input_processor@DV?$stream_input_adapter@D@__crt_stdio_input@@@__crt_stdio_input@@AEAA_NXZ 0000000180046804 f i libucrt:input.obj
 0001:000458a4       ??$process_string_specifier_tchar@D@?$input_processor@DV?$stream_input_adapter@D@__crt_stdio_input@@@__crt_stdio_input@@AEAA_NW4conversion_mode@1@D@Z 00000001800468a4 f i libucrt:input.obj
 0001:00045a40       ??$process_string_specifier_tchar@_W@?$input_processor@DV?$stream_input_adapter@D@__crt_stdio_input@@@__crt_stdio_input@@AEAA_NW4conversion_mode@1@_W@Z 0000000180046a40 f i libucrt:input.obj
 0001:00045c14       ??$skip_whitespace@Vstream_input_adapter@__crt_stdio_input@@D@__crt_stdio_input@@YAHAEAV?$stream_input_adapter@D@0@QEAU__crt_locale_pointers@@@Z 0000000180046c14 f i libucrt:input.obj
 0001:00045e00       ?advance@?$format_string_parser@D@__crt_stdio_input@@QEAA_NXZ 0000000180046e00 f i libucrt:input.obj
 0001:00045fcc       ?as_double@floating_point_value@__crt_strtox@@QEBAAEANXZ 0000000180046fcc f i libucrt:input.obj
 0001:00046008       ?as_float@floating_point_value@__crt_strtox@@QEBAAEAMXZ 0000000180047008 f i libucrt:input.obj
 0001:00046044       ?assemble_floating_point_value@__crt_strtox@@YA?AW4SLD_STATUS@@_KH_N1AEBVfloating_point_value@1@@Z 0000000180047044 f i libucrt:input.obj
 0001:000463f8       ?assemble_floating_point_value_from_big_integer@__crt_strtox@@YA?AW4SLD_STATUS@@AEBUbig_integer@1@I_N1AEBVfloating_point_value@1@@Z 00000001800473f8 f i libucrt:input.obj
 0001:00046578       ?convert_decimal_string_to_floating_type_common@__crt_strtox@@YA?AW4SLD_STATUS@@AEBUfloating_point_string@1@AEBVfloating_point_value@1@@Z 0000000180047578 f i libucrt:input.obj
 0001:00048368       ?convert_hexadecimal_string_to_floating_type_common@__crt_strtox@@YA?AW4SLD_STATUS@@AEBUfloating_point_string@1@AEBVfloating_point_value@1@@Z 0000000180049368 f i libucrt:input.obj
 0001:00048420       ?divide@__crt_strtox@@YA_KAEAUbig_integer@1@AEBU21@@Z 0000000180049420 f i libucrt:input.obj
 0001:000488b4       ?length@?$format_string_parser@D@__crt_stdio_input@@QEBA_KXZ 00000001800498b4 f i libucrt:input.obj
 0001:00048950       ?process@?$input_processor@DV?$stream_input_adapter@D@__crt_stdio_input@@@__crt_stdio_input@@QEAAHXZ 0000000180049950 f i libucrt:input.obj
 0001:00048a34       ?process_conversion_specifier@?$input_processor@DV?$stream_input_adapter@D@__crt_stdio_input@@@__crt_stdio_input@@AEAA_NXZ 0000000180049a34 f i libucrt:input.obj
 0001:00048b50       ?process_floating_point_specifier@?$input_processor@DV?$stream_input_adapter@D@__crt_stdio_input@@@__crt_stdio_input@@AEAA_NXZ 0000000180049b50 f i libucrt:input.obj
 0001:00048bb4       ?process_integer_specifier@?$input_processor@DV?$stream_input_adapter@D@__crt_stdio_input@@@__crt_stdio_input@@AEAA_NI_N@Z 0000000180049bb4 f i libucrt:input.obj
 0001:00048c60       ?process_literal_character_tchar@?$input_processor@DV?$stream_input_adapter@D@__crt_stdio_input@@@__crt_stdio_input@@AEAA_ND@Z 0000000180049c60 f i libucrt:input.obj
 0001:00048cd4       ?process_state@?$input_processor@DV?$stream_input_adapter@D@__crt_stdio_input@@@__crt_stdio_input@@AEAA_NXZ 0000000180049cd4 f i libucrt:input.obj
 0001:00048d80       ?process_string_specifier@?$input_processor@DV?$stream_input_adapter@D@__crt_stdio_input@@@__crt_stdio_input@@AEAA_NW4conversion_mode@2@@Z 0000000180049d80 f i libucrt:input.obj
 0001:00048e00       ?scan_conversion_specifier@?$format_string_parser@D@__crt_stdio_input@@AEAA_NXZ 0000000180049e00 f i libucrt:input.obj
 0001:00048fc8       ?scan_optional_field_width@?$format_string_parser@D@__crt_stdio_input@@AEAA_NXZ 0000000180049fc8 f i libucrt:input.obj
 0001:00049070       ?scan_optional_length_modifier@?$format_string_parser@D@__crt_stdio_input@@AEAAXXZ 000000018004a070 f i libucrt:input.obj
 0001:0004919c       ?scan_scanset_range@?$format_string_parser@D@__crt_stdio_input@@AEAA_NXZ 000000018004a19c f i libucrt:input.obj
 0001:0004931c       ?write_character@?$input_processor@DV?$stream_input_adapter@D@__crt_stdio_input@@@__crt_stdio_input@@AEAA_NQEFA_W_KAEAPEFA_WAEA_KD@Z 000000018004a31c f i libucrt:input.obj
 0001:000493b0       ?write_integer@?$input_processor@DV?$stream_input_adapter@D@__crt_stdio_input@@@__crt_stdio_input@@AEAA_N_K@Z 000000018004a3b0 f i libucrt:input.obj
 0001:00049424       __stdio_common_vfscanf     000000018004a424 f   libucrt:input.obj
 0001:00049724       _wdupenv_s                 000000018004a724 f   libucrt:getenv.obj
 0001:00049744       _wgetenv                   000000018004a744 f   libucrt:getenv.obj
 0001:0004974c       _wsystem                   000000018004a74c f   libucrt:system.obj
 0001:00049888       wcscmp                     000000018004a888 f   libucrt:wcscmp.obj
 0001:000498c0       _initterm                  000000018004a8c0 f   libucrt:initterm.obj
 0001:00049924       _initterm_e                000000018004a924 f   libucrt:initterm.obj
 0001:00049964       _seh_filter_dll            000000018004a964 f   libucrt:exception_filter.obj
 0001:00049978       _seh_filter_exe            000000018004a978 f   libucrt:exception_filter.obj
 0001:00049d84       __acrt_initialize_thread_local_exit_callback 000000018004ad84 f   libucrt:exit.obj
 0001:00049d8c       _cexit                     000000018004ad8c f   libucrt:exit.obj
 0001:00049d9c       _exit                      000000018004ad9c f   libucrt:exit.obj
 0001:00049da8       _is_c_termination_complete 000000018004ada8 f   libucrt:exit.obj
 0001:00049f6c       __acrt_allocate_buffer_for_argv 000000018004af6c f   libucrt:argv_parsing.obj
 0001:00049fcc       _configure_narrow_argv     000000018004afcc f   libucrt:argv_parsing.obj
 0001:0004a578       __dcrt_get_or_create_wide_environment_nolock 000000018004b578 f   libucrt:environment_initialization.obj
 0001:0004a5b4       __dcrt_uninitialize_environments_nolock 000000018004b5b4 f   libucrt:environment_initialization.obj
 0001:0004a5ec       _initialize_narrow_environment 000000018004b5ec f   libucrt:environment_initialization.obj
 0001:0004a77c       _execute_onexit_table      000000018004b77c f   libucrt:onexit.obj
 0001:0004a7b8       _initialize_onexit_table   000000018004b7b8 f   libucrt:onexit.obj
 0001:0004a830       __acrt_uninitialize_command_line 000000018004b830 f   libucrt:argv_data.obj
 0001:0004a93c       __acrt_initialize          000000018004b93c f   libucrt:initialization.obj
 0001:0004a950       __acrt_thread_attach       000000018004b950 f   libucrt:initialization.obj
 0001:0004a964       __acrt_thread_detach       000000018004b964 f   libucrt:initialization.obj
 0001:0004a974       __acrt_uninitialize        000000018004b974 f   libucrt:initialization.obj
 0001:0004a9ac       __acrt_uninitialize_critical 000000018004b9ac f   libucrt:initialization.obj
 0001:0004a9bc       terminate                  000000018004b9bc f   libucrt:terminate.obj
 0001:0004abdc       strupr                     000000018004bbdc f   libucrt:strupr.obj
 0001:0004abdc       _strupr                    000000018004bbdc f   libucrt:strupr.obj
 0001:0004ac34       _strupr_s_l                000000018004bc34 f   libucrt:strupr.obj
 0001:0004ac80       strcpy_s                   000000018004bc80 f   libucrt:strcpy_s.obj
 0001:0004ace0       ??$parse_integer@KV?$c_string_character_source@D@__crt_strtox@@@__crt_strtox@@YAKQEAU__crt_locale_pointers@@V?$c_string_character_source@D@0@H_N@Z 000000018004bce0 f i libucrt:atox.obj
 0001:0004affc       ??$parse_integer@KV?$c_string_character_source@_W@__crt_strtox@@@__crt_strtox@@YAKQEAU__crt_locale_pointers@@V?$c_string_character_source@_W@0@H_N@Z 000000018004bffc f i libucrt:atox.obj
 0001:0004b6c0       ??$parse_integer@_KV?$c_string_character_source@D@__crt_strtox@@@__crt_strtox@@YA_KQEAU__crt_locale_pointers@@V?$c_string_character_source@D@0@H_N@Z 000000018004c6c0 f i libucrt:atox.obj
 0001:0004b9e4       abort                      000000018004c9e4 f   libucrt:abort.obj
 0001:0004ba3c       calloc                     000000018004ca3c f   libucrt:calloc.obj
 0001:0004ba44       wcsncmp                    000000018004ca44 f   libucrt:wcsncmp.obj
 0001:0004ba70       __acrt_call_reportfault    000000018004ca70 f   libucrt:invalid_parameter.obj
 0001:0004bbcc       __acrt_initialize_invalid_parameter_handler 000000018004cbcc f   libucrt:invalid_parameter.obj
 0001:0004bbd4       _invalid_parameter         000000018004cbd4 f   libucrt:invalid_parameter.obj
 0001:0004bc84       _invalid_parameter_noinfo  000000018004cc84 f   libucrt:invalid_parameter.obj
 0001:0004bca4       _invoke_watson             000000018004cca4 f   libucrt:invalid_parameter.obj
 0001:0004bd30       _tolower_l                 000000018004cd30 f   libucrt:tolower_toupper.obj
 0001:0004be70       tolower                    000000018004ce70 f   libucrt:tolower_toupper.obj
 0001:0004be9c       _free_base                 000000018004ce9c f   libucrt:free_base.obj
 0001:0004bedc       _malloc_base               000000018004cedc f   libucrt:malloc_base.obj
 0001:0004bf3c       strtol                     000000018004cf3c f   libucrt:strtox.obj
 0001:0004bf68       strtoull                   000000018004cf68 f   libucrt:strtox.obj
 0001:0004bf94       wcstol                     000000018004cf94 f   libucrt:strtox.obj
 0001:0004bfc0       _mbtowc_l                  000000018004cfc0 f   libucrt:mbtowc.obj
 0001:0004c108       mbtowc                     000000018004d108 f   libucrt:mbtowc.obj
 0001:0004c110       _wctomb_s_l                000000018004d110 f   libucrt:wctomb.obj
 0001:0004c294       wctomb_s                   000000018004d294 f   libucrt:wctomb.obj
 0001:0004c2a8       strnlen                    000000018004d2a8 f   libucrt:strnlen.obj
 0001:0004c3ec       wcsnlen                    000000018004d3ec f   libucrt:strnlen.obj
 0001:0004c92c       __acrt_freeptd             000000018004d92c f   libucrt:per_thread_data.obj
 0001:0004c970       __acrt_getptd              000000018004d970 f   libucrt:per_thread_data.obj
 0001:0004ca3c       __acrt_getptd_head         000000018004da3c f   libucrt:per_thread_data.obj
 0001:0004cae4       __acrt_getptd_noexit       000000018004dae4 f   libucrt:per_thread_data.obj
 0001:0004cbb4       __acrt_initialize_ptd      000000018004dbb4 f   libucrt:per_thread_data.obj
 0001:0004cbf0       __acrt_uninitialize_ptd    000000018004dbf0 f   libucrt:per_thread_data.obj
 0001:0004cc14       __acrt_update_locale_info  000000018004dc14 f   libucrt:locale_update.obj
 0001:0004cc48       __acrt_update_multibyte_info 000000018004dc48 f   libucrt:locale_update.obj
 0001:0004d638       __acrt_fp_format           000000018004e638 f   libucrt:cvt.obj
 0001:0004d8c0       _fileno                    000000018004e8c0 f   libucrt:fileno.obj
 0001:0004d8e8       _fputc_nolock              000000018004e8e8 f   libucrt:fputc.obj
 0001:0004d900       _get_printf_count_output   000000018004e900 f   libucrt:printf_count_output.obj
 0001:0004d918       __acrt_stdio_begin_temporary_buffering_nolock 000000018004e918 f   libucrt:_sftbuf.obj
 0001:0004d9e8       __acrt_stdio_end_temporary_buffering_nolock 000000018004e9e8 f   libucrt:_sftbuf.obj
 0001:0004da94       __acrt_set_locale_changed  000000018004ea94 f   libucrt:wsetlocale.obj
 0001:0004daa0       __acrt_uninitialize_locale 000000018004eaa0 f   libucrt:wsetlocale.obj
 0001:0004dcb8       __acrt_initialize_lowio    000000018004ecb8 f   libucrt:ioinit.obj
 0001:0004dcf4       __acrt_uninitialize_lowio  000000018004ecf4 f   libucrt:ioinit.obj
 0001:0004dd34       wcscpy_s                   000000018004ed34 f   libucrt:wcscpy_s.obj
 0001:0004dd9c       ?__acrt_stdio_allocate_stream@@YA?AV__crt_stdio_stream@@XZ 000000018004ed9c f   libucrt:stream.obj
 0001:0004ddf4       ?__acrt_stdio_free_stream@@YAXV__crt_stdio_stream@@@Z 000000018004edf4 f   libucrt:stream.obj
 0001:0004defc       ??$__acrt_stdio_parse_mode@_W@@YA?AU__acrt_stdio_stream_mode@@QEB_W@Z 000000018004eefc f i libucrt:openfile.obj
 0001:0004e1dc       _wopenfile                 000000018004f1dc f   libucrt:openfile.obj
 0001:0004e2ec       _close                     000000018004f2ec f   libucrt:close.obj
 0001:0004e390       _close_nolock              000000018004f390 f   libucrt:close.obj
 0001:0004e44c       __acrt_stdio_free_buffer_nolock 000000018004f44c f   libucrt:_freebuf.obj
 0001:0004e4a0       _get_fpsr                  000000018004f4a0 f   libucrt:fpsr.obj
 0001:0004e4b0       _set_fpsr                  000000018004f4b0 f   libucrt:fpsr.obj
 0001:0004e4ba       _fclrf                     000000018004f4ba f   libucrt:fpsr.obj
 0001:0004e4ce       _frnd                      000000018004f4ce f   libucrt:fpsr.obj
 0001:0004e4f0       _calloc_base               000000018004f4f0 f   libucrt:calloc_base.obj
 0001:0004e568       __sys_errlist              000000018004f568 f   libucrt:syserr.obj
 0001:0004e570       __sys_nerr                 000000018004f570 f   libucrt:syserr.obj
 0001:0004e578       strncpy_s                  000000018004f578 f   libucrt:strncpy_s.obj
 0001:0004e824       __acrt_AppPolicyGetProcessTerminationMethodInternal 000000018004f824 f   libucrt:winapi_thunks.obj
 0001:0004e874       __acrt_AreFileApisANSI     000000018004f874 f   libucrt:winapi_thunks.obj
 0001:0004e8b0       __acrt_CompareStringEx     000000018004f8b0 f   libucrt:winapi_thunks.obj
 0001:0004e98c       __acrt_FlsAlloc            000000018004f98c f   libucrt:winapi_thunks.obj
 0001:0004e9d4       __acrt_FlsFree             000000018004f9d4 f   libucrt:winapi_thunks.obj
 0001:0004ea1c       __acrt_FlsGetValue         000000018004fa1c f   libucrt:winapi_thunks.obj
 0001:0004ea64       __acrt_FlsSetValue         000000018004fa64 f   libucrt:winapi_thunks.obj
 0001:0004eab8       __acrt_InitializeCriticalSectionEx 000000018004fab8 f   libucrt:winapi_thunks.obj
 0001:0004eb1c       __acrt_LCMapStringEx       000000018004fb1c f   libucrt:winapi_thunks.obj
 0001:0004ebf8       __acrt_LocaleNameToLCID    000000018004fbf8 f   libucrt:winapi_thunks.obj
 0001:0004ec48       __acrt_initialize_winapi_thunks 000000018004fc48 f   libucrt:winapi_thunks.obj
 0001:0004ec90       __acrt_uninitialize_winapi_thunks 000000018004fc90 f   libucrt:winapi_thunks.obj
 0001:0004ecd4       _fcloseall                 000000018004fcd4 f   libucrt:closeall.obj
 0001:0004f324       _read                      0000000180050324 f   libucrt:read.obj
 0001:0004f440       _read_nolock               0000000180050440 f   libucrt:read.obj
 0001:0004f8cc       __acrt_stdio_refill_and_read_narrow_nolock 00000001800508cc f   libucrt:_filbuf.obj
 0001:0004fd98       _lseek                     0000000180050d98 f   libucrt:lseek.obj
 0001:0004fda0       _lseeki64                  0000000180050da0 f   libucrt:lseek.obj
 0001:0004fda8       _lseeki64_nolock           0000000180050da8 f   libucrt:lseek.obj
 0001:0004fdb0       __acrt_stdio_allocate_buffer_nolock 0000000180050db0 f   libucrt:_getbuf.obj
 0001:0004fe14       __acrt_GetStringTypeW      0000000180050e14 f   libucrt:getstringtypew.obj
 0001:0004fe1c       __pctype_func              0000000180050e1c f   libucrt:ctype.obj
 0001:0004fe4c       _isctype_l                 0000000180050e4c f   libucrt:isctype.obj
 0001:0004ff5c       _towlower_l                0000000180050f5c f   libucrt:towlower.obj
 0001:00050020       _recalloc                  0000000180051020 f   libucrt:recalloc.obj
 0001:00050028       _recalloc_base             0000000180051028 f   libucrt:recalloc.obj
 0001:000500c0       wcscat_s                   00000001800510c0 f   libucrt:wcscat_s.obj
 0001:00050140       _cwait                     0000000180051140 f   libucrt:wait.obj
 0001:000501f8       __acrt_wgetpath            00000001800511f8 f   libucrt:getpath.obj
 0001:000502d4       __acrt_initialize_locks    00000001800512d4 f   libucrt:locks.obj
 0001:0005031c       __acrt_lock                000000018005131c f   libucrt:locks.obj
 0001:00050338       __acrt_uninitialize_locks  0000000180051338 f   libucrt:locks.obj
 0001:00050370       __acrt_unlock              0000000180051370 f   libucrt:locks.obj
 0001:0005038c       _waccess_s                 000000018005138c f   libucrt:waccess.obj
 0001:00050438       _pipe                      0000000180051438 f   libucrt:pipe.obj
 0001:000507b0       _wfdopen                   00000001800517b0 f   libucrt:fdopen.obj
 0001:00050844       _commit                    0000000180051844 f   libucrt:commit.obj
 0001:00050e90       _write                     0000000180051e90 f   libucrt:write.obj
 0001:00050f7c       _write_nolock              0000000180051f7c f   libucrt:write.obj
 0001:000513a0       __acrt_stdio_flush_and_write_narrow_nolock 00000001800523a0 f   libucrt:_flsbuf.obj
 0001:00051588       _ui64toa_s                 0000000180052588 f   libucrt:xtoa.obj
 0001:0005159c       _strdup                    000000018005259c f   libucrt:strdup.obj
 0001:00051614       __acrt_GetTempPathA        0000000180052614 f   libucrt:gettemppath.obj
 0001:00051da4       _sopen_nolock              0000000180052da4 f   libucrt:open.obj
 0001:00051e34       _sopen_s                   0000000180052e34 f   libucrt:open.obj
 0001:00051e68       _wsopen_nolock             0000000180052e68 f   libucrt:open.obj
 0001:00052254       _wsopen_s                  0000000180053254 f   libucrt:open.obj
 0001:00052288       __acrt_uninitialize_tmpfile 0000000180053288 f   libucrt:rmtmp.obj
 0001:0005229c       _rmtmp                     000000018005329c f   libucrt:rmtmp.obj
 0001:00052330       fegetround                 0000000180053330 f   libucrt:fegetround.obj
 0001:00052344       _wcsnicoll                 0000000180053344 f   libucrt:wcsnicol.obj
 0001:000523d8       _wcsnicoll_l               00000001800533d8 f   libucrt:wcsnicol.obj
 0001:00052c8c       _wspawnve                  0000000180053c8c f   libucrt:spawnv.obj
 0001:00052fd0       _wspawnvpe                 0000000180053fd0 f   libucrt:spawnvp.obj
 0001:00052fd8       __acrt_get_process_end_policy 0000000180053fd8 f   libucrt:win_policies.obj
 0001:00053578       __acrt_expand_narrow_argv_wildcards 0000000180054578 f   libucrt:argv_wildcards.obj
 0001:00053cc0       __acrt_initialize_multibyte 0000000180054cc0 f   libucrt:mbctype.obj
 0001:00053d20       __acrt_update_thread_multibyte_data 0000000180054d20 f   libucrt:mbctype.obj
 0001:00053d3c       _setmbcp_nolock            0000000180054d3c f   libucrt:mbctype.obj
 0001:00054074       _ismbblead                 0000000180055074 f   libucrt:ismbbyte.obj
 0001:00054088       __acrt_initialize_command_line 0000000180055088 f   libucrt:argv_data.obj
 0001:000540b0       __dcrt_get_narrow_environment_from_os 00000001800550b0 f   libucrt:get_environment_from_os.obj
 0001:000541b4       __dcrt_get_wide_environment_from_os 00000001800551b4 f   libucrt:get_environment_from_os.obj
 0001:00054668       __dcrt_set_variable_in_wide_environment_nolock 0000000180055668 f   libucrt:setenv.obj
 0001:00054670       __acrt_initialize_heap     0000000180055670 f   libucrt:heap_handle.obj
 0001:0005468c       __acrt_uninitialize_heap   000000018005568c f   libucrt:heap_handle.obj
 0001:00054698       __acrt_execute_initializers 0000000180055698 f   libucrt:shared_initialization.obj
 0001:00054718       __acrt_execute_uninitializers 0000000180055718 f   libucrt:shared_initialization.obj
 0001:00054754       __acrt_initialize_new_handler 0000000180055754 f   libucrt:new_handler.obj
 0001:0005475c       _callnewh                  000000018005575c f   libucrt:new_handler.obj
 0001:0005478c       _query_new_handler         000000018005578c f   libucrt:new_handler.obj
 0001:00054808       __acrt_get_sigabrt_handler 0000000180055808 f   libucrt:signal.obj
 0001:00054838       __acrt_initialize_signal_handlers 0000000180055838 f   libucrt:signal.obj
 0001:00054858       raise                      0000000180055858 f   libucrt:signal.obj
 0001:00054acc       __acrt_has_user_matherr    0000000180055acc f   libucrt:matherr.obj
 0001:00054aec       __acrt_initialize_user_matherr 0000000180055aec f   libucrt:matherr.obj
 0001:00054af4       __acrt_invoke_user_matherr 0000000180055af4 f   libucrt:matherr.obj
 0001:00054e3c       __acrt_LCMapStringA        0000000180055e3c f   libucrt:lcmapstringa.obj
 0001:00054ed4       _isleadbyte_l              0000000180055ed4 f i libucrt:_wctype.obj
 0001:00054f14       _query_new_mode            0000000180055f14 f   libucrt:new_mode.obj
 0001:00054f1c       __acrt_MultiByteToWideChar 0000000180055f1c f   libucrt:multibytetowidechar.obj
 0001:00054f24       __acrt_WideCharToMultiByte 0000000180055f24 f   libucrt:widechartomultibyte.obj
 0001:00054f2c       __acrt_add_locale_ref      0000000180055f2c f   libucrt:locale_refcounting.obj
 0001:00054fb8       __acrt_free_locale         0000000180055fb8 f   libucrt:locale_refcounting.obj
 0001:00055130       __acrt_locale_add_lc_time_reference 0000000180056130 f   libucrt:locale_refcounting.obj
 0001:00055158       __acrt_locale_free_lc_time_if_unreferenced 0000000180056158 f   libucrt:locale_refcounting.obj
 0001:00055190       __acrt_locale_release_lc_time_reference 0000000180056190 f   libucrt:locale_refcounting.obj
 0001:000551b8       __acrt_release_locale_ref  00000001800561b8 f   libucrt:locale_refcounting.obj
 0001:00055260       __acrt_update_thread_locale_data 0000000180056260 f   libucrt:locale_refcounting.obj
 0001:000552d0       _updatetlocinfoEx_nolock   00000001800562d0 f   libucrt:locale_refcounting.obj
 0001:00055338       __acrt_fp_strflt_to_string 0000000180056338 f   libucrt:_fptostr.obj
 0001:000553f8       __acrt_fltout              00000001800563f8 f   libucrt:cfout.obj
 0001:0005674c       _isatty                    000000018005774c f   libucrt:isatty.obj
 0001:000567ac       __acrt_locale_free_monetary 00000001800577ac f   libucrt:initmon.obj
 0001:000568b8       __acrt_locale_free_numeric 00000001800578b8 f   libucrt:initnum.obj
 0001:00056978       __acrt_locale_free_time    0000000180057978 f   libucrt:inittime.obj
 0001:00056a80       __acrt_GetStringTypeA      0000000180057a80 f   libucrt:getstringtypea.obj
 0001:00056c10       __acrt_lowio_create_handle_array 0000000180057c10 f   libucrt:osfinfo.obj
 0001:00056ca8       __acrt_lowio_destroy_handle_array 0000000180057ca8 f   libucrt:osfinfo.obj
 0001:00056cf8       __acrt_lowio_ensure_fh_exists 0000000180057cf8 f   libucrt:osfinfo.obj
 0001:00056da0       __acrt_lowio_lock_fh       0000000180057da0 f   libucrt:osfinfo.obj
 0001:00056dc4       __acrt_lowio_set_os_handle 0000000180057dc4 f   libucrt:osfinfo.obj
 0001:00056e84       __acrt_lowio_unlock_fh     0000000180057e84 f   libucrt:osfinfo.obj
 0001:00056ea8       _alloc_osfhnd              0000000180057ea8 f   libucrt:osfinfo.obj
 0001:00056fcc       _free_osfhnd               0000000180057fcc f   libucrt:osfinfo.obj
 0001:00057088       _get_osfhandle             0000000180058088 f   libucrt:osfinfo.obj
 0001:00057100       _wcsnicmp                  0000000180058100 f   libucrt:wcsnicmp.obj
 0001:00057198       _wcsnicmp_l                0000000180058198 f   libucrt:wcsnicmp.obj
 0001:0005737c       __acrt_DownlevelLocaleNameToLCID 000000018005837c f   libucrt:lcidtoname_downlevel.obj
 0001:000573b0       __acrt_LCMapStringW        00000001800583b0 f   libucrt:lcmapstringw.obj
 0001:00057438       _msize                     0000000180058438 f   libucrt:msize.obj
 0001:00057440       _msize_base                0000000180058440 f   libucrt:msize.obj
 0001:0005747c       _realloc_base              000000018005847c f   libucrt:realloc_base.obj
 0001:000574f8       __acrt_copy_path_to_wide_string 00000001800584f8 f   libucrt:string_utilities.obj
 0001:000575f0       _get_fmode                 00000001800585f0 f   libucrt:setmode.obj
 0001:00057620       _setmode_nolock            0000000180058620 f   libucrt:setmode.obj
 0001:00057700       _putwch_nolock             0000000180058700 f   libucrt:putwch.obj
 0001:0005773c       _chsize_nolock             000000018005873c f   libucrt:chsize.obj
 0001:000578b8       __acrt_fenv_get_common_round_control 00000001800588b8 f   libucrt:_fenvutils.obj
 0001:000578c4       __acrt_fenv_get_control    00000001800588c4 f   libucrt:_fenvutils.obj
 0001:000579c4       __acrt_fenv_get_status     00000001800589c4 f   libucrt:_fenvutils.obj
 0001:00057a1c       __acrt_fenv_set_control    0000000180058a1c f   libucrt:_fenvutils.obj
 0001:00057b64       __acrt_fenv_set_status     0000000180058b64 f   libucrt:_fenvutils.obj
 0001:00057be8       __acrt_CompareStringW      0000000180058be8 f   libucrt:comparestringw.obj
 0001:00058004       __acrt_pack_wide_command_line_and_environment 0000000180059004 f   libucrt:cenvarg.obj
 0001:00058180       qsort                      0000000180059180 f   libucrt:qsort.obj
 0001:00058530       _mbsdec                    0000000180059530 f   libucrt:mbsdec.obj
 0001:00058538       _mbsdec_l                  0000000180059538 f   libucrt:mbsdec.obj
 0001:000585e0       __strncnt                  00000001800595e0 f   libucrt:strncnt.obj
 0001:000585f8       fegetenv                   00000001800595f8 f   libucrt:fegetenv.obj
 0001:00058618       fesetenv                   0000000180059618 f   libucrt:fesetenv.obj
 0001:00058668       feholdexcept               0000000180059668 f   libucrt:feholdexcept.obj
 0001:000586b8       ceil                       00000001800596b8 f   libucrt:ceil.obj
 0001:00058780       log10                      0000000180059780 f   libucrt:log10.obj
 0001:00058d2c       _query_app_type            0000000180059d2c f   libucrt:report_runtime_error.obj
 0001:00058d34       __dcrt_lowio_ensure_console_output_initialized 0000000180059d34 f   libucrt:initcon.obj
 0001:00058d88       __dcrt_terminate_console_output 0000000180059d88 f   libucrt:initcon.obj
 0001:00058da4       __dcrt_write_console_w     0000000180059da4 f   libucrt:initcon.obj
 0001:00058f88       _handle_error              0000000180059f88 f   libucrt:libm_error.obj
 0001:000590b0       _handle_nan                000000018005a0b0 f   libucrt:libm_error.obj
 0001:000590d0       __acrt_initialize_fma3     000000018005a0d0 f   libucrt:fma3_available.obj
 0001:00059140       _log10_special             000000018005a140 f   libucrt:log_special.obj
 0001:000591f8       _raise_exc                 000000018005a1f8 f   libucrt:fpexcept.obj
 0001:00059220       _raise_exc_ex              000000018005a220 f   libucrt:fpexcept.obj
 0001:00059528       _set_errno_from_matherr    000000018005a528 f   libucrt:fpexcept.obj
 0001:00059558       _clrfp                     000000018005a558 f   libucrt:fpctrl.obj
 0001:00059578       _ctrlfp                    000000018005a578 f   libucrt:fpctrl.obj
 0001:000595f4       _set_statfp                000000018005a5f4 f   libucrt:fpctrl.obj
 0001:00059614       _statfp                    000000018005a614 f   libucrt:fpctrl.obj
 0001:00059625       IsProcessorFeaturePresent  000000018005a625 f   kernel32:KERNEL32.dll
 0001:0005962b       RtlUnwindEx                000000018005a62b f   kernel32:KERNEL32.dll
 0001:00059640       _FindPESection             000000018005a640 f   LIBCMT:pesect.obj
 0001:00059690       _IsNonwritableInCurrentImage 000000018005a690 f   LIBCMT:pesect.obj
 0001:000596e0       _ValidateImageBase         000000018005a6e0 f   LIBCMT:pesect.obj
 0001:00059710       __GSHandlerCheck           000000018005a710 f   LIBCMT:_gshandler_.obj
 0001:00059730       __GSHandlerCheckCommon     000000018005a730 f   LIBCMT:_gshandler_.obj
 0001:000597a0       __security_check_cookie    000000018005a7a0 f   LIBCMT:_amdsecgs_.obj
 0001:000597c4       __raise_securityfailure    000000018005a7c4 f   LIBCMT:gs_report.obj
 0001:000597f8       __report_gsfailure         000000018005a7f8 f   LIBCMT:gs_report.obj
 0001:000598cc       __report_rangecheckfailure 000000018005a8cc f   LIBCMT:gs_report.obj
 0001:000598e0       __report_securityfailure   000000018005a8e0 f   LIBCMT:gs_report.obj
 0001:00059a60       __GSHandlerCheck_SEH       000000018005aa60 f   LIBCMT:_gshandlerseh_.obj
 0001:00059b00       _guard_dispatch_icall_nop  000000018005ab00 f   LIBCMT:_guard_dispatch_.obj
 0002:00000000       Keys                       000000018005f000     flags.obj
 0002:00001650       VirtualKeyStrings          0000000180060650     service.obj
 0002:000054fc       _fltused                   00000001800644fc     LIBCMT:fltused.obj
 0002:00005500       __scrt_native_dllmain_reason 0000000180064500     LIBCMT:utility.obj
 0002:00005508       __security_cookie          0000000180064508     LIBCMT:gs_cookie.obj
 0002:00005510       __security_cookie_complement 0000000180064510     LIBCMT:gs_cookie.obj
 0002:00005518       __isa_available            0000000180064518     LIBCMT:_cpu_disp_.obj
 0002:0000551c       __isa_enabled              000000018006451c     LIBCMT:_cpu_disp_.obj
 0002:00005520       __memcpy_nt_iters          0000000180064520     LIBCMT:_cpu_disp_.obj
 0002:00005550       _iob                       0000000180064550     libucrt:_file.obj
 0002:00005660       __abort_behavior           0000000180064660     libucrt:abort.obj
 0002:00005670       __acrt_initial_locale_data 0000000180064670     libucrt:nlsdata.obj
 0002:000057c8       __acrt_initial_locale_pointers 00000001800647c8     libucrt:nlsdata.obj
 0002:000057d8       __acrt_wide_c_locale_string 00000001800647d8     libucrt:nlsdata.obj
 0002:000057e0       __badioinfo                00000001800647e0     libucrt:ioinit.obj
 0002:00005820       _lookuptrailbytes          0000000180064820     libucrt:read.obj
 0002:00005920       _pwctype                   0000000180064920     libucrt:ctype.obj
 0002:00005930       __acrt_initial_multibyte_data 0000000180064930     libucrt:mbctype.obj
 0002:00005e70       __globallocalestatus       0000000180064e70     libucrt:glstatus.obj
 0002:00005e80       __acrt_lconv_c             0000000180064e80     libucrt:localeconv.obj
 0002:00005f18       __acrt_lconv_static_decimal 0000000180064f18     libucrt:localeconv.obj
 0002:00005f1c       __acrt_lconv_static_W_decimal 0000000180064f1c     libucrt:localeconv.obj
 0002:00005f60       ?__type_info_root_node@@3U__type_info_node@@A 0000000180064f60     LIBCMT:tncleanup.obj
 0002:00005f70       __scrt_current_native_startup_state 0000000180064f70     LIBCMT:utility.obj
 0002:00005f78       __scrt_native_startup_lock 0000000180064f78     LIBCMT:utility.obj
 0002:00005fb4       __scrt_debugger_hook_flag  0000000180064fb4     LIBCMT:utility_desktop.obj
 0002:00005fb8       __favor                    0000000180064fb8     LIBCMT:_cpu_disp_.obj
 0002:00005fc0       ?m_pGetParameter@UnDecorator@@0P6APEADJ@ZEA 0000000180064fc0     libvcruntime:undname.obj
 0002:00005fc8       ?m_CHPENameOffset@UnDecorator@@0KA 0000000180064fc8     libvcruntime:undname.obj
 0002:00005fcc       ?m_recursionLevel@UnDecorator@@0KA 0000000180064fcc     libvcruntime:undname.obj
 0002:00005fd0       ?pArgList@UnDecorator@@0PEAVReplicator@@EA 0000000180064fd0     libvcruntime:undname.obj
 0002:00005fd8       ?pZNameList@UnDecorator@@0PEAVReplicator@@EA 0000000180064fd8     libvcruntime:undname.obj
 0002:00005fe0       ?pTemplateArgList@UnDecorator@@0PEAVReplicator@@EA 0000000180064fe0     libvcruntime:undname.obj
 0002:00005fe8       ?gName@UnDecorator@@0PEBDEB 0000000180064fe8     libvcruntime:undname.obj
 0002:00005ff0       ?name@UnDecorator@@0PEBDEB 0000000180064ff0     libvcruntime:undname.obj
 0002:00005ff8       ?disableFlags@UnDecorator@@0KA 0000000180064ff8     libvcruntime:undname.obj
 0002:00005ffc       ?fExplicitTemplateParams@UnDecorator@@0_NA 0000000180064ffc     libvcruntime:undname.obj
 0002:00005ffd       ?fGetTemplateArgumentList@UnDecorator@@0_NA 0000000180064ffd     libvcruntime:undname.obj
 0002:00006118       __pPurecall                0000000180065118     libvcruntime:purevirt_data.obj
 0002:00006120       ?__WinRTOutOfMemoryExceptionCallback@@3P6APEAXXZEA 0000000180065120     libvcruntime:ehhelpers.obj
 0002:00006128       _nstream                   0000000180065128     libucrt:_file.obj
 0002:00006130       __piob                     0000000180065130     libucrt:_file.obj
 0002:00006138       _cflush                    0000000180065138     libucrt:_file.obj
 0002:00006190       ?c_exit_complete@?1???R<lambda_6e4b09c48022b2350581041d5f6b0c4c>@@QEBA@XZ@4_NA 0000000180065190     libucrt:exit.obj
 0002:000062a8       _environ_table             00000001800652a8     libucrt:environment_initialization.obj
 0002:000062b0       _wenviron_table            00000001800652b0     libucrt:environment_initialization.obj
 0002:000062b8       __dcrt_initial_wide_environment 00000001800652b8     libucrt:environment_initialization.obj
 0002:000062c0       __dcrt_initial_narrow_environment 00000001800652c0     libucrt:environment_initialization.obj
 0002:000062c8       __acrt_atexit_table        00000001800652c8     libucrt:onexit.obj
 0002:000062e0       __acrt_at_quick_exit_table 00000001800652e0     libucrt:onexit.obj
 0002:00006308       __acrt_stdout_buffer       0000000180065308     libucrt:_sftbuf.obj
 0002:00006310       __acrt_stderr_buffer       0000000180065310     libucrt:_sftbuf.obj
 0002:00006318       __acrt_locale_changed_data 0000000180065318     libucrt:wsetlocale.obj
 0002:00006320       __acrt_current_locale_data 0000000180065320     libucrt:nlsdata.obj
 0002:00006330       __pioinfo                  0000000180065330     libucrt:ioinit.obj
 0002:00006730       _nhandle                   0000000180065730     libucrt:ioinit.obj
 0002:00006b24       _commode                   0000000180065b24     libucrt:ncommode.obj
 0002:00006b28       __acrt_current_multibyte_data 0000000180065b28     libucrt:mbctype.obj
 0002:00006b30       _mbctype                   0000000180065b30     libucrt:mbctype.obj
 0002:00006b38       _mbcasemap                 0000000180065b38     libucrt:mbctype.obj
 0002:00006b48       __argc                     0000000180065b48     libucrt:argv_data.obj
 0002:00006b50       __argv                     0000000180065b50     libucrt:argv_data.obj
 0002:00006b58       __wargv                    0000000180065b58     libucrt:argv_data.obj
 0002:00006b60       _acmdln                    0000000180065b60     libucrt:argv_data.obj
 0002:00006b68       _wcmdln                    0000000180065b68     libucrt:argv_data.obj
 0002:00006b70       _pgmptr                    0000000180065b70     libucrt:argv_data.obj
 0002:00006b78       __acrt_heap                0000000180065b78     libucrt:heap_handle.obj
 0002:00006bb4       __acrt_lconv_static_null   0000000180065bb4     libucrt:localeconv.obj
 0002:00006bb8       __acrt_lconv_static_W_null 0000000180065bb8     libucrt:localeconv.obj
 0002:00006bbc       _umaskval                  0000000180065bbc     libucrt:umask.obj
 0002:00006bc4       _fmode                     0000000180065bc4     libucrt:txtmode.obj
 0002:00006bc8       __fma3_is_available        0000000180065bc8     libucrt:fma3_available.obj
 0002:00006bcc       __use_fma3_lib             0000000180065bcc     libucrt:fma3_available.obj
 0002:00007140       EnumCP                     0000000180066140     <common>
 0002:00007150       ?_OptionsStorage@?1??__local_stdio_scanf_options@@9@9 0000000180066150     <common>
 0002:00007158       ?_OptionsStorage@?1??__local_stdio_printf_options@@9@9 0000000180066158     <common>
 0002:00007160       __scrt_ucrt_dll_is_in_use  0000000180066160     <common>
 0002:00007168       __dyn_tls_init_callback    0000000180066168     <common>
 0004:00000000       __imp_RegEnumValueW        000000018006b000     advapi32:ADVAPI32.dll
 0004:00000008       __imp_RegEnumKeyExW        000000018006b008     advapi32:ADVAPI32.dll
 0004:00000010       __imp_RegDeleteValueW      000000018006b010     advapi32:ADVAPI32.dll
 0004:00000018       __imp_RegDeleteKeyW        000000018006b018     advapi32:ADVAPI32.dll
 0004:00000020       __imp_RegSetValueExW       000000018006b020     advapi32:ADVAPI32.dll
 0004:00000028       __imp_RegQueryValueExW     000000018006b028     advapi32:ADVAPI32.dll
 0004:00000030       __imp_RegOpenKeyExW        000000018006b030     advapi32:ADVAPI32.dll
 0004:00000038       __imp_RegCreateKeyExW      000000018006b038     advapi32:ADVAPI32.dll
 0004:00000040       __imp_RegCloseKey          000000018006b040     advapi32:ADVAPI32.dll
 0004:00000048       \177ADVAPI32_NULL_THUNK_DATA 000000018006b048     advapi32:ADVAPI32.dll
 0004:00000050       __imp_GetConsoleScreenBufferInfo 000000018006b050     kernel32:KERNEL32.dll
 0004:00000058       __imp_FreeLibrary          000000018006b058     kernel32:KERNEL32.dll
 0004:00000060       __imp_GetModuleFileNameW   000000018006b060     kernel32:KERNEL32.dll
 0004:00000068       __imp_LoadLibraryW         000000018006b068     kernel32:KERNEL32.dll
 0004:00000070       __imp_SetCurrentDirectoryW 000000018006b070     kernel32:KERNEL32.dll
 0004:00000078       __imp_GetCurrentDirectoryW 000000018006b078     kernel32:KERNEL32.dll
 0004:00000080       __imp_SearchPathW          000000018006b080     kernel32:KERNEL32.dll
 0004:00000088       __imp_GetDriveTypeW        000000018006b088     kernel32:KERNEL32.dll
 0004:00000090       __imp_GetLogicalDriveStringsW 000000018006b090     kernel32:KERNEL32.dll
 0004:00000098       __imp_SetFileAttributesW   000000018006b098     kernel32:KERNEL32.dll
 0004:000000a0       __imp_OutputDebugStringW   000000018006b0a0     kernel32:KERNEL32.dll
 0004:000000a8       __imp_GetLastError         000000018006b0a8     kernel32:KERNEL32.dll
 0004:000000b0       __imp_Sleep                000000018006b0b0     kernel32:KERNEL32.dll
 0004:000000b8       __imp_GlobalMemoryStatusEx 000000018006b0b8     kernel32:KERNEL32.dll
 0004:000000c0       __imp_FormatMessageW       000000018006b0c0     kernel32:KERNEL32.dll
 0004:000000c8       __imp_MultiByteToWideChar  000000018006b0c8     kernel32:KERNEL32.dll
 0004:000000d0       __imp_WideCharToMultiByte  000000018006b0d0     kernel32:KERNEL32.dll
 0004:000000d8       __imp_GetACP               000000018006b0d8     kernel32:KERNEL32.dll
 0004:000000e0       __imp_GetOEMCP             000000018006b0e0     kernel32:KERNEL32.dll
 0004:000000e8       __imp_GetProcAddress       000000018006b0e8     kernel32:KERNEL32.dll
 0004:000000f0       __imp_EnumSystemCodePagesW 000000018006b0f0     kernel32:KERNEL32.dll
 0004:000000f8       __imp_SetEnvironmentVariableW 000000018006b0f8     kernel32:KERNEL32.dll
 0004:00000100       __imp_CreateDirectoryW     000000018006b100     kernel32:KERNEL32.dll
 0004:00000108       __imp_DeleteFileW          000000018006b108     kernel32:KERNEL32.dll
 0004:00000110       __imp_FileTimeToLocalFileTime 000000018006b110     kernel32:KERNEL32.dll
 0004:00000118       __imp_FindClose            000000018006b118     kernel32:KERNEL32.dll
 0004:00000120       __imp_FindFirstFileW       000000018006b120     kernel32:KERNEL32.dll
 0004:00000128       __imp_RemoveDirectoryW     000000018006b128     kernel32:KERNEL32.dll
 0004:00000130       __imp_GetSystemTimeAsFileTime 000000018006b130     kernel32:KERNEL32.dll
 0004:00000138       __imp_GetModuleHandleW     000000018006b138     kernel32:KERNEL32.dll
 0004:00000140       __imp_CopyFileW            000000018006b140     kernel32:KERNEL32.dll
 0004:00000148       __imp_MoveFileExW          000000018006b148     kernel32:KERNEL32.dll
 0004:00000150       __imp_FileTimeToSystemTime 000000018006b150     kernel32:KERNEL32.dll
 0004:00000158       __imp_SystemTimeToFileTime 000000018006b158     kernel32:KERNEL32.dll
 0004:00000160       __imp_CompareStringW       000000018006b160     kernel32:KERNEL32.dll
 0004:00000168       __imp_PeekConsoleInputW    000000018006b168     kernel32:KERNEL32.dll
 0004:00000170       __imp_ReadConsoleInputW    000000018006b170     kernel32:KERNEL32.dll
 0004:00000178       __imp_SetEndOfFile         000000018006b178     kernel32:KERNEL32.dll
 0004:00000180       __imp_HeapReAlloc          000000018006b180     kernel32:KERNEL32.dll
 0004:00000188       __imp_HeapSize             000000018006b188     kernel32:KERNEL32.dll
 0004:00000190       __imp_GetModuleHandleA     000000018006b190     kernel32:KERNEL32.dll
 0004:00000198       __imp_DeleteTimerQueueTimer 000000018006b198     kernel32:KERNEL32.dll
 0004:000001a0       __imp_ChangeTimerQueueTimer 000000018006b1a0     kernel32:KERNEL32.dll
 0004:000001a8       __imp_CreateTimerQueueTimer 000000018006b1a8     kernel32:KERNEL32.dll
 0004:000001b0       __imp_CreateTimerQueue     000000018006b1b0     kernel32:KERNEL32.dll
 0004:000001b8       __imp_GetFileAttributesW   000000018006b1b8     kernel32:KERNEL32.dll
 0004:000001c0       __imp_GetEnvironmentVariableW 000000018006b1c0     kernel32:KERNEL32.dll
 0004:000001c8       __imp_GetStdHandle         000000018006b1c8     kernel32:KERNEL32.dll
 0004:000001d0       __imp_GetCPInfoExW         000000018006b1d0     kernel32:KERNEL32.dll
 0004:000001d8       __imp_DeleteTimerQueueEx   000000018006b1d8     kernel32:KERNEL32.dll
 0004:000001e0       __imp_SetStdHandle         000000018006b1e0     kernel32:KERNEL32.dll
 0004:000001e8       __imp_GetProcessHeap       000000018006b1e8     kernel32:KERNEL32.dll
 0004:000001f0       __imp_FreeEnvironmentStringsW 000000018006b1f0     kernel32:KERNEL32.dll
 0004:000001f8       __imp_GetEnvironmentStringsW 000000018006b1f8     kernel32:KERNEL32.dll
 0004:00000200       __imp_GetCommandLineW      000000018006b200     kernel32:KERNEL32.dll
 0004:00000208       __imp_GetCommandLineA      000000018006b208     kernel32:KERNEL32.dll
 0004:00000210       __imp_GetCPInfo            000000018006b210     kernel32:KERNEL32.dll
 0004:00000218       __imp_IsValidCodePage      000000018006b218     kernel32:KERNEL32.dll
 0004:00000220       __imp_FindNextFileA        000000018006b220     kernel32:KERNEL32.dll
 0004:00000228       __imp_FindFirstFileExA     000000018006b228     kernel32:KERNEL32.dll
 0004:00000230       __imp_CreateFileW          000000018006b230     kernel32:KERNEL32.dll
 0004:00000238       __imp_GetConsoleCP         000000018006b238     kernel32:KERNEL32.dll
 0004:00000240       __imp_WriteFile            000000018006b240     kernel32:KERNEL32.dll
 0004:00000248       __imp_FlushFileBuffers     000000018006b248     kernel32:KERNEL32.dll
 0004:00000250       __imp_CreatePipe           000000018006b250     kernel32:KERNEL32.dll
 0004:00000258       __imp_GetFileAttributesExW 000000018006b258     kernel32:KERNEL32.dll
 0004:00000260       __imp_GetExitCodeProcess   000000018006b260     kernel32:KERNEL32.dll
 0004:00000268       __imp_WaitForSingleObject  000000018006b268     kernel32:KERNEL32.dll
 0004:00000270       __imp_GetStringTypeW       000000018006b270     kernel32:KERNEL32.dll
 0004:00000278       __imp_SetFilePointerEx     000000018006b278     kernel32:KERNEL32.dll
 0004:00000280       __imp_ReadConsoleW         000000018006b280     kernel32:KERNEL32.dll
 0004:00000288       __imp_GetConsoleMode       000000018006b288     kernel32:KERNEL32.dll
 0004:00000290       __imp_LCMapStringW         000000018006b290     kernel32:KERNEL32.dll
 0004:00000298       __imp_GetFileType          000000018006b298     kernel32:KERNEL32.dll
 0004:000002a0       __imp_HeapAlloc            000000018006b2a0     kernel32:KERNEL32.dll
 0004:000002a8       __imp_HeapFree             000000018006b2a8     kernel32:KERNEL32.dll
 0004:000002b0       __imp_GetModuleFileNameA   000000018006b2b0     kernel32:KERNEL32.dll
 0004:000002b8       __imp_GetModuleHandleExW   000000018006b2b8     kernel32:KERNEL32.dll
 0004:000002c0       __imp_TerminateProcess     000000018006b2c0     kernel32:KERNEL32.dll
 0004:000002c8       __imp_ExitProcess          000000018006b2c8     kernel32:KERNEL32.dll
 0004:000002d0       __imp_GetTempPathW         000000018006b2d0     kernel32:KERNEL32.dll
 0004:000002d8       __imp_ReadFile             000000018006b2d8     kernel32:KERNEL32.dll
 0004:000002e0       __imp_CreateProcessW       000000018006b2e0     kernel32:KERNEL32.dll
 0004:000002e8       __imp_GetCurrentProcess    000000018006b2e8     kernel32:KERNEL32.dll
 0004:000002f0       __imp_DuplicateHandle      000000018006b2f0     kernel32:KERNEL32.dll
 0004:000002f8       __imp_CloseHandle          000000018006b2f8     kernel32:KERNEL32.dll
 0004:00000300       __imp_RaiseException       000000018006b300     kernel32:KERNEL32.dll
 0004:00000308       __imp_LoadLibraryExW       000000018006b308     kernel32:KERNEL32.dll
 0004:00000310       __imp_TlsFree              000000018006b310     kernel32:KERNEL32.dll
 0004:00000318       __imp_TlsSetValue          000000018006b318     kernel32:KERNEL32.dll
 0004:00000320       __imp_TlsGetValue          000000018006b320     kernel32:KERNEL32.dll
 0004:00000328       __imp_TlsAlloc             000000018006b328     kernel32:KERNEL32.dll
 0004:00000330       __imp_InitializeCriticalSectionAndSpinCount 000000018006b330     kernel32:KERNEL32.dll
 0004:00000338       __imp_DeleteCriticalSection 000000018006b338     kernel32:KERNEL32.dll
 0004:00000340       __imp_WriteConsoleW        000000018006b340     kernel32:KERNEL32.dll
 0004:00000348       __imp_LeaveCriticalSection 000000018006b348     kernel32:KERNEL32.dll
 0004:00000350       __imp_EnterCriticalSection 000000018006b350     kernel32:KERNEL32.dll
 0004:00000358       __imp_SetLastError         000000018006b358     kernel32:KERNEL32.dll
 0004:00000360       __imp_InterlockedFlushSList 000000018006b360     kernel32:KERNEL32.dll
 0004:00000368       __imp_RtlUnwindEx          000000018006b368     kernel32:KERNEL32.dll
 0004:00000370       __imp_IsProcessorFeaturePresent 000000018006b370     kernel32:KERNEL32.dll
 0004:00000378       __imp_GetStartupInfoW      000000018006b378     kernel32:KERNEL32.dll
 0004:00000380       __imp_SetUnhandledExceptionFilter 000000018006b380     kernel32:KERNEL32.dll
 0004:00000388       __imp_UnhandledExceptionFilter 000000018006b388     kernel32:KERNEL32.dll
 0004:00000390       __imp_IsDebuggerPresent    000000018006b390     kernel32:KERNEL32.dll
 0004:00000398       __imp_RtlVirtualUnwind     000000018006b398     kernel32:KERNEL32.dll
 0004:000003a0       __imp_RtlLookupFunctionEntry 000000018006b3a0     kernel32:KERNEL32.dll
 0004:000003a8       __imp_RtlCaptureContext    000000018006b3a8     kernel32:KERNEL32.dll
 0004:000003b0       __imp_InitializeSListHead  000000018006b3b0     kernel32:KERNEL32.dll
 0004:000003b8       __imp_GetCurrentThreadId   000000018006b3b8     kernel32:KERNEL32.dll
 0004:000003c0       __imp_GetCurrentProcessId  000000018006b3c0     kernel32:KERNEL32.dll
 0004:000003c8       __imp_QueryPerformanceCounter 000000018006b3c8     kernel32:KERNEL32.dll
 0004:000003d0       \177KERNEL32_NULL_THUNK_DATA 000000018006b3d0     kernel32:KERNEL32.dll
 0004:000003d8       __imp_RpcStringFreeA       000000018006b3d8     rpcrt4:RPCRT4.dll
 0004:000003e0       __imp_UuidCreate           000000018006b3e0     rpcrt4:RPCRT4.dll
 0004:000003e8       __imp_UuidToStringA        000000018006b3e8     rpcrt4:RPCRT4.dll
 0004:000003f0       __imp_UuidFromStringA      000000018006b3f0     rpcrt4:RPCRT4.dll
 0004:000003f8       \177RPCRT4_NULL_THUNK_DATA 000000018006b3f8     rpcrt4:RPCRT4.dll
 0004:00000400       __imp_ShellExecuteW        000000018006b400     shell32:SHELL32.dll
 0004:00000408       __imp_SHGetFolderPathW     000000018006b408     shell32:SHELL32.dll
 0004:00000410       \177SHELL32_NULL_THUNK_DATA 000000018006b410     shell32:SHELL32.dll
 0004:00000418       __imp_GetKeyState          000000018006b418     user32:USER32.dll
 0004:00000420       \177USER32_NULL_THUNK_DATA 000000018006b420     user32:USER32.dll
 0004:00000428       __imp_luaL_gsub            000000018006b428     lua51:lua51.dll
 0004:00000430       __imp_lua_isuserdata       000000018006b430     lua51:lua51.dll
 0004:00000438       __imp_lua_iscfunction      000000018006b438     lua51:lua51.dll
 0004:00000440       __imp_luaL_checkoption     000000018006b440     lua51:lua51.dll
 0004:00000448       __imp_lua_tocfunction      000000018006b448     lua51:lua51.dll
 0004:00000450       __imp_luaL_prepbuffer      000000018006b450     lua51:lua51.dll
 0004:00000458       __imp_luaL_checkstack      000000018006b458     lua51:lua51.dll
 0004:00000460       __imp_lua_dump             000000018006b460     lua51:lua51.dll
 0004:00000468       __imp_luaL_typerror        000000018006b468     lua51:lua51.dll
 0004:00000470       __imp_lua_setallocf        000000018006b470     lua51:lua51.dll
 0004:00000478       __imp_lua_getallocf        000000018006b478     lua51:lua51.dll
 0004:00000480       __imp_lua_next             000000018006b480     lua51:lua51.dll
 0004:00000488       __imp_lua_setfenv          000000018006b488     lua51:lua51.dll
 0004:00000490       __imp_lua_rawset           000000018006b490     lua51:lua51.dll
 0004:00000498       __imp_lua_settable         000000018006b498     lua51:lua51.dll
 0004:000004a0       __imp_lua_getfenv          000000018006b4a0     lua51:lua51.dll
 0004:000004a8       __imp_lua_rawget           000000018006b4a8     lua51:lua51.dll
 0004:000004b0       __imp_luaopen_debug        000000018006b4b0     lua51:lua51.dll
 0004:000004b8       __imp_luaopen_math         000000018006b4b8     lua51:lua51.dll
 0004:000004c0       __imp_luaopen_string       000000018006b4c0     lua51:lua51.dll
 0004:000004c8       __imp_luaopen_os           000000018006b4c8     lua51:lua51.dll
 0004:000004d0       __imp_luaopen_table        000000018006b4d0     lua51:lua51.dll
 0004:000004d8       __imp_luaopen_base         000000018006b4d8     lua51:lua51.dll
 0004:000004e0       __imp_luaL_checktype       000000018006b4e0     lua51:lua51.dll
 0004:000004e8       __imp_lua_getinfo          000000018006b4e8     lua51:lua51.dll
 0004:000004f0       __imp_lua_getstack         000000018006b4f0     lua51:lua51.dll
 0004:000004f8       __imp_luaL_error           000000018006b4f8     lua51:lua51.dll
 0004:00000500       __imp_luaL_checkudata      000000018006b500     lua51:lua51.dll
 0004:00000508       __imp_luaL_optinteger      000000018006b508     lua51:lua51.dll
 0004:00000510       __imp_luaL_optlstring      000000018006b510     lua51:lua51.dll
 0004:00000518       __imp_luaL_checklstring    000000018006b518     lua51:lua51.dll
 0004:00000520       __imp_lua_checkstack       000000018006b520     lua51:lua51.dll
 0004:00000528       __imp_lua_replace          000000018006b528     lua51:lua51.dll
 0004:00000530       __imp_luaL_pushresult      000000018006b530     lua51:lua51.dll
 0004:00000538       __imp_luaL_addlstring      000000018006b538     lua51:lua51.dll
 0004:00000540       __imp_luaL_buffinit        000000018006b540     lua51:lua51.dll
 0004:00000548       __imp_lua_concat           000000018006b548     lua51:lua51.dll
 0004:00000550       __imp_lua_typename         000000018006b550     lua51:lua51.dll
 0004:00000558       __imp_lua_load             000000018006b558     lua51:lua51.dll
 0004:00000560       __imp_lua_pushfstring      000000018006b560     lua51:lua51.dll
 0004:00000568       __imp_luaL_loadstring      000000018006b568     lua51:lua51.dll
 0004:00000570       __imp_luaL_unref           000000018006b570     lua51:lua51.dll
 0004:00000578       __imp_luaL_ref             000000018006b578     lua51:lua51.dll
 0004:00000580       __imp_lua_gc               000000018006b580     lua51:lua51.dll
 0004:00000588       __imp_lua_pcall            000000018006b588     lua51:lua51.dll
 0004:00000590       __imp_lua_call             000000018006b590     lua51:lua51.dll
 0004:00000598       __imp_lua_rawseti          000000018006b598     lua51:lua51.dll
 0004:000005a0       __imp_lua_setfield         000000018006b5a0     lua51:lua51.dll
 0004:000005a8       __imp_lua_createtable      000000018006b5a8     lua51:lua51.dll
 0004:000005b0       __imp_lua_rawgeti          000000018006b5b0     lua51:lua51.dll
 0004:000005b8       __imp_lua_gettable         000000018006b5b8     lua51:lua51.dll
 0004:000005c0       __imp_lua_pushlightuserdata 000000018006b5c0     lua51:lua51.dll
 0004:000005c8       __imp_lua_pushcclosure     000000018006b5c8     lua51:lua51.dll
 0004:000005d0       __imp_lua_pushlstring      000000018006b5d0     lua51:lua51.dll
 0004:000005d8       __imp_lua_pushinteger      000000018006b5d8     lua51:lua51.dll
 0004:000005e0       __imp_lua_objlen           000000018006b5e0     lua51:lua51.dll
 0004:000005e8       __imp_lua_toboolean        000000018006b5e8     lua51:lua51.dll
 0004:000005f0       __imp_lua_tointeger        000000018006b5f0     lua51:lua51.dll
 0004:000005f8       __imp_lua_isstring         000000018006b5f8     lua51:lua51.dll
 0004:00000600       __imp_lua_isnumber         000000018006b600     lua51:lua51.dll
 0004:00000608       __imp_lua_insert           000000018006b608     lua51:lua51.dll
 0004:00000610       __imp_lua_remove           000000018006b610     lua51:lua51.dll
 0004:00000618       __imp_lua_pushvalue        000000018006b618     lua51:lua51.dll
 0004:00000620       __imp_luaL_newmetatable    000000018006b620     lua51:lua51.dll
 0004:00000628       __imp_luaL_checkinteger    000000018006b628     lua51:lua51.dll
 0004:00000630       __imp_luaL_argerror        000000018006b630     lua51:lua51.dll
 0004:00000638       __imp_luaL_register        000000018006b638     lua51:lua51.dll
 0004:00000640       __imp_lua_setmetatable     000000018006b640     lua51:lua51.dll
 0004:00000648       __imp_lua_getmetatable     000000018006b648     lua51:lua51.dll
 0004:00000650       __imp_lua_newuserdata      000000018006b650     lua51:lua51.dll
 0004:00000658       __imp_lua_getfield         000000018006b658     lua51:lua51.dll
 0004:00000660       __imp_lua_pushboolean      000000018006b660     lua51:lua51.dll
 0004:00000668       __imp_lua_pushstring       000000018006b668     lua51:lua51.dll
 0004:00000670       __imp_lua_pushnumber       000000018006b670     lua51:lua51.dll
 0004:00000678       __imp_lua_pushnil          000000018006b678     lua51:lua51.dll
 0004:00000680       __imp_lua_touserdata       000000018006b680     lua51:lua51.dll
 0004:00000688       __imp_lua_tolstring        000000018006b688     lua51:lua51.dll
 0004:00000690       __imp_lua_tonumber         000000018006b690     lua51:lua51.dll
 0004:00000698       __imp_lua_rawequal         000000018006b698     lua51:lua51.dll
 0004:000006a0       __imp_lua_type             000000018006b6a0     lua51:lua51.dll
 0004:000006a8       __imp_lua_settop           000000018006b6a8     lua51:lua51.dll
 0004:000006b0       __imp_lua_gettop           000000018006b6b0     lua51:lua51.dll
 0004:000006b8       __imp_luaL_findtable       000000018006b6b8     lua51:lua51.dll
 0004:000006c0       __imp_luaL_checkany        000000018006b6c0     lua51:lua51.dll
 0004:000006c8       __imp_luaL_optnumber       000000018006b6c8     lua51:lua51.dll
 0004:000006d0       __imp_lua_error            000000018006b6d0     lua51:lua51.dll
 0004:000006d8       __imp_luaL_checknumber     000000018006b6d8     lua51:lua51.dll
 0004:000006e0       __imp_luaL_addvalue        000000018006b6e0     lua51:lua51.dll
 0004:000006e8       \177lua51_NULL_THUNK_DATA  000000018006b6e8     lua51:lua51.dll
 0004:000006f0       __guard_check_icall_fptr   000000018006b6f0     LIBCMT:guard_support.obj
 0004:000006f8       __guard_dispatch_icall_fptr 000000018006b6f8     LIBCMT:guard_support.obj
 0004:00000700       __IMPORT_DESCRIPTOR_KERNEL32 000000018006b700     kernel32:KERNEL32.dll
 0004:00000714       __IMPORT_DESCRIPTOR_USER32 000000018006b714     user32:USER32.dll
 0004:00000728       __IMPORT_DESCRIPTOR_ADVAPI32 000000018006b728     advapi32:ADVAPI32.dll
 0004:0000073c       __IMPORT_DESCRIPTOR_SHELL32 000000018006b73c     shell32:SHELL32.dll
 0004:00000750       __IMPORT_DESCRIPTOR_lua51  000000018006b750     lua51:lua51.dll
 0004:00000764       __IMPORT_DESCRIPTOR_RPCRT4 000000018006b764     rpcrt4:RPCRT4.dll
 0004:00000778       __NULL_IMPORT_DESCRIPTOR   000000018006b778     kernel32:KERNEL32.dll

 entry point at        0001:0003b49c

 Static symbols

 0001:00000080       funcs                      0000000180001080     bit64.obj
 0001:000001a0       metamethods                00000001800011a0     bit64.obj
 0001:00000360       FCF_FG_4BIT                0000000180001360     exported.obj
 0001:00000368       FCF_BG_4BIT                0000000180001368     exported.obj
 0001:00000370       FCF_4BITMASK               0000000180001370     exported.obj
 0001:00000378       FCF_RAWATTR_MASK           0000000180001378     exported.obj
 0001:00000380       FCF_EXTENDEDFLAGS          0000000180001380     exported.obj
 0001:00000388       FCF_FG_BOLD                0000000180001388     exported.obj
 0001:00000390       FCF_FG_ITALIC              0000000180001390     exported.obj
 0001:00000398       FCF_FG_UNDERLINE           0000000180001398     exported.obj
 0001:000003a0       FCF_STYLEMASK              00000001800013a0     exported.obj
 0001:000003a8       FCF_NONE                   00000001800013a8     exported.obj
 0001:000003b0       CDF_NONE                   00000001800013b0     exported.obj
 0001:000003b8       FMSG_WARNING               00000001800013b8     exported.obj
 0001:000003c0       FMSG_ERRORTYPE             00000001800013c0     exported.obj
 0001:000003c8       FMSG_KEEPBACKGROUND        00000001800013c8     exported.obj
 0001:000003d0       FMSG_LEFTALIGN             00000001800013d0     exported.obj
 0001:000003d8       FMSG_ALLINONE              00000001800013d8     exported.obj
 0001:000003e0       FMSG_MB_OK                 00000001800013e0     exported.obj
 0001:000003e8       FMSG_MB_OKCANCEL           00000001800013e8     exported.obj
 0001:000003f0       FMSG_MB_ABORTRETRYIGNORE   00000001800013f0     exported.obj
 0001:000003f8       FMSG_MB_YESNO              00000001800013f8     exported.obj
 0001:00000400       FMSG_MB_YESNOCANCEL        0000000180001400     exported.obj
 0001:00000408       FMSG_MB_RETRYCANCEL        0000000180001408     exported.obj
 0001:00000410       FMSG_NONE                  0000000180001410     exported.obj
 0001:00000418       DIF_BOXCOLOR               0000000180001418     exported.obj
 0001:00000420       DIF_GROUP                  0000000180001420     exported.obj
 0001:00000428       DIF_LEFTTEXT               0000000180001428     exported.obj
 0001:00000430       DIF_MOVESELECT             0000000180001430     exported.obj
 0001:00000438       DIF_SHOWAMPERSAND          0000000180001438     exported.obj
 0001:00000440       DIF_CENTERGROUP            0000000180001440     exported.obj
 0001:00000448       DIF_NOBRACKETS             0000000180001448     exported.obj
 0001:00000450       DIF_MANUALADDHISTORY       0000000180001450     exported.obj
 0001:00000458       DIF_SEPARATOR              0000000180001458     exported.obj
 0001:00000460       DIF_SEPARATOR2             0000000180001460     exported.obj
 0001:00000468       DIF_EDITOR                 0000000180001468     exported.obj
 0001:00000470       DIF_LISTNOAMPERSAND        0000000180001470     exported.obj
 0001:00000478       DIF_LISTNOBOX              0000000180001478     exported.obj
 0001:00000480       DIF_HISTORY                0000000180001480     exported.obj
 0001:00000488       DIF_BTNNOCLOSE             0000000180001488     exported.obj
 0001:00000490       DIF_CENTERTEXT             0000000180001490     exported.obj
 0001:00000498       DIF_SEPARATORUSER          0000000180001498     exported.obj
 0001:000004a0       DIF_SETSHIELD              00000001800014a0     exported.obj
 0001:000004a8       DIF_EDITEXPAND             00000001800014a8     exported.obj
 0001:000004b0       DIF_DROPDOWNLIST           00000001800014b0     exported.obj
 0001:000004b8       DIF_USELASTHISTORY         00000001800014b8     exported.obj
 0001:000004c0       DIF_MASKEDIT               00000001800014c0     exported.obj
 0001:000004c8       DIF_LISTTRACKMOUSE         00000001800014c8     exported.obj
 0001:000004d0       DIF_LISTTRACKMOUSEINFOCUS  00000001800014d0     exported.obj
 0001:000004d8       DIF_SELECTONENTRY          00000001800014d8     exported.obj
 0001:000004e0       DIF_3STATE                 00000001800014e0     exported.obj
 0001:000004e8       DIF_EDITPATH               00000001800014e8     exported.obj
 0001:000004f0       DIF_LISTWRAPMODE           00000001800014f0     exported.obj
 0001:000004f8       DIF_NOAUTOCOMPLETE         00000001800014f8     exported.obj
 0001:00000500       DIF_LISTAUTOHIGHLIGHT      0000000180001500     exported.obj
 0001:00000508       DIF_LISTNOCLOSE            0000000180001508     exported.obj
 0001:00000510       DIF_EDITPATHEXEC           0000000180001510     exported.obj
 0001:00000518       DIF_HIDDEN                 0000000180001518     exported.obj
 0001:00000520       DIF_READONLY               0000000180001520     exported.obj
 0001:00000528       DIF_NOFOCUS                0000000180001528     exported.obj
 0001:00000530       DIF_DISABLE                0000000180001530     exported.obj
 0001:00000538       DIF_DEFAULTBUTTON          0000000180001538     exported.obj
 0001:00000540       DIF_FOCUS                  0000000180001540     exported.obj
 0001:00000548       DIF_RIGHTTEXT              0000000180001548     exported.obj
 0001:00000550       DIF_WORDWRAP               0000000180001550     exported.obj
 0001:00000558       DIF_NONE                   0000000180001558     exported.obj
 0001:00000560       LIF_SELECTED               0000000180001560     exported.obj
 0001:00000568       LIF_CHECKED                0000000180001568     exported.obj
 0001:00000570       LIF_SEPARATOR              0000000180001570     exported.obj
 0001:00000578       LIF_DISABLE                0000000180001578     exported.obj
 0001:00000580       LIF_GRAYED                 0000000180001580     exported.obj
 0001:00000588       LIF_HIDDEN                 0000000180001588     exported.obj
 0001:00000590       LIF_DELETEUSERDATA         0000000180001590     exported.obj
 0001:00000598       LIF_NONE                   0000000180001598     exported.obj
 0001:000005a0       LIFIND_EXACTMATCH          00000001800015a0     exported.obj
 0001:000005a8       LIFIND_NONE                00000001800015a8     exported.obj
 0001:000005b0       LINFO_SHOWNOBOX            00000001800015b0     exported.obj
 0001:000005b8       LINFO_AUTOHIGHLIGHT        00000001800015b8     exported.obj
 0001:000005c0       LINFO_REVERSEHIGHLIGHT     00000001800015c0     exported.obj
 0001:000005c8       LINFO_WRAPMODE             00000001800015c8     exported.obj
 0001:000005d0       LINFO_SHOWAMPERSAND        00000001800015d0     exported.obj
 0001:000005d8       LINFO_NONE                 00000001800015d8     exported.obj
 0001:000005e0       FDLG_WARNING               00000001800015e0     exported.obj
 0001:000005e8       FDLG_SMALLDIALOG           00000001800015e8     exported.obj
 0001:000005f0       FDLG_NODRAWSHADOW          00000001800015f0     exported.obj
 0001:000005f8       FDLG_NODRAWPANEL           00000001800015f8     exported.obj
 0001:00000600       FDLG_KEEPCONSOLETITLE      0000000180001600     exported.obj
 0001:00000608       FDLG_NONMODAL              0000000180001608     exported.obj
 0001:00000610       FDLG_NONE                  0000000180001610     exported.obj
 0001:00000618       MIF_SELECTED               0000000180001618     exported.obj
 0001:00000620       MIF_CHECKED                0000000180001620     exported.obj
 0001:00000628       MIF_SEPARATOR              0000000180001628     exported.obj
 0001:00000630       MIF_DISABLE                0000000180001630     exported.obj
 0001:00000638       MIF_GRAYED                 0000000180001638     exported.obj
 0001:00000640       MIF_HIDDEN                 0000000180001640     exported.obj
 0001:00000648       MIF_NONE                   0000000180001648     exported.obj
 0001:00000650       FMENU_SHOWAMPERSAND        0000000180001650     exported.obj
 0001:00000658       FMENU_WRAPMODE             0000000180001658     exported.obj
 0001:00000660       FMENU_AUTOHIGHLIGHT        0000000180001660     exported.obj
 0001:00000668       FMENU_REVERSEAUTOHIGHLIGHT 0000000180001668     exported.obj
 0001:00000670       FMENU_CHANGECONSOLETITLE   0000000180001670     exported.obj
 0001:00000678       FMENU_NONE                 0000000180001678     exported.obj
 0001:00000680       PPIF_SELECTED              0000000180001680     exported.obj
 0001:00000688       PPIF_PROCESSDESCR          0000000180001688     exported.obj
 0001:00000690       PPIF_NONE                  0000000180001690     exported.obj
 0001:00000698       PFLAGS_SHOWHIDDEN          0000000180001698     exported.obj
 0001:000006a0       PFLAGS_HIGHLIGHT           00000001800016a0     exported.obj
 0001:000006a8       PFLAGS_REVERSESORTORDER    00000001800016a8     exported.obj
 0001:000006b0       PFLAGS_USESORTGROUPS       00000001800016b0     exported.obj
 0001:000006b8       PFLAGS_SELECTEDFIRST       00000001800016b8     exported.obj
 0001:000006c0       PFLAGS_REALNAMES           00000001800016c0     exported.obj
 0001:000006c8       PFLAGS_PANELLEFT           00000001800016c8     exported.obj
 0001:000006d0       PFLAGS_DIRECTORIESFIRST    00000001800016d0     exported.obj
 0001:000006d8       PFLAGS_USECRC32            00000001800016d8     exported.obj
 0001:000006e0       PFLAGS_PLUGIN              00000001800016e0     exported.obj
 0001:000006e8       PFLAGS_VISIBLE             00000001800016e8     exported.obj
 0001:000006f0       PFLAGS_FOCUS               00000001800016f0     exported.obj
 0001:000006f8       PFLAGS_ALTERNATIVENAMES    00000001800016f8     exported.obj
 0001:00000700       PFLAGS_SHORTCUT            0000000180001700     exported.obj
 0001:00000708       PFLAGS_NONE                0000000180001708     exported.obj
 0001:00000710       VF_NONMODAL                0000000180001710     exported.obj
 0001:00000718       VF_DELETEONCLOSE           0000000180001718     exported.obj
 0001:00000720       VF_ENABLE_F6               0000000180001720     exported.obj
 0001:00000728       VF_DISABLEHISTORY          0000000180001728     exported.obj
 0001:00000730       VF_IMMEDIATERETURN         0000000180001730     exported.obj
 0001:00000738       VF_DELETEONLYFILEONCLOSE   0000000180001738     exported.obj
 0001:00000740       VF_NONE                    0000000180001740     exported.obj
 0001:00000748       EF_NONMODAL                0000000180001748     exported.obj
 0001:00000750       EF_CREATENEW               0000000180001750     exported.obj
 0001:00000758       EF_ENABLE_F6               0000000180001758     exported.obj
 0001:00000760       EF_DISABLEHISTORY          0000000180001760     exported.obj
 0001:00000768       EF_DELETEONCLOSE           0000000180001768     exported.obj
 0001:00000770       EF_IMMEDIATERETURN         0000000180001770     exported.obj
 0001:00000778       EF_DELETEONLYFILEONCLOSE   0000000180001778     exported.obj
 0001:00000780       EF_LOCKED                  0000000180001780     exported.obj
 0001:00000788       EF_DISABLESAVEPOS          0000000180001788     exported.obj
 0001:00000790       EF_OPENMODE_MASK           0000000180001790     exported.obj
 0001:00000798       EF_OPENMODE_QUERY          0000000180001798     exported.obj
 0001:000007a0       EF_OPENMODE_NEWIFOPEN      00000001800017a0     exported.obj
 0001:000007a8       EF_OPENMODE_USEEXISTING    00000001800017a8     exported.obj
 0001:000007b0       EF_OPENMODE_BREAKIFOPEN    00000001800017b0     exported.obj
 0001:000007b8       EF_OPENMODE_RELOADIFOPEN   00000001800017b8     exported.obj
 0001:000007c0       EN_NONE                    00000001800017c0     exported.obj
 0001:000007c8       FHELP_NOSHOWERROR          00000001800017c8     exported.obj
 0001:000007d0       FHELP_SELFHELP             00000001800017d0     exported.obj
 0001:000007d8       FHELP_FARHELP              00000001800017d8     exported.obj
 0001:000007e0       FHELP_CUSTOMFILE           00000001800017e0     exported.obj
 0001:000007e8       FHELP_CUSTOMPATH           00000001800017e8     exported.obj
 0001:000007f0       FHELP_GUID                 00000001800017f0     exported.obj
 0001:000007f8       FHELP_USECONTENTS          00000001800017f8     exported.obj
 0001:00000800       FHELP_NONE                 0000000180001800     exported.obj
 0001:00000808       KMFLAGS_SILENTCHECK        0000000180001808     exported.obj
 0001:00000810       KMFLAGS_NOSENDKEYSTOPLUGINS 0000000180001810     exported.obj
 0001:00000818       KMFLAGS_ENABLEOUTPUT       0000000180001818     exported.obj
 0001:00000820       KMFLAGS_LANGMASK           0000000180001820     exported.obj
 0001:00000828       KMFLAGS_LUA                0000000180001828     exported.obj
 0001:00000830       KMFLAGS_MOONSCRIPT         0000000180001830     exported.obj
 0001:00000838       KMFLAGS_NONE               0000000180001838     exported.obj
 0001:00000840       AKMFLAGS_NONE              0000000180001840     exported.obj
 0001:00000848       FSETCLR_REDRAW             0000000180001848     exported.obj
 0001:00000850       FSETCLR_NONE               0000000180001850     exported.obj
 0001:00000858       WIF_MODIFIED               0000000180001858     exported.obj
 0001:00000860       WIF_CURRENT                0000000180001860     exported.obj
 0001:00000868       WIF_MODAL                  0000000180001868     exported.obj
 0001:00000870       WIF_NONE                   0000000180001870     exported.obj
 0001:00000878       VOPT_SAVEFILEPOSITION      0000000180001878     exported.obj
 0001:00000880       VOPT_AUTODETECTCODEPAGE    0000000180001880     exported.obj
 0001:00000888       VOPT_SHOWTITLEBAR          0000000180001888     exported.obj
 0001:00000890       VOPT_SHOWKEYBAR            0000000180001890     exported.obj
 0001:00000898       VOPT_SHOWSCROLLBAR         0000000180001898     exported.obj
 0001:000008a0       VOPT_QUICKVIEW             00000001800018a0     exported.obj
 0001:000008a8       VOPT_NONE                  00000001800018a8     exported.obj
 0001:000008b0       VSMFL_REDRAW               00000001800018b0     exported.obj
 0001:000008b8       VSMFL_NONE                 00000001800018b8     exported.obj
 0001:000008c0       VSP_NOREDRAW               00000001800018c0     exported.obj
 0001:000008c8       VSP_PERCENT                00000001800018c8     exported.obj
 0001:000008d0       VSP_RELATIVE               00000001800018d0     exported.obj
 0001:000008d8       VSP_NORETNEWPOS            00000001800018d8     exported.obj
 0001:000008e0       VSP_NONE                   00000001800018e0     exported.obj
 0001:000008e8       VMF_WRAP                   00000001800018e8     exported.obj
 0001:000008f0       VMF_WORDWRAP               00000001800018f0     exported.obj
 0001:000008f8       VMF_NONE                   00000001800018f8     exported.obj
 0001:00000900       ECF_TABMARKFIRST           0000000180001900     exported.obj
 0001:00000908       ECF_TABMARKCURRENT         0000000180001908     exported.obj
 0001:00000910       ECF_AUTODELETE             0000000180001910     exported.obj
 0001:00000918       ECF_NONE                   0000000180001918     exported.obj
 0001:00000920       FIB_ENABLEEMPTY            0000000180001920     exported.obj
 0001:00000928       FIB_PASSWORD               0000000180001928     exported.obj
 0001:00000930       FIB_EXPANDENV              0000000180001930     exported.obj
 0001:00000938       FIB_NOUSELASTHISTORY       0000000180001938     exported.obj
 0001:00000940       FIB_BUTTONS                0000000180001940     exported.obj
 0001:00000948       FIB_NOAMPERSAND            0000000180001948     exported.obj
 0001:00000950       FIB_EDITPATH               0000000180001950     exported.obj
 0001:00000958       FIB_EDITPATHEXEC           0000000180001958     exported.obj
 0001:00000960       FIB_NONE                   0000000180001960     exported.obj
 0001:00000968       FPF_LOADED                 0000000180001968     exported.obj
 0001:00000970       FPF_ANSI                   0000000180001970     exported.obj
 0001:00000978       FPF_NONE                   0000000180001978     exported.obj
 0001:00000980       PN_CMPNAME                 0000000180001980     exported.obj
 0001:00000988       PN_CMPNAMELIST             0000000180001988     exported.obj
 0001:00000990       PN_GENERATENAME            0000000180001990     exported.obj
 0001:00000998       PN_CHECKMASK               0000000180001998     exported.obj
 0001:000009a0       PN_SKIPPATH                00000001800019a0     exported.obj
 0001:000009a8       PN_SHOWERRORMESSAGE        00000001800019a8     exported.obj
 0001:000009b0       PN_NONE                    00000001800019b0     exported.obj
 0001:000009b8       XLAT_SWITCHKEYBLAYOUT      00000001800019b8     exported.obj
 0001:000009c0       XLAT_SWITCHKEYBBEEP        00000001800019c0     exported.obj
 0001:000009c8       XLAT_USEKEYBLAYOUTNAME     00000001800019c8     exported.obj
 0001:000009d0       XLAT_CONVERTALLCMDLINE     00000001800019d0     exported.obj
 0001:000009d8       XLAT_NONE                  00000001800019d8     exported.obj
 0001:000009e0       FRS_RETUPDIR               00000001800019e0     exported.obj
 0001:000009e8       FRS_RECUR                  00000001800019e8     exported.obj
 0001:000009f0       FRS_SCANSYMLINK            00000001800019f0     exported.obj
 0001:000009f8       FRS_NONE                   00000001800019f8     exported.obj
 0001:00000a00       MLF_SHOWERRMSG             0000000180001a00     exported.obj
 0001:00000a08       MLF_DONOTUPDATEPANEL       0000000180001a08     exported.obj
 0001:00000a10       MLF_HOLDTARGET             0000000180001a10     exported.obj
 0001:00000a18       MLF_NONE                   0000000180001a18     exported.obj
 0001:00000a20       FFFS_COMMAS                0000000180001a20     exported.obj
 0001:00000a28       FFFS_FLOATSIZE             0000000180001a28     exported.obj
 0001:00000a30       FFFS_SHOWBYTESINDEX        0000000180001a30     exported.obj
 0001:00000a38       FFFS_ECONOMIC              0000000180001a38     exported.obj
 0001:00000a40       FFFS_THOUSAND              0000000180001a40     exported.obj
 0001:00000a48       FFFS_MINSIZEINDEX          0000000180001a48     exported.obj
 0001:00000a50       FFFS_MINSIZEINDEX_MASK     0000000180001a50     exported.obj
 0001:00000a58       FFFS_NONE                  0000000180001a58     exported.obj
 0001:00000a60       PF_PRELOAD                 0000000180001a60     exported.obj
 0001:00000a68       PF_DISABLEPANELS           0000000180001a68     exported.obj
 0001:00000a70       PF_EDITOR                  0000000180001a70     exported.obj
 0001:00000a78       PF_VIEWER                  0000000180001a78     exported.obj
 0001:00000a80       PF_FULLCMDLINE             0000000180001a80     exported.obj
 0001:00000a88       PF_DIALOG                  0000000180001a88     exported.obj
 0001:00000a90       PF_NONE                    0000000180001a90     exported.obj
 0001:00000a98       IPLFLAGS_SEPARATOR         0000000180001a98     exported.obj
 0001:00000aa0       IPLFLAGS_NONE              0000000180001aa0     exported.obj
 0001:00000aa8       PMFLAGS_FULLSCREEN         0000000180001aa8     exported.obj
 0001:00000ab0       PMFLAGS_DETAILEDSTATUS     0000000180001ab0     exported.obj
 0001:00000ab8       PMFLAGS_ALIGNEXTENSIONS    0000000180001ab8     exported.obj
 0001:00000ac0       PMFLAGS_CASECONVERSION     0000000180001ac0     exported.obj
 0001:00000ac8       PMFLAGS_NONE               0000000180001ac8     exported.obj
 0001:00000ad0       OPIF_DISABLEFILTER         0000000180001ad0     exported.obj
 0001:00000ad8       OPIF_DISABLESORTGROUPS     0000000180001ad8     exported.obj
 0001:00000ae0       OPIF_DISABLEHIGHLIGHTING   0000000180001ae0     exported.obj
 0001:00000ae8       OPIF_ADDDOTS               0000000180001ae8     exported.obj
 0001:00000af0       OPIF_RAWSELECTION          0000000180001af0     exported.obj
 0001:00000af8       OPIF_REALNAMES             0000000180001af8     exported.obj
 0001:00000b00       OPIF_SHOWNAMESONLY         0000000180001b00     exported.obj
 0001:00000b08       OPIF_SHOWRIGHTALIGNNAMES   0000000180001b08     exported.obj
 0001:00000b10       OPIF_SHOWPRESERVECASE      0000000180001b10     exported.obj
 0001:00000b18       OPIF_COMPAREFATTIME        0000000180001b18     exported.obj
 0001:00000b20       OPIF_EXTERNALGET           0000000180001b20     exported.obj
 0001:00000b28       OPIF_EXTERNALPUT           0000000180001b28     exported.obj
 0001:00000b30       OPIF_EXTERNALDELETE        0000000180001b30     exported.obj
 0001:00000b38       OPIF_EXTERNALMKDIR         0000000180001b38     exported.obj
 0001:00000b40       OPIF_USEATTRHIGHLIGHTING   0000000180001b40     exported.obj
 0001:00000b48       OPIF_USECRC32              0000000180001b48     exported.obj
 0001:00000b50       OPIF_USEFREESIZE           0000000180001b50     exported.obj
 0001:00000b58       OPIF_SHORTCUT              0000000180001b58     exported.obj
 0001:00000b60       OPIF_NONE                  0000000180001b60     exported.obj
 0001:00000b68       OPM_SILENT                 0000000180001b68     exported.obj
 0001:00000b70       OPM_FIND                   0000000180001b70     exported.obj
 0001:00000b78       OPM_VIEW                   0000000180001b78     exported.obj
 0001:00000b80       OPM_EDIT                   0000000180001b80     exported.obj
 0001:00000b88       OPM_TOPLEVEL               0000000180001b88     exported.obj
 0001:00000b90       OPM_DESCR                  0000000180001b90     exported.obj
 0001:00000b98       OPM_QUICKVIEW              0000000180001b98     exported.obj
 0001:00000ba0       OPM_PGDN                   0000000180001ba0     exported.obj
 0001:00000ba8       OPM_COMMANDS               0000000180001ba8     exported.obj
 0001:00000bb0       OPM_NONE                   0000000180001bb0     exported.obj
 0001:00000bb8       FOSF_ACTIVE                0000000180001bb8     exported.obj
 0001:00000bc0       FOSF_NONE                  0000000180001bc0     exported.obj
 0001:00000bc8       PCIF_NONE                  0000000180001bc8     exported.obj
 0001:00000bd0       FarGuid                    0000000180001bd0     exported.obj
 0001:00000be0       PDF_DIALOGEVENTDRAWENABLE  0000000180001be0     exported.obj
 0001:00000be8       PDF_PROCESSINGERROR        0000000180001be8     exported.obj
 0001:000012e0       FCF_FG_4BIT                00000001800022e0     flags.obj
 0001:000012e8       FCF_BG_4BIT                00000001800022e8     flags.obj
 0001:000012f0       FCF_4BITMASK               00000001800022f0     flags.obj
 0001:000012f8       FCF_RAWATTR_MASK           00000001800022f8     flags.obj
 0001:00001300       FCF_EXTENDEDFLAGS          0000000180002300     flags.obj
 0001:00001308       FCF_FG_BOLD                0000000180002308     flags.obj
 0001:00001310       FCF_FG_ITALIC              0000000180002310     flags.obj
 0001:00001318       FCF_FG_UNDERLINE           0000000180002318     flags.obj
 0001:00001320       FCF_STYLEMASK              0000000180002320     flags.obj
 0001:00001328       FCF_NONE                   0000000180002328     flags.obj
 0001:00001330       CDF_NONE                   0000000180002330     flags.obj
 0001:00001338       FMSG_WARNING               0000000180002338     flags.obj
 0001:00001340       FMSG_ERRORTYPE             0000000180002340     flags.obj
 0001:00001348       FMSG_KEEPBACKGROUND        0000000180002348     flags.obj
 0001:00001350       FMSG_LEFTALIGN             0000000180002350     flags.obj
 0001:00001358       FMSG_ALLINONE              0000000180002358     flags.obj
 0001:00001360       FMSG_MB_OK                 0000000180002360     flags.obj
 0001:00001368       FMSG_MB_OKCANCEL           0000000180002368     flags.obj
 0001:00001370       FMSG_MB_ABORTRETRYIGNORE   0000000180002370     flags.obj
 0001:00001378       FMSG_MB_YESNO              0000000180002378     flags.obj
 0001:00001380       FMSG_MB_YESNOCANCEL        0000000180002380     flags.obj
 0001:00001388       FMSG_MB_RETRYCANCEL        0000000180002388     flags.obj
 0001:00001390       FMSG_NONE                  0000000180002390     flags.obj
 0001:00001398       DIF_BOXCOLOR               0000000180002398     flags.obj
 0001:000013a0       DIF_GROUP                  00000001800023a0     flags.obj
 0001:000013a8       DIF_LEFTTEXT               00000001800023a8     flags.obj
 0001:000013b0       DIF_MOVESELECT             00000001800023b0     flags.obj
 0001:000013b8       DIF_SHOWAMPERSAND          00000001800023b8     flags.obj
 0001:000013c0       DIF_CENTERGROUP            00000001800023c0     flags.obj
 0001:000013c8       DIF_NOBRACKETS             00000001800023c8     flags.obj
 0001:000013d0       DIF_MANUALADDHISTORY       00000001800023d0     flags.obj
 0001:000013d8       DIF_SEPARATOR              00000001800023d8     flags.obj
 0001:000013e0       DIF_SEPARATOR2             00000001800023e0     flags.obj
 0001:000013e8       DIF_EDITOR                 00000001800023e8     flags.obj
 0001:000013f0       DIF_LISTNOAMPERSAND        00000001800023f0     flags.obj
 0001:000013f8       DIF_LISTNOBOX              00000001800023f8     flags.obj
 0001:00001400       DIF_HISTORY                0000000180002400     flags.obj
 0001:00001408       DIF_BTNNOCLOSE             0000000180002408     flags.obj
 0001:00001410       DIF_CENTERTEXT             0000000180002410     flags.obj
 0001:00001418       DIF_SEPARATORUSER          0000000180002418     flags.obj
 0001:00001420       DIF_SETSHIELD              0000000180002420     flags.obj
 0001:00001428       DIF_EDITEXPAND             0000000180002428     flags.obj
 0001:00001430       DIF_DROPDOWNLIST           0000000180002430     flags.obj
 0001:00001438       DIF_USELASTHISTORY         0000000180002438     flags.obj
 0001:00001440       DIF_MASKEDIT               0000000180002440     flags.obj
 0001:00001448       DIF_LISTTRACKMOUSE         0000000180002448     flags.obj
 0001:00001450       DIF_LISTTRACKMOUSEINFOCUS  0000000180002450     flags.obj
 0001:00001458       DIF_SELECTONENTRY          0000000180002458     flags.obj
 0001:00001460       DIF_3STATE                 0000000180002460     flags.obj
 0001:00001468       DIF_EDITPATH               0000000180002468     flags.obj
 0001:00001470       DIF_LISTWRAPMODE           0000000180002470     flags.obj
 0001:00001478       DIF_NOAUTOCOMPLETE         0000000180002478     flags.obj
 0001:00001480       DIF_LISTAUTOHIGHLIGHT      0000000180002480     flags.obj
 0001:00001488       DIF_LISTNOCLOSE            0000000180002488     flags.obj
 0001:00001490       DIF_EDITPATHEXEC           0000000180002490     flags.obj
 0001:00001498       DIF_HIDDEN                 0000000180002498     flags.obj
 0001:000014a0       DIF_READONLY               00000001800024a0     flags.obj
 0001:000014a8       DIF_NOFOCUS                00000001800024a8     flags.obj
 0001:000014b0       DIF_DISABLE                00000001800024b0     flags.obj
 0001:000014b8       DIF_DEFAULTBUTTON          00000001800024b8     flags.obj
 0001:000014c0       DIF_FOCUS                  00000001800024c0     flags.obj
 0001:000014c8       DIF_RIGHTTEXT              00000001800024c8     flags.obj
 0001:000014d0       DIF_WORDWRAP               00000001800024d0     flags.obj
 0001:000014d8       DIF_NONE                   00000001800024d8     flags.obj
 0001:000014e0       LIF_SELECTED               00000001800024e0     flags.obj
 0001:000014e8       LIF_CHECKED                00000001800024e8     flags.obj
 0001:000014f0       LIF_SEPARATOR              00000001800024f0     flags.obj
 0001:000014f8       LIF_DISABLE                00000001800024f8     flags.obj
 0001:00001500       LIF_GRAYED                 0000000180002500     flags.obj
 0001:00001508       LIF_HIDDEN                 0000000180002508     flags.obj
 0001:00001510       LIF_DELETEUSERDATA         0000000180002510     flags.obj
 0001:00001518       LIF_NONE                   0000000180002518     flags.obj
 0001:00001520       LIFIND_EXACTMATCH          0000000180002520     flags.obj
 0001:00001528       LIFIND_NONE                0000000180002528     flags.obj
 0001:00001530       LINFO_SHOWNOBOX            0000000180002530     flags.obj
 0001:00001538       LINFO_AUTOHIGHLIGHT        0000000180002538     flags.obj
 0001:00001540       LINFO_REVERSEHIGHLIGHT     0000000180002540     flags.obj
 0001:00001548       LINFO_WRAPMODE             0000000180002548     flags.obj
 0001:00001550       LINFO_SHOWAMPERSAND        0000000180002550     flags.obj
 0001:00001558       LINFO_NONE                 0000000180002558     flags.obj
 0001:00001560       FDLG_WARNING               0000000180002560     flags.obj
 0001:00001568       FDLG_SMALLDIALOG           0000000180002568     flags.obj
 0001:00001570       FDLG_NODRAWSHADOW          0000000180002570     flags.obj
 0001:00001578       FDLG_NODRAWPANEL           0000000180002578     flags.obj
 0001:00001580       FDLG_KEEPCONSOLETITLE      0000000180002580     flags.obj
 0001:00001588       FDLG_NONMODAL              0000000180002588     flags.obj
 0001:00001590       FDLG_NONE                  0000000180002590     flags.obj
 0001:00001598       MIF_SELECTED               0000000180002598     flags.obj
 0001:000015a0       MIF_CHECKED                00000001800025a0     flags.obj
 0001:000015a8       MIF_SEPARATOR              00000001800025a8     flags.obj
 0001:000015b0       MIF_DISABLE                00000001800025b0     flags.obj
 0001:000015b8       MIF_GRAYED                 00000001800025b8     flags.obj
 0001:000015c0       MIF_HIDDEN                 00000001800025c0     flags.obj
 0001:000015c8       MIF_NONE                   00000001800025c8     flags.obj
 0001:000015d0       FMENU_SHOWAMPERSAND        00000001800025d0     flags.obj
 0001:000015d8       FMENU_WRAPMODE             00000001800025d8     flags.obj
 0001:000015e0       FMENU_AUTOHIGHLIGHT        00000001800025e0     flags.obj
 0001:000015e8       FMENU_REVERSEAUTOHIGHLIGHT 00000001800025e8     flags.obj
 0001:000015f0       FMENU_CHANGECONSOLETITLE   00000001800025f0     flags.obj
 0001:000015f8       FMENU_NONE                 00000001800025f8     flags.obj
 0001:00001600       PPIF_SELECTED              0000000180002600     flags.obj
 0001:00001608       PPIF_PROCESSDESCR          0000000180002608     flags.obj
 0001:00001610       PPIF_NONE                  0000000180002610     flags.obj
 0001:00001618       PFLAGS_SHOWHIDDEN          0000000180002618     flags.obj
 0001:00001620       PFLAGS_HIGHLIGHT           0000000180002620     flags.obj
 0001:00001628       PFLAGS_REVERSESORTORDER    0000000180002628     flags.obj
 0001:00001630       PFLAGS_USESORTGROUPS       0000000180002630     flags.obj
 0001:00001638       PFLAGS_SELECTEDFIRST       0000000180002638     flags.obj
 0001:00001640       PFLAGS_REALNAMES           0000000180002640     flags.obj
 0001:00001648       PFLAGS_PANELLEFT           0000000180002648     flags.obj
 0001:00001650       PFLAGS_DIRECTORIESFIRST    0000000180002650     flags.obj
 0001:00001658       PFLAGS_USECRC32            0000000180002658     flags.obj
 0001:00001660       PFLAGS_PLUGIN              0000000180002660     flags.obj
 0001:00001668       PFLAGS_VISIBLE             0000000180002668     flags.obj
 0001:00001670       PFLAGS_FOCUS               0000000180002670     flags.obj
 0001:00001678       PFLAGS_ALTERNATIVENAMES    0000000180002678     flags.obj
 0001:00001680       PFLAGS_SHORTCUT            0000000180002680     flags.obj
 0001:00001688       PFLAGS_NONE                0000000180002688     flags.obj
 0001:00001690       VF_NONMODAL                0000000180002690     flags.obj
 0001:00001698       VF_DELETEONCLOSE           0000000180002698     flags.obj
 0001:000016a0       VF_ENABLE_F6               00000001800026a0     flags.obj
 0001:000016a8       VF_DISABLEHISTORY          00000001800026a8     flags.obj
 0001:000016b0       VF_IMMEDIATERETURN         00000001800026b0     flags.obj
 0001:000016b8       VF_DELETEONLYFILEONCLOSE   00000001800026b8     flags.obj
 0001:000016c0       VF_NONE                    00000001800026c0     flags.obj
 0001:000016c8       EF_NONMODAL                00000001800026c8     flags.obj
 0001:000016d0       EF_CREATENEW               00000001800026d0     flags.obj
 0001:000016d8       EF_ENABLE_F6               00000001800026d8     flags.obj
 0001:000016e0       EF_DISABLEHISTORY          00000001800026e0     flags.obj
 0001:000016e8       EF_DELETEONCLOSE           00000001800026e8     flags.obj
 0001:000016f0       EF_IMMEDIATERETURN         00000001800026f0     flags.obj
 0001:000016f8       EF_DELETEONLYFILEONCLOSE   00000001800026f8     flags.obj
 0001:00001700       EF_LOCKED                  0000000180002700     flags.obj
 0001:00001708       EF_DISABLESAVEPOS          0000000180002708     flags.obj
 0001:00001710       EF_OPENMODE_MASK           0000000180002710     flags.obj
 0001:00001718       EF_OPENMODE_QUERY          0000000180002718     flags.obj
 0001:00001720       EF_OPENMODE_NEWIFOPEN      0000000180002720     flags.obj
 0001:00001728       EF_OPENMODE_USEEXISTING    0000000180002728     flags.obj
 0001:00001730       EF_OPENMODE_BREAKIFOPEN    0000000180002730     flags.obj
 0001:00001738       EF_OPENMODE_RELOADIFOPEN   0000000180002738     flags.obj
 0001:00001740       EN_NONE                    0000000180002740     flags.obj
 0001:00001748       FHELP_NOSHOWERROR          0000000180002748     flags.obj
 0001:00001750       FHELP_SELFHELP             0000000180002750     flags.obj
 0001:00001758       FHELP_FARHELP              0000000180002758     flags.obj
 0001:00001760       FHELP_CUSTOMFILE           0000000180002760     flags.obj
 0001:00001768       FHELP_CUSTOMPATH           0000000180002768     flags.obj
 0001:00001770       FHELP_GUID                 0000000180002770     flags.obj
 0001:00001778       FHELP_USECONTENTS          0000000180002778     flags.obj
 0001:00001780       FHELP_NONE                 0000000180002780     flags.obj
 0001:00001788       KMFLAGS_SILENTCHECK        0000000180002788     flags.obj
 0001:00001790       KMFLAGS_NOSENDKEYSTOPLUGINS 0000000180002790     flags.obj
 0001:00001798       KMFLAGS_ENABLEOUTPUT       0000000180002798     flags.obj
 0001:000017a0       KMFLAGS_LANGMASK           00000001800027a0     flags.obj
 0001:000017a8       KMFLAGS_LUA                00000001800027a8     flags.obj
 0001:000017b0       KMFLAGS_MOONSCRIPT         00000001800027b0     flags.obj
 0001:000017b8       KMFLAGS_NONE               00000001800027b8     flags.obj
 0001:000017c0       AKMFLAGS_NONE              00000001800027c0     flags.obj
 0001:000017c8       FSETCLR_REDRAW             00000001800027c8     flags.obj
 0001:000017d0       FSETCLR_NONE               00000001800027d0     flags.obj
 0001:000017d8       WIF_MODIFIED               00000001800027d8     flags.obj
 0001:000017e0       WIF_CURRENT                00000001800027e0     flags.obj
 0001:000017e8       WIF_MODAL                  00000001800027e8     flags.obj
 0001:000017f0       WIF_NONE                   00000001800027f0     flags.obj
 0001:000017f8       VOPT_SAVEFILEPOSITION      00000001800027f8     flags.obj
 0001:00001800       VOPT_AUTODETECTCODEPAGE    0000000180002800     flags.obj
 0001:00001808       VOPT_SHOWTITLEBAR          0000000180002808     flags.obj
 0001:00001810       VOPT_SHOWKEYBAR            0000000180002810     flags.obj
 0001:00001818       VOPT_SHOWSCROLLBAR         0000000180002818     flags.obj
 0001:00001820       VOPT_QUICKVIEW             0000000180002820     flags.obj
 0001:00001828       VOPT_NONE                  0000000180002828     flags.obj
 0001:00001830       VSMFL_REDRAW               0000000180002830     flags.obj
 0001:00001838       VSMFL_NONE                 0000000180002838     flags.obj
 0001:00001840       VSP_NOREDRAW               0000000180002840     flags.obj
 0001:00001848       VSP_PERCENT                0000000180002848     flags.obj
 0001:00001850       VSP_RELATIVE               0000000180002850     flags.obj
 0001:00001858       VSP_NORETNEWPOS            0000000180002858     flags.obj
 0001:00001860       VSP_NONE                   0000000180002860     flags.obj
 0001:00001868       VMF_WRAP                   0000000180002868     flags.obj
 0001:00001870       VMF_WORDWRAP               0000000180002870     flags.obj
 0001:00001878       VMF_NONE                   0000000180002878     flags.obj
 0001:00001880       ECF_TABMARKFIRST           0000000180002880     flags.obj
 0001:00001888       ECF_TABMARKCURRENT         0000000180002888     flags.obj
 0001:00001890       ECF_AUTODELETE             0000000180002890     flags.obj
 0001:00001898       ECF_NONE                   0000000180002898     flags.obj
 0001:000018a0       FIB_ENABLEEMPTY            00000001800028a0     flags.obj
 0001:000018a8       FIB_PASSWORD               00000001800028a8     flags.obj
 0001:000018b0       FIB_EXPANDENV              00000001800028b0     flags.obj
 0001:000018b8       FIB_NOUSELASTHISTORY       00000001800028b8     flags.obj
 0001:000018c0       FIB_BUTTONS                00000001800028c0     flags.obj
 0001:000018c8       FIB_NOAMPERSAND            00000001800028c8     flags.obj
 0001:000018d0       FIB_EDITPATH               00000001800028d0     flags.obj
 0001:000018d8       FIB_EDITPATHEXEC           00000001800028d8     flags.obj
 0001:000018e0       FIB_NONE                   00000001800028e0     flags.obj
 0001:000018e8       FPF_LOADED                 00000001800028e8     flags.obj
 0001:000018f0       FPF_ANSI                   00000001800028f0     flags.obj
 0001:000018f8       FPF_NONE                   00000001800028f8     flags.obj
 0001:00001900       PN_CMPNAME                 0000000180002900     flags.obj
 0001:00001908       PN_CMPNAMELIST             0000000180002908     flags.obj
 0001:00001910       PN_GENERATENAME            0000000180002910     flags.obj
 0001:00001918       PN_CHECKMASK               0000000180002918     flags.obj
 0001:00001920       PN_SKIPPATH                0000000180002920     flags.obj
 0001:00001928       PN_SHOWERRORMESSAGE        0000000180002928     flags.obj
 0001:00001930       PN_NONE                    0000000180002930     flags.obj
 0001:00001938       XLAT_SWITCHKEYBLAYOUT      0000000180002938     flags.obj
 0001:00001940       XLAT_SWITCHKEYBBEEP        0000000180002940     flags.obj
 0001:00001948       XLAT_USEKEYBLAYOUTNAME     0000000180002948     flags.obj
 0001:00001950       XLAT_CONVERTALLCMDLINE     0000000180002950     flags.obj
 0001:00001958       XLAT_NONE                  0000000180002958     flags.obj
 0001:00001960       FRS_RETUPDIR               0000000180002960     flags.obj
 0001:00001968       FRS_RECUR                  0000000180002968     flags.obj
 0001:00001970       FRS_SCANSYMLINK            0000000180002970     flags.obj
 0001:00001978       FRS_NONE                   0000000180002978     flags.obj
 0001:00001980       MLF_SHOWERRMSG             0000000180002980     flags.obj
 0001:00001988       MLF_DONOTUPDATEPANEL       0000000180002988     flags.obj
 0001:00001990       MLF_HOLDTARGET             0000000180002990     flags.obj
 0001:00001998       MLF_NONE                   0000000180002998     flags.obj
 0001:000019a0       FFFS_COMMAS                00000001800029a0     flags.obj
 0001:000019a8       FFFS_FLOATSIZE             00000001800029a8     flags.obj
 0001:000019b0       FFFS_SHOWBYTESINDEX        00000001800029b0     flags.obj
 0001:000019b8       FFFS_ECONOMIC              00000001800029b8     flags.obj
 0001:000019c0       FFFS_THOUSAND              00000001800029c0     flags.obj
 0001:000019c8       FFFS_MINSIZEINDEX          00000001800029c8     flags.obj
 0001:000019d0       FFFS_MINSIZEINDEX_MASK     00000001800029d0     flags.obj
 0001:000019d8       FFFS_NONE                  00000001800029d8     flags.obj
 0001:000019e0       PF_PRELOAD                 00000001800029e0     flags.obj
 0001:000019e8       PF_DISABLEPANELS           00000001800029e8     flags.obj
 0001:000019f0       PF_EDITOR                  00000001800029f0     flags.obj
 0001:000019f8       PF_VIEWER                  00000001800029f8     flags.obj
 0001:00001a00       PF_FULLCMDLINE             0000000180002a00     flags.obj
 0001:00001a08       PF_DIALOG                  0000000180002a08     flags.obj
 0001:00001a10       PF_NONE                    0000000180002a10     flags.obj
 0001:00001a18       IPLFLAGS_SEPARATOR         0000000180002a18     flags.obj
 0001:00001a20       IPLFLAGS_NONE              0000000180002a20     flags.obj
 0001:00001a28       PMFLAGS_FULLSCREEN         0000000180002a28     flags.obj
 0001:00001a30       PMFLAGS_DETAILEDSTATUS     0000000180002a30     flags.obj
 0001:00001a38       PMFLAGS_ALIGNEXTENSIONS    0000000180002a38     flags.obj
 0001:00001a40       PMFLAGS_CASECONVERSION     0000000180002a40     flags.obj
 0001:00001a48       PMFLAGS_NONE               0000000180002a48     flags.obj
 0001:00001a50       OPIF_DISABLEFILTER         0000000180002a50     flags.obj
 0001:00001a58       OPIF_DISABLESORTGROUPS     0000000180002a58     flags.obj
 0001:00001a60       OPIF_DISABLEHIGHLIGHTING   0000000180002a60     flags.obj
 0001:00001a68       OPIF_ADDDOTS               0000000180002a68     flags.obj
 0001:00001a70       OPIF_RAWSELECTION          0000000180002a70     flags.obj
 0001:00001a78       OPIF_REALNAMES             0000000180002a78     flags.obj
 0001:00001a80       OPIF_SHOWNAMESONLY         0000000180002a80     flags.obj
 0001:00001a88       OPIF_SHOWRIGHTALIGNNAMES   0000000180002a88     flags.obj
 0001:00001a90       OPIF_SHOWPRESERVECASE      0000000180002a90     flags.obj
 0001:00001a98       OPIF_COMPAREFATTIME        0000000180002a98     flags.obj
 0001:00001aa0       OPIF_EXTERNALGET           0000000180002aa0     flags.obj
 0001:00001aa8       OPIF_EXTERNALPUT           0000000180002aa8     flags.obj
 0001:00001ab0       OPIF_EXTERNALDELETE        0000000180002ab0     flags.obj
 0001:00001ab8       OPIF_EXTERNALMKDIR         0000000180002ab8     flags.obj
 0001:00001ac0       OPIF_USEATTRHIGHLIGHTING   0000000180002ac0     flags.obj
 0001:00001ac8       OPIF_USECRC32              0000000180002ac8     flags.obj
 0001:00001ad0       OPIF_USEFREESIZE           0000000180002ad0     flags.obj
 0001:00001ad8       OPIF_SHORTCUT              0000000180002ad8     flags.obj
 0001:00001ae0       OPIF_NONE                  0000000180002ae0     flags.obj
 0001:00001ae8       OPM_SILENT                 0000000180002ae8     flags.obj
 0001:00001af0       OPM_FIND                   0000000180002af0     flags.obj
 0001:00001af8       OPM_VIEW                   0000000180002af8     flags.obj
 0001:00001b00       OPM_EDIT                   0000000180002b00     flags.obj
 0001:00001b08       OPM_TOPLEVEL               0000000180002b08     flags.obj
 0001:00001b10       OPM_DESCR                  0000000180002b10     flags.obj
 0001:00001b18       OPM_QUICKVIEW              0000000180002b18     flags.obj
 0001:00001b20       OPM_PGDN                   0000000180002b20     flags.obj
 0001:00001b28       OPM_COMMANDS               0000000180002b28     flags.obj
 0001:00001b30       OPM_NONE                   0000000180002b30     flags.obj
 0001:00001b38       FOSF_ACTIVE                0000000180002b38     flags.obj
 0001:00001b40       FOSF_NONE                  0000000180002b40     flags.obj
 0001:00001b48       PCIF_NONE                  0000000180002b48     flags.obj
 0001:00001b50       FarGuid                    0000000180002b50     flags.obj
 0001:00006680       colors                     0000000180007680     keysandcolors.obj
 0001:000075e0       guids                      00000001800085e0     keysandcolors.obj
 0001:00008960       FCF_FG_4BIT                0000000180009960     lflua.obj
 0001:00008968       FCF_BG_4BIT                0000000180009968     lflua.obj
 0001:00008970       FCF_4BITMASK               0000000180009970     lflua.obj
 0001:00008978       FCF_RAWATTR_MASK           0000000180009978     lflua.obj
 0001:00008980       FCF_EXTENDEDFLAGS          0000000180009980     lflua.obj
 0001:00008988       FCF_FG_BOLD                0000000180009988     lflua.obj
 0001:00008990       FCF_FG_ITALIC              0000000180009990     lflua.obj
 0001:00008998       FCF_FG_UNDERLINE           0000000180009998     lflua.obj
 0001:000089a0       FCF_STYLEMASK              00000001800099a0     lflua.obj
 0001:000089a8       FCF_NONE                   00000001800099a8     lflua.obj
 0001:000089b0       CDF_NONE                   00000001800099b0     lflua.obj
 0001:000089b8       FMSG_WARNING               00000001800099b8     lflua.obj
 0001:000089c0       FMSG_ERRORTYPE             00000001800099c0     lflua.obj
 0001:000089c8       FMSG_KEEPBACKGROUND        00000001800099c8     lflua.obj
 0001:000089d0       FMSG_LEFTALIGN             00000001800099d0     lflua.obj
 0001:000089d8       FMSG_ALLINONE              00000001800099d8     lflua.obj
 0001:000089e0       FMSG_MB_OK                 00000001800099e0     lflua.obj
 0001:000089e8       FMSG_MB_OKCANCEL           00000001800099e8     lflua.obj
 0001:000089f0       FMSG_MB_ABORTRETRYIGNORE   00000001800099f0     lflua.obj
 0001:000089f8       FMSG_MB_YESNO              00000001800099f8     lflua.obj
 0001:00008a00       FMSG_MB_YESNOCANCEL        0000000180009a00     lflua.obj
 0001:00008a08       FMSG_MB_RETRYCANCEL        0000000180009a08     lflua.obj
 0001:00008a10       FMSG_NONE                  0000000180009a10     lflua.obj
 0001:00008a18       DIF_BOXCOLOR               0000000180009a18     lflua.obj
 0001:00008a20       DIF_GROUP                  0000000180009a20     lflua.obj
 0001:00008a28       DIF_LEFTTEXT               0000000180009a28     lflua.obj
 0001:00008a30       DIF_MOVESELECT             0000000180009a30     lflua.obj
 0001:00008a38       DIF_SHOWAMPERSAND          0000000180009a38     lflua.obj
 0001:00008a40       DIF_CENTERGROUP            0000000180009a40     lflua.obj
 0001:00008a48       DIF_NOBRACKETS             0000000180009a48     lflua.obj
 0001:00008a50       DIF_MANUALADDHISTORY       0000000180009a50     lflua.obj
 0001:00008a58       DIF_SEPARATOR              0000000180009a58     lflua.obj
 0001:00008a60       DIF_SEPARATOR2             0000000180009a60     lflua.obj
 0001:00008a68       DIF_EDITOR                 0000000180009a68     lflua.obj
 0001:00008a70       DIF_LISTNOAMPERSAND        0000000180009a70     lflua.obj
 0001:00008a78       DIF_LISTNOBOX              0000000180009a78     lflua.obj
 0001:00008a80       DIF_HISTORY                0000000180009a80     lflua.obj
 0001:00008a88       DIF_BTNNOCLOSE             0000000180009a88     lflua.obj
 0001:00008a90       DIF_CENTERTEXT             0000000180009a90     lflua.obj
 0001:00008a98       DIF_SEPARATORUSER          0000000180009a98     lflua.obj
 0001:00008aa0       DIF_SETSHIELD              0000000180009aa0     lflua.obj
 0001:00008aa8       DIF_EDITEXPAND             0000000180009aa8     lflua.obj
 0001:00008ab0       DIF_DROPDOWNLIST           0000000180009ab0     lflua.obj
 0001:00008ab8       DIF_USELASTHISTORY         0000000180009ab8     lflua.obj
 0001:00008ac0       DIF_MASKEDIT               0000000180009ac0     lflua.obj
 0001:00008ac8       DIF_LISTTRACKMOUSE         0000000180009ac8     lflua.obj
 0001:00008ad0       DIF_LISTTRACKMOUSEINFOCUS  0000000180009ad0     lflua.obj
 0001:00008ad8       DIF_SELECTONENTRY          0000000180009ad8     lflua.obj
 0001:00008ae0       DIF_3STATE                 0000000180009ae0     lflua.obj
 0001:00008ae8       DIF_EDITPATH               0000000180009ae8     lflua.obj
 0001:00008af0       DIF_LISTWRAPMODE           0000000180009af0     lflua.obj
 0001:00008af8       DIF_NOAUTOCOMPLETE         0000000180009af8     lflua.obj
 0001:00008b00       DIF_LISTAUTOHIGHLIGHT      0000000180009b00     lflua.obj
 0001:00008b08       DIF_LISTNOCLOSE            0000000180009b08     lflua.obj
 0001:00008b10       DIF_EDITPATHEXEC           0000000180009b10     lflua.obj
 0001:00008b18       DIF_HIDDEN                 0000000180009b18     lflua.obj
 0001:00008b20       DIF_READONLY               0000000180009b20     lflua.obj
 0001:00008b28       DIF_NOFOCUS                0000000180009b28     lflua.obj
 0001:00008b30       DIF_DISABLE                0000000180009b30     lflua.obj
 0001:00008b38       DIF_DEFAULTBUTTON          0000000180009b38     lflua.obj
 0001:00008b40       DIF_FOCUS                  0000000180009b40     lflua.obj
 0001:00008b48       DIF_RIGHTTEXT              0000000180009b48     lflua.obj
 0001:00008b50       DIF_WORDWRAP               0000000180009b50     lflua.obj
 0001:00008b58       DIF_NONE                   0000000180009b58     lflua.obj
 0001:00008b60       LIF_SELECTED               0000000180009b60     lflua.obj
 0001:00008b68       LIF_CHECKED                0000000180009b68     lflua.obj
 0001:00008b70       LIF_SEPARATOR              0000000180009b70     lflua.obj
 0001:00008b78       LIF_DISABLE                0000000180009b78     lflua.obj
 0001:00008b80       LIF_GRAYED                 0000000180009b80     lflua.obj
 0001:00008b88       LIF_HIDDEN                 0000000180009b88     lflua.obj
 0001:00008b90       LIF_DELETEUSERDATA         0000000180009b90     lflua.obj
 0001:00008b98       LIF_NONE                   0000000180009b98     lflua.obj
 0001:00008ba0       LIFIND_EXACTMATCH          0000000180009ba0     lflua.obj
 0001:00008ba8       LIFIND_NONE                0000000180009ba8     lflua.obj
 0001:00008bb0       LINFO_SHOWNOBOX            0000000180009bb0     lflua.obj
 0001:00008bb8       LINFO_AUTOHIGHLIGHT        0000000180009bb8     lflua.obj
 0001:00008bc0       LINFO_REVERSEHIGHLIGHT     0000000180009bc0     lflua.obj
 0001:00008bc8       LINFO_WRAPMODE             0000000180009bc8     lflua.obj
 0001:00008bd0       LINFO_SHOWAMPERSAND        0000000180009bd0     lflua.obj
 0001:00008bd8       LINFO_NONE                 0000000180009bd8     lflua.obj
 0001:00008be0       FDLG_WARNING               0000000180009be0     lflua.obj
 0001:00008be8       FDLG_SMALLDIALOG           0000000180009be8     lflua.obj
 0001:00008bf0       FDLG_NODRAWSHADOW          0000000180009bf0     lflua.obj
 0001:00008bf8       FDLG_NODRAWPANEL           0000000180009bf8     lflua.obj
 0001:00008c00       FDLG_KEEPCONSOLETITLE      0000000180009c00     lflua.obj
 0001:00008c08       FDLG_NONMODAL              0000000180009c08     lflua.obj
 0001:00008c10       FDLG_NONE                  0000000180009c10     lflua.obj
 0001:00008c18       MIF_SELECTED               0000000180009c18     lflua.obj
 0001:00008c20       MIF_CHECKED                0000000180009c20     lflua.obj
 0001:00008c28       MIF_SEPARATOR              0000000180009c28     lflua.obj
 0001:00008c30       MIF_DISABLE                0000000180009c30     lflua.obj
 0001:00008c38       MIF_GRAYED                 0000000180009c38     lflua.obj
 0001:00008c40       MIF_HIDDEN                 0000000180009c40     lflua.obj
 0001:00008c48       MIF_NONE                   0000000180009c48     lflua.obj
 0001:00008c50       FMENU_SHOWAMPERSAND        0000000180009c50     lflua.obj
 0001:00008c58       FMENU_WRAPMODE             0000000180009c58     lflua.obj
 0001:00008c60       FMENU_AUTOHIGHLIGHT        0000000180009c60     lflua.obj
 0001:00008c68       FMENU_REVERSEAUTOHIGHLIGHT 0000000180009c68     lflua.obj
 0001:00008c70       FMENU_CHANGECONSOLETITLE   0000000180009c70     lflua.obj
 0001:00008c78       FMENU_NONE                 0000000180009c78     lflua.obj
 0001:00008c80       PPIF_SELECTED              0000000180009c80     lflua.obj
 0001:00008c88       PPIF_PROCESSDESCR          0000000180009c88     lflua.obj
 0001:00008c90       PPIF_NONE                  0000000180009c90     lflua.obj
 0001:00008c98       PFLAGS_SHOWHIDDEN          0000000180009c98     lflua.obj
 0001:00008ca0       PFLAGS_HIGHLIGHT           0000000180009ca0     lflua.obj
 0001:00008ca8       PFLAGS_REVERSESORTORDER    0000000180009ca8     lflua.obj
 0001:00008cb0       PFLAGS_USESORTGROUPS       0000000180009cb0     lflua.obj
 0001:00008cb8       PFLAGS_SELECTEDFIRST       0000000180009cb8     lflua.obj
 0001:00008cc0       PFLAGS_REALNAMES           0000000180009cc0     lflua.obj
 0001:00008cc8       PFLAGS_PANELLEFT           0000000180009cc8     lflua.obj
 0001:00008cd0       PFLAGS_DIRECTORIESFIRST    0000000180009cd0     lflua.obj
 0001:00008cd8       PFLAGS_USECRC32            0000000180009cd8     lflua.obj
 0001:00008ce0       PFLAGS_PLUGIN              0000000180009ce0     lflua.obj
 0001:00008ce8       PFLAGS_VISIBLE             0000000180009ce8     lflua.obj
 0001:00008cf0       PFLAGS_FOCUS               0000000180009cf0     lflua.obj
 0001:00008cf8       PFLAGS_ALTERNATIVENAMES    0000000180009cf8     lflua.obj
 0001:00008d00       PFLAGS_SHORTCUT            0000000180009d00     lflua.obj
 0001:00008d08       PFLAGS_NONE                0000000180009d08     lflua.obj
 0001:00008d10       VF_NONMODAL                0000000180009d10     lflua.obj
 0001:00008d18       VF_DELETEONCLOSE           0000000180009d18     lflua.obj
 0001:00008d20       VF_ENABLE_F6               0000000180009d20     lflua.obj
 0001:00008d28       VF_DISABLEHISTORY          0000000180009d28     lflua.obj
 0001:00008d30       VF_IMMEDIATERETURN         0000000180009d30     lflua.obj
 0001:00008d38       VF_DELETEONLYFILEONCLOSE   0000000180009d38     lflua.obj
 0001:00008d40       VF_NONE                    0000000180009d40     lflua.obj
 0001:00008d48       EF_NONMODAL                0000000180009d48     lflua.obj
 0001:00008d50       EF_CREATENEW               0000000180009d50     lflua.obj
 0001:00008d58       EF_ENABLE_F6               0000000180009d58     lflua.obj
 0001:00008d60       EF_DISABLEHISTORY          0000000180009d60     lflua.obj
 0001:00008d68       EF_DELETEONCLOSE           0000000180009d68     lflua.obj
 0001:00008d70       EF_IMMEDIATERETURN         0000000180009d70     lflua.obj
 0001:00008d78       EF_DELETEONLYFILEONCLOSE   0000000180009d78     lflua.obj
 0001:00008d80       EF_LOCKED                  0000000180009d80     lflua.obj
 0001:00008d88       EF_DISABLESAVEPOS          0000000180009d88     lflua.obj
 0001:00008d90       EF_OPENMODE_MASK           0000000180009d90     lflua.obj
 0001:00008d98       EF_OPENMODE_QUERY          0000000180009d98     lflua.obj
 0001:00008da0       EF_OPENMODE_NEWIFOPEN      0000000180009da0     lflua.obj
 0001:00008da8       EF_OPENMODE_USEEXISTING    0000000180009da8     lflua.obj
 0001:00008db0       EF_OPENMODE_BREAKIFOPEN    0000000180009db0     lflua.obj
 0001:00008db8       EF_OPENMODE_RELOADIFOPEN   0000000180009db8     lflua.obj
 0001:00008dc0       EN_NONE                    0000000180009dc0     lflua.obj
 0001:00008dc8       FHELP_NOSHOWERROR          0000000180009dc8     lflua.obj
 0001:00008dd0       FHELP_SELFHELP             0000000180009dd0     lflua.obj
 0001:00008dd8       FHELP_FARHELP              0000000180009dd8     lflua.obj
 0001:00008de0       FHELP_CUSTOMFILE           0000000180009de0     lflua.obj
 0001:00008de8       FHELP_CUSTOMPATH           0000000180009de8     lflua.obj
 0001:00008df0       FHELP_GUID                 0000000180009df0     lflua.obj
 0001:00008df8       FHELP_USECONTENTS          0000000180009df8     lflua.obj
 0001:00008e00       FHELP_NONE                 0000000180009e00     lflua.obj
 0001:00008e08       KMFLAGS_SILENTCHECK        0000000180009e08     lflua.obj
 0001:00008e10       KMFLAGS_NOSENDKEYSTOPLUGINS 0000000180009e10     lflua.obj
 0001:00008e18       KMFLAGS_ENABLEOUTPUT       0000000180009e18     lflua.obj
 0001:00008e20       KMFLAGS_LANGMASK           0000000180009e20     lflua.obj
 0001:00008e28       KMFLAGS_LUA                0000000180009e28     lflua.obj
 0001:00008e30       KMFLAGS_MOONSCRIPT         0000000180009e30     lflua.obj
 0001:00008e38       KMFLAGS_NONE               0000000180009e38     lflua.obj
 0001:00008e40       AKMFLAGS_NONE              0000000180009e40     lflua.obj
 0001:00008e48       FSETCLR_REDRAW             0000000180009e48     lflua.obj
 0001:00008e50       FSETCLR_NONE               0000000180009e50     lflua.obj
 0001:00008e58       WIF_MODIFIED               0000000180009e58     lflua.obj
 0001:00008e60       WIF_CURRENT                0000000180009e60     lflua.obj
 0001:00008e68       WIF_MODAL                  0000000180009e68     lflua.obj
 0001:00008e70       WIF_NONE                   0000000180009e70     lflua.obj
 0001:00008e78       VOPT_SAVEFILEPOSITION      0000000180009e78     lflua.obj
 0001:00008e80       VOPT_AUTODETECTCODEPAGE    0000000180009e80     lflua.obj
 0001:00008e88       VOPT_SHOWTITLEBAR          0000000180009e88     lflua.obj
 0001:00008e90       VOPT_SHOWKEYBAR            0000000180009e90     lflua.obj
 0001:00008e98       VOPT_SHOWSCROLLBAR         0000000180009e98     lflua.obj
 0001:00008ea0       VOPT_QUICKVIEW             0000000180009ea0     lflua.obj
 0001:00008ea8       VOPT_NONE                  0000000180009ea8     lflua.obj
 0001:00008eb0       VSMFL_REDRAW               0000000180009eb0     lflua.obj
 0001:00008eb8       VSMFL_NONE                 0000000180009eb8     lflua.obj
 0001:00008ec0       VSP_NOREDRAW               0000000180009ec0     lflua.obj
 0001:00008ec8       VSP_PERCENT                0000000180009ec8     lflua.obj
 0001:00008ed0       VSP_RELATIVE               0000000180009ed0     lflua.obj
 0001:00008ed8       VSP_NORETNEWPOS            0000000180009ed8     lflua.obj
 0001:00008ee0       VSP_NONE                   0000000180009ee0     lflua.obj
 0001:00008ee8       VMF_WRAP                   0000000180009ee8     lflua.obj
 0001:00008ef0       VMF_WORDWRAP               0000000180009ef0     lflua.obj
 0001:00008ef8       VMF_NONE                   0000000180009ef8     lflua.obj
 0001:00008f00       ECF_TABMARKFIRST           0000000180009f00     lflua.obj
 0001:00008f08       ECF_TABMARKCURRENT         0000000180009f08     lflua.obj
 0001:00008f10       ECF_AUTODELETE             0000000180009f10     lflua.obj
 0001:00008f18       ECF_NONE                   0000000180009f18     lflua.obj
 0001:00008f20       FIB_ENABLEEMPTY            0000000180009f20     lflua.obj
 0001:00008f28       FIB_PASSWORD               0000000180009f28     lflua.obj
 0001:00008f30       FIB_EXPANDENV              0000000180009f30     lflua.obj
 0001:00008f38       FIB_NOUSELASTHISTORY       0000000180009f38     lflua.obj
 0001:00008f40       FIB_BUTTONS                0000000180009f40     lflua.obj
 0001:00008f48       FIB_NOAMPERSAND            0000000180009f48     lflua.obj
 0001:00008f50       FIB_EDITPATH               0000000180009f50     lflua.obj
 0001:00008f58       FIB_EDITPATHEXEC           0000000180009f58     lflua.obj
 0001:00008f60       FIB_NONE                   0000000180009f60     lflua.obj
 0001:00008f68       FPF_LOADED                 0000000180009f68     lflua.obj
 0001:00008f70       FPF_ANSI                   0000000180009f70     lflua.obj
 0001:00008f78       FPF_NONE                   0000000180009f78     lflua.obj
 0001:00008f80       PN_CMPNAME                 0000000180009f80     lflua.obj
 0001:00008f88       PN_CMPNAMELIST             0000000180009f88     lflua.obj
 0001:00008f90       PN_GENERATENAME            0000000180009f90     lflua.obj
 0001:00008f98       PN_CHECKMASK               0000000180009f98     lflua.obj
 0001:00008fa0       PN_SKIPPATH                0000000180009fa0     lflua.obj
 0001:00008fa8       PN_SHOWERRORMESSAGE        0000000180009fa8     lflua.obj
 0001:00008fb0       PN_NONE                    0000000180009fb0     lflua.obj
 0001:00008fb8       XLAT_SWITCHKEYBLAYOUT      0000000180009fb8     lflua.obj
 0001:00008fc0       XLAT_SWITCHKEYBBEEP        0000000180009fc0     lflua.obj
 0001:00008fc8       XLAT_USEKEYBLAYOUTNAME     0000000180009fc8     lflua.obj
 0001:00008fd0       XLAT_CONVERTALLCMDLINE     0000000180009fd0     lflua.obj
 0001:00008fd8       XLAT_NONE                  0000000180009fd8     lflua.obj
 0001:00008fe0       FRS_RETUPDIR               0000000180009fe0     lflua.obj
 0001:00008fe8       FRS_RECUR                  0000000180009fe8     lflua.obj
 0001:00008ff0       FRS_SCANSYMLINK            0000000180009ff0     lflua.obj
 0001:00008ff8       FRS_NONE                   0000000180009ff8     lflua.obj
 0001:00009000       MLF_SHOWERRMSG             000000018000a000     lflua.obj
 0001:00009008       MLF_DONOTUPDATEPANEL       000000018000a008     lflua.obj
 0001:00009010       MLF_HOLDTARGET             000000018000a010     lflua.obj
 0001:00009018       MLF_NONE                   000000018000a018     lflua.obj
 0001:00009020       FFFS_COMMAS                000000018000a020     lflua.obj
 0001:00009028       FFFS_FLOATSIZE             000000018000a028     lflua.obj
 0001:00009030       FFFS_SHOWBYTESINDEX        000000018000a030     lflua.obj
 0001:00009038       FFFS_ECONOMIC              000000018000a038     lflua.obj
 0001:00009040       FFFS_THOUSAND              000000018000a040     lflua.obj
 0001:00009048       FFFS_MINSIZEINDEX          000000018000a048     lflua.obj
 0001:00009050       FFFS_MINSIZEINDEX_MASK     000000018000a050     lflua.obj
 0001:00009058       FFFS_NONE                  000000018000a058     lflua.obj
 0001:00009060       PF_PRELOAD                 000000018000a060     lflua.obj
 0001:00009068       PF_DISABLEPANELS           000000018000a068     lflua.obj
 0001:00009070       PF_EDITOR                  000000018000a070     lflua.obj
 0001:00009078       PF_VIEWER                  000000018000a078     lflua.obj
 0001:00009080       PF_FULLCMDLINE             000000018000a080     lflua.obj
 0001:00009088       PF_DIALOG                  000000018000a088     lflua.obj
 0001:00009090       PF_NONE                    000000018000a090     lflua.obj
 0001:00009098       IPLFLAGS_SEPARATOR         000000018000a098     lflua.obj
 0001:000090a0       IPLFLAGS_NONE              000000018000a0a0     lflua.obj
 0001:000090a8       PMFLAGS_FULLSCREEN         000000018000a0a8     lflua.obj
 0001:000090b0       PMFLAGS_DETAILEDSTATUS     000000018000a0b0     lflua.obj
 0001:000090b8       PMFLAGS_ALIGNEXTENSIONS    000000018000a0b8     lflua.obj
 0001:000090c0       PMFLAGS_CASECONVERSION     000000018000a0c0     lflua.obj
 0001:000090c8       PMFLAGS_NONE               000000018000a0c8     lflua.obj
 0001:000090d0       OPIF_DISABLEFILTER         000000018000a0d0     lflua.obj
 0001:000090d8       OPIF_DISABLESORTGROUPS     000000018000a0d8     lflua.obj
 0001:000090e0       OPIF_DISABLEHIGHLIGHTING   000000018000a0e0     lflua.obj
 0001:000090e8       OPIF_ADDDOTS               000000018000a0e8     lflua.obj
 0001:000090f0       OPIF_RAWSELECTION          000000018000a0f0     lflua.obj
 0001:000090f8       OPIF_REALNAMES             000000018000a0f8     lflua.obj
 0001:00009100       OPIF_SHOWNAMESONLY         000000018000a100     lflua.obj
 0001:00009108       OPIF_SHOWRIGHTALIGNNAMES   000000018000a108     lflua.obj
 0001:00009110       OPIF_SHOWPRESERVECASE      000000018000a110     lflua.obj
 0001:00009118       OPIF_COMPAREFATTIME        000000018000a118     lflua.obj
 0001:00009120       OPIF_EXTERNALGET           000000018000a120     lflua.obj
 0001:00009128       OPIF_EXTERNALPUT           000000018000a128     lflua.obj
 0001:00009130       OPIF_EXTERNALDELETE        000000018000a130     lflua.obj
 0001:00009138       OPIF_EXTERNALMKDIR         000000018000a138     lflua.obj
 0001:00009140       OPIF_USEATTRHIGHLIGHTING   000000018000a140     lflua.obj
 0001:00009148       OPIF_USECRC32              000000018000a148     lflua.obj
 0001:00009150       OPIF_USEFREESIZE           000000018000a150     lflua.obj
 0001:00009158       OPIF_SHORTCUT              000000018000a158     lflua.obj
 0001:00009160       OPIF_NONE                  000000018000a160     lflua.obj
 0001:00009168       OPM_SILENT                 000000018000a168     lflua.obj
 0001:00009170       OPM_FIND                   000000018000a170     lflua.obj
 0001:00009178       OPM_VIEW                   000000018000a178     lflua.obj
 0001:00009180       OPM_EDIT                   000000018000a180     lflua.obj
 0001:00009188       OPM_TOPLEVEL               000000018000a188     lflua.obj
 0001:00009190       OPM_DESCR                  000000018000a190     lflua.obj
 0001:00009198       OPM_QUICKVIEW              000000018000a198     lflua.obj
 0001:000091a0       OPM_PGDN                   000000018000a1a0     lflua.obj
 0001:000091a8       OPM_COMMANDS               000000018000a1a8     lflua.obj
 0001:000091b0       OPM_NONE                   000000018000a1b0     lflua.obj
 0001:000091b8       FOSF_ACTIVE                000000018000a1b8     lflua.obj
 0001:000091c0       FOSF_NONE                  000000018000a1c0     lflua.obj
 0001:000091c8       PCIF_NONE                  000000018000a1c8     lflua.obj
 0001:000091d0       FarGuid                    000000018000a1d0     lflua.obj
 0001:000091e0       PDF_DIALOGEVENTDRAWENABLE  000000018000a1e0     lflua.obj
 0001:000091e8       PDF_PROCESSINGERROR        000000018000a1e8     lflua.obj
 0001:00009240       FCF_FG_4BIT                000000018000a240     lregex.obj
 0001:00009248       FCF_BG_4BIT                000000018000a248     lregex.obj
 0001:00009250       FCF_4BITMASK               000000018000a250     lregex.obj
 0001:00009258       FCF_RAWATTR_MASK           000000018000a258     lregex.obj
 0001:00009260       FCF_EXTENDEDFLAGS          000000018000a260     lregex.obj
 0001:00009268       FCF_FG_BOLD                000000018000a268     lregex.obj
 0001:00009270       FCF_FG_ITALIC              000000018000a270     lregex.obj
 0001:00009278       FCF_FG_UNDERLINE           000000018000a278     lregex.obj
 0001:00009280       FCF_STYLEMASK              000000018000a280     lregex.obj
 0001:00009288       FCF_NONE                   000000018000a288     lregex.obj
 0001:00009290       CDF_NONE                   000000018000a290     lregex.obj
 0001:00009298       FMSG_WARNING               000000018000a298     lregex.obj
 0001:000092a0       FMSG_ERRORTYPE             000000018000a2a0     lregex.obj
 0001:000092a8       FMSG_KEEPBACKGROUND        000000018000a2a8     lregex.obj
 0001:000092b0       FMSG_LEFTALIGN             000000018000a2b0     lregex.obj
 0001:000092b8       FMSG_ALLINONE              000000018000a2b8     lregex.obj
 0001:000092c0       FMSG_MB_OK                 000000018000a2c0     lregex.obj
 0001:000092c8       FMSG_MB_OKCANCEL           000000018000a2c8     lregex.obj
 0001:000092d0       FMSG_MB_ABORTRETRYIGNORE   000000018000a2d0     lregex.obj
 0001:000092d8       FMSG_MB_YESNO              000000018000a2d8     lregex.obj
 0001:000092e0       FMSG_MB_YESNOCANCEL        000000018000a2e0     lregex.obj
 0001:000092e8       FMSG_MB_RETRYCANCEL        000000018000a2e8     lregex.obj
 0001:000092f0       FMSG_NONE                  000000018000a2f0     lregex.obj
 0001:000092f8       DIF_BOXCOLOR               000000018000a2f8     lregex.obj
 0001:00009300       DIF_GROUP                  000000018000a300     lregex.obj
 0001:00009308       DIF_LEFTTEXT               000000018000a308     lregex.obj
 0001:00009310       DIF_MOVESELECT             000000018000a310     lregex.obj
 0001:00009318       DIF_SHOWAMPERSAND          000000018000a318     lregex.obj
 0001:00009320       DIF_CENTERGROUP            000000018000a320     lregex.obj
 0001:00009328       DIF_NOBRACKETS             000000018000a328     lregex.obj
 0001:00009330       DIF_MANUALADDHISTORY       000000018000a330     lregex.obj
 0001:00009338       DIF_SEPARATOR              000000018000a338     lregex.obj
 0001:00009340       DIF_SEPARATOR2             000000018000a340     lregex.obj
 0001:00009348       DIF_EDITOR                 000000018000a348     lregex.obj
 0001:00009350       DIF_LISTNOAMPERSAND        000000018000a350     lregex.obj
 0001:00009358       DIF_LISTNOBOX              000000018000a358     lregex.obj
 0001:00009360       DIF_HISTORY                000000018000a360     lregex.obj
 0001:00009368       DIF_BTNNOCLOSE             000000018000a368     lregex.obj
 0001:00009370       DIF_CENTERTEXT             000000018000a370     lregex.obj
 0001:00009378       DIF_SEPARATORUSER          000000018000a378     lregex.obj
 0001:00009380       DIF_SETSHIELD              000000018000a380     lregex.obj
 0001:00009388       DIF_EDITEXPAND             000000018000a388     lregex.obj
 0001:00009390       DIF_DROPDOWNLIST           000000018000a390     lregex.obj
 0001:00009398       DIF_USELASTHISTORY         000000018000a398     lregex.obj
 0001:000093a0       DIF_MASKEDIT               000000018000a3a0     lregex.obj
 0001:000093a8       DIF_LISTTRACKMOUSE         000000018000a3a8     lregex.obj
 0001:000093b0       DIF_LISTTRACKMOUSEINFOCUS  000000018000a3b0     lregex.obj
 0001:000093b8       DIF_SELECTONENTRY          000000018000a3b8     lregex.obj
 0001:000093c0       DIF_3STATE                 000000018000a3c0     lregex.obj
 0001:000093c8       DIF_EDITPATH               000000018000a3c8     lregex.obj
 0001:000093d0       DIF_LISTWRAPMODE           000000018000a3d0     lregex.obj
 0001:000093d8       DIF_NOAUTOCOMPLETE         000000018000a3d8     lregex.obj
 0001:000093e0       DIF_LISTAUTOHIGHLIGHT      000000018000a3e0     lregex.obj
 0001:000093e8       DIF_LISTNOCLOSE            000000018000a3e8     lregex.obj
 0001:000093f0       DIF_EDITPATHEXEC           000000018000a3f0     lregex.obj
 0001:000093f8       DIF_HIDDEN                 000000018000a3f8     lregex.obj
 0001:00009400       DIF_READONLY               000000018000a400     lregex.obj
 0001:00009408       DIF_NOFOCUS                000000018000a408     lregex.obj
 0001:00009410       DIF_DISABLE                000000018000a410     lregex.obj
 0001:00009418       DIF_DEFAULTBUTTON          000000018000a418     lregex.obj
 0001:00009420       DIF_FOCUS                  000000018000a420     lregex.obj
 0001:00009428       DIF_RIGHTTEXT              000000018000a428     lregex.obj
 0001:00009430       DIF_WORDWRAP               000000018000a430     lregex.obj
 0001:00009438       DIF_NONE                   000000018000a438     lregex.obj
 0001:00009440       LIF_SELECTED               000000018000a440     lregex.obj
 0001:00009448       LIF_CHECKED                000000018000a448     lregex.obj
 0001:00009450       LIF_SEPARATOR              000000018000a450     lregex.obj
 0001:00009458       LIF_DISABLE                000000018000a458     lregex.obj
 0001:00009460       LIF_GRAYED                 000000018000a460     lregex.obj
 0001:00009468       LIF_HIDDEN                 000000018000a468     lregex.obj
 0001:00009470       LIF_DELETEUSERDATA         000000018000a470     lregex.obj
 0001:00009478       LIF_NONE                   000000018000a478     lregex.obj
 0001:00009480       LIFIND_EXACTMATCH          000000018000a480     lregex.obj
 0001:00009488       LIFIND_NONE                000000018000a488     lregex.obj
 0001:00009490       LINFO_SHOWNOBOX            000000018000a490     lregex.obj
 0001:00009498       LINFO_AUTOHIGHLIGHT        000000018000a498     lregex.obj
 0001:000094a0       LINFO_REVERSEHIGHLIGHT     000000018000a4a0     lregex.obj
 0001:000094a8       LINFO_WRAPMODE             000000018000a4a8     lregex.obj
 0001:000094b0       LINFO_SHOWAMPERSAND        000000018000a4b0     lregex.obj
 0001:000094b8       LINFO_NONE                 000000018000a4b8     lregex.obj
 0001:000094c0       FDLG_WARNING               000000018000a4c0     lregex.obj
 0001:000094c8       FDLG_SMALLDIALOG           000000018000a4c8     lregex.obj
 0001:000094d0       FDLG_NODRAWSHADOW          000000018000a4d0     lregex.obj
 0001:000094d8       FDLG_NODRAWPANEL           000000018000a4d8     lregex.obj
 0001:000094e0       FDLG_KEEPCONSOLETITLE      000000018000a4e0     lregex.obj
 0001:000094e8       FDLG_NONMODAL              000000018000a4e8     lregex.obj
 0001:000094f0       FDLG_NONE                  000000018000a4f0     lregex.obj
 0001:000094f8       MIF_SELECTED               000000018000a4f8     lregex.obj
 0001:00009500       MIF_CHECKED                000000018000a500     lregex.obj
 0001:00009508       MIF_SEPARATOR              000000018000a508     lregex.obj
 0001:00009510       MIF_DISABLE                000000018000a510     lregex.obj
 0001:00009518       MIF_GRAYED                 000000018000a518     lregex.obj
 0001:00009520       MIF_HIDDEN                 000000018000a520     lregex.obj
 0001:00009528       MIF_NONE                   000000018000a528     lregex.obj
 0001:00009530       FMENU_SHOWAMPERSAND        000000018000a530     lregex.obj
 0001:00009538       FMENU_WRAPMODE             000000018000a538     lregex.obj
 0001:00009540       FMENU_AUTOHIGHLIGHT        000000018000a540     lregex.obj
 0001:00009548       FMENU_REVERSEAUTOHIGHLIGHT 000000018000a548     lregex.obj
 0001:00009550       FMENU_CHANGECONSOLETITLE   000000018000a550     lregex.obj
 0001:00009558       FMENU_NONE                 000000018000a558     lregex.obj
 0001:00009560       PPIF_SELECTED              000000018000a560     lregex.obj
 0001:00009568       PPIF_PROCESSDESCR          000000018000a568     lregex.obj
 0001:00009570       PPIF_NONE                  000000018000a570     lregex.obj
 0001:00009578       PFLAGS_SHOWHIDDEN          000000018000a578     lregex.obj
 0001:00009580       PFLAGS_HIGHLIGHT           000000018000a580     lregex.obj
 0001:00009588       PFLAGS_REVERSESORTORDER    000000018000a588     lregex.obj
 0001:00009590       PFLAGS_USESORTGROUPS       000000018000a590     lregex.obj
 0001:00009598       PFLAGS_SELECTEDFIRST       000000018000a598     lregex.obj
 0001:000095a0       PFLAGS_REALNAMES           000000018000a5a0     lregex.obj
 0001:000095a8       PFLAGS_PANELLEFT           000000018000a5a8     lregex.obj
 0001:000095b0       PFLAGS_DIRECTORIESFIRST    000000018000a5b0     lregex.obj
 0001:000095b8       PFLAGS_USECRC32            000000018000a5b8     lregex.obj
 0001:000095c0       PFLAGS_PLUGIN              000000018000a5c0     lregex.obj
 0001:000095c8       PFLAGS_VISIBLE             000000018000a5c8     lregex.obj
 0001:000095d0       PFLAGS_FOCUS               000000018000a5d0     lregex.obj
 0001:000095d8       PFLAGS_ALTERNATIVENAMES    000000018000a5d8     lregex.obj
 0001:000095e0       PFLAGS_SHORTCUT            000000018000a5e0     lregex.obj
 0001:000095e8       PFLAGS_NONE                000000018000a5e8     lregex.obj
 0001:000095f0       VF_NONMODAL                000000018000a5f0     lregex.obj
 0001:000095f8       VF_DELETEONCLOSE           000000018000a5f8     lregex.obj
 0001:00009600       VF_ENABLE_F6               000000018000a600     lregex.obj
 0001:00009608       VF_DISABLEHISTORY          000000018000a608     lregex.obj
 0001:00009610       VF_IMMEDIATERETURN         000000018000a610     lregex.obj
 0001:00009618       VF_DELETEONLYFILEONCLOSE   000000018000a618     lregex.obj
 0001:00009620       VF_NONE                    000000018000a620     lregex.obj
 0001:00009628       EF_NONMODAL                000000018000a628     lregex.obj
 0001:00009630       EF_CREATENEW               000000018000a630     lregex.obj
 0001:00009638       EF_ENABLE_F6               000000018000a638     lregex.obj
 0001:00009640       EF_DISABLEHISTORY          000000018000a640     lregex.obj
 0001:00009648       EF_DELETEONCLOSE           000000018000a648     lregex.obj
 0001:00009650       EF_IMMEDIATERETURN         000000018000a650     lregex.obj
 0001:00009658       EF_DELETEONLYFILEONCLOSE   000000018000a658     lregex.obj
 0001:00009660       EF_LOCKED                  000000018000a660     lregex.obj
 0001:00009668       EF_DISABLESAVEPOS          000000018000a668     lregex.obj
 0001:00009670       EF_OPENMODE_MASK           000000018000a670     lregex.obj
 0001:00009678       EF_OPENMODE_QUERY          000000018000a678     lregex.obj
 0001:00009680       EF_OPENMODE_NEWIFOPEN      000000018000a680     lregex.obj
 0001:00009688       EF_OPENMODE_USEEXISTING    000000018000a688     lregex.obj
 0001:00009690       EF_OPENMODE_BREAKIFOPEN    000000018000a690     lregex.obj
 0001:00009698       EF_OPENMODE_RELOADIFOPEN   000000018000a698     lregex.obj
 0001:000096a0       EN_NONE                    000000018000a6a0     lregex.obj
 0001:000096a8       FHELP_NOSHOWERROR          000000018000a6a8     lregex.obj
 0001:000096b0       FHELP_SELFHELP             000000018000a6b0     lregex.obj
 0001:000096b8       FHELP_FARHELP              000000018000a6b8     lregex.obj
 0001:000096c0       FHELP_CUSTOMFILE           000000018000a6c0     lregex.obj
 0001:000096c8       FHELP_CUSTOMPATH           000000018000a6c8     lregex.obj
 0001:000096d0       FHELP_GUID                 000000018000a6d0     lregex.obj
 0001:000096d8       FHELP_USECONTENTS          000000018000a6d8     lregex.obj
 0001:000096e0       FHELP_NONE                 000000018000a6e0     lregex.obj
 0001:000096e8       KMFLAGS_SILENTCHECK        000000018000a6e8     lregex.obj
 0001:000096f0       KMFLAGS_NOSENDKEYSTOPLUGINS 000000018000a6f0     lregex.obj
 0001:000096f8       KMFLAGS_ENABLEOUTPUT       000000018000a6f8     lregex.obj
 0001:00009700       KMFLAGS_LANGMASK           000000018000a700     lregex.obj
 0001:00009708       KMFLAGS_LUA                000000018000a708     lregex.obj
 0001:00009710       KMFLAGS_MOONSCRIPT         000000018000a710     lregex.obj
 0001:00009718       KMFLAGS_NONE               000000018000a718     lregex.obj
 0001:00009720       AKMFLAGS_NONE              000000018000a720     lregex.obj
 0001:00009728       FSETCLR_REDRAW             000000018000a728     lregex.obj
 0001:00009730       FSETCLR_NONE               000000018000a730     lregex.obj
 0001:00009738       WIF_MODIFIED               000000018000a738     lregex.obj
 0001:00009740       WIF_CURRENT                000000018000a740     lregex.obj
 0001:00009748       WIF_MODAL                  000000018000a748     lregex.obj
 0001:00009750       WIF_NONE                   000000018000a750     lregex.obj
 0001:00009758       VOPT_SAVEFILEPOSITION      000000018000a758     lregex.obj
 0001:00009760       VOPT_AUTODETECTCODEPAGE    000000018000a760     lregex.obj
 0001:00009768       VOPT_SHOWTITLEBAR          000000018000a768     lregex.obj
 0001:00009770       VOPT_SHOWKEYBAR            000000018000a770     lregex.obj
 0001:00009778       VOPT_SHOWSCROLLBAR         000000018000a778     lregex.obj
 0001:00009780       VOPT_QUICKVIEW             000000018000a780     lregex.obj
 0001:00009788       VOPT_NONE                  000000018000a788     lregex.obj
 0001:00009790       VSMFL_REDRAW               000000018000a790     lregex.obj
 0001:00009798       VSMFL_NONE                 000000018000a798     lregex.obj
 0001:000097a0       VSP_NOREDRAW               000000018000a7a0     lregex.obj
 0001:000097a8       VSP_PERCENT                000000018000a7a8     lregex.obj
 0001:000097b0       VSP_RELATIVE               000000018000a7b0     lregex.obj
 0001:000097b8       VSP_NORETNEWPOS            000000018000a7b8     lregex.obj
 0001:000097c0       VSP_NONE                   000000018000a7c0     lregex.obj
 0001:000097c8       VMF_WRAP                   000000018000a7c8     lregex.obj
 0001:000097d0       VMF_WORDWRAP               000000018000a7d0     lregex.obj
 0001:000097d8       VMF_NONE                   000000018000a7d8     lregex.obj
 0001:000097e0       ECF_TABMARKFIRST           000000018000a7e0     lregex.obj
 0001:000097e8       ECF_TABMARKCURRENT         000000018000a7e8     lregex.obj
 0001:000097f0       ECF_AUTODELETE             000000018000a7f0     lregex.obj
 0001:000097f8       ECF_NONE                   000000018000a7f8     lregex.obj
 0001:00009800       FIB_ENABLEEMPTY            000000018000a800     lregex.obj
 0001:00009808       FIB_PASSWORD               000000018000a808     lregex.obj
 0001:00009810       FIB_EXPANDENV              000000018000a810     lregex.obj
 0001:00009818       FIB_NOUSELASTHISTORY       000000018000a818     lregex.obj
 0001:00009820       FIB_BUTTONS                000000018000a820     lregex.obj
 0001:00009828       FIB_NOAMPERSAND            000000018000a828     lregex.obj
 0001:00009830       FIB_EDITPATH               000000018000a830     lregex.obj
 0001:00009838       FIB_EDITPATHEXEC           000000018000a838     lregex.obj
 0001:00009840       FIB_NONE                   000000018000a840     lregex.obj
 0001:00009848       FPF_LOADED                 000000018000a848     lregex.obj
 0001:00009850       FPF_ANSI                   000000018000a850     lregex.obj
 0001:00009858       FPF_NONE                   000000018000a858     lregex.obj
 0001:00009860       PN_CMPNAME                 000000018000a860     lregex.obj
 0001:00009868       PN_CMPNAMELIST             000000018000a868     lregex.obj
 0001:00009870       PN_GENERATENAME            000000018000a870     lregex.obj
 0001:00009878       PN_CHECKMASK               000000018000a878     lregex.obj
 0001:00009880       PN_SKIPPATH                000000018000a880     lregex.obj
 0001:00009888       PN_SHOWERRORMESSAGE        000000018000a888     lregex.obj
 0001:00009890       PN_NONE                    000000018000a890     lregex.obj
 0001:00009898       XLAT_SWITCHKEYBLAYOUT      000000018000a898     lregex.obj
 0001:000098a0       XLAT_SWITCHKEYBBEEP        000000018000a8a0     lregex.obj
 0001:000098a8       XLAT_USEKEYBLAYOUTNAME     000000018000a8a8     lregex.obj
 0001:000098b0       XLAT_CONVERTALLCMDLINE     000000018000a8b0     lregex.obj
 0001:000098b8       XLAT_NONE                  000000018000a8b8     lregex.obj
 0001:000098c0       FRS_RETUPDIR               000000018000a8c0     lregex.obj
 0001:000098c8       FRS_RECUR                  000000018000a8c8     lregex.obj
 0001:000098d0       FRS_SCANSYMLINK            000000018000a8d0     lregex.obj
 0001:000098d8       FRS_NONE                   000000018000a8d8     lregex.obj
 0001:000098e0       MLF_SHOWERRMSG             000000018000a8e0     lregex.obj
 0001:000098e8       MLF_DONOTUPDATEPANEL       000000018000a8e8     lregex.obj
 0001:000098f0       MLF_HOLDTARGET             000000018000a8f0     lregex.obj
 0001:000098f8       MLF_NONE                   000000018000a8f8     lregex.obj
 0001:00009900       FFFS_COMMAS                000000018000a900     lregex.obj
 0001:00009908       FFFS_FLOATSIZE             000000018000a908     lregex.obj
 0001:00009910       FFFS_SHOWBYTESINDEX        000000018000a910     lregex.obj
 0001:00009918       FFFS_ECONOMIC              000000018000a918     lregex.obj
 0001:00009920       FFFS_THOUSAND              000000018000a920     lregex.obj
 0001:00009928       FFFS_MINSIZEINDEX          000000018000a928     lregex.obj
 0001:00009930       FFFS_MINSIZEINDEX_MASK     000000018000a930     lregex.obj
 0001:00009938       FFFS_NONE                  000000018000a938     lregex.obj
 0001:00009940       PF_PRELOAD                 000000018000a940     lregex.obj
 0001:00009948       PF_DISABLEPANELS           000000018000a948     lregex.obj
 0001:00009950       PF_EDITOR                  000000018000a950     lregex.obj
 0001:00009958       PF_VIEWER                  000000018000a958     lregex.obj
 0001:00009960       PF_FULLCMDLINE             000000018000a960     lregex.obj
 0001:00009968       PF_DIALOG                  000000018000a968     lregex.obj
 0001:00009970       PF_NONE                    000000018000a970     lregex.obj
 0001:00009978       IPLFLAGS_SEPARATOR         000000018000a978     lregex.obj
 0001:00009980       IPLFLAGS_NONE              000000018000a980     lregex.obj
 0001:00009988       PMFLAGS_FULLSCREEN         000000018000a988     lregex.obj
 0001:00009990       PMFLAGS_DETAILEDSTATUS     000000018000a990     lregex.obj
 0001:00009998       PMFLAGS_ALIGNEXTENSIONS    000000018000a998     lregex.obj
 0001:000099a0       PMFLAGS_CASECONVERSION     000000018000a9a0     lregex.obj
 0001:000099a8       PMFLAGS_NONE               000000018000a9a8     lregex.obj
 0001:000099b0       OPIF_DISABLEFILTER         000000018000a9b0     lregex.obj
 0001:000099b8       OPIF_DISABLESORTGROUPS     000000018000a9b8     lregex.obj
 0001:000099c0       OPIF_DISABLEHIGHLIGHTING   000000018000a9c0     lregex.obj
 0001:000099c8       OPIF_ADDDOTS               000000018000a9c8     lregex.obj
 0001:000099d0       OPIF_RAWSELECTION          000000018000a9d0     lregex.obj
 0001:000099d8       OPIF_REALNAMES             000000018000a9d8     lregex.obj
 0001:000099e0       OPIF_SHOWNAMESONLY         000000018000a9e0     lregex.obj
 0001:000099e8       OPIF_SHOWRIGHTALIGNNAMES   000000018000a9e8     lregex.obj
 0001:000099f0       OPIF_SHOWPRESERVECASE      000000018000a9f0     lregex.obj
 0001:000099f8       OPIF_COMPAREFATTIME        000000018000a9f8     lregex.obj
 0001:00009a00       OPIF_EXTERNALGET           000000018000aa00     lregex.obj
 0001:00009a08       OPIF_EXTERNALPUT           000000018000aa08     lregex.obj
 0001:00009a10       OPIF_EXTERNALDELETE        000000018000aa10     lregex.obj
 0001:00009a18       OPIF_EXTERNALMKDIR         000000018000aa18     lregex.obj
 0001:00009a20       OPIF_USEATTRHIGHLIGHTING   000000018000aa20     lregex.obj
 0001:00009a28       OPIF_USECRC32              000000018000aa28     lregex.obj
 0001:00009a30       OPIF_USEFREESIZE           000000018000aa30     lregex.obj
 0001:00009a38       OPIF_SHORTCUT              000000018000aa38     lregex.obj
 0001:00009a40       OPIF_NONE                  000000018000aa40     lregex.obj
 0001:00009a48       OPM_SILENT                 000000018000aa48     lregex.obj
 0001:00009a50       OPM_FIND                   000000018000aa50     lregex.obj
 0001:00009a58       OPM_VIEW                   000000018000aa58     lregex.obj
 0001:00009a60       OPM_EDIT                   000000018000aa60     lregex.obj
 0001:00009a68       OPM_TOPLEVEL               000000018000aa68     lregex.obj
 0001:00009a70       OPM_DESCR                  000000018000aa70     lregex.obj
 0001:00009a78       OPM_QUICKVIEW              000000018000aa78     lregex.obj
 0001:00009a80       OPM_PGDN                   000000018000aa80     lregex.obj
 0001:00009a88       OPM_COMMANDS               000000018000aa88     lregex.obj
 0001:00009a90       OPM_NONE                   000000018000aa90     lregex.obj
 0001:00009a98       FOSF_ACTIVE                000000018000aa98     lregex.obj
 0001:00009aa0       FOSF_NONE                  000000018000aaa0     lregex.obj
 0001:00009aa8       PCIF_NONE                  000000018000aaa8     lregex.obj
 0001:00009ab0       FarGuid                    000000018000aab0     lregex.obj
 0001:00009ac0       PDF_DIALOGEVENTDRAWENABLE  000000018000aac0     lregex.obj
 0001:00009ac8       PDF_PROCESSINGERROR        000000018000aac8     lregex.obj
 0001:00009d90       FCF_FG_4BIT                000000018000ad90     luamacro.obj
 0001:00009d98       FCF_BG_4BIT                000000018000ad98     luamacro.obj
 0001:00009da0       FCF_4BITMASK               000000018000ada0     luamacro.obj
 0001:00009da8       FCF_RAWATTR_MASK           000000018000ada8     luamacro.obj
 0001:00009db0       FCF_EXTENDEDFLAGS          000000018000adb0     luamacro.obj
 0001:00009db8       FCF_FG_BOLD                000000018000adb8     luamacro.obj
 0001:00009dc0       FCF_FG_ITALIC              000000018000adc0     luamacro.obj
 0001:00009dc8       FCF_FG_UNDERLINE           000000018000adc8     luamacro.obj
 0001:00009dd0       FCF_STYLEMASK              000000018000add0     luamacro.obj
 0001:00009dd8       FCF_NONE                   000000018000add8     luamacro.obj
 0001:00009de0       CDF_NONE                   000000018000ade0     luamacro.obj
 0001:00009de8       FMSG_WARNING               000000018000ade8     luamacro.obj
 0001:00009df0       FMSG_ERRORTYPE             000000018000adf0     luamacro.obj
 0001:00009df8       FMSG_KEEPBACKGROUND        000000018000adf8     luamacro.obj
 0001:00009e00       FMSG_LEFTALIGN             000000018000ae00     luamacro.obj
 0001:00009e08       FMSG_ALLINONE              000000018000ae08     luamacro.obj
 0001:00009e10       FMSG_MB_OK                 000000018000ae10     luamacro.obj
 0001:00009e18       FMSG_MB_OKCANCEL           000000018000ae18     luamacro.obj
 0001:00009e20       FMSG_MB_ABORTRETRYIGNORE   000000018000ae20     luamacro.obj
 0001:00009e28       FMSG_MB_YESNO              000000018000ae28     luamacro.obj
 0001:00009e30       FMSG_MB_YESNOCANCEL        000000018000ae30     luamacro.obj
 0001:00009e38       FMSG_MB_RETRYCANCEL        000000018000ae38     luamacro.obj
 0001:00009e40       FMSG_NONE                  000000018000ae40     luamacro.obj
 0001:00009e48       DIF_BOXCOLOR               000000018000ae48     luamacro.obj
 0001:00009e50       DIF_GROUP                  000000018000ae50     luamacro.obj
 0001:00009e58       DIF_LEFTTEXT               000000018000ae58     luamacro.obj
 0001:00009e60       DIF_MOVESELECT             000000018000ae60     luamacro.obj
 0001:00009e68       DIF_SHOWAMPERSAND          000000018000ae68     luamacro.obj
 0001:00009e70       DIF_CENTERGROUP            000000018000ae70     luamacro.obj
 0001:00009e78       DIF_NOBRACKETS             000000018000ae78     luamacro.obj
 0001:00009e80       DIF_MANUALADDHISTORY       000000018000ae80     luamacro.obj
 0001:00009e88       DIF_SEPARATOR              000000018000ae88     luamacro.obj
 0001:00009e90       DIF_SEPARATOR2             000000018000ae90     luamacro.obj
 0001:00009e98       DIF_EDITOR                 000000018000ae98     luamacro.obj
 0001:00009ea0       DIF_LISTNOAMPERSAND        000000018000aea0     luamacro.obj
 0001:00009ea8       DIF_LISTNOBOX              000000018000aea8     luamacro.obj
 0001:00009eb0       DIF_HISTORY                000000018000aeb0     luamacro.obj
 0001:00009eb8       DIF_BTNNOCLOSE             000000018000aeb8     luamacro.obj
 0001:00009ec0       DIF_CENTERTEXT             000000018000aec0     luamacro.obj
 0001:00009ec8       DIF_SEPARATORUSER          000000018000aec8     luamacro.obj
 0001:00009ed0       DIF_SETSHIELD              000000018000aed0     luamacro.obj
 0001:00009ed8       DIF_EDITEXPAND             000000018000aed8     luamacro.obj
 0001:00009ee0       DIF_DROPDOWNLIST           000000018000aee0     luamacro.obj
 0001:00009ee8       DIF_USELASTHISTORY         000000018000aee8     luamacro.obj
 0001:00009ef0       DIF_MASKEDIT               000000018000aef0     luamacro.obj
 0001:00009ef8       DIF_LISTTRACKMOUSE         000000018000aef8     luamacro.obj
 0001:00009f00       DIF_LISTTRACKMOUSEINFOCUS  000000018000af00     luamacro.obj
 0001:00009f08       DIF_SELECTONENTRY          000000018000af08     luamacro.obj
 0001:00009f10       DIF_3STATE                 000000018000af10     luamacro.obj
 0001:00009f18       DIF_EDITPATH               000000018000af18     luamacro.obj
 0001:00009f20       DIF_LISTWRAPMODE           000000018000af20     luamacro.obj
 0001:00009f28       DIF_NOAUTOCOMPLETE         000000018000af28     luamacro.obj
 0001:00009f30       DIF_LISTAUTOHIGHLIGHT      000000018000af30     luamacro.obj
 0001:00009f38       DIF_LISTNOCLOSE            000000018000af38     luamacro.obj
 0001:00009f40       DIF_EDITPATHEXEC           000000018000af40     luamacro.obj
 0001:00009f48       DIF_HIDDEN                 000000018000af48     luamacro.obj
 0001:00009f50       DIF_READONLY               000000018000af50     luamacro.obj
 0001:00009f58       DIF_NOFOCUS                000000018000af58     luamacro.obj
 0001:00009f60       DIF_DISABLE                000000018000af60     luamacro.obj
 0001:00009f68       DIF_DEFAULTBUTTON          000000018000af68     luamacro.obj
 0001:00009f70       DIF_FOCUS                  000000018000af70     luamacro.obj
 0001:00009f78       DIF_RIGHTTEXT              000000018000af78     luamacro.obj
 0001:00009f80       DIF_WORDWRAP               000000018000af80     luamacro.obj
 0001:00009f88       DIF_NONE                   000000018000af88     luamacro.obj
 0001:00009f90       LIF_SELECTED               000000018000af90     luamacro.obj
 0001:00009f98       LIF_CHECKED                000000018000af98     luamacro.obj
 0001:00009fa0       LIF_SEPARATOR              000000018000afa0     luamacro.obj
 0001:00009fa8       LIF_DISABLE                000000018000afa8     luamacro.obj
 0001:00009fb0       LIF_GRAYED                 000000018000afb0     luamacro.obj
 0001:00009fb8       LIF_HIDDEN                 000000018000afb8     luamacro.obj
 0001:00009fc0       LIF_DELETEUSERDATA         000000018000afc0     luamacro.obj
 0001:00009fc8       LIF_NONE                   000000018000afc8     luamacro.obj
 0001:00009fd0       LIFIND_EXACTMATCH          000000018000afd0     luamacro.obj
 0001:00009fd8       LIFIND_NONE                000000018000afd8     luamacro.obj
 0001:00009fe0       LINFO_SHOWNOBOX            000000018000afe0     luamacro.obj
 0001:00009fe8       LINFO_AUTOHIGHLIGHT        000000018000afe8     luamacro.obj
 0001:00009ff0       LINFO_REVERSEHIGHLIGHT     000000018000aff0     luamacro.obj
 0001:00009ff8       LINFO_WRAPMODE             000000018000aff8     luamacro.obj
 0001:0000a000       LINFO_SHOWAMPERSAND        000000018000b000     luamacro.obj
 0001:0000a008       LINFO_NONE                 000000018000b008     luamacro.obj
 0001:0000a010       FDLG_WARNING               000000018000b010     luamacro.obj
 0001:0000a018       FDLG_SMALLDIALOG           000000018000b018     luamacro.obj
 0001:0000a020       FDLG_NODRAWSHADOW          000000018000b020     luamacro.obj
 0001:0000a028       FDLG_NODRAWPANEL           000000018000b028     luamacro.obj
 0001:0000a030       FDLG_KEEPCONSOLETITLE      000000018000b030     luamacro.obj
 0001:0000a038       FDLG_NONMODAL              000000018000b038     luamacro.obj
 0001:0000a040       FDLG_NONE                  000000018000b040     luamacro.obj
 0001:0000a048       MIF_SELECTED               000000018000b048     luamacro.obj
 0001:0000a050       MIF_CHECKED                000000018000b050     luamacro.obj
 0001:0000a058       MIF_SEPARATOR              000000018000b058     luamacro.obj
 0001:0000a060       MIF_DISABLE                000000018000b060     luamacro.obj
 0001:0000a068       MIF_GRAYED                 000000018000b068     luamacro.obj
 0001:0000a070       MIF_HIDDEN                 000000018000b070     luamacro.obj
 0001:0000a078       MIF_NONE                   000000018000b078     luamacro.obj
 0001:0000a080       FMENU_SHOWAMPERSAND        000000018000b080     luamacro.obj
 0001:0000a088       FMENU_WRAPMODE             000000018000b088     luamacro.obj
 0001:0000a090       FMENU_AUTOHIGHLIGHT        000000018000b090     luamacro.obj
 0001:0000a098       FMENU_REVERSEAUTOHIGHLIGHT 000000018000b098     luamacro.obj
 0001:0000a0a0       FMENU_CHANGECONSOLETITLE   000000018000b0a0     luamacro.obj
 0001:0000a0a8       FMENU_NONE                 000000018000b0a8     luamacro.obj
 0001:0000a0b0       PPIF_SELECTED              000000018000b0b0     luamacro.obj
 0001:0000a0b8       PPIF_PROCESSDESCR          000000018000b0b8     luamacro.obj
 0001:0000a0c0       PPIF_NONE                  000000018000b0c0     luamacro.obj
 0001:0000a0c8       PFLAGS_SHOWHIDDEN          000000018000b0c8     luamacro.obj
 0001:0000a0d0       PFLAGS_HIGHLIGHT           000000018000b0d0     luamacro.obj
 0001:0000a0d8       PFLAGS_REVERSESORTORDER    000000018000b0d8     luamacro.obj
 0001:0000a0e0       PFLAGS_USESORTGROUPS       000000018000b0e0     luamacro.obj
 0001:0000a0e8       PFLAGS_SELECTEDFIRST       000000018000b0e8     luamacro.obj
 0001:0000a0f0       PFLAGS_REALNAMES           000000018000b0f0     luamacro.obj
 0001:0000a0f8       PFLAGS_PANELLEFT           000000018000b0f8     luamacro.obj
 0001:0000a100       PFLAGS_DIRECTORIESFIRST    000000018000b100     luamacro.obj
 0001:0000a108       PFLAGS_USECRC32            000000018000b108     luamacro.obj
 0001:0000a110       PFLAGS_PLUGIN              000000018000b110     luamacro.obj
 0001:0000a118       PFLAGS_VISIBLE             000000018000b118     luamacro.obj
 0001:0000a120       PFLAGS_FOCUS               000000018000b120     luamacro.obj
 0001:0000a128       PFLAGS_ALTERNATIVENAMES    000000018000b128     luamacro.obj
 0001:0000a130       PFLAGS_SHORTCUT            000000018000b130     luamacro.obj
 0001:0000a138       PFLAGS_NONE                000000018000b138     luamacro.obj
 0001:0000a140       VF_NONMODAL                000000018000b140     luamacro.obj
 0001:0000a148       VF_DELETEONCLOSE           000000018000b148     luamacro.obj
 0001:0000a150       VF_ENABLE_F6               000000018000b150     luamacro.obj
 0001:0000a158       VF_DISABLEHISTORY          000000018000b158     luamacro.obj
 0001:0000a160       VF_IMMEDIATERETURN         000000018000b160     luamacro.obj
 0001:0000a168       VF_DELETEONLYFILEONCLOSE   000000018000b168     luamacro.obj
 0001:0000a170       VF_NONE                    000000018000b170     luamacro.obj
 0001:0000a178       EF_NONMODAL                000000018000b178     luamacro.obj
 0001:0000a180       EF_CREATENEW               000000018000b180     luamacro.obj
 0001:0000a188       EF_ENABLE_F6               000000018000b188     luamacro.obj
 0001:0000a190       EF_DISABLEHISTORY          000000018000b190     luamacro.obj
 0001:0000a198       EF_DELETEONCLOSE           000000018000b198     luamacro.obj
 0001:0000a1a0       EF_IMMEDIATERETURN         000000018000b1a0     luamacro.obj
 0001:0000a1a8       EF_DELETEONLYFILEONCLOSE   000000018000b1a8     luamacro.obj
 0001:0000a1b0       EF_LOCKED                  000000018000b1b0     luamacro.obj
 0001:0000a1b8       EF_DISABLESAVEPOS          000000018000b1b8     luamacro.obj
 0001:0000a1c0       EF_OPENMODE_MASK           000000018000b1c0     luamacro.obj
 0001:0000a1c8       EF_OPENMODE_QUERY          000000018000b1c8     luamacro.obj
 0001:0000a1d0       EF_OPENMODE_NEWIFOPEN      000000018000b1d0     luamacro.obj
 0001:0000a1d8       EF_OPENMODE_USEEXISTING    000000018000b1d8     luamacro.obj
 0001:0000a1e0       EF_OPENMODE_BREAKIFOPEN    000000018000b1e0     luamacro.obj
 0001:0000a1e8       EF_OPENMODE_RELOADIFOPEN   000000018000b1e8     luamacro.obj
 0001:0000a1f0       EN_NONE                    000000018000b1f0     luamacro.obj
 0001:0000a1f8       FHELP_NOSHOWERROR          000000018000b1f8     luamacro.obj
 0001:0000a200       FHELP_SELFHELP             000000018000b200     luamacro.obj
 0001:0000a208       FHELP_FARHELP              000000018000b208     luamacro.obj
 0001:0000a210       FHELP_CUSTOMFILE           000000018000b210     luamacro.obj
 0001:0000a218       FHELP_CUSTOMPATH           000000018000b218     luamacro.obj
 0001:0000a220       FHELP_GUID                 000000018000b220     luamacro.obj
 0001:0000a228       FHELP_USECONTENTS          000000018000b228     luamacro.obj
 0001:0000a230       FHELP_NONE                 000000018000b230     luamacro.obj
 0001:0000a238       KMFLAGS_SILENTCHECK        000000018000b238     luamacro.obj
 0001:0000a240       KMFLAGS_NOSENDKEYSTOPLUGINS 000000018000b240     luamacro.obj
 0001:0000a248       KMFLAGS_ENABLEOUTPUT       000000018000b248     luamacro.obj
 0001:0000a250       KMFLAGS_LANGMASK           000000018000b250     luamacro.obj
 0001:0000a258       KMFLAGS_LUA                000000018000b258     luamacro.obj
 0001:0000a260       KMFLAGS_MOONSCRIPT         000000018000b260     luamacro.obj
 0001:0000a268       KMFLAGS_NONE               000000018000b268     luamacro.obj
 0001:0000a270       AKMFLAGS_NONE              000000018000b270     luamacro.obj
 0001:0000a278       FSETCLR_REDRAW             000000018000b278     luamacro.obj
 0001:0000a280       FSETCLR_NONE               000000018000b280     luamacro.obj
 0001:0000a288       WIF_MODIFIED               000000018000b288     luamacro.obj
 0001:0000a290       WIF_CURRENT                000000018000b290     luamacro.obj
 0001:0000a298       WIF_MODAL                  000000018000b298     luamacro.obj
 0001:0000a2a0       WIF_NONE                   000000018000b2a0     luamacro.obj
 0001:0000a2a8       VOPT_SAVEFILEPOSITION      000000018000b2a8     luamacro.obj
 0001:0000a2b0       VOPT_AUTODETECTCODEPAGE    000000018000b2b0     luamacro.obj
 0001:0000a2b8       VOPT_SHOWTITLEBAR          000000018000b2b8     luamacro.obj
 0001:0000a2c0       VOPT_SHOWKEYBAR            000000018000b2c0     luamacro.obj
 0001:0000a2c8       VOPT_SHOWSCROLLBAR         000000018000b2c8     luamacro.obj
 0001:0000a2d0       VOPT_QUICKVIEW             000000018000b2d0     luamacro.obj
 0001:0000a2d8       VOPT_NONE                  000000018000b2d8     luamacro.obj
 0001:0000a2e0       VSMFL_REDRAW               000000018000b2e0     luamacro.obj
 0001:0000a2e8       VSMFL_NONE                 000000018000b2e8     luamacro.obj
 0001:0000a2f0       VSP_NOREDRAW               000000018000b2f0     luamacro.obj
 0001:0000a2f8       VSP_PERCENT                000000018000b2f8     luamacro.obj
 0001:0000a300       VSP_RELATIVE               000000018000b300     luamacro.obj
 0001:0000a308       VSP_NORETNEWPOS            000000018000b308     luamacro.obj
 0001:0000a310       VSP_NONE                   000000018000b310     luamacro.obj
 0001:0000a318       VMF_WRAP                   000000018000b318     luamacro.obj
 0001:0000a320       VMF_WORDWRAP               000000018000b320     luamacro.obj
 0001:0000a328       VMF_NONE                   000000018000b328     luamacro.obj
 0001:0000a330       ECF_TABMARKFIRST           000000018000b330     luamacro.obj
 0001:0000a338       ECF_TABMARKCURRENT         000000018000b338     luamacro.obj
 0001:0000a340       ECF_AUTODELETE             000000018000b340     luamacro.obj
 0001:0000a348       ECF_NONE                   000000018000b348     luamacro.obj
 0001:0000a350       FIB_ENABLEEMPTY            000000018000b350     luamacro.obj
 0001:0000a358       FIB_PASSWORD               000000018000b358     luamacro.obj
 0001:0000a360       FIB_EXPANDENV              000000018000b360     luamacro.obj
 0001:0000a368       FIB_NOUSELASTHISTORY       000000018000b368     luamacro.obj
 0001:0000a370       FIB_BUTTONS                000000018000b370     luamacro.obj
 0001:0000a378       FIB_NOAMPERSAND            000000018000b378     luamacro.obj
 0001:0000a380       FIB_EDITPATH               000000018000b380     luamacro.obj
 0001:0000a388       FIB_EDITPATHEXEC           000000018000b388     luamacro.obj
 0001:0000a390       FIB_NONE                   000000018000b390     luamacro.obj
 0001:0000a398       FPF_LOADED                 000000018000b398     luamacro.obj
 0001:0000a3a0       FPF_ANSI                   000000018000b3a0     luamacro.obj
 0001:0000a3a8       FPF_NONE                   000000018000b3a8     luamacro.obj
 0001:0000a3b0       PN_CMPNAME                 000000018000b3b0     luamacro.obj
 0001:0000a3b8       PN_CMPNAMELIST             000000018000b3b8     luamacro.obj
 0001:0000a3c0       PN_GENERATENAME            000000018000b3c0     luamacro.obj
 0001:0000a3c8       PN_CHECKMASK               000000018000b3c8     luamacro.obj
 0001:0000a3d0       PN_SKIPPATH                000000018000b3d0     luamacro.obj
 0001:0000a3d8       PN_SHOWERRORMESSAGE        000000018000b3d8     luamacro.obj
 0001:0000a3e0       PN_NONE                    000000018000b3e0     luamacro.obj
 0001:0000a3e8       XLAT_SWITCHKEYBLAYOUT      000000018000b3e8     luamacro.obj
 0001:0000a3f0       XLAT_SWITCHKEYBBEEP        000000018000b3f0     luamacro.obj
 0001:0000a3f8       XLAT_USEKEYBLAYOUTNAME     000000018000b3f8     luamacro.obj
 0001:0000a400       XLAT_CONVERTALLCMDLINE     000000018000b400     luamacro.obj
 0001:0000a408       XLAT_NONE                  000000018000b408     luamacro.obj
 0001:0000a410       FRS_RETUPDIR               000000018000b410     luamacro.obj
 0001:0000a418       FRS_RECUR                  000000018000b418     luamacro.obj
 0001:0000a420       FRS_SCANSYMLINK            000000018000b420     luamacro.obj
 0001:0000a428       FRS_NONE                   000000018000b428     luamacro.obj
 0001:0000a430       MLF_SHOWERRMSG             000000018000b430     luamacro.obj
 0001:0000a438       MLF_DONOTUPDATEPANEL       000000018000b438     luamacro.obj
 0001:0000a440       MLF_HOLDTARGET             000000018000b440     luamacro.obj
 0001:0000a448       MLF_NONE                   000000018000b448     luamacro.obj
 0001:0000a450       FFFS_COMMAS                000000018000b450     luamacro.obj
 0001:0000a458       FFFS_FLOATSIZE             000000018000b458     luamacro.obj
 0001:0000a460       FFFS_SHOWBYTESINDEX        000000018000b460     luamacro.obj
 0001:0000a468       FFFS_ECONOMIC              000000018000b468     luamacro.obj
 0001:0000a470       FFFS_THOUSAND              000000018000b470     luamacro.obj
 0001:0000a478       FFFS_MINSIZEINDEX          000000018000b478     luamacro.obj
 0001:0000a480       FFFS_MINSIZEINDEX_MASK     000000018000b480     luamacro.obj
 0001:0000a488       FFFS_NONE                  000000018000b488     luamacro.obj
 0001:0000a490       PF_PRELOAD                 000000018000b490     luamacro.obj
 0001:0000a498       PF_DISABLEPANELS           000000018000b498     luamacro.obj
 0001:0000a4a0       PF_EDITOR                  000000018000b4a0     luamacro.obj
 0001:0000a4a8       PF_VIEWER                  000000018000b4a8     luamacro.obj
 0001:0000a4b0       PF_FULLCMDLINE             000000018000b4b0     luamacro.obj
 0001:0000a4b8       PF_DIALOG                  000000018000b4b8     luamacro.obj
 0001:0000a4c0       PF_NONE                    000000018000b4c0     luamacro.obj
 0001:0000a4c8       IPLFLAGS_SEPARATOR         000000018000b4c8     luamacro.obj
 0001:0000a4d0       IPLFLAGS_NONE              000000018000b4d0     luamacro.obj
 0001:0000a4d8       PMFLAGS_FULLSCREEN         000000018000b4d8     luamacro.obj
 0001:0000a4e0       PMFLAGS_DETAILEDSTATUS     000000018000b4e0     luamacro.obj
 0001:0000a4e8       PMFLAGS_ALIGNEXTENSIONS    000000018000b4e8     luamacro.obj
 0001:0000a4f0       PMFLAGS_CASECONVERSION     000000018000b4f0     luamacro.obj
 0001:0000a4f8       PMFLAGS_NONE               000000018000b4f8     luamacro.obj
 0001:0000a500       OPIF_DISABLEFILTER         000000018000b500     luamacro.obj
 0001:0000a508       OPIF_DISABLESORTGROUPS     000000018000b508     luamacro.obj
 0001:0000a510       OPIF_DISABLEHIGHLIGHTING   000000018000b510     luamacro.obj
 0001:0000a518       OPIF_ADDDOTS               000000018000b518     luamacro.obj
 0001:0000a520       OPIF_RAWSELECTION          000000018000b520     luamacro.obj
 0001:0000a528       OPIF_REALNAMES             000000018000b528     luamacro.obj
 0001:0000a530       OPIF_SHOWNAMESONLY         000000018000b530     luamacro.obj
 0001:0000a538       OPIF_SHOWRIGHTALIGNNAMES   000000018000b538     luamacro.obj
 0001:0000a540       OPIF_SHOWPRESERVECASE      000000018000b540     luamacro.obj
 0001:0000a548       OPIF_COMPAREFATTIME        000000018000b548     luamacro.obj
 0001:0000a550       OPIF_EXTERNALGET           000000018000b550     luamacro.obj
 0001:0000a558       OPIF_EXTERNALPUT           000000018000b558     luamacro.obj
 0001:0000a560       OPIF_EXTERNALDELETE        000000018000b560     luamacro.obj
 0001:0000a568       OPIF_EXTERNALMKDIR         000000018000b568     luamacro.obj
 0001:0000a570       OPIF_USEATTRHIGHLIGHTING   000000018000b570     luamacro.obj
 0001:0000a578       OPIF_USECRC32              000000018000b578     luamacro.obj
 0001:0000a580       OPIF_USEFREESIZE           000000018000b580     luamacro.obj
 0001:0000a588       OPIF_SHORTCUT              000000018000b588     luamacro.obj
 0001:0000a590       OPIF_NONE                  000000018000b590     luamacro.obj
 0001:0000a598       OPM_SILENT                 000000018000b598     luamacro.obj
 0001:0000a5a0       OPM_FIND                   000000018000b5a0     luamacro.obj
 0001:0000a5a8       OPM_VIEW                   000000018000b5a8     luamacro.obj
 0001:0000a5b0       OPM_EDIT                   000000018000b5b0     luamacro.obj
 0001:0000a5b8       OPM_TOPLEVEL               000000018000b5b8     luamacro.obj
 0001:0000a5c0       OPM_DESCR                  000000018000b5c0     luamacro.obj
 0001:0000a5c8       OPM_QUICKVIEW              000000018000b5c8     luamacro.obj
 0001:0000a5d0       OPM_PGDN                   000000018000b5d0     luamacro.obj
 0001:0000a5d8       OPM_COMMANDS               000000018000b5d8     luamacro.obj
 0001:0000a5e0       OPM_NONE                   000000018000b5e0     luamacro.obj
 0001:0000a5e8       FOSF_ACTIVE                000000018000b5e8     luamacro.obj
 0001:0000a5f0       FOSF_NONE                  000000018000b5f0     luamacro.obj
 0001:0000a5f8       PCIF_NONE                  000000018000b5f8     luamacro.obj
 0001:0000a600       FarGuid                    000000018000b600     luamacro.obj
 0001:0000a610       PDF_DIALOGEVENTDRAWENABLE  000000018000b610     luamacro.obj
 0001:0000a618       PDF_PROCESSINGERROR        000000018000b618     luamacro.obj
 0001:0000a620       LuamacroGuid               000000018000b620     luamacro.obj
 0001:0000a700       FCF_FG_4BIT                000000018000b700     lusercontrol.obj
 0001:0000a708       FCF_BG_4BIT                000000018000b708     lusercontrol.obj
 0001:0000a710       FCF_4BITMASK               000000018000b710     lusercontrol.obj
 0001:0000a718       FCF_RAWATTR_MASK           000000018000b718     lusercontrol.obj
 0001:0000a720       FCF_EXTENDEDFLAGS          000000018000b720     lusercontrol.obj
 0001:0000a728       FCF_FG_BOLD                000000018000b728     lusercontrol.obj
 0001:0000a730       FCF_FG_ITALIC              000000018000b730     lusercontrol.obj
 0001:0000a738       FCF_FG_UNDERLINE           000000018000b738     lusercontrol.obj
 0001:0000a740       FCF_STYLEMASK              000000018000b740     lusercontrol.obj
 0001:0000a748       FCF_NONE                   000000018000b748     lusercontrol.obj
 0001:0000a750       CDF_NONE                   000000018000b750     lusercontrol.obj
 0001:0000a758       FMSG_WARNING               000000018000b758     lusercontrol.obj
 0001:0000a760       FMSG_ERRORTYPE             000000018000b760     lusercontrol.obj
 0001:0000a768       FMSG_KEEPBACKGROUND        000000018000b768     lusercontrol.obj
 0001:0000a770       FMSG_LEFTALIGN             000000018000b770     lusercontrol.obj
 0001:0000a778       FMSG_ALLINONE              000000018000b778     lusercontrol.obj
 0001:0000a780       FMSG_MB_OK                 000000018000b780     lusercontrol.obj
 0001:0000a788       FMSG_MB_OKCANCEL           000000018000b788     lusercontrol.obj
 0001:0000a790       FMSG_MB_ABORTRETRYIGNORE   000000018000b790     lusercontrol.obj
 0001:0000a798       FMSG_MB_YESNO              000000018000b798     lusercontrol.obj
 0001:0000a7a0       FMSG_MB_YESNOCANCEL        000000018000b7a0     lusercontrol.obj
 0001:0000a7a8       FMSG_MB_RETRYCANCEL        000000018000b7a8     lusercontrol.obj
 0001:0000a7b0       FMSG_NONE                  000000018000b7b0     lusercontrol.obj
 0001:0000a7b8       DIF_BOXCOLOR               000000018000b7b8     lusercontrol.obj
 0001:0000a7c0       DIF_GROUP                  000000018000b7c0     lusercontrol.obj
 0001:0000a7c8       DIF_LEFTTEXT               000000018000b7c8     lusercontrol.obj
 0001:0000a7d0       DIF_MOVESELECT             000000018000b7d0     lusercontrol.obj
 0001:0000a7d8       DIF_SHOWAMPERSAND          000000018000b7d8     lusercontrol.obj
 0001:0000a7e0       DIF_CENTERGROUP            000000018000b7e0     lusercontrol.obj
 0001:0000a7e8       DIF_NOBRACKETS             000000018000b7e8     lusercontrol.obj
 0001:0000a7f0       DIF_MANUALADDHISTORY       000000018000b7f0     lusercontrol.obj
 0001:0000a7f8       DIF_SEPARATOR              000000018000b7f8     lusercontrol.obj
 0001:0000a800       DIF_SEPARATOR2             000000018000b800     lusercontrol.obj
 0001:0000a808       DIF_EDITOR                 000000018000b808     lusercontrol.obj
 0001:0000a810       DIF_LISTNOAMPERSAND        000000018000b810     lusercontrol.obj
 0001:0000a818       DIF_LISTNOBOX              000000018000b818     lusercontrol.obj
 0001:0000a820       DIF_HISTORY                000000018000b820     lusercontrol.obj
 0001:0000a828       DIF_BTNNOCLOSE             000000018000b828     lusercontrol.obj
 0001:0000a830       DIF_CENTERTEXT             000000018000b830     lusercontrol.obj
 0001:0000a838       DIF_SEPARATORUSER          000000018000b838     lusercontrol.obj
 0001:0000a840       DIF_SETSHIELD              000000018000b840     lusercontrol.obj
 0001:0000a848       DIF_EDITEXPAND             000000018000b848     lusercontrol.obj
 0001:0000a850       DIF_DROPDOWNLIST           000000018000b850     lusercontrol.obj
 0001:0000a858       DIF_USELASTHISTORY         000000018000b858     lusercontrol.obj
 0001:0000a860       DIF_MASKEDIT               000000018000b860     lusercontrol.obj
 0001:0000a868       DIF_LISTTRACKMOUSE         000000018000b868     lusercontrol.obj
 0001:0000a870       DIF_LISTTRACKMOUSEINFOCUS  000000018000b870     lusercontrol.obj
 0001:0000a878       DIF_SELECTONENTRY          000000018000b878     lusercontrol.obj
 0001:0000a880       DIF_3STATE                 000000018000b880     lusercontrol.obj
 0001:0000a888       DIF_EDITPATH               000000018000b888     lusercontrol.obj
 0001:0000a890       DIF_LISTWRAPMODE           000000018000b890     lusercontrol.obj
 0001:0000a898       DIF_NOAUTOCOMPLETE         000000018000b898     lusercontrol.obj
 0001:0000a8a0       DIF_LISTAUTOHIGHLIGHT      000000018000b8a0     lusercontrol.obj
 0001:0000a8a8       DIF_LISTNOCLOSE            000000018000b8a8     lusercontrol.obj
 0001:0000a8b0       DIF_EDITPATHEXEC           000000018000b8b0     lusercontrol.obj
 0001:0000a8b8       DIF_HIDDEN                 000000018000b8b8     lusercontrol.obj
 0001:0000a8c0       DIF_READONLY               000000018000b8c0     lusercontrol.obj
 0001:0000a8c8       DIF_NOFOCUS                000000018000b8c8     lusercontrol.obj
 0001:0000a8d0       DIF_DISABLE                000000018000b8d0     lusercontrol.obj
 0001:0000a8d8       DIF_DEFAULTBUTTON          000000018000b8d8     lusercontrol.obj
 0001:0000a8e0       DIF_FOCUS                  000000018000b8e0     lusercontrol.obj
 0001:0000a8e8       DIF_RIGHTTEXT              000000018000b8e8     lusercontrol.obj
 0001:0000a8f0       DIF_WORDWRAP               000000018000b8f0     lusercontrol.obj
 0001:0000a8f8       DIF_NONE                   000000018000b8f8     lusercontrol.obj
 0001:0000a900       LIF_SELECTED               000000018000b900     lusercontrol.obj
 0001:0000a908       LIF_CHECKED                000000018000b908     lusercontrol.obj
 0001:0000a910       LIF_SEPARATOR              000000018000b910     lusercontrol.obj
 0001:0000a918       LIF_DISABLE                000000018000b918     lusercontrol.obj
 0001:0000a920       LIF_GRAYED                 000000018000b920     lusercontrol.obj
 0001:0000a928       LIF_HIDDEN                 000000018000b928     lusercontrol.obj
 0001:0000a930       LIF_DELETEUSERDATA         000000018000b930     lusercontrol.obj
 0001:0000a938       LIF_NONE                   000000018000b938     lusercontrol.obj
 0001:0000a940       LIFIND_EXACTMATCH          000000018000b940     lusercontrol.obj
 0001:0000a948       LIFIND_NONE                000000018000b948     lusercontrol.obj
 0001:0000a950       LINFO_SHOWNOBOX            000000018000b950     lusercontrol.obj
 0001:0000a958       LINFO_AUTOHIGHLIGHT        000000018000b958     lusercontrol.obj
 0001:0000a960       LINFO_REVERSEHIGHLIGHT     000000018000b960     lusercontrol.obj
 0001:0000a968       LINFO_WRAPMODE             000000018000b968     lusercontrol.obj
 0001:0000a970       LINFO_SHOWAMPERSAND        000000018000b970     lusercontrol.obj
 0001:0000a978       LINFO_NONE                 000000018000b978     lusercontrol.obj
 0001:0000a980       FDLG_WARNING               000000018000b980     lusercontrol.obj
 0001:0000a988       FDLG_SMALLDIALOG           000000018000b988     lusercontrol.obj
 0001:0000a990       FDLG_NODRAWSHADOW          000000018000b990     lusercontrol.obj
 0001:0000a998       FDLG_NODRAWPANEL           000000018000b998     lusercontrol.obj
 0001:0000a9a0       FDLG_KEEPCONSOLETITLE      000000018000b9a0     lusercontrol.obj
 0001:0000a9a8       FDLG_NONMODAL              000000018000b9a8     lusercontrol.obj
 0001:0000a9b0       FDLG_NONE                  000000018000b9b0     lusercontrol.obj
 0001:0000a9b8       MIF_SELECTED               000000018000b9b8     lusercontrol.obj
 0001:0000a9c0       MIF_CHECKED                000000018000b9c0     lusercontrol.obj
 0001:0000a9c8       MIF_SEPARATOR              000000018000b9c8     lusercontrol.obj
 0001:0000a9d0       MIF_DISABLE                000000018000b9d0     lusercontrol.obj
 0001:0000a9d8       MIF_GRAYED                 000000018000b9d8     lusercontrol.obj
 0001:0000a9e0       MIF_HIDDEN                 000000018000b9e0     lusercontrol.obj
 0001:0000a9e8       MIF_NONE                   000000018000b9e8     lusercontrol.obj
 0001:0000a9f0       FMENU_SHOWAMPERSAND        000000018000b9f0     lusercontrol.obj
 0001:0000a9f8       FMENU_WRAPMODE             000000018000b9f8     lusercontrol.obj
 0001:0000aa00       FMENU_AUTOHIGHLIGHT        000000018000ba00     lusercontrol.obj
 0001:0000aa08       FMENU_REVERSEAUTOHIGHLIGHT 000000018000ba08     lusercontrol.obj
 0001:0000aa10       FMENU_CHANGECONSOLETITLE   000000018000ba10     lusercontrol.obj
 0001:0000aa18       FMENU_NONE                 000000018000ba18     lusercontrol.obj
 0001:0000aa20       PPIF_SELECTED              000000018000ba20     lusercontrol.obj
 0001:0000aa28       PPIF_PROCESSDESCR          000000018000ba28     lusercontrol.obj
 0001:0000aa30       PPIF_NONE                  000000018000ba30     lusercontrol.obj
 0001:0000aa38       PFLAGS_SHOWHIDDEN          000000018000ba38     lusercontrol.obj
 0001:0000aa40       PFLAGS_HIGHLIGHT           000000018000ba40     lusercontrol.obj
 0001:0000aa48       PFLAGS_REVERSESORTORDER    000000018000ba48     lusercontrol.obj
 0001:0000aa50       PFLAGS_USESORTGROUPS       000000018000ba50     lusercontrol.obj
 0001:0000aa58       PFLAGS_SELECTEDFIRST       000000018000ba58     lusercontrol.obj
 0001:0000aa60       PFLAGS_REALNAMES           000000018000ba60     lusercontrol.obj
 0001:0000aa68       PFLAGS_PANELLEFT           000000018000ba68     lusercontrol.obj
 0001:0000aa70       PFLAGS_DIRECTORIESFIRST    000000018000ba70     lusercontrol.obj
 0001:0000aa78       PFLAGS_USECRC32            000000018000ba78     lusercontrol.obj
 0001:0000aa80       PFLAGS_PLUGIN              000000018000ba80     lusercontrol.obj
 0001:0000aa88       PFLAGS_VISIBLE             000000018000ba88     lusercontrol.obj
 0001:0000aa90       PFLAGS_FOCUS               000000018000ba90     lusercontrol.obj
 0001:0000aa98       PFLAGS_ALTERNATIVENAMES    000000018000ba98     lusercontrol.obj
 0001:0000aaa0       PFLAGS_SHORTCUT            000000018000baa0     lusercontrol.obj
 0001:0000aaa8       PFLAGS_NONE                000000018000baa8     lusercontrol.obj
 0001:0000aab0       VF_NONMODAL                000000018000bab0     lusercontrol.obj
 0001:0000aab8       VF_DELETEONCLOSE           000000018000bab8     lusercontrol.obj
 0001:0000aac0       VF_ENABLE_F6               000000018000bac0     lusercontrol.obj
 0001:0000aac8       VF_DISABLEHISTORY          000000018000bac8     lusercontrol.obj
 0001:0000aad0       VF_IMMEDIATERETURN         000000018000bad0     lusercontrol.obj
 0001:0000aad8       VF_DELETEONLYFILEONCLOSE   000000018000bad8     lusercontrol.obj
 0001:0000aae0       VF_NONE                    000000018000bae0     lusercontrol.obj
 0001:0000aae8       EF_NONMODAL                000000018000bae8     lusercontrol.obj
 0001:0000aaf0       EF_CREATENEW               000000018000baf0     lusercontrol.obj
 0001:0000aaf8       EF_ENABLE_F6               000000018000baf8     lusercontrol.obj
 0001:0000ab00       EF_DISABLEHISTORY          000000018000bb00     lusercontrol.obj
 0001:0000ab08       EF_DELETEONCLOSE           000000018000bb08     lusercontrol.obj
 0001:0000ab10       EF_IMMEDIATERETURN         000000018000bb10     lusercontrol.obj
 0001:0000ab18       EF_DELETEONLYFILEONCLOSE   000000018000bb18     lusercontrol.obj
 0001:0000ab20       EF_LOCKED                  000000018000bb20     lusercontrol.obj
 0001:0000ab28       EF_DISABLESAVEPOS          000000018000bb28     lusercontrol.obj
 0001:0000ab30       EF_OPENMODE_MASK           000000018000bb30     lusercontrol.obj
 0001:0000ab38       EF_OPENMODE_QUERY          000000018000bb38     lusercontrol.obj
 0001:0000ab40       EF_OPENMODE_NEWIFOPEN      000000018000bb40     lusercontrol.obj
 0001:0000ab48       EF_OPENMODE_USEEXISTING    000000018000bb48     lusercontrol.obj
 0001:0000ab50       EF_OPENMODE_BREAKIFOPEN    000000018000bb50     lusercontrol.obj
 0001:0000ab58       EF_OPENMODE_RELOADIFOPEN   000000018000bb58     lusercontrol.obj
 0001:0000ab60       EN_NONE                    000000018000bb60     lusercontrol.obj
 0001:0000ab68       FHELP_NOSHOWERROR          000000018000bb68     lusercontrol.obj
 0001:0000ab70       FHELP_SELFHELP             000000018000bb70     lusercontrol.obj
 0001:0000ab78       FHELP_FARHELP              000000018000bb78     lusercontrol.obj
 0001:0000ab80       FHELP_CUSTOMFILE           000000018000bb80     lusercontrol.obj
 0001:0000ab88       FHELP_CUSTOMPATH           000000018000bb88     lusercontrol.obj
 0001:0000ab90       FHELP_GUID                 000000018000bb90     lusercontrol.obj
 0001:0000ab98       FHELP_USECONTENTS          000000018000bb98     lusercontrol.obj
 0001:0000aba0       FHELP_NONE                 000000018000bba0     lusercontrol.obj
 0001:0000aba8       KMFLAGS_SILENTCHECK        000000018000bba8     lusercontrol.obj
 0001:0000abb0       KMFLAGS_NOSENDKEYSTOPLUGINS 000000018000bbb0     lusercontrol.obj
 0001:0000abb8       KMFLAGS_ENABLEOUTPUT       000000018000bbb8     lusercontrol.obj
 0001:0000abc0       KMFLAGS_LANGMASK           000000018000bbc0     lusercontrol.obj
 0001:0000abc8       KMFLAGS_LUA                000000018000bbc8     lusercontrol.obj
 0001:0000abd0       KMFLAGS_MOONSCRIPT         000000018000bbd0     lusercontrol.obj
 0001:0000abd8       KMFLAGS_NONE               000000018000bbd8     lusercontrol.obj
 0001:0000abe0       AKMFLAGS_NONE              000000018000bbe0     lusercontrol.obj
 0001:0000abe8       FSETCLR_REDRAW             000000018000bbe8     lusercontrol.obj
 0001:0000abf0       FSETCLR_NONE               000000018000bbf0     lusercontrol.obj
 0001:0000abf8       WIF_MODIFIED               000000018000bbf8     lusercontrol.obj
 0001:0000ac00       WIF_CURRENT                000000018000bc00     lusercontrol.obj
 0001:0000ac08       WIF_MODAL                  000000018000bc08     lusercontrol.obj
 0001:0000ac10       WIF_NONE                   000000018000bc10     lusercontrol.obj
 0001:0000ac18       VOPT_SAVEFILEPOSITION      000000018000bc18     lusercontrol.obj
 0001:0000ac20       VOPT_AUTODETECTCODEPAGE    000000018000bc20     lusercontrol.obj
 0001:0000ac28       VOPT_SHOWTITLEBAR          000000018000bc28     lusercontrol.obj
 0001:0000ac30       VOPT_SHOWKEYBAR            000000018000bc30     lusercontrol.obj
 0001:0000ac38       VOPT_SHOWSCROLLBAR         000000018000bc38     lusercontrol.obj
 0001:0000ac40       VOPT_QUICKVIEW             000000018000bc40     lusercontrol.obj
 0001:0000ac48       VOPT_NONE                  000000018000bc48     lusercontrol.obj
 0001:0000ac50       VSMFL_REDRAW               000000018000bc50     lusercontrol.obj
 0001:0000ac58       VSMFL_NONE                 000000018000bc58     lusercontrol.obj
 0001:0000ac60       VSP_NOREDRAW               000000018000bc60     lusercontrol.obj
 0001:0000ac68       VSP_PERCENT                000000018000bc68     lusercontrol.obj
 0001:0000ac70       VSP_RELATIVE               000000018000bc70     lusercontrol.obj
 0001:0000ac78       VSP_NORETNEWPOS            000000018000bc78     lusercontrol.obj
 0001:0000ac80       VSP_NONE                   000000018000bc80     lusercontrol.obj
 0001:0000ac88       VMF_WRAP                   000000018000bc88     lusercontrol.obj
 0001:0000ac90       VMF_WORDWRAP               000000018000bc90     lusercontrol.obj
 0001:0000ac98       VMF_NONE                   000000018000bc98     lusercontrol.obj
 0001:0000aca0       ECF_TABMARKFIRST           000000018000bca0     lusercontrol.obj
 0001:0000aca8       ECF_TABMARKCURRENT         000000018000bca8     lusercontrol.obj
 0001:0000acb0       ECF_AUTODELETE             000000018000bcb0     lusercontrol.obj
 0001:0000acb8       ECF_NONE                   000000018000bcb8     lusercontrol.obj
 0001:0000acc0       FIB_ENABLEEMPTY            000000018000bcc0     lusercontrol.obj
 0001:0000acc8       FIB_PASSWORD               000000018000bcc8     lusercontrol.obj
 0001:0000acd0       FIB_EXPANDENV              000000018000bcd0     lusercontrol.obj
 0001:0000acd8       FIB_NOUSELASTHISTORY       000000018000bcd8     lusercontrol.obj
 0001:0000ace0       FIB_BUTTONS                000000018000bce0     lusercontrol.obj
 0001:0000ace8       FIB_NOAMPERSAND            000000018000bce8     lusercontrol.obj
 0001:0000acf0       FIB_EDITPATH               000000018000bcf0     lusercontrol.obj
 0001:0000acf8       FIB_EDITPATHEXEC           000000018000bcf8     lusercontrol.obj
 0001:0000ad00       FIB_NONE                   000000018000bd00     lusercontrol.obj
 0001:0000ad08       FPF_LOADED                 000000018000bd08     lusercontrol.obj
 0001:0000ad10       FPF_ANSI                   000000018000bd10     lusercontrol.obj
 0001:0000ad18       FPF_NONE                   000000018000bd18     lusercontrol.obj
 0001:0000ad20       PN_CMPNAME                 000000018000bd20     lusercontrol.obj
 0001:0000ad28       PN_CMPNAMELIST             000000018000bd28     lusercontrol.obj
 0001:0000ad30       PN_GENERATENAME            000000018000bd30     lusercontrol.obj
 0001:0000ad38       PN_CHECKMASK               000000018000bd38     lusercontrol.obj
 0001:0000ad40       PN_SKIPPATH                000000018000bd40     lusercontrol.obj
 0001:0000ad48       PN_SHOWERRORMESSAGE        000000018000bd48     lusercontrol.obj
 0001:0000ad50       PN_NONE                    000000018000bd50     lusercontrol.obj
 0001:0000ad58       XLAT_SWITCHKEYBLAYOUT      000000018000bd58     lusercontrol.obj
 0001:0000ad60       XLAT_SWITCHKEYBBEEP        000000018000bd60     lusercontrol.obj
 0001:0000ad68       XLAT_USEKEYBLAYOUTNAME     000000018000bd68     lusercontrol.obj
 0001:0000ad70       XLAT_CONVERTALLCMDLINE     000000018000bd70     lusercontrol.obj
 0001:0000ad78       XLAT_NONE                  000000018000bd78     lusercontrol.obj
 0001:0000ad80       FRS_RETUPDIR               000000018000bd80     lusercontrol.obj
 0001:0000ad88       FRS_RECUR                  000000018000bd88     lusercontrol.obj
 0001:0000ad90       FRS_SCANSYMLINK            000000018000bd90     lusercontrol.obj
 0001:0000ad98       FRS_NONE                   000000018000bd98     lusercontrol.obj
 0001:0000ada0       MLF_SHOWERRMSG             000000018000bda0     lusercontrol.obj
 0001:0000ada8       MLF_DONOTUPDATEPANEL       000000018000bda8     lusercontrol.obj
 0001:0000adb0       MLF_HOLDTARGET             000000018000bdb0     lusercontrol.obj
 0001:0000adb8       MLF_NONE                   000000018000bdb8     lusercontrol.obj
 0001:0000adc0       FFFS_COMMAS                000000018000bdc0     lusercontrol.obj
 0001:0000adc8       FFFS_FLOATSIZE             000000018000bdc8     lusercontrol.obj
 0001:0000add0       FFFS_SHOWBYTESINDEX        000000018000bdd0     lusercontrol.obj
 0001:0000add8       FFFS_ECONOMIC              000000018000bdd8     lusercontrol.obj
 0001:0000ade0       FFFS_THOUSAND              000000018000bde0     lusercontrol.obj
 0001:0000ade8       FFFS_MINSIZEINDEX          000000018000bde8     lusercontrol.obj
 0001:0000adf0       FFFS_MINSIZEINDEX_MASK     000000018000bdf0     lusercontrol.obj
 0001:0000adf8       FFFS_NONE                  000000018000bdf8     lusercontrol.obj
 0001:0000ae00       PF_PRELOAD                 000000018000be00     lusercontrol.obj
 0001:0000ae08       PF_DISABLEPANELS           000000018000be08     lusercontrol.obj
 0001:0000ae10       PF_EDITOR                  000000018000be10     lusercontrol.obj
 0001:0000ae18       PF_VIEWER                  000000018000be18     lusercontrol.obj
 0001:0000ae20       PF_FULLCMDLINE             000000018000be20     lusercontrol.obj
 0001:0000ae28       PF_DIALOG                  000000018000be28     lusercontrol.obj
 0001:0000ae30       PF_NONE                    000000018000be30     lusercontrol.obj
 0001:0000ae38       IPLFLAGS_SEPARATOR         000000018000be38     lusercontrol.obj
 0001:0000ae40       IPLFLAGS_NONE              000000018000be40     lusercontrol.obj
 0001:0000ae48       PMFLAGS_FULLSCREEN         000000018000be48     lusercontrol.obj
 0001:0000ae50       PMFLAGS_DETAILEDSTATUS     000000018000be50     lusercontrol.obj
 0001:0000ae58       PMFLAGS_ALIGNEXTENSIONS    000000018000be58     lusercontrol.obj
 0001:0000ae60       PMFLAGS_CASECONVERSION     000000018000be60     lusercontrol.obj
 0001:0000ae68       PMFLAGS_NONE               000000018000be68     lusercontrol.obj
 0001:0000ae70       OPIF_DISABLEFILTER         000000018000be70     lusercontrol.obj
 0001:0000ae78       OPIF_DISABLESORTGROUPS     000000018000be78     lusercontrol.obj
 0001:0000ae80       OPIF_DISABLEHIGHLIGHTING   000000018000be80     lusercontrol.obj
 0001:0000ae88       OPIF_ADDDOTS               000000018000be88     lusercontrol.obj
 0001:0000ae90       OPIF_RAWSELECTION          000000018000be90     lusercontrol.obj
 0001:0000ae98       OPIF_REALNAMES             000000018000be98     lusercontrol.obj
 0001:0000aea0       OPIF_SHOWNAMESONLY         000000018000bea0     lusercontrol.obj
 0001:0000aea8       OPIF_SHOWRIGHTALIGNNAMES   000000018000bea8     lusercontrol.obj
 0001:0000aeb0       OPIF_SHOWPRESERVECASE      000000018000beb0     lusercontrol.obj
 0001:0000aeb8       OPIF_COMPAREFATTIME        000000018000beb8     lusercontrol.obj
 0001:0000aec0       OPIF_EXTERNALGET           000000018000bec0     lusercontrol.obj
 0001:0000aec8       OPIF_EXTERNALPUT           000000018000bec8     lusercontrol.obj
 0001:0000aed0       OPIF_EXTERNALDELETE        000000018000bed0     lusercontrol.obj
 0001:0000aed8       OPIF_EXTERNALMKDIR         000000018000bed8     lusercontrol.obj
 0001:0000aee0       OPIF_USEATTRHIGHLIGHTING   000000018000bee0     lusercontrol.obj
 0001:0000aee8       OPIF_USECRC32              000000018000bee8     lusercontrol.obj
 0001:0000aef0       OPIF_USEFREESIZE           000000018000bef0     lusercontrol.obj
 0001:0000aef8       OPIF_SHORTCUT              000000018000bef8     lusercontrol.obj
 0001:0000af00       OPIF_NONE                  000000018000bf00     lusercontrol.obj
 0001:0000af08       OPM_SILENT                 000000018000bf08     lusercontrol.obj
 0001:0000af10       OPM_FIND                   000000018000bf10     lusercontrol.obj
 0001:0000af18       OPM_VIEW                   000000018000bf18     lusercontrol.obj
 0001:0000af20       OPM_EDIT                   000000018000bf20     lusercontrol.obj
 0001:0000af28       OPM_TOPLEVEL               000000018000bf28     lusercontrol.obj
 0001:0000af30       OPM_DESCR                  000000018000bf30     lusercontrol.obj
 0001:0000af38       OPM_QUICKVIEW              000000018000bf38     lusercontrol.obj
 0001:0000af40       OPM_PGDN                   000000018000bf40     lusercontrol.obj
 0001:0000af48       OPM_COMMANDS               000000018000bf48     lusercontrol.obj
 0001:0000af50       OPM_NONE                   000000018000bf50     lusercontrol.obj
 0001:0000af58       FOSF_ACTIVE                000000018000bf58     lusercontrol.obj
 0001:0000af60       FOSF_NONE                  000000018000bf60     lusercontrol.obj
 0001:0000af68       PCIF_NONE                  000000018000bf68     lusercontrol.obj
 0001:0000af70       FarGuid                    000000018000bf70     lusercontrol.obj
 0001:0000b168       FCF_FG_4BIT                000000018000c168     service.obj
 0001:0000b170       FCF_BG_4BIT                000000018000c170     service.obj
 0001:0000b178       FCF_4BITMASK               000000018000c178     service.obj
 0001:0000b180       FCF_RAWATTR_MASK           000000018000c180     service.obj
 0001:0000b188       FCF_EXTENDEDFLAGS          000000018000c188     service.obj
 0001:0000b190       FCF_FG_BOLD                000000018000c190     service.obj
 0001:0000b198       FCF_FG_ITALIC              000000018000c198     service.obj
 0001:0000b1a0       FCF_FG_UNDERLINE           000000018000c1a0     service.obj
 0001:0000b1a8       FCF_STYLEMASK              000000018000c1a8     service.obj
 0001:0000b1b0       FCF_NONE                   000000018000c1b0     service.obj
 0001:0000b1b8       CDF_NONE                   000000018000c1b8     service.obj
 0001:0000b1c0       FMSG_WARNING               000000018000c1c0     service.obj
 0001:0000b1c8       FMSG_ERRORTYPE             000000018000c1c8     service.obj
 0001:0000b1d0       FMSG_KEEPBACKGROUND        000000018000c1d0     service.obj
 0001:0000b1d8       FMSG_LEFTALIGN             000000018000c1d8     service.obj
 0001:0000b1e0       FMSG_ALLINONE              000000018000c1e0     service.obj
 0001:0000b1e8       FMSG_MB_OK                 000000018000c1e8     service.obj
 0001:0000b1f0       FMSG_MB_OKCANCEL           000000018000c1f0     service.obj
 0001:0000b1f8       FMSG_MB_ABORTRETRYIGNORE   000000018000c1f8     service.obj
 0001:0000b200       FMSG_MB_YESNO              000000018000c200     service.obj
 0001:0000b208       FMSG_MB_YESNOCANCEL        000000018000c208     service.obj
 0001:0000b210       FMSG_MB_RETRYCANCEL        000000018000c210     service.obj
 0001:0000b218       FMSG_NONE                  000000018000c218     service.obj
 0001:0000b220       DIF_BOXCOLOR               000000018000c220     service.obj
 0001:0000b228       DIF_GROUP                  000000018000c228     service.obj
 0001:0000b230       DIF_LEFTTEXT               000000018000c230     service.obj
 0001:0000b238       DIF_MOVESELECT             000000018000c238     service.obj
 0001:0000b240       DIF_SHOWAMPERSAND          000000018000c240     service.obj
 0001:0000b248       DIF_CENTERGROUP            000000018000c248     service.obj
 0001:0000b250       ?key@?3??far_Menu@@9@9     000000018000c250     service.obj
 0001:0000b258       DIF_NOBRACKETS             000000018000c258     service.obj
 0001:0000b260       DIF_MANUALADDHISTORY       000000018000c260     service.obj
 0001:0000b268       DIF_SEPARATOR              000000018000c268     service.obj
 0001:0000b270       DIF_SEPARATOR2             000000018000c270     service.obj
 0001:0000b278       DIF_EDITOR                 000000018000c278     service.obj
 0001:0000b280       DIF_LISTNOAMPERSAND        000000018000c280     service.obj
 0001:0000b288       DIF_LISTNOBOX              000000018000c288     service.obj
 0001:0000b290       DIF_HISTORY                000000018000c290     service.obj
 0001:0000b298       DIF_BTNNOCLOSE             000000018000c298     service.obj
 0001:0000b2a0       DIF_CENTERTEXT             000000018000c2a0     service.obj
 0001:0000b2a8       DIF_SEPARATORUSER          000000018000c2a8     service.obj
 0001:0000b2b0       DIF_SETSHIELD              000000018000c2b0     service.obj
 0001:0000b2b8       DIF_EDITEXPAND             000000018000c2b8     service.obj
 0001:0000b2c0       DIF_DROPDOWNLIST           000000018000c2c0     service.obj
 0001:0000b2c8       DIF_USELASTHISTORY         000000018000c2c8     service.obj
 0001:0000b2d0       DIF_MASKEDIT               000000018000c2d0     service.obj
 0001:0000b2d8       DIF_LISTTRACKMOUSE         000000018000c2d8     service.obj
 0001:0000b2e0       DIF_LISTTRACKMOUSEINFOCUS  000000018000c2e0     service.obj
 0001:0000b2e8       DIF_SELECTONENTRY          000000018000c2e8     service.obj
 0001:0000b2f0       DIF_3STATE                 000000018000c2f0     service.obj
 0001:0000b2f8       DIF_EDITPATH               000000018000c2f8     service.obj
 0001:0000b300       DIF_LISTWRAPMODE           000000018000c300     service.obj
 0001:0000b308       DIF_NOAUTOCOMPLETE         000000018000c308     service.obj
 0001:0000b310       DIF_LISTAUTOHIGHLIGHT      000000018000c310     service.obj
 0001:0000b318       DIF_LISTNOCLOSE            000000018000c318     service.obj
 0001:0000b320       DIF_EDITPATHEXEC           000000018000c320     service.obj
 0001:0000b328       DIF_HIDDEN                 000000018000c328     service.obj
 0001:0000b330       DIF_READONLY               000000018000c330     service.obj
 0001:0000b338       DIF_NOFOCUS                000000018000c338     service.obj
 0001:0000b340       DIF_DISABLE                000000018000c340     service.obj
 0001:0000b348       DIF_DEFAULTBUTTON          000000018000c348     service.obj
 0001:0000b350       DIF_FOCUS                  000000018000c350     service.obj
 0001:0000b358       DIF_RIGHTTEXT              000000018000c358     service.obj
 0001:0000b360       DIF_WORDWRAP               000000018000c360     service.obj
 0001:0000b368       DIF_NONE                   000000018000c368     service.obj
 0001:0000b370       LIF_SELECTED               000000018000c370     service.obj
 0001:0000b378       LIF_CHECKED                000000018000c378     service.obj
 0001:0000b380       LIF_SEPARATOR              000000018000c380     service.obj
 0001:0000b388       LIF_DISABLE                000000018000c388     service.obj
 0001:0000b390       LIF_GRAYED                 000000018000c390     service.obj
 0001:0000b398       LIF_HIDDEN                 000000018000c398     service.obj
 0001:0000b3a0       LIF_DELETEUSERDATA         000000018000c3a0     service.obj
 0001:0000b3a8       LIF_NONE                   000000018000c3a8     service.obj
 0001:0000b3b0       LIFIND_EXACTMATCH          000000018000c3b0     service.obj
 0001:0000b3b8       LIFIND_NONE                000000018000c3b8     service.obj
 0001:0000b3c0       LINFO_SHOWNOBOX            000000018000c3c0     service.obj
 0001:0000b3c8       LINFO_AUTOHIGHLIGHT        000000018000c3c8     service.obj
 0001:0000b3d0       LINFO_REVERSEHIGHLIGHT     000000018000c3d0     service.obj
 0001:0000b3d8       LINFO_WRAPMODE             000000018000c3d8     service.obj
 0001:0000b3e0       LINFO_SHOWAMPERSAND        000000018000c3e0     service.obj
 0001:0000b3e8       LINFO_NONE                 000000018000c3e8     service.obj
 0001:0000b3f0       FDLG_WARNING               000000018000c3f0     service.obj
 0001:0000b3f8       FDLG_SMALLDIALOG           000000018000c3f8     service.obj
 0001:0000b400       FDLG_NODRAWSHADOW          000000018000c400     service.obj
 0001:0000b408       FDLG_NODRAWPANEL           000000018000c408     service.obj
 0001:0000b410       FDLG_KEEPCONSOLETITLE      000000018000c410     service.obj
 0001:0000b418       FDLG_NONMODAL              000000018000c418     service.obj
 0001:0000b420       FDLG_NONE                  000000018000c420     service.obj
 0001:0000b428       MIF_SELECTED               000000018000c428     service.obj
 0001:0000b430       MIF_CHECKED                000000018000c430     service.obj
 0001:0000b438       MIF_SEPARATOR              000000018000c438     service.obj
 0001:0000b440       MIF_DISABLE                000000018000c440     service.obj
 0001:0000b448       MIF_GRAYED                 000000018000c448     service.obj
 0001:0000b450       MIF_HIDDEN                 000000018000c450     service.obj
 0001:0000b458       MIF_NONE                   000000018000c458     service.obj
 0001:0000b460       FMENU_SHOWAMPERSAND        000000018000c460     service.obj
 0001:0000b468       FMENU_WRAPMODE             000000018000c468     service.obj
 0001:0000b470       FMENU_AUTOHIGHLIGHT        000000018000c470     service.obj
 0001:0000b478       FMENU_REVERSEAUTOHIGHLIGHT 000000018000c478     service.obj
 0001:0000b480       FMENU_CHANGECONSOLETITLE   000000018000c480     service.obj
 0001:0000b488       FMENU_NONE                 000000018000c488     service.obj
 0001:0000b490       PPIF_SELECTED              000000018000c490     service.obj
 0001:0000b498       PPIF_PROCESSDESCR          000000018000c498     service.obj
 0001:0000b4a0       PPIF_NONE                  000000018000c4a0     service.obj
 0001:0000b4a8       PFLAGS_SHOWHIDDEN          000000018000c4a8     service.obj
 0001:0000b4b0       PFLAGS_HIGHLIGHT           000000018000c4b0     service.obj
 0001:0000b4b8       PFLAGS_REVERSESORTORDER    000000018000c4b8     service.obj
 0001:0000b4c0       PFLAGS_USESORTGROUPS       000000018000c4c0     service.obj
 0001:0000b4c8       PFLAGS_SELECTEDFIRST       000000018000c4c8     service.obj
 0001:0000b4d0       PFLAGS_REALNAMES           000000018000c4d0     service.obj
 0001:0000b4d8       PFLAGS_PANELLEFT           000000018000c4d8     service.obj
 0001:0000b4e0       PFLAGS_DIRECTORIESFIRST    000000018000c4e0     service.obj
 0001:0000b4e8       PFLAGS_USECRC32            000000018000c4e8     service.obj
 0001:0000b4f0       PFLAGS_PLUGIN              000000018000c4f0     service.obj
 0001:0000b4f8       PFLAGS_VISIBLE             000000018000c4f8     service.obj
 0001:0000b500       PFLAGS_FOCUS               000000018000c500     service.obj
 0001:0000b508       PFLAGS_ALTERNATIVENAMES    000000018000c508     service.obj
 0001:0000b510       PFLAGS_SHORTCUT            000000018000c510     service.obj
 0001:0000b518       PFLAGS_NONE                000000018000c518     service.obj
 0001:0000b520       VF_NONMODAL                000000018000c520     service.obj
 0001:0000b528       VF_DELETEONCLOSE           000000018000c528     service.obj
 0001:0000b530       VF_ENABLE_F6               000000018000c530     service.obj
 0001:0000b538       VF_DISABLEHISTORY          000000018000c538     service.obj
 0001:0000b540       VF_IMMEDIATERETURN         000000018000c540     service.obj
 0001:0000b548       VF_DELETEONLYFILEONCLOSE   000000018000c548     service.obj
 0001:0000b550       VF_NONE                    000000018000c550     service.obj
 0001:0000b558       EF_NONMODAL                000000018000c558     service.obj
 0001:0000b560       EF_CREATENEW               000000018000c560     service.obj
 0001:0000b568       EF_ENABLE_F6               000000018000c568     service.obj
 0001:0000b570       EF_DISABLEHISTORY          000000018000c570     service.obj
 0001:0000b578       EF_DELETEONCLOSE           000000018000c578     service.obj
 0001:0000b580       EF_IMMEDIATERETURN         000000018000c580     service.obj
 0001:0000b588       EF_DELETEONLYFILEONCLOSE   000000018000c588     service.obj
 0001:0000b590       EF_LOCKED                  000000018000c590     service.obj
 0001:0000b598       EF_DISABLESAVEPOS          000000018000c598     service.obj
 0001:0000b5a0       EF_OPENMODE_MASK           000000018000c5a0     service.obj
 0001:0000b5a8       EF_OPENMODE_QUERY          000000018000c5a8     service.obj
 0001:0000b5b0       EF_OPENMODE_NEWIFOPEN      000000018000c5b0     service.obj
 0001:0000b5b8       EF_OPENMODE_USEEXISTING    000000018000c5b8     service.obj
 0001:0000b5c0       EF_OPENMODE_BREAKIFOPEN    000000018000c5c0     service.obj
 0001:0000b5c8       EF_OPENMODE_RELOADIFOPEN   000000018000c5c8     service.obj
 0001:0000b5d0       EN_NONE                    000000018000c5d0     service.obj
 0001:0000b5d8       FHELP_NOSHOWERROR          000000018000c5d8     service.obj
 0001:0000b5e0       FHELP_SELFHELP             000000018000c5e0     service.obj
 0001:0000b5e8       FHELP_FARHELP              000000018000c5e8     service.obj
 0001:0000b5f0       FHELP_CUSTOMFILE           000000018000c5f0     service.obj
 0001:0000b5f8       FHELP_CUSTOMPATH           000000018000c5f8     service.obj
 0001:0000b600       FHELP_GUID                 000000018000c600     service.obj
 0001:0000b608       FHELP_USECONTENTS          000000018000c608     service.obj
 0001:0000b610       FHELP_NONE                 000000018000c610     service.obj
 0001:0000b618       KMFLAGS_SILENTCHECK        000000018000c618     service.obj
 0001:0000b620       KMFLAGS_NOSENDKEYSTOPLUGINS 000000018000c620     service.obj
 0001:0000b628       KMFLAGS_ENABLEOUTPUT       000000018000c628     service.obj
 0001:0000b630       KMFLAGS_LANGMASK           000000018000c630     service.obj
 0001:0000b638       KMFLAGS_LUA                000000018000c638     service.obj
 0001:0000b640       KMFLAGS_MOONSCRIPT         000000018000c640     service.obj
 0001:0000b648       KMFLAGS_NONE               000000018000c648     service.obj
 0001:0000b650       AKMFLAGS_NONE              000000018000c650     service.obj
 0001:0000b658       FSETCLR_REDRAW             000000018000c658     service.obj
 0001:0000b660       FSETCLR_NONE               000000018000c660     service.obj
 0001:0000b668       WIF_MODIFIED               000000018000c668     service.obj
 0001:0000b670       WIF_CURRENT                000000018000c670     service.obj
 0001:0000b678       WIF_MODAL                  000000018000c678     service.obj
 0001:0000b680       WIF_NONE                   000000018000c680     service.obj
 0001:0000b688       VOPT_SAVEFILEPOSITION      000000018000c688     service.obj
 0001:0000b690       VOPT_AUTODETECTCODEPAGE    000000018000c690     service.obj
 0001:0000b698       VOPT_SHOWTITLEBAR          000000018000c698     service.obj
 0001:0000b6a0       VOPT_SHOWKEYBAR            000000018000c6a0     service.obj
 0001:0000b6a8       VOPT_SHOWSCROLLBAR         000000018000c6a8     service.obj
 0001:0000b6b0       VOPT_QUICKVIEW             000000018000c6b0     service.obj
 0001:0000b6b8       VOPT_NONE                  000000018000c6b8     service.obj
 0001:0000b6c0       VSMFL_REDRAW               000000018000c6c0     service.obj
 0001:0000b6c8       VSMFL_NONE                 000000018000c6c8     service.obj
 0001:0000b6d0       VSP_NOREDRAW               000000018000c6d0     service.obj
 0001:0000b6d8       VSP_PERCENT                000000018000c6d8     service.obj
 0001:0000b6e0       VSP_RELATIVE               000000018000c6e0     service.obj
 0001:0000b6e8       VSP_NORETNEWPOS            000000018000c6e8     service.obj
 0001:0000b6f0       VSP_NONE                   000000018000c6f0     service.obj
 0001:0000b6f8       VMF_WRAP                   000000018000c6f8     service.obj
 0001:0000b700       VMF_WORDWRAP               000000018000c700     service.obj
 0001:0000b708       VMF_NONE                   000000018000c708     service.obj
 0001:0000b710       ECF_TABMARKFIRST           000000018000c710     service.obj
 0001:0000b718       ECF_TABMARKCURRENT         000000018000c718     service.obj
 0001:0000b720       ECF_AUTODELETE             000000018000c720     service.obj
 0001:0000b728       ECF_NONE                   000000018000c728     service.obj
 0001:0000b730       FIB_ENABLEEMPTY            000000018000c730     service.obj
 0001:0000b738       FIB_PASSWORD               000000018000c738     service.obj
 0001:0000b740       FIB_EXPANDENV              000000018000c740     service.obj
 0001:0000b748       FIB_NOUSELASTHISTORY       000000018000c748     service.obj
 0001:0000b750       FIB_BUTTONS                000000018000c750     service.obj
 0001:0000b758       FIB_NOAMPERSAND            000000018000c758     service.obj
 0001:0000b760       FIB_EDITPATH               000000018000c760     service.obj
 0001:0000b768       FIB_EDITPATHEXEC           000000018000c768     service.obj
 0001:0000b770       FIB_NONE                   000000018000c770     service.obj
 0001:0000b778       FPF_LOADED                 000000018000c778     service.obj
 0001:0000b780       FPF_ANSI                   000000018000c780     service.obj
 0001:0000b788       FPF_NONE                   000000018000c788     service.obj
 0001:0000b790       ?C@?3??far_InputRecordToName@@9@9 000000018000c790     service.obj
 0001:0000b798       ?A@?3??far_InputRecordToName@@9@9 000000018000c798     service.obj
 0001:0000b7a0       ?S@?3??far_InputRecordToName@@9@9 000000018000c7a0     service.obj
 0001:0000b7a8       PN_CMPNAME                 000000018000c7a8     service.obj
 0001:0000b7b0       PN_CMPNAMELIST             000000018000c7b0     service.obj
 0001:0000b7b8       PN_GENERATENAME            000000018000c7b8     service.obj
 0001:0000b7c0       PN_CHECKMASK               000000018000c7c0     service.obj
 0001:0000b7c8       PN_SKIPPATH                000000018000c7c8     service.obj
 0001:0000b7d0       PN_SHOWERRORMESSAGE        000000018000c7d0     service.obj
 0001:0000b7d8       PN_NONE                    000000018000c7d8     service.obj
 0001:0000b7e0       XLAT_SWITCHKEYBLAYOUT      000000018000c7e0     service.obj
 0001:0000b7e8       XLAT_SWITCHKEYBBEEP        000000018000c7e8     service.obj
 0001:0000b7f0       XLAT_USEKEYBLAYOUTNAME     000000018000c7f0     service.obj
 0001:0000b7f8       XLAT_CONVERTALLCMDLINE     000000018000c7f8     service.obj
 0001:0000b800       XLAT_NONE                  000000018000c800     service.obj
 0001:0000b808       FRS_RETUPDIR               000000018000c808     service.obj
 0001:0000b810       FRS_RECUR                  000000018000c810     service.obj
 0001:0000b818       FRS_SCANSYMLINK            000000018000c818     service.obj
 0001:0000b820       FRS_NONE                   000000018000c820     service.obj
 0001:0000b828       MLF_SHOWERRMSG             000000018000c828     service.obj
 0001:0000b830       MLF_DONOTUPDATEPANEL       000000018000c830     service.obj
 0001:0000b838       MLF_HOLDTARGET             000000018000c838     service.obj
 0001:0000b840       MLF_NONE                   000000018000c840     service.obj
 0001:0000b848       FFFS_COMMAS                000000018000c848     service.obj
 0001:0000b850       FFFS_FLOATSIZE             000000018000c850     service.obj
 0001:0000b858       FFFS_SHOWBYTESINDEX        000000018000c858     service.obj
 0001:0000b860       FFFS_ECONOMIC              000000018000c860     service.obj
 0001:0000b868       FFFS_THOUSAND              000000018000c868     service.obj
 0001:0000b870       FFFS_MINSIZEINDEX          000000018000c870     service.obj
 0001:0000b878       FFFS_MINSIZEINDEX_MASK     000000018000c878     service.obj
 0001:0000b880       FFFS_NONE                  000000018000c880     service.obj
 0001:0000b888       PF_PRELOAD                 000000018000c888     service.obj
 0001:0000b890       PF_DISABLEPANELS           000000018000c890     service.obj
 0001:0000b898       PF_EDITOR                  000000018000c898     service.obj
 0001:0000b8a0       PF_VIEWER                  000000018000c8a0     service.obj
 0001:0000b8a8       PF_FULLCMDLINE             000000018000c8a8     service.obj
 0001:0000b8b0       PF_DIALOG                  000000018000c8b0     service.obj
 0001:0000b8b8       PF_NONE                    000000018000c8b8     service.obj
 0001:0000b8c0       IPLFLAGS_SEPARATOR         000000018000c8c0     service.obj
 0001:0000b8c8       IPLFLAGS_NONE              000000018000c8c8     service.obj
 0001:0000b8d0       PMFLAGS_FULLSCREEN         000000018000c8d0     service.obj
 0001:0000b8d8       PMFLAGS_DETAILEDSTATUS     000000018000c8d8     service.obj
 0001:0000b8e0       PMFLAGS_ALIGNEXTENSIONS    000000018000c8e0     service.obj
 0001:0000b8e8       PMFLAGS_CASECONVERSION     000000018000c8e8     service.obj
 0001:0000b8f0       PMFLAGS_NONE               000000018000c8f0     service.obj
 0001:0000b8f8       OPIF_DISABLEFILTER         000000018000c8f8     service.obj
 0001:0000b900       OPIF_DISABLESORTGROUPS     000000018000c900     service.obj
 0001:0000b908       OPIF_DISABLEHIGHLIGHTING   000000018000c908     service.obj
 0001:0000b910       OPIF_ADDDOTS               000000018000c910     service.obj
 0001:0000b918       OPIF_RAWSELECTION          000000018000c918     service.obj
 0001:0000b920       OPIF_REALNAMES             000000018000c920     service.obj
 0001:0000b928       OPIF_SHOWNAMESONLY         000000018000c928     service.obj
 0001:0000b930       OPIF_SHOWRIGHTALIGNNAMES   000000018000c930     service.obj
 0001:0000b938       OPIF_SHOWPRESERVECASE      000000018000c938     service.obj
 0001:0000b940       OPIF_COMPAREFATTIME        000000018000c940     service.obj
 0001:0000b948       OPIF_EXTERNALGET           000000018000c948     service.obj
 0001:0000b950       OPIF_EXTERNALPUT           000000018000c950     service.obj
 0001:0000b958       OPIF_EXTERNALDELETE        000000018000c958     service.obj
 0001:0000b960       OPIF_EXTERNALMKDIR         000000018000c960     service.obj
 0001:0000b968       OPIF_USEATTRHIGHLIGHTING   000000018000c968     service.obj
 0001:0000b970       OPIF_USECRC32              000000018000c970     service.obj
 0001:0000b978       OPIF_USEFREESIZE           000000018000c978     service.obj
 0001:0000b980       OPIF_SHORTCUT              000000018000c980     service.obj
 0001:0000b988       OPIF_NONE                  000000018000c988     service.obj
 0001:0000b990       OPM_SILENT                 000000018000c990     service.obj
 0001:0000b998       OPM_FIND                   000000018000c998     service.obj
 0001:0000b9a0       OPM_VIEW                   000000018000c9a0     service.obj
 0001:0000b9a8       OPM_EDIT                   000000018000c9a8     service.obj
 0001:0000b9b0       OPM_TOPLEVEL               000000018000c9b0     service.obj
 0001:0000b9b8       OPM_DESCR                  000000018000c9b8     service.obj
 0001:0000b9c0       OPM_QUICKVIEW              000000018000c9c0     service.obj
 0001:0000b9c8       OPM_PGDN                   000000018000c9c8     service.obj
 0001:0000b9d0       OPM_COMMANDS               000000018000c9d0     service.obj
 0001:0000b9d8       OPM_NONE                   000000018000c9d8     service.obj
 0001:0000b9e0       FOSF_ACTIVE                000000018000c9e0     service.obj
 0001:0000b9e8       FOSF_NONE                  000000018000c9e8     service.obj
 0001:0000b9f0       PCIF_NONE                  000000018000c9f0     service.obj
 0001:0000b9f8       FarGuid                    000000018000c9f8     service.obj
 0001:0000ba08       ?FarGuid@?1??far_CreateSettings@@9@9 000000018000ca08     service.obj
 0001:0000ba18       PDF_DIALOGEVENTDRAWENABLE  000000018000ca18     service.obj
 0001:0000c7d0       lualibs                    000000018000d7d0     service.obj
 0001:0000c950       PDF_PROCESSINGERROR        000000018000d950     service.obj
 0001:0000e6c0       uniclib                    000000018000f6c0     slnunico.obj
 0001:0000ea90       fnames                     000000018000fa90     uliolib51.obj
 0001:0000eaa0       ?mode@?1??f_seek@@9@9      000000018000faa0     uliolib51.obj
 0001:0000eab0       ?modenames@?1??f_seek@@9@9 000000018000fab0     uliolib51.obj
 0001:0000ead0       ?mode@?1??f_setvbuf@@9@9   000000018000fad0     uliolib51.obj
 0001:0000eae0       ?modenames@?1??f_setvbuf@@9@9 000000018000fae0     uliolib51.obj
 0001:0000eb00       iolib                      000000018000fb00     uliolib51.obj
 0001:0000ebc0       flib                       000000018000fbc0     uliolib51.obj
 0001:0000ee48       sentinel_                  000000018000fe48     uloadlib51.obj
 0001:0000ee50       pk_funcs                   000000018000fe50     uloadlib51.obj
 0001:0000ee80       ll_funcs                   000000018000fe80     uloadlib51.obj
 0001:0000eeb0       loaders                    000000018000feb0     uloadlib51.obj
 0001:0000f780       FCF_FG_4BIT                0000000180010780     util.obj
 0001:0000f788       FCF_BG_4BIT                0000000180010788     util.obj
 0001:0000f790       FCF_4BITMASK               0000000180010790     util.obj
 0001:0000f798       FCF_RAWATTR_MASK           0000000180010798     util.obj
 0001:0000f7a0       FCF_EXTENDEDFLAGS          00000001800107a0     util.obj
 0001:0000f7a8       FCF_FG_BOLD                00000001800107a8     util.obj
 0001:0000f7b0       FCF_FG_ITALIC              00000001800107b0     util.obj
 0001:0000f7b8       FCF_FG_UNDERLINE           00000001800107b8     util.obj
 0001:0000f7c0       FCF_STYLEMASK              00000001800107c0     util.obj
 0001:0000f7c8       FCF_NONE                   00000001800107c8     util.obj
 0001:0000f7d0       CDF_NONE                   00000001800107d0     util.obj
 0001:0000f7d8       FMSG_WARNING               00000001800107d8     util.obj
 0001:0000f7e0       FMSG_ERRORTYPE             00000001800107e0     util.obj
 0001:0000f7e8       FMSG_KEEPBACKGROUND        00000001800107e8     util.obj
 0001:0000f7f0       FMSG_LEFTALIGN             00000001800107f0     util.obj
 0001:0000f7f8       FMSG_ALLINONE              00000001800107f8     util.obj
 0001:0000f800       FMSG_MB_OK                 0000000180010800     util.obj
 0001:0000f808       FMSG_MB_OKCANCEL           0000000180010808     util.obj
 0001:0000f810       FMSG_MB_ABORTRETRYIGNORE   0000000180010810     util.obj
 0001:0000f818       FMSG_MB_YESNO              0000000180010818     util.obj
 0001:0000f820       FMSG_MB_YESNOCANCEL        0000000180010820     util.obj
 0001:0000f828       FMSG_MB_RETRYCANCEL        0000000180010828     util.obj
 0001:0000f830       FMSG_NONE                  0000000180010830     util.obj
 0001:0000f838       DIF_BOXCOLOR               0000000180010838     util.obj
 0001:0000f840       DIF_GROUP                  0000000180010840     util.obj
 0001:0000f848       DIF_LEFTTEXT               0000000180010848     util.obj
 0001:0000f850       DIF_MOVESELECT             0000000180010850     util.obj
 0001:0000f858       DIF_SHOWAMPERSAND          0000000180010858     util.obj
 0001:0000f860       DIF_CENTERGROUP            0000000180010860     util.obj
 0001:0000f868       DIF_NOBRACKETS             0000000180010868     util.obj
 0001:0000f870       DIF_MANUALADDHISTORY       0000000180010870     util.obj
 0001:0000f878       DIF_SEPARATOR              0000000180010878     util.obj
 0001:0000f880       DIF_SEPARATOR2             0000000180010880     util.obj
 0001:0000f888       DIF_EDITOR                 0000000180010888     util.obj
 0001:0000f890       DIF_LISTNOAMPERSAND        0000000180010890     util.obj
 0001:0000f898       DIF_LISTNOBOX              0000000180010898     util.obj
 0001:0000f8a0       DIF_HISTORY                00000001800108a0     util.obj
 0001:0000f8a8       DIF_BTNNOCLOSE             00000001800108a8     util.obj
 0001:0000f8b0       DIF_CENTERTEXT             00000001800108b0     util.obj
 0001:0000f8b8       DIF_SEPARATORUSER          00000001800108b8     util.obj
 0001:0000f8c0       DIF_SETSHIELD              00000001800108c0     util.obj
 0001:0000f8c8       DIF_EDITEXPAND             00000001800108c8     util.obj
 0001:0000f8d0       DIF_DROPDOWNLIST           00000001800108d0     util.obj
 0001:0000f8d8       DIF_USELASTHISTORY         00000001800108d8     util.obj
 0001:0000f8e0       DIF_MASKEDIT               00000001800108e0     util.obj
 0001:0000f8e8       DIF_LISTTRACKMOUSE         00000001800108e8     util.obj
 0001:0000f8f0       DIF_LISTTRACKMOUSEINFOCUS  00000001800108f0     util.obj
 0001:0000f8f8       DIF_SELECTONENTRY          00000001800108f8     util.obj
 0001:0000f900       DIF_3STATE                 0000000180010900     util.obj
 0001:0000f908       DIF_EDITPATH               0000000180010908     util.obj
 0001:0000f910       DIF_LISTWRAPMODE           0000000180010910     util.obj
 0001:0000f918       DIF_NOAUTOCOMPLETE         0000000180010918     util.obj
 0001:0000f920       DIF_LISTAUTOHIGHLIGHT      0000000180010920     util.obj
 0001:0000f928       DIF_LISTNOCLOSE            0000000180010928     util.obj
 0001:0000f930       DIF_EDITPATHEXEC           0000000180010930     util.obj
 0001:0000f938       DIF_HIDDEN                 0000000180010938     util.obj
 0001:0000f940       DIF_READONLY               0000000180010940     util.obj
 0001:0000f948       DIF_NOFOCUS                0000000180010948     util.obj
 0001:0000f950       DIF_DISABLE                0000000180010950     util.obj
 0001:0000f958       DIF_DEFAULTBUTTON          0000000180010958     util.obj
 0001:0000f960       DIF_FOCUS                  0000000180010960     util.obj
 0001:0000f968       DIF_RIGHTTEXT              0000000180010968     util.obj
 0001:0000f970       DIF_WORDWRAP               0000000180010970     util.obj
 0001:0000f978       DIF_NONE                   0000000180010978     util.obj
 0001:0000f980       LIF_SELECTED               0000000180010980     util.obj
 0001:0000f988       LIF_CHECKED                0000000180010988     util.obj
 0001:0000f990       LIF_SEPARATOR              0000000180010990     util.obj
 0001:0000f998       LIF_DISABLE                0000000180010998     util.obj
 0001:0000f9a0       LIF_GRAYED                 00000001800109a0     util.obj
 0001:0000f9a8       LIF_HIDDEN                 00000001800109a8     util.obj
 0001:0000f9b0       LIF_DELETEUSERDATA         00000001800109b0     util.obj
 0001:0000f9b8       LIF_NONE                   00000001800109b8     util.obj
 0001:0000f9c0       LIFIND_EXACTMATCH          00000001800109c0     util.obj
 0001:0000f9c8       LIFIND_NONE                00000001800109c8     util.obj
 0001:0000f9d0       LINFO_SHOWNOBOX            00000001800109d0     util.obj
 0001:0000f9d8       LINFO_AUTOHIGHLIGHT        00000001800109d8     util.obj
 0001:0000f9e0       LINFO_REVERSEHIGHLIGHT     00000001800109e0     util.obj
 0001:0000f9e8       LINFO_WRAPMODE             00000001800109e8     util.obj
 0001:0000f9f0       LINFO_SHOWAMPERSAND        00000001800109f0     util.obj
 0001:0000f9f8       LINFO_NONE                 00000001800109f8     util.obj
 0001:0000fa00       FDLG_WARNING               0000000180010a00     util.obj
 0001:0000fa08       FDLG_SMALLDIALOG           0000000180010a08     util.obj
 0001:0000fa10       FDLG_NODRAWSHADOW          0000000180010a10     util.obj
 0001:0000fa18       FDLG_NODRAWPANEL           0000000180010a18     util.obj
 0001:0000fa20       FDLG_KEEPCONSOLETITLE      0000000180010a20     util.obj
 0001:0000fa28       FDLG_NONMODAL              0000000180010a28     util.obj
 0001:0000fa30       FDLG_NONE                  0000000180010a30     util.obj
 0001:0000fa38       MIF_SELECTED               0000000180010a38     util.obj
 0001:0000fa40       MIF_CHECKED                0000000180010a40     util.obj
 0001:0000fa48       MIF_SEPARATOR              0000000180010a48     util.obj
 0001:0000fa50       MIF_DISABLE                0000000180010a50     util.obj
 0001:0000fa58       MIF_GRAYED                 0000000180010a58     util.obj
 0001:0000fa60       MIF_HIDDEN                 0000000180010a60     util.obj
 0001:0000fa68       MIF_NONE                   0000000180010a68     util.obj
 0001:0000fa70       FMENU_SHOWAMPERSAND        0000000180010a70     util.obj
 0001:0000fa78       FMENU_WRAPMODE             0000000180010a78     util.obj
 0001:0000fa80       FMENU_AUTOHIGHLIGHT        0000000180010a80     util.obj
 0001:0000fa88       FMENU_REVERSEAUTOHIGHLIGHT 0000000180010a88     util.obj
 0001:0000fa90       FMENU_CHANGECONSOLETITLE   0000000180010a90     util.obj
 0001:0000fa98       FMENU_NONE                 0000000180010a98     util.obj
 0001:0000faa0       PPIF_SELECTED              0000000180010aa0     util.obj
 0001:0000faa8       PPIF_PROCESSDESCR          0000000180010aa8     util.obj
 0001:0000fab0       PPIF_NONE                  0000000180010ab0     util.obj
 0001:0000fab8       PFLAGS_SHOWHIDDEN          0000000180010ab8     util.obj
 0001:0000fac0       PFLAGS_HIGHLIGHT           0000000180010ac0     util.obj
 0001:0000fac8       PFLAGS_REVERSESORTORDER    0000000180010ac8     util.obj
 0001:0000fad0       PFLAGS_USESORTGROUPS       0000000180010ad0     util.obj
 0001:0000fad8       PFLAGS_SELECTEDFIRST       0000000180010ad8     util.obj
 0001:0000fae0       PFLAGS_REALNAMES           0000000180010ae0     util.obj
 0001:0000fae8       PFLAGS_PANELLEFT           0000000180010ae8     util.obj
 0001:0000faf0       PFLAGS_DIRECTORIESFIRST    0000000180010af0     util.obj
 0001:0000faf8       PFLAGS_USECRC32            0000000180010af8     util.obj
 0001:0000fb00       PFLAGS_PLUGIN              0000000180010b00     util.obj
 0001:0000fb08       PFLAGS_VISIBLE             0000000180010b08     util.obj
 0001:0000fb10       PFLAGS_FOCUS               0000000180010b10     util.obj
 0001:0000fb18       PFLAGS_ALTERNATIVENAMES    0000000180010b18     util.obj
 0001:0000fb20       PFLAGS_SHORTCUT            0000000180010b20     util.obj
 0001:0000fb28       PFLAGS_NONE                0000000180010b28     util.obj
 0001:0000fb30       VF_NONMODAL                0000000180010b30     util.obj
 0001:0000fb38       VF_DELETEONCLOSE           0000000180010b38     util.obj
 0001:0000fb40       VF_ENABLE_F6               0000000180010b40     util.obj
 0001:0000fb48       VF_DISABLEHISTORY          0000000180010b48     util.obj
 0001:0000fb50       VF_IMMEDIATERETURN         0000000180010b50     util.obj
 0001:0000fb58       VF_DELETEONLYFILEONCLOSE   0000000180010b58     util.obj
 0001:0000fb60       VF_NONE                    0000000180010b60     util.obj
 0001:0000fb68       EF_NONMODAL                0000000180010b68     util.obj
 0001:0000fb70       EF_CREATENEW               0000000180010b70     util.obj
 0001:0000fb78       EF_ENABLE_F6               0000000180010b78     util.obj
 0001:0000fb80       EF_DISABLEHISTORY          0000000180010b80     util.obj
 0001:0000fb88       EF_DELETEONCLOSE           0000000180010b88     util.obj
 0001:0000fb90       EF_IMMEDIATERETURN         0000000180010b90     util.obj
 0001:0000fb98       EF_DELETEONLYFILEONCLOSE   0000000180010b98     util.obj
 0001:0000fba0       EF_LOCKED                  0000000180010ba0     util.obj
 0001:0000fba8       EF_DISABLESAVEPOS          0000000180010ba8     util.obj
 0001:0000fbb0       EF_OPENMODE_MASK           0000000180010bb0     util.obj
 0001:0000fbb8       EF_OPENMODE_QUERY          0000000180010bb8     util.obj
 0001:0000fbc0       EF_OPENMODE_NEWIFOPEN      0000000180010bc0     util.obj
 0001:0000fbc8       EF_OPENMODE_USEEXISTING    0000000180010bc8     util.obj
 0001:0000fbd0       EF_OPENMODE_BREAKIFOPEN    0000000180010bd0     util.obj
 0001:0000fbd8       EF_OPENMODE_RELOADIFOPEN   0000000180010bd8     util.obj
 0001:0000fbe0       EN_NONE                    0000000180010be0     util.obj
 0001:0000fbe8       FHELP_NOSHOWERROR          0000000180010be8     util.obj
 0001:0000fbf0       FHELP_SELFHELP             0000000180010bf0     util.obj
 0001:0000fbf8       FHELP_FARHELP              0000000180010bf8     util.obj
 0001:0000fc00       FHELP_CUSTOMFILE           0000000180010c00     util.obj
 0001:0000fc08       FHELP_CUSTOMPATH           0000000180010c08     util.obj
 0001:0000fc10       FHELP_GUID                 0000000180010c10     util.obj
 0001:0000fc18       FHELP_USECONTENTS          0000000180010c18     util.obj
 0001:0000fc20       FHELP_NONE                 0000000180010c20     util.obj
 0001:0000fc28       KMFLAGS_SILENTCHECK        0000000180010c28     util.obj
 0001:0000fc30       KMFLAGS_NOSENDKEYSTOPLUGINS 0000000180010c30     util.obj
 0001:0000fc38       KMFLAGS_ENABLEOUTPUT       0000000180010c38     util.obj
 0001:0000fc40       KMFLAGS_LANGMASK           0000000180010c40     util.obj
 0001:0000fc48       KMFLAGS_LUA                0000000180010c48     util.obj
 0001:0000fc50       KMFLAGS_MOONSCRIPT         0000000180010c50     util.obj
 0001:0000fc58       KMFLAGS_NONE               0000000180010c58     util.obj
 0001:0000fc60       AKMFLAGS_NONE              0000000180010c60     util.obj
 0001:0000fc68       FSETCLR_REDRAW             0000000180010c68     util.obj
 0001:0000fc70       FSETCLR_NONE               0000000180010c70     util.obj
 0001:0000fc78       WIF_MODIFIED               0000000180010c78     util.obj
 0001:0000fc80       WIF_CURRENT                0000000180010c80     util.obj
 0001:0000fc88       WIF_MODAL                  0000000180010c88     util.obj
 0001:0000fc90       WIF_NONE                   0000000180010c90     util.obj
 0001:0000fc98       VOPT_SAVEFILEPOSITION      0000000180010c98     util.obj
 0001:0000fca0       VOPT_AUTODETECTCODEPAGE    0000000180010ca0     util.obj
 0001:0000fca8       VOPT_SHOWTITLEBAR          0000000180010ca8     util.obj
 0001:0000fcb0       VOPT_SHOWKEYBAR            0000000180010cb0     util.obj
 0001:0000fcb8       VOPT_SHOWSCROLLBAR         0000000180010cb8     util.obj
 0001:0000fcc0       VOPT_QUICKVIEW             0000000180010cc0     util.obj
 0001:0000fcc8       VOPT_NONE                  0000000180010cc8     util.obj
 0001:0000fcd0       VSMFL_REDRAW               0000000180010cd0     util.obj
 0001:0000fcd8       VSMFL_NONE                 0000000180010cd8     util.obj
 0001:0000fce0       VSP_NOREDRAW               0000000180010ce0     util.obj
 0001:0000fce8       VSP_PERCENT                0000000180010ce8     util.obj
 0001:0000fcf0       VSP_RELATIVE               0000000180010cf0     util.obj
 0001:0000fcf8       VSP_NORETNEWPOS            0000000180010cf8     util.obj
 0001:0000fd00       VSP_NONE                   0000000180010d00     util.obj
 0001:0000fd08       VMF_WRAP                   0000000180010d08     util.obj
 0001:0000fd10       VMF_WORDWRAP               0000000180010d10     util.obj
 0001:0000fd18       VMF_NONE                   0000000180010d18     util.obj
 0001:0000fd20       ECF_TABMARKFIRST           0000000180010d20     util.obj
 0001:0000fd28       ECF_TABMARKCURRENT         0000000180010d28     util.obj
 0001:0000fd30       ECF_AUTODELETE             0000000180010d30     util.obj
 0001:0000fd38       ECF_NONE                   0000000180010d38     util.obj
 0001:0000fd40       FIB_ENABLEEMPTY            0000000180010d40     util.obj
 0001:0000fd48       FIB_PASSWORD               0000000180010d48     util.obj
 0001:0000fd50       FIB_EXPANDENV              0000000180010d50     util.obj
 0001:0000fd58       FIB_NOUSELASTHISTORY       0000000180010d58     util.obj
 0001:0000fd60       FIB_BUTTONS                0000000180010d60     util.obj
 0001:0000fd68       FIB_NOAMPERSAND            0000000180010d68     util.obj
 0001:0000fd70       FIB_EDITPATH               0000000180010d70     util.obj
 0001:0000fd78       FIB_EDITPATHEXEC           0000000180010d78     util.obj
 0001:0000fd80       FIB_NONE                   0000000180010d80     util.obj
 0001:0000fd88       FPF_LOADED                 0000000180010d88     util.obj
 0001:0000fd90       FPF_ANSI                   0000000180010d90     util.obj
 0001:0000fd98       FPF_NONE                   0000000180010d98     util.obj
 0001:0000fda0       PN_CMPNAME                 0000000180010da0     util.obj
 0001:0000fda8       PN_CMPNAMELIST             0000000180010da8     util.obj
 0001:0000fdb0       PN_GENERATENAME            0000000180010db0     util.obj
 0001:0000fdb8       PN_CHECKMASK               0000000180010db8     util.obj
 0001:0000fdc0       PN_SKIPPATH                0000000180010dc0     util.obj
 0001:0000fdc8       PN_SHOWERRORMESSAGE        0000000180010dc8     util.obj
 0001:0000fdd0       PN_NONE                    0000000180010dd0     util.obj
 0001:0000fdd8       XLAT_SWITCHKEYBLAYOUT      0000000180010dd8     util.obj
 0001:0000fde0       XLAT_SWITCHKEYBBEEP        0000000180010de0     util.obj
 0001:0000fde8       XLAT_USEKEYBLAYOUTNAME     0000000180010de8     util.obj
 0001:0000fdf0       XLAT_CONVERTALLCMDLINE     0000000180010df0     util.obj
 0001:0000fdf8       XLAT_NONE                  0000000180010df8     util.obj
 0001:0000fe00       FRS_RETUPDIR               0000000180010e00     util.obj
 0001:0000fe08       FRS_RECUR                  0000000180010e08     util.obj
 0001:0000fe10       FRS_SCANSYMLINK            0000000180010e10     util.obj
 0001:0000fe18       FRS_NONE                   0000000180010e18     util.obj
 0001:0000fe20       MLF_SHOWERRMSG             0000000180010e20     util.obj
 0001:0000fe28       MLF_DONOTUPDATEPANEL       0000000180010e28     util.obj
 0001:0000fe30       MLF_HOLDTARGET             0000000180010e30     util.obj
 0001:0000fe38       MLF_NONE                   0000000180010e38     util.obj
 0001:0000fe40       FFFS_COMMAS                0000000180010e40     util.obj
 0001:0000fe48       FFFS_FLOATSIZE             0000000180010e48     util.obj
 0001:0000fe50       FFFS_SHOWBYTESINDEX        0000000180010e50     util.obj
 0001:0000fe58       FFFS_ECONOMIC              0000000180010e58     util.obj
 0001:0000fe60       FFFS_THOUSAND              0000000180010e60     util.obj
 0001:0000fe68       FFFS_MINSIZEINDEX          0000000180010e68     util.obj
 0001:0000fe70       FFFS_MINSIZEINDEX_MASK     0000000180010e70     util.obj
 0001:0000fe78       FFFS_NONE                  0000000180010e78     util.obj
 0001:0000fe80       PF_PRELOAD                 0000000180010e80     util.obj
 0001:0000fe88       PF_DISABLEPANELS           0000000180010e88     util.obj
 0001:0000fe90       PF_EDITOR                  0000000180010e90     util.obj
 0001:0000fe98       PF_VIEWER                  0000000180010e98     util.obj
 0001:0000fea0       PF_FULLCMDLINE             0000000180010ea0     util.obj
 0001:0000fea8       PF_DIALOG                  0000000180010ea8     util.obj
 0001:0000feb0       PF_NONE                    0000000180010eb0     util.obj
 0001:0000feb8       IPLFLAGS_SEPARATOR         0000000180010eb8     util.obj
 0001:0000fec0       IPLFLAGS_NONE              0000000180010ec0     util.obj
 0001:0000fec8       PMFLAGS_FULLSCREEN         0000000180010ec8     util.obj
 0001:0000fed0       PMFLAGS_DETAILEDSTATUS     0000000180010ed0     util.obj
 0001:0000fed8       PMFLAGS_ALIGNEXTENSIONS    0000000180010ed8     util.obj
 0001:0000fee0       PMFLAGS_CASECONVERSION     0000000180010ee0     util.obj
 0001:0000fee8       PMFLAGS_NONE               0000000180010ee8     util.obj
 0001:0000fef0       OPIF_DISABLEFILTER         0000000180010ef0     util.obj
 0001:0000fef8       OPIF_DISABLESORTGROUPS     0000000180010ef8     util.obj
 0001:0000ff00       OPIF_DISABLEHIGHLIGHTING   0000000180010f00     util.obj
 0001:0000ff08       OPIF_ADDDOTS               0000000180010f08     util.obj
 0001:0000ff10       OPIF_RAWSELECTION          0000000180010f10     util.obj
 0001:0000ff18       OPIF_REALNAMES             0000000180010f18     util.obj
 0001:0000ff20       OPIF_SHOWNAMESONLY         0000000180010f20     util.obj
 0001:0000ff28       OPIF_SHOWRIGHTALIGNNAMES   0000000180010f28     util.obj
 0001:0000ff30       OPIF_SHOWPRESERVECASE      0000000180010f30     util.obj
 0001:0000ff38       OPIF_COMPAREFATTIME        0000000180010f38     util.obj
 0001:0000ff40       OPIF_EXTERNALGET           0000000180010f40     util.obj
 0001:0000ff48       OPIF_EXTERNALPUT           0000000180010f48     util.obj
 0001:0000ff50       OPIF_EXTERNALDELETE        0000000180010f50     util.obj
 0001:0000ff58       OPIF_EXTERNALMKDIR         0000000180010f58     util.obj
 0001:0000ff60       OPIF_USEATTRHIGHLIGHTING   0000000180010f60     util.obj
 0001:0000ff68       OPIF_USECRC32              0000000180010f68     util.obj
 0001:0000ff70       OPIF_USEFREESIZE           0000000180010f70     util.obj
 0001:0000ff78       OPIF_SHORTCUT              0000000180010f78     util.obj
 0001:0000ff80       OPIF_NONE                  0000000180010f80     util.obj
 0001:0000ff88       OPM_SILENT                 0000000180010f88     util.obj
 0001:0000ff90       OPM_FIND                   0000000180010f90     util.obj
 0001:0000ff98       OPM_VIEW                   0000000180010f98     util.obj
 0001:0000ffa0       OPM_EDIT                   0000000180010fa0     util.obj
 0001:0000ffa8       OPM_TOPLEVEL               0000000180010fa8     util.obj
 0001:0000ffb0       OPM_DESCR                  0000000180010fb0     util.obj
 0001:0000ffb8       OPM_QUICKVIEW              0000000180010fb8     util.obj
 0001:0000ffc0       OPM_PGDN                   0000000180010fc0     util.obj
 0001:0000ffc8       OPM_COMMANDS               0000000180010fc8     util.obj
 0001:0000ffd0       OPM_NONE                   0000000180010fd0     util.obj
 0001:0000ffd8       FOSF_ACTIVE                0000000180010fd8     util.obj
 0001:0000ffe0       FOSF_NONE                  0000000180010fe0     util.obj
 0001:0000ffe8       PCIF_NONE                  0000000180010fe8     util.obj
 0001:0000fff0       FarGuid                    0000000180010ff0     util.obj
 0001:00010090       FCF_FG_4BIT                0000000180011090     win.obj
 0001:00010098       FCF_BG_4BIT                0000000180011098     win.obj
 0001:000100a0       FCF_4BITMASK               00000001800110a0     win.obj
 0001:000100a8       FCF_RAWATTR_MASK           00000001800110a8     win.obj
 0001:000100b0       FCF_EXTENDEDFLAGS          00000001800110b0     win.obj
 0001:000100b8       FCF_FG_BOLD                00000001800110b8     win.obj
 0001:000100c0       FCF_FG_ITALIC              00000001800110c0     win.obj
 0001:000100c8       FCF_FG_UNDERLINE           00000001800110c8     win.obj
 0001:000100d0       FCF_STYLEMASK              00000001800110d0     win.obj
 0001:000100d8       FCF_NONE                   00000001800110d8     win.obj
 0001:000100e0       CDF_NONE                   00000001800110e0     win.obj
 0001:000100e8       FMSG_WARNING               00000001800110e8     win.obj
 0001:000100f0       FMSG_ERRORTYPE             00000001800110f0     win.obj
 0001:000100f8       FMSG_KEEPBACKGROUND        00000001800110f8     win.obj
 0001:00010100       FMSG_LEFTALIGN             0000000180011100     win.obj
 0001:00010108       FMSG_ALLINONE              0000000180011108     win.obj
 0001:00010110       FMSG_MB_OK                 0000000180011110     win.obj
 0001:00010118       FMSG_MB_OKCANCEL           0000000180011118     win.obj
 0001:00010120       FMSG_MB_ABORTRETRYIGNORE   0000000180011120     win.obj
 0001:00010128       FMSG_MB_YESNO              0000000180011128     win.obj
 0001:00010130       FMSG_MB_YESNOCANCEL        0000000180011130     win.obj
 0001:00010138       FMSG_MB_RETRYCANCEL        0000000180011138     win.obj
 0001:00010140       FMSG_NONE                  0000000180011140     win.obj
 0001:00010148       DIF_BOXCOLOR               0000000180011148     win.obj
 0001:00010150       DIF_GROUP                  0000000180011150     win.obj
 0001:00010158       DIF_LEFTTEXT               0000000180011158     win.obj
 0001:00010160       DIF_MOVESELECT             0000000180011160     win.obj
 0001:00010168       DIF_SHOWAMPERSAND          0000000180011168     win.obj
 0001:00010170       DIF_CENTERGROUP            0000000180011170     win.obj
 0001:00010178       DIF_NOBRACKETS             0000000180011178     win.obj
 0001:00010180       DIF_MANUALADDHISTORY       0000000180011180     win.obj
 0001:00010188       DIF_SEPARATOR              0000000180011188     win.obj
 0001:00010190       DIF_SEPARATOR2             0000000180011190     win.obj
 0001:00010198       DIF_EDITOR                 0000000180011198     win.obj
 0001:000101a0       DIF_LISTNOAMPERSAND        00000001800111a0     win.obj
 0001:000101a8       DIF_LISTNOBOX              00000001800111a8     win.obj
 0001:000101b0       DIF_HISTORY                00000001800111b0     win.obj
 0001:000101b8       DIF_BTNNOCLOSE             00000001800111b8     win.obj
 0001:000101c0       DIF_CENTERTEXT             00000001800111c0     win.obj
 0001:000101c8       DIF_SEPARATORUSER          00000001800111c8     win.obj
 0001:000101d0       DIF_SETSHIELD              00000001800111d0     win.obj
 0001:000101d8       DIF_EDITEXPAND             00000001800111d8     win.obj
 0001:000101e0       DIF_DROPDOWNLIST           00000001800111e0     win.obj
 0001:000101e8       DIF_USELASTHISTORY         00000001800111e8     win.obj
 0001:000101f0       DIF_MASKEDIT               00000001800111f0     win.obj
 0001:000101f8       DIF_LISTTRACKMOUSE         00000001800111f8     win.obj
 0001:00010200       DIF_LISTTRACKMOUSEINFOCUS  0000000180011200     win.obj
 0001:00010208       DIF_SELECTONENTRY          0000000180011208     win.obj
 0001:00010210       DIF_3STATE                 0000000180011210     win.obj
 0001:00010218       DIF_EDITPATH               0000000180011218     win.obj
 0001:00010220       DIF_LISTWRAPMODE           0000000180011220     win.obj
 0001:00010228       DIF_NOAUTOCOMPLETE         0000000180011228     win.obj
 0001:00010230       DIF_LISTAUTOHIGHLIGHT      0000000180011230     win.obj
 0001:00010238       DIF_LISTNOCLOSE            0000000180011238     win.obj
 0001:00010240       DIF_EDITPATHEXEC           0000000180011240     win.obj
 0001:00010248       DIF_HIDDEN                 0000000180011248     win.obj
 0001:00010250       DIF_READONLY               0000000180011250     win.obj
 0001:00010258       DIF_NOFOCUS                0000000180011258     win.obj
 0001:00010260       DIF_DISABLE                0000000180011260     win.obj
 0001:00010268       DIF_DEFAULTBUTTON          0000000180011268     win.obj
 0001:00010270       DIF_FOCUS                  0000000180011270     win.obj
 0001:00010278       DIF_RIGHTTEXT              0000000180011278     win.obj
 0001:00010280       DIF_WORDWRAP               0000000180011280     win.obj
 0001:00010288       DIF_NONE                   0000000180011288     win.obj
 0001:00010290       LIF_SELECTED               0000000180011290     win.obj
 0001:00010298       LIF_CHECKED                0000000180011298     win.obj
 0001:000102a0       LIF_SEPARATOR              00000001800112a0     win.obj
 0001:000102a8       LIF_DISABLE                00000001800112a8     win.obj
 0001:000102b0       LIF_GRAYED                 00000001800112b0     win.obj
 0001:000102b8       LIF_HIDDEN                 00000001800112b8     win.obj
 0001:000102c0       LIF_DELETEUSERDATA         00000001800112c0     win.obj
 0001:000102c8       LIF_NONE                   00000001800112c8     win.obj
 0001:000102d0       LIFIND_EXACTMATCH          00000001800112d0     win.obj
 0001:000102d8       LIFIND_NONE                00000001800112d8     win.obj
 0001:000102e0       LINFO_SHOWNOBOX            00000001800112e0     win.obj
 0001:000102e8       LINFO_AUTOHIGHLIGHT        00000001800112e8     win.obj
 0001:000102f0       LINFO_REVERSEHIGHLIGHT     00000001800112f0     win.obj
 0001:000102f8       LINFO_WRAPMODE             00000001800112f8     win.obj
 0001:00010300       LINFO_SHOWAMPERSAND        0000000180011300     win.obj
 0001:00010308       LINFO_NONE                 0000000180011308     win.obj
 0001:00010310       FDLG_WARNING               0000000180011310     win.obj
 0001:00010318       FDLG_SMALLDIALOG           0000000180011318     win.obj
 0001:00010320       FDLG_NODRAWSHADOW          0000000180011320     win.obj
 0001:00010328       FDLG_NODRAWPANEL           0000000180011328     win.obj
 0001:00010330       FDLG_KEEPCONSOLETITLE      0000000180011330     win.obj
 0001:00010338       FDLG_NONMODAL              0000000180011338     win.obj
 0001:00010340       FDLG_NONE                  0000000180011340     win.obj
 0001:00010348       MIF_SELECTED               0000000180011348     win.obj
 0001:00010350       MIF_CHECKED                0000000180011350     win.obj
 0001:00010358       MIF_SEPARATOR              0000000180011358     win.obj
 0001:00010360       MIF_DISABLE                0000000180011360     win.obj
 0001:00010368       MIF_GRAYED                 0000000180011368     win.obj
 0001:00010370       MIF_HIDDEN                 0000000180011370     win.obj
 0001:00010378       MIF_NONE                   0000000180011378     win.obj
 0001:00010380       FMENU_SHOWAMPERSAND        0000000180011380     win.obj
 0001:00010388       FMENU_WRAPMODE             0000000180011388     win.obj
 0001:00010390       FMENU_AUTOHIGHLIGHT        0000000180011390     win.obj
 0001:00010398       FMENU_REVERSEAUTOHIGHLIGHT 0000000180011398     win.obj
 0001:000103a0       FMENU_CHANGECONSOLETITLE   00000001800113a0     win.obj
 0001:000103a8       FMENU_NONE                 00000001800113a8     win.obj
 0001:000103b0       PPIF_SELECTED              00000001800113b0     win.obj
 0001:000103b8       PPIF_PROCESSDESCR          00000001800113b8     win.obj
 0001:000103c0       PPIF_NONE                  00000001800113c0     win.obj
 0001:000103c8       PFLAGS_SHOWHIDDEN          00000001800113c8     win.obj
 0001:000103d0       PFLAGS_HIGHLIGHT           00000001800113d0     win.obj
 0001:000103d8       PFLAGS_REVERSESORTORDER    00000001800113d8     win.obj
 0001:000103e0       PFLAGS_USESORTGROUPS       00000001800113e0     win.obj
 0001:000103e8       PFLAGS_SELECTEDFIRST       00000001800113e8     win.obj
 0001:000103f0       PFLAGS_REALNAMES           00000001800113f0     win.obj
 0001:000103f8       PFLAGS_PANELLEFT           00000001800113f8     win.obj
 0001:00010400       PFLAGS_DIRECTORIESFIRST    0000000180011400     win.obj
 0001:00010408       PFLAGS_USECRC32            0000000180011408     win.obj
 0001:00010410       PFLAGS_PLUGIN              0000000180011410     win.obj
 0001:00010418       PFLAGS_VISIBLE             0000000180011418     win.obj
 0001:00010420       PFLAGS_FOCUS               0000000180011420     win.obj
 0001:00010428       PFLAGS_ALTERNATIVENAMES    0000000180011428     win.obj
 0001:00010430       PFLAGS_SHORTCUT            0000000180011430     win.obj
 0001:00010438       PFLAGS_NONE                0000000180011438     win.obj
 0001:00010440       VF_NONMODAL                0000000180011440     win.obj
 0001:00010448       VF_DELETEONCLOSE           0000000180011448     win.obj
 0001:00010450       VF_ENABLE_F6               0000000180011450     win.obj
 0001:00010458       VF_DISABLEHISTORY          0000000180011458     win.obj
 0001:00010460       VF_IMMEDIATERETURN         0000000180011460     win.obj
 0001:00010468       VF_DELETEONLYFILEONCLOSE   0000000180011468     win.obj
 0001:00010470       VF_NONE                    0000000180011470     win.obj
 0001:00010478       EF_NONMODAL                0000000180011478     win.obj
 0001:00010480       EF_CREATENEW               0000000180011480     win.obj
 0001:00010488       EF_ENABLE_F6               0000000180011488     win.obj
 0001:00010490       EF_DISABLEHISTORY          0000000180011490     win.obj
 0001:00010498       EF_DELETEONCLOSE           0000000180011498     win.obj
 0001:000104a0       EF_IMMEDIATERETURN         00000001800114a0     win.obj
 0001:000104a8       EF_DELETEONLYFILEONCLOSE   00000001800114a8     win.obj
 0001:000104b0       EF_LOCKED                  00000001800114b0     win.obj
 0001:000104b8       EF_DISABLESAVEPOS          00000001800114b8     win.obj
 0001:000104c0       EF_OPENMODE_MASK           00000001800114c0     win.obj
 0001:000104c8       EF_OPENMODE_QUERY          00000001800114c8     win.obj
 0001:000104d0       EF_OPENMODE_NEWIFOPEN      00000001800114d0     win.obj
 0001:000104d8       EF_OPENMODE_USEEXISTING    00000001800114d8     win.obj
 0001:000104e0       EF_OPENMODE_BREAKIFOPEN    00000001800114e0     win.obj
 0001:000104e8       EF_OPENMODE_RELOADIFOPEN   00000001800114e8     win.obj
 0001:000104f0       EN_NONE                    00000001800114f0     win.obj
 0001:000104f8       FHELP_NOSHOWERROR          00000001800114f8     win.obj
 0001:00010500       FHELP_SELFHELP             0000000180011500     win.obj
 0001:00010508       FHELP_FARHELP              0000000180011508     win.obj
 0001:00010510       FHELP_CUSTOMFILE           0000000180011510     win.obj
 0001:00010518       FHELP_CUSTOMPATH           0000000180011518     win.obj
 0001:00010520       FHELP_GUID                 0000000180011520     win.obj
 0001:00010528       FHELP_USECONTENTS          0000000180011528     win.obj
 0001:00010530       FHELP_NONE                 0000000180011530     win.obj
 0001:00010538       KMFLAGS_SILENTCHECK        0000000180011538     win.obj
 0001:00010540       KMFLAGS_NOSENDKEYSTOPLUGINS 0000000180011540     win.obj
 0001:00010548       KMFLAGS_ENABLEOUTPUT       0000000180011548     win.obj
 0001:00010550       KMFLAGS_LANGMASK           0000000180011550     win.obj
 0001:00010558       KMFLAGS_LUA                0000000180011558     win.obj
 0001:00010560       KMFLAGS_MOONSCRIPT         0000000180011560     win.obj
 0001:00010568       KMFLAGS_NONE               0000000180011568     win.obj
 0001:00010570       AKMFLAGS_NONE              0000000180011570     win.obj
 0001:00010578       FSETCLR_REDRAW             0000000180011578     win.obj
 0001:00010580       FSETCLR_NONE               0000000180011580     win.obj
 0001:00010588       WIF_MODIFIED               0000000180011588     win.obj
 0001:00010590       WIF_CURRENT                0000000180011590     win.obj
 0001:00010598       WIF_MODAL                  0000000180011598     win.obj
 0001:000105a0       WIF_NONE                   00000001800115a0     win.obj
 0001:000105a8       VOPT_SAVEFILEPOSITION      00000001800115a8     win.obj
 0001:000105b0       VOPT_AUTODETECTCODEPAGE    00000001800115b0     win.obj
 0001:000105b8       VOPT_SHOWTITLEBAR          00000001800115b8     win.obj
 0001:000105c0       VOPT_SHOWKEYBAR            00000001800115c0     win.obj
 0001:000105c8       VOPT_SHOWSCROLLBAR         00000001800115c8     win.obj
 0001:000105d0       VOPT_QUICKVIEW             00000001800115d0     win.obj
 0001:000105d8       VOPT_NONE                  00000001800115d8     win.obj
 0001:000105e0       VSMFL_REDRAW               00000001800115e0     win.obj
 0001:000105e8       VSMFL_NONE                 00000001800115e8     win.obj
 0001:000105f0       VSP_NOREDRAW               00000001800115f0     win.obj
 0001:000105f8       VSP_PERCENT                00000001800115f8     win.obj
 0001:00010600       VSP_RELATIVE               0000000180011600     win.obj
 0001:00010608       VSP_NORETNEWPOS            0000000180011608     win.obj
 0001:00010610       VSP_NONE                   0000000180011610     win.obj
 0001:00010618       VMF_WRAP                   0000000180011618     win.obj
 0001:00010620       VMF_WORDWRAP               0000000180011620     win.obj
 0001:00010628       VMF_NONE                   0000000180011628     win.obj
 0001:00010630       ECF_TABMARKFIRST           0000000180011630     win.obj
 0001:00010638       ECF_TABMARKCURRENT         0000000180011638     win.obj
 0001:00010640       ECF_AUTODELETE             0000000180011640     win.obj
 0001:00010648       ECF_NONE                   0000000180011648     win.obj
 0001:00010650       FIB_ENABLEEMPTY            0000000180011650     win.obj
 0001:00010658       FIB_PASSWORD               0000000180011658     win.obj
 0001:00010660       FIB_EXPANDENV              0000000180011660     win.obj
 0001:00010668       FIB_NOUSELASTHISTORY       0000000180011668     win.obj
 0001:00010670       FIB_BUTTONS                0000000180011670     win.obj
 0001:00010678       FIB_NOAMPERSAND            0000000180011678     win.obj
 0001:00010680       FIB_EDITPATH               0000000180011680     win.obj
 0001:00010688       FIB_EDITPATHEXEC           0000000180011688     win.obj
 0001:00010690       FIB_NONE                   0000000180011690     win.obj
 0001:00010698       FPF_LOADED                 0000000180011698     win.obj
 0001:000106a0       FPF_ANSI                   00000001800116a0     win.obj
 0001:000106a8       FPF_NONE                   00000001800116a8     win.obj
 0001:000106b0       PN_CMPNAME                 00000001800116b0     win.obj
 0001:000106b8       PN_CMPNAMELIST             00000001800116b8     win.obj
 0001:000106c0       PN_GENERATENAME            00000001800116c0     win.obj
 0001:000106c8       PN_CHECKMASK               00000001800116c8     win.obj
 0001:000106d0       PN_SKIPPATH                00000001800116d0     win.obj
 0001:000106d8       PN_SHOWERRORMESSAGE        00000001800116d8     win.obj
 0001:000106e0       PN_NONE                    00000001800116e0     win.obj
 0001:000106e8       XLAT_SWITCHKEYBLAYOUT      00000001800116e8     win.obj
 0001:000106f0       XLAT_SWITCHKEYBBEEP        00000001800116f0     win.obj
 0001:000106f8       XLAT_USEKEYBLAYOUTNAME     00000001800116f8     win.obj
 0001:00010700       XLAT_CONVERTALLCMDLINE     0000000180011700     win.obj
 0001:00010708       XLAT_NONE                  0000000180011708     win.obj
 0001:00010710       FRS_RETUPDIR               0000000180011710     win.obj
 0001:00010718       FRS_RECUR                  0000000180011718     win.obj
 0001:00010720       FRS_SCANSYMLINK            0000000180011720     win.obj
 0001:00010728       FRS_NONE                   0000000180011728     win.obj
 0001:00010730       MLF_SHOWERRMSG             0000000180011730     win.obj
 0001:00010738       MLF_DONOTUPDATEPANEL       0000000180011738     win.obj
 0001:00010740       MLF_HOLDTARGET             0000000180011740     win.obj
 0001:00010748       MLF_NONE                   0000000180011748     win.obj
 0001:00010750       FFFS_COMMAS                0000000180011750     win.obj
 0001:00010758       FFFS_FLOATSIZE             0000000180011758     win.obj
 0001:00010760       FFFS_SHOWBYTESINDEX        0000000180011760     win.obj
 0001:00010768       FFFS_ECONOMIC              0000000180011768     win.obj
 0001:00010770       FFFS_THOUSAND              0000000180011770     win.obj
 0001:00010778       FFFS_MINSIZEINDEX          0000000180011778     win.obj
 0001:00010780       FFFS_MINSIZEINDEX_MASK     0000000180011780     win.obj
 0001:00010788       FFFS_NONE                  0000000180011788     win.obj
 0001:00010790       PF_PRELOAD                 0000000180011790     win.obj
 0001:00010798       PF_DISABLEPANELS           0000000180011798     win.obj
 0001:000107a0       PF_EDITOR                  00000001800117a0     win.obj
 0001:000107a8       PF_VIEWER                  00000001800117a8     win.obj
 0001:000107b0       PF_FULLCMDLINE             00000001800117b0     win.obj
 0001:000107b8       PF_DIALOG                  00000001800117b8     win.obj
 0001:000107c0       PF_NONE                    00000001800117c0     win.obj
 0001:000107c8       IPLFLAGS_SEPARATOR         00000001800117c8     win.obj
 0001:000107d0       IPLFLAGS_NONE              00000001800117d0     win.obj
 0001:000107d8       PMFLAGS_FULLSCREEN         00000001800117d8     win.obj
 0001:000107e0       PMFLAGS_DETAILEDSTATUS     00000001800117e0     win.obj
 0001:000107e8       PMFLAGS_ALIGNEXTENSIONS    00000001800117e8     win.obj
 0001:000107f0       PMFLAGS_CASECONVERSION     00000001800117f0     win.obj
 0001:000107f8       PMFLAGS_NONE               00000001800117f8     win.obj
 0001:00010800       OPIF_DISABLEFILTER         0000000180011800     win.obj
 0001:00010808       OPIF_DISABLESORTGROUPS     0000000180011808     win.obj
 0001:00010810       OPIF_DISABLEHIGHLIGHTING   0000000180011810     win.obj
 0001:00010818       OPIF_ADDDOTS               0000000180011818     win.obj
 0001:00010820       OPIF_RAWSELECTION          0000000180011820     win.obj
 0001:00010828       OPIF_REALNAMES             0000000180011828     win.obj
 0001:00010830       OPIF_SHOWNAMESONLY         0000000180011830     win.obj
 0001:00010838       OPIF_SHOWRIGHTALIGNNAMES   0000000180011838     win.obj
 0001:00010840       OPIF_SHOWPRESERVECASE      0000000180011840     win.obj
 0001:00010848       OPIF_COMPAREFATTIME        0000000180011848     win.obj
 0001:00010850       OPIF_EXTERNALGET           0000000180011850     win.obj
 0001:00010858       OPIF_EXTERNALPUT           0000000180011858     win.obj
 0001:00010860       OPIF_EXTERNALDELETE        0000000180011860     win.obj
 0001:00010868       OPIF_EXTERNALMKDIR         0000000180011868     win.obj
 0001:00010870       OPIF_USEATTRHIGHLIGHTING   0000000180011870     win.obj
 0001:00010878       OPIF_USECRC32              0000000180011878     win.obj
 0001:00010880       OPIF_USEFREESIZE           0000000180011880     win.obj
 0001:00010888       OPIF_SHORTCUT              0000000180011888     win.obj
 0001:00010890       OPIF_NONE                  0000000180011890     win.obj
 0001:00010898       OPM_SILENT                 0000000180011898     win.obj
 0001:000108a0       OPM_FIND                   00000001800118a0     win.obj
 0001:000108a8       OPM_VIEW                   00000001800118a8     win.obj
 0001:000108b0       OPM_EDIT                   00000001800118b0     win.obj
 0001:000108b8       OPM_TOPLEVEL               00000001800118b8     win.obj
 0001:000108c0       OPM_DESCR                  00000001800118c0     win.obj
 0001:000108c8       OPM_QUICKVIEW              00000001800118c8     win.obj
 0001:000108d0       OPM_PGDN                   00000001800118d0     win.obj
 0001:000108d8       OPM_COMMANDS               00000001800118d8     win.obj
 0001:000108e0       OPM_NONE                   00000001800118e0     win.obj
 0001:000108e8       FOSF_ACTIVE                00000001800118e8     win.obj
 0001:000108f0       FOSF_NONE                  00000001800118f0     win.obj
 0001:000108f8       PCIF_NONE                  00000001800118f8     win.obj
 0001:00010900       FarGuid                    0000000180011900     win.obj
 0001:00010ed0       ?tokenTable@@3QBQEBDB      0000000180011ed0     libvcruntime:undname.obj
 0001:00010f48       ?rttiTable@@3QBQEBDB       0000000180011f48     libvcruntime:undname.obj
 0001:00010f70       ?nameTable@@3QBQEBDB       0000000180011f70     libvcruntime:undname.obj
 0001:00011878       ?module_names@?A0x89697e75@@3QBQEB_WB 0000000180012878     libvcruntime:winapi_downlevel.obj
 0001:00011948       ?candidate_modules@?1??try_get_FlsAlloc@@YAP6AKP6AXPEAX@Z@ZXZ@4QBW4module_id@?A0x89697e75@@B 0000000180012948     libvcruntime:winapi_downlevel.obj
 0001:00011960       ?candidate_modules@?1??try_get_FlsFree@@YAP6AHK@ZXZ@4QBW4module_id@?A0x89697e75@@B 0000000180012960     libvcruntime:winapi_downlevel.obj
 0001:00011970       ?candidate_modules@?1??try_get_FlsGetValue@@YAP6APEAXK@ZXZ@4QBW4module_id@?A0x89697e75@@B 0000000180012970     libvcruntime:winapi_downlevel.obj
 0001:00011988       ?candidate_modules@?1??try_get_FlsSetValue@@YAP6AHKPEAX@ZXZ@4QBW4module_id@?A0x89697e75@@B 0000000180012988     libvcruntime:winapi_downlevel.obj
 0001:000119a0       ?candidate_modules@?1??try_get_InitializeCriticalSectionEx@@YAP6AHPEAU_RTL_CRITICAL_SECTION@@KK@ZXZ@4QBW4module_id@?A0x89697e75@@B 00000001800129a0     libvcruntime:winapi_downlevel.obj
 0001:00011a50       ?errtable@@3QBUerrentry@?A0x31fdb9ec@@B 0000000180012a50     libucrt:errno.obj
 0001:00011bf0       ?default_cmd_exe@?1???$common_popen_nolock@_W@@YAPEAU_iobuf@@QEB_W0HAEAY01H@Z@4QB_WB 0000000180012bf0     libucrt:popen.obj
 0001:00011c00       ?slash_c@?1???$common_popen_nolock@_W@@YAPEAU_iobuf@@QEB_W0HAEAY01H@Z@4QB_WB 0000000180012c00     libucrt:popen.obj
 0001:00011c10       ?comspec_name@?1???$get_comspec@_W@@YAPEB_WXZ@4QB_WB 0000000180012c10     libucrt:popen.obj
 0001:00011c20       ?backslash@?L@???$get_executable_path@_W@@YAPEB_WQEB_W@Z@4QB_WB 0000000180012c20     libucrt:popen.obj
 0001:00011c28       ?path_name@?1???$get_path@_W@@YAPEB_WXZ@4QB_WB 0000000180012c28     libucrt:popen.obj
 0001:00012830       ?comspec_name@?1???$common_system@_W@@YAHQEB_W@Z@4QB_WB 0000000180013830     libucrt:system.obj
 0001:00012840       ?cmd_exe@?1???$common_system@_W@@YAHQEB_W@Z@4QB_WB 0000000180013840     libucrt:system.obj
 0001:00012850       ?slash_c@?1???$common_system@_W@@YAHQEB_W@Z@4QB_WB 0000000180013850     libucrt:system.obj
 0001:00012960       __acrt_initializers        0000000180013960     libucrt:initialization.obj
 0001:00013180       __real@433fffffffffffff    0000000180014180     libucrt:fpsr.obj
 0001:00013188       __real@c33fffffffffffff    0000000180014188     libucrt:fpsr.obj
 0001:00013690       ?module_names@?A0x391cf84c@@3QBQEB_WB 0000000180014690     libucrt:winapi_thunks.obj
 0001:00013b88       ?candidate_modules@?1??try_get_AreFileApisANSI@@YAP6AHXZXZ@4QBW4module_id@?A0x391cf84c@@B 0000000180014b88     libucrt:winapi_thunks.obj
 0001:00013ba0       ?candidate_modules@?1??try_get_CompareStringEx@@YAP6AHPEB_WK0H0HPEAU_nlsversioninfo@@PEAX_J@ZXZ@4QBW4module_id@?A0x391cf84c@@B 0000000180014ba0     libucrt:winapi_thunks.obj
 0001:00013bb8       ?candidate_modules@?1??try_get_FlsAlloc@@YAP6AKP6AXPEAX@Z@ZXZ@4QBW4module_id@?A0x391cf84c@@B 0000000180014bb8     libucrt:winapi_thunks.obj
 0001:00013bc0       ?candidate_modules@?1??try_get_FlsFree@@YAP6AHK@ZXZ@4QBW4module_id@?A0x391cf84c@@B 0000000180014bc0     libucrt:winapi_thunks.obj
 0001:00013bc8       ?candidate_modules@?1??try_get_FlsGetValue@@YAP6APEAXK@ZXZ@4QBW4module_id@?A0x391cf84c@@B 0000000180014bc8     libucrt:winapi_thunks.obj
 0001:00013bd0       ?candidate_modules@?1??try_get_FlsSetValue@@YAP6AHKPEAX@ZXZ@4QBW4module_id@?A0x391cf84c@@B 0000000180014bd0     libucrt:winapi_thunks.obj
 0001:00013bd8       ?candidate_modules@?1??try_get_InitializeCriticalSectionEx@@YAP6AHPEAU_RTL_CRITICAL_SECTION@@KK@ZXZ@4QBW4module_id@?A0x391cf84c@@B 0000000180014bd8     libucrt:winapi_thunks.obj
 0001:00013be0       ?candidate_modules@?1??try_get_LCMapStringEx@@YAP6AHPEB_WK0HPEA_WHPEAU_nlsversioninfo@@PEAX_J@ZXZ@4QBW4module_id@?A0x391cf84c@@B 0000000180014be0     libucrt:winapi_thunks.obj
 0001:00013bf8       ?candidate_modules@?1??try_get_LocaleNameToLCID@@YAP6AKPEB_WK@ZXZ@4QBW4module_id@?A0x391cf84c@@B 0000000180014bf8     libucrt:winapi_thunks.obj
 0001:00013c14       ?candidate_modules@?1??try_get_AppPolicyGetProcessTerminationMethod@@YAP6AJPEAXPEAW4AppPolicyProcessTerminationMethod@@@ZXZ@4QBW4module_id@?A0x391cf84c@@B 0000000180014c14     libucrt:winapi_thunks.obj
 0001:00014444       ?dot_slash@?CB@???$common_spawnv@_W@@YA_JHQEB_WQEBQEB_W1@Z@4QB_WB 0000000180015444     libucrt:spawnv.obj
 0001:00014450       ?extensions@?CP@???$common_spawnv@_W@@YA_JHQEB_WQEBQEB_W1@Z@4QAY04$$CB_WA 0000000180015450     libucrt:spawnv.obj
 0001:00014478       ?_mb_locale_names@@3QBQEB_WB 0000000180015478     libucrt:mbctype.obj
 0001:00014ee0       ?LocaleNameToIndexTable@?A0x881e4c05@@3QBULocaleNameIndex@1@B 0000000180015ee0     libucrt:lcidtoname_downlevel.obj
 0001:00016780       ?LcidToLocaleNameTable@?A0x881e4c05@@3QBULcidToLocaleName@1@B 0000000180017780     libucrt:lcidtoname_downlevel.obj
 0001:000177ec       ?equal_sign@?BD@???$construct_environment_block@_W@@YAHQEBQEB_WQEAPEA_W@Z@4QB_WB 00000001800187ec     libucrt:cenvarg.obj
 0001:000177f0       __real_ninf                00000001800187f0     libucrt:log10.obj
 0001:00017800       __real_inf                 0000000180018800     libucrt:log10.obj
 0001:00017810       __real_neg_qnan            0000000180018810     libucrt:log10.obj
 0001:00017820       __real_qnanbit             0000000180018820     libucrt:log10.obj
 0001:00017830       __int_1023                 0000000180018830     libucrt:log10.obj
 0001:00017840       __mask_001                 0000000180018840     libucrt:log10.obj
 0001:00017850       __mask_mant                0000000180018850     libucrt:log10.obj
 0001:00017860       __mask_mant_top8           0000000180018860     libucrt:log10.obj
 0001:00017870       __mask_mant9               0000000180018870     libucrt:log10.obj
 0001:00017880       __real_log10_e             0000000180018880     libucrt:log10.obj
 0001:00017890       __real_log10_e_lead        0000000180018890     libucrt:log10.obj
 0001:000178a0       __real_log10_e_tail        00000001800188a0     libucrt:log10.obj
 0001:000178b0       __real_log10_2_lead        00000001800188b0     libucrt:log10.obj
 0001:000178c0       __real_log10_2_tail        00000001800188c0     libucrt:log10.obj
 0001:000178d0       __real_two                 00000001800188d0     libucrt:log10.obj
 0001:000178e0       __real_one                 00000001800188e0     libucrt:log10.obj
 0001:000178f0       __real_half                00000001800188f0     libucrt:log10.obj
 0001:00017900       __mask_100                 0000000180018900     libucrt:log10.obj
 0001:00017910       __real_1_over_512          0000000180018910     libucrt:log10.obj
 0001:00017920       __real_1_over_2            0000000180018920     libucrt:log10.obj
 0001:00017930       __real_1_over_3            0000000180018930     libucrt:log10.obj
 0001:00017940       __real_1_over_4            0000000180018940     libucrt:log10.obj
 0001:00017950       __real_1_over_5            0000000180018950     libucrt:log10.obj
 0001:00017960       __real_1_over_6            0000000180018960     libucrt:log10.obj
 0001:00017970       __real_neg_1023            0000000180018970     libucrt:log10.obj
 0001:00017980       __mask_2045                0000000180018980     libucrt:log10.obj
 0001:00017990       __real_threshold           0000000180018990     libucrt:log10.obj
 0001:000179a0       __real_near_one_lt         00000001800189a0     libucrt:log10.obj
 0001:000179b0       __real_near_one_gt         00000001800189b0     libucrt:log10.obj
 0001:000179c0       __real_min_norm            00000001800189c0     libucrt:log10.obj
 0001:000179d0       __real_notsign             00000001800189d0     libucrt:log10.obj
 0001:000179e0       __real_ca1                 00000001800189e0     libucrt:log10.obj
 0001:000179f0       __real_ca2                 00000001800189f0     libucrt:log10.obj
 0001:00017a00       __real_ca3                 0000000180018a00     libucrt:log10.obj
 0001:00017a10       __real_ca4                 0000000180018a10     libucrt:log10.obj
 0001:00017a20       __mask_lower               0000000180018a20     libucrt:log10.obj
 0001:00017a30       __flag_x_zero              0000000180018a30     libucrt:log10.obj
 0001:00017a34       __flag_x_neg               0000000180018a34     libucrt:log10.obj
 0001:00017a38       __flag_x_nan               0000000180018a38     libucrt:log10.obj
 0001:00019288       GS_ExceptionPointers       000000018001a288     LIBCMT:gs_report.obj
 0001:00019660       $$000000                   000000018001a660     chkstk.obj
 0001:000196d0       f_unm                      000000018001a6d0 f   bit64.obj
 0001:00019700       f_eq                       000000018001a700 f   bit64.obj
 0001:00019750       f_lt                       000000018001a750 f   bit64.obj
 0001:000197a0       f_le                       000000018001a7a0 f   bit64.obj
 0001:000197f0       band                       000000018001a7f0 f   bit64.obj
 0001:000198c0       bor                        000000018001a8c0 f   bit64.obj
 0001:00019990       bxor                       000000018001a990 f   bit64.obj
 0001:00019a60       bnot                       000000018001aa60 f   bit64.obj
 0001:00019a90       lshift                     000000018001aa90 f   bit64.obj
 0001:00019ae0       rshift                     000000018001aae0 f   bit64.obj
 0001:00019b30       arshift                    000000018001ab30 f   bit64.obj
 0001:00019b90       f_new                      000000018001ab90 f   bit64.obj
 0001:00019e00       f_tostring                 000000018001ae00 f   bit64.obj
 0001:00019e50       f_type                     000000018001ae50 f   bit64.obj
 0001:00019ef0       f_add                      000000018001aef0 f   bit64.obj
 0001:00019fc0       f_sub                      000000018001afc0 f   bit64.obj
 0001:0001a010       f_mul                      000000018001b010 f   bit64.obj
 0001:0001a0e0       f_div                      000000018001b0e0 f   bit64.obj
 0001:0001a160       f_mod                      000000018001b160 f   bit64.obj
 0001:0001a360       check64                    000000018001b360 f   bit64.obj
 0001:0001a6e0       FillFarMacroCall           000000018001b6e0 f   exported.obj
 0001:0001a920       FillFarMacroCall_Callback  000000018001b920 f   exported.obj
 0001:0001de70       PushAnalyseInfo            000000018001ee70 f   exported.obj
 0001:0001e060       RegisterObject             000000018001f060 f   exported.obj
 0001:0001ebc0       errfile                    000000018001fbc0 f   lflua.obj
 0001:0001ec40       getF                       000000018001fc40 f   lflua.obj
 0001:0001ff40       FL_PushParams              0000000180020f40 f   luamacro.obj
 0001:0001ffe0       InitMPR                    0000000180020fe0 f   luamacro.obj
 0001:00020050       MacroCallFarCallback       0000000180021050 f   luamacro.obj
 0001:00020720       uc_tostring                0000000180021720 f   lusercontrol.obj
 0001:000207a0       uc_index                   00000001800217a0 f   lusercontrol.obj
 0001:000208a0       uc_newindex                00000001800218a0 f   lusercontrol.obj
 0001:000209b0       uc_New                     00000001800219b0 f   lusercontrol.obj
 0001:00020d40       far_GetFileOwner           0000000180021d40 f   service.obj
 0001:00020df0       far_GetNumberOfLinks       0000000180021df0 f   service.obj
 0001:00020e50       far_PluginStartupInfo      0000000180021e50 f   service.obj
 0001:00020f20       far_GetCurrentDirectory    0000000180021f20 f   service.obj
 0001:00020fa0       editor_GetFileName         0000000180021fa0 f   service.obj
 0001:00021070       editor_GetInfo             0000000180022070 f   service.obj
 0001:000213f0       editor_GetString           00000001800223f0 f   service.obj
 0001:00021400       editor_GetStringW          0000000180022400 f   service.obj
 0001:00021410       editor_SetString           0000000180022410 f   service.obj
 0001:00021420       editor_SetStringW          0000000180022420 f   service.obj
 0001:00021430       editor_InsertString        0000000180022430 f   service.obj
 0001:000214c0       editor_DeleteString        00000001800224c0 f   service.obj
 0001:00021530       editor_InsertText          0000000180022530 f   service.obj
 0001:000215b0       editor_InsertTextW         00000001800225b0 f   service.obj
 0001:000215c0       editor_DeleteChar          00000001800225c0 f   service.obj
 0001:00021630       editor_DeleteBlock         0000000180022630 f   service.obj
 0001:000216a0       editor_UndoRedo            00000001800226a0 f   service.obj
 0001:00021730       editor_SetKeyBar           0000000180022730 f   service.obj
 0001:00021740       viewer_SetKeyBar           0000000180022740 f   service.obj
 0001:00021750       editor_SetParam            0000000180022750 f   service.obj
 0001:000218b0       editor_SetPosition         00000001800228b0 f   service.obj
 0001:000219e0       editor_Redraw              00000001800229e0 f   service.obj
 0001:00021a50       editor_ExpandTabs          0000000180022a50 f   service.obj
 0001:00021ae0       editor_GetBookmarks        0000000180022ae0 f   service.obj
 0001:00021af0       editor_GetSessionBookmarks 0000000180022af0 f   service.obj
 0001:00021b00       editor_AddSessionBookmark  0000000180022b00 f   service.obj
 0001:00021b70       editor_ClearSessionBookmarks 0000000180022b70 f   service.obj
 0001:00021be0       editor_DeleteSessionBookmark 0000000180022be0 f   service.obj
 0001:00021c70       editor_NextSessionBookmark 0000000180022c70 f   service.obj
 0001:00021ce0       editor_PrevSessionBookmark 0000000180022ce0 f   service.obj
 0001:00021d50       editor_SetTitle            0000000180022d50 f   service.obj
 0001:00021dd0       editor_GetTitle            0000000180022dd0 f   service.obj
 0001:00021e90       editor_Quit                0000000180022e90 f   service.obj
 0001:00021f00       editor_Select              0000000180022f00 f   service.obj
 0001:00022030       editor_GetSelection        0000000180023030 f   service.obj
 0001:000223d0       editor_TabToReal           00000001800233d0 f   service.obj
 0001:000223e0       editor_RealToTab           00000001800233e0 f   service.obj
 0001:000223f0       editor_AddColor            00000001800233f0 f   service.obj
 0001:000225d0       editor_DelColor            00000001800235d0 f   service.obj
 0001:00022700       editor_GetColor            0000000180023700 f   service.obj
 0001:000228f0       editor_SaveFile            00000001800238f0 f   service.obj
 0001:000229b0       editor_ReadInput           00000001800239b0 f   service.obj
 0001:00022a30       editor_ProcessInput        0000000180023a30 f   service.obj
 0001:00022ac0       editor_SubscribeChangeEvent 0000000180023ac0 f   service.obj
 0001:00022b50       far_Menu                   0000000180023b50 f   service.obj
 0001:000235e0       far_Message                00000001800245e0 f   service.obj
 0001:000237a0       panel_CheckPanelsExist     00000001800247a0 f   service.obj
 0001:00023800       panel_ClosePanel           0000000180024800 f   service.obj
 0001:00023870       panel_GetPanelInfo         0000000180024870 f   service.obj
 0001:00023b10       panel_GetPanelItem         0000000180024b10 f   service.obj
 0001:00023b20       panel_GetSelectedPanelItem 0000000180024b20 f   service.obj
 0001:00023b30       panel_GetCurrentPanelItem  0000000180024b30 f   service.obj
 0001:00023b40       panel_GetPanelFormat       0000000180024b40 f   service.obj
 0001:00023b50       panel_GetPanelHostFile     0000000180024b50 f   service.obj
 0001:00023b60       panel_GetColumnTypes       0000000180024b60 f   service.obj
 0001:00023b70       panel_GetColumnWidths      0000000180024b70 f   service.obj
 0001:00023b80       panel_GetPanelPrefix       0000000180024b80 f   service.obj
 0001:00023b90       panel_RedrawPanel          0000000180024b90 f   service.obj
 0001:00023ca0       panel_SetSortOrder         0000000180024ca0 f   service.obj
 0001:00023cb0       panel_SetDirectoriesFirst  0000000180024cb0 f   service.obj
 0001:00023cc0       panel_UpdatePanel          0000000180024cc0 f   service.obj
 0001:00023cd0       panel_SetSortMode          0000000180024cd0 f   service.obj
 0001:00023ce0       panel_SetViewMode          0000000180024ce0 f   service.obj
 0001:00023cf0       panel_GetPanelDirectory    0000000180024cf0 f   service.obj
 0001:00023e50       panel_SetPanelDirectory    0000000180024e50 f   service.obj
 0001:00024040       panel_GetCmdLine           0000000180025040 f   service.obj
 0001:000240e0       panel_SetCmdLine           00000001800250e0 f   service.obj
 0001:00024160       panel_GetCmdLinePos        0000000180025160 f   service.obj
 0001:000241e0       panel_SetCmdLinePos        00000001800251e0 f   service.obj
 0001:00024260       panel_InsertCmdLine        0000000180025260 f   service.obj
 0001:000242e0       panel_GetCmdLineSelection  00000001800252e0 f   service.obj
 0001:00024390       panel_SetCmdLineSelection  0000000180025390 f   service.obj
 0001:00024450       panel_SetSelection         0000000180025450 f   service.obj
 0001:00024460       panel_ClearSelection       0000000180025460 f   service.obj
 0001:00024470       panel_SetUserScreen        0000000180025470 f   service.obj
 0001:000244f0       panel_GetUserScreen        00000001800254f0 f   service.obj
 0001:00024570       panel_IsActivePanel        0000000180025570 f   service.obj
 0001:000245d0       panel_SetActivePanel       00000001800255d0 f   service.obj
 0001:00024670       far_GetDirList             0000000180025670 f   service.obj
 0001:000249d0       far_GetPluginDirList       00000001800259d0 f   service.obj
 0001:00024a70       far_RestoreScreen          0000000180025a70 f   service.obj
 0001:00024b00       far_SaveScreen             0000000180025b00 f   service.obj
 0001:00024be0       far_SendDlgMessage         0000000180025be0 f   service.obj
 0001:00025e60       $LN154                     0000000180026e60     service.obj
 0001:00025e6c       $LN153                     0000000180026e6c     service.obj
 0001:00025eb0       $LN152                     0000000180026eb0     service.obj
 0001:00025f38       $LN151                     0000000180026f38     service.obj
 0001:00025f80       far_DialogInit             0000000180026f80 f   service.obj
 0001:00026360       far_DialogRun              0000000180027360 f   service.obj
 0001:00026400       far_DialogFree             0000000180027400 f   service.obj
 0001:00026430       dialog_tostring            0000000180027430 f   service.obj
 0001:00026490       dialog_rawhandle           0000000180027490 f   service.obj
 0001:000264e0       far_GetDlgItem             00000001800274e0 f   service.obj
 0001:00026590       far_SetDlgItem             0000000180027590 f   service.obj
 0001:00026630       far_SubscribeDialogDrawEvents 0000000180027630 f   service.obj
 0001:00026650       editor_Editor              0000000180027650 f   service.obj
 0001:000267f0       viewer_Viewer              00000001800277f0 f   service.obj
 0001:00026950       viewer_GetFileName         0000000180027950 f   service.obj
 0001:00026a20       viewer_GetInfo             0000000180027a20 f   service.obj
 0001:00026cf0       viewer_Quit                0000000180027cf0 f   service.obj
 0001:00026d50       viewer_Redraw              0000000180027d50 f   service.obj
 0001:00026db0       viewer_Select              0000000180027db0 f   service.obj
 0001:00026e60       viewer_SetPosition         0000000180027e60 f   service.obj
 0001:00027030       viewer_SetMode             0000000180028030 f   service.obj
 0001:00027170       far_ShowHelp               0000000180028170 f   service.obj
 0001:00027240       far_InputBox               0000000180028240 f   service.obj
 0001:00027430       far_GetMsg                 0000000180028430 f   service.obj
 0001:000274b0       far_Text                   00000001800284b0 f   service.obj
 0001:00027560       far_CopyToClipboard        0000000180028560 f   service.obj
 0001:00027650       far_PasteFromClipboard     0000000180028650 f   service.obj
 0001:00027730       far_InputRecordToName      0000000180028730 f   service.obj
 0001:00027930       far_NameToInputRecord      0000000180028930 f   service.obj
 0001:000279b0       far_LStricmp               00000001800289b0 f   service.obj
 0001:00027a30       far_LStrnicmp              0000000180028a30 f   service.obj
 0001:00027ad0       far_ProcessName            0000000180028ad0 f   service.obj
 0001:00027ce0       far_GetReparsePointInfo    0000000180028ce0 f   service.obj
 0001:00027d80       far_LIsAlpha               0000000180028d80 f   service.obj
 0001:00027de0       far_LIsAlphanum            0000000180028de0 f   service.obj
 0001:00027e40       far_LIsLower               0000000180028e40 f   service.obj
 0001:00027ea0       far_LIsUpper               0000000180028ea0 f   service.obj
 0001:00027f00       far_LLowerBuf              0000000180028f00 f   service.obj
 0001:00027f70       far_LUpperBuf              0000000180028f70 f   service.obj
 0001:00027fe0       far_MkTemp                 0000000180028fe0 f   service.obj
 0001:00028070       far_MkLink                 0000000180029070 f   service.obj
 0001:00028150       far_GetPathRoot            0000000180029150 f   service.obj
 0001:000281f0       far_TruncPathStr           00000001800291f0 f   service.obj
 0001:00028200       far_TruncStr               0000000180029200 f   service.obj
 0001:00028210       far_RecursiveSearch        0000000180029210 f   service.obj
 0001:00028360       far_ConvertPath            0000000180029360 f   service.obj
 0001:00028430       far_AdvControl             0000000180029430 f   service.obj
 0001:00028c2c       $LN62                      0000000180029c2c     service.obj
 0001:00028ca0       far_MacroLoadAll           0000000180029ca0 f   service.obj
 0001:00028d70       far_MacroSaveAll           0000000180029d70 f   service.obj
 0001:00028dc0       far_MacroGetState          0000000180029dc0 f   service.obj
 0001:00028e10       far_MacroGetArea           0000000180029e10 f   service.obj
 0001:00028e60       far_MacroPost              0000000180029e60 f   service.obj
 0001:00028e70       far_MacroCheck             0000000180029e70 f   service.obj
 0001:00028e80       far_MacroGetLastError      0000000180029e80 f   service.obj
 0001:00028f80       far_MacroAdd               0000000180029f80 f   service.obj
 0001:00029220       far_MacroDelete            000000018002a220 f   service.obj
 0001:000292e0       far_MacroExecute           000000018002a2e0 f   service.obj
 0001:00029460       far_CPluginStartupInfo     000000018002a460 f   service.obj
 0001:00029490       far_MakeMenuItems          000000018002a490 f   service.obj
 0001:00029830       far_Show                   000000018002a830 f   service.obj
 0001:000298e0       far_CreateFileFilter       000000018002a8e0 f   service.obj
 0001:000299a0       filefilter_Free            000000018002a9a0 f   service.obj
 0001:00029a30       filefilter_gc              000000018002aa30 f   service.obj
 0001:00029ac0       filefilter_tostring        000000018002aac0 f   service.obj
 0001:00029b20       filefilter_OpenMenu        000000018002ab20 f   service.obj
 0001:00029bb0       filefilter_Starting        000000018002abb0 f   service.obj
 0001:00029c40       filefilter_IsFileInFilter  000000018002ac40 f   service.obj
 0001:00029d10       far_LoadPlugin             000000018002ad10 f   service.obj
 0001:00029d20       far_ForcedLoadPlugin       000000018002ad20 f   service.obj
 0001:00029d30       far_UnloadPlugin           000000018002ad30 f   service.obj
 0001:00029da0       far_FindPlugin             000000018002ada0 f   service.obj
 0001:00029e50       far_GetPluginInformation   000000018002ae50 f   service.obj
 0001:0002a0f0       far_GetPlugins             000000018002b0f0 f   service.obj
 0001:0002a210       far_IsPluginLoaded         000000018002b210 f   service.obj
 0001:0002a320       far_XLat                   000000018002b320 f   service.obj
 0001:0002a420       far_FormatFileSize         000000018002b420 f   service.obj
 0001:0002a550       far_FarClock               000000018002b550 f   service.obj
 0001:0002a5a0       far_Timer                  000000018002b5a0 f   service.obj
 0001:0002a790       timer_gc                   000000018002b790 f   service.obj
 0001:0002a830       timer_tostring             000000018002b830 f   service.obj
 0001:0002a890       timer_index                000000018002b890 f   service.obj
 0001:0002aa00       timer_newindex             000000018002ba00 f   service.obj
 0001:0002abb0       far_CreateSettings         000000018002bbb0 f   service.obj
 0001:0002ad80       Settings_set               000000018002bd80 f   service.obj
 0001:0002aeb0       Settings_get               000000018002beb0 f   service.obj
 0001:0002b000       Settings_delete            000000018002c000 f   service.obj
 0001:0002b0d0       Settings_createsubkey      000000018002c0d0 f   service.obj
 0001:0002b210       Settings_opensubkey        000000018002c210 f   service.obj
 0001:0002b2f0       Settings_enum              000000018002c2f0 f   service.obj
 0001:0002b610       Settings_free              000000018002c610 f   service.obj
 0001:0002b6b0       far_FreeSettings           000000018002c6b0 f   service.obj
 0001:0002b750       Settings_tostring          000000018002c750 f   service.obj
 0001:0002b7b0       far_ColorDialog            000000018002c7b0 f   service.obj
 0001:0002b900       far_RunDefaultScript       000000018002c900 f   service.obj
 0001:0002b930       AddMacroData_gc            000000018002c930 f   service.obj
 0001:0002b9e0       ChangePanelSelection       000000018002c9e0 f   service.obj
 0001:0002bc80       CheckFlags                 000000018002cc80 f   service.obj
 0001:0002bcd0       CheckFlagsFromTable        000000018002ccd0 f   service.obj
 0001:0002c050       CustomAllocator            000000018002d050 f   service.obj
 0001:0002c180       FillEditorSelect           000000018002d180 f   service.obj
 0001:0002c280       FillEditorSetPosition      000000018002d280 f   service.obj
 0001:0002c590       FillKeyBarTitles           000000018002d590 f   service.obj
 0001:0002c780       FrsUserFunc                000000018002d780 f   service.obj
 0001:0002da40       MacroSendString            000000018002ea40 f   service.obj
 0001:0002de30       OptInputRecord             000000018002ee30 f   service.obj
 0001:0002e1a0       PushBookmarks              000000018002f1a0 f   service.obj
 0001:0002e3f4       $LN15                      000000018002f3f4     service.obj
 0001:0002e400       $LN14                      000000018002f400     service.obj
 0001:0002e6a0       $LN32                      000000018002f6a0     service.obj
 0001:0002e6ac       $LN31                      000000018002f6ac     service.obj
 0001:0002e6c4       $LN30                      000000018002f6c4     service.obj
 0001:0002e720       PushDlgItem                000000018002f720 f   service.obj
 0001:0002e980       PushDlgItemNum             000000018002f980 f   service.obj
 0001:0002f200       PushPluginHandle           0000000180030200 f   service.obj
 0001:0002f2a0       PutPluginMenuItemToTable   00000001800302a0 f   service.obj
 0001:0002f3c0       PutVersionInfoToTable      00000001800303c0 f   service.obj
 0001:0002f460       SetDlgItem                 0000000180030460 f   service.obj
 0001:0002f520       SetFarDialogItem           0000000180030520 f   service.obj
 0001:0002f8b0       SetKeyBar                  00000001800308b0 f   service.obj
 0001:0002fa10       SetPanelBooleanProperty    0000000180030a10 f   service.obj
 0001:0002fac0       SetPanelIntegerProperty    0000000180030ac0 f   service.obj
 0001:0002fbc0       _EditorGetString           0000000180030bc0 f   service.obj
 0001:0002fe60       _EditorInsertText          0000000180030e60 f   service.obj
 0001:0002ff70       _EditorSetString           0000000180030f70 f   service.obj
 0001:000300b0       _EditorTabConvert          00000001800310b0 f   service.obj
 0001:00030170       check_env_flag             0000000180031170 f   service.obj
 0001:00030290       free_dialog                0000000180031290 f   service.obj
 0001:00030300       get_env_flag               0000000180031300 f   service.obj
 0001:00030430       get_panel_item             0000000180031430 f   service.obj
 0001:00030540       get_string_info            0000000180031540 f   service.obj
 0001:00030630       luaopen_far                0000000180031630 f   service.obj
 0001:00030a00       plugin_load                0000000180031a00 f   service.obj
 0001:00030b00       timer_Close                0000000180031b00 f   service.obj
 0001:00030bc0       truncstring                0000000180031bc0 f   service.obj
 0001:00030cb0       unic_len                   0000000180031cb0 f   slnunico.obj
 0001:00030d50       unic_sub                   0000000180031d50 f   slnunico.obj
 0001:00030fa0       str_reverse                0000000180031fa0 f   slnunico.obj
 0001:00031170       unic_lower                 0000000180032170 f   slnunico.obj
 0001:000312f0       unic_upper                 00000001800322f0 f   slnunico.obj
 0001:00031470       str_rep                    0000000180032470 f   slnunico.obj
 0001:00031500       unic_byte                  0000000180032500 f   slnunico.obj
 0001:000316e0       unic_char                  00000001800326e0 f   slnunico.obj
 0001:00031800       str_dump                   0000000180032800 f   slnunico.obj
 0001:00031880       unic_find                  0000000180032880 f   slnunico.obj
 0001:00031890       unic_match                 0000000180032890 f   slnunico.obj
 0001:000318a0       gmatch                     00000001800328a0 f   slnunico.obj
 0001:00031970       gfind_nodef                0000000180032970 f   slnunico.obj
 0001:00031980       unic_gsub                  0000000180032980 f   slnunico.obj
 0001:00031be0       str_format                 0000000180032be0 f   slnunico.obj
 0001:00032124       $LN73                      0000000180033124     slnunico.obj
 0001:00032140       $LN72                      0000000180033140     slnunico.obj
 0001:00032180       utf8_valid                 0000000180033180 f   slnunico.obj
 0001:000322f0       add_value                  00000001800332f0 f   slnunico.obj
 0001:00032510       gmatch_aux                 0000000180033510 f   slnunico.obj
 0001:00032710       grab_one_utf8              0000000180033710 f   slnunico.obj
 0001:00032950       match                      0000000180033950 f   slnunico.obj
 0001:00032d20       match_class                0000000180033d20 f   slnunico.obj
 0001:00032e88       $LN26                      0000000180033e88     slnunico.obj
 0001:00032ef0       max_expand                 0000000180033ef0 f   slnunico.obj
 0001:00033060       min_expand                 0000000180034060 f   slnunico.obj
 0001:00033340       push_captures              0000000180034340 f   slnunico.obj
 0001:00033440       push_onecapture            0000000180034440 f   slnunico.obj
 0001:000334f0       singlematch                00000001800344f0 f   slnunico.obj
 0001:00033780       start_capture              0000000180034780 f   slnunico.obj
 0001:00033810       unic_find_aux              0000000180034810 f   slnunico.obj
 0001:00033b60       utf8_count                 0000000180034b60 f   slnunico.obj
 0001:00033c40       utf8_deco                  0000000180034c40 f   slnunico.obj
 0001:00033d20       utf8_enco                  0000000180034d20 f   slnunico.obj
 0001:00033e40       utf8_graphext              0000000180034e40 f   slnunico.obj
 0001:00033f90       utf8_oced                  0000000180034f90 f   slnunico.obj
 0001:00034080       writer                     0000000180035080 f   slnunico.obj
 0001:000340a0       io_type                    00000001800350a0 f   uliolib51.obj
 0001:00034170       io_close                   0000000180035170 f   uliolib51.obj
 0001:00034200       io_gc                      0000000180035200 f   uliolib51.obj
 0001:00034260       io_tostring                0000000180035260 f   uliolib51.obj
 0001:000342c0       io_open                    00000001800352c0 f   uliolib51.obj
 0001:000343e0       io_popen                   00000001800353e0 f   uliolib51.obj
 0001:000344a0       io_tmpfile                 00000001800354a0 f   uliolib51.obj
 0001:00034550       io_input                   0000000180035550 f   uliolib51.obj
 0001:00034570       io_output                  0000000180035570 f   uliolib51.obj
 0001:00034590       f_lines                    0000000180035590 f   uliolib51.obj
 0001:00034600       io_lines                   0000000180035600 f   uliolib51.obj
 0001:00034750       io_read                    0000000180035750 f   uliolib51.obj
 0001:000347c0       f_read                     00000001800357c0 f   uliolib51.obj
 0001:00034820       io_write                   0000000180035820 f   uliolib51.obj
 0001:00034890       f_write                    0000000180035890 f   uliolib51.obj
 0001:000348f0       f_seek                     00000001800358f0 f   uliolib51.obj
 0001:000349f0       f_setvbuf                  00000001800359f0 f   uliolib51.obj
 0001:00034ae0       io_flush                   0000000180035ae0 f   uliolib51.obj
 0001:00034ba0       f_flush                    0000000180035ba0 f   uliolib51.obj
 0001:00034c50       f_rawhandle                0000000180035c50 f   uliolib51.obj
 0001:00034cc0       aux_close                  0000000180035cc0 f   uliolib51.obj
 0001:00034d00       fileerror                  0000000180035d00 f   uliolib51.obj
 0001:00034dd0       g_iofile                   0000000180035dd0 f   uliolib51.obj
 0001:00034ee0       g_read                     0000000180035ee0 f   uliolib51.obj
 0001:000350e0       g_write                    00000001800360e0 f   uliolib51.obj
 0001:000351f0       io_fclose                  00000001800361f0 f   uliolib51.obj
 0001:00035290       io_noclose                 0000000180036290 f   uliolib51.obj
 0001:000352c0       io_pclose                  00000001800362c0 f   uliolib51.obj
 0001:00035370       io_readline                0000000180036370 f   uliolib51.obj
 0001:00035750       newfile                    0000000180036750 f   uliolib51.obj
 0001:000357a0       pushresult                 00000001800367a0 f   uliolib51.obj
 0001:00035870       read_chars                 0000000180036870 f   uliolib51.obj
 0001:00035920       read_line                  0000000180036920 f   uliolib51.obj
 0001:00035a10       ll_loadlib                 0000000180036a10 f   uloadlib51.obj
 0001:00035aa0       loader_Lua                 0000000180036aa0 f   uloadlib51.obj
 0001:00035b00       loader_C                   0000000180036b00 f   uloadlib51.obj
 0001:00035b80       loader_Croot               0000000180036b80 f   uloadlib51.obj
 0001:00035c50       loader_preload             0000000180036c50 f   uloadlib51.obj
 0001:00035cf0       ll_require                 0000000180036cf0 f   uloadlib51.obj
 0001:00035f40       ll_module                  0000000180036f40 f   uloadlib51.obj
 0001:00036190       ll_seeall                  0000000180037190 f   uloadlib51.obj
 0001:00036210       findfile                   0000000180037210 f   uloadlib51.obj
 0001:00036430       gctm                       0000000180037430 f   uloadlib51.obj
 0001:00036480       ll_loadfunc                0000000180037480 f   uloadlib51.obj
 0001:000365f0       loaderror                  00000001800375f0 f   uloadlib51.obj
 0001:00036850       mkfuncname                 0000000180037850 f   uloadlib51.obj
 0001:000368c0       setpath                    00000001800378c0 f   uloadlib51.obj
 0001:00037604       $LN12                      0000000180038604     ustring.obj
 0001:00038070       ustring_OutputDebugString  0000000180039070 f   ustring.obj
 0001:000382a0       ustring_system             00000001800392a0 f   ustring.obj
 0001:00039540       win_GetEnv                 000000018003a540 f   win.obj
 0001:00039610       win_SetEnv                 000000018003a610 f   win.obj
 0001:00039670       win_SetRegKey              000000018003a670 f   win.obj
 0001:000398a0       win_GetRegKey              000000018003a8a0 f   win.obj
 0001:00039a70       win_DeleteRegKey           000000018003aa70 f   win.obj
 0001:00039b30       win_DeleteRegValue         000000018003ab30 f   win.obj
 0001:00039bf0       win_EnumRegKey             000000018003abf0 f   win.obj
 0001:00039d20       win_EnumRegValue           000000018003ad20 f   win.obj
 0001:00039e50       win_ExtractKey             000000018003ae50 f   win.obj
 0001:00039f10       win_ExtractKeyEx           000000018003af10 f   win.obj
 0001:00039fb0       win_GetFileInfo            000000018003afb0 f   win.obj
 0001:0003a0e0       win_GetSystemTimeAsFileTime 000000018003b0e0 f   win.obj
 0001:0003a110       win_FileTimeToSystemTime   000000018003b110 f   win.obj
 0001:0003a220       win_SystemTimeToFileTime   000000018003b220 f   win.obj
 0001:0003a340       win_FileTimeToLocalFileTime 000000018003b340 f   win.obj
 0001:0003a3b0       win_CompareString          000000018003b3b0 f   win.obj
 0001:0003a540       win_wcscmp                 000000018003b540 f   win.obj
 0001:0003a5c0       win_GetVirtualKeys         000000018003b5c0 f   win.obj
 0001:0003a5e0       win_GetConsoleScreenBufferInfo 000000018003b5e0 f   win.obj
 0001:0003a720       win_CopyFile               000000018003b720 f   win.obj
 0001:0003a7c0       win_MoveFile               000000018003b7c0 f   win.obj
 0001:0003a8d0       win_DeleteFile             000000018003b8d0 f   win.obj
 0001:0003a920       win_CreateDir              000000018003b920 f   win.obj
 0001:0003aa40       win_RemoveDir              000000018003ba40 f   win.obj
 0001:0003aa90       win_ShellExecute           000000018003ba90 f   win.obj
 0001:0003ab70       win_IsProcess64bit         000000018003bb70 f   win.obj
 0001:0003ab90       CheckHKey                  000000018003bb90 f   win.obj
 0001:0003ad60       mkdir                      000000018003bd60 f   win.obj
 0001:0003b17c       ?dllmain_crt_dispatch@@YAHQEAUHINSTANCE__@@KQEAX@Z 000000018003c17c f   LIBCMT:dll_dllmain.obj
 0001:0003b1cc       ?dllmain_crt_process_attach@@YAHQEAUHINSTANCE__@@QEAX@Z 000000018003c1cc f   LIBCMT:dll_dllmain.obj
 0001:0003b2e4       ?dllmain_crt_process_detach@@YAH_N@Z 000000018003c2e4 f   LIBCMT:dll_dllmain.obj
 0001:0003b368       ?dllmain_dispatch@@YAHQEAUHINSTANCE__@@KQEAX@Z 000000018003c368 f   LIBCMT:dll_dllmain.obj
 0001:0003bdb0       $$000000                   000000018003cdb0     libvcruntime:memcpy.obj
 0001:0003be57       MoveSmall                  000000018003ce57     libvcruntime:memcpy.obj
 0001:0003c210       $$000000                   000000018003d210     libvcruntime:memset.obj
 0001:0003c30c       MsetTab                    000000018003d30c     libvcruntime:memset.obj
 0001:0003c710       $$000000                   000000018003d710     libvcruntime:memchr.obj
 0001:0003c790       $$000000                   000000018003d790     libvcruntime:memcmp.obj
 0001:0003cc80       $$000000                   000000018003dc80     libvcruntime:_jmpuwind_.obj
 0001:0003cf48       ?try_get_function@@YAPEAXW4function_id@?A0x89697e75@@QEBDQEBW4module_id@2@2@Z 000000018003df48 f   libvcruntime:winapi_downlevel.obj
 0001:0003d330       $$000000                   000000018003e330     libvcruntime:handlers.obj
 0001:0003d3f8       ??$?RV<lambda_a62c933ada0517137acf5807a1eeac1f>@@AEAV<lambda_a31071773b9a94e445cbd5d04ef99106>@@V<lambda_56065050dbf3ada7e59a83db45153de3>@@@?$__crt_seh_guarded_call@H@@QEAAH$$QEAV<lambda_a62c933ada0517137acf5807a1eeac1f>@@AEAV<lambda_a31071773b9a94e445cbd5d04ef99106>@@$$QEAV<lambda_56065050dbf3ada7e59a83db45153de3>@@@Z 000000018003e3f8 f   libucrt:output.obj
 0001:0003d438       ??$common_vsprintf@Vstandard_base@__crt_stdio_output@@D@@YAH_KQEAD0QEBDQEAU__crt_locale_pointers@@1@Z 000000018003e438 f   libucrt:output.obj
 0001:0003d604       ??$common_vsprintf@Vstandard_base@__crt_stdio_output@@_W@@YAH_KQEA_W0QEB_WQEAU__crt_locale_pointers@@QEAD@Z 000000018003e604 f   libucrt:output.obj
 0001:0003dda0       ??R<lambda_a31071773b9a94e445cbd5d04ef99106>@@QEBAHXZ 000000018003eda0 f   libucrt:output.obj
 0001:0004093c       ??$common_fsopen@_W@@YAPEAU_iobuf@@QEB_W0H@Z 000000018004193c f   libucrt:fopen.obj
 0001:00040b70       common_control87           0000000180041b70 f   libucrt:ieee.obj
 0001:00041154       ??$common_freopen@_W@@YAHQEAPEAU_iobuf@@QEB_W1V__crt_stdio_stream@@H@Z 0000000180042154 f   libucrt:freopen.obj
 0001:000419c0       $$000000                   00000001800429c0     libucrt:strcmp.obj
 0001:00041d50       $$000000                   0000000180042d50     libucrt:strncmp.obj
 0001:00041de0       $$000000                   0000000180042de0     libucrt:strncpy.obj
 0001:00041f54       fallbackMethod             0000000180042f54 f   libucrt:strpbrk.obj
 0001:00042324       $LN78                      0000000180043324     libucrt:strpbrk.obj
 0001:00042360       $LN77                      0000000180043360     libucrt:strpbrk.obj
 0001:000423a0       $LN76                      00000001800433a0     libucrt:strpbrk.obj
 0001:000423e0       ??$common_popen@_W@@YAPEAU_iobuf@@QEB_W0@Z 00000001800433e0 f   libucrt:popen.obj
 0001:000425ac       ??$common_popen_nolock@_W@@YAPEAU_iobuf@@QEB_W0HAEAY01H@Z 00000001800435ac f   libucrt:popen.obj
 0001:000428f4       ??$get_executable_path@_W@@YAPEB_WQEB_W@Z 00000001800438f4 f   libucrt:popen.obj
 0001:00042aa4       ?idtab@@YAPEAUprocess_handle_pair@?A0xe43b7539@@QEAU_iobuf@@@Z 0000000180043aa4 f   libucrt:popen.obj
 0001:00042cc0       ??$?RV<lambda_842d9ff0dc9ef11c61343bbaebe7f885>@@AEAV<lambda_c5860995281e5c4ce005b3de8f5874ee>@@V<lambda_d90129c13df834fdcbf8d2b88dafcf2d>@@@?$__crt_seh_guarded_call@X@@QEAAX$$QEAV<lambda_842d9ff0dc9ef11c61343bbaebe7f885>@@AEAV<lambda_c5860995281e5c4ce005b3de8f5874ee>@@$$QEAV<lambda_d90129c13df834fdcbf8d2b88dafcf2d>@@@Z 0000000180043cc0 f   libucrt:fflush.obj
 0001:00042d5c       ??$?RV<lambda_886d6c58226a84441f68b9f2b8217b83>@@AEAV<lambda_ab61a845afdef5b7c387490eaf3616ee>@@V<lambda_f7f22ab5edc0698d5f6905b0d3f44752>@@@?$__crt_seh_guarded_call@X@@QEAAX$$QEAV<lambda_886d6c58226a84441f68b9f2b8217b83>@@AEAV<lambda_ab61a845afdef5b7c387490eaf3616ee>@@$$QEAV<lambda_f7f22ab5edc0698d5f6905b0d3f44752>@@@Z 0000000180043d5c f   libucrt:fflush.obj
 0001:00042e44       ??$?RV<lambda_c376a267cfb53b6959b3b692ec76b120>@@AEAV<lambda_9a32fed5bf61b6b509b2d3f6003082a1>@@V<lambda_572fbb9fa0ab338edf41edfd4b5fcc8d>@@@?$__crt_seh_guarded_call@H@@QEAAH$$QEAV<lambda_c376a267cfb53b6959b3b692ec76b120>@@AEAV<lambda_9a32fed5bf61b6b509b2d3f6003082a1>@@$$QEAV<lambda_572fbb9fa0ab338edf41edfd4b5fcc8d>@@@Z 0000000180043e44 f   libucrt:fflush.obj
 0001:00042e84       ?common_flush_all@@YAH_N@Z 0000000180043e84 f   libucrt:fflush.obj
 0001:0004301c       ??$common_fgets@D@@YAPEADQEADHV__crt_stdio_stream@@@Z 000000018004401c f   libucrt:fgets.obj
 0001:000430f4       ?common_fseek@@YAHV__crt_stdio_stream@@_JH@Z 00000001800440f4 f   libucrt:fseek.obj
 0001:00043160       ?common_fseek_binary_mode_read_only_fast_track_nolock@@YA_NV__crt_stdio_stream@@_JH@Z 0000000180044160 f   libucrt:fseek.obj
 0001:00043240       ?common_fseek_nolock@@YAHV__crt_stdio_stream@@_JH@Z 0000000180044240 f   libucrt:fseek.obj
 0001:00043314       ??$common_ftell@J@@YAJV__crt_stdio_stream@@@Z 0000000180044314 f   libucrt:ftell.obj
 0001:00043384       ??$common_ftell_nolock@_J@@YA_JV__crt_stdio_stream@@@Z 0000000180044384 f   libucrt:ftell.obj
 0001:000434c0       ?common_ftell_read_mode_nolock@@YA_JV__crt_stdio_stream@@_J1@Z 00000001800444c0 f   libucrt:ftell.obj
 0001:0004360c       ?common_ftell_translated_utf8_nolock@@YA_JV__crt_stdio_stream@@_J@Z 000000018004460c f   libucrt:ftell.obj
 0001:00043788       ?count_newline_bytes@@YA_JQEBD0W4__crt_lowio_text_mode@@@Z 0000000180044788 f   libucrt:ftell.obj
 0001:00043824       ??$?RV<lambda_bdbcead8b570fa3d5ec6d9679862a6e5>@@AEAV<lambda_96f4279ff90247a4c5c5d9824f56f8c1>@@V<lambda_4606be27f17b5e5579e09050fab91818>@@@?$__crt_seh_guarded_call@_K@@QEAA_K$$QEAV<lambda_bdbcead8b570fa3d5ec6d9679862a6e5>@@AEAV<lambda_96f4279ff90247a4c5c5d9824f56f8c1>@@$$QEAV<lambda_4606be27f17b5e5579e09050fab91818>@@@Z 0000000180044824 f   libucrt:fwrite.obj
 0001:00043864       ??R<lambda_96f4279ff90247a4c5c5d9824f56f8c1>@@QEBA_KXZ 0000000180044864 f   libucrt:fwrite.obj
 0001:00043ae4       ??$?RV<lambda_84ec643ea9557e2f7dc01bb0e9624395>@@AEAV<lambda_ca71763b3c0644891230e4f79ea54fa6>@@V<lambda_439a761618c59b0600e24586724d733b>@@@?$__crt_seh_guarded_call@H@@QEAAH$$QEAV<lambda_84ec643ea9557e2f7dc01bb0e9624395>@@AEAV<lambda_ca71763b3c0644891230e4f79ea54fa6>@@$$QEAV<lambda_439a761618c59b0600e24586724d733b>@@@Z 0000000180044ae4 f   libucrt:setvbuf.obj
 0001:00043b24       ??R<lambda_ca71763b3c0644891230e4f79ea54fa6>@@QEBAHXZ 0000000180044b24 f   libucrt:setvbuf.obj
 0001:00043cb0       ??$generate_tmpfile_file_name@D@@YA_NQEAD_K@Z 0000000180044cb0 f   libucrt:tmpfile.obj
 0001:00043d4c       ??$get_tmpfile_buffer_nolock@D@@YAPEADW4buffer_id@?A0x5b9a7937@@@Z 0000000180044d4c f   libucrt:tmpfile.obj
 0001:00043d90       ??$initialize_tmpfile_buffer_nolock@D@@YA_NW4buffer_id@?A0x5b9a7937@@@Z 0000000180044d90 f   libucrt:tmpfile.obj
 0001:00043e54       ?common_tmpfile@@YAHQEAPEAU_iobuf@@H@Z 0000000180044e54 f   libucrt:tmpfile.obj
 0001:00043ebc       ?common_tmpfile_nolock@@YAHQEAPEAU_iobuf@@H@Z 0000000180044ebc f   libucrt:tmpfile.obj
 0001:000440ec       ??$?RV<lambda_082dd7c0feb7dbdaf245f261e54a6583>@@AEAV<lambda_f3caf1ecae5fe01a9a1a6239afa44510>@@V<lambda_c640b76c0755ae85b317b35c67c61e6b>@@@?$__crt_seh_guarded_call@H@@QEAAH$$QEAV<lambda_082dd7c0feb7dbdaf245f261e54a6583>@@AEAV<lambda_f3caf1ecae5fe01a9a1a6239afa44510>@@$$QEAV<lambda_c640b76c0755ae85b317b35c67c61e6b>@@@Z 00000001800450ec f   libucrt:input.obj
 0001:00045c98       ??R<lambda_156378f40168adef48d7ddfcff3a1264>@@QEBA_NXZ 0000000180046c98 f   libucrt:input.obj
 0001:00045d10       ??R<lambda_f3caf1ecae5fe01a9a1a6239afa44510>@@QEBAHXZ 0000000180046d10 f   libucrt:input.obj
 0001:000494b0       memcpy_s                   000000018004a4b0 f   libucrt:input.obj
 0001:000494b0       memcpy_s                   000000018004a4b0 f   libucrt:cfout.obj
 0001:00049538       ??$common_dupenv_s@_W@@YAHQEAPEA_WQEA_KQEB_WHQEBDH@Z 000000018004a538 f   libucrt:getenv.obj
 0001:0004962c       ??$common_getenv@_W@@YAPEA_WQEB_W@Z 000000018004a62c f   libucrt:getenv.obj
 0001:0004968c       ??$common_getenv_nolock@_W@@YAPEA_WQEB_W@Z 000000018004a68c f   libucrt:getenv.obj
 0001:00049b04       ??$?RV<lambda_d80eeec6fff315bfe5c115232f3240e3>@@AEAV<lambda_6e4b09c48022b2350581041d5f6b0c4c>@@V<lambda_2358e3775559c9db80273638284d5e45>@@@?$__crt_seh_guarded_call@X@@QEAAX$$QEAV<lambda_d80eeec6fff315bfe5c115232f3240e3>@@AEAV<lambda_6e4b09c48022b2350581041d5f6b0c4c>@@$$QEAV<lambda_2358e3775559c9db80273638284d5e45>@@@Z 000000018004ab04 f   libucrt:exit.obj
 0001:00049b3c       ??R<lambda_6e4b09c48022b2350581041d5f6b0c4c>@@QEBA@XZ 000000018004ab3c f   libucrt:exit.obj
 0001:00049c14       ?atexit_exception_filter@@YAHK@Z 000000018004ac14 f   libucrt:exit.obj
 0001:00049c20       ?common_exit@@YAXHW4_crt_exit_cleanup_mode@@W4_crt_exit_return_mode@@@Z 000000018004ac20 f   libucrt:exit.obj
 0001:00049cdc       ?exit_or_terminate_process@@YAXI@Z 000000018004acdc f   libucrt:exit.obj
 0001:00049d28       ?try_cor_exit_process@@YAXI@Z 000000018004ad28 f   libucrt:exit.obj
 0001:00049db0       ??$parse_command_line@D@@YAXPEADPEAPEAD0PEA_K2@Z 000000018004adb0 f   libucrt:argv_parsing.obj
 0001:0004a154       ??$common_initialize_environment_nolock@D@@YAHXZ 000000018004b154 f   libucrt:environment_initialization.obj
 0001:0004a1c0       ??$common_initialize_environment_nolock@_W@@YAHXZ 000000018004b1c0 f   libucrt:environment_initialization.obj
 0001:0004a228       ??$create_environment@D@@YAQEAPEADQEAD@Z 000000018004b228 f   libucrt:environment_initialization.obj
 0001:0004a334       ??$create_environment@_W@@YAQEAPEA_WQEA_W@Z 000000018004b334 f   libucrt:environment_initialization.obj
 0001:0004a44c       ??$free_environment@_W@@YAXQEAPEA_W@Z 000000018004b44c f   libucrt:environment_initialization.obj
 0001:0004a44c       ??$free_environment@D@@YAXQEAPEAD@Z 000000018004b44c f   libucrt:environment_initialization.obj
 0001:0004a490       ??$initialize_environment_by_cloning_nolock@_W@@YAHXZ 000000018004b490 f   libucrt:environment_initialization.obj
 0001:0004a540       ??$uninitialize_environment_internal@D@@YAXAEAPEAPEAD@Z 000000018004b540 f   libucrt:environment_initialization.obj
 0001:0004a55c       ??$uninitialize_environment_internal@_W@@YAXAEAPEAPEA_W@Z 000000018004b55c f   libucrt:environment_initialization.obj
 0001:0004a5f4       ??$?RV<lambda_7777bce6b2f8c936911f934f8298dc43>@@AEAV<lambda_f03950bc5685219e0bcd2087efbe011e>@@V<lambda_3883c3dff614d5e0c5f61bb1ac94921c>@@@?$__crt_seh_guarded_call@H@@QEAAH$$QEAV<lambda_7777bce6b2f8c936911f934f8298dc43>@@AEAV<lambda_f03950bc5685219e0bcd2087efbe011e>@@$$QEAV<lambda_3883c3dff614d5e0c5f61bb1ac94921c>@@@Z 000000018004b5f4 f   libucrt:onexit.obj
 0001:0004a630       ??R<lambda_f03950bc5685219e0bcd2087efbe011e>@@QEBAHXZ 000000018004b630 f   libucrt:onexit.obj
 0001:0004a7f8       initialize_global_variables 000000018004b7f8 f   libucrt:initialization.obj
 0001:0004a80c       initialize_c               000000018004b80c f   libucrt:initialization.obj
 0001:0004a830       initialize_environment     000000018004b830 f   libucrt:initialization.obj
 0001:0004a830       initialize_global_state_isolation 000000018004b830 f   libucrt:initialization.obj
 0001:0004a830       report_memory_leaks        000000018004b830 f   libucrt:initialization.obj
 0001:0004a830       uninitialize_c             000000018004b830 f   libucrt:initialization.obj
 0001:0004a830       uninitialize_global_state_isolation 000000018004b830 f   libucrt:initialization.obj
 0001:0004a834       uninitialize_environment   000000018004b834 f   libucrt:initialization.obj
 0001:0004a844       initialize_pointers        000000018004b844 f   libucrt:initialization.obj
 0001:0004a898       uninitialize_vcruntime     000000018004b898 f   libucrt:initialization.obj
 0001:0004a8a0       uninitialize_allocated_memory 000000018004b8a0 f   libucrt:initialization.obj
 0001:0004a8e0       uninitialize_allocated_io_buffers 000000018004b8e0 f   libucrt:initialization.obj
 0001:0004a9dc       ?_strupr_s_l_stat@@YAHQEAD_KQEAU__crt_locale_pointers@@@Z 000000018004b9dc f   libucrt:strupr.obj
 0001:0004bcec       ?internal_isupper_l@@YA_NHQEAU__crt_locale_pointers@@@Z 000000018004ccec f   libucrt:tolower_toupper.obj
 0001:0004c5b4       ??$?RV<lambda_0ae27a3a962d80f24befdcbee591983d>@@AEAV<lambda_8d0ee55de4b1038c4002e0adecdf1839>@@V<lambda_dc504788e8f1664fe9b84e20bfb512f2>@@@?$__crt_seh_guarded_call@X@@QEAAX$$QEAV<lambda_0ae27a3a962d80f24befdcbee591983d>@@AEAV<lambda_8d0ee55de4b1038c4002e0adecdf1839>@@$$QEAV<lambda_dc504788e8f1664fe9b84e20bfb512f2>@@@Z 000000018004d5b4 f   libucrt:per_thread_data.obj
 0001:0004c5f4       ??$?RV<lambda_2d41944a1d46af3157314b8a01080d33>@@AEAV<lambda_8f455de75cd7d7f24b4096f044d8b9e6>@@V<lambda_aa500f224e6afead328df44964fe2772>@@@?$__crt_seh_guarded_call@X@@QEAAX$$QEAV<lambda_2d41944a1d46af3157314b8a01080d33>@@AEAV<lambda_8f455de75cd7d7f24b4096f044d8b9e6>@@$$QEAV<lambda_aa500f224e6afead328df44964fe2772>@@@Z 000000018004d5f4 f   libucrt:per_thread_data.obj
 0001:0004c634       ??$?RV<lambda_aa87e3671a710a21b5dc78c0bdf72e11>@@AEAV<lambda_92619d2358a28f41a33ba319515a20b9>@@V<lambda_6992ecaafeb10aed2b74cb1fae11a551>@@@?$__crt_seh_guarded_call@X@@QEAAX$$QEAV<lambda_aa87e3671a710a21b5dc78c0bdf72e11>@@AEAV<lambda_92619d2358a28f41a33ba319515a20b9>@@$$QEAV<lambda_6992ecaafeb10aed2b74cb1fae11a551>@@@Z 000000018004d634 f   libucrt:per_thread_data.obj
 0001:0004c67c       ??$?RV<lambda_f2e299630e499de9f9a165e60fcd3db5>@@AEAV<lambda_2ae9d31cdba2644fcbeaf08da7c24588>@@V<lambda_40d01ff24d0e7b3814fdbdcee8eab3c7>@@@?$__crt_seh_guarded_call@X@@QEAAX$$QEAV<lambda_f2e299630e499de9f9a165e60fcd3db5>@@AEAV<lambda_2ae9d31cdba2644fcbeaf08da7c24588>@@$$QEAV<lambda_40d01ff24d0e7b3814fdbdcee8eab3c7>@@@Z 000000018004d67c f   libucrt:per_thread_data.obj
 0001:0004c6dc       ?construct_ptd_array@@YAXQEAU__acrt_ptd@@@Z 000000018004d6dc f   libucrt:per_thread_data.obj
 0001:0004c7ac       ?destroy_fls@@YAXPEAX@Z    000000018004d7ac f   libucrt:per_thread_data.obj
 0001:0004c7cc       ?destroy_ptd_array@@YAXQEAU__acrt_ptd@@@Z 000000018004d7cc f   libucrt:per_thread_data.obj
 0001:0004c8c4       ?replace_current_thread_locale_nolock@@YAXQEAU__acrt_ptd@@QEAU__crt_locale_data@@@Z 000000018004d8c4 f   libucrt:per_thread_data.obj
 0001:0004cc7c       ?fp_format_a@@YAHQEBNPEAD_KQEAD2H_NIQEAU__crt_locale_pointers@@@Z 000000018004dc7c f   libucrt:cvt.obj
 0001:0004cfd0       ?fp_format_e@@YAHQEBNQEAD_K12H_NIQEAU__crt_locale_pointers@@@Z 000000018004dfd0 f   libucrt:cvt.obj
 0001:0004d0ac       ?fp_format_e_internal@@YAHQEAD_KH_NIQEAU_strflt@@2QEAU__crt_locale_pointers@@@Z 000000018004e0ac f   libucrt:cvt.obj
 0001:0004d280       ?fp_format_f_internal@@YAHQEAD_KHQEAU_strflt@@_NQEAU__crt_locale_pointers@@@Z 000000018004e280 f   libucrt:cvt.obj
 0001:0004d3c8       ?fp_format_g@@YAHQEBNQEAD_K12H_NIQEAU__crt_locale_pointers@@@Z 000000018004e3c8 f   libucrt:cvt.obj
 0001:0004d4fc       ?fp_format_nan_or_infinity@@YAHW4__acrt_fp_class@@_NPEAD_K1@Z 000000018004e4fc f   libucrt:cvt.obj
 0001:0004da24       ??$?RV<lambda_410d79af7f07d98d83a3f525b3859a53>@@AEAV<lambda_3e16ef9562a7dcce91392c22ab16ea36>@@V<lambda_38119f0e861e05405d8a144b9b982f0a>@@@?$__crt_seh_guarded_call@X@@QEAAX$$QEAV<lambda_410d79af7f07d98d83a3f525b3859a53>@@AEAV<lambda_3e16ef9562a7dcce91392c22ab16ea36>@@$$QEAV<lambda_38119f0e861e05405d8a144b9b982f0a>@@@Z 000000018004ea24 f   libucrt:wsetlocale.obj
 0001:0004dad0       ?initialize_inherited_file_handles_nolock@@YAXXZ 000000018004ead0 f   libucrt:ioinit.obj
 0001:0004dbbc       ?initialize_stdio_handles_nolock@@YAXXZ 000000018004ebbc f   libucrt:ioinit.obj
 0001:0004de10       ?find_or_allocate_unused_stream_nolock@@YA?AV__crt_stdio_stream@@XZ 000000018004ee10 f   libucrt:stream.obj
 0001:0004e278       ??$?RV<lambda_751a882b2c74d4b022dec766aa51a29a>@@AEAV<lambda_628dfdc04ba53c8bfc02c9951375f3f5>@@V<lambda_f6c7be5f7998530c34de24c7437d6b54>@@@?$__crt_seh_guarded_call@H@@QEAAH$$QEAV<lambda_751a882b2c74d4b022dec766aa51a29a>@@AEAV<lambda_628dfdc04ba53c8bfc02c9951375f3f5>@@$$QEAV<lambda_f6c7be5f7998530c34de24c7437d6b54>@@@Z 000000018004f278 f   libucrt:close.obj
 0001:0004e490       $$000000                   000000018004f490     libucrt:fpsr.obj
 0001:0004e64c       ?try_get_function@@YAPEAXW4function_id@?A0x391cf84c@@QEBDQEBW4module_id@2@2@Z 000000018004f64c f   libucrt:winapi_thunks.obj
 0001:0004ed88       ??$translate_text_mode_nolock@D@@YAHHQEAD_K@Z 000000018004fd88 f   libucrt:read.obj
 0001:0004ef44       ??$translate_text_mode_nolock@_W@@YAHHQEA_W_K@Z 000000018004ff44 f   libucrt:read.obj
 0001:0004f17c       ?translate_ansi_or_utf8_nolock@@YAHHQEAD_KQEA_W1@Z 000000018005017c f   libucrt:read.obj
 0001:0004fa2c       ??$common_lseek@J@@YAJHJH@Z 0000000180050a2c f   libucrt:lseek.obj
 0001:0004fb18       ??$common_lseek@_J@@YA_JH_JH@Z 0000000180050b18 f   libucrt:lseek.obj
 0001:0004fc08       ??$common_lseek_nolock@J@@YAJHJH@Z 0000000180050c08 f   libucrt:lseek.obj
 0001:0004fcfc       ??$common_lseek_nolock@_J@@YA_JH_JH@Z 0000000180050cfc f   libucrt:lseek.obj
 0001:000506c4       ??$common_fdopen@_W@@YAPEAU_iobuf@@HQEB_W@Z 00000001800516c4 f   libucrt:fdopen.obj
 0001:000507b8       ??$?RV<lambda_a37b2b86f63e897a80ea819b0eb08c01>@@AEAV<lambda_38ce7e780aa69e748d6df282ebc68efe>@@V<lambda_99fb1378e971ab6e7edea83e3a7a83a2>@@@?$__crt_seh_guarded_call@H@@QEAAH$$QEAV<lambda_a37b2b86f63e897a80ea819b0eb08c01>@@AEAV<lambda_38ce7e780aa69e748d6df282ebc68efe>@@$$QEAV<lambda_99fb1378e971ab6e7edea83e3a7a83a2>@@@Z 00000001800517b8 f   libucrt:commit.obj
 0001:000508d8       ?write_double_translated_ansi_nolock@@YA?AUwrite_result@?A0x17268360@@HQEBDI@Z 00000001800518d8 f   libucrt:write.obj
 0001:00050afc       ?write_text_ansi_nolock@@YA?AUwrite_result@?A0x17268360@@HQEBDI@Z 0000000180051afc f   libucrt:write.obj
 0001:00050c00       ?write_text_utf16le_nolock@@YA?AUwrite_result@?A0x17268360@@HQEBDI@Z 0000000180051c00 f   libucrt:write.obj
 0001:00050d1c       ?write_text_utf8_nolock@@YA?AUwrite_result@?A0x17268360@@HQEBDI@Z 0000000180051d1c f   libucrt:write.obj
 0001:000512c0       ??$write_buffer_nolock@D@@YA_NDV__crt_stdio_stream@@@Z 00000001800522c0 f   libucrt:_flsbuf.obj
 0001:00051488       ??$common_xtox@_KD@@YAH_KQEAD0I_N@Z 0000000180052488 f   libucrt:xtoa.obj
 0001:00051520       ??$common_xtox_s@_KD@@YAH_KQEAD0I_N@Z 0000000180052520 f   libucrt:xtoa.obj
 0001:000516bc       ??$common_sopen_dispatch@D@@YAHQEBDHHHQEAHH@Z 00000001800526bc f   libucrt:open.obj
 0001:00051780       ??$common_sopen_dispatch@_W@@YAHQEB_WHHHQEAHH@Z 0000000180052780 f   libucrt:open.obj
 0001:00051844       ?configure_text_mode@@YAHHUfile_options@?A0xa9d50aae@@HAEAW4__crt_lowio_text_mode@@@Z 0000000180052844 f   libucrt:open.obj
 0001:00051ad8       ?decode_options@@YA?AUfile_options@?A0xa9d50aae@@HHH@Z 0000000180052ad8 f   libucrt:open.obj
 0001:00051ce0       ?truncate_ctrl_z_if_present@@YAHH@Z 0000000180052ce0 f   libucrt:open.obj
 0001:0005250c       ??$?RV<lambda_a22f0c497e5168315e06dae667770027>@@AEAV<lambda_a094494068278ba5130ab06e1292f60a>@@V<lambda_24dc10c13f43218c635520766e23e324>@@@?$__crt_seh_guarded_call@_N@@QEAA_N$$QEAV<lambda_a22f0c497e5168315e06dae667770027>@@AEAV<lambda_a094494068278ba5130ab06e1292f60a>@@$$QEAV<lambda_24dc10c13f43218c635520766e23e324>@@@Z 000000018005350c f   libucrt:spawnv.obj
 0001:0005254c       ??$common_spawnv@_W@@YA_JHQEB_WQEBQEB_W1@Z 000000018005354c f   libucrt:spawnv.obj
 0001:000527e0       ??$execute_command@_W@@YA_JHQEB_WQEBQEB_W1@Z 00000001800537e0 f   libucrt:spawnv.obj
 0001:00052a3c       ??R<lambda_a094494068278ba5130ab06e1292f60a>@@QEBA_NXZ 0000000180053a3c f   libucrt:spawnv.obj
 0001:00052c34       ?accumulate_inheritable_handles@@YA_NQEAPEAEQEA_K_N@Z 0000000180053c34 f   libucrt:spawnv.obj
 0001:00052c94       ??$common_spawnvp@_W@@YA_JHQEB_WQEBQEB_W1@Z 0000000180053c94 f   libucrt:spawnvp.obj
 0001:00053014       ?<lambda_invoker_cdecl>@<lambda_c2303d2482d7c3675ea2e24c4cfb6115>@@CAHPEBX0@Z 0000000180054014 f   libucrt:argv_wildcards.obj
 0001:00053028       ??$common_expand_argv_wildcards@D@@YAHQEAPEADQEAPEAPEAD@Z 0000000180054028 f   libucrt:argv_wildcards.obj
 0001:00053234       ??$copy_and_add_argument_to_buffer@D@@YAHQEBD0_KAEAV?$argument_list@D@?A0x5f5c8891@@@Z 0000000180054234 f   libucrt:argv_wildcards.obj
 0001:000533cc       ??$expand_argument_wildcards@D@@YAHQEAD0AEAV?$argument_list@D@?A0x5f5c8891@@@Z 00000001800543cc f   libucrt:argv_wildcards.obj
 0001:00053580       ??$?RV<lambda_efdfa57d1f175319df784efa44bb7b81>@@AEAV<lambda_5f0a4c1567f8adc6734073e5d1e1b35c>@@V<lambda_2e8a7d3640ea6ccb4c2413664c2db6fd>@@@?$__crt_seh_guarded_call@X@@QEAAX$$QEAV<lambda_efdfa57d1f175319df784efa44bb7b81>@@AEAV<lambda_5f0a4c1567f8adc6734073e5d1e1b35c>@@$$QEAV<lambda_2e8a7d3640ea6ccb4c2413664c2db6fd>@@@Z 0000000180054580 f   libucrt:mbctype.obj
 0001:00053754       ?getSystemCP@@YAHH@Z       0000000180054754 f   libucrt:mbctype.obj
 0001:000537d4       ?setSBCS@@YAXPEAU__crt_multibyte_data@@@Z 00000001800547d4 f   libucrt:mbctype.obj
 0001:00053864       ?setSBUpLow@@YAXPEAU__crt_multibyte_data@@@Z 0000000180054864 f   libucrt:mbctype.obj
 0001:00053a44       ?setmbcp_internal@@YAHH_NQEAU__acrt_ptd@@QEAPEAU__crt_multibyte_data@@@Z 0000000180054a44 f   libucrt:mbctype.obj
 0001:00053c08       ?update_thread_multibyte_data_internal@@YAPEAU__crt_multibyte_data@@QEAU__acrt_ptd@@QEAPEAU1@@Z 0000000180054c08 f   libucrt:mbctype.obj
 0001:00053ffc       ?x_ismbbtype_l@@YAHPEAU__crt_locale_pointers@@IHH@Z 0000000180054ffc f   libucrt:ismbbyte.obj
 0001:00054254       ??$common_set_variable_in_environment_nolock@_W@@YAHQEA_WH@Z 0000000180055254 f   libucrt:setenv.obj
 0001:00054574       ??$copy_environment@_W@@YAPEAPEA_WQEAPEA_W@Z 0000000180055574 f   libucrt:setenv.obj
 0001:000547c0       ??$?RV<lambda_450d765d439847d4c735a33c368b5fc0>@@AEAV<lambda_44731a7d0e6d81c3e6aa82d741081786>@@V<lambda_601a2a7da3b7a96e9554ac7215c4b07c>@@@?$__crt_seh_guarded_call@P6AXH@Z@@QEAAP6AXH@Z$$QEAV<lambda_450d765d439847d4c735a33c368b5fc0>@@AEAV<lambda_44731a7d0e6d81c3e6aa82d741081786>@@$$QEAV<lambda_601a2a7da3b7a96e9554ac7215c4b07c>@@@Z 00000001800557c0 f   libucrt:signal.obj
 0001:00054b24       ?__acrt_LCMapStringA_stat@@YAHPEAU__crt_locale_pointers@@PEB_WKPEBDHPEADHHH@Z 0000000180055b24 f   libucrt:lcmapstringa.obj
 0001:00056924       ?free_crt_array_internal@@YAXQEAPEBX_K@Z 0000000180057924 f   libucrt:inittime.obj
 0001:000572b0       ?GetTableIndexFromLocaleName@@YAHPEB_W@Z 00000001800582b0 f   libucrt:lcidtoname_downlevel.obj
 0001:00057ca8       ??$construct_environment_block@_W@@YAHQEBQEB_WQEAPEA_W@Z 0000000180058ca8 f   libucrt:cenvarg.obj
 0001:000585c8       ?initialize_multibyte@@YAHXZ 00000001800595c8 f   libucrt:multibyte_initializer.obj
 0001:00058780       $$000000                   0000000180059780     libucrt:log10.obj
 0001:00058e64       _call_matherr              0000000180059e64 f   libucrt:libm_error.obj
 0001:00058ecc       _exception_enabled         0000000180059ecc f   libucrt:libm_error.obj
 0001:00059160       _log_special_common        000000018005a160 f   libucrt:log_special.obj
 0001:00059790       $$000000                   000000018005a790     LIBCMT:_amdsecgs_.obj
 0001:0005997c       capture_current_context    000000018005a97c f   LIBCMT:gs_report.obj
 0001:000599ec       capture_previous_context   000000018005a9ec f   LIBCMT:gs_report.obj
 0001:00059af0       $$000000                   000000018005aaf0     LIBCMT:_guard_dispatch_.obj
 0001:00059b10       ?fin$0@?0??dllmain_crt_process_attach@@YAHQEAUHINSTANCE__@@QEAX@Z@4HA 000000018005ab10 f   LIBCMT:dll_dllmain.obj
 0001:00059b27       ?fin$0@?0??dllmain_crt_process_detach@@YAH_N@Z@4HA 000000018005ab27 f   LIBCMT:dll_dllmain.obj
 0001:00059b43       ?filt$0@?0??dllmain_dispatch@@YAHQEAUHINSTANCE__@@KQEAX@Z@4HA 000000018005ab43 f   LIBCMT:dll_dllmain.obj
 0001:00059b79       __scrt_is_nonwritable_in_current_image$filt$0 000000018005ab79 f   LIBCMT:utility.obj
 0001:00059b91       __DestructExceptionObject$filt$0 000000018005ab91 f   libvcruntime:ehhelpers.obj
 0001:00059ba9       ?fin$0@?0???$?RV<lambda_082dd7c0feb7dbdaf245f261e54a6583>@@AEAV<lambda_f3caf1ecae5fe01a9a1a6239afa44510>@@V<lambda_c640b76c0755ae85b317b35c67c61e6b>@@@?$__crt_seh_guarded_call@H@@QEAAH$$QEAV<lambda_082dd7c0feb7dbdaf245f261e54a6583>@@AEAV<lambda_f3caf1ecae5fe01a9a1a6239afa44510>@@$$QEAV<lambda_c640b76c0755ae85b317b35c67c61e6b>@@@Z@4HA 000000018005aba9 f   libucrt:input.obj
 0001:00059ba9       ?fin$0@?0???$?RV<lambda_a62c933ada0517137acf5807a1eeac1f>@@AEAV<lambda_a31071773b9a94e445cbd5d04ef99106>@@V<lambda_56065050dbf3ada7e59a83db45153de3>@@@?$__crt_seh_guarded_call@H@@QEAAH$$QEAV<lambda_a62c933ada0517137acf5807a1eeac1f>@@AEAV<lambda_a31071773b9a94e445cbd5d04ef99106>@@$$QEAV<lambda_56065050dbf3ada7e59a83db45153de3>@@@Z@4HA 000000018005aba9 f   libucrt:output.obj
 0001:00059ba9       ?fin$0@?0???$?RV<lambda_84ec643ea9557e2f7dc01bb0e9624395>@@AEAV<lambda_ca71763b3c0644891230e4f79ea54fa6>@@V<lambda_439a761618c59b0600e24586724d733b>@@@?$__crt_seh_guarded_call@H@@QEAAH$$QEAV<lambda_84ec643ea9557e2f7dc01bb0e9624395>@@AEAV<lambda_ca71763b3c0644891230e4f79ea54fa6>@@$$QEAV<lambda_439a761618c59b0600e24586724d733b>@@@Z@4HA 000000018005aba9 f   libucrt:setvbuf.obj
 0001:00059ba9       ?fin$0@?0???$?RV<lambda_842d9ff0dc9ef11c61343bbaebe7f885>@@AEAV<lambda_c5860995281e5c4ce005b3de8f5874ee>@@V<lambda_d90129c13df834fdcbf8d2b88dafcf2d>@@@?$__crt_seh_guarded_call@X@@QEAAX$$QEAV<lambda_842d9ff0dc9ef11c61343bbaebe7f885>@@AEAV<lambda_c5860995281e5c4ce005b3de8f5874ee>@@$$QEAV<lambda_d90129c13df834fdcbf8d2b88dafcf2d>@@@Z@4HA 000000018005aba9 f   libucrt:fflush.obj
 0001:00059ba9       ?fin$0@?0???$?RV<lambda_bdbcead8b570fa3d5ec6d9679862a6e5>@@AEAV<lambda_96f4279ff90247a4c5c5d9824f56f8c1>@@V<lambda_4606be27f17b5e5579e09050fab91818>@@@?$__crt_seh_guarded_call@_K@@QEAA_K$$QEAV<lambda_bdbcead8b570fa3d5ec6d9679862a6e5>@@AEAV<lambda_96f4279ff90247a4c5c5d9824f56f8c1>@@$$QEAV<lambda_4606be27f17b5e5579e09050fab91818>@@@Z@4HA 000000018005aba9 f   libucrt:fwrite.obj
 0001:00059ba9       ?fin$0@?0???$?RV<lambda_c376a267cfb53b6959b3b692ec76b120>@@AEAV<lambda_9a32fed5bf61b6b509b2d3f6003082a1>@@V<lambda_572fbb9fa0ab338edf41edfd4b5fcc8d>@@@?$__crt_seh_guarded_call@H@@QEAAH$$QEAV<lambda_c376a267cfb53b6959b3b692ec76b120>@@AEAV<lambda_9a32fed5bf61b6b509b2d3f6003082a1>@@$$QEAV<lambda_572fbb9fa0ab338edf41edfd4b5fcc8d>@@@Z@4HA 000000018005aba9 f   libucrt:fflush.obj
 0001:00059bc4       ?fin$0@?0???$common_fsopen@_W@@YAPEAU_iobuf@@QEB_W0H@Z@4HA 000000018005abc4 f   libucrt:fopen.obj
 0001:00059bef       clearerr_s$fin$0           000000018005abef f   libucrt:clearerr.obj
 0001:00059bef       ?fin$0@?0???$common_ftell@J@@YAJV__crt_stdio_stream@@@Z@4HA 000000018005abef f   libucrt:ftell.obj
 0001:00059bef       rewind$fin$0               000000018005abef f   libucrt:rewind.obj
 0001:00059bef       ?fin$0@?0??common_fseek@@YAHV__crt_stdio_stream@@_JH@Z@4HA 000000018005abef f   libucrt:fseek.obj
 0001:00059bef       fclose$fin$0               000000018005abef f   libucrt:fclose.obj
 0001:00059c07       _ctrlfp$filt$0             000000018005ac07 f   libucrt:fpctrl.obj
 0001:00059c07       common_control87$filt$0    000000018005ac07 f   libucrt:ieee.obj
 0001:00059c33       ?fin$0@?0???$common_freopen@_W@@YAHQEAPEAU_iobuf@@QEB_W1V__crt_stdio_stream@@H@Z@4HA 000000018005ac33 f   libucrt:freopen.obj
 0001:00059c4b       fread_s$fin$0              000000018005ac4b f   libucrt:fread.obj
 0001:00059c63       fgetc$fin$0                000000018005ac63 f   libucrt:fgetc.obj
 0001:00059c7d       ungetc$fin$0               000000018005ac7d f   libucrt:ungetc.obj
 0001:00059c95       ?fin$0@?0???$common_popen@_W@@YAPEAU_iobuf@@QEB_W0@Z@4HA 000000018005ac95 f   libucrt:popen.obj
 0001:00059cb0       _pclose$fin$0              000000018005acb0 f   libucrt:popen.obj
 0001:00059cc9       ?fin$0@?0???$?RV<lambda_886d6c58226a84441f68b9f2b8217b83>@@AEAV<lambda_ab61a845afdef5b7c387490eaf3616ee>@@V<lambda_f7f22ab5edc0698d5f6905b0d3f44752>@@@?$__crt_seh_guarded_call@X@@QEAAX$$QEAV<lambda_886d6c58226a84441f68b9f2b8217b83>@@AEAV<lambda_ab61a845afdef5b7c387490eaf3616ee>@@$$QEAV<lambda_f7f22ab5edc0698d5f6905b0d3f44752>@@@Z@4HA 000000018005acc9 f   libucrt:fflush.obj
 0001:00059ce6       ?fin$0@?0???$common_fgets@D@@YAPEADQEADHV__crt_stdio_stream@@@Z@4HA 000000018005ace6 f   libucrt:fgets.obj
 0001:00059cfe       ?fin$0@?0??common_tmpfile@@YAHQEAPEAU_iobuf@@H@Z@4HA 000000018005acfe f   libucrt:tmpfile.obj
 0001:00059d17       ?fin$0@?0??common_tmpfile_nolock@@YAHQEAPEAU_iobuf@@H@Z@4HA 000000018005ad17 f   libucrt:tmpfile.obj
 0001:00059d40       ?fin$0@?0???$common_dupenv_s@_W@@YAHQEAPEA_WQEA_KQEB_WHQEBDH@Z@4HA 000000018005ad40 f   libucrt:getenv.obj
 0001:00059d59       ?fin$0@?0???$common_getenv@_W@@YAPEA_WQEB_W@Z@4HA 000000018005ad59 f   libucrt:getenv.obj
 0001:00059d72       ?fin$0@?0???$?RV<lambda_f2e299630e499de9f9a165e60fcd3db5>@@AEAV<lambda_2ae9d31cdba2644fcbeaf08da7c24588>@@V<lambda_40d01ff24d0e7b3814fdbdcee8eab3c7>@@@?$__crt_seh_guarded_call@X@@QEAAX$$QEAV<lambda_f2e299630e499de9f9a165e60fcd3db5>@@AEAV<lambda_2ae9d31cdba2644fcbeaf08da7c24588>@@$$QEAV<lambda_40d01ff24d0e7b3814fdbdcee8eab3c7>@@@Z@4HA 000000018005ad72 f   libucrt:per_thread_data.obj
 0001:00059d72       ?fin$0@?0???$?RV<lambda_2d41944a1d46af3157314b8a01080d33>@@AEAV<lambda_8f455de75cd7d7f24b4096f044d8b9e6>@@V<lambda_aa500f224e6afead328df44964fe2772>@@@?$__crt_seh_guarded_call@X@@QEAAX$$QEAV<lambda_2d41944a1d46af3157314b8a01080d33>@@AEAV<lambda_8f455de75cd7d7f24b4096f044d8b9e6>@@$$QEAV<lambda_aa500f224e6afead328df44964fe2772>@@@Z@4HA 000000018005ad72 f   libucrt:per_thread_data.obj
 0001:00059d72       ?fin$0@?0???$?RV<lambda_7777bce6b2f8c936911f934f8298dc43>@@AEAV<lambda_f03950bc5685219e0bcd2087efbe011e>@@V<lambda_3883c3dff614d5e0c5f61bb1ac94921c>@@@?$__crt_seh_guarded_call@H@@QEAAH$$QEAV<lambda_7777bce6b2f8c936911f934f8298dc43>@@AEAV<lambda_f03950bc5685219e0bcd2087efbe011e>@@$$QEAV<lambda_3883c3dff614d5e0c5f61bb1ac94921c>@@@Z@4HA 000000018005ad72 f   libucrt:onexit.obj
 0001:00059d72       ?fin$0@?0???$?RV<lambda_450d765d439847d4c735a33c368b5fc0>@@AEAV<lambda_44731a7d0e6d81c3e6aa82d741081786>@@V<lambda_601a2a7da3b7a96e9554ac7215c4b07c>@@@?$__crt_seh_guarded_call@P6AXH@Z@@QEAAP6AXH@Z$$QEAV<lambda_450d765d439847d4c735a33c368b5fc0>@@AEAV<lambda_44731a7d0e6d81c3e6aa82d741081786>@@$$QEAV<lambda_601a2a7da3b7a96e9554ac7215c4b07c>@@@Z@4HA 000000018005ad72 f   libucrt:signal.obj
 0001:00059d72       ?fin$0@?0???$?RV<lambda_efdfa57d1f175319df784efa44bb7b81>@@AEAV<lambda_5f0a4c1567f8adc6734073e5d1e1b35c>@@V<lambda_2e8a7d3640ea6ccb4c2413664c2db6fd>@@@?$__crt_seh_guarded_call@X@@QEAAX$$QEAV<lambda_efdfa57d1f175319df784efa44bb7b81>@@AEAV<lambda_5f0a4c1567f8adc6734073e5d1e1b35c>@@$$QEAV<lambda_2e8a7d3640ea6ccb4c2413664c2db6fd>@@@Z@4HA 000000018005ad72 f   libucrt:mbctype.obj
 0001:00059d72       ?fin$0@?0???$?RV<lambda_d80eeec6fff315bfe5c115232f3240e3>@@AEAV<lambda_6e4b09c48022b2350581041d5f6b0c4c>@@V<lambda_2358e3775559c9db80273638284d5e45>@@@?$__crt_seh_guarded_call@X@@QEAAX$$QEAV<lambda_d80eeec6fff315bfe5c115232f3240e3>@@AEAV<lambda_6e4b09c48022b2350581041d5f6b0c4c>@@$$QEAV<lambda_2358e3775559c9db80273638284d5e45>@@@Z@4HA 000000018005ad72 f   libucrt:exit.obj
 0001:00059d72       ?fin$0@?0???$?RV<lambda_aa87e3671a710a21b5dc78c0bdf72e11>@@AEAV<lambda_92619d2358a28f41a33ba319515a20b9>@@V<lambda_6992ecaafeb10aed2b74cb1fae11a551>@@@?$__crt_seh_guarded_call@X@@QEAAX$$QEAV<lambda_aa87e3671a710a21b5dc78c0bdf72e11>@@AEAV<lambda_92619d2358a28f41a33ba319515a20b9>@@$$QEAV<lambda_6992ecaafeb10aed2b74cb1fae11a551>@@@Z@4HA 000000018005ad72 f   libucrt:per_thread_data.obj
 0001:00059d72       ?fin$0@?0???$?RV<lambda_a22f0c497e5168315e06dae667770027>@@AEAV<lambda_a094494068278ba5130ab06e1292f60a>@@V<lambda_24dc10c13f43218c635520766e23e324>@@@?$__crt_seh_guarded_call@_N@@QEAA_N$$QEAV<lambda_a22f0c497e5168315e06dae667770027>@@AEAV<lambda_a094494068278ba5130ab06e1292f60a>@@$$QEAV<lambda_24dc10c13f43218c635520766e23e324>@@@Z@4HA 000000018005ad72 f   libucrt:spawnv.obj
 0001:00059d72       ?fin$0@?0???$?RV<lambda_0ae27a3a962d80f24befdcbee591983d>@@AEAV<lambda_8d0ee55de4b1038c4002e0adecdf1839>@@V<lambda_dc504788e8f1664fe9b84e20bfb512f2>@@@?$__crt_seh_guarded_call@X@@QEAAX$$QEAV<lambda_0ae27a3a962d80f24befdcbee591983d>@@AEAV<lambda_8d0ee55de4b1038c4002e0adecdf1839>@@$$QEAV<lambda_dc504788e8f1664fe9b84e20bfb512f2>@@@Z@4HA 000000018005ad72 f   libucrt:per_thread_data.obj
 0001:00059d8c       ?filt$0@?0???R<lambda_6e4b09c48022b2350581041d5f6b0c4c>@@QEBA@XZ@4HA 000000018005ad8c f   libucrt:exit.obj
 0001:00059da7       ?fin$0@?0???$?RV<lambda_410d79af7f07d98d83a3f525b3859a53>@@AEAV<lambda_3e16ef9562a7dcce91392c22ab16ea36>@@V<lambda_38119f0e861e05405d8a144b9b982f0a>@@@?$__crt_seh_guarded_call@X@@QEAAX$$QEAV<lambda_410d79af7f07d98d83a3f525b3859a53>@@AEAV<lambda_3e16ef9562a7dcce91392c22ab16ea36>@@$$QEAV<lambda_38119f0e861e05405d8a144b9b982f0a>@@@Z@4HA 000000018005ada7 f   libucrt:wsetlocale.obj
 0001:00059dc1       __acrt_initialize_lowio$fin$0 000000018005adc1 f   libucrt:ioinit.obj
 0001:00059dc1       _alloc_osfhnd$fin$0        000000018005adc1 f   libucrt:osfinfo.obj
 0001:00059dc1       __acrt_lowio_ensure_fh_exists$fin$0 000000018005adc1 f   libucrt:osfinfo.obj
 0001:00059dda       ?fin$0@?0??__acrt_stdio_allocate_stream@@YA?AV__crt_stdio_stream@@XZ@4HA 000000018005adda f   libucrt:stream.obj
 0001:00059dda       _fcloseall$fin$0           000000018005adda f   libucrt:closeall.obj
 0001:00059df3       ?fin$0@?0???$?RV<lambda_a37b2b86f63e897a80ea819b0eb08c01>@@AEAV<lambda_38ce7e780aa69e748d6df282ebc68efe>@@V<lambda_99fb1378e971ab6e7edea83e3a7a83a2>@@@?$__crt_seh_guarded_call@H@@QEAAH$$QEAV<lambda_a37b2b86f63e897a80ea819b0eb08c01>@@AEAV<lambda_38ce7e780aa69e748d6df282ebc68efe>@@$$QEAV<lambda_99fb1378e971ab6e7edea83e3a7a83a2>@@@Z@4HA 000000018005adf3 f   libucrt:commit.obj
 0001:00059df3       ?fin$0@?0???$?RV<lambda_751a882b2c74d4b022dec766aa51a29a>@@AEAV<lambda_628dfdc04ba53c8bfc02c9951375f3f5>@@V<lambda_f6c7be5f7998530c34de24c7437d6b54>@@@?$__crt_seh_guarded_call@H@@QEAAH$$QEAV<lambda_751a882b2c74d4b022dec766aa51a29a>@@AEAV<lambda_628dfdc04ba53c8bfc02c9951375f3f5>@@$$QEAV<lambda_f6c7be5f7998530c34de24c7437d6b54>@@@Z@4HA 000000018005adf3 f   libucrt:close.obj
 0001:00059e0d       _read$fin$0                000000018005ae0d f   libucrt:read.obj
 0001:00059e24       ?fin$0@?0???$common_lseek@J@@YAJHJH@Z@4HA 000000018005ae24 f   libucrt:lseek.obj
 0001:00059e24       ?fin$0@?0???$common_lseek@_J@@YA_JH_JH@Z@4HA 000000018005ae24 f   libucrt:lseek.obj
 0001:00059e24       _write$fin$0               000000018005ae24 f   libucrt:write.obj
 0001:00059e3b       _pipe$fin$1                000000018005ae3b f   libucrt:pipe.obj
 0001:00059e57       _pipe$fin$0                000000018005ae57 f   libucrt:pipe.obj
 0001:00059e73       ?fin$0@?0???$common_fdopen@_W@@YAPEAU_iobuf@@HQEB_W@Z@4HA 000000018005ae73 f   libucrt:fdopen.obj
 0001:00059e8d       ?fin$0@?0???$common_sopen_dispatch@_W@@YAHQEB_WHHHQEAHH@Z@4HA 000000018005ae8d f   libucrt:open.obj
 0001:00059e8d       ?fin$0@?0???$common_sopen_dispatch@D@@YAHQEBDHHHQEAHH@Z@4HA 000000018005ae8d f   libucrt:open.obj
 0001:00059ee0       _rmtmp$fin$0               000000018005aee0 f   libucrt:rmtmp.obj
 0001:00059efa       _rmtmp$fin$1               000000018005aefa f   libucrt:rmtmp.obj
 0001:00059f13       ?fin$0@?0??update_thread_multibyte_data_internal@@YAPEAU__crt_multibyte_data@@QEAU__acrt_ptd@@QEAPEAU1@@Z@4HA 000000018005af13 f   libucrt:mbctype.obj
 0001:00059f2c       _query_new_handler$fin$0   000000018005af2c f   libucrt:new_handler.obj
 0001:00059f42       raise$fin$0                000000018005af42 f   libucrt:signal.obj
 0001:00059f63       __acrt_update_thread_locale_data$fin$0 000000018005af63 f   libucrt:locale_refcounting.obj
 0001:00059f80       _IsNonwritableInCurrentImage$filt$0 000000018005af80 f   LIBCMT:pesect.obj
 0001:00059fa0       $xdatasym                  000000018005afa0     chkstk.obj
 0001:00059fa8       $unwind$fprintf            000000018005afa8     service.obj
 0001:00059fa8       $unwind$fscanf             000000018005afa8     uliolib51.obj
 0001:00059fa8       $unwind$sprintf            000000018005afa8     bit64.obj
 0001:00059fb4       $unwind$GetAttrFromTable   000000018005afb4     util.obj
 0001:00059fb4       $unwind$editor_DeleteChar  000000018005afb4     service.obj
 0001:00059fb4       $unwind$__acrt_wgetpath    000000018005afb4     libucrt:getpath.obj
 0001:00059fb4       $unwind$func_New           000000018005afb4     lregex.obj
 0001:00059fb4       $unwind$GetFileSizeFromTable 000000018005afb4     util.obj
 0001:00059fb4       $unwind$LF_FreeContentData 000000018005afb4     exported.obj
 0001:00059fb4       $unwind$_close_nolock      000000018005afb4     libucrt:close.obj
 0001:00059fb4       $unwind$editor_DeleteString 000000018005afb4     service.obj
 0001:00059fb4       $unwind$??$common_initialize_environment_nolock@_W@@YAHXZ 000000018005afb4     libucrt:environment_initialization.obj
 0001:00059fb4       $unwind$GetExportFunction  000000018005afb4     exported.obj
 0001:00059fb4       $unwind$?type_case_c_tchar@?$output_processor@DV?$string_output_adapter@D@__crt_stdio_output@@V?$standard_base@DV?$string_output_adapter@D@__crt_stdio_output@@@2@@__crt_stdio_output@@AEAA_ND@Z 000000018005afb4     libucrt:output.obj
 0001:00059fb4       $unwind$ustring_EnumSystemCodePages 000000018005afb4     ustring.obj
 0001:00059fb4       $unwind$??$common_initialize_environment_nolock@D@@YAHXZ 000000018005afb4     libucrt:environment_initialization.obj
 0001:00059fb4       $unwind$strncpy_s          000000018005afb4     libucrt:strncpy_s.obj
 0001:00059fb4       $unwind$LF_ExitFAR         000000018005afb4     exported.obj
 0001:00059fb4       $unwind$LF_FreeFindData    000000018005afb4     exported.obj
 0001:00059fb4       $unwind$free_dialog        000000018005afb4     service.obj
 0001:00059fb4       $unwind$unic_len           000000018005afb4     slnunico.obj
 0001:00059fb4       $unwind$_RTC_Initialize    000000018005afb4     LIBCMT:_initsect_.obj
 0001:00059fb4       $unwind$_RTC_Terminate     000000018005afb4     LIBCMT:_initsect_.obj
 0001:00059fb4       $unwind$?common_fseek_binary_mode_read_only_fast_track_nolock@@YA_NV__crt_stdio_stream@@_JH@Z 000000018005afb4     libucrt:fseek.obj
 0001:00059fb4       $unwind$editor_DeleteBlock 000000018005afb4     service.obj
 0001:00059fb4       $unwind$editor_Redraw      000000018005afb4     service.obj
 0001:00059fb4       $unwind$bit64_pushuserdata 000000018005afb4     bit64.obj
 0001:00059fb4       $unwind$bit64_push         000000018005afb4     bit64.obj
 0001:00059fb4       $unwind$viewer_Quit        000000018005afb4     service.obj
 0001:00059fb4       $unwind$LF_Analyse         000000018005afb4     exported.obj
 0001:00059fb4       $unwind$?type_case_c_tchar@?$output_processor@DV?$stream_output_adapter@D@__crt_stdio_output@@V?$standard_base@DV?$stream_output_adapter@D@__crt_stdio_output@@@2@@__crt_stdio_output@@AEAA_ND@Z 000000018005afb4     libucrt:output.obj
 0001:00059fb4       $unwind$ustring_GetKeyState 000000018005afb4     ustring.obj
 0001:00059fb4       $unwind$method_tostring    000000018005afb4     lregex.obj
 0001:00059fb4       $unwind$?force_decimal_point@__crt_stdio_output@@YAXPEADQEAU__crt_locale_pointers@@@Z 000000018005afb4     libucrt:output.obj
 0001:00059fb4       $unwind$FillEditorSetPosition 000000018005afb4     service.obj
 0001:00059fb4       $unwind$method_gc          000000018005afb4     lregex.obj
 0001:00059fb4       $unwind$far_GetNumberOfLinks 000000018005afb4     service.obj
 0001:00059fb4       $unwind$__acrt_uninitialize_lowio 000000018005afb4     libucrt:ioinit.obj
 0001:00059fb4       $unwind$??0_LocaleUpdate@@QEAA@QEAU__crt_locale_pointers@@@Z 000000018005afb4     libucrt:output.obj
 0001:00059fb4       $unwind$far_Show           000000018005afb4     service.obj
 0001:00059fb4       $unwind$lshift             000000018005afb4     bit64.obj
 0001:00059fb4       $unwind$rshift             000000018005afb4     bit64.obj
 0001:00059fb4       $unwind$PushPluginHandle   000000018005afb4     service.obj
 0001:00059fb4       $unwind$viewer_Redraw      000000018005afb4     service.obj
 0001:00059fb4       $unwind$PutFlagsToTable    000000018005afb4     service.obj
 0001:00059fb4       $unwind$__vcrt_FlsSetValue 000000018005afb4     libvcruntime:winapi_downlevel.obj
 0001:00059fb4       $unwind$GetFlagsFromTable  000000018005afb4     service.obj
 0001:00059fb4       $unwind$arshift            000000018005afb4     bit64.obj
 0001:00059fb4       $unwind$CheckFlagsFromTable 000000018005afb4     service.obj
 0001:00059fb4       $unwind$filefilter_Free    000000018005afb4     service.obj
 0001:00059fb4       $unwind$filefilter_gc      000000018005afb4     service.obj
 0001:00059fb4       $unwind$RegisterObject     000000018005afb4     exported.obj
 0001:00059fb4       $unwind$CheckFlags         000000018005afb4     service.obj
 0001:00059fb4       $unwind$PushAnalyseInfo    000000018005afb4     exported.obj
 0001:00059fb4       $unwind$DialogHandleEqual  000000018005afb4     service.obj
 0001:00059fb4       $unwind$PushFarMacroValue  000000018005afb4     exported.obj
 0001:00059fb4       $unwind$_realloc_base      000000018005afb4     libucrt:realloc_base.obj
 0001:00059fb4       $unwind$__acrt_stdio_begin_temporary_buffering_nolock 000000018005afb4     libucrt:_sftbuf.obj
 0001:00059fb4       $unwind$filefilter_OpenMenu 000000018005afb4     service.obj
 0001:00059fb4       $unwind$filefilter_Starting 000000018005afb4     service.obj
 0001:00059fb4       $unwind$win_SetEnv         000000018005afb4     win.obj
 0001:00059fb4       $unwind$far_UnloadPlugin   000000018005afb4     service.obj
 0001:00059fb4       $unwind$?state_case_normal_tchar@?$output_processor@DV?$stream_output_adapter@D@__crt_stdio_output@@V?$standard_base@DV?$stream_output_adapter@D@__crt_stdio_output@@@2@@__crt_stdio_output@@AEAA_ND@Z 000000018005afb4     libucrt:output.obj
 0001:00059fb4       $unwind$CheckHKey          000000018005afb4     win.obj
 0001:00059fb4       $unwind$GetLuaStateTimerQueue 000000018005afb4     service.obj
 0001:00059fb4       $unwind$_ungetc_nolock     000000018005afb4     libucrt:ungetc.obj
 0001:00059fb4       $unwind$far_LIsUpper       000000018005afb4     service.obj
 0001:00059fb4       $unwind$io_type            000000018005afb4     uliolib51.obj
 0001:00059fb4       $unwind$f_sub              000000018005afb4     bit64.obj
 0001:00059fb4       $unwind$newfile            000000018005afb4     uliolib51.obj
 0001:00059fb4       $unwind$??$get_tmpfile_buffer_nolock@D@@YAPEADW4buffer_id@?A0x5b9a7937@@@Z 000000018005afb4     libucrt:tmpfile.obj
 0001:00059fb4       $unwind$Settings_free      000000018005afb4     service.obj
 0001:00059fb4       $unwind$PushFarColor       000000018005afb4     service.obj
 0001:00059fb4       $unwind$far_GetMsg         000000018005afb4     service.obj
 0001:00059fb4       $unwind$far_LIsLower       000000018005afb4     service.obj
 0001:00059fb4       $unwind$far_LIsAlphanum    000000018005afb4     service.obj
 0001:00059fb4       $unwind$f_div              000000018005afb4     bit64.obj
 0001:00059fb4       $unwind$far_LIsAlpha       000000018005afb4     service.obj
 0001:00059fb4       $unwind$panel_IsActivePanel 000000018005afb4     service.obj
 0001:00059fb4       $unwind$io_tmpfile         000000018005afb4     uliolib51.obj
 0001:00059fb4       $unwind$?process_state@?$input_processor@DV?$stream_input_adapter@D@__crt_stdio_input@@@__crt_stdio_input@@AEAA_NXZ 000000018005afb4     libucrt:input.obj
 0001:00059fb4       $unwind$editor_AddSessionBookmark 000000018005afb4     service.obj
 0001:00059fb4       $unwind$io_read            000000018005afb4     uliolib51.obj
 0001:00059fb4       $unwind$editor_ClearSessionBookmarks 000000018005afb4     service.obj
 0001:00059fb4       $unwind$?process_literal_character_tchar@?$input_processor@DV?$stream_input_adapter@D@__crt_stdio_input@@@__crt_stdio_input@@AEAA_ND@Z 000000018005afb4     libucrt:input.obj
 0001:00059fb4       $unwind$f_eq               000000018005afb4     bit64.obj
 0001:00059fb4       $unwind$f_lt               000000018005afb4     bit64.obj
 0001:00059fb4       $unwind$editor_NextSessionBookmark 000000018005afb4     service.obj
 0001:00059fb4       $unwind$f_le               000000018005afb4     bit64.obj
 0001:00059fb4       $unwind$editor_PrevSessionBookmark 000000018005afb4     service.obj
 0001:00059fb4       $unwind$f_read             000000018005afb4     uliolib51.obj
 0001:00059fb4       $unwind$?process_conversion_specifier@?$input_processor@DV?$stream_input_adapter@D@__crt_stdio_input@@@__crt_stdio_input@@AEAA_NXZ 000000018005afb4     libucrt:input.obj
 0001:00059fb4       $unwind$PutStrToTable      000000018005afb4     ustring.obj
 0001:00059fb4       $unwind$PutStrToArray      000000018005afb4     ustring.obj
 0001:00059fb4       $unwind$PutNumToTable      000000018005afb4     ustring.obj
 0001:00059fb4       $unwind$PutLStrToTable     000000018005afb4     ustring.obj
 0001:00059fb4       $unwind$panel_GetCmdLinePos 000000018005afb4     service.obj
 0001:00059fb4       $unwind$?replace_current_thread_locale_nolock@@YAXQEAU__acrt_ptd@@QEAU__crt_locale_data@@@Z 000000018005afb4     libucrt:per_thread_data.obj
 0001:00059fb4       $unwind$io_write           000000018005afb4     uliolib51.obj
 0001:00059fb4       $unwind$editor_Quit        000000018005afb4     service.obj
 0001:00059fb4       $unwind$LF_InitLuaState2   000000018005afb4     service.obj
 0001:00059fb4       $unwind$?process_floating_point_specifier@?$input_processor@DV?$stream_input_adapter@D@__crt_stdio_input@@@__crt_stdio_input@@AEAA_NXZ 000000018005afb4     libucrt:input.obj
 0001:00059fb4       $unwind$LF_ProcessEditorInput 000000018005afb4     exported.obj
 0001:00059fb4       $unwind$f_write            000000018005afb4     uliolib51.obj
 0001:00059fb4       $unwind$?write_integer@?$input_processor@DV?$stream_input_adapter@D@__crt_stdio_input@@@__crt_stdio_input@@AEAA_N_K@Z 000000018005afb4     libucrt:input.obj
 0001:00059fb4       $unwind$PutIntToTable      000000018005afb4     ustring.obj
 0001:00059fb4       $unwind$_fclose_nolock     000000018005afb4     libucrt:fclose.obj
 0001:00059fb4       $unwind$PutIntToArray      000000018005afb4     ustring.obj
 0001:00059fb4       $unwind$__acrt_LocaleNameToLCID 000000018005afb4     libucrt:winapi_thunks.obj
 0001:00059fb4       $unwind$__acrt_getptd      000000018005afb4     libucrt:per_thread_data.obj
 0001:00059fb4       $unwind$LF_GetLuafarAPI    000000018005afb4     service.obj
 0001:00059fb4       $unwind$f_rawhandle        000000018005afb4     uliolib51.obj
 0001:00059fb4       $unwind$PutBoolToTable     000000018005afb4     ustring.obj
 0001:00059fb4       $unwind$__acrt_getptd_noexit 000000018005afb4     libucrt:per_thread_data.obj
 0001:00059fb4       $unwind$__acrt_execute_uninitializers 000000018005afb4     libucrt:shared_initialization.obj
 0001:00059fb4       $unwind$GetOptIntFromTable 000000018005afb4     ustring.obj
 0001:00059fb4       $unwind$_updatetlocinfoEx_nolock 000000018005afb4     libucrt:locale_refcounting.obj
 0001:00059fb4       $unwind$GetOptIntFromArray 000000018005afb4     ustring.obj
 0001:00059fb4       $unwind$GetOptBoolFromTable 000000018005afb4     ustring.obj
 0001:00059fb4       $unwind$GetBoolFromTable   000000018005afb4     ustring.obj
 0001:00059fb4       $unwind$SysErrorReturn     000000018005afb4     ustring.obj
 0001:00059fb4       $unwind$method_bracketscount 000000018005afb4     lregex.obj
 0001:00059fb4       $unwind$PushInputRecord    000000018005afb4     service.obj
 0001:00059fb4       $unwind$??R<lambda_156378f40168adef48d7ddfcff3a1264>@@QEBA_NXZ 000000018005afb4     libucrt:input.obj
 0001:00059fb4       $unwind$ll_loadlib         000000018005afb4     uloadlib51.obj
 0001:00059fb4       $unwind$_initterm_e        000000018005afb4     libucrt:initterm.obj
 0001:00059fb4       $unwind$loader_Lua         000000018005afb4     uloadlib51.obj
 0001:00059fb4       $unwind$panel_CheckPanelsExist 000000018005afb4     service.obj
 0001:00059fb4       $unwind$mkfuncname         000000018005afb4     uloadlib51.obj
 0001:00059fb4       $unwind$__acrt_FlsSetValue 000000018005afb4     libucrt:winapi_thunks.obj
 0001:00059fb4       $unwind$__acrt_errno_map_os_error 000000018005afb4     libucrt:errno.obj
 0001:00059fb4       $unwind$loader_preload     000000018005afb4     uloadlib51.obj
 0001:00059fc0       $unwind$_cwait             000000018005afc0     libucrt:wait.obj
 0001:00059fc0       $unwind$LF_ProcessEditorEvent 000000018005afc0     exported.obj
 0001:00059fc0       $unwind$?type_case_c_tchar@?$output_processor@_WV?$string_output_adapter@_W@__crt_stdio_output@@V?$standard_base@_WV?$string_output_adapter@_W@__crt_stdio_output@@@2@@__crt_stdio_output@@AEAA_N_W@Z 000000018005afc0     libucrt:output.obj
 0001:00059fc0       $unwind$??R<lambda_ca71763b3c0644891230e4f79ea54fa6>@@QEBAHXZ 000000018005afc0     libucrt:setvbuf.obj
 0001:00059fc0       $unwind$bit64_getvalue     000000018005afc0     bit64.obj
 0001:00059fc0       $unwind$LF_ProcessConsoleInput 000000018005afc0     exported.obj
 0001:00059fd0       $chain$0$bit64_getvalue    000000018005afd0     bit64.obj
 0001:00059fe4       $chain$1$bit64_getvalue    000000018005afe4     bit64.obj
 0001:00059ff4       $unwind$check64            000000018005aff4     bit64.obj
 0001:0005a004       $chain$0$check64           000000018005b004     bit64.obj
 0001:0005a018       $chain$1$check64           000000018005b018     bit64.obj
 0001:0005a028       $unwind$InitMPR            000000018005b028     luamacro.obj
 0001:0005a028       $unwind$FillInputRecord    000000018005b028     service.obj
 0001:0005a028       $unwind$pcall_msg          000000018005b028     exported.obj
 0001:0005a028       $unwind$timer_index        000000018005b028     service.obj
 0001:0005a028       $unwind$??$skip_whitespace@Vstream_input_adapter@__crt_stdio_input@@D@__crt_stdio_input@@YAHAEAV?$stream_input_adapter@D@0@QEAU__crt_locale_pointers@@@Z 000000018005b028     libucrt:input.obj
 0001:0005a028       $unwind$PackMacroValues    000000018005b028     exported.obj
 0001:0005a028       $unwind$?find_or_allocate_unused_stream_nolock@@YA?AV__crt_stdio_stream@@XZ 000000018005b028     libucrt:stream.obj
 0001:0005a028       $unwind$AddBufToCollector  000000018005b028     exported.obj
 0001:0005a028       $unwind$OptInputRecord     000000018005b028     service.obj
 0001:0005a028       $unwind$_seh_filter_exe    000000018005b028     libucrt:exception_filter.obj
 0001:0005a028       $unwind$?common_fseek_nolock@@YAHV__crt_stdio_stream@@_JH@Z 000000018005b028     libucrt:fseek.obj
 0001:0005a028       $unwind$push_far_regex     000000018005b028     lregex.obj
 0001:0005a028       $unwind$__scrt_dllmain_exception_filter 000000018005b028     LIBCMT:utility.obj
 0001:0005a028       $unwind$__acrt_free_locale 000000018005b028     libucrt:locale_refcounting.obj
 0001:0005a028       $unwind$_initterm          000000018005b028     libucrt:initterm.obj
 0001:0005a028       $unwind$findfile           000000018005b028     uloadlib51.obj
 0001:0005a028       $unwind$FillPluginPanelItem 000000018005b028     exported.obj
 0001:0005a028       $unwind$band               000000018005b028     bit64.obj
 0001:0005a028       $unwind$bor                000000018005b028     bit64.obj
 0001:0005a028       $unwind$bxor               000000018005b028     bit64.obj
 0001:0005a028       $unwind$??$ensure_buffer_is_big_enough@_W@formatting_buffer@__crt_stdio_output@@QEAA_N_K@Z 000000018005b028     libucrt:output.obj
 0001:0005a028       $unwind$??$common_ftell_nolock@_J@@YA_JV__crt_stdio_stream@@@Z 000000018005b028     libucrt:ftell.obj
 0001:0005a028       $unwind$__acrt_lowio_create_handle_array 000000018005b028     libucrt:osfinfo.obj
 0001:0005a028       $unwind$??$common_getenv_nolock@_W@@YAPEA_WQEB_W@Z 000000018005b028     libucrt:getenv.obj
 0001:0005a028       $unwind$__dcrt_get_wide_environment_from_os 000000018005b028     libucrt:get_environment_from_os.obj
 0001:0005a028       $unwind$win_CopyFile       000000018005b028     win.obj
 0001:0005a028       $unwind$_recalloc_base     000000018005b028     libucrt:recalloc.obj
 0001:0005a028       $unwind$??$ensure_buffer_is_big_enough@D@formatting_buffer@__crt_stdio_output@@QEAA_N_K@Z 000000018005b028     libucrt:output.obj
 0001:0005a028       $unwind$uc_New             000000018005b028     lusercontrol.obj
 0001:0005a028       $unwind$pushresult         000000018005b028     uliolib51.obj
 0001:0005a028       $unwind$?setSBCS@@YAXPEAU__crt_multibyte_data@@@Z 000000018005b028     libucrt:mbctype.obj
 0001:0005a028       $unwind$f_add              000000018005b028     bit64.obj
 0001:0005a028       $unwind$win_DeleteRegKey   000000018005b028     win.obj
 0001:0005a028       $unwind$io_popen           000000018005b028     uliolib51.obj
 0001:0005a028       $unwind$f_mul              000000018005b028     bit64.obj
 0001:0005a03c       $unwind$win_GetSystemTimeAsFileTime 000000018005b03c     win.obj
 0001:0005a03c       $unwind$io_gc              000000018005b03c     uliolib51.obj
 0001:0005a03c       $unwind$io_close           000000018005b03c     uliolib51.obj
 0001:0005a03c       $unwind$__raise_securityfailure 000000018005b03c     LIBCMT:gs_report.obj
 0001:0005a03c       $unwind$aux_close          000000018005b03c     uliolib51.obj
 0001:0005a03c       $unwind$__scrt_release_startup_lock 000000018005b03c     LIBCMT:utility.obj
 0001:0005a03c       $unwind$_malloc_base       000000018005b03c     libucrt:malloc_base.obj
 0001:0005a03c       $unwind$io_tostring        000000018005b03c     uliolib51.obj
 0001:0005a03c       $unwind$io_noclose         000000018005b03c     uliolib51.obj
 0001:0005a03c       $unwind$__vcrt_freeptd     000000018005b03c     libvcruntime:per_thread_data.obj
 0001:0005a03c       $unwind$?internal_isupper_l@@YA_NHQEAU__crt_locale_pointers@@@Z 000000018005b03c     libucrt:tolower_toupper.obj
 0001:0005a03c       $unwind$uc_tostring        000000018005b03c     lusercontrol.obj
 0001:0005a03c       $unwind$__acrt_update_multibyte_info 000000018005b03c     libucrt:locale_update.obj
 0001:0005a03c       $unwind$uc_len             000000018005b03c     lusercontrol.obj
 0001:0005a03c       $unwind$far_FreeSettings   000000018005b03c     service.obj
 0001:0005a03c       $unwind$??$common_xtox@_KD@@YAH_KQEAD0I_N@Z 000000018005b03c     libucrt:xtoa.obj
 0001:0005a03c       $unwind$far_CopyToClipboard 000000018005b03c     service.obj
 0001:0005a03c       $unwind$__scrt_initialize_crt 000000018005b03c     LIBCMT:utility.obj
 0001:0005a03c       $unwind$DeleteLuaStateTimerQueue 000000018005b03c     service.obj
 0001:0005a03c       $unwind$f_lines            000000018005b03c     uliolib51.obj
 0001:0005a03c       $unwind$SetFarColors       000000018005b03c     keysandcolors.obj
 0001:0005a03c       $unwind$feholdexcept       000000018005b03c     libucrt:feholdexcept.obj
 0001:0005a03c       $unwind$luaopen_usercontrol 000000018005b03c     lusercontrol.obj
 0001:0005a03c       $unwind$fesetenv           000000018005b03c     libucrt:fesetenv.obj
 0001:0005a03c       $unwind$_fflush_nolock     000000018005b03c     libucrt:fflush.obj
 0001:0005a03c       $unwind$Settings_tostring  000000018005b03c     service.obj
 0001:0005a03c       $unwind$fegetenv           000000018005b03c     libucrt:fegetenv.obj
 0001:0005a03c       $unwind$_callnewh          000000018005b03c     libucrt:new_handler.obj
 0001:0005a03c       $unwind$OptHandle          000000018005b03c     service.obj
 0001:0005a03c       $unwind$__vcrt_initialize_locks 000000018005b03c     libvcruntime:locks.obj
 0001:0005a03c       $unwind$f_unm              000000018005b03c     bit64.obj
 0001:0005a03c       $unwind$__scrt_uninitialize_crt 000000018005b03c     LIBCMT:utility.obj
 0001:0005a03c       $unwind$win_DeleteFile     000000018005b03c     win.obj
 0001:0005a03c       $unwind$win_RemoveDir      000000018005b03c     win.obj
 0001:0005a03c       $unwind$__vcrt_FlsAlloc    000000018005b03c     libvcruntime:winapi_downlevel.obj
 0001:0005a03c       $unwind$filefilter_tostring 000000018005b03c     service.obj
 0001:0005a03c       $unwind$strcpy_s           000000018005b03c     libucrt:strcpy_s.obj
 0001:0005a03c       $unwind$luaopen_win        000000018005b03c     win.obj
 0001:0005a03c       $unwind$far_RunDefaultScript 000000018005b03c     service.obj
 0001:0005a03c       $unwind$__acrt_uninitialize_stdio 000000018005b03c     libucrt:_file.obj
 0001:0005a03c       $unwind$_strupr            000000018005b03c     libucrt:strupr.obj
 0001:0005a03c       $unwind$__vcrt_FlsFree     000000018005b03c     libvcruntime:winapi_downlevel.obj
 0001:0005a03c       $unwind$luaopen_bit64      000000018005b03c     bit64.obj
 0001:0005a03c       $unwind$__vcrt_FlsGetValue 000000018005b03c     libvcruntime:winapi_downlevel.obj
 0001:0005a03c       $unwind$luaB_loadfileW     000000018005b03c     lflua.obj
 0001:0005a03c       $unwind$luaopen_unicode    000000018005b03c     slnunico.obj
 0001:0005a03c       $unwind$__acrt_allocate_buffer_for_argv 000000018005b03c     libucrt:argv_parsing.obj
 0001:0005a03c       $unwind$_set_statfp        000000018005b03c     libucrt:fpctrl.obj
 0001:0005a03c       $unwind$uninitialize_allocated_memory 000000018005b03c     libucrt:initialization.obj
 0001:0005a03c       $unwind$initialize_pointers 000000018005b03c     libucrt:initialization.obj
 0001:0005a03c       $unwind$bnot               000000018005b03c     bit64.obj
 0001:0005a03c       $unwind$__acrt_update_locale_info 000000018005b03c     libucrt:locale_update.obj
 0001:0005a03c       $unwind$?exit_or_terminate_process@@YAXI@Z 000000018005b03c     libucrt:exit.obj
 0001:0005a03c       $unwind$timer_tostring     000000018005b03c     service.obj
 0001:0005a03c       $unwind$__acrt_freeptd     000000018005b03c     libucrt:per_thread_data.obj
 0001:0005a03c       $unwind$far_MacroGetArea   000000018005b03c     service.obj
 0001:0005a03c       $unwind$FarPanelItemFreeCallback 000000018005b03c     exported.obj
 0001:0005a03c       $unwind$?idtab@@YAPEAUprocess_handle_pair@?A0xe43b7539@@QEAU_iobuf@@@Z 000000018005b03c     libucrt:popen.obj
 0001:0005a03c       $unwind$far_CPluginStartupInfo 000000018005b03c     service.obj
 0001:0005a03c       $unwind$wcscpy_s           000000018005b03c     libucrt:wcscpy_s.obj
 0001:0005a03c       $unwind$?try_cor_exit_process@@YAXI@Z 000000018005b03c     libucrt:exit.obj
 0001:0005a03c       $unwind$?state_case_normal@?$output_processor@DV?$stream_output_adapter@D@__crt_stdio_output@@V?$standard_base@DV?$stream_output_adapter@D@__crt_stdio_output@@@2@@__crt_stdio_output@@AEAA_NXZ 000000018005b03c     libucrt:output.obj
 0001:0005a03c       $unwind$__acrt_stdio_allocate_buffer_nolock 000000018005b03c     libucrt:_getbuf.obj
 0001:0005a03c       $unwind$_clrfp             000000018005b03c     libucrt:fpctrl.obj
 0001:0005a03c       $unwind$?type_case_s@?$output_processor@DV?$stream_output_adapter@D@__crt_stdio_output@@V?$standard_base@DV?$stream_output_adapter@D@__crt_stdio_output@@@2@@__crt_stdio_output@@AEAA_NXZ 000000018005b03c     libucrt:output.obj
 0001:0005a03c       $unwind$win_FileTimeToLocalFileTime 000000018005b03c     win.obj
 0001:0005a03c       $unwind$far_MacroGetState  000000018005b03c     service.obj
 0001:0005a03c       $unwind$far_MacroSaveAll   000000018005b03c     service.obj
 0001:0005a03c       $unwind$?scan_optional_field_width@?$format_string_parser@D@__crt_stdio_input@@AEAA_NXZ 000000018005b03c     libucrt:input.obj
 0001:0005a03c       $unwind$__acrt_AppPolicyGetProcessTerminationMethodInternal 000000018005b03c     libucrt:winapi_thunks.obj
 0001:0005a03c       $unwind$?state_case_normal@?$output_processor@DV?$string_output_adapter@D@__crt_stdio_output@@V?$standard_base@DV?$string_output_adapter@D@__crt_stdio_output@@@2@@__crt_stdio_output@@AEAA_NXZ 000000018005b03c     libucrt:output.obj
 0001:0005a03c       $unwind$__acrt_FlsAlloc    000000018005b03c     libucrt:winapi_thunks.obj
 0001:0005a03c       $unwind$_clearfp           000000018005b03c     libucrt:ieee.obj
 0001:0005a03c       $unwind$__acrt_getptd_head 000000018005b03c     libucrt:per_thread_data.obj
 0001:0005a03c       $unwind$__std_type_info_destroy_list 000000018005b03c     libvcruntime:std_type_info.obj
 0001:0005a03c       $unwind$check_utf16_string 000000018005b03c     ustring.obj
 0001:0005a03c       $unwind$__acrt_uninitialize_winapi_thunks 000000018005b03c     libucrt:winapi_thunks.obj
 0001:0005a03c       $unwind$TimerCallback      000000018005b03c     service.obj
 0001:0005a03c       $unwind$PutAttrToTable     000000018005b03c     ustring.obj
 0001:0005a03c       $unwind$ustring_GetACP     000000018005b03c     ustring.obj
 0001:0005a03c       $unwind$push_onecapture    000000018005b03c     slnunico.obj
 0001:0005a03c       $unwind$luaopen_regex      000000018005b03c     lregex.obj
 0001:0005a03c       $unwind$ustring_GetOEMCP   000000018005b03c     ustring.obj
 0001:0005a03c       $unwind$ReplacePluginInfoCollector 000000018005b03c     exported.obj
 0001:0005a03c       $unwind$PushPluginObject   000000018005b03c     exported.obj
 0001:0005a03c       $unwind$__acrt_FlsFree     000000018005b03c     libucrt:winapi_thunks.obj
 0001:0005a03c       $unwind$pusherror          000000018005b03c     ustring.obj
 0001:0005a03c       $unwind$dialog_tostring    000000018005b03c     service.obj
 0001:0005a03c       $unwind$ustring_GetDriveType 000000018005b03c     ustring.obj
 0001:0005a03c       $unwind$ustring_len        000000018005b03c     ustring.obj
 0001:0005a03c       $unwind$traceback          000000018005b03c     exported.obj
 0001:0005a03c       $unwind$dialog_rawhandle   000000018005b03c     service.obj
 0001:0005a03c       $unwind$?type_case_s@?$output_processor@DV?$string_output_adapter@D@__crt_stdio_output@@V?$standard_base@DV?$string_output_adapter@D@__crt_stdio_output@@@2@@__crt_stdio_output@@AEAA_NXZ 000000018005b03c     libucrt:output.obj
 0001:0005a03c       $unwind$ustring_system     000000018005b03c     ustring.obj
 0001:0005a03c       $unwind$gctm               000000018005b03c     uloadlib51.obj
 0001:0005a03c       $unwind$GetFileTimeFromTable 000000018005b03c     util.obj
 0001:0005a03c       $unwind$__acrt_FlsGetValue 000000018005b03c     libucrt:winapi_thunks.obj
 0001:0005a03c       $unwind$luaopen_ustring    000000018005b03c     ustring.obj
 0001:0005a03c       $unwind$__acrt_fp_strflt_to_string 000000018005b03c     libucrt:_fptostr.obj
 0001:0005a03c       $unwind$__acrt_uninitialize_locks 000000018005b03c     libucrt:locks.obj
 0001:0005a03c       $unwind$ll_seeall          000000018005b03c     uloadlib51.obj
 0001:0005a03c       $unwind$__acrt_stdio_free_buffer_nolock 000000018005b03c     libucrt:_freebuf.obj
 0001:0005a03c       $unwind$__acrt_initialize_locks 000000018005b03c     libucrt:locks.obj
 0001:0005a03c       $unwind$_calloc_base       000000018005b03c     libucrt:calloc_base.obj
 0001:0005a03c       $unwind$__acrt_get_process_end_policy 000000018005b03c     libucrt:win_policies.obj
 0001:0005a03c       $unwind$wcscat_s           000000018005b03c     libucrt:wcscat_s.obj
 0001:0005a03c       $unwind$__vcrt_uninitialize_locks 000000018005b03c     libvcruntime:locks.obj
 0001:0005a03c       $unwind$far_FarClock       000000018005b03c     service.obj
 0001:0005a044       $unwind$f_new              000000018005b044     bit64.obj
 0001:0005a054       $chain$0$f_new             000000018005b054     bit64.obj
 0001:0005a068       $chain$1$f_new             000000018005b068     bit64.obj
 0001:0005a078       $unwind$__dcrt_lowio_ensure_console_output_initialized 000000018005b078     libucrt:initcon.obj
 0001:0005a078       $unwind$isspace            000000018005b078     libucrt:_ctype.obj
 0001:0005a078       $unwind$far_FarMacroCallToLua 000000018005b078     luamacro.obj
 0001:0005a078       $unwind$?getSystemCP@@YAHH@Z 000000018005b078     libucrt:mbctype.obj
 0001:0005a078       $unwind$win_GetConsoleScreenBufferInfo 000000018005b078     win.obj
 0001:0005a078       $unwind$f_tostring         000000018005b078     bit64.obj
 0001:0005a078       $unwind$_isleadbyte_l      000000018005b078     libucrt:_wctype.obj
 0001:0005a078       $unwind$isdigit            000000018005b078     libucrt:_ctype.obj
 0001:0005a080       $unwind$io_lines           000000018005b080     uliolib51.obj
 0001:0005a080       $unwind$f_type             000000018005b080     bit64.obj
 0001:0005a088       $chain$0$f_type            000000018005b088     bit64.obj
 0001:0005a09c       $chain$1$f_type            000000018005b09c     bit64.obj
 0001:0005a0ac       $unwind$far_DialogRun      000000018005b0ac     service.obj
 0001:0005a0ac       $unwind$OptFlags           000000018005b0ac     service.obj
 0001:0005a0ac       $unwind$luaB_dofileW       000000018005b0ac     lflua.obj
 0001:0005a0ac       $unwind$?type_case_Z@?$output_processor@_WV?$string_output_adapter@_W@__crt_stdio_output@@V?$standard_base@_WV?$string_output_adapter@_W@__crt_stdio_output@@@2@@__crt_stdio_output@@AEAA_NXZ 000000018005b0ac     libucrt:output.obj
 0001:0005a0ac       $unwind$GetFarColor        000000018005b0ac     service.obj
 0001:0005a0ac       $unwind$LF_ProcessViewerEvent 000000018005b0ac     exported.obj
 0001:0005a0ac       $unwind$LF_ClosePanel      000000018005b0ac     exported.obj
 0001:0005a0ac       $unwind$?type_case_s@?$output_processor@_WV?$string_output_adapter@_W@__crt_stdio_output@@V?$standard_base@_WV?$string_output_adapter@_W@__crt_stdio_output@@@2@@__crt_stdio_output@@AEAA_NXZ 000000018005b0ac     libucrt:output.obj
 0001:0005a0ac       $unwind$utf8_enco          000000018005b0ac     slnunico.obj
 0001:0005a0ac       $unwind$LF_SetDirectory    000000018005b0ac     exported.obj
 0001:0005a0ac       $unwind$LF_SetFindList     000000018005b0ac     exported.obj
 0001:0005a0ac       $unwind$?type_case_n@?$output_processor@DV?$stream_output_adapter@D@__crt_stdio_output@@V?$standard_base@DV?$stream_output_adapter@D@__crt_stdio_output@@@2@@__crt_stdio_output@@AEAA_NXZ 000000018005b0ac     libucrt:output.obj
 0001:0005a0ac       $unwind$__vcrt_InitializeCriticalSectionEx 000000018005b0ac     libvcruntime:winapi_downlevel.obj
 0001:0005a0ac       $unwind$_DllMainCRTStartup 000000018005b0ac     LIBCMT:dll_dllmain.obj
 0001:0005a0ac       $unwind$PushDMParams       000000018005b0ac     service.obj
 0001:0005a0ac       $unwind$__acrt_stdio_flush_and_write_narrow_nolock 000000018005b0ac     libucrt:_flsbuf.obj
 0001:0005a0ac       $unwind$??R<lambda_96f4279ff90247a4c5c5d9824f56f8c1>@@QEBA_KXZ 000000018005b0ac     libucrt:fwrite.obj
 0001:0005a0ac       $unwind$uc_newindex        000000018005b0ac     lusercontrol.obj
 0001:0005a0ac       $unwind$fileerror          000000018005b0ac     uliolib51.obj
 0001:0005a0ac       $unwind$__acrt_stdio_free_tmpfile_name_buffers_nolock 000000018005b0ac     libucrt:tmpfile.obj
 0001:0005a0ac       $unwind$?type_case_n@?$output_processor@_WV?$string_output_adapter@_W@__crt_stdio_output@@V?$standard_base@_WV?$string_output_adapter@_W@__crt_stdio_output@@@2@@__crt_stdio_output@@AEAA_NXZ 000000018005b0ac     libucrt:output.obj
 0001:0005a0ac       $unwind$io_fclose          000000018005b0ac     uliolib51.obj
 0001:0005a0ac       $unwind$memcpy_s           000000018005b0ac     libucrt:input.obj
 0001:0005a0ac       $unwind$io_readline        000000018005b0ac     uliolib51.obj
 0001:0005a0ac       $unwind$push_flags_table   000000018005b0ac     flags.obj
 0001:0005a0ac       $unwind$?process@?$input_processor@DV?$stream_input_adapter@D@__crt_stdio_input@@@__crt_stdio_input@@QEAAHXZ 000000018005b0ac     libucrt:input.obj
 0001:0005a0ac       $unwind$__acrt_stdio_flush_nolock 000000018005b0ac     libucrt:fflush.obj
 0001:0005a0ac       $unwind$LF_PutFiles        000000018005b0ac     exported.obj
 0001:0005a0ac       $unwind$?process_string_specifier@?$input_processor@DV?$stream_input_adapter@D@__crt_stdio_input@@@__crt_stdio_input@@AEAA_NW4conversion_mode@2@@Z 000000018005b0ac     libucrt:input.obj
 0001:0005a0ac       $unwind$f_seek             000000018005b0ac     uliolib51.obj
 0001:0005a0ac       $unwind$?advance@?$format_string_parser@D@__crt_stdio_input@@QEAA_NXZ 000000018005b0ac     libucrt:input.obj
 0001:0005a0ac       $unwind$f_setvbuf          000000018005b0ac     uliolib51.obj
 0001:0005a0ac       $unwind$io_flush           000000018005b0ac     uliolib51.obj
 0001:0005a0ac       $unwind$win_wcscmp         000000018005b0ac     win.obj
 0001:0005a0ac       $unwind$?scan_scanset_range@?$format_string_parser@D@__crt_stdio_input@@AEAA_NXZ 000000018005b0ac     libucrt:input.obj
 0001:0005a0ac       $unwind$f_flush            000000018005b0ac     uliolib51.obj
 0001:0005a0ac       $unwind$__vcrt_getptd_noexit 000000018005b0ac     libvcruntime:per_thread_data.obj
 0001:0005a0ac       $unwind$luaopen_uio        000000018005b0ac     uliolib51.obj
 0001:0005a0ac       $unwind$memcpy_s           000000018005b0ac     libucrt:cfout.obj
 0001:0005a0ac       $unwind$__acrt_execute_initializers 000000018005b0ac     libucrt:shared_initialization.obj
 0001:0005a0ac       $unwind$loader_C           000000018005b0ac     uloadlib51.obj
 0001:0005a0ac       $unwind$ll_require         000000018005b0ac     uloadlib51.obj
 0001:0005a0ac       $unwind$__acrt_InitializeCriticalSectionEx 000000018005b0ac     libucrt:winapi_thunks.obj
 0001:0005a0ac       $unwind$?type_case_n@?$output_processor@DV?$string_output_adapter@D@__crt_stdio_output@@V?$standard_base@DV?$string_output_adapter@D@__crt_stdio_output@@@2@@__crt_stdio_output@@AEAA_NXZ 000000018005b0ac     libucrt:output.obj
 0001:0005a0ac       $unwind$get_env_flag       000000018005b0ac     service.obj
 0001:0005a0ac       $unwind$LF_ProcessPanelInput 000000018005b0ac     exported.obj
 0001:0005a0ac       $unwind$_exception_enabled 000000018005b0ac     libucrt:libm_error.obj
 0001:0005a0ac       $unwind$??$common_lseek_nolock@_J@@YA_JH_JH@Z 000000018005b0ac     libucrt:lseek.obj
 0001:0005a0ac       $unwind$PutVersionInfoToTable 000000018005b0ac     service.obj
 0001:0005a0ac       $unwind$FillEditorSelect   000000018005b0ac     service.obj
 0001:0005a0ac       $unwind$check_env_flag     000000018005b0ac     service.obj
 0001:0005a0ac       $unwind$?free_crt_array_internal@@YAXQEAPEBX_K@Z 000000018005b0ac     libucrt:inittime.obj
 0001:0005a0ac       $unwind$LF_ProcessHostFile 000000018005b0ac     exported.obj
 0001:0005a0ac       $unwind$LF_InitLuaState1   000000018005b0ac     service.obj
 0001:0005a0ac       $unwind$LF_Configure       000000018005b0ac     exported.obj
 0001:0005a0ac       $unwind$io_pclose          000000018005b0ac     uliolib51.obj
 0001:0005a0ac       $unwind$f_mod              000000018005b0ac     bit64.obj
 0001:0005a0bc       $unwind$_AddStringToCollector 000000018005b0bc     exported.obj
 0001:0005a0bc       $unwind$LF_GetFindData     000000018005b0bc     exported.obj
 0001:0005a0bc       $unwind$LF_MakeDirectory   000000018005b0bc     exported.obj
 0001:0005a0bc       $unwind$LF_Compare         000000018005b0bc     exported.obj
 0001:0005a0bc       $unwind$LF_GetFiles        000000018005b0bc     exported.obj
 0001:0005a0c8       $chain$0$LF_Compare        000000018005b0c8     exported.obj
 0001:0005a0dc       $chain$2$LF_Compare        000000018005b0dc     exported.obj
 0001:0005a0f0       $chain$3$LF_Compare        000000018005b0f0     exported.obj
 0001:0005a100       $unwind$LF_ProcessPanelEvent 000000018005b100     exported.obj
 0001:0005a100       $unwind$LF_DeleteFiles     000000018005b100     exported.obj
 0001:0005a110       $chain$0$LF_DeleteFiles    000000018005b110     exported.obj
 0001:0005a124       $chain$2$LF_DeleteFiles    000000018005b124     exported.obj
 0001:0005a138       $chain$3$LF_DeleteFiles    000000018005b138     exported.obj
 0001:0005a148       $chain$0$LF_GetFiles       000000018005b148     exported.obj
 0001:0005a15c       $chain$2$LF_GetFiles       000000018005b15c     exported.obj
 0001:0005a170       $chain$3$LF_GetFiles       000000018005b170     exported.obj
 0001:0005a180       $chain$0$LF_GetFindData    000000018005b180     exported.obj
 0001:0005a194       $chain$1$LF_GetFindData    000000018005b194     exported.obj
 0001:0005a1a4       $unwind$LF_GetGlobalInfo   000000018005b1a4     exported.obj
 0001:0005a1b8       $chain$1$LF_GetGlobalInfo  000000018005b1b8     exported.obj
 0001:0005a1cc       $chain$2$LF_GetGlobalInfo  000000018005b1cc     exported.obj
 0001:0005a1e0       $chain$3$LF_GetGlobalInfo  000000018005b1e0     exported.obj
 0001:0005a1f0       $chain$4$LF_GetGlobalInfo  000000018005b1f0     exported.obj
 0001:0005a200       $unwind$LF_GetOpenPanelInfo 000000018005b200     exported.obj
 0001:0005a20c       $chain$1$LF_GetOpenPanelInfo 000000018005b20c     exported.obj
 0001:0005a224       $chain$3$LF_GetOpenPanelInfo 000000018005b224     exported.obj
 0001:0005a23c       $chain$7$LF_GetOpenPanelInfo 000000018005b23c     exported.obj
 0001:0005a25c       $chain$8$LF_GetOpenPanelInfo 000000018005b25c     exported.obj
 0001:0005a26c       $chain$9$LF_GetOpenPanelInfo 000000018005b26c     exported.obj
 0001:0005a27c       $unwind$LF_GetPluginInfo   000000018005b27c     exported.obj
 0001:0005a288       $chain$0$LF_GetPluginInfo  000000018005b288     exported.obj
 0001:0005a29c       $chain$1$LF_GetPluginInfo  000000018005b29c     exported.obj
 0001:0005a2ac       $chain$0$LF_MakeDirectory  000000018005b2ac     exported.obj
 0001:0005a2c0       $chain$2$LF_MakeDirectory  000000018005b2c0     exported.obj
 0001:0005a2d4       $chain$3$LF_MakeDirectory  000000018005b2d4     exported.obj
 0001:0005a2e4       $unwind$LF_DoFile          000000018005b2e4     service.obj
 0001:0005a2e4       $unwind$win_MoveFile       000000018005b2e4     win.obj
 0001:0005a2e4       $unwind$FrsUserFunc        000000018005b2e4     service.obj
 0001:0005a2e4       $unwind$PushDNParams       000000018005b2e4     service.obj
 0001:0005a2e4       $unwind$start_capture      000000018005b2e4     slnunico.obj
 0001:0005a2e4       $unwind$LF_Open            000000018005b2e4     exported.obj
 0001:0005a2e4       $unwind$LF_ProcessDialogEvent 000000018005b2e4     exported.obj
 0001:0005a2e4       $unwind$timer_newindex     000000018005b2e4     service.obj
 0001:0005a2e4       $unwind$win_CreateDir      000000018005b2e4     win.obj
 0001:0005a2e4       $unwind$ll_loadfunc        000000018005b2e4     uloadlib51.obj
 0001:0005a2fc       $chain$0$LF_ProcessEditorEvent 000000018005b2fc     exported.obj
 0001:0005a310       $chain$1$LF_ProcessEditorEvent 000000018005b310     exported.obj
 0001:0005a320       $chain$0$LF_ProcessPanelEvent 000000018005b320     exported.obj
 0001:0005a334       $chain$2$LF_ProcessPanelEvent 000000018005b334     exported.obj
 0001:0005a348       $chain$3$LF_ProcessPanelEvent 000000018005b348     exported.obj
 0001:0005a358       $chain$0$LF_ProcessConsoleInput 000000018005b358     exported.obj
 0001:0005a36c       $chain$1$LF_ProcessConsoleInput 000000018005b36c     exported.obj
 0001:0005a37c       $unwind$LF_ProcessSynchroEvent 000000018005b37c     exported.obj
 0001:0005a37c       $unwind$capture_previous_context 000000018005b37c     LIBCMT:gs_report.obj
 0001:0005a388       $chain$1$LF_ProcessSynchroEvent 000000018005b388     exported.obj
 0001:0005a3a0       $chain$2$LF_ProcessSynchroEvent 000000018005b3a0     exported.obj
 0001:0005a3b4       $chain$3$LF_ProcessSynchroEvent 000000018005b3b4     exported.obj
 0001:0005a3c4       $chain$5$LF_ProcessSynchroEvent 000000018005b3c4     exported.obj
 0001:0005a3d8       $chain$6$LF_ProcessSynchroEvent 000000018005b3d8     exported.obj
 0001:0005a3e8       $unwind$?parse_int_from_format_string@?$output_processor@_WV?$string_output_adapter@_W@__crt_stdio_output@@V?$standard_base@_WV?$string_output_adapter@_W@__crt_stdio_output@@@2@@__crt_stdio_output@@AEAA_NQEAH@Z 000000018005b3e8     libucrt:output.obj
 0001:0005a3e8       $unwind$PutPluginMenuItemToTable 000000018005b3e8     service.obj
 0001:0005a3e8       $unwind$LF_GetContentData  000000018005b3e8     exported.obj
 0001:0005a3e8       $unwind$LF_GetContentFields 000000018005b3e8     exported.obj
 0001:0005a3fc       $chain$0$LF_GetContentFields 000000018005b3fc     exported.obj
 0001:0005a410       $chain$1$LF_GetContentFields 000000018005b410     exported.obj
 0001:0005a420       $chain$0$LF_GetContentData 000000018005b420     exported.obj
 0001:0005a434       $chain$1$LF_GetContentData 000000018005b434     exported.obj
 0001:0005a444       $chain$0$_AddStringToCollector 000000018005b444     exported.obj
 0001:0005a458       $chain$1$_AddStringToCollector 000000018005b458     exported.obj
 0001:0005a468       $unwind$CreateStringsArray 000000018005b468     exported.obj
 0001:0005a478       $chain$0$CreateStringsArray 000000018005b478     exported.obj
 0001:0005a48c       $chain$1$CreateStringsArray 000000018005b48c     exported.obj
 0001:0005a4a0       $chain$2$CreateStringsArray 000000018005b4a0     exported.obj
 0001:0005a4b0       $chain$3$CreateStringsArray 000000018005b4b0     exported.obj
 0001:0005a4c0       $unwind$FillFindData       000000018005b4c0     exported.obj
 0001:0005a4d4       $chain$1$FillFindData      000000018005b4d4     exported.obj
 0001:0005a4ec       $chain$2$FillFindData      000000018005b4ec     exported.obj
 0001:0005a4fc       $unwind$UpdateFileSelection 000000018005b4fc     exported.obj
 0001:0005a50c       $chain$0$UpdateFileSelection 000000018005b50c     exported.obj
 0001:0005a520       $chain$1$UpdateFileSelection 000000018005b520     exported.obj
 0001:0005a530       $unwind$RunDefaultScript   000000018005b530     exported.obj
 0001:0005a548       $chain$0$RunDefaultScript  000000018005b548     exported.obj
 0001:0005a55c       $chain$1$RunDefaultScript  000000018005b55c     exported.obj
 0001:0005a56c       $unwind$FillFarMacroCall_Callback 000000018005b56c     exported.obj
 0001:0005a578       $chain$0$FillFarMacroCall_Callback 000000018005b578     exported.obj
 0001:0005a58c       $chain$1$FillFarMacroCall_Callback 000000018005b58c     exported.obj
 0001:0005a59c       $unwind$FillFarMacroCall   000000018005b59c     exported.obj
 0001:0005a5ac       $chain$3$FillFarMacroCall  000000018005b5ac     exported.obj
 0001:0005a5cc       $chain$4$FillFarMacroCall  000000018005b5cc     exported.obj
 0001:0005a5dc       $unwind$getPluginMenuItems 000000018005b5dc     exported.obj
 0001:0005a5f4       $unwind$LF_Gsub            000000018005b5f4     lflua.obj
 0001:0005a614       $unwind$LF_LoadFile        000000018005b614     lflua.obj
 0001:0005a628       $chain$1$LF_LoadFile       000000018005b628     lflua.obj
 0001:0005a640       $chain$2$LF_LoadFile       000000018005b640     lflua.obj
 0001:0005a640       $chain$4$LF_LoadFile       000000018005b640     lflua.obj
 0001:0005a650       $chain$3$LF_LoadFile       000000018005b650     lflua.obj
 0001:0005a668       $unwind$getF               000000018005b668     lflua.obj
 0001:0005a678       $unwind$??$common_lseek_nolock@J@@YAJHJH@Z 000000018005b678     libucrt:lseek.obj
 0001:0005a678       $unwind$luaLF_FieldError   000000018005b678     util.obj
 0001:0005a678       $unwind$_invalid_parameter 000000018005b678     libucrt:invalid_parameter.obj
 0001:0005a678       $unwind$_wcsdup            000000018005b678     libucrt:wcsdup.obj
 0001:0005a678       $unwind$luaLF_SlotError    000000018005b678     util.obj
 0001:0005a678       $unwind$errfile            000000018005b678     lflua.obj
 0001:0005a68c       $unwind$check_regex_pattern 000000018005b68c     lregex.obj
 0001:0005a69c       $chain$1$check_regex_pattern 000000018005b69c     lregex.obj
 0001:0005a6b4       $chain$2$check_regex_pattern 000000018005b6b4     lregex.obj
 0001:0005a6c4       $unwind$_regex_gmatch_closure 000000018005b6c4     lregex.obj
 0001:0005a6d4       $chain$1$_regex_gmatch_closure 000000018005b6d4     lregex.obj
 0001:0005a6ec       $chain$2$_regex_gmatch_closure 000000018005b6ec     lregex.obj
 0001:0005a700       $chain$3$_regex_gmatch_closure 000000018005b700     lregex.obj
 0001:0005a710       $unwind$match              000000018005b710     slnunico.obj
 0001:0005a710       $unwind$_Gmatch            000000018005b710     lregex.obj
 0001:0005a728       $unwind$rx_find_match      000000018005b728     lregex.obj
 0001:0005a744       $unwind$rx_gsub            000000018005b744     lregex.obj
 0001:0005a760       $unwind$FL_PushParams      000000018005b760     luamacro.obj
 0001:0005a76c       $chain$0$FL_PushParams     000000018005b76c     luamacro.obj
 0001:0005a780       $chain$1$FL_PushParams     000000018005b780     luamacro.obj
 0001:0005a794       $chain$2$FL_PushParams     000000018005b794     luamacro.obj
 0001:0005a7a8       $chain$3$FL_PushParams     000000018005b7a8     luamacro.obj
 0001:0005a7b8       $chain$4$FL_PushParams     000000018005b7b8     luamacro.obj
 0001:0005a7c8       $chain$5$FL_PushParams     000000018005b7c8     luamacro.obj
 0001:0005a7d8       $unwind$Open_Luamacro      000000018005b7d8     luamacro.obj
 0001:0005a7ec       $chain$0$Open_Luamacro     000000018005b7ec     luamacro.obj
 0001:0005a800       $chain$1$Open_Luamacro     000000018005b800     luamacro.obj
 0001:0005a810       $unwind$far_MacroCallFar   000000018005b810     luamacro.obj
 0001:0005a820       $chain$1$far_MacroCallFar  000000018005b820     luamacro.obj
 0001:0005a838       $chain$3$far_MacroCallFar  000000018005b838     luamacro.obj
 0001:0005a850       $chain$4$far_MacroCallFar  000000018005b850     luamacro.obj
 0001:0005a860       $chain$5$far_MacroCallFar  000000018005b860     luamacro.obj
 0001:0005a870       $chain$0$far_FarMacroCallToLua 000000018005b870     luamacro.obj
 0001:0005a884       $chain$1$far_FarMacroCallToLua 000000018005b884     luamacro.obj
 0001:0005a894       $unwind$uc_index           000000018005b894     lusercontrol.obj
 0001:0005a8a4       $unwind$CreateRegKey       000000018005b8a4     reg.obj
 0001:0005a8ac       $unwind$??$parse_floating_point_write_result@N@__crt_strtox@@YA?AW4SLD_STATUS@@W4floating_point_parse_result@0@AEBUfloating_point_string@0@QEAN@Z 000000018005b8ac     libucrt:input.obj
 0001:0005a8ac       $unwind$??$parse_floating_point_write_result@M@__crt_strtox@@YA?AW4SLD_STATUS@@W4floating_point_parse_result@0@AEBUfloating_point_string@0@QEAM@Z 000000018005b8ac     libucrt:input.obj
 0001:0005a8ac       $unwind$_log10_special     000000018005b8ac     libucrt:log_special.obj
 0001:0005a8ac       $unwind$_wsopen_s          000000018005b8ac     libucrt:open.obj
 0001:0005a8ac       $unwind$_sopen_s           000000018005b8ac     libucrt:open.obj
 0001:0005a8ac       $unwind$_wdupenv_s         000000018005b8ac     libucrt:getenv.obj
 0001:0005a8ac       $unwind$_ui64toa_s         000000018005b8ac     libucrt:xtoa.obj
 0001:0005a8ac       $unwind$OpenRegKey         000000018005b8ac     reg.obj
 0001:0005a8ac       $unwind$?as_float@floating_point_value@__crt_strtox@@QEBAAEAMXZ 000000018005b8ac     libucrt:input.obj
 0001:0005a8ac       $unwind$wctomb_s           000000018005b8ac     libucrt:wctomb.obj
 0001:0005a8ac       $unwind$strtoull           000000018005b8ac     libucrt:strtox.obj
 0001:0005a8ac       $unwind$strtol             000000018005b8ac     libucrt:strtox.obj
 0001:0005a8ac       $unwind$wcstol             000000018005b8ac     libucrt:strtox.obj
 0001:0005a8ac       $unwind$fflush             000000018005b8ac     libucrt:fflush.obj
 0001:0005a8ac       $unwind$_invalid_parameter_noinfo 000000018005b8ac     libucrt:invalid_parameter.obj
 0001:0005a8ac       $unwind$check_utf8_string  000000018005b8ac     ustring.obj
 0001:0005a8ac       $unwind$utf8_to_utf16      000000018005b8ac     ustring.obj
 0001:0005a8ac       $unwind$push_utf8_string   000000018005b8ac     ustring.obj
 0001:0005a8ac       $unwind$PushAttrString     000000018005b8ac     ustring.obj
 0001:0005a8ac       $unwind$?as_double@floating_point_value@__crt_strtox@@QEBAAEANXZ 000000018005b8ac     libucrt:input.obj
 0001:0005a8ac       $unwind$fread              000000018005b8ac     libucrt:fread.obj
 0001:0005a8ac       $unwind$_wfreopen          000000018005b8ac     libucrt:freopen.obj
 0001:0005a8b4       $unwind$SetRegKeyStr       000000018005b8b4     reg.obj
 0001:0005a8b4       $unwind$SetRegKeyArr       000000018005b8b4     reg.obj
 0001:0005a8c4       $unwind$SetRegKeyDword     000000018005b8c4     reg.obj
 0001:0005a8d0       $unwind$__scrt_dllmain_uninitialize_critical 000000018005b8d0     LIBCMT:utility.obj
 0001:0005a8d0       $unwind$__scrt_dllmain_crt_thread_attach 000000018005b8d0     LIBCMT:utility.obj
 0001:0005a8d0       $unwind$__scrt_dllmain_crt_thread_detach 000000018005b8d0     LIBCMT:utility.obj
 0001:0005a8d0       $unwind$__vcrt_initialize  000000018005b8d0     libvcruntime:initialization.obj
 0001:0005a8d0       $unwind$__vcrt_uninitialize 000000018005b8d0     libvcruntime:initialization.obj
 0001:0005a8d0       $unwind$__vcrt_uninitialize_critical 000000018005b8d0     libvcruntime:initialization.obj
 0001:0005a8d0       $unwind$__scrt_acquire_startup_lock 000000018005b8d0     LIBCMT:utility.obj
 0001:0005a8d0       $unwind$__scrt_initialize_default_local_stdio_options 000000018005b8d0     LIBCMT:default_local_stdio_options.obj
 0001:0005a8d0       $unwind$__vcrt_thread_attach 000000018005b8d0     libvcruntime:initialization.obj
 0001:0005a8d0       $unwind$__acrt_update_thread_multibyte_data 000000018005b8d0     libucrt:mbctype.obj
 0001:0005a8d0       $unwind$__acrt_initialize_multibyte 000000018005b8d0     libucrt:mbctype.obj
 0001:0005a8d0       $unwind$_wcsnicoll         000000018005b8d0     libucrt:wcsnicol.obj
 0001:0005a8d0       $unwind$fegetround         000000018005b8d0     libucrt:fegetround.obj
 0001:0005a8d0       $unwind$?dllmain_crt_dispatch@@YAHQEAUHINSTANCE__@@KQEAX@Z 000000018005b8d0     LIBCMT:dll_dllmain.obj
 0001:0005a8d0       $unwind$__acrt_initialize_command_line 000000018005b8d0     libucrt:argv_data.obj
 0001:0005a8d0       $unwind$__acrt_uninitialize_tmpfile 000000018005b8d0     libucrt:rmtmp.obj
 0001:0005a8d0       $unwind$__vcrt_thread_detach 000000018005b8d0     libvcruntime:initialization.obj
 0001:0005a8d0       $unwind$__report_rangecheckfailure 000000018005b8d0     LIBCMT:gs_report.obj
 0001:0005a8d0       $unwind$__acrt_initialize_heap 000000018005b8d0     libucrt:heap_handle.obj
 0001:0005a8d0       $unwind$__vcrt_initialize_ptd 000000018005b8d0     libvcruntime:per_thread_data.obj
 0001:0005a8d0       $unwind$__vcrt_uninitialize_ptd 000000018005b8d0     libvcruntime:per_thread_data.obj
 0001:0005a8d0       $unwind$__dcrt_terminate_console_output 000000018005b8d0     libucrt:initcon.obj
 0001:0005a8d0       $unwind$__vcrt_freefls     000000018005b8d0     libvcruntime:per_thread_data.obj
 0001:0005a8d0       $unwind$tmpfile            000000018005b8d0     libucrt:tmpfile.obj
 0001:0005a8d0       $unwind$GetPluginData      000000018005b8d0     service.obj
 0001:0005a8d0       $unwind$?validate_stream_is_ansi_if_required@?$__acrt_stdio_char_traits@D@@SA_NQEAU_iobuf@@@Z 000000018005b8d0     libucrt:output.obj
 0001:0005a8d0       $unwind$__scrt_dllmain_before_initialize_c 000000018005b8d0     LIBCMT:utility.obj
 0001:0005a8d0       $unwind$DllMain            000000018005b8d0     service.obj
 0001:0005a8d0       $unwind$?state_case_normal_tchar@?$output_processor@DV?$string_output_adapter@D@__crt_stdio_output@@V?$standard_base@DV?$string_output_adapter@D@__crt_stdio_output@@@2@@__crt_stdio_output@@AEAA_ND@Z 000000018005b8d0     libucrt:output.obj
 0001:0005a8d0       $unwind$tolower            000000018005b8d0     libucrt:tolower_toupper.obj
 0001:0005a8d0       $unwind$?state_case_size@?$output_processor@DV?$string_output_adapter@D@__crt_stdio_output@@V?$standard_base@DV?$string_output_adapter@D@__crt_stdio_output@@@2@@__crt_stdio_output@@AEAA_NXZ 000000018005b8d0     libucrt:output.obj
 0001:0005a8d0       $unwind$__acrt_release_locale_ref 000000018005b8d0     libucrt:locale_refcounting.obj
 0001:0005a8d0       $unwind$?state_case_size@?$output_processor@_WV?$string_output_adapter@_W@__crt_stdio_output@@V?$standard_base@_WV?$string_output_adapter@_W@__crt_stdio_output@@@2@@__crt_stdio_output@@AEAA_NXZ 000000018005b8d0     libucrt:output.obj
 0001:0005a8d0       $unwind$_errno             000000018005b8d0     libucrt:errno.obj
 0001:0005a8d0       $unwind$__doserrno         000000018005b8d0     libucrt:errno.obj
 0001:0005a8d0       $unwind$__pctype_func      000000018005b8d0     libucrt:ctype.obj
 0001:0005a8d0       $unwind$dir_exist          000000018005b8d0     service.obj
 0001:0005a8d0       $unwind$_fileno            000000018005b8d0     libucrt:fileno.obj
 0001:0005a8d0       $unwind$_isatty            000000018005b8d0     libucrt:isatty.obj
 0001:0005a8d0       $unwind$??$uninitialize_environment_internal@_W@@YAXAEAPEAPEA_W@Z 000000018005b8d0     libucrt:environment_initialization.obj
 0001:0005a8d0       $unwind$?initialize_multibyte@@YAHXZ 000000018005b8d0     libucrt:multibyte_initializer.obj
 0001:0005a8d0       $unwind$feof               000000018005b8d0     libucrt:feoferr.obj
 0001:0005a8d0       $unwind$ferror             000000018005b8d0     libucrt:feoferr.obj
 0001:0005a8d0       $unwind$_get_osfhandle     000000018005b8d0     libucrt:osfinfo.obj
 0001:0005a8d0       $unwind$??$uninitialize_environment_internal@D@@YAXAEAPEAPEAD@Z 000000018005b8d0     libucrt:environment_initialization.obj
 0001:0005a8d0       $unwind$_wcsnicmp          000000018005b8d0     libucrt:wcsnicmp.obj
 0001:0005a8d0       $unwind$__scrt_dllmain_after_initialize_c 000000018005b8d0     LIBCMT:utility.obj
 0001:0005a8d0       $unwind$__acrt_uninitialize_ptd 000000018005b8d0     libucrt:per_thread_data.obj
 0001:0005a8d0       $unwind$win_IsProcess64bit 000000018005b8d0     win.obj
 0001:0005a8d0       $unwind$__acrt_DownlevelLocaleNameToLCID 000000018005b8d0     libucrt:lcidtoname_downlevel.obj
 0001:0005a8d0       $unwind$_msize_base        000000018005b8d0     libucrt:msize.obj
 0001:0005a8d0       $unwind$_invoke_watson     000000018005b8d0     libucrt:invalid_parameter.obj
 0001:0005a8d0       $unwind$_get_fmode         000000018005b8d0     libucrt:setmode.obj
 0001:0005a8d0       $unwind$_fgetc_nolock      000000018005b8d0     libucrt:fgetc.obj
 0001:0005a8d0       $unwind$?state_case_size@?$output_processor@DV?$stream_output_adapter@D@__crt_stdio_output@@V?$standard_base@DV?$stream_output_adapter@D@__crt_stdio_output@@@2@@__crt_stdio_output@@AEAA_NXZ 000000018005b8d0     libucrt:output.obj
 0001:0005a8d0       $unwind$abort              000000018005b8d0     libucrt:abort.obj
 0001:0005a8d0       $unwind$_set_errno_from_matherr 000000018005b8d0     libucrt:fpexcept.obj
 0001:0005a8d0       $unwind$_wcsicmp           000000018005b8d0     libucrt:wcsicmp.obj
 0001:0005a8d0       $unwind$__acrt_initialize_ptd 000000018005b8d0     libucrt:per_thread_data.obj
 0001:0005a8d0       $unwind$win_GetVirtualKeys 000000018005b8d0     win.obj
 0001:0005a8d0       $unwind$__scrt_dllmain_uninitialize_c 000000018005b8d0     LIBCMT:utility.obj
 0001:0005a8d0       $unwind$uninitialize_allocated_io_buffers 000000018005b8d0     libucrt:initialization.obj
 0001:0005a8d0       $unwind$uninitialize_environment 000000018005b8d0     libucrt:initialization.obj
 0001:0005a8d0       $unwind$ustring_Sleep      000000018005b8d0     ustring.obj
 0001:0005a8d0       $unwind$initialize_c       000000018005b8d0     libucrt:initialization.obj
 0001:0005a8d0       $unwind$__acrt_thread_detach 000000018005b8d0     libucrt:initialization.obj
 0001:0005a8d0       $unwind$__acrt_thread_attach 000000018005b8d0     libucrt:initialization.obj
 0001:0005a8d0       $unwind$_statfp            000000018005b8d0     libucrt:fpctrl.obj
 0001:0005a8d0       $unwind$far_DialogFree     000000018005b8d0     service.obj
 0001:0005a8d0       $unwind$__dcrt_uninitialize_environments_nolock 000000018005b8d0     libucrt:environment_initialization.obj
 0001:0005a8d0       $unwind$__acrt_uninitialize_critical 000000018005b8d0     libucrt:initialization.obj
 0001:0005a8d0       $unwind$far_SubscribeDialogDrawEvents 000000018005b8d0     service.obj
 0001:0005a8d0       $unwind$__acrt_uninitialize 000000018005b8d0     libucrt:initialization.obj
 0001:0005a8d0       $unwind$__dcrt_get_or_create_wide_environment_nolock 000000018005b8d0     libucrt:environment_initialization.obj
 0001:0005a8d0       $unwind$__acrt_AreFileApisANSI 000000018005b8d0     libucrt:winapi_thunks.obj
 0001:0005a8d0       $unwind$writer             000000018005b8d0     slnunico.obj
 0001:0005a8d0       $unwind$__GSHandlerCheck   000000018005b8d0     LIBCMT:_gshandler_.obj
 0001:0005a8d8       $unwind$LF_DlgProc         000000018005b8d8     service.obj
 0001:0005a8e8       $chain$1$LF_DlgProc        000000018005b8e8     service.obj
 0001:0005a900       $chain$2$LF_DlgProc        000000018005b900     service.obj
 0001:0005a910       $unwind$LF_Message         000000018005b910     service.obj
 0001:0005a92c       $unwind$LF_RunLuafarInit   000000018005b92c     service.obj
 0001:0005a938       $unwind$PushPanelItem      000000018005b938     service.obj
 0001:0005a944       $chain$0$PushPanelItem     000000018005b944     service.obj
 0001:0005a958       $chain$1$PushPanelItem     000000018005b958     service.obj
 0001:0005a968       $chain$3$PushPanelItem     000000018005b968     service.obj
 0001:0005a980       $chain$4$PushPanelItem     000000018005b980     service.obj
 0001:0005a990       $unwind$PushPanelItems     000000018005b990     service.obj
 0001:0005a9a0       $chain$3$PushPanelItems    000000018005b9a0     service.obj
 0001:0005a9c0       $chain$4$PushPanelItems    000000018005b9c0     service.obj
 0001:0005a9d0       $unwind$luaopen_far        000000018005b9d0     service.obj
 0001:0005a9d0       $unwind$panel_GetCmdLine   000000018005b9d0     service.obj
 0001:0005a9d0       $unwind$far_GetPluginInformation 000000018005b9d0     service.obj
 0001:0005a9d0       $unwind$NewDialogData      000000018005b9d0     service.obj
 0001:0005a9d0       $unwind$viewer_GetFileName 000000018005b9d0     service.obj
 0001:0005a9d0       $unwind$editor_GetFileName 000000018005b9d0     service.obj
 0001:0005a9d0       $unwind$far_GetPathRoot    000000018005b9d0     service.obj
 0001:0005a9d0       $unwind$far_MkLink         000000018005b9d0     service.obj
 0001:0005a9d0       $unwind$far_ShowHelp       000000018005b9d0     service.obj
 0001:0005a9d0       $unwind$editor_GetTitle    000000018005b9d0     service.obj
 0001:0005a9e4       $chain$0$DllMain           000000018005b9e4     service.obj
 0001:0005a9f8       $chain$1$DllMain           000000018005b9f8     service.obj
 0001:0005aa08       $unwind$GetFlagCombination 000000018005ba08     service.obj
 0001:0005aa20       $unwind$plugin_load        000000018005ba20     service.obj
 0001:0005aa20       $unwind$ConvertLuaValue    000000018005ba20     service.obj
 0001:0005aa34       $unwind$far_GetFileOwner   000000018005ba34     service.obj
 0001:0005aa48       $unwind$AddMacroData_gc    000000018005ba48     service.obj
 0001:0005aa48       $unwind$ustring_sub        000000018005ba48     ustring.obj
 0001:0005aa48       $unwind$utf8_valid         000000018005ba48     slnunico.obj
 0001:0005aa48       $unwind$editor_InsertText  000000018005ba48     service.obj
 0001:0005aa48       $unwind$far_MacroDelete    000000018005ba48     service.obj
 0001:0005aa48       $unwind$panel_SetCmdLine   000000018005ba48     service.obj
 0001:0005aa48       $unwind$panel_SetCmdLinePos 000000018005ba48     service.obj
 0001:0005aa48       $unwind$editor_DeleteSessionBookmark 000000018005ba48     service.obj
 0001:0005aa48       $unwind$gmatch             000000018005ba48     slnunico.obj
 0001:0005aa48       $unwind$editor_SetTitle    000000018005ba48     service.obj
 0001:0005aa48       $unwind$panel_InsertCmdLine 000000018005ba48     service.obj
 0001:0005aa48       $unwind$far_LStricmp       000000018005ba48     service.obj
 0001:0005aa48       $unwind$far_PluginStartupInfo 000000018005ba48     service.obj
 0001:0005aa48       $unwind$panel_ClosePanel   000000018005ba48     service.obj
 0001:0005aa48       $unwind$panel_SetUserScreen 000000018005ba48     service.obj
 0001:0005aa48       $unwind$far_MkTemp         000000018005ba48     service.obj
 0001:0005aa48       $unwind$panel_SetActivePanel 000000018005ba48     service.obj
 0001:0005aa48       $unwind$panel_GetUserScreen 000000018005ba48     service.obj
 0001:0005aa58       $unwind$far_CreateFileFilter 000000018005ba58     service.obj
 0001:0005aa58       $unwind$far_GetCurrentDirectory 000000018005ba58     service.obj
 0001:0005aa58       $unwind$far_LStrnicmp      000000018005ba58     service.obj
 0001:0005aa6c       $unwind$editor_GetInfo     000000018005ba6c     service.obj
 0001:0005aa7c       $chain$2$editor_GetInfo    000000018005ba7c     service.obj
 0001:0005aa98       $chain$3$editor_GetInfo    000000018005ba98     service.obj
 0001:0005aaac       $chain$4$editor_GetInfo    000000018005baac     service.obj
 0001:0005aabc       $chain$5$editor_GetInfo    000000018005babc     service.obj
 0001:0005aad0       $unwind$_EditorGetString   000000018005bad0     service.obj
 0001:0005aaec       $unwind$_EditorSetString   000000018005baec     service.obj
 0001:0005aafc       $unwind$far_FindPlugin     000000018005bafc     service.obj
 0001:0005aafc       $unwind$editor_InsertString 000000018005bafc     service.obj
 0001:0005aafc       $unwind$editor_ExpandTabs  000000018005bafc     service.obj
 0001:0005aafc       $unwind$far_LUpperBuf      000000018005bafc     service.obj
 0001:0005aafc       $unwind$far_LLowerBuf      000000018005bafc     service.obj
 0001:0005ab0c       $unwind$_EditorInsertText  000000018005bb0c     service.obj
 0001:0005ab1c       $unwind$strerror           000000018005bb1c     libucrt:strerror.obj
 0001:0005ab1c       $unwind$editor_UndoRedo    000000018005bb1c     service.obj
 0001:0005ab1c       $unwind$EnumCodePagesProc  000000018005bb1c     ustring.obj
 0001:0005ab1c       $unwind$?convert_hexadecimal_string_to_floating_type_common@__crt_strtox@@YA?AW4SLD_STATUS@@AEBUfloating_point_string@1@AEBVfloating_point_value@1@@Z 000000018005bb1c     libucrt:input.obj
 0001:0005ab1c       $unwind$PutWStrToTable     000000018005bb1c     ustring.obj
 0001:0005ab28       $unwind$FillKeyBarTitles   000000018005bb28     service.obj
 0001:0005ab3c       $chain$1$FillKeyBarTitles  000000018005bb3c     service.obj
 0001:0005ab54       $chain$2$FillKeyBarTitles  000000018005bb54     service.obj
 0001:0005ab64       $unwind$SetKeyBar          000000018005bb64     service.obj
 0001:0005ab7c       $unwind$editor_SetParam    000000018005bb7c     service.obj
 0001:0005ab90       $unwind$editor_SetPosition 000000018005bb90     service.obj
 0001:0005aba0       $unwind$PushBookmarks      000000018005bba0     service.obj
 0001:0005abb4       $chain$0$PushBookmarks     000000018005bbb4     service.obj
 0001:0005abc8       $chain$1$PushBookmarks     000000018005bbc8     service.obj
 0001:0005abd8       $unwind$editor_Select      000000018005bbd8     service.obj
 0001:0005abe8       $unwind$editor_GetSelection 000000018005bbe8     service.obj
 0001:0005ac04       $unwind$_EditorTabConvert  000000018005bc04     service.obj
 0001:0005ac18       $unwind$editor_AddColor    000000018005bc18     service.obj
 0001:0005ac2c       $unwind$editor_DelColor    000000018005bc2c     service.obj
 0001:0005ac40       $unwind$editor_GetColor    000000018005bc40     service.obj
 0001:0005ac50       $unwind$editor_SaveFile    000000018005bc50     service.obj
 0001:0005ac50       $unwind$viewer_Select      000000018005bc50     service.obj
 0001:0005ac50       $unwind$panel_SetCmdLineSelection 000000018005bc50     service.obj
 0001:0005ac60       $unwind$Settings_delete    000000018005bc60     service.obj
 0001:0005ac60       $unwind$_mbsdec_l          000000018005bc60     libucrt:mbsdec.obj
 0001:0005ac60       $unwind$viewer_SetMode     000000018005bc60     service.obj
 0001:0005ac60       $unwind$editor_ProcessInput 000000018005bc60     service.obj
 0001:0005ac60       $unwind$win_ExtractKey     000000018005bc60     win.obj
 0001:0005ac60       $unwind$LF_Error           000000018005bc60     service.obj
 0001:0005ac60       $unwind$panel_GetCmdLineSelection 000000018005bc60     service.obj
 0001:0005ac60       $unwind$editor_SubscribeChangeEvent 000000018005bc60     service.obj
 0001:0005ac60       $unwind$win_ExtractKeyEx   000000018005bc60     win.obj
 0001:0005ac60       $unwind$editor_ReadInput   000000018005bc60     service.obj
 0001:0005ac60       $unwind$far_NameToInputRecord 000000018005bc60     service.obj
 0001:0005ac60       $unwind$Settings_opensubkey 000000018005bc60     service.obj
 0001:0005ac60       $unwind$_strupr_s_l        000000018005bc60     libucrt:strupr.obj
 0001:0005ac6c       $unwind$far_Menu           000000018005bc6c     service.obj
 0001:0005ac88       $unwind$far_Message        000000018005bc88     service.obj
 0001:0005aca4       $unwind$panel_GetPanelInfo 000000018005bca4     service.obj
 0001:0005acb4       $chain$0$panel_GetPanelInfo 000000018005bcb4     service.obj
 0001:0005acc8       $chain$1$panel_GetPanelInfo 000000018005bcc8     service.obj
 0001:0005acd8       $unwind$get_panel_item     000000018005bcd8     service.obj
 0001:0005acec       $unwind$get_string_info    000000018005bcec     service.obj
 0001:0005ad04       $unwind$panel_RedrawPanel  000000018005bd04     service.obj
 0001:0005ad18       $unwind$SetPanelBooleanProperty 000000018005bd18     service.obj
 0001:0005ad18       $unwind$SetPanelIntegerProperty 000000018005bd18     service.obj
 0001:0005ad18       $unwind$g_write            000000018005bd18     uliolib51.obj
 0001:0005ad18       $unwind$truncstring        000000018005bd18     service.obj
 0001:0005ad2c       $unwind$panel_GetPanelDirectory 000000018005bd2c     service.obj
 0001:0005ad40       $unwind$panel_SetPanelDirectory 000000018005bd40     service.obj
 0001:0005ad50       $unwind$ChangePanelSelection 000000018005bd50     service.obj
 0001:0005ad64       $chain$1$ChangePanelSelection 000000018005bd64     service.obj
 0001:0005ad7c       $chain$2$ChangePanelSelection 000000018005bd7c     service.obj
 0001:0005ad8c       $unwind$far_GetDirList     000000018005bd8c     service.obj
 0001:0005ad98       $chain$0$far_GetDirList    000000018005bd98     service.obj
 0001:0005adac       $chain$6$far_GetDirList    000000018005bdac     service.obj
 0001:0005add4       $chain$7$far_GetDirList    000000018005bdd4     service.obj
 0001:0005ade4       $chain$8$far_GetDirList    000000018005bde4     service.obj
 0001:0005adf4       $unwind$far_GetPluginDirList 000000018005bdf4     service.obj
 0001:0005ae00       $unwind$far_RestoreScreen  000000018005be00     service.obj
 0001:0005ae0c       $unwind$far_SaveScreen     000000018005be0c     service.obj
 0001:0005ae24       $unwind$CreateList         000000018005be24     service.obj
 0001:0005ae34       $chain$2$CreateList        000000018005be34     service.obj
 0001:0005ae50       $chain$3$CreateList        000000018005be50     service.obj
 0001:0005ae60       $unwind$far_ConvertPath    000000018005be60     service.obj
 0001:0005ae60       $unwind$SetFarDialogItem   000000018005be60     service.obj
 0001:0005ae78       $unwind$PushDlgItem        000000018005be78     service.obj
 0001:0005ae8c       $chain$1$PushDlgItem       000000018005be8c     service.obj
 0001:0005aea0       $chain$2$PushDlgItem       000000018005bea0     service.obj
 0001:0005aeb0       $unwind$PushDlgItemNum     000000018005beb0     service.obj
 0001:0005aec8       $unwind$SetDlgItem         000000018005bec8     service.obj
 0001:0005aee0       $unwind$far_SendDlgMessage 000000018005bee0     service.obj
 0001:0005aefc       $unwind$ProcessDNResult    000000018005befc     service.obj
 0001:0005af0c       $chain$0$ProcessDNResult   000000018005bf0c     service.obj
 0001:0005af20       $chain$1$ProcessDNResult   000000018005bf20     service.obj
 0001:0005af34       $chain$2$ProcessDNResult   000000018005bf34     service.obj
 0001:0005af44       $chain$3$ProcessDNResult   000000018005bf44     service.obj
 0001:0005af54       $unwind$far_DialogInit     000000018005bf54     service.obj
 0001:0005af6c       $chain$0$far_DialogInit    000000018005bf6c     service.obj
 0001:0005af80       $chain$1$far_DialogInit    000000018005bf80     service.obj
 0001:0005af90       $unwind$far_SetDlgItem     000000018005bf90     service.obj
 0001:0005af90       $unwind$far_GetDlgItem     000000018005bf90     service.obj
 0001:0005afa4       $unwind$far_InputBox       000000018005bfa4     service.obj
 0001:0005afa4       $unwind$editor_Editor      000000018005bfa4     service.obj
 0001:0005afbc       $unwind$viewer_Viewer      000000018005bfbc     service.obj
 0001:0005afd4       $unwind$viewer_GetInfo     000000018005bfd4     service.obj
 0001:0005afe0       $chain$1$viewer_GetInfo    000000018005bfe0     service.obj
 0001:0005aff8       $chain$2$viewer_GetInfo    000000018005bff8     service.obj
 0001:0005b00c       $chain$3$viewer_GetInfo    000000018005c00c     service.obj
 0001:0005b01c       $chain$4$viewer_GetInfo    000000018005c01c     service.obj
 0001:0005b02c       $unwind$viewer_SetPosition 000000018005c02c     service.obj
 0001:0005b034       $chain$2$viewer_SetPosition 000000018005c034     service.obj
 0001:0005b050       $chain$3$viewer_SetPosition 000000018005c050     service.obj
 0001:0005b060       $unwind$far_Text           000000018005c060     service.obj
 0001:0005b074       $chain$1$far_CopyToClipboard 000000018005c074     service.obj
 0001:0005b08c       $chain$2$far_CopyToClipboard 000000018005c08c     service.obj
 0001:0005b09c       $unwind$far_PasteFromClipboard 000000018005c09c     service.obj
 0001:0005b0b0       $unwind$pusherrorcode      000000018005c0b0     ustring.obj
 0001:0005b0b0       $unwind$far_InputRecordToName 000000018005c0b0     service.obj
 0001:0005b0c0       $unwind$far_ProcessName    000000018005c0c0     service.obj
 0001:0005b0d4       $chain$1$far_ProcessName   000000018005c0d4     service.obj
 0001:0005b0e8       $chain$2$far_ProcessName   000000018005c0e8     service.obj
 0001:0005b0fc       $chain$3$far_ProcessName   000000018005c0fc     service.obj
 0001:0005b10c       $chain$6$far_ProcessName   000000018005c10c     service.obj
 0001:0005b10c       $chain$4$far_ProcessName   000000018005c10c     service.obj
 0001:0005b11c       $chain$5$far_ProcessName   000000018005c11c     service.obj
 0001:0005b130       $unwind$far_GetReparsePointInfo 000000018005c130     service.obj
 0001:0005b140       $chain$0$far_GetReparsePointInfo 000000018005c140     service.obj
 0001:0005b154       $chain$1$far_GetReparsePointInfo 000000018005c154     service.obj
 0001:0005b164       $unwind$far_RecursiveSearch 000000018005c164     service.obj
 0001:0005b164       $unwind$?process_integer_specifier@?$input_processor@DV?$stream_input_adapter@D@__crt_stdio_input@@@__crt_stdio_input@@AEAA_NI_N@Z 000000018005c164     libucrt:input.obj
 0001:0005b178       $unwind$far_AdvControl     000000018005c178     service.obj
 0001:0005b198       $chain$0$far_AdvControl    000000018005c198     service.obj
 0001:0005b1ac       $chain$1$far_AdvControl    000000018005c1ac     service.obj
 0001:0005b1bc       $unwind$far_MacroLoadAll   000000018005c1bc     service.obj
 0001:0005b1bc       $unwind$capture_current_context 000000018005c1bc     LIBCMT:gs_report.obj
 0001:0005b1c8       $chain$0$far_MacroLoadAll  000000018005c1c8     service.obj
 0001:0005b1dc       $chain$1$far_MacroLoadAll  000000018005c1dc     service.obj
 0001:0005b1ec       $unwind$MacroSendString    000000018005c1ec     service.obj
 0001:0005b200       $unwind$far_MacroGetLastError 000000018005c200     service.obj
 0001:0005b210       $chain$0$far_MacroGetLastError 000000018005c210     service.obj
 0001:0005b224       $chain$1$far_MacroGetLastError 000000018005c224     service.obj
 0001:0005b234       $unwind$MacroAddCallback   000000018005c234     service.obj
 0001:0005b248       $unwind$far_MacroAdd       000000018005c248     service.obj
 0001:0005b25c       $unwind$far_MacroExecute   000000018005c25c     service.obj
 0001:0005b264       $chain$2$far_MacroExecute  000000018005c264     service.obj
 0001:0005b280       $chain$3$far_MacroExecute  000000018005c280     service.obj
 0001:0005b290       $unwind$far_MakeMenuItems  000000018005c290     service.obj
 0001:0005b29c       $chain$1$far_MakeMenuItems 000000018005c29c     service.obj
 0001:0005b2b4       $chain$5$far_MakeMenuItems 000000018005c2b4     service.obj
 0001:0005b2d4       $chain$6$far_MakeMenuItems 000000018005c2d4     service.obj
 0001:0005b2e4       $chain$8$far_MakeMenuItems 000000018005c2e4     service.obj
 0001:0005b2fc       $chain$9$far_MakeMenuItems 000000018005c2fc     service.obj
 0001:0005b30c       $unwind$??$parse_floating_point_possible_nan_is_ind@DV?$input_adapter_character_source@V?$stream_input_adapter@D@__crt_stdio_input@@@__crt_strtox@@@__crt_strtox@@YA_NAEADAEAV?$input_adapter_character_source@V?$stream_input_adapter@D@__crt_stdio_input@@@0@@Z 000000018005c30c     libucrt:input.obj
 0001:0005b30c       $unwind$_chsize_nolock     000000018005c30c     libucrt:chsize.obj
 0001:0005b30c       $unwind$NewVirtualKeyTable 000000018005c30c     service.obj
 0001:0005b30c       $unwind$gmatch_aux         000000018005c30c     slnunico.obj
 0001:0005b30c       $unwind$??$parse_floating_point_possible_nan_is_snan@DV?$input_adapter_character_source@V?$stream_input_adapter@D@__crt_stdio_input@@@__crt_strtox@@@__crt_strtox@@YA_NAEADAEAV?$input_adapter_character_source@V?$stream_input_adapter@D@__crt_stdio_input@@@0@@Z 000000018005c30c     libucrt:input.obj
 0001:0005b30c       $unwind$?type_case_integer@?$output_processor@_WV?$string_output_adapter@_W@__crt_stdio_output@@V?$standard_base@_WV?$string_output_adapter@_W@__crt_stdio_output@@@2@@__crt_stdio_output@@AEAA_NI_N@Z 000000018005c30c     libucrt:output.obj
 0001:0005b30c       $unwind$??$parse_floating_point_possible_infinity@DV?$input_adapter_character_source@V?$stream_input_adapter@D@__crt_stdio_input@@@__crt_strtox@@_K@__crt_strtox@@YA?AW4floating_point_parse_result@0@AEADAEAV?$input_adapter_character_source@V?$stream_input_adapter@D@__crt_stdio_input@@@0@_K@Z 000000018005c30c     libucrt:input.obj
 0001:0005b30c       $unwind$?type_case_integer@?$output_processor@DV?$string_output_adapter@D@__crt_stdio_output@@V?$standard_base@DV?$string_output_adapter@D@__crt_stdio_output@@@2@@__crt_stdio_output@@AEAA_NI_N@Z 000000018005c30c     libucrt:output.obj
 0001:0005b30c       $unwind$?type_case_integer@?$output_processor@DV?$stream_output_adapter@D@__crt_stdio_output@@V?$standard_base@DV?$stream_output_adapter@D@__crt_stdio_output@@@2@@__crt_stdio_output@@AEAA_NI_N@Z 000000018005c30c     libucrt:output.obj
 0001:0005b30c       $unwind$io_open            000000018005c30c     uliolib51.obj
 0001:0005b324       $unwind$filefilter_IsFileInFilter 000000018005c324     service.obj
 0001:0005b338       $chain$0$PutPluginMenuItemToTable 000000018005c338     service.obj
 0001:0005b34c       $chain$1$PutPluginMenuItemToTable 000000018005c34c     service.obj
 0001:0005b35c       $unwind$far_GetPlugins     000000018005c35c     service.obj
 0001:0005b368       $chain$1$far_GetPlugins    000000018005c368     service.obj
 0001:0005b380       $chain$2$far_GetPlugins    000000018005c380     service.obj
 0001:0005b394       $chain$3$far_GetPlugins    000000018005c394     service.obj
 0001:0005b3a4       $chain$4$far_GetPlugins    000000018005c3a4     service.obj
 0001:0005b3b4       $unwind$far_IsPluginLoaded 000000018005c3b4     service.obj
 0001:0005b3c4       $chain$0$far_IsPluginLoaded 000000018005c3c4     service.obj
 0001:0005b3d8       $chain$1$far_IsPluginLoaded 000000018005c3d8     service.obj
 0001:0005b3e8       $unwind$far_XLat           000000018005c3e8     service.obj
 0001:0005b3fc       $unwind$far_FormatFileSize 000000018005c3fc     service.obj
 0001:0005b414       $unwind$far_Timer          000000018005c414     service.obj
 0001:0005b42c       $unwind$timer_Close        000000018005c42c     service.obj
 0001:0005b42c       $unwind$iswctype           000000018005c42c     libucrt:iswctype.obj
 0001:0005b42c       $unwind$timer_gc           000000018005c42c     service.obj
 0001:0005b438       $chain$0$timer_Close       000000018005c438     service.obj
 0001:0005b44c       $chain$1$timer_Close       000000018005c44c     service.obj
 0001:0005b45c       $chain$0$timer_gc          000000018005c45c     service.obj
 0001:0005b470       $chain$1$timer_gc          000000018005c470     service.obj
 0001:0005b480       $unwind$far_CreateSettings 000000018005c480     service.obj
 0001:0005b490       $unwind$Settings_get       000000018005c490     service.obj
 0001:0005b490       $unwind$Settings_set       000000018005c490     service.obj
 0001:0005b49c       $unwind$Settings_createsubkey 000000018005c49c     service.obj
 0001:0005b4b0       $unwind$Settings_enum      000000018005c4b0     service.obj
 0001:0005b4c0       $chain$0$Settings_enum     000000018005c4c0     service.obj
 0001:0005b4d4       $chain$2$Settings_enum     000000018005c4d4     service.obj
 0001:0005b4ec       $chain$3$Settings_enum     000000018005c4ec     service.obj
 0001:0005b4fc       $chain$5$Settings_enum     000000018005c4fc     service.obj
 0001:0005b510       $chain$6$Settings_enum     000000018005c510     service.obj
 0001:0005b520       $unwind$far_ColorDialog    000000018005c520     service.obj
 0001:0005b530       $unwind$_snwprintf         000000018005c530     slnunico.obj
 0001:0005b540       $unwind$??$write_multiple_characters@V?$string_output_adapter@D@__crt_stdio_output@@D@__crt_stdio_output@@YAXAEBV?$string_output_adapter@D@0@DHQEAH@Z 000000018005c540     libucrt:output.obj
 0001:0005b540       $unwind$??$type_case_integer_parse_into_buffer@I@?$output_processor@DV?$stream_output_adapter@D@__crt_stdio_output@@V?$standard_base@DV?$stream_output_adapter@D@__crt_stdio_output@@@2@@__crt_stdio_output@@AEAAXII_N@Z 000000018005c540     libucrt:output.obj
 0001:0005b540       $unwind$??$type_case_integer_parse_into_buffer@_K@?$output_processor@_WV?$string_output_adapter@_W@__crt_stdio_output@@V?$standard_base@_WV?$string_output_adapter@_W@__crt_stdio_output@@@2@@__crt_stdio_output@@AEAAX_KI_N@Z 000000018005c540     libucrt:output.obj
 0001:0005b540       $unwind$??$type_case_integer_parse_into_buffer@_K@?$output_processor@DV?$string_output_adapter@D@__crt_stdio_output@@V?$standard_base@DV?$string_output_adapter@D@__crt_stdio_output@@@2@@__crt_stdio_output@@AEAAX_KI_N@Z 000000018005c540     libucrt:output.obj
 0001:0005b540       $unwind$??$type_case_integer_parse_into_buffer@_K@?$output_processor@DV?$stream_output_adapter@D@__crt_stdio_output@@V?$standard_base@DV?$stream_output_adapter@D@__crt_stdio_output@@@2@@__crt_stdio_output@@AEAAX_KI_N@Z 000000018005c540     libucrt:output.obj
 0001:0005b540       $unwind$utf8_oced          000000018005c540     slnunico.obj
 0001:0005b540       $unwind$??$type_case_integer_parse_into_buffer@I@?$output_processor@DV?$string_output_adapter@D@__crt_stdio_output@@V?$standard_base@DV?$string_output_adapter@D@__crt_stdio_output@@@2@@__crt_stdio_output@@AEAAXII_N@Z 000000018005c540     libucrt:output.obj
 0001:0005b540       $unwind$??$type_case_integer_parse_into_buffer@I@?$output_processor@_WV?$string_output_adapter@_W@__crt_stdio_output@@V?$standard_base@_WV?$string_output_adapter@_W@__crt_stdio_output@@@2@@__crt_stdio_output@@AEAAXII_N@Z 000000018005c540     libucrt:output.obj
 0001:0005b548       $unwind$__GSHandlerCheckCommon 000000018005c548     LIBCMT:_gshandler_.obj
 0001:0005b548       $unwind$utf8_graphext      000000018005c548     slnunico.obj
 0001:0005b550       $chain$0$utf8_graphext     000000018005c550     slnunico.obj
 0001:0005b564       $chain$1$utf8_graphext     000000018005c564     slnunico.obj
 0001:0005b574       $unwind$utf8_count         000000018005c574     slnunico.obj
 0001:0005b584       $chain$0$utf8_count        000000018005c584     slnunico.obj
 0001:0005b598       $chain$1$utf8_count        000000018005c598     slnunico.obj
 0001:0005b5ac       $chain$2$utf8_count        000000018005c5ac     slnunico.obj
 0001:0005b5bc       $chain$3$utf8_count        000000018005c5bc     slnunico.obj
 0001:0005b5cc       $unwind$unic_sub           000000018005c5cc     slnunico.obj
 0001:0005b5e4       $unwind$unic_lower         000000018005c5e4     slnunico.obj
 0001:0005b5e4       $unwind$str_reverse        000000018005c5e4     slnunico.obj
 0001:0005b5e4       $unwind$unic_upper         000000018005c5e4     slnunico.obj
 0001:0005b5f8       $chain$0$str_reverse       000000018005c5f8     slnunico.obj
 0001:0005b60c       $chain$1$str_reverse       000000018005c60c     slnunico.obj
 0001:0005b61c       $chain$0$unic_lower        000000018005c61c     slnunico.obj
 0001:0005b630       $chain$1$unic_lower        000000018005c630     slnunico.obj
 0001:0005b640       $chain$0$unic_upper        000000018005c640     slnunico.obj
 0001:0005b654       $chain$1$unic_upper        000000018005c654     slnunico.obj
 0001:0005b664       $unwind$str_rep            000000018005c664     slnunico.obj
 0001:0005b678       $unwind$unic_byte          000000018005c678     slnunico.obj
 0001:0005b690       $unwind$unic_char          000000018005c690     slnunico.obj
 0001:0005b6a8       $chain$0$unic_char         000000018005c6a8     slnunico.obj
 0001:0005b6bc       $chain$1$unic_char         000000018005c6bc     slnunico.obj
 0001:0005b6cc       $unwind$str_dump           000000018005c6cc     slnunico.obj
 0001:0005b6d8       $unwind$match_class        000000018005c6d8     slnunico.obj
 0001:0005b6e8       $unwind$singlematch        000000018005c6e8     slnunico.obj
 0001:0005b704       $unwind$max_expand         000000018005c704     slnunico.obj
 0001:0005b718       $chain$0$max_expand        000000018005c718     slnunico.obj
 0001:0005b72c       $chain$1$max_expand        000000018005c72c     slnunico.obj
 0001:0005b73c       $unwind$min_expand         000000018005c73c     slnunico.obj
 0001:0005b754       $chain$0$push_onecapture   000000018005c754     slnunico.obj
 0001:0005b768       $chain$1$push_onecapture   000000018005c768     slnunico.obj
 0001:0005b77c       $chain$2$push_onecapture   000000018005c77c     slnunico.obj
 0001:0005b78c       $chain$4$push_onecapture   000000018005c78c     slnunico.obj
 0001:0005b7a0       $unwind$push_captures      000000018005c7a0     slnunico.obj
 0001:0005b7b4       $chain$1$push_captures     000000018005c7b4     slnunico.obj
 0001:0005b7cc       $chain$2$push_captures     000000018005c7cc     slnunico.obj
 0001:0005b7dc       $unwind$unic_find_aux      000000018005c7dc     slnunico.obj
 0001:0005b7f8       $unwind$add_value          000000018005c7f8     slnunico.obj
 0001:0005b80c       $chain$0$add_value         000000018005c80c     slnunico.obj
 0001:0005b820       $chain$1$add_value         000000018005c820     slnunico.obj
 0001:0005b830       $unwind$unic_gsub          000000018005c830     slnunico.obj
 0001:0005b850       $unwind$str_format         000000018005c850     slnunico.obj
 0001:0005b86c       $unwind$g_iofile           000000018005c86c     uliolib51.obj
 0001:0005b87c       $chain$0$g_iofile          000000018005c87c     uliolib51.obj
 0001:0005b890       $chain$1$g_iofile          000000018005c890     uliolib51.obj
 0001:0005b8a4       $chain$2$g_iofile          000000018005c8a4     uliolib51.obj
 0001:0005b8b4       $chain$3$g_iofile          000000018005c8b4     uliolib51.obj
 0001:0005b8c4       $chain$1$io_lines          000000018005c8c4     uliolib51.obj
 0001:0005b8dc       $chain$2$io_lines          000000018005c8dc     uliolib51.obj
 0001:0005b8f0       $unwind$read_line          000000018005c8f0     uliolib51.obj
 0001:0005b904       $unwind$read_chars         000000018005c904     uliolib51.obj
 0001:0005b91c       $unwind$g_read             000000018005c91c     uliolib51.obj
 0001:0005b934       $unwind$strpbrk            000000018005c934     libucrt:strpbrk.obj
 0001:0005b934       $unwind$GetIntFromArray    000000018005c934     util.obj
 0001:0005b934       $unwind$_strdup            000000018005c934     libucrt:strdup.obj
 0001:0005b934       $unwind$PutWStrToArray     000000018005c934     ustring.obj
 0001:0005b934       $unwind$loaderror          000000018005c934     uloadlib51.obj
 0001:0005b934       $unwind$??$initialize_tmpfile_buffer_nolock@D@@YA_NW4buffer_id@?A0x5b9a7937@@@Z 000000018005c934     libucrt:tmpfile.obj
 0001:0005b934       $unwind$??$generate_tmpfile_file_name@D@@YA_NQEAD_K@Z 000000018005c934     libucrt:tmpfile.obj
 0001:0005b944       $unwind$loader_Croot       000000018005c944     uloadlib51.obj
 0001:0005b954       $unwind$ll_module          000000018005c954     uloadlib51.obj
 0001:0005b968       $chain$0$ll_module         000000018005c968     uloadlib51.obj
 0001:0005b97c       $chain$1$ll_module         000000018005c97c     uloadlib51.obj
 0001:0005b98c       $unwind$setpath            000000018005c98c     uloadlib51.obj
 0001:0005b9a0       $unwind$_free_osfhnd       000000018005c9a0     libucrt:osfinfo.obj
 0001:0005b9a0       $unwind$__acrt_stdio_refill_and_read_narrow_nolock 000000018005c9a0     libucrt:_filbuf.obj
 0001:0005b9a0       $unwind$?initialize_stdio_handles_nolock@@YAXXZ 000000018005c9a0     libucrt:ioinit.obj
 0001:0005b9a0       $unwind$luaopen_upackage   000000018005c9a0     uloadlib51.obj
 0001:0005b9b4       $unwind$GetOptNumFromTable 000000018005c9b4     ustring.obj
 0001:0005b9c0       $unwind$opt_utf8_string    000000018005c9c0     ustring.obj
 0001:0005b9d8       $unwind$convert_multibyte_string 000000018005c9d8     ustring.obj
 0001:0005b9f4       $unwind$push_multibyte_string 000000018005c9f4     ustring.obj
 0001:0005ba08       $chain$2$push_multibyte_string 000000018005ca08     ustring.obj
 0001:0005ba20       $chain$3$push_multibyte_string 000000018005ca20     ustring.obj
 0001:0005ba34       $unwind$ustring_WideCharToMultiByte 000000018005ca34     ustring.obj
 0001:0005ba48       $chain$1$ustring_WideCharToMultiByte 000000018005ca48     ustring.obj
 0001:0005ba60       $chain$2$ustring_WideCharToMultiByte 000000018005ca60     ustring.obj
 0001:0005ba70       $unwind$ustring_MultiByteToWideChar 000000018005ca70     ustring.obj
 0001:0005ba8c       $unwind$ustring_OemToUtf8  000000018005ca8c     ustring.obj
 0001:0005ba98       $chain$1$ustring_OemToUtf8 000000018005ca98     ustring.obj
 0001:0005bab0       $chain$2$ustring_OemToUtf8 000000018005cab0     ustring.obj
 0001:0005bac0       $unwind$?decode_options@@YA?AUfile_options@?A0xa9d50aae@@HHH@Z 000000018005cac0     libucrt:open.obj
 0001:0005bac0       $unwind$win_DeleteRegValue 000000018005cac0     win.obj
 0001:0005bac0       $unwind$ustring_Utf8ToOem  000000018005cac0     ustring.obj
 0001:0005bad4       $unwind$win_FileTimeToSystemTime 000000018005cad4     win.obj
 0001:0005bad4       $unwind$ustring_Utf16ToUtf8 000000018005cad4     ustring.obj
 0001:0005bad4       $unwind$ustring_Uuid       000000018005cad4     ustring.obj
 0001:0005bad4       $unwind$??$common_xtox_s@_KD@@YAH_KQEAD0I_N@Z 000000018005cad4     libucrt:xtoa.obj
 0001:0005bad4       $unwind$win_SystemTimeToFileTime 000000018005cad4     win.obj
 0001:0005badc       $unwind$ustring_Utf8ToUtf16 000000018005cadc     ustring.obj
 0001:0005baec       $chain$0$ustring_Utf8ToUtf16 000000018005caec     ustring.obj
 0001:0005bb00       $chain$1$ustring_Utf8ToUtf16 000000018005cb00     ustring.obj
 0001:0005bb10       $unwind$ustring_GetCPInfo  000000018005cb10     ustring.obj
 0001:0005bb28       $unwind$ustring_GetLogicalDriveStrings 000000018005cb28     ustring.obj
 0001:0005bb38       $chain$0$ustring_GetLogicalDriveStrings 000000018005cb38     ustring.obj
 0001:0005bb4c       $chain$1$ustring_GetLogicalDriveStrings 000000018005cb4c     ustring.obj
 0001:0005bb5c       $unwind$ustring_SearchPath 000000018005cb5c     ustring.obj
 0001:0005bb74       $unwind$ustring_GlobalMemoryStatus 000000018005cb74     ustring.obj
 0001:0005bb7c       $chain$0$ustring_GlobalMemoryStatus 000000018005cb7c     ustring.obj
 0001:0005bb90       $chain$2$ustring_GlobalMemoryStatus 000000018005cb90     ustring.obj
 0001:0005bba4       $unwind$ustring_SetFileAttr 000000018005cba4     ustring.obj
 0001:0005bbb0       $chain$2$ustring_SetFileAttr 000000018005cbb0     ustring.obj
 0001:0005bbcc       $chain$3$ustring_SetFileAttr 000000018005cbcc     ustring.obj
 0001:0005bbe0       $chain$4$ustring_SetFileAttr 000000018005cbe0     ustring.obj
 0001:0005bbf0       $chain$5$ustring_SetFileAttr 000000018005cbf0     ustring.obj
 0001:0005bc00       $unwind$ustring_GetFileAttr 000000018005cc00     ustring.obj
 0001:0005bc00       $unwind$ustring_SetCurrentDir 000000018005cc00     ustring.obj
 0001:0005bc0c       $chain$2$ustring_GetFileAttr 000000018005cc0c     ustring.obj
 0001:0005bc28       $chain$3$ustring_GetFileAttr 000000018005cc28     ustring.obj
 0001:0005bc38       $unwind$ustring_SHGetFolderPath 000000018005cc38     ustring.obj
 0001:0005bc48       $chain$1$ustring_SHGetFolderPath 000000018005cc48     ustring.obj
 0001:0005bc60       $chain$2$ustring_SHGetFolderPath 000000018005cc60     ustring.obj
 0001:0005bc70       $unwind$ustring_OutputDebugString 000000018005cc70     ustring.obj
 0001:0005bc84       $chain$0$ustring_OutputDebugString 000000018005cc84     ustring.obj
 0001:0005bc98       $chain$1$ustring_OutputDebugString 000000018005cc98     ustring.obj
 0001:0005bca8       $unwind$ustring_GetCurrentDir 000000018005cca8     ustring.obj
 0001:0005bcbc       $chain$0$ustring_GetCurrentDir 000000018005ccbc     ustring.obj
 0001:0005bcd0       $chain$1$ustring_GetCurrentDir 000000018005ccd0     ustring.obj
 0001:0005bce4       $chain$2$ustring_GetCurrentDir 000000018005cce4     ustring.obj
 0001:0005bcf4       $chain$3$ustring_GetCurrentDir 000000018005ccf4     ustring.obj
 0001:0005bd04       $chain$2$ustring_SetCurrentDir 000000018005cd04     ustring.obj
 0001:0005bd20       $chain$3$ustring_SetCurrentDir 000000018005cd20     ustring.obj
 0001:0005bd30       $unwind$win_GetEnv         000000018005cd30     win.obj
 0001:0005bd44       $chain$0$win_GetEnv        000000018005cd44     win.obj
 0001:0005bd58       $chain$1$win_GetEnv        000000018005cd58     win.obj
 0001:0005bd68       $unwind$win_SetRegKey      000000018005cd68     win.obj
 0001:0005bd80       $unwind$win_GetRegKey      000000018005cd80     win.obj
 0001:0005bd94       $unwind$win_EnumRegValue   000000018005cd94     win.obj
 0001:0005bd94       $unwind$win_EnumRegKey     000000018005cd94     win.obj
 0001:0005bda8       $unwind$win_GetFileInfo    000000018005cda8     win.obj
 0001:0005bdb8       $unwind$win_CompareString  000000018005cdb8     win.obj
 0001:0005bdd0       $unwind$mkdir              000000018005cdd0     win.obj
 0001:0005bde8       $chain$0$mkdir             000000018005cde8     win.obj
 0001:0005bdfc       $unwind$win_ShellExecute   000000018005cdfc     win.obj
 0001:0005bdfc       $unwind$??$create_environment@_W@@YAQEAPEA_WQEA_W@Z 000000018005cdfc     libucrt:environment_initialization.obj
 0001:0005bdfc       $unwind$__acrt_copy_path_to_wide_string 000000018005cdfc     libucrt:string_utilities.obj
 0001:0005bdfc       $unwind$??$create_environment@D@@YAQEAPEADQEAD@Z 000000018005cdfc     libucrt:environment_initialization.obj
 0001:0005be14       $unwind$?dllmain_crt_process_attach@@YAHQEAUHINSTANCE__@@QEAX@Z 000000018005ce14     LIBCMT:dll_dllmain.obj
 0001:0005be50       $unwind$?fin$0@?0???$?RV<lambda_f2e299630e499de9f9a165e60fcd3db5>@@AEAV<lambda_2ae9d31cdba2644fcbeaf08da7c24588>@@V<lambda_40d01ff24d0e7b3814fdbdcee8eab3c7>@@@?$__crt_seh_guarded_call@X@@QEAAX$$QEAV<lambda_f2e299630e499de9f9a165e60fcd3db5>@@AEAV<lambda_2ae9d31cdba2644fcbeaf08da7c24588>@@$$QEAV<lambda_40d01ff24d0e7b3814fdbdcee8eab3c7>@@@Z@4HA 000000018005ce50     libucrt:per_thread_data.obj
 0001:0005be50       $unwind$common_control87$filt$0 000000018005ce50     libucrt:ieee.obj
 0001:0005be50       $unwind$?fin$0@?0???$?RV<lambda_aa87e3671a710a21b5dc78c0bdf72e11>@@AEAV<lambda_92619d2358a28f41a33ba319515a20b9>@@V<lambda_6992ecaafeb10aed2b74cb1fae11a551>@@@?$__crt_seh_guarded_call@X@@QEAAX$$QEAV<lambda_aa87e3671a710a21b5dc78c0bdf72e11>@@AEAV<lambda_92619d2358a28f41a33ba319515a20b9>@@$$QEAV<lambda_6992ecaafeb10aed2b74cb1fae11a551>@@@Z@4HA 000000018005ce50     libucrt:per_thread_data.obj
 0001:0005be50       $unwind$?fin$0@?0??__acrt_stdio_allocate_stream@@YA?AV__crt_stdio_stream@@XZ@4HA 000000018005ce50     libucrt:stream.obj
 0001:0005be50       $unwind$_query_new_handler$fin$0 000000018005ce50     libucrt:new_handler.obj
 0001:0005be50       $unwind$?fin$0@?0???$common_freopen@_W@@YAHQEAPEAU_iobuf@@QEB_W1V__crt_stdio_stream@@H@Z@4HA 000000018005ce50     libucrt:freopen.obj
 0001:0005be50       $unwind$?fin$0@?0???$?RV<lambda_0ae27a3a962d80f24befdcbee591983d>@@AEAV<lambda_8d0ee55de4b1038c4002e0adecdf1839>@@V<lambda_dc504788e8f1664fe9b84e20bfb512f2>@@@?$__crt_seh_guarded_call@X@@QEAAX$$QEAV<lambda_0ae27a3a962d80f24befdcbee591983d>@@AEAV<lambda_8d0ee55de4b1038c4002e0adecdf1839>@@$$QEAV<lambda_dc504788e8f1664fe9b84e20bfb512f2>@@@Z@4HA 000000018005ce50     libucrt:per_thread_data.obj
 0001:0005be50       $unwind$fgetc$fin$0        000000018005ce50     libucrt:fgetc.obj
 0001:0005be50       $unwind$?fin$0@?0???$?RV<lambda_082dd7c0feb7dbdaf245f261e54a6583>@@AEAV<lambda_f3caf1ecae5fe01a9a1a6239afa44510>@@V<lambda_c640b76c0755ae85b317b35c67c61e6b>@@@?$__crt_seh_guarded_call@H@@QEAAH$$QEAV<lambda_082dd7c0feb7dbdaf245f261e54a6583>@@AEAV<lambda_f3caf1ecae5fe01a9a1a6239afa44510>@@$$QEAV<lambda_c640b76c0755ae85b317b35c67c61e6b>@@@Z@4HA 000000018005ce50     libucrt:input.obj
 0001:0005be50       $unwind$rewind$fin$0       000000018005ce50     libucrt:rewind.obj
 0001:0005be50       $unwind$ungetc$fin$0       000000018005ce50     libucrt:ungetc.obj
 0001:0005be50       $unwind$?fin$0@?0??dllmain_crt_process_detach@@YAH_N@Z@4HA 000000018005ce50     LIBCMT:dll_dllmain.obj
 0001:0005be50       $unwind$_read$fin$0        000000018005ce50     libucrt:read.obj
 0001:0005be50       $unwind$__acrt_update_thread_locale_data$fin$0 000000018005ce50     libucrt:locale_refcounting.obj
 0001:0005be50       $unwind$?fin$0@?0??dllmain_crt_process_attach@@YAHQEAUHINSTANCE__@@QEAX@Z@4HA 000000018005ce50     LIBCMT:dll_dllmain.obj
 0001:0005be50       $unwind$?fin$0@?0???$?RV<lambda_751a882b2c74d4b022dec766aa51a29a>@@AEAV<lambda_628dfdc04ba53c8bfc02c9951375f3f5>@@V<lambda_f6c7be5f7998530c34de24c7437d6b54>@@@?$__crt_seh_guarded_call@H@@QEAAH$$QEAV<lambda_751a882b2c74d4b022dec766aa51a29a>@@AEAV<lambda_628dfdc04ba53c8bfc02c9951375f3f5>@@$$QEAV<lambda_f6c7be5f7998530c34de24c7437d6b54>@@@Z@4HA 000000018005ce50     libucrt:close.obj
 0001:0005be50       $unwind$_pclose$fin$0      000000018005ce50     libucrt:popen.obj
 0001:0005be50       $unwind$fclose$fin$0       000000018005ce50     libucrt:fclose.obj
 0001:0005be50       $unwind$?fin$0@?0???$common_getenv@_W@@YAPEA_WQEB_W@Z@4HA 000000018005ce50     libucrt:getenv.obj
 0001:0005be50       $unwind$?fin$0@?0???$common_fdopen@_W@@YAPEAU_iobuf@@HQEB_W@Z@4HA 000000018005ce50     libucrt:fdopen.obj
 0001:0005be50       $unwind$clearerr_s$fin$0   000000018005ce50     libucrt:clearerr.obj
 0001:0005be50       $unwind$__acrt_initialize_lowio$fin$0 000000018005ce50     libucrt:ioinit.obj
 0001:0005be50       $unwind$?fin$0@?0???$?RV<lambda_a37b2b86f63e897a80ea819b0eb08c01>@@AEAV<lambda_38ce7e780aa69e748d6df282ebc68efe>@@V<lambda_99fb1378e971ab6e7edea83e3a7a83a2>@@@?$__crt_seh_guarded_call@H@@QEAAH$$QEAV<lambda_a37b2b86f63e897a80ea819b0eb08c01>@@AEAV<lambda_38ce7e780aa69e748d6df282ebc68efe>@@$$QEAV<lambda_99fb1378e971ab6e7edea83e3a7a83a2>@@@Z@4HA 000000018005ce50     libucrt:commit.obj
 0001:0005be50       $unwind$_write$fin$0       000000018005ce50     libucrt:write.obj
 0001:0005be50       $unwind$?fin$0@?0???$?RV<lambda_842d9ff0dc9ef11c61343bbaebe7f885>@@AEAV<lambda_c5860995281e5c4ce005b3de8f5874ee>@@V<lambda_d90129c13df834fdcbf8d2b88dafcf2d>@@@?$__crt_seh_guarded_call@X@@QEAAX$$QEAV<lambda_842d9ff0dc9ef11c61343bbaebe7f885>@@AEAV<lambda_c5860995281e5c4ce005b3de8f5874ee>@@$$QEAV<lambda_d90129c13df834fdcbf8d2b88dafcf2d>@@@Z@4HA 000000018005ce50     libucrt:fflush.obj
 0001:0005be50       $unwind$?fin$0@?0???$?RV<lambda_886d6c58226a84441f68b9f2b8217b83>@@AEAV<lambda_ab61a845afdef5b7c387490eaf3616ee>@@V<lambda_f7f22ab5edc0698d5f6905b0d3f44752>@@@?$__crt_seh_guarded_call@X@@QEAAX$$QEAV<lambda_886d6c58226a84441f68b9f2b8217b83>@@AEAV<lambda_ab61a845afdef5b7c387490eaf3616ee>@@$$QEAV<lambda_f7f22ab5edc0698d5f6905b0d3f44752>@@@Z@4HA 000000018005ce50     libucrt:fflush.obj
 0001:0005be50       $unwind$?fin$0@?0???$?RV<lambda_c376a267cfb53b6959b3b692ec76b120>@@AEAV<lambda_9a32fed5bf61b6b509b2d3f6003082a1>@@V<lambda_572fbb9fa0ab338edf41edfd4b5fcc8d>@@@?$__crt_seh_guarded_call@H@@QEAAH$$QEAV<lambda_c376a267cfb53b6959b3b692ec76b120>@@AEAV<lambda_9a32fed5bf61b6b509b2d3f6003082a1>@@$$QEAV<lambda_572fbb9fa0ab338edf41edfd4b5fcc8d>@@@Z@4HA 000000018005ce50     libucrt:fflush.obj
 0001:0005be50       $unwind$?fin$0@?0???$common_fsopen@_W@@YAPEAU_iobuf@@QEB_W0H@Z@4HA 000000018005ce50     libucrt:fopen.obj
 0001:0005be50       $unwind$?fin$0@?0???$common_fgets@D@@YAPEADQEADHV__crt_stdio_stream@@@Z@4HA 000000018005ce50     libucrt:fgets.obj
 0001:0005be50       $unwind$?fin$0@?0???$?RV<lambda_a62c933ada0517137acf5807a1eeac1f>@@AEAV<lambda_a31071773b9a94e445cbd5d04ef99106>@@V<lambda_56065050dbf3ada7e59a83db45153de3>@@@?$__crt_seh_guarded_call@H@@QEAAH$$QEAV<lambda_a62c933ada0517137acf5807a1eeac1f>@@AEAV<lambda_a31071773b9a94e445cbd5d04ef99106>@@$$QEAV<lambda_56065050dbf3ada7e59a83db45153de3>@@@Z@4HA 000000018005ce50     libucrt:output.obj
 0001:0005be50       $unwind$_fcloseall$fin$0   000000018005ce50     libucrt:closeall.obj
 0001:0005be50       $unwind$_alloc_osfhnd$fin$0 000000018005ce50     libucrt:osfinfo.obj
 0001:0005be50       $unwind$?fin$0@?0???$?RV<lambda_2d41944a1d46af3157314b8a01080d33>@@AEAV<lambda_8f455de75cd7d7f24b4096f044d8b9e6>@@V<lambda_aa500f224e6afead328df44964fe2772>@@@?$__crt_seh_guarded_call@X@@QEAAX$$QEAV<lambda_2d41944a1d46af3157314b8a01080d33>@@AEAV<lambda_8f455de75cd7d7f24b4096f044d8b9e6>@@$$QEAV<lambda_aa500f224e6afead328df44964fe2772>@@@Z@4HA 000000018005ce50     libucrt:per_thread_data.obj
 0001:0005be50       $unwind$?fin$0@?0???$common_lseek@_J@@YA_JH_JH@Z@4HA 000000018005ce50     libucrt:lseek.obj
 0001:0005be50       $unwind$?fin$0@?0??common_fseek@@YAHV__crt_stdio_stream@@_JH@Z@4HA 000000018005ce50     libucrt:fseek.obj
 0001:0005be50       $unwind$raise$fin$0        000000018005ce50     libucrt:signal.obj
 0001:0005be50       $unwind$?fin$0@?0???$common_ftell@J@@YAJV__crt_stdio_stream@@@Z@4HA 000000018005ce50     libucrt:ftell.obj
 0001:0005be50       $unwind$_rmtmp$fin$0       000000018005ce50     libucrt:rmtmp.obj
 0001:0005be50       $unwind$?fin$0@?0???$?RV<lambda_efdfa57d1f175319df784efa44bb7b81>@@AEAV<lambda_5f0a4c1567f8adc6734073e5d1e1b35c>@@V<lambda_2e8a7d3640ea6ccb4c2413664c2db6fd>@@@?$__crt_seh_guarded_call@X@@QEAAX$$QEAV<lambda_efdfa57d1f175319df784efa44bb7b81>@@AEAV<lambda_5f0a4c1567f8adc6734073e5d1e1b35c>@@$$QEAV<lambda_2e8a7d3640ea6ccb4c2413664c2db6fd>@@@Z@4HA 000000018005ce50     libucrt:mbctype.obj
 0001:0005be50       $unwind$?fin$0@?0???$?RV<lambda_7777bce6b2f8c936911f934f8298dc43>@@AEAV<lambda_f03950bc5685219e0bcd2087efbe011e>@@V<lambda_3883c3dff614d5e0c5f61bb1ac94921c>@@@?$__crt_seh_guarded_call@H@@QEAAH$$QEAV<lambda_7777bce6b2f8c936911f934f8298dc43>@@AEAV<lambda_f03950bc5685219e0bcd2087efbe011e>@@$$QEAV<lambda_3883c3dff614d5e0c5f61bb1ac94921c>@@@Z@4HA 000000018005ce50     libucrt:onexit.obj
 0001:0005be50       $unwind$__acrt_lowio_ensure_fh_exists$fin$0 000000018005ce50     libucrt:osfinfo.obj
 0001:0005be50       $unwind$?fin$0@?0???$common_lseek@J@@YAJHJH@Z@4HA 000000018005ce50     libucrt:lseek.obj
 0001:0005be50       $unwind$?fin$0@?0???$?RV<lambda_450d765d439847d4c735a33c368b5fc0>@@AEAV<lambda_44731a7d0e6d81c3e6aa82d741081786>@@V<lambda_601a2a7da3b7a96e9554ac7215c4b07c>@@@?$__crt_seh_guarded_call@P6AXH@Z@@QEAAP6AXH@Z$$QEAV<lambda_450d765d439847d4c735a33c368b5fc0>@@AEAV<lambda_44731a7d0e6d81c3e6aa82d741081786>@@$$QEAV<lambda_601a2a7da3b7a96e9554ac7215c4b07c>@@@Z@4HA 000000018005ce50     libucrt:signal.obj
 0001:0005be50       $unwind$_rmtmp$fin$1       000000018005ce50     libucrt:rmtmp.obj
 0001:0005be50       $unwind$?fin$0@?0???$?RV<lambda_bdbcead8b570fa3d5ec6d9679862a6e5>@@AEAV<lambda_96f4279ff90247a4c5c5d9824f56f8c1>@@V<lambda_4606be27f17b5e5579e09050fab91818>@@@?$__crt_seh_guarded_call@_K@@QEAA_K$$QEAV<lambda_bdbcead8b570fa3d5ec6d9679862a6e5>@@AEAV<lambda_96f4279ff90247a4c5c5d9824f56f8c1>@@$$QEAV<lambda_4606be27f17b5e5579e09050fab91818>@@@Z@4HA 000000018005ce50     libucrt:fwrite.obj
 0001:0005be50       $unwind$_IsNonwritableInCurrentImage$filt$0 000000018005ce50     LIBCMT:pesect.obj
 0001:0005be50       $unwind$_ctrlfp$filt$0     000000018005ce50     libucrt:fpctrl.obj
 0001:0005be50       $unwind$?filt$0@?0???R<lambda_6e4b09c48022b2350581041d5f6b0c4c>@@QEBA@XZ@4HA 000000018005ce50     libucrt:exit.obj
 0001:0005be50       $unwind$?fin$0@?0???$?RV<lambda_84ec643ea9557e2f7dc01bb0e9624395>@@AEAV<lambda_ca71763b3c0644891230e4f79ea54fa6>@@V<lambda_439a761618c59b0600e24586724d733b>@@@?$__crt_seh_guarded_call@H@@QEAAH$$QEAV<lambda_84ec643ea9557e2f7dc01bb0e9624395>@@AEAV<lambda_ca71763b3c0644891230e4f79ea54fa6>@@$$QEAV<lambda_439a761618c59b0600e24586724d733b>@@@Z@4HA 000000018005ce50     libucrt:setvbuf.obj
 0001:0005be50       $unwind$__DestructExceptionObject$filt$0 000000018005ce50     libvcruntime:ehhelpers.obj
 0001:0005be50       $unwind$?fin$0@?0???$?RV<lambda_410d79af7f07d98d83a3f525b3859a53>@@AEAV<lambda_3e16ef9562a7dcce91392c22ab16ea36>@@V<lambda_38119f0e861e05405d8a144b9b982f0a>@@@?$__crt_seh_guarded_call@X@@QEAAX$$QEAV<lambda_410d79af7f07d98d83a3f525b3859a53>@@AEAV<lambda_3e16ef9562a7dcce91392c22ab16ea36>@@$$QEAV<lambda_38119f0e861e05405d8a144b9b982f0a>@@@Z@4HA 000000018005ce50     libucrt:wsetlocale.obj
 0001:0005be50       $unwind$?fin$0@?0???$common_popen@_W@@YAPEAU_iobuf@@QEB_W0@Z@4HA 000000018005ce50     libucrt:popen.obj
 0001:0005be50       $unwind$?fin$0@?0???$?RV<lambda_a22f0c497e5168315e06dae667770027>@@AEAV<lambda_a094494068278ba5130ab06e1292f60a>@@V<lambda_24dc10c13f43218c635520766e23e324>@@@?$__crt_seh_guarded_call@_N@@QEAA_N$$QEAV<lambda_a22f0c497e5168315e06dae667770027>@@AEAV<lambda_a094494068278ba5130ab06e1292f60a>@@$$QEAV<lambda_24dc10c13f43218c635520766e23e324>@@@Z@4HA 000000018005ce50     libucrt:spawnv.obj
 0001:0005be50       $unwind$?fin$0@?0??common_tmpfile@@YAHQEAPEAU_iobuf@@H@Z@4HA 000000018005ce50     libucrt:tmpfile.obj
 0001:0005be50       $unwind$?fin$0@?0??update_thread_multibyte_data_internal@@YAPEAU__crt_multibyte_data@@QEAU__acrt_ptd@@QEAPEAU1@@Z@4HA 000000018005ce50     libucrt:mbctype.obj
 0001:0005be50       $unwind$?fin$0@?0???$?RV<lambda_d80eeec6fff315bfe5c115232f3240e3>@@AEAV<lambda_6e4b09c48022b2350581041d5f6b0c4c>@@V<lambda_2358e3775559c9db80273638284d5e45>@@@?$__crt_seh_guarded_call@X@@QEAAX$$QEAV<lambda_d80eeec6fff315bfe5c115232f3240e3>@@AEAV<lambda_6e4b09c48022b2350581041d5f6b0c4c>@@$$QEAV<lambda_2358e3775559c9db80273638284d5e45>@@@Z@4HA 000000018005ce50     libucrt:exit.obj
 0001:0005be58       $unwind$?dllmain_crt_process_detach@@YAH_N@Z 000000018005ce58     LIBCMT:dll_dllmain.obj
 0001:0005be8c       $unwind$?dllmain_dispatch@@YAHQEAUHINSTANCE__@@KQEAX@Z 000000018005ce8c     LIBCMT:dll_dllmain.obj
 0001:0005beb4       $unwind$_pipe$fin$1        000000018005ceb4     libucrt:pipe.obj
 0001:0005beb4       $unwind$?fin$0@?0???$common_dupenv_s@_W@@YAHQEAPEA_WQEA_KQEB_WHQEBDH@Z@4HA 000000018005ceb4     libucrt:getenv.obj
 0001:0005beb4       $unwind$_pipe$fin$0        000000018005ceb4     libucrt:pipe.obj
 0001:0005beb4       $unwind$?fin$0@?0??common_tmpfile_nolock@@YAHQEAPEAU_iobuf@@H@Z@4HA 000000018005ceb4     libucrt:tmpfile.obj
 0001:0005beb4       $unwind$?filt$0@?0??dllmain_dispatch@@YAHQEAUHINSTANCE__@@KQEAX@Z@4HA 000000018005ceb4     LIBCMT:dll_dllmain.obj
 0001:0005beb4       $unwind$fread_s$fin$0      000000018005ceb4     libucrt:fread.obj
 0001:0005bebc       $unwind$__security_init_cookie 000000018005cebc     LIBCMT:gs_support.obj
 0001:0005bec8       $unwind$__scrt_is_nonwritable_in_current_image 000000018005cec8     LIBCMT:utility.obj
 0001:0005bee8       $unwind$__scrt_is_nonwritable_in_current_image$filt$0 000000018005cee8     LIBCMT:utility.obj
 0001:0005bef0       $unwind$__scrt_initialize_onexit_tables 000000018005cef0     LIBCMT:utility.obj
 0001:0005befc       $unwind$__scrt_fastfail    000000018005cefc     LIBCMT:utility_desktop.obj
 0001:0005bf0c       $unwind$__isa_available_init 000000018005cf0c     LIBCMT:_cpu_disp_.obj
 0001:0005bf20       $xdatasym                  000000018005cf20     LIBCMT:_guard_dispatch_.obj
 0001:0005bf28       $xdatasym                  000000018005cf28     libvcruntime:memcpy.obj
 0001:0005bf30       $xdatasym                  000000018005cf30     libvcruntime:memset.obj
 0001:0005bf34       $unwind$wcsstr             000000018005cf34     libvcruntime:wcsstr.obj
 0001:0005bf48       $unwind$strrchr            000000018005cf48     libvcruntime:strrchr.obj
 0001:0005bf48       $unwind$strchr             000000018005cf48     libvcruntime:strchr.obj
 0001:0005bf48       $unwind$wcschr             000000018005cf48     libvcruntime:wcschr.obj
 0001:0005bf50       $xdatasym                  000000018005cf50     libvcruntime:memchr.obj
 0001:0005bf58       $xdatasym                  000000018005cf58     libvcruntime:memcmp.obj
 0001:0005bf5c       $unwind$__C_specific_handler 000000018005cf5c     libvcruntime:_riscchandler_.obj
 0001:0005bf78       $xdatasym                  000000018005cf78     libvcruntime:_jmpuwind_.obj
 0001:0005bf8c       $unwind$__vcrt_initialize_winapi_thunks 000000018005cf8c     libvcruntime:winapi_downlevel.obj
 0001:0005bf8c       $unwind$wcsncpy            000000018005cf8c     libucrt:wcsncpy.obj
 0001:0005bf8c       $unwind$__acrt_initialize_winapi_thunks 000000018005cf8c     libucrt:winapi_thunks.obj
 0001:0005bf94       $unwind$__vcrt_uninitialize_winapi_thunks 000000018005cf94     libvcruntime:winapi_downlevel.obj
 0001:0005bf94       $unwind$__acrt_stdio_end_temporary_buffering_nolock 000000018005cf94     libucrt:_sftbuf.obj
 0001:0005bf9c       $unwind$??$process_string_specifier_tchar@D@?$input_processor@DV?$stream_input_adapter@D@__crt_stdio_input@@@__crt_stdio_input@@AEAA_NW4conversion_mode@1@D@Z 000000018005cf9c     libucrt:input.obj
 0001:0005bf9c       $unwind$?try_get_function@@YAPEAXW4function_id@?A0x391cf84c@@QEBDQEBW4module_id@2@2@Z 000000018005cf9c     libucrt:winapi_thunks.obj
 0001:0005bf9c       $unwind$?try_get_function@@YAPEAXW4function_id@?A0x89697e75@@QEBDQEBW4module_id@2@2@Z 000000018005cf9c     libvcruntime:winapi_downlevel.obj
 0001:0005bf9c       $unwind$??R<lambda_f03950bc5685219e0bcd2087efbe011e>@@QEBAHXZ 000000018005cf9c     libucrt:onexit.obj
 0001:0005bf9c       $unwind$_fwrite_nolock     000000018005cf9c     libucrt:fwrite.obj
 0001:0005bfb8       $xdatasym                  000000018005cfb8     libvcruntime:handlers.obj
 0001:0005bfc0       $unwind$__DestructExceptionObject 000000018005cfc0     libvcruntime:ehhelpers.obj
 0001:0005bfe0       $unwind$__stdio_common_vfprintf 000000018005cfe0     libucrt:output.obj
 0001:0005bfe0       $unwind$__stdio_common_vfscanf 000000018005cfe0     libucrt:input.obj
 0001:0005bfe8       $unwind$??$common_vsprintf@Vstandard_base@__crt_stdio_output@@_W@@YAH_KQEA_W0QEB_WQEAU__crt_locale_pointers@@QEAD@Z 000000018005cfe8     libucrt:output.obj
 0001:0005bfe8       $unwind$??$common_vsprintf@Vstandard_base@__crt_stdio_output@@D@@YAH_KQEAD0QEBDQEAU__crt_locale_pointers@@1@Z 000000018005cfe8     libucrt:output.obj
 0001:0005c008       $unwind$??$parse_command_line@D@@YAXPEADPEAPEAD0PEA_K2@Z 000000018005d008     libucrt:argv_parsing.obj
 0001:0005c008       $unwind$?write_string_impl@?$output_adapter_common@DV?$stream_output_adapter@D@__crt_stdio_output@@@__crt_stdio_output@@IEBAXQEBDHQEAHAEAV__crt_deferred_errno_cache@@@Z 000000018005d008     libucrt:output.obj
 0001:0005c024       $unwind$?process@?$output_processor@DV?$string_output_adapter@D@__crt_stdio_output@@V?$standard_base@DV?$string_output_adapter@D@__crt_stdio_output@@@2@@__crt_stdio_output@@QEAAHXZ 000000018005d024     libucrt:output.obj
 0001:0005c024       $unwind$?process@?$output_processor@DV?$stream_output_adapter@D@__crt_stdio_output@@V?$standard_base@DV?$stream_output_adapter@D@__crt_stdio_output@@@2@@__crt_stdio_output@@QEAAHXZ 000000018005d024     libucrt:output.obj
 0001:0005c034       $unwind$?parse_int_from_format_string@?$output_processor@DV?$stream_output_adapter@D@__crt_stdio_output@@V?$standard_base@DV?$stream_output_adapter@D@__crt_stdio_output@@@2@@__crt_stdio_output@@AEAA_NQEAH@Z 000000018005d034     libucrt:output.obj
 0001:0005c034       $unwind$?parse_int_from_format_string@?$output_processor@DV?$string_output_adapter@D@__crt_stdio_output@@V?$standard_base@DV?$string_output_adapter@D@__crt_stdio_output@@@2@@__crt_stdio_output@@AEAA_NQEAH@Z 000000018005d034     libucrt:output.obj
 0001:0005c048       $unwind$?state_case_type@?$output_processor@DV?$stream_output_adapter@D@__crt_stdio_output@@V?$standard_base@DV?$stream_output_adapter@D@__crt_stdio_output@@@2@@__crt_stdio_output@@AEAA_NXZ 000000018005d048     libucrt:output.obj
 0001:0005c048       $unwind$?state_case_type@?$output_processor@DV?$string_output_adapter@D@__crt_stdio_output@@V?$standard_base@DV?$string_output_adapter@D@__crt_stdio_output@@@2@@__crt_stdio_output@@AEAA_NXZ 000000018005d048     libucrt:output.obj
 0001:0005c048       $unwind$?configure_text_mode@@YAHHUfile_options@?A0xa9d50aae@@HAEAW4__crt_lowio_text_mode@@@Z 000000018005d048     libucrt:open.obj
 0001:0005c060       $unwind$?type_case_a@?$output_processor@DV?$string_output_adapter@D@__crt_stdio_output@@V?$standard_base@DV?$string_output_adapter@D@__crt_stdio_output@@@2@@__crt_stdio_output@@AEAA_NXZ 000000018005d060     libucrt:output.obj
 0001:0005c060       $unwind$?type_case_a@?$output_processor@DV?$stream_output_adapter@D@__crt_stdio_output@@V?$standard_base@DV?$stream_output_adapter@D@__crt_stdio_output@@@2@@__crt_stdio_output@@AEAA_NXZ 000000018005d060     libucrt:output.obj
 0001:0005c06c       $unwind$?write_stored_string_tchar@?$output_processor@DV?$stream_output_adapter@D@__crt_stdio_output@@V?$standard_base@DV?$stream_output_adapter@D@__crt_stdio_output@@@2@@__crt_stdio_output@@AEAA_ND@Z 000000018005d06c     libucrt:output.obj
 0001:0005c06c       $unwind$?write_stored_string_tchar@?$output_processor@DV?$string_output_adapter@D@__crt_stdio_output@@V?$standard_base@DV?$string_output_adapter@D@__crt_stdio_output@@@2@@__crt_stdio_output@@AEAA_ND@Z 000000018005d06c     libucrt:output.obj
 0001:0005c084       $unwind$??R<lambda_a31071773b9a94e445cbd5d04ef99106>@@QEBAHXZ 000000018005d084     libucrt:output.obj
 0001:0005c0a4       $unwind$?write_string@?$string_output_adapter@D@__crt_stdio_output@@QEBAXQEBDHQEAHAEAV__crt_deferred_errno_cache@@@Z 000000018005d0a4     libucrt:output.obj
 0001:0005c0bc       $unwind$?write_string@?$string_output_adapter@_W@__crt_stdio_output@@QEBAXQEB_WHQEAHAEAV__crt_deferred_errno_cache@@@Z 000000018005d0bc     libucrt:output.obj
 0001:0005c0d4       $unwind$??$__acrt_stdio_parse_mode@_W@@YA?AU__acrt_stdio_stream_mode@@QEB_W@Z 000000018005d0d4     libucrt:openfile.obj
 0001:0005c0d4       $unwind$__acrt_initialize_stdio 000000018005d0d4     libucrt:_file.obj
 0001:0005c0d4       $unwind$__GSHandlerCheck_SEH 000000018005d0d4     LIBCMT:_gshandlerseh_.obj
 0001:0005c0d4       $unwind$__acrt_lowio_set_os_handle 000000018005d0d4     libucrt:osfinfo.obj
 0001:0005c0d4       $unwind$?process@?$output_processor@_WV?$string_output_adapter@_W@__crt_stdio_output@@V?$standard_base@_WV?$string_output_adapter@_W@__crt_stdio_output@@@2@@__crt_stdio_output@@QEAAHXZ 000000018005d0d4     libucrt:output.obj
 0001:0005c0ec       $unwind$?state_case_type@?$output_processor@_WV?$string_output_adapter@_W@__crt_stdio_output@@V?$standard_base@_WV?$string_output_adapter@_W@__crt_stdio_output@@@2@@__crt_stdio_output@@AEAA_NXZ 000000018005d0ec     libucrt:output.obj
 0001:0005c110       $unwind$?type_case_a@?$output_processor@_WV?$string_output_adapter@_W@__crt_stdio_output@@V?$standard_base@_WV?$string_output_adapter@_W@__crt_stdio_output@@@2@@__crt_stdio_output@@AEAA_NXZ 000000018005d110     libucrt:output.obj
 0001:0005c120       $unwind$?write_stored_string_tchar@?$output_processor@_WV?$string_output_adapter@_W@__crt_stdio_output@@V?$standard_base@_WV?$string_output_adapter@_W@__crt_stdio_output@@@2@@__crt_stdio_output@@AEAA_N_W@Z 000000018005d120     libucrt:output.obj
 0001:0005c134       $unwind$??$write_multiple_characters@V?$string_output_adapter@_W@__crt_stdio_output@@D@__crt_stdio_output@@YAXAEBV?$string_output_adapter@_W@0@DHQEAH@Z 000000018005d134     libucrt:output.obj
 0001:0005c140       $unwind$??$write_multiple_characters@V?$stream_output_adapter@D@__crt_stdio_output@@D@__crt_stdio_output@@YAXAEBV?$stream_output_adapter@D@0@DHQEAH@Z 000000018005d140     libucrt:output.obj
 0001:0005c158       $unwind$??$?RV<lambda_a62c933ada0517137acf5807a1eeac1f>@@AEAV<lambda_a31071773b9a94e445cbd5d04ef99106>@@V<lambda_56065050dbf3ada7e59a83db45153de3>@@@?$__crt_seh_guarded_call@H@@QEAAH$$QEAV<lambda_a62c933ada0517137acf5807a1eeac1f>@@AEAV<lambda_a31071773b9a94e445cbd5d04ef99106>@@$$QEAV<lambda_56065050dbf3ada7e59a83db45153de3>@@@Z 000000018005d158     libucrt:output.obj
 0001:0005c17c       $unwind$??$common_fsopen@_W@@YAPEAU_iobuf@@QEB_W0H@Z 000000018005d17c     libucrt:fopen.obj
 0001:0005c1a8       $unwind$fclose             000000018005d1a8     libucrt:fclose.obj
 0001:0005c1cc       $unwind$common_control87   000000018005d1cc     libucrt:ieee.obj
 0001:0005c1f8       $unwind$??$common_freopen@_W@@YAHQEAPEAU_iobuf@@QEB_W1V__crt_stdio_stream@@H@Z 000000018005d1f8     libucrt:freopen.obj
 0001:0005c224       $unwind$fread_s            000000018005d224     libucrt:fread.obj
 0001:0005c254       $unwind$_fread_nolock_s    000000018005d254     libucrt:fread.obj
 0001:0005c26c       $unwind$fgetc              000000018005d26c     libucrt:fgetc.obj
 0001:0005c2a0       $unwind$rewind             000000018005d2a0     libucrt:rewind.obj
 0001:0005c2c4       $unwind$ungetc             000000018005d2c4     libucrt:ungetc.obj
 0001:0005c2e8       $xdatasym                  000000018005d2e8     libucrt:strcmp.obj
 0001:0005c2ec       $unwind$_wcsicmp_l         000000018005d2ec     libucrt:wcsicmp.obj
 0001:0005c2ec       $unwind$__dcrt_write_console_w 000000018005d2ec     libucrt:initcon.obj
 0001:0005c300       $xdatasym                  000000018005d300     libucrt:strncmp.obj
 0001:0005c308       $xdatasym                  000000018005d308     libucrt:strncpy.obj
 0001:0005c30c       $unwind$fallbackMethod     000000018005d30c     libucrt:strpbrk.obj
 0001:0005c31c       $unwind$_pclose            000000018005d31c     libucrt:popen.obj
 0001:0005c344       $unwind$??$common_popen@_W@@YAPEAU_iobuf@@QEB_W0@Z 000000018005d344     libucrt:popen.obj
 0001:0005c374       $unwind$??$common_popen_nolock@_W@@YAPEAU_iobuf@@QEB_W0HAEAY01H@Z 000000018005d374     libucrt:popen.obj
 0001:0005c394       $unwind$??$get_executable_path@_W@@YAPEB_WQEB_W@Z 000000018005d394     libucrt:popen.obj
 0001:0005c3ac       $unwind$clearerr_s         000000018005d3ac     libucrt:clearerr.obj
 0001:0005c3d4       $unwind$?common_flush_all@@YAH_N@Z 000000018005d3d4     libucrt:fflush.obj
 0001:0005c3dc       $unwind$??$?RV<lambda_842d9ff0dc9ef11c61343bbaebe7f885>@@AEAV<lambda_c5860995281e5c4ce005b3de8f5874ee>@@V<lambda_d90129c13df834fdcbf8d2b88dafcf2d>@@@?$__crt_seh_guarded_call@X@@QEAAX$$QEAV<lambda_842d9ff0dc9ef11c61343bbaebe7f885>@@AEAV<lambda_c5860995281e5c4ce005b3de8f5874ee>@@$$QEAV<lambda_d90129c13df834fdcbf8d2b88dafcf2d>@@@Z 000000018005d3dc     libucrt:fflush.obj
 0001:0005c400       $unwind$??$?RV<lambda_886d6c58226a84441f68b9f2b8217b83>@@AEAV<lambda_ab61a845afdef5b7c387490eaf3616ee>@@V<lambda_f7f22ab5edc0698d5f6905b0d3f44752>@@@?$__crt_seh_guarded_call@X@@QEAAX$$QEAV<lambda_886d6c58226a84441f68b9f2b8217b83>@@AEAV<lambda_ab61a845afdef5b7c387490eaf3616ee>@@$$QEAV<lambda_f7f22ab5edc0698d5f6905b0d3f44752>@@@Z 000000018005d400     libucrt:fflush.obj
 0001:0005c428       $unwind$??$?RV<lambda_c376a267cfb53b6959b3b692ec76b120>@@AEAV<lambda_9a32fed5bf61b6b509b2d3f6003082a1>@@V<lambda_572fbb9fa0ab338edf41edfd4b5fcc8d>@@@?$__crt_seh_guarded_call@H@@QEAAH$$QEAV<lambda_c376a267cfb53b6959b3b692ec76b120>@@AEAV<lambda_9a32fed5bf61b6b509b2d3f6003082a1>@@$$QEAV<lambda_572fbb9fa0ab338edf41edfd4b5fcc8d>@@@Z 000000018005d428     libucrt:fflush.obj
 0001:0005c44c       $unwind$??$common_fgets@D@@YAPEADQEADHV__crt_stdio_stream@@@Z 000000018005d44c     libucrt:fgets.obj
 0001:0005c478       $unwind$?common_fseek@@YAHV__crt_stdio_stream@@_JH@Z 000000018005d478     libucrt:fseek.obj
 0001:0005c4a0       $unwind$?common_ftell_translated_utf8_nolock@@YA_JV__crt_stdio_stream@@_J@Z 000000018005d4a0     libucrt:ftell.obj
 0001:0005c4c8       $unwind$?common_ftell_read_mode_nolock@@YA_JV__crt_stdio_stream@@_J1@Z 000000018005d4c8     libucrt:ftell.obj
 0001:0005c4e0       $unwind$??$common_ftell@J@@YAJV__crt_stdio_stream@@@Z 000000018005d4e0     libucrt:ftell.obj
 0001:0005c504       $unwind$fwrite             000000018005d504     libucrt:fwrite.obj
 0001:0005c50c       $unwind$??$?RV<lambda_bdbcead8b570fa3d5ec6d9679862a6e5>@@AEAV<lambda_96f4279ff90247a4c5c5d9824f56f8c1>@@V<lambda_4606be27f17b5e5579e09050fab91818>@@@?$__crt_seh_guarded_call@_K@@QEAA_K$$QEAV<lambda_bdbcead8b570fa3d5ec6d9679862a6e5>@@AEAV<lambda_96f4279ff90247a4c5c5d9824f56f8c1>@@$$QEAV<lambda_4606be27f17b5e5579e09050fab91818>@@@Z 000000018005d50c     libucrt:fwrite.obj
 0001:0005c530       $unwind$setvbuf            000000018005d530     libucrt:setvbuf.obj
 0001:0005c538       $unwind$??$?RV<lambda_84ec643ea9557e2f7dc01bb0e9624395>@@AEAV<lambda_ca71763b3c0644891230e4f79ea54fa6>@@V<lambda_439a761618c59b0600e24586724d733b>@@@?$__crt_seh_guarded_call@H@@QEAAH$$QEAV<lambda_84ec643ea9557e2f7dc01bb0e9624395>@@AEAV<lambda_ca71763b3c0644891230e4f79ea54fa6>@@$$QEAV<lambda_439a761618c59b0600e24586724d733b>@@@Z 000000018005d538     libucrt:setvbuf.obj
 0001:0005c55c       $unwind$?common_tmpfile_nolock@@YAHQEAPEAU_iobuf@@H@Z 000000018005d55c     libucrt:tmpfile.obj
 0001:0005c588       $unwind$?common_tmpfile@@YAHQEAPEAU_iobuf@@H@Z 000000018005d588     libucrt:tmpfile.obj
 0001:0005c5ac       $unwind$?divide@__crt_strtox@@YA_KAEAUbig_integer@1@AEBU21@@Z 000000018005d5ac     libucrt:input.obj
 0001:0005c5cc       $chain$5$?divide@__crt_strtox@@YA_KAEAUbig_integer@1@AEBU21@@Z 000000018005d5cc     libucrt:input.obj
 0001:0005c5e0       $chain$6$?divide@__crt_strtox@@YA_KAEAUbig_integer@1@AEBU21@@Z 000000018005d5e0     libucrt:input.obj
 0001:0005c5f0       $unwind$?assemble_floating_point_value@__crt_strtox@@YA?AW4SLD_STATUS@@_KH_N1AEBVfloating_point_value@1@@Z 000000018005d5f0     libucrt:input.obj
 0001:0005c608       $unwind$?assemble_floating_point_value_from_big_integer@__crt_strtox@@YA?AW4SLD_STATUS@@AEBUbig_integer@1@I_N1AEBVfloating_point_value@1@@Z 000000018005d608     libucrt:input.obj
 0001:0005c624       $unwind$?convert_decimal_string_to_floating_type_common@__crt_strtox@@YA?AW4SLD_STATUS@@AEBUfloating_point_string@1@AEBVfloating_point_value@1@@Z 000000018005d624     libucrt:input.obj
 0001:0005c648       $unwind$?write_character@?$input_processor@DV?$stream_input_adapter@D@__crt_stdio_input@@@__crt_stdio_input@@AEAA_NQEFA_W_KAEAPEFA_WAEA_KD@Z 000000018005d648     libucrt:input.obj
 0001:0005c658       $unwind$??R<lambda_f3caf1ecae5fe01a9a1a6239afa44510>@@QEBAHXZ 000000018005d658     libucrt:input.obj
 0001:0005c678       $unwind$??$process_floating_point_specifier_t@N@?$input_processor@DV?$stream_input_adapter@D@__crt_stdio_input@@@__crt_stdio_input@@AEAA_NXZ 000000018005d678     libucrt:input.obj
 0001:0005c678       $unwind$??$process_floating_point_specifier_t@M@?$input_processor@DV?$stream_input_adapter@D@__crt_stdio_input@@@__crt_stdio_input@@AEAA_NXZ 000000018005d678     libucrt:input.obj
 0001:0005c684       $unwind$??$parse_integer@_KV?$input_adapter_character_source@V?$stream_input_adapter@D@__crt_stdio_input@@@__crt_strtox@@@__crt_strtox@@YA_KQEAU__crt_locale_pointers@@V?$input_adapter_character_source@V?$stream_input_adapter@D@__crt_stdio_input@@@0@H_N@Z 000000018005d684     libucrt:input.obj
 0001:0005c6a0       $unwind$??$process_string_specifier_tchar@_W@?$input_processor@DV?$stream_input_adapter@D@__crt_stdio_input@@@__crt_stdio_input@@AEAA_NW4conversion_mode@1@_W@Z 000000018005d6a0     libucrt:input.obj
 0001:0005c6b8       $unwind$??$?RV<lambda_082dd7c0feb7dbdaf245f261e54a6583>@@AEAV<lambda_f3caf1ecae5fe01a9a1a6239afa44510>@@V<lambda_c640b76c0755ae85b317b35c67c61e6b>@@@?$__crt_seh_guarded_call@H@@QEAAH$$QEAV<lambda_082dd7c0feb7dbdaf245f261e54a6583>@@AEAV<lambda_f3caf1ecae5fe01a9a1a6239afa44510>@@$$QEAV<lambda_c640b76c0755ae85b317b35c67c61e6b>@@@Z 000000018005d6b8     libucrt:input.obj
 0001:0005c6dc       $unwind$??$parse_floating_point@V?$input_adapter_character_source@V?$stream_input_adapter@D@__crt_stdio_input@@@__crt_strtox@@M@__crt_strtox@@YA?AW4SLD_STATUS@@QEAU__crt_locale_pointers@@V?$input_adapter_character_source@V?$stream_input_adapter@D@__crt_stdio_input@@@0@QEAM@Z 000000018005d6dc     libucrt:input.obj
 0001:0005c6dc       $unwind$??$parse_floating_point@V?$input_adapter_character_source@V?$stream_input_adapter@D@__crt_stdio_input@@@__crt_strtox@@N@__crt_strtox@@YA?AW4SLD_STATUS@@QEAU__crt_locale_pointers@@V?$input_adapter_character_source@V?$stream_input_adapter@D@__crt_stdio_input@@@0@QEAN@Z 000000018005d6dc     libucrt:input.obj
 0001:0005c6f4       $unwind$??$parse_floating_point_from_source@V?$input_adapter_character_source@V?$stream_input_adapter@D@__crt_stdio_input@@@__crt_strtox@@@__crt_strtox@@YA?AW4floating_point_parse_result@0@QEAU__crt_locale_pointers@@AEAV?$input_adapter_character_source@V?$stream_input_adapter@D@__crt_stdio_input@@@0@AEAUfloating_point_string@0@@Z 000000018005d6f4     libucrt:input.obj
 0001:0005c70c       $unwind$??$parse_floating_point_possible_nan@DV?$input_adapter_character_source@V?$stream_input_adapter@D@__crt_stdio_input@@@__crt_strtox@@_K@__crt_strtox@@YA?AW4floating_point_parse_result@0@AEADAEAV?$input_adapter_character_source@V?$stream_input_adapter@D@__crt_stdio_input@@@0@_K@Z 000000018005d70c     libucrt:input.obj
 0001:0005c720       $unwind$??$common_getenv@_W@@YAPEA_WQEB_W@Z 000000018005d720     libucrt:getenv.obj
 0001:0005c740       $unwind$??$common_dupenv_s@_W@@YAHQEAPEA_WQEA_KQEB_WHQEBDH@Z 000000018005d740     libucrt:getenv.obj
 0001:0005c780       $unwind$_wsystem           000000018005d780     libucrt:system.obj
 0001:0005c798       $unwind$?common_exit@@YAXHW4_crt_exit_cleanup_mode@@W4_crt_exit_return_mode@@@Z 000000018005d798     libucrt:exit.obj
 0001:0005c7a4       $unwind$??R<lambda_6e4b09c48022b2350581041d5f6b0c4c>@@QEBA@XZ 000000018005d7a4     libucrt:exit.obj
 0001:0005c7c4       $unwind$??$?RV<lambda_d80eeec6fff315bfe5c115232f3240e3>@@AEAV<lambda_6e4b09c48022b2350581041d5f6b0c4c>@@V<lambda_2358e3775559c9db80273638284d5e45>@@@?$__crt_seh_guarded_call@X@@QEAAX$$QEAV<lambda_d80eeec6fff315bfe5c115232f3240e3>@@AEAV<lambda_6e4b09c48022b2350581041d5f6b0c4c>@@$$QEAV<lambda_2358e3775559c9db80273638284d5e45>@@@Z 000000018005d7c4     libucrt:exit.obj
 0001:0005c7e8       $unwind$_configure_narrow_argv 000000018005d7e8     libucrt:argv_parsing.obj
 0001:0005c7fc       $unwind$??$free_environment@D@@YAXQEAPEAD@Z 000000018005d7fc     libucrt:environment_initialization.obj
 0001:0005c7fc       $unwind$??$free_environment@_W@@YAXQEAPEA_W@Z 000000018005d7fc     libucrt:environment_initialization.obj
 0001:0005c808       $unwind$??$initialize_environment_by_cloning_nolock@_W@@YAHXZ 000000018005d808     libucrt:environment_initialization.obj
 0001:0005c818       $unwind$_execute_onexit_table 000000018005d818     libucrt:onexit.obj
 0001:0005c820       $unwind$??$?RV<lambda_7777bce6b2f8c936911f934f8298dc43>@@AEAV<lambda_f03950bc5685219e0bcd2087efbe011e>@@V<lambda_3883c3dff614d5e0c5f61bb1ac94921c>@@@?$__crt_seh_guarded_call@H@@QEAAH$$QEAV<lambda_7777bce6b2f8c936911f934f8298dc43>@@AEAV<lambda_f03950bc5685219e0bcd2087efbe011e>@@$$QEAV<lambda_3883c3dff614d5e0c5f61bb1ac94921c>@@@Z 000000018005d820     libucrt:onexit.obj
 0001:0005c844       $unwind$terminate          000000018005d844     libucrt:terminate.obj
 0001:0005c864       $unwind$?_strupr_s_l_stat@@YAHQEAD_KQEAU__crt_locale_pointers@@@Z 000000018005d864     libucrt:strupr.obj
 0001:0005c888       $unwind$??$parse_integer@_KV?$c_string_character_source@D@__crt_strtox@@@__crt_strtox@@YA_KQEAU__crt_locale_pointers@@V?$c_string_character_source@D@0@H_N@Z 000000018005d888     libucrt:atox.obj
 0001:0005c888       $unwind$??$parse_integer@KV?$c_string_character_source@D@__crt_strtox@@@__crt_strtox@@YAKQEAU__crt_locale_pointers@@V?$c_string_character_source@D@0@H_N@Z 000000018005d888     libucrt:atox.obj
 0001:0005c8a4       $unwind$??$parse_integer@KV?$c_string_character_source@_W@__crt_strtox@@@__crt_strtox@@YAKQEAU__crt_locale_pointers@@V?$c_string_character_source@_W@0@H_N@Z 000000018005d8a4     libucrt:atox.obj
 0001:0005c8bc       $unwind$__acrt_call_reportfault 000000018005d8bc     libucrt:invalid_parameter.obj
 0001:0005c8dc       $unwind$_tolower_l         000000018005d8dc     libucrt:tolower_toupper.obj
 0001:0005c8ec       $unwind$__acrt_locale_free_numeric 000000018005d8ec     libucrt:initnum.obj
 0001:0005c8ec       $unwind$__acrt_locale_free_lc_time_if_unreferenced 000000018005d8ec     libucrt:locale_refcounting.obj
 0001:0005c8ec       $unwind$?destroy_fls@@YAXPEAX@Z 000000018005d8ec     libucrt:per_thread_data.obj
 0001:0005c8ec       $unwind$_free_base         000000018005d8ec     libucrt:free_base.obj
 0001:0005c8f4       $unwind$_mbtowc_l          000000018005d8f4     libucrt:mbtowc.obj
 0001:0005c8f4       $unwind$_wcsnicoll_l       000000018005d8f4     libucrt:wcsnicol.obj
 0001:0005c8f4       $unwind$__acrt_CompareStringW 000000018005d8f4     libucrt:comparestringw.obj
 0001:0005c90c       $unwind$_wctomb_s_l        000000018005d90c     libucrt:wctomb.obj
 0001:0005c91c       $unwind$?construct_ptd_array@@YAXQEAU__acrt_ptd@@@Z 000000018005d91c     libucrt:per_thread_data.obj
 0001:0005c924       $unwind$?destroy_ptd_array@@YAXQEAU__acrt_ptd@@@Z 000000018005d924     libucrt:per_thread_data.obj
 0001:0005c92c       $unwind$??$?RV<lambda_0ae27a3a962d80f24befdcbee591983d>@@AEAV<lambda_8d0ee55de4b1038c4002e0adecdf1839>@@V<lambda_dc504788e8f1664fe9b84e20bfb512f2>@@@?$__crt_seh_guarded_call@X@@QEAAX$$QEAV<lambda_0ae27a3a962d80f24befdcbee591983d>@@AEAV<lambda_8d0ee55de4b1038c4002e0adecdf1839>@@$$QEAV<lambda_dc504788e8f1664fe9b84e20bfb512f2>@@@Z 000000018005d92c     libucrt:per_thread_data.obj
 0001:0005c950       $unwind$??$?RV<lambda_aa87e3671a710a21b5dc78c0bdf72e11>@@AEAV<lambda_92619d2358a28f41a33ba319515a20b9>@@V<lambda_6992ecaafeb10aed2b74cb1fae11a551>@@@?$__crt_seh_guarded_call@X@@QEAAX$$QEAV<lambda_aa87e3671a710a21b5dc78c0bdf72e11>@@AEAV<lambda_92619d2358a28f41a33ba319515a20b9>@@$$QEAV<lambda_6992ecaafeb10aed2b74cb1fae11a551>@@@Z 000000018005d950     libucrt:per_thread_data.obj
 0001:0005c974       $unwind$??$?RV<lambda_f2e299630e499de9f9a165e60fcd3db5>@@AEAV<lambda_2ae9d31cdba2644fcbeaf08da7c24588>@@V<lambda_40d01ff24d0e7b3814fdbdcee8eab3c7>@@@?$__crt_seh_guarded_call@X@@QEAAX$$QEAV<lambda_f2e299630e499de9f9a165e60fcd3db5>@@AEAV<lambda_2ae9d31cdba2644fcbeaf08da7c24588>@@$$QEAV<lambda_40d01ff24d0e7b3814fdbdcee8eab3c7>@@@Z 000000018005d974     libucrt:per_thread_data.obj
 0001:0005c998       $unwind$??$?RV<lambda_2d41944a1d46af3157314b8a01080d33>@@AEAV<lambda_8f455de75cd7d7f24b4096f044d8b9e6>@@V<lambda_aa500f224e6afead328df44964fe2772>@@@?$__crt_seh_guarded_call@X@@QEAAX$$QEAV<lambda_2d41944a1d46af3157314b8a01080d33>@@AEAV<lambda_8f455de75cd7d7f24b4096f044d8b9e6>@@$$QEAV<lambda_aa500f224e6afead328df44964fe2772>@@@Z 000000018005d998     libucrt:per_thread_data.obj
 0001:0005c9bc       $unwind$__acrt_fp_format   000000018005d9bc     libucrt:cvt.obj
 0001:0005c9d0       $unwind$?fp_format_nan_or_infinity@@YAHW4__acrt_fp_class@@_NPEAD_K1@Z 000000018005d9d0     libucrt:cvt.obj
 0001:0005c9e4       $unwind$?fp_format_e_internal@@YAHQEAD_KH_NIQEAU_strflt@@2QEAU__crt_locale_pointers@@@Z 000000018005d9e4     libucrt:cvt.obj
 0001:0005c9fc       $unwind$?fp_format_e@@YAHQEBNQEAD_K12H_NIQEAU__crt_locale_pointers@@@Z 000000018005d9fc     libucrt:cvt.obj
 0001:0005c9fc       $unwind$__acrt_CompareStringEx 000000018005d9fc     libucrt:winapi_thunks.obj
 0001:0005c9fc       $unwind$__acrt_LCMapStringW 000000018005d9fc     libucrt:lcmapstringw.obj
 0001:0005c9fc       $unwind$__acrt_LCMapStringEx 000000018005d9fc     libucrt:winapi_thunks.obj
 0001:0005c9fc       $unwind$_sopen_nolock      000000018005d9fc     libucrt:open.obj
 0001:0005ca10       $unwind$?fp_format_a@@YAHQEBNPEAD_KQEAD2H_NIQEAU__crt_locale_pointers@@@Z 000000018005da10     libucrt:cvt.obj
 0001:0005ca2c       $unwind$_wcsnicmp_l        000000018005da2c     libucrt:wcsnicmp.obj
 0001:0005ca2c       $unwind$?fp_format_f_internal@@YAHQEAD_KHQEAU_strflt@@_NQEAU__crt_locale_pointers@@@Z 000000018005da2c     libucrt:cvt.obj
 0001:0005ca2c       $unwind$__dcrt_get_narrow_environment_from_os 000000018005da2c     libucrt:get_environment_from_os.obj
 0001:0005ca44       $unwind$?fp_format_g@@YAHQEBNQEAD_K12H_NIQEAU__crt_locale_pointers@@@Z 000000018005da44     libucrt:cvt.obj
 0001:0005ca58       $unwind$__acrt_get_sigabrt_handler 000000018005da58     libucrt:signal.obj
 0001:0005ca58       $unwind$__acrt_uninitialize_locale 000000018005da58     libucrt:wsetlocale.obj
 0001:0005ca60       $unwind$??$?RV<lambda_410d79af7f07d98d83a3f525b3859a53>@@AEAV<lambda_3e16ef9562a7dcce91392c22ab16ea36>@@V<lambda_38119f0e861e05405d8a144b9b982f0a>@@@?$__crt_seh_guarded_call@X@@QEAAX$$QEAV<lambda_410d79af7f07d98d83a3f525b3859a53>@@AEAV<lambda_3e16ef9562a7dcce91392c22ab16ea36>@@$$QEAV<lambda_38119f0e861e05405d8a144b9b982f0a>@@@Z 000000018005da60     libucrt:wsetlocale.obj
 0001:0005ca88       $unwind$__acrt_initialize_lowio 000000018005da88     libucrt:ioinit.obj
 0001:0005caa8       $unwind$?initialize_inherited_file_handles_nolock@@YAXXZ 000000018005daa8     libucrt:ioinit.obj
 0001:0005cac4       $unwind$?__acrt_stdio_allocate_stream@@YA?AV__crt_stdio_stream@@XZ 000000018005dac4     libucrt:stream.obj
 0001:0005cae4       $unwind$_wopenfile         000000018005dae4     libucrt:openfile.obj
 0001:0005caf8       $unwind$_commit            000000018005daf8     libucrt:commit.obj
 0001:0005caf8       $unwind$_close             000000018005daf8     libucrt:close.obj
 0001:0005cb00       $unwind$??$?RV<lambda_751a882b2c74d4b022dec766aa51a29a>@@AEAV<lambda_628dfdc04ba53c8bfc02c9951375f3f5>@@V<lambda_f6c7be5f7998530c34de24c7437d6b54>@@@?$__crt_seh_guarded_call@H@@QEAAH$$QEAV<lambda_751a882b2c74d4b022dec766aa51a29a>@@AEAV<lambda_628dfdc04ba53c8bfc02c9951375f3f5>@@$$QEAV<lambda_f6c7be5f7998530c34de24c7437d6b54>@@@Z 000000018005db00     libucrt:close.obj
 0001:0005cb28       $xdatasym                  000000018005db28     libucrt:fpsr.obj
 0001:0005cb30       $unwind$_fcloseall         000000018005db30     libucrt:closeall.obj
 0001:0005cb54       $unwind$_read              000000018005db54     libucrt:read.obj
 0001:0005cb84       $unwind$_read_nolock       000000018005db84     libucrt:read.obj
 0001:0005cb9c       $unwind$?translate_ansi_or_utf8_nolock@@YAHHQEAD_KQEA_W1@Z 000000018005db9c     libucrt:read.obj
 0001:0005cbb8       $unwind$??$translate_text_mode_nolock@D@@YAHHQEAD_K@Z 000000018005dbb8     libucrt:read.obj
 0001:0005cbd0       $unwind$??$translate_text_mode_nolock@_W@@YAHHQEA_W_K@Z 000000018005dbd0     libucrt:read.obj
 0001:0005cbe8       $unwind$??$common_lseek@J@@YAJHJH@Z 000000018005dbe8     libucrt:lseek.obj
 0001:0005cc18       $unwind$??$common_lseek@_J@@YA_JH_JH@Z 000000018005dc18     libucrt:lseek.obj
 0001:0005cc48       $unwind$_isctype_l         000000018005dc48     libucrt:isctype.obj
 0001:0005cc64       $unwind$_towlower_l        000000018005dc64     libucrt:towlower.obj
 0001:0005cc6c       $unwind$_waccess_s         000000018005dc6c     libucrt:waccess.obj
 0001:0005cc7c       $unwind$_pipe              000000018005dc7c     libucrt:pipe.obj
 0001:0005ccbc       $unwind$??$common_fdopen@_W@@YAPEAU_iobuf@@HQEB_W@Z 000000018005dcbc     libucrt:fdopen.obj
 0001:0005ccdc       $unwind$??$?RV<lambda_a37b2b86f63e897a80ea819b0eb08c01>@@AEAV<lambda_38ce7e780aa69e748d6df282ebc68efe>@@V<lambda_99fb1378e971ab6e7edea83e3a7a83a2>@@@?$__crt_seh_guarded_call@H@@QEAAH$$QEAV<lambda_a37b2b86f63e897a80ea819b0eb08c01>@@AEAV<lambda_38ce7e780aa69e748d6df282ebc68efe>@@$$QEAV<lambda_99fb1378e971ab6e7edea83e3a7a83a2>@@@Z 000000018005dcdc     libucrt:commit.obj
 0001:0005cd00       $unwind$_write             000000018005dd00     libucrt:write.obj
 0001:0005cd30       $unwind$_write_nolock      000000018005dd30     libucrt:write.obj
 0001:0005cd48       $unwind$?write_double_translated_ansi_nolock@@YA?AUwrite_result@?A0x17268360@@HQEBDI@Z 000000018005dd48     libucrt:write.obj
 0001:0005cd68       $unwind$?write_text_ansi_nolock@@YA?AUwrite_result@?A0x17268360@@HQEBDI@Z 000000018005dd68     libucrt:write.obj
 0001:0005cd68       $unwind$?write_text_utf16le_nolock@@YA?AUwrite_result@?A0x17268360@@HQEBDI@Z 000000018005dd68     libucrt:write.obj
 0001:0005cd88       $unwind$?write_text_utf8_nolock@@YA?AUwrite_result@?A0x17268360@@HQEBDI@Z 000000018005dd88     libucrt:write.obj
 0001:0005cdac       $unwind$??$write_buffer_nolock@D@@YA_NDV__crt_stdio_stream@@@Z 000000018005ddac     libucrt:_flsbuf.obj
 0001:0005cdbc       $unwind$__acrt_GetTempPathA 000000018005ddbc     libucrt:gettemppath.obj
 0001:0005cdd4       $unwind$_wsopen_nolock     000000018005ddd4     libucrt:open.obj
 0001:0005cdf0       $unwind$??$common_sopen_dispatch@D@@YAHQEBDHHHQEAHH@Z 000000018005ddf0     libucrt:open.obj
 0001:0005ce14       $unwind$?fin$0@?0???$common_sopen_dispatch@_W@@YAHQEB_WHHHQEAHH@Z@4HA 000000018005de14     libucrt:open.obj
 0001:0005ce14       $unwind$?fin$0@?0???$common_sopen_dispatch@D@@YAHQEBDHHHQEAHH@Z@4HA 000000018005de14     libucrt:open.obj
 0001:0005ce1c       $unwind$??$common_sopen_dispatch@_W@@YAHQEB_WHHHQEAHH@Z 000000018005de1c     libucrt:open.obj
 0001:0005ce40       $unwind$?truncate_ctrl_z_if_present@@YAHH@Z 000000018005de40     libucrt:open.obj
 0001:0005ce50       $unwind$_rmtmp             000000018005de50     libucrt:rmtmp.obj
 0001:0005ce84       $unwind$?accumulate_inheritable_handles@@YA_NQEAPEAEQEA_K_N@Z 000000018005de84     libucrt:spawnv.obj
 0001:0005ce8c       $unwind$??R<lambda_a094494068278ba5130ab06e1292f60a>@@QEBA_NXZ 000000018005de8c     libucrt:spawnv.obj
 0001:0005cea8       $unwind$??$common_spawnv@_W@@YA_JHQEB_WQEBQEB_W1@Z 000000018005dea8     libucrt:spawnv.obj
 0001:0005cec4       $unwind$??$?RV<lambda_a22f0c497e5168315e06dae667770027>@@AEAV<lambda_a094494068278ba5130ab06e1292f60a>@@V<lambda_24dc10c13f43218c635520766e23e324>@@@?$__crt_seh_guarded_call@_N@@QEAA_N$$QEAV<lambda_a22f0c497e5168315e06dae667770027>@@AEAV<lambda_a094494068278ba5130ab06e1292f60a>@@$$QEAV<lambda_24dc10c13f43218c635520766e23e324>@@@Z 000000018005dec4     libucrt:spawnv.obj
 0001:0005cee8       $unwind$??$execute_command@_W@@YA_JHQEB_WQEBQEB_W1@Z 000000018005dee8     libucrt:spawnv.obj
 0001:0005cf04       $unwind$??$common_spawnvp@_W@@YA_JHQEB_WQEBQEB_W1@Z 000000018005df04     libucrt:spawnvp.obj
 0001:0005cf24       $unwind$??$common_expand_argv_wildcards@D@@YAHQEAPEADQEAPEAPEAD@Z 000000018005df24     libucrt:argv_wildcards.obj
 0001:0005cf3c       $unwind$??$copy_and_add_argument_to_buffer@D@@YAHQEBD0_KAEAV?$argument_list@D@?A0x5f5c8891@@@Z 000000018005df3c     libucrt:argv_wildcards.obj
 0001:0005cf3c       $unwind$??$common_set_variable_in_environment_nolock@_W@@YAHQEA_WH@Z 000000018005df3c     libucrt:setenv.obj
 0001:0005cf58       $unwind$??$expand_argument_wildcards@D@@YAHQEAD0AEAV?$argument_list@D@?A0x5f5c8891@@@Z 000000018005df58     libucrt:argv_wildcards.obj
 0001:0005cf78       $unwind$_setmbcp_nolock    000000018005df78     libucrt:mbctype.obj
 0001:0005cf98       $unwind$?update_thread_multibyte_data_internal@@YAPEAU__crt_multibyte_data@@QEAU__acrt_ptd@@QEAPEAU1@@Z 000000018005df98     libucrt:mbctype.obj
 0001:0005cfc0       $unwind$?setmbcp_internal@@YAHH_NQEAU__acrt_ptd@@QEAPEAU__crt_multibyte_data@@@Z 000000018005dfc0     libucrt:mbctype.obj
 0001:0005cfd0       $unwind$?setSBUpLow@@YAXPEAU__crt_multibyte_data@@@Z 000000018005dfd0     libucrt:mbctype.obj
 0001:0005cfec       $unwind$??$?RV<lambda_efdfa57d1f175319df784efa44bb7b81>@@AEAV<lambda_5f0a4c1567f8adc6734073e5d1e1b35c>@@V<lambda_2e8a7d3640ea6ccb4c2413664c2db6fd>@@@?$__crt_seh_guarded_call@X@@QEAAX$$QEAV<lambda_efdfa57d1f175319df784efa44bb7b81>@@AEAV<lambda_5f0a4c1567f8adc6734073e5d1e1b35c>@@$$QEAV<lambda_2e8a7d3640ea6ccb4c2413664c2db6fd>@@@Z 000000018005dfec     libucrt:mbctype.obj
 0001:0005d014       $unwind$?x_ismbbtype_l@@YAHPEAU__crt_locale_pointers@@IHH@Z 000000018005e014     libucrt:ismbbyte.obj
 0001:0005d024       $unwind$??$copy_environment@_W@@YAPEAPEA_WQEAPEA_W@Z 000000018005e024     libucrt:setenv.obj
 0001:0005d03c       $unwind$_query_new_handler 000000018005e03c     libucrt:new_handler.obj
 0001:0005d05c       $unwind$raise              000000018005e05c     libucrt:signal.obj
 0001:0005d088       $unwind$??$?RV<lambda_450d765d439847d4c735a33c368b5fc0>@@AEAV<lambda_44731a7d0e6d81c3e6aa82d741081786>@@V<lambda_601a2a7da3b7a96e9554ac7215c4b07c>@@@?$__crt_seh_guarded_call@P6AXH@Z@@QEAAP6AXH@Z$$QEAV<lambda_450d765d439847d4c735a33c368b5fc0>@@AEAV<lambda_44731a7d0e6d81c3e6aa82d741081786>@@$$QEAV<lambda_601a2a7da3b7a96e9554ac7215c4b07c>@@@Z 000000018005e088     libucrt:signal.obj
 0001:0005d0ac       $unwind$__acrt_LCMapStringA 000000018005e0ac     libucrt:lcmapstringa.obj
 0001:0005d0bc       $unwind$?__acrt_LCMapStringA_stat@@YAHPEAU__crt_locale_pointers@@PEB_WKPEBDHPEADHHH@Z 000000018005e0bc     libucrt:lcmapstringa.obj
 0001:0005d0e4       $unwind$__acrt_update_thread_locale_data 000000018005e0e4     libucrt:locale_refcounting.obj
 0001:0005d108       $unwind$__acrt_fltout      000000018005e108     libucrt:cfout.obj
 0001:0005d128       $unwind$__acrt_locale_free_monetary 000000018005e128     libucrt:initmon.obj
 0001:0005d130       $unwind$__acrt_locale_free_time 000000018005e130     libucrt:inittime.obj
 0001:0005d140       $unwind$__acrt_GetStringTypeA 000000018005e140     libucrt:getstringtypea.obj
 0001:0005d168       $unwind$_alloc_osfhnd      000000018005e168     libucrt:osfinfo.obj
 0001:0005d198       $unwind$__acrt_lowio_destroy_handle_array 000000018005e198     libucrt:osfinfo.obj
 0001:0005d1a8       $unwind$__acrt_lowio_ensure_fh_exists 000000018005e1a8     libucrt:osfinfo.obj
 0001:0005d1d4       $unwind$?GetTableIndexFromLocaleName@@YAHPEB_W@Z 000000018005e1d4     libucrt:lcidtoname_downlevel.obj
 0001:0005d1ec       $unwind$_setmode_nolock    000000018005e1ec     libucrt:setmode.obj
 0001:0005d1fc       $unwind$_putwch_nolock     000000018005e1fc     libucrt:putwch.obj
 0001:0005d204       $unwind$__acrt_fenv_set_control 000000018005e204     libucrt:_fenvutils.obj
 0001:0005d214       $unwind$__acrt_pack_wide_command_line_and_environment 000000018005e214     libucrt:cenvarg.obj
 0001:0005d230       $unwind$??$construct_environment_block@_W@@YAHQEBQEB_WQEAPEA_W@Z 000000018005e230     libucrt:cenvarg.obj
 0001:0005d250       $unwind$qsort              000000018005e250     libucrt:qsort.obj
 0001:0005d268       $chain$4$qsort             000000018005e268     libucrt:qsort.obj
 0001:0005d28c       $chain$5$qsort             000000018005e28c     libucrt:qsort.obj
 0001:0005d2a0       $xdatasym                  000000018005e2a0     libucrt:log10.obj
 0001:0005d2ac       $unwind$_call_matherr      000000018005e2ac     libucrt:libm_error.obj
 0001:0005d2b4       $unwind$_handle_error      000000018005e2b4     libucrt:libm_error.obj
 0001:0005d2d4       $unwind$__acrt_initialize_fma3 000000018005e2d4     libucrt:fma3_available.obj
 0001:0005d2dc       $unwind$_log_special_common 000000018005e2dc     libucrt:log_special.obj
 0001:0005d2e8       $unwind$_raise_exc         000000018005e2e8     libucrt:fpexcept.obj
 0001:0005d2f0       $unwind$_raise_exc_ex      000000018005e2f0     libucrt:fpexcept.obj
 0001:0005d304       $unwind$_ctrlfp            000000018005e304     libucrt:fpctrl.obj
 0001:0005d32c       $unwind$_IsNonwritableInCurrentImage 000000018005e32c     LIBCMT:pesect.obj
 0001:0005d350       $xdatasym                  000000018005e350     LIBCMT:_amdsecgs_.obj
 0001:0005d354       $unwind$__report_securityfailure 000000018005e354     LIBCMT:gs_report.obj
 0001:0005d35c       $unwind$__report_gsfailure 000000018005e35c     LIBCMT:gs_report.obj
 0001:0005d370       .edata                     000000018005e370     luafar3.exp
 0001:0005d398       rgpv                       000000018005e398     luafar3.exp
 0001:0005d440       rgszName                   000000018005e440     luafar3.exp
 0001:0005d4e8       rgwOrd                     000000018005e4e8     luafar3.exp
 0001:0005d53c       szName                     000000018005e53c     luafar3.exp
 0001:0005d548       $N00001                    000000018005e548     luafar3.exp
 0001:0005d553       $N00002                    000000018005e553     luafar3.exp
 0001:0005d563       $N00003                    000000018005e563     luafar3.exp
 0001:0005d571       $N00004                    000000018005e571     luafar3.exp
 0001:0005d57c       $N00005                    000000018005e57c     luafar3.exp
 0001:0005d589       $N00006                    000000018005e589     luafar3.exp
 0001:0005d598       $N00007                    000000018005e598     luafar3.exp
 0001:0005d5a3       $N00008                    000000018005e5a3     luafar3.exp
 0001:0005d5ad       $N00009                    000000018005e5ad     luafar3.exp
 0001:0005d5b8       $N00010                    000000018005e5b8     luafar3.exp
 0001:0005d5cb       $N00011                    000000018005e5cb     luafar3.exp
 0001:0005d5db       $N00012                    000000018005e5db     luafar3.exp
 0001:0005d5ed       $N00013                    000000018005e5ed     luafar3.exp
 0001:0005d601       $N00014                    000000018005e601     luafar3.exp
 0001:0005d60d       $N00015                    000000018005e60d     luafar3.exp
 0001:0005d61c       $N00016                    000000018005e61c     luafar3.exp
 0001:0005d62d       $N00017                    000000018005e62d     luafar3.exp
 0001:0005d63d       $N00018                    000000018005e63d     luafar3.exp
 0001:0005d651       $N00019                    000000018005e651     luafar3.exp
 0001:0005d662       $N00020                    000000018005e662     luafar3.exp
 0001:0005d66a       $N00021                    000000018005e66a     luafar3.exp
 0001:0005d67b       $N00022                    000000018005e67b     luafar3.exp
 0001:0005d68c       $N00023                    000000018005e68c     luafar3.exp
 0001:0005d698       $N00024                    000000018005e698     luafar3.exp
 0001:0005d6a9       $N00025                    000000018005e6a9     luafar3.exp
 0001:0005d6ba       $N00026                    000000018005e6ba     luafar3.exp
 0001:0005d6c5       $N00027                    000000018005e6c5     luafar3.exp
 0001:0005d6cd       $N00028                    000000018005e6cd     luafar3.exp
 0001:0005d6e4       $N00029                    000000018005e6e4     luafar3.exp
 0001:0005d6fa       $N00030                    000000018005e6fa     luafar3.exp
 0001:0005d710       $N00031                    000000018005e710     luafar3.exp
 0001:0005d726       $N00032                    000000018005e726     luafar3.exp
 0001:0005d738       $N00033                    000000018005e738     luafar3.exp
 0001:0005d74b       $N00034                    000000018005e74b     luafar3.exp
 0001:0005d760       $N00035                    000000018005e760     luafar3.exp
 0001:0005d775       $N00036                    000000018005e775     luafar3.exp
 0001:0005d78c       $N00037                    000000018005e78c     luafar3.exp
 0001:0005d7a2       $N00038                    000000018005e7a2     luafar3.exp
 0001:0005d7ae       $N00039                    000000018005e7ae     luafar3.exp
 0001:0005d7c2       $N00040                    000000018005e7c2     luafar3.exp
 0001:0005d7d3       $N00041                    000000018005e7d3     luafar3.exp
 0001:0005d7e3       $N00042                    000000018005e7e3     luafar3.exp
 0002:00001e50       pageMap                    0000000180060e50     slnunico.obj
 0002:00003550       groupMap                   0000000180062550     slnunico.obj
 0002:00005300       groups                     0000000180064300     slnunico.obj
 0002:00005530       ?__vcrt_flsindex@@3KA      0000000180064530     libvcruntime:per_thread_data.obj
 0002:00005540       ?dazSupported@?1??common_control87@@9@9 0000000180064540     libucrt:ieee.obj
 0002:00005544       ?errno_no_memory@@3HA      0000000180064544     libucrt:errno.obj
 0002:00005548       ?doserrno_no_memory@@3KA   0000000180064548     libucrt:errno.obj
 0002:00005664       ?__acrt_flsindex@@3KA      0000000180064664     libucrt:per_thread_data.obj
 0002:00005b60       _mbctypes                  0000000180064b60     libucrt:mbctype.obj
 0002:00005c70       _mbcasemaps                0000000180064c70     libucrt:mbctype.obj
 0002:00005d70       ?__rgctypeflag@@3PADA      0000000180064d70     libucrt:mbctype.obj
 0002:00005d80       ?__rgcode_page_info@@3PAUcode_page_info@@A 0000000180064d80     libucrt:mbctype.obj
 0002:00005f20       ?__dcrt_lowio_console_output_handle@@3PEAXEA 0000000180064f20     libucrt:initcon.obj
 0002:00005f30       ?dazSupported@?1??_ctrlfp@@9@9 0000000180064f30     libucrt:fpctrl.obj
 0002:00005f40       luaopen_bit                0000000180064f40     service.obj
 0002:00005f48       luaopen_ffi                0000000180064f48     service.obj
 0002:00005f50       luaopen_jit                0000000180064f50     service.obj
 0002:00005f58       ?__proc_attached@@3HA      0000000180064f58     LIBCMT:dll_dllmain.obj
 0002:00005f74       ?module_local_atexit_table_initialized@@3_NA 0000000180064f74     LIBCMT:utility.obj
 0002:00005f80       ?module_local_atexit_table@@3U_onexit_table_t@@A 0000000180064f80     LIBCMT:utility.obj
 0002:00005f98       ?module_local_at_quick_exit_table@@3U_onexit_table_t@@A 0000000180064f98     LIBCMT:utility.obj
 0002:00005fb0       ?is_initialized_as_dll@@3_NA 0000000180064fb0     LIBCMT:utility.obj
 0002:00006000       ?heap@@3V_HeapManager@@A   0000000180065000     libvcruntime:undname.obj
 0002:00006030       ?__vcrt_startup_thread_ptd@@3U__vcrt_ptd@@A 0000000180065030     libvcruntime:per_thread_data.obj
 0002:000060a8       __vcrt_lock_table          00000001800650a8     libvcruntime:locks.obj
 0002:000060d0       __vcrt_locks_initialized   00000001800650d0     libvcruntime:locks.obj
 0002:000060d8       ?module_handles@@3PAPEAUHINSTANCE__@@A 00000001800650d8     libvcruntime:winapi_downlevel.obj
 0002:000060f0       ?encoded_function_pointers@@3PAPEAXA 00000001800650f0     libvcruntime:winapi_downlevel.obj
 0002:00006140       ?__idtabsiz@@3IA           0000000180065140     libucrt:popen.obj
 0002:00006148       ?__idpairs@@3PEAUprocess_handle_pair@?A0xe43b7539@@EA 0000000180065148     libucrt:popen.obj
 0002:00006150       ?narrow_tmpfile_buffer_pointers@@3PAPEADA 0000000180065150     libucrt:tmpfile.obj
 0002:00006168       ?wide_tmpfile_buffer_pointers@@3PAPEA_WA 0000000180065168     libucrt:tmpfile.obj
 0002:00006180       ?c_termination_complete@@3JA 0000000180065180     libucrt:exit.obj
 0002:00006188       ?thread_local_exit_callback_func@@3P6AXPEAXK0@ZEA 0000000180065188     libucrt:exit.obj
 0002:000061a0       ?program_name@?1???$common_configure_argv@D@@YAHW4_crt_argv_mode@@@Z@4PADA 00000001800651a0     libucrt:argv_parsing.obj
 0002:000062f8       ?__acrt_invalid_parameter_handler@@3V?$dual_state_global@P6AXPEB_W00I_K@Z@__crt_state_management@@A 00000001800652f8     libucrt:invalid_parameter.obj
 0002:00006300       ?enable_percent_n@@3_KA    0000000180065300     libucrt:printf_count_output.obj
 0002:00006740       ?module_handles@@3PAPEAUHINSTANCE__@@A 0000000180065740     libucrt:winapi_thunks.obj
 0002:000067e0       ?encoded_function_pointers@@3PAPEAXA 00000001800657e0     libucrt:winapi_thunks.obj
 0002:000068f0       ?__acrt_lock_table@@3PAU_RTL_CRITICAL_SECTION@@A 00000001800658f0     libucrt:locks.obj
 0002:00006b20       ?__acrt_locks_initialized@@3IA 0000000180065b20     libucrt:locks.obj
 0002:00006b40       ?fSystemSet@@3HA           0000000180065b40     libucrt:mbctype.obj
 0002:00006b44       ?initialized@?1??__acrt_initialize_multibyte@@9@4_NA 0000000180065b44     libucrt:mbctype.obj
 0002:00006b80       ?__acrt_new_handler@@3V?$dual_state_global@P6AH_K@Z@__crt_state_management@@A 0000000180065b80     libucrt:new_handler.obj
 0002:00006b88       ?ctrlc_action@@3V?$dual_state_global@P6AXH@Z@__crt_state_management@@A 0000000180065b88     libucrt:signal.obj
 0002:00006b90       ?ctrlbreak_action@@3V?$dual_state_global@P6AXH@Z@__crt_state_management@@A 0000000180065b90     libucrt:signal.obj
 0002:00006b98       ?abort_action@@3V?$dual_state_global@P6AXH@Z@__crt_state_management@@A 0000000180065b98     libucrt:signal.obj
 0002:00006ba0       ?term_action@@3V?$dual_state_global@P6AXH@Z@__crt_state_management@@A 0000000180065ba0     libucrt:signal.obj
 0002:00006ba8       ?user_matherr@@3V?$dual_state_global@P6AHPEAU_exception@@@Z@__crt_state_management@@A 0000000180065ba8     libucrt:matherr.obj
 0002:00006bb0       ?__acrt_global_new_mode@@3V?$dual_state_global@J@__crt_state_management@@A 0000000180065bb0     libucrt:new_mode.obj
 0002:00006bc0       ?__acrt_app_type@@3W4_crt_app_type@@A 0000000180065bc0     libucrt:report_runtime_error.obj
 0002:00006bd0       GS_ExceptionRecord         0000000180065bd0     LIBCMT:gs_report.obj
 0002:00006c70       GS_ContextRecord           0000000180065c70     LIBCMT:gs_report.obj
 0003:0000018c       $pdata$sprintf             000000018006718c     bit64.obj
 0003:00000150       $pdata$bit64_pushuserdata  0000000180067150     bit64.obj
 0003:00000144       $pdata$bit64_push          0000000180067144     bit64.obj
 0003:00000120       $pdata$bit64_getvalue      0000000180067120     bit64.obj
 0003:0000012c       $pdata$0$bit64_getvalue    000000018006712c     bit64.obj
 0003:00000138       $pdata$1$bit64_getvalue    0000000180067138     bit64.obj
 0003:0000015c       $pdata$check64             000000018006715c     bit64.obj
 0003:00000168       $pdata$0$check64           0000000180067168     bit64.obj
 0003:00000174       $pdata$1$check64           0000000180067174     bit64.obj
 0003:0000003c       $pdata$band                000000018006703c     bit64.obj
 0003:00000048       $pdata$bor                 0000000180067048     bit64.obj
 0003:00000054       $pdata$bxor                0000000180067054     bit64.obj
 0003:00000060       $pdata$bnot                0000000180067060     bit64.obj
 0003:0000006c       $pdata$lshift              000000018006706c     bit64.obj
 0003:00000078       $pdata$rshift              0000000180067078     bit64.obj
 0003:00000084       $pdata$arshift             0000000180067084     bit64.obj
 0003:00000090       $pdata$f_new               0000000180067090     bit64.obj
 0003:0000009c       $pdata$0$f_new             000000018006709c     bit64.obj
 0003:000000a8       $pdata$1$f_new             00000001800670a8     bit64.obj
 0003:000000b4       $pdata$f_tostring          00000001800670b4     bit64.obj
 0003:000000c0       $pdata$f_type              00000001800670c0     bit64.obj
 0003:000000cc       $pdata$0$f_type            00000001800670cc     bit64.obj
 0003:000000d8       $pdata$1$f_type            00000001800670d8     bit64.obj
 0003:000000e4       $pdata$f_add               00000001800670e4     bit64.obj
 0003:000000f0       $pdata$f_sub               00000001800670f0     bit64.obj
 0003:000000fc       $pdata$f_mul               00000001800670fc     bit64.obj
 0003:00000108       $pdata$f_div               0000000180067108     bit64.obj
 0003:00000114       $pdata$f_mod               0000000180067114     bit64.obj
 0003:0000000c       $pdata$f_unm               000000018006700c     bit64.obj
 0003:00000018       $pdata$f_eq                0000000180067018     bit64.obj
 0003:00000024       $pdata$f_lt                0000000180067024     bit64.obj
 0003:00000030       $pdata$f_le                0000000180067030     bit64.obj
 0003:00000180       $pdata$luaopen_bit64       0000000180067180     bit64.obj
 0003:00000270       $pdata$LF_Analyse          0000000180067270     exported.obj
 0003:0000027c       $pdata$LF_ClosePanel       000000018006727c     exported.obj
 0003:00000288       $pdata$LF_Compare          0000000180067288     exported.obj
 0003:00000294       $pdata$0$LF_Compare        0000000180067294     exported.obj
 0003:000002a0       $pdata$2$LF_Compare        00000001800672a0     exported.obj
 0003:000002ac       $pdata$3$LF_Compare        00000001800672ac     exported.obj
 0003:000002b8       $pdata$LF_Configure        00000001800672b8     exported.obj
 0003:000002c4       $pdata$LF_DeleteFiles      00000001800672c4     exported.obj
 0003:000002d0       $pdata$0$LF_DeleteFiles    00000001800672d0     exported.obj
 0003:000002dc       $pdata$2$LF_DeleteFiles    00000001800672dc     exported.obj
 0003:000002e8       $pdata$3$LF_DeleteFiles    00000001800672e8     exported.obj
 0003:000002f4       $pdata$LF_ExitFAR          00000001800672f4     exported.obj
 0003:0000030c       $pdata$LF_FreeFindData     000000018006730c     exported.obj
 0003:00000360       $pdata$LF_GetFiles         0000000180067360     exported.obj
 0003:0000036c       $pdata$0$LF_GetFiles       000000018006736c     exported.obj
 0003:00000378       $pdata$2$LF_GetFiles       0000000180067378     exported.obj
 0003:00000384       $pdata$3$LF_GetFiles       0000000180067384     exported.obj
 0003:00000390       $pdata$LF_GetFindData      0000000180067390     exported.obj
 0003:0000039c       $pdata$0$LF_GetFindData    000000018006739c     exported.obj
 0003:000003a8       $pdata$1$LF_GetFindData    00000001800673a8     exported.obj
 0003:000003b4       $pdata$LF_GetGlobalInfo    00000001800673b4     exported.obj
 0003:000003c0       $pdata$1$LF_GetGlobalInfo  00000001800673c0     exported.obj
 0003:000003cc       $pdata$2$LF_GetGlobalInfo  00000001800673cc     exported.obj
 0003:000003d8       $pdata$3$LF_GetGlobalInfo  00000001800673d8     exported.obj
 0003:000003e4       $pdata$4$LF_GetGlobalInfo  00000001800673e4     exported.obj
 0003:000003f0       $pdata$LF_GetOpenPanelInfo 00000001800673f0     exported.obj
 0003:000003fc       $pdata$1$LF_GetOpenPanelInfo 00000001800673fc     exported.obj
 0003:00000408       $pdata$3$LF_GetOpenPanelInfo 0000000180067408     exported.obj
 0003:00000414       $pdata$7$LF_GetOpenPanelInfo 0000000180067414     exported.obj
 0003:00000420       $pdata$8$LF_GetOpenPanelInfo 0000000180067420     exported.obj
 0003:0000042c       $pdata$9$LF_GetOpenPanelInfo 000000018006742c     exported.obj
 0003:00000438       $pdata$LF_GetPluginInfo    0000000180067438     exported.obj
 0003:00000444       $pdata$0$LF_GetPluginInfo  0000000180067444     exported.obj
 0003:00000450       $pdata$1$LF_GetPluginInfo  0000000180067450     exported.obj
 0003:0000045c       $pdata$LF_MakeDirectory    000000018006745c     exported.obj
 0003:00000468       $pdata$0$LF_MakeDirectory  0000000180067468     exported.obj
 0003:00000474       $pdata$2$LF_MakeDirectory  0000000180067474     exported.obj
 0003:00000480       $pdata$3$LF_MakeDirectory  0000000180067480     exported.obj
 0003:0000048c       $pdata$LF_Open             000000018006748c     exported.obj
 0003:000004bc       $pdata$LF_ProcessDialogEvent 00000001800674bc     exported.obj
 0003:000004c8       $pdata$LF_ProcessEditorEvent 00000001800674c8     exported.obj
 0003:000004d4       $pdata$0$LF_ProcessEditorEvent 00000001800674d4     exported.obj
 0003:000004e0       $pdata$1$LF_ProcessEditorEvent 00000001800674e0     exported.obj
 0003:000004ec       $pdata$LF_ProcessEditorInput 00000001800674ec     exported.obj
 0003:000004f8       $pdata$LF_ProcessHostFile  00000001800674f8     exported.obj
 0003:00000504       $pdata$LF_ProcessPanelEvent 0000000180067504     exported.obj
 0003:00000510       $pdata$0$LF_ProcessPanelEvent 0000000180067510     exported.obj
 0003:0000051c       $pdata$2$LF_ProcessPanelEvent 000000018006751c     exported.obj
 0003:00000528       $pdata$3$LF_ProcessPanelEvent 0000000180067528     exported.obj
 0003:00000534       $pdata$LF_ProcessPanelInput 0000000180067534     exported.obj
 0003:00000498       $pdata$LF_ProcessConsoleInput 0000000180067498     exported.obj
 0003:000004a4       $pdata$0$LF_ProcessConsoleInput 00000001800674a4     exported.obj
 0003:000004b0       $pdata$1$LF_ProcessConsoleInput 00000001800674b0     exported.obj
 0003:00000540       $pdata$LF_ProcessSynchroEvent 0000000180067540     exported.obj
 0003:0000054c       $pdata$1$LF_ProcessSynchroEvent 000000018006754c     exported.obj
 0003:00000558       $pdata$2$LF_ProcessSynchroEvent 0000000180067558     exported.obj
 0003:00000564       $pdata$3$LF_ProcessSynchroEvent 0000000180067564     exported.obj
 0003:00000570       $pdata$5$LF_ProcessSynchroEvent 0000000180067570     exported.obj
 0003:0000057c       $pdata$6$LF_ProcessSynchroEvent 000000018006757c     exported.obj
 0003:00000588       $pdata$LF_ProcessViewerEvent 0000000180067588     exported.obj
 0003:00000594       $pdata$LF_PutFiles         0000000180067594     exported.obj
 0003:000005a0       $pdata$LF_SetDirectory     00000001800675a0     exported.obj
 0003:000005ac       $pdata$LF_SetFindList      00000001800675ac     exported.obj
 0003:0000033c       $pdata$LF_GetContentFields 000000018006733c     exported.obj
 0003:00000348       $pdata$0$LF_GetContentFields 0000000180067348     exported.obj
 0003:00000354       $pdata$1$LF_GetContentFields 0000000180067354     exported.obj
 0003:00000318       $pdata$LF_GetContentData   0000000180067318     exported.obj
 0003:00000324       $pdata$0$LF_GetContentData 0000000180067324     exported.obj
 0003:00000330       $pdata$1$LF_GetContentData 0000000180067330     exported.obj
 0003:00000300       $pdata$LF_FreeContentData  0000000180067300     exported.obj
 0003:000005b8       $pdata$PackMacroValues     00000001800675b8     exported.obj
 0003:00000684       $pdata$traceback           0000000180067684     exported.obj
 0003:00000264       $pdata$GetExportFunction   0000000180067264     exported.obj
 0003:00000678       $pdata$pcall_msg           0000000180067678     exported.obj
 0003:000005dc       $pdata$PushPluginObject    00000001800675dc     exported.obj
 0003:000005f4       $pdata$ReplacePluginInfoCollector 00000001800675f4     exported.obj
 0003:00000648       $pdata$_AddStringToCollector 0000000180067648     exported.obj
 0003:00000654       $pdata$0$_AddStringToCollector 0000000180067654     exported.obj
 0003:00000660       $pdata$1$_AddStringToCollector 0000000180067660     exported.obj
 0003:00000198       $pdata$AddBufToCollector   0000000180067198     exported.obj
 0003:000001a4       $pdata$CreateStringsArray  00000001800671a4     exported.obj
 0003:000001b0       $pdata$0$CreateStringsArray 00000001800671b0     exported.obj
 0003:000001bc       $pdata$1$CreateStringsArray 00000001800671bc     exported.obj
 0003:000001c8       $pdata$2$CreateStringsArray 00000001800671c8     exported.obj
 0003:000001d4       $pdata$3$CreateStringsArray 00000001800671d4     exported.obj
 0003:000001e0       $pdata$FarPanelItemFreeCallback 00000001800671e0     exported.obj
 0003:00000258       $pdata$FillPluginPanelItem 0000000180067258     exported.obj
 0003:00000234       $pdata$FillFindData        0000000180067234     exported.obj
 0003:00000240       $pdata$1$FillFindData      0000000180067240     exported.obj
 0003:0000024c       $pdata$2$FillFindData      000000018006724c     exported.obj
 0003:00000624       $pdata$UpdateFileSelection 0000000180067624     exported.obj
 0003:00000630       $pdata$0$UpdateFileSelection 0000000180067630     exported.obj
 0003:0000063c       $pdata$1$UpdateFileSelection 000000018006763c     exported.obj
 0003:00000600       $pdata$RunDefaultScript    0000000180067600     exported.obj
 0003:0000060c       $pdata$0$RunDefaultScript  000000018006760c     exported.obj
 0003:00000618       $pdata$1$RunDefaultScript  0000000180067618     exported.obj
 0003:000005e8       $pdata$RegisterObject      00000001800675e8     exported.obj
 0003:000005c4       $pdata$PushAnalyseInfo     00000001800675c4     exported.obj
 0003:000005d0       $pdata$PushFarMacroValue   00000001800675d0     exported.obj
 0003:00000210       $pdata$FillFarMacroCall_Callback 0000000180067210     exported.obj
 0003:0000021c       $pdata$0$FillFarMacroCall_Callback 000000018006721c     exported.obj
 0003:00000228       $pdata$1$FillFarMacroCall_Callback 0000000180067228     exported.obj
 0003:000001ec       $pdata$FillFarMacroCall    00000001800671ec     exported.obj
 0003:000001f8       $pdata$3$FillFarMacroCall  00000001800671f8     exported.obj
 0003:00000204       $pdata$4$FillFarMacroCall  0000000180067204     exported.obj
 0003:0000066c       $pdata$getPluginMenuItems  000000018006766c     exported.obj
 0003:00000690       $pdata$push_flags_table    0000000180067690     flags.obj
 0003:0000069c       $pdata$SetFarColors        000000018006769c     keysandcolors.obj
 0003:000006a8       $pdata$LF_Gsub             00000001800676a8     lflua.obj
 0003:000006b4       $pdata$LF_LoadFile         00000001800676b4     lflua.obj
 0003:000006c0       $pdata$1$LF_LoadFile       00000001800676c0     lflua.obj
 0003:000006cc       $pdata$2$LF_LoadFile       00000001800676cc     lflua.obj
 0003:000006d8       $pdata$3$LF_LoadFile       00000001800676d8     lflua.obj
 0003:000006e4       $pdata$4$LF_LoadFile       00000001800676e4     lflua.obj
 0003:000006fc       $pdata$getF                00000001800676fc     lflua.obj
 0003:000006f0       $pdata$errfile             00000001800676f0     lflua.obj
 0003:00000714       $pdata$luaB_loadfileW      0000000180067714     lflua.obj
 0003:00000708       $pdata$luaB_dofileW        0000000180067708     lflua.obj
 0003:00000720       $pdata$method_gc           0000000180067720     lregex.obj
 0003:0000072c       $pdata$method_tostring     000000018006772c     lregex.obj
 0003:0000078c       $pdata$check_regex_pattern 000000018006778c     lregex.obj
 0003:00000798       $pdata$1$check_regex_pattern 0000000180067798     lregex.obj
 0003:000007a4       $pdata$2$check_regex_pattern 00000001800677a4     lregex.obj
 0003:000007bc       $pdata$push_far_regex      00000001800677bc     lregex.obj
 0003:0000075c       $pdata$_regex_gmatch_closure 000000018006775c     lregex.obj
 0003:00000768       $pdata$1$_regex_gmatch_closure 0000000180067768     lregex.obj
 0003:00000774       $pdata$2$_regex_gmatch_closure 0000000180067774     lregex.obj
 0003:00000780       $pdata$3$_regex_gmatch_closure 0000000180067780     lregex.obj
 0003:00000750       $pdata$_Gmatch             0000000180067750     lregex.obj
 0003:000007c8       $pdata$rx_find_match       00000001800677c8     lregex.obj
 0003:00000738       $pdata$method_bracketscount 0000000180067738     lregex.obj
 0003:000007d4       $pdata$rx_gsub             00000001800677d4     lregex.obj
 0003:00000744       $pdata$func_New            0000000180067744     lregex.obj
 0003:000007b0       $pdata$luaopen_regex       00000001800677b0     lregex.obj
 0003:000007e0       $pdata$FL_PushParams       00000001800677e0     luamacro.obj
 0003:000007ec       $pdata$0$FL_PushParams     00000001800677ec     luamacro.obj
 0003:000007f8       $pdata$1$FL_PushParams     00000001800677f8     luamacro.obj
 0003:00000804       $pdata$2$FL_PushParams     0000000180067804     luamacro.obj
 0003:00000810       $pdata$3$FL_PushParams     0000000180067810     luamacro.obj
 0003:0000081c       $pdata$4$FL_PushParams     000000018006781c     luamacro.obj
 0003:00000828       $pdata$5$FL_PushParams     0000000180067828     luamacro.obj
 0003:00000834       $pdata$InitMPR             0000000180067834     luamacro.obj
 0003:00000840       $pdata$Open_Luamacro       0000000180067840     luamacro.obj
 0003:0000084c       $pdata$0$Open_Luamacro     000000018006784c     luamacro.obj
 0003:00000858       $pdata$1$Open_Luamacro     0000000180067858     luamacro.obj
 0003:00000888       $pdata$far_MacroCallFar    0000000180067888     luamacro.obj
 0003:00000894       $pdata$1$far_MacroCallFar  0000000180067894     luamacro.obj
 0003:000008a0       $pdata$3$far_MacroCallFar  00000001800678a0     luamacro.obj
 0003:000008ac       $pdata$4$far_MacroCallFar  00000001800678ac     luamacro.obj
 0003:000008b8       $pdata$5$far_MacroCallFar  00000001800678b8     luamacro.obj
 0003:00000864       $pdata$far_FarMacroCallToLua 0000000180067864     luamacro.obj
 0003:00000870       $pdata$0$far_FarMacroCallToLua 0000000180067870     luamacro.obj
 0003:0000087c       $pdata$1$far_FarMacroCallToLua 000000018006787c     luamacro.obj
 0003:000008c4       $pdata$uc_tostring         00000001800678c4     lusercontrol.obj
 0003:000008d0       $pdata$uc_len              00000001800678d0     lusercontrol.obj
 0003:000008dc       $pdata$uc_index            00000001800678dc     lusercontrol.obj
 0003:000008e8       $pdata$uc_newindex         00000001800678e8     lusercontrol.obj
 0003:000008f4       $pdata$uc_New              00000001800678f4     lusercontrol.obj
 0003:00000900       $pdata$luaopen_usercontrol 0000000180067900     lusercontrol.obj
 0003:0000090c       $pdata$CreateRegKey        000000018006790c     reg.obj
 0003:00000918       $pdata$OpenRegKey          0000000180067918     reg.obj
 0003:0000093c       $pdata$SetRegKeyStr        000000018006793c     reg.obj
 0003:00000930       $pdata$SetRegKeyDword      0000000180067930     reg.obj
 0003:00000924       $pdata$SetRegKeyArr        0000000180067924     reg.obj
 0003:00001674       $pdata$fprintf             0000000180068674     service.obj
 0003:000013a4       $pdata$GetPluginData       00000001800683a4     service.obj
 0003:000013ec       $pdata$LF_GetLuafarAPI     00000001800683ec     service.obj
 0003:000013b0       $pdata$LF_DlgProc          00000001800683b0     service.obj
 0003:000013bc       $pdata$1$LF_DlgProc        00000001800683bc     service.obj
 0003:000013c8       $pdata$2$LF_DlgProc        00000001800683c8     service.obj
 0003:000013f8       $pdata$LF_InitLuaState1    00000001800683f8     service.obj
 0003:00001404       $pdata$LF_InitLuaState2    0000000180068404     service.obj
 0003:000013d4       $pdata$LF_DoFile           00000001800683d4     service.obj
 0003:00001410       $pdata$LF_Message          0000000180068410     service.obj
 0003:0000141c       $pdata$LF_RunLuafarInit    000000018006841c     service.obj
 0003:0000153c       $pdata$PushPanelItem       000000018006853c     service.obj
 0003:00001548       $pdata$0$PushPanelItem     0000000180068548     service.obj
 0003:00001554       $pdata$1$PushPanelItem     0000000180068554     service.obj
 0003:00001560       $pdata$3$PushPanelItem     0000000180068560     service.obj
 0003:0000156c       $pdata$4$PushPanelItem     000000018006856c     service.obj
 0003:00001578       $pdata$PushPanelItems      0000000180068578     service.obj
 0003:00001584       $pdata$3$PushPanelItems    0000000180068584     service.obj
 0003:00001590       $pdata$4$PushPanelItems    0000000180068590     service.obj
 0003:00001440       $pdata$NewDialogData       0000000180068440     service.obj
 0003:00001374       $pdata$GetFarColor         0000000180068374     service.obj
 0003:00001524       $pdata$PushFarColor        0000000180068524     service.obj
 0003:000012fc       $pdata$DllMain             00000001800682fc     service.obj
 0003:00001308       $pdata$0$DllMain           0000000180068308     service.obj
 0003:00001314       $pdata$1$DllMain           0000000180068314     service.obj
 0003:00001398       $pdata$GetLuaStateTimerQueue 0000000180068398     service.obj
 0003:000012e4       $pdata$DeleteLuaStateTimerQueue 00000001800682e4     service.obj
 0003:00001464       $pdata$OptHandle           0000000180068464     service.obj
 0003:0000168c       $pdata$get_env_flag        000000018006868c     service.obj
 0003:0000165c       $pdata$check_env_flag      000000018006865c     service.obj
 0003:00001380       $pdata$GetFlagCombination  0000000180068380     service.obj
 0003:0000129c       $pdata$CheckFlags          000000018006829c     service.obj
 0003:00001458       $pdata$OptFlags            0000000180068458     service.obj
 0003:000012a8       $pdata$CheckFlagsFromTable 00000001800682a8     service.obj
 0003:0000138c       $pdata$GetFlagsFromTable   000000018006838c     service.obj
 0003:000015a8       $pdata$PutFlagsToTable     00000001800685a8     service.obj
 0003:0000159c       $pdata$PushPluginHandle    000000018006859c     service.obj
 0003:000012b4       $pdata$ConvertLuaValue     00000001800682b4     service.obj
 0003:00000948       $pdata$far_GetFileOwner    0000000180067948     service.obj
 0003:00000954       $pdata$far_GetNumberOfLinks 0000000180067954     service.obj
 0003:0000132c       $pdata$FillEditorSetPosition 000000018006832c     service.obj
 0003:00000960       $pdata$far_PluginStartupInfo 0000000180067960     service.obj
 0003:0000096c       $pdata$far_GetCurrentDirectory 000000018006796c     service.obj
 0003:00000978       $pdata$editor_GetFileName  0000000180067978     service.obj
 0003:00000984       $pdata$editor_GetInfo      0000000180067984     service.obj
 0003:00000990       $pdata$2$editor_GetInfo    0000000180067990     service.obj
 0003:0000099c       $pdata$3$editor_GetInfo    000000018006799c     service.obj
 0003:000009a8       $pdata$4$editor_GetInfo    00000001800679a8     service.obj
 0003:000009b4       $pdata$5$editor_GetInfo    00000001800679b4     service.obj
 0003:0000162c       $pdata$_EditorGetString    000000018006862c     service.obj
 0003:00001644       $pdata$_EditorSetString    0000000180068644     service.obj
 0003:000009c0       $pdata$editor_InsertString 00000001800679c0     service.obj
 0003:000009cc       $pdata$editor_DeleteString 00000001800679cc     service.obj
 0003:00001638       $pdata$_EditorInsertText   0000000180068638     service.obj
 0003:000009d8       $pdata$editor_InsertText   00000001800679d8     service.obj
 0003:000009e4       $pdata$editor_DeleteChar   00000001800679e4     service.obj
 0003:000009f0       $pdata$editor_DeleteBlock  00000001800679f0     service.obj
 0003:000009fc       $pdata$editor_UndoRedo     00000001800679fc     service.obj
 0003:00001344       $pdata$FillKeyBarTitles    0000000180068344     service.obj
 0003:00001350       $pdata$1$FillKeyBarTitles  0000000180068350     service.obj
 0003:0000135c       $pdata$2$FillKeyBarTitles  000000018006835c     service.obj
 0003:000015fc       $pdata$SetKeyBar           00000001800685fc     service.obj
 0003:00000a08       $pdata$editor_SetParam     0000000180067a08     service.obj
 0003:00000a14       $pdata$editor_SetPosition  0000000180067a14     service.obj
 0003:00000a20       $pdata$editor_Redraw       0000000180067a20     service.obj
 0003:00000a2c       $pdata$editor_ExpandTabs   0000000180067a2c     service.obj
 0003:000014b8       $pdata$PushBookmarks       00000001800684b8     service.obj
 0003:000014c4       $pdata$0$PushBookmarks     00000001800684c4     service.obj
 0003:000014d0       $pdata$1$PushBookmarks     00000001800684d0     service.obj
 0003:00000a38       $pdata$editor_AddSessionBookmark 0000000180067a38     service.obj
 0003:00000a44       $pdata$editor_ClearSessionBookmarks 0000000180067a44     service.obj
 0003:00000a50       $pdata$editor_DeleteSessionBookmark 0000000180067a50     service.obj
 0003:00000a5c       $pdata$editor_NextSessionBookmark 0000000180067a5c     service.obj
 0003:00000a68       $pdata$editor_PrevSessionBookmark 0000000180067a68     service.obj
 0003:00000a74       $pdata$editor_SetTitle     0000000180067a74     service.obj
 0003:00000a80       $pdata$editor_GetTitle     0000000180067a80     service.obj
 0003:00000a8c       $pdata$editor_Quit         0000000180067a8c     service.obj
 0003:00001320       $pdata$FillEditorSelect    0000000180068320     service.obj
 0003:00000a98       $pdata$editor_Select       0000000180067a98     service.obj
 0003:00000aa4       $pdata$editor_GetSelection 0000000180067aa4     service.obj
 0003:00001650       $pdata$_EditorTabConvert   0000000180068650     service.obj
 0003:00000ab0       $pdata$editor_AddColor     0000000180067ab0     service.obj
 0003:00000abc       $pdata$editor_DelColor     0000000180067abc     service.obj
 0003:00000ac8       $pdata$editor_GetColor     0000000180067ac8     service.obj
 0003:00000ad4       $pdata$editor_SaveFile     0000000180067ad4     service.obj
 0003:00001530       $pdata$PushInputRecord     0000000180068530     service.obj
 0003:00000ae0       $pdata$editor_ReadInput    0000000180067ae0     service.obj
 0003:00001338       $pdata$FillInputRecord     0000000180068338     service.obj
 0003:00001470       $pdata$OptInputRecord      0000000180068470     service.obj
 0003:00000aec       $pdata$editor_ProcessInput 0000000180067aec     service.obj
 0003:00000af8       $pdata$editor_SubscribeChangeEvent 0000000180067af8     service.obj
 0003:00000b04       $pdata$far_Menu            0000000180067b04     service.obj
 0003:000013e0       $pdata$LF_Error            00000001800683e0     service.obj
 0003:00000b10       $pdata$far_Message         0000000180067b10     service.obj
 0003:00000b1c       $pdata$panel_CheckPanelsExist 0000000180067b1c     service.obj
 0003:00000b28       $pdata$panel_ClosePanel    0000000180067b28     service.obj
 0003:00000b34       $pdata$panel_GetPanelInfo  0000000180067b34     service.obj
 0003:00000b40       $pdata$0$panel_GetPanelInfo 0000000180067b40     service.obj
 0003:00000b4c       $pdata$1$panel_GetPanelInfo 0000000180067b4c     service.obj
 0003:00001698       $pdata$get_panel_item      0000000180068698     service.obj
 0003:000016a4       $pdata$get_string_info     00000001800686a4     service.obj
 0003:00000b58       $pdata$panel_RedrawPanel   0000000180067b58     service.obj
 0003:00001608       $pdata$SetPanelBooleanProperty 0000000180068608     service.obj
 0003:00001614       $pdata$SetPanelIntegerProperty 0000000180068614     service.obj
 0003:00000b64       $pdata$panel_GetPanelDirectory 0000000180067b64     service.obj
 0003:00000b70       $pdata$panel_SetPanelDirectory 0000000180067b70     service.obj
 0003:00000b7c       $pdata$panel_GetCmdLine    0000000180067b7c     service.obj
 0003:00000b88       $pdata$panel_SetCmdLine    0000000180067b88     service.obj
 0003:00000b94       $pdata$panel_GetCmdLinePos 0000000180067b94     service.obj
 0003:00000ba0       $pdata$panel_SetCmdLinePos 0000000180067ba0     service.obj
 0003:00000bac       $pdata$panel_InsertCmdLine 0000000180067bac     service.obj
 0003:00000bb8       $pdata$panel_GetCmdLineSelection 0000000180067bb8     service.obj
 0003:00000bc4       $pdata$panel_SetCmdLineSelection 0000000180067bc4     service.obj
 0003:00001278       $pdata$ChangePanelSelection 0000000180068278     service.obj
 0003:00001284       $pdata$1$ChangePanelSelection 0000000180068284     service.obj
 0003:00001290       $pdata$2$ChangePanelSelection 0000000180068290     service.obj
 0003:00000bd0       $pdata$panel_SetUserScreen 0000000180067bd0     service.obj
 0003:00000bdc       $pdata$panel_GetUserScreen 0000000180067bdc     service.obj
 0003:00000be8       $pdata$panel_IsActivePanel 0000000180067be8     service.obj
 0003:00000bf4       $pdata$panel_SetActivePanel 0000000180067bf4     service.obj
 0003:00000c00       $pdata$far_GetDirList      0000000180067c00     service.obj
 0003:00000c0c       $pdata$0$far_GetDirList    0000000180067c0c     service.obj
 0003:00000c18       $pdata$6$far_GetDirList    0000000180067c18     service.obj
 0003:00000c24       $pdata$7$far_GetDirList    0000000180067c24     service.obj
 0003:00000c30       $pdata$8$far_GetDirList    0000000180067c30     service.obj
 0003:00000c3c       $pdata$far_GetPluginDirList 0000000180067c3c     service.obj
 0003:00000c48       $pdata$far_RestoreScreen   0000000180067c48     service.obj
 0003:00000c54       $pdata$far_SaveScreen      0000000180067c54     service.obj
 0003:000012c0       $pdata$CreateList          00000001800682c0     service.obj
 0003:000012cc       $pdata$2$CreateList        00000001800682cc     service.obj
 0003:000012d8       $pdata$3$CreateList        00000001800682d8     service.obj
 0003:000015f0       $pdata$SetFarDialogItem    00000001800685f0     service.obj
 0003:000014f4       $pdata$PushDlgItem         00000001800684f4     service.obj
 0003:00001500       $pdata$1$PushDlgItem       0000000180068500     service.obj
 0003:0000150c       $pdata$2$PushDlgItem       000000018006850c     service.obj
 0003:00001518       $pdata$PushDlgItemNum      0000000180068518     service.obj
 0003:000015e4       $pdata$SetDlgItem          00000001800685e4     service.obj
 0003:000012f0       $pdata$DialogHandleEqual   00000001800682f0     service.obj
 0003:000014dc       $pdata$PushDMParams        00000001800684dc     service.obj
 0003:00000c60       $pdata$far_SendDlgMessage  0000000180067c60     service.obj
 0003:000014e8       $pdata$PushDNParams        00000001800684e8     service.obj
 0003:0000147c       $pdata$ProcessDNResult     000000018006847c     service.obj
 0003:00001488       $pdata$0$ProcessDNResult   0000000180068488     service.obj
 0003:00001494       $pdata$1$ProcessDNResult   0000000180068494     service.obj
 0003:000014a0       $pdata$2$ProcessDNResult   00000001800684a0     service.obj
 0003:000014ac       $pdata$3$ProcessDNResult   00000001800684ac     service.obj
 0003:00000c6c       $pdata$far_DialogInit      0000000180067c6c     service.obj
 0003:00000c78       $pdata$0$far_DialogInit    0000000180067c78     service.obj
 0003:00000c84       $pdata$1$far_DialogInit    0000000180067c84     service.obj
 0003:00001680       $pdata$free_dialog         0000000180068680     service.obj
 0003:00000c90       $pdata$far_DialogRun       0000000180067c90     service.obj
 0003:00000c9c       $pdata$far_DialogFree      0000000180067c9c     service.obj
 0003:00000ca8       $pdata$dialog_tostring     0000000180067ca8     service.obj
 0003:00000cb4       $pdata$dialog_rawhandle    0000000180067cb4     service.obj
 0003:00000cc0       $pdata$far_GetDlgItem      0000000180067cc0     service.obj
 0003:00000ccc       $pdata$far_SetDlgItem      0000000180067ccc     service.obj
 0003:00000cd8       $pdata$far_SubscribeDialogDrawEvents 0000000180067cd8     service.obj
 0003:00000ce4       $pdata$editor_Editor       0000000180067ce4     service.obj
 0003:00000cf0       $pdata$viewer_Viewer       0000000180067cf0     service.obj
 0003:00000cfc       $pdata$viewer_GetFileName  0000000180067cfc     service.obj
 0003:00000d08       $pdata$viewer_GetInfo      0000000180067d08     service.obj
 0003:00000d14       $pdata$1$viewer_GetInfo    0000000180067d14     service.obj
 0003:00000d20       $pdata$2$viewer_GetInfo    0000000180067d20     service.obj
 0003:00000d2c       $pdata$3$viewer_GetInfo    0000000180067d2c     service.obj
 0003:00000d38       $pdata$4$viewer_GetInfo    0000000180067d38     service.obj
 0003:00000d44       $pdata$viewer_Quit         0000000180067d44     service.obj
 0003:00000d50       $pdata$viewer_Redraw       0000000180067d50     service.obj
 0003:00000d5c       $pdata$viewer_Select       0000000180067d5c     service.obj
 0003:00000d68       $pdata$viewer_SetPosition  0000000180067d68     service.obj
 0003:00000d74       $pdata$2$viewer_SetPosition 0000000180067d74     service.obj
 0003:00000d80       $pdata$3$viewer_SetPosition 0000000180067d80     service.obj
 0003:00000d8c       $pdata$viewer_SetMode      0000000180067d8c     service.obj
 0003:00000d98       $pdata$far_ShowHelp        0000000180067d98     service.obj
 0003:00000da4       $pdata$far_InputBox        0000000180067da4     service.obj
 0003:00000db0       $pdata$far_GetMsg          0000000180067db0     service.obj
 0003:00000dbc       $pdata$far_Text            0000000180067dbc     service.obj
 0003:00000dc8       $pdata$far_CopyToClipboard 0000000180067dc8     service.obj
 0003:00000dd4       $pdata$1$far_CopyToClipboard 0000000180067dd4     service.obj
 0003:00000de0       $pdata$2$far_CopyToClipboard 0000000180067de0     service.obj
 0003:00000dec       $pdata$far_PasteFromClipboard 0000000180067dec     service.obj
 0003:00000df8       $pdata$far_InputRecordToName 0000000180067df8     service.obj
 0003:00000e04       $pdata$far_NameToInputRecord 0000000180067e04     service.obj
 0003:00000e10       $pdata$far_LStricmp        0000000180067e10     service.obj
 0003:00000e1c       $pdata$far_LStrnicmp       0000000180067e1c     service.obj
 0003:00000e28       $pdata$far_ProcessName     0000000180067e28     service.obj
 0003:00000e34       $pdata$1$far_ProcessName   0000000180067e34     service.obj
 0003:00000e40       $pdata$2$far_ProcessName   0000000180067e40     service.obj
 0003:00000e4c       $pdata$3$far_ProcessName   0000000180067e4c     service.obj
 0003:00000e58       $pdata$4$far_ProcessName   0000000180067e58     service.obj
 0003:00000e64       $pdata$5$far_ProcessName   0000000180067e64     service.obj
 0003:00000e70       $pdata$6$far_ProcessName   0000000180067e70     service.obj
 0003:00000e7c       $pdata$far_GetReparsePointInfo 0000000180067e7c     service.obj
 0003:00000e88       $pdata$0$far_GetReparsePointInfo 0000000180067e88     service.obj
 0003:00000e94       $pdata$1$far_GetReparsePointInfo 0000000180067e94     service.obj
 0003:00000ea0       $pdata$far_LIsAlpha        0000000180067ea0     service.obj
 0003:00000eac       $pdata$far_LIsAlphanum     0000000180067eac     service.obj
 0003:00000eb8       $pdata$far_LIsLower        0000000180067eb8     service.obj
 0003:00000ec4       $pdata$far_LIsUpper        0000000180067ec4     service.obj
 0003:00000ed0       $pdata$far_LLowerBuf       0000000180067ed0     service.obj
 0003:00000edc       $pdata$far_LUpperBuf       0000000180067edc     service.obj
 0003:00000ee8       $pdata$far_MkTemp          0000000180067ee8     service.obj
 0003:00000ef4       $pdata$far_MkLink          0000000180067ef4     service.obj
 0003:00000f00       $pdata$far_GetPathRoot     0000000180067f00     service.obj
 0003:000016ec       $pdata$truncstring         00000001800686ec     service.obj
 0003:00001368       $pdata$FrsUserFunc         0000000180068368     service.obj
 0003:00000f0c       $pdata$far_RecursiveSearch 0000000180067f0c     service.obj
 0003:00000f18       $pdata$far_ConvertPath     0000000180067f18     service.obj
 0003:00000f24       $pdata$far_AdvControl      0000000180067f24     service.obj
 0003:00000f30       $pdata$0$far_AdvControl    0000000180067f30     service.obj
 0003:00000f3c       $pdata$1$far_AdvControl    0000000180067f3c     service.obj
 0003:00000f48       $pdata$far_MacroLoadAll    0000000180067f48     service.obj
 0003:00000f54       $pdata$0$far_MacroLoadAll  0000000180067f54     service.obj
 0003:00000f60       $pdata$1$far_MacroLoadAll  0000000180067f60     service.obj
 0003:00000f6c       $pdata$far_MacroSaveAll    0000000180067f6c     service.obj
 0003:00000f78       $pdata$far_MacroGetState   0000000180067f78     service.obj
 0003:00000f84       $pdata$far_MacroGetArea    0000000180067f84     service.obj
 0003:00001434       $pdata$MacroSendString     0000000180068434     service.obj
 0003:00000f90       $pdata$far_MacroGetLastError 0000000180067f90     service.obj
 0003:00000f9c       $pdata$0$far_MacroGetLastError 0000000180067f9c     service.obj
 0003:00000fa8       $pdata$1$far_MacroGetLastError 0000000180067fa8     service.obj
 0003:00001428       $pdata$MacroAddCallback    0000000180068428     service.obj
 0003:00000fb4       $pdata$far_MacroAdd        0000000180067fb4     service.obj
 0003:00000fc0       $pdata$far_MacroDelete     0000000180067fc0     service.obj
 0003:0000126c       $pdata$AddMacroData_gc     000000018006826c     service.obj
 0003:00000fcc       $pdata$far_MacroExecute    0000000180067fcc     service.obj
 0003:00000fd8       $pdata$2$far_MacroExecute  0000000180067fd8     service.obj
 0003:00000fe4       $pdata$3$far_MacroExecute  0000000180067fe4     service.obj
 0003:00000ff0       $pdata$far_CPluginStartupInfo 0000000180067ff0     service.obj
 0003:00000ffc       $pdata$far_MakeMenuItems   0000000180067ffc     service.obj
 0003:00001008       $pdata$1$far_MakeMenuItems 0000000180068008     service.obj
 0003:00001014       $pdata$5$far_MakeMenuItems 0000000180068014     service.obj
 0003:00001020       $pdata$6$far_MakeMenuItems 0000000180068020     service.obj
 0003:0000102c       $pdata$8$far_MakeMenuItems 000000018006802c     service.obj
 0003:00001038       $pdata$9$far_MakeMenuItems 0000000180068038     service.obj
 0003:00001044       $pdata$far_Show            0000000180068044     service.obj
 0003:0000144c       $pdata$NewVirtualKeyTable  000000018006844c     service.obj
 0003:00001050       $pdata$far_CreateFileFilter 0000000180068050     service.obj
 0003:0000105c       $pdata$filefilter_Free     000000018006805c     service.obj
 0003:00001068       $pdata$filefilter_gc       0000000180068068     service.obj
 0003:00001074       $pdata$filefilter_tostring 0000000180068074     service.obj
 0003:00001080       $pdata$filefilter_OpenMenu 0000000180068080     service.obj
 0003:0000108c       $pdata$filefilter_Starting 000000018006808c     service.obj
 0003:00001098       $pdata$filefilter_IsFileInFilter 0000000180068098     service.obj
 0003:000016bc       $pdata$plugin_load         00000001800686bc     service.obj
 0003:000010a4       $pdata$far_UnloadPlugin    00000001800680a4     service.obj
 0003:000010b0       $pdata$far_FindPlugin      00000001800680b0     service.obj
 0003:000015b4       $pdata$PutPluginMenuItemToTable 00000001800685b4     service.obj
 0003:000015c0       $pdata$0$PutPluginMenuItemToTable 00000001800685c0     service.obj
 0003:000015cc       $pdata$1$PutPluginMenuItemToTable 00000001800685cc     service.obj
 0003:000015d8       $pdata$PutVersionInfoToTable 00000001800685d8     service.obj
 0003:000010bc       $pdata$far_GetPluginInformation 00000001800680bc     service.obj
 0003:000010c8       $pdata$far_GetPlugins      00000001800680c8     service.obj
 0003:000010d4       $pdata$1$far_GetPlugins    00000001800680d4     service.obj
 0003:000010e0       $pdata$2$far_GetPlugins    00000001800680e0     service.obj
 0003:000010ec       $pdata$3$far_GetPlugins    00000001800680ec     service.obj
 0003:000010f8       $pdata$4$far_GetPlugins    00000001800680f8     service.obj
 0003:00001104       $pdata$far_IsPluginLoaded  0000000180068104     service.obj
 0003:00001110       $pdata$0$far_IsPluginLoaded 0000000180068110     service.obj
 0003:0000111c       $pdata$1$far_IsPluginLoaded 000000018006811c     service.obj
 0003:00001128       $pdata$far_XLat            0000000180068128     service.obj
 0003:00001134       $pdata$far_FormatFileSize  0000000180068134     service.obj
 0003:00001140       $pdata$far_FarClock        0000000180068140     service.obj
 0003:00001620       $pdata$TimerCallback       0000000180068620     service.obj
 0003:0000114c       $pdata$far_Timer           000000018006814c     service.obj
 0003:000016c8       $pdata$timer_Close         00000001800686c8     service.obj
 0003:000016d4       $pdata$0$timer_Close       00000001800686d4     service.obj
 0003:000016e0       $pdata$1$timer_Close       00000001800686e0     service.obj
 0003:00001158       $pdata$timer_gc            0000000180068158     service.obj
 0003:00001164       $pdata$0$timer_gc          0000000180068164     service.obj
 0003:00001170       $pdata$1$timer_gc          0000000180068170     service.obj
 0003:0000117c       $pdata$timer_tostring      000000018006817c     service.obj
 0003:00001188       $pdata$timer_index         0000000180068188     service.obj
 0003:00001194       $pdata$timer_newindex      0000000180068194     service.obj
 0003:00001668       $pdata$dir_exist           0000000180068668     service.obj
 0003:000011a0       $pdata$far_CreateSettings  00000001800681a0     service.obj
 0003:000011ac       $pdata$Settings_set        00000001800681ac     service.obj
 0003:000011b8       $pdata$Settings_get        00000001800681b8     service.obj
 0003:000011c4       $pdata$Settings_delete     00000001800681c4     service.obj
 0003:000011d0       $pdata$Settings_createsubkey 00000001800681d0     service.obj
 0003:000011dc       $pdata$Settings_opensubkey 00000001800681dc     service.obj
 0003:000011e8       $pdata$Settings_enum       00000001800681e8     service.obj
 0003:000011f4       $pdata$0$Settings_enum     00000001800681f4     service.obj
 0003:00001200       $pdata$2$Settings_enum     0000000180068200     service.obj
 0003:0000120c       $pdata$3$Settings_enum     000000018006820c     service.obj
 0003:00001218       $pdata$5$Settings_enum     0000000180068218     service.obj
 0003:00001224       $pdata$6$Settings_enum     0000000180068224     service.obj
 0003:00001230       $pdata$Settings_free       0000000180068230     service.obj
 0003:0000123c       $pdata$far_FreeSettings    000000018006823c     service.obj
 0003:00001248       $pdata$Settings_tostring   0000000180068248     service.obj
 0003:00001254       $pdata$far_ColorDialog     0000000180068254     service.obj
 0003:00001260       $pdata$far_RunDefaultScript 0000000180068260     service.obj
 0003:000016b0       $pdata$luaopen_far         00000001800686b0     service.obj
 0003:000017f4       $pdata$_snwprintf          00000001800687f4     slnunico.obj
 0003:00001944       $pdata$utf8_enco           0000000180068944     slnunico.obj
 0003:00001974       $pdata$utf8_oced           0000000180068974     slnunico.obj
 0003:00001950       $pdata$utf8_graphext       0000000180068950     slnunico.obj
 0003:0000195c       $pdata$0$utf8_graphext     000000018006895c     slnunico.obj
 0003:00001968       $pdata$1$utf8_graphext     0000000180068968     slnunico.obj
 0003:00001908       $pdata$utf8_count          0000000180068908     slnunico.obj
 0003:00001914       $pdata$0$utf8_count        0000000180068914     slnunico.obj
 0003:00001920       $pdata$1$utf8_count        0000000180068920     slnunico.obj
 0003:0000192c       $pdata$2$utf8_count        000000018006892c     slnunico.obj
 0003:00001938       $pdata$3$utf8_count        0000000180068938     slnunico.obj
 0003:000016f8       $pdata$unic_len            00000001800686f8     slnunico.obj
 0003:00001704       $pdata$unic_sub            0000000180068704     slnunico.obj
 0003:00001710       $pdata$str_reverse         0000000180068710     slnunico.obj
 0003:0000171c       $pdata$0$str_reverse       000000018006871c     slnunico.obj
 0003:00001728       $pdata$1$str_reverse       0000000180068728     slnunico.obj
 0003:00001734       $pdata$unic_lower          0000000180068734     slnunico.obj
 0003:00001740       $pdata$0$unic_lower        0000000180068740     slnunico.obj
 0003:0000174c       $pdata$1$unic_lower        000000018006874c     slnunico.obj
 0003:00001758       $pdata$unic_upper          0000000180068758     slnunico.obj
 0003:00001764       $pdata$0$unic_upper        0000000180068764     slnunico.obj
 0003:00001770       $pdata$1$unic_upper        0000000180068770     slnunico.obj
 0003:0000177c       $pdata$str_rep             000000018006877c     slnunico.obj
 0003:00001788       $pdata$unic_byte           0000000180068788     slnunico.obj
 0003:00001794       $pdata$unic_char           0000000180068794     slnunico.obj
 0003:000017a0       $pdata$0$unic_char         00000001800687a0     slnunico.obj
 0003:000017ac       $pdata$1$unic_char         00000001800687ac     slnunico.obj
 0003:00001980       $pdata$writer              0000000180068980     slnunico.obj
 0003:000017b8       $pdata$str_dump            00000001800687b8     slnunico.obj
 0003:00001848       $pdata$match_class         0000000180068848     slnunico.obj
 0003:000018e4       $pdata$singlematch         00000001800688e4     slnunico.obj
 0003:0000183c       $pdata$match               000000018006883c     slnunico.obj
 0003:00001854       $pdata$max_expand          0000000180068854     slnunico.obj
 0003:00001860       $pdata$0$max_expand        0000000180068860     slnunico.obj
 0003:0000186c       $pdata$1$max_expand        000000018006886c     slnunico.obj
 0003:00001878       $pdata$min_expand          0000000180068878     slnunico.obj
 0003:000018f0       $pdata$start_capture       00000001800688f0     slnunico.obj
 0003:000018a8       $pdata$push_onecapture     00000001800688a8     slnunico.obj
 0003:000018b4       $pdata$0$push_onecapture   00000001800688b4     slnunico.obj
 0003:000018c0       $pdata$1$push_onecapture   00000001800688c0     slnunico.obj
 0003:000018cc       $pdata$2$push_onecapture   00000001800688cc     slnunico.obj
 0003:000018d8       $pdata$4$push_onecapture   00000001800688d8     slnunico.obj
 0003:00001884       $pdata$push_captures       0000000180068884     slnunico.obj
 0003:00001890       $pdata$1$push_captures     0000000180068890     slnunico.obj
 0003:0000189c       $pdata$2$push_captures     000000018006889c     slnunico.obj
 0003:000018fc       $pdata$unic_find_aux       00000001800688fc     slnunico.obj
 0003:00001824       $pdata$gmatch_aux          0000000180068824     slnunico.obj
 0003:000017c4       $pdata$gmatch              00000001800687c4     slnunico.obj
 0003:00001800       $pdata$add_value           0000000180068800     slnunico.obj
 0003:0000180c       $pdata$0$add_value         000000018006880c     slnunico.obj
 0003:00001818       $pdata$1$add_value         0000000180068818     slnunico.obj
 0003:000017d0       $pdata$unic_gsub           00000001800687d0     slnunico.obj
 0003:000017dc       $pdata$str_format          00000001800687dc     slnunico.obj
 0003:000017e8       $pdata$utf8_valid          00000001800687e8     slnunico.obj
 0003:00001830       $pdata$luaopen_unicode     0000000180068830     slnunico.obj
 0003:00001a94       $pdata$fscanf              0000000180068a94     uliolib51.obj
 0003:00001b3c       $pdata$pushresult          0000000180068b3c     uliolib51.obj
 0003:00001a88       $pdata$fileerror           0000000180068a88     uliolib51.obj
 0003:0000198c       $pdata$io_type             000000018006898c     uliolib51.obj
 0003:00001b30       $pdata$newfile             0000000180068b30     uliolib51.obj
 0003:00001b00       $pdata$io_noclose          0000000180068b00     uliolib51.obj
 0003:00001b0c       $pdata$io_pclose           0000000180068b0c     uliolib51.obj
 0003:00001af4       $pdata$io_fclose           0000000180068af4     uliolib51.obj
 0003:00001a7c       $pdata$aux_close           0000000180068a7c     uliolib51.obj
 0003:00001998       $pdata$io_close            0000000180068998     uliolib51.obj
 0003:000019a4       $pdata$io_gc               00000001800689a4     uliolib51.obj
 0003:000019b0       $pdata$io_tostring         00000001800689b0     uliolib51.obj
 0003:000019bc       $pdata$io_open             00000001800689bc     uliolib51.obj
 0003:000019c8       $pdata$io_popen            00000001800689c8     uliolib51.obj
 0003:000019d4       $pdata$io_tmpfile          00000001800689d4     uliolib51.obj
 0003:00001aa0       $pdata$g_iofile            0000000180068aa0     uliolib51.obj
 0003:00001aac       $pdata$0$g_iofile          0000000180068aac     uliolib51.obj
 0003:00001ab8       $pdata$1$g_iofile          0000000180068ab8     uliolib51.obj
 0003:00001ac4       $pdata$2$g_iofile          0000000180068ac4     uliolib51.obj
 0003:00001ad0       $pdata$3$g_iofile          0000000180068ad0     uliolib51.obj
 0003:00001b18       $pdata$io_readline         0000000180068b18     uliolib51.obj
 0003:000019e0       $pdata$f_lines             00000001800689e0     uliolib51.obj
 0003:000019ec       $pdata$io_lines            00000001800689ec     uliolib51.obj
 0003:000019f8       $pdata$1$io_lines          00000001800689f8     uliolib51.obj
 0003:00001a04       $pdata$2$io_lines          0000000180068a04     uliolib51.obj
 0003:00001b54       $pdata$read_line           0000000180068b54     uliolib51.obj
 0003:00001b48       $pdata$read_chars          0000000180068b48     uliolib51.obj
 0003:00001adc       $pdata$g_read              0000000180068adc     uliolib51.obj
 0003:00001a10       $pdata$io_read             0000000180068a10     uliolib51.obj
 0003:00001a1c       $pdata$f_read              0000000180068a1c     uliolib51.obj
 0003:00001ae8       $pdata$g_write             0000000180068ae8     uliolib51.obj
 0003:00001a28       $pdata$io_write            0000000180068a28     uliolib51.obj
 0003:00001a34       $pdata$f_write             0000000180068a34     uliolib51.obj
 0003:00001a40       $pdata$f_seek              0000000180068a40     uliolib51.obj
 0003:00001a4c       $pdata$f_setvbuf           0000000180068a4c     uliolib51.obj
 0003:00001a58       $pdata$io_flush            0000000180068a58     uliolib51.obj
 0003:00001a64       $pdata$f_flush             0000000180068a64     uliolib51.obj
 0003:00001a70       $pdata$f_rawhandle         0000000180068a70     uliolib51.obj
 0003:00001b24       $pdata$luaopen_uio         0000000180068b24     uliolib51.obj
 0003:00001be4       $pdata$gctm                0000000180068be4     uloadlib51.obj
 0003:00001bf0       $pdata$ll_loadfunc         0000000180068bf0     uloadlib51.obj
 0003:00001b60       $pdata$ll_loadlib          0000000180068b60     uloadlib51.obj
 0003:00001bd8       $pdata$findfile            0000000180068bd8     uloadlib51.obj
 0003:00001bfc       $pdata$loaderror           0000000180068bfc     uloadlib51.obj
 0003:00001b6c       $pdata$loader_Lua          0000000180068b6c     uloadlib51.obj
 0003:00001c14       $pdata$mkfuncname          0000000180068c14     uloadlib51.obj
 0003:00001b78       $pdata$loader_C            0000000180068b78     uloadlib51.obj
 0003:00001b84       $pdata$loader_Croot        0000000180068b84     uloadlib51.obj
 0003:00001b90       $pdata$loader_preload      0000000180068b90     uloadlib51.obj
 0003:00001b9c       $pdata$ll_require          0000000180068b9c     uloadlib51.obj
 0003:00001ba8       $pdata$ll_module           0000000180068ba8     uloadlib51.obj
 0003:00001bb4       $pdata$0$ll_module         0000000180068bb4     uloadlib51.obj
 0003:00001bc0       $pdata$1$ll_module         0000000180068bc0     uloadlib51.obj
 0003:00001bcc       $pdata$ll_seeall           0000000180068bcc     uloadlib51.obj
 0003:00001c20       $pdata$setpath             0000000180068c20     uloadlib51.obj
 0003:00001c08       $pdata$luaopen_upackage    0000000180068c08     uloadlib51.obj
 0003:00001f98       $pdata$luaopen_ustring     0000000180068f98     ustring.obj
 0003:00001fec       $pdata$pusherrorcode       0000000180068fec     ustring.obj
 0003:00001fe0       $pdata$pusherror           0000000180068fe0     ustring.obj
 0003:00001f68       $pdata$SysErrorReturn      0000000180068f68     ustring.obj
 0003:00001ea8       $pdata$GetBoolFromTable    0000000180068ea8     ustring.obj
 0003:00001eb4       $pdata$GetOptBoolFromTable 0000000180068eb4     ustring.obj
 0003:00001ec0       $pdata$GetOptIntFromArray  0000000180068ec0     ustring.obj
 0003:00001ecc       $pdata$GetOptIntFromTable  0000000180068ecc     ustring.obj
 0003:00001ed8       $pdata$GetOptNumFromTable  0000000180068ed8     ustring.obj
 0003:00001efc       $pdata$PutBoolToTable      0000000180068efc     ustring.obj
 0003:00001f08       $pdata$PutIntToArray       0000000180068f08     ustring.obj
 0003:00001f14       $pdata$PutIntToTable       0000000180068f14     ustring.obj
 0003:00001f20       $pdata$PutLStrToTable      0000000180068f20     ustring.obj
 0003:00001f2c       $pdata$PutNumToTable       0000000180068f2c     ustring.obj
 0003:00001f38       $pdata$PutStrToArray       0000000180068f38     ustring.obj
 0003:00001f44       $pdata$PutStrToTable       0000000180068f44     ustring.obj
 0003:00001f50       $pdata$PutWStrToArray      0000000180068f50     ustring.obj
 0003:00001f5c       $pdata$PutWStrToTable      0000000180068f5c     ustring.obj
 0003:00001f80       $pdata$check_utf8_string   0000000180068f80     ustring.obj
 0003:00001ff8       $pdata$utf8_to_utf16       0000000180068ff8     ustring.obj
 0003:00001fa4       $pdata$opt_utf8_string     0000000180068fa4     ustring.obj
 0003:00001fd4       $pdata$push_utf8_string    0000000180068fd4     ustring.obj
 0003:00001f74       $pdata$check_utf16_string  0000000180068f74     ustring.obj
 0003:00001ee4       $pdata$PushAttrString      0000000180068ee4     ustring.obj
 0003:00001ef0       $pdata$PutAttrToTable      0000000180068ef0     ustring.obj
 0003:00001f8c       $pdata$convert_multibyte_string 0000000180068f8c     ustring.obj
 0003:00001fb0       $pdata$push_multibyte_string 0000000180068fb0     ustring.obj
 0003:00001fbc       $pdata$2$push_multibyte_string 0000000180068fbc     ustring.obj
 0003:00001fc8       $pdata$3$push_multibyte_string 0000000180068fc8     ustring.obj
 0003:00001c2c       $pdata$ustring_WideCharToMultiByte 0000000180068c2c     ustring.obj
 0003:00001c38       $pdata$1$ustring_WideCharToMultiByte 0000000180068c38     ustring.obj
 0003:00001c44       $pdata$2$ustring_WideCharToMultiByte 0000000180068c44     ustring.obj
 0003:00001c50       $pdata$ustring_MultiByteToWideChar 0000000180068c50     ustring.obj
 0003:00001c5c       $pdata$ustring_OemToUtf8   0000000180068c5c     ustring.obj
 0003:00001c68       $pdata$1$ustring_OemToUtf8 0000000180068c68     ustring.obj
 0003:00001c74       $pdata$2$ustring_OemToUtf8 0000000180068c74     ustring.obj
 0003:00001c80       $pdata$ustring_Utf8ToOem   0000000180068c80     ustring.obj
 0003:00001c8c       $pdata$ustring_Utf16ToUtf8 0000000180068c8c     ustring.obj
 0003:00001c98       $pdata$ustring_Utf8ToUtf16 0000000180068c98     ustring.obj
 0003:00001ca4       $pdata$0$ustring_Utf8ToUtf16 0000000180068ca4     ustring.obj
 0003:00001cb0       $pdata$1$ustring_Utf8ToUtf16 0000000180068cb0     ustring.obj
 0003:00001cbc       $pdata$ustring_GetACP      0000000180068cbc     ustring.obj
 0003:00001cc8       $pdata$ustring_GetOEMCP    0000000180068cc8     ustring.obj
 0003:00001e9c       $pdata$EnumCodePagesProc   0000000180068e9c     ustring.obj
 0003:00001cd4       $pdata$ustring_EnumSystemCodePages 0000000180068cd4     ustring.obj
 0003:00001ce0       $pdata$ustring_GetCPInfo   0000000180068ce0     ustring.obj
 0003:00001cec       $pdata$ustring_GetLogicalDriveStrings 0000000180068cec     ustring.obj
 0003:00001cf8       $pdata$0$ustring_GetLogicalDriveStrings 0000000180068cf8     ustring.obj
 0003:00001d04       $pdata$1$ustring_GetLogicalDriveStrings 0000000180068d04     ustring.obj
 0003:00001d10       $pdata$ustring_GetDriveType 0000000180068d10     ustring.obj
 0003:00001d1c       $pdata$ustring_Uuid        0000000180068d1c     ustring.obj
 0003:00001d28       $pdata$ustring_SearchPath  0000000180068d28     ustring.obj
 0003:00001d34       $pdata$ustring_GlobalMemoryStatus 0000000180068d34     ustring.obj
 0003:00001d40       $pdata$0$ustring_GlobalMemoryStatus 0000000180068d40     ustring.obj
 0003:00001d4c       $pdata$2$ustring_GlobalMemoryStatus 0000000180068d4c     ustring.obj
 0003:00001d58       $pdata$ustring_Sleep       0000000180068d58     ustring.obj
 0003:00001d64       $pdata$ustring_SetFileAttr 0000000180068d64     ustring.obj
 0003:00001d70       $pdata$2$ustring_SetFileAttr 0000000180068d70     ustring.obj
 0003:00001d7c       $pdata$3$ustring_SetFileAttr 0000000180068d7c     ustring.obj
 0003:00001d88       $pdata$4$ustring_SetFileAttr 0000000180068d88     ustring.obj
 0003:00001d94       $pdata$5$ustring_SetFileAttr 0000000180068d94     ustring.obj
 0003:00001da0       $pdata$ustring_GetFileAttr 0000000180068da0     ustring.obj
 0003:00001dac       $pdata$2$ustring_GetFileAttr 0000000180068dac     ustring.obj
 0003:00001db8       $pdata$3$ustring_GetFileAttr 0000000180068db8     ustring.obj
 0003:00001dc4       $pdata$ustring_SHGetFolderPath 0000000180068dc4     ustring.obj
 0003:00001dd0       $pdata$1$ustring_SHGetFolderPath 0000000180068dd0     ustring.obj
 0003:00001ddc       $pdata$2$ustring_SHGetFolderPath 0000000180068ddc     ustring.obj
 0003:00001de8       $pdata$ustring_sub         0000000180068de8     ustring.obj
 0003:00001df4       $pdata$ustring_len         0000000180068df4     ustring.obj
 0003:00001e00       $pdata$ustring_OutputDebugString 0000000180068e00     ustring.obj
 0003:00001e0c       $pdata$0$ustring_OutputDebugString 0000000180068e0c     ustring.obj
 0003:00001e18       $pdata$1$ustring_OutputDebugString 0000000180068e18     ustring.obj
 0003:00001e24       $pdata$ustring_system      0000000180068e24     ustring.obj
 0003:00001e30       $pdata$ustring_GetCurrentDir 0000000180068e30     ustring.obj
 0003:00001e3c       $pdata$0$ustring_GetCurrentDir 0000000180068e3c     ustring.obj
 0003:00001e48       $pdata$1$ustring_GetCurrentDir 0000000180068e48     ustring.obj
 0003:00001e54       $pdata$2$ustring_GetCurrentDir 0000000180068e54     ustring.obj
 0003:00001e60       $pdata$3$ustring_GetCurrentDir 0000000180068e60     ustring.obj
 0003:00001e6c       $pdata$ustring_SetCurrentDir 0000000180068e6c     ustring.obj
 0003:00001e78       $pdata$2$ustring_SetCurrentDir 0000000180068e78     ustring.obj
 0003:00001e84       $pdata$3$ustring_SetCurrentDir 0000000180068e84     ustring.obj
 0003:00001e90       $pdata$ustring_GetKeyState 0000000180068e90     ustring.obj
 0003:00002004       $pdata$GetAttrFromTable    0000000180069004     util.obj
 0003:00002028       $pdata$GetIntFromArray     0000000180069028     util.obj
 0003:00002034       $pdata$luaLF_FieldError    0000000180069034     util.obj
 0003:00002040       $pdata$luaLF_SlotError     0000000180069040     util.obj
 0003:00002010       $pdata$GetFileSizeFromTable 0000000180069010     util.obj
 0003:0000201c       $pdata$GetFileTimeFromTable 000000018006901c     util.obj
 0003:0000204c       $pdata$win_GetEnv          000000018006904c     win.obj
 0003:00002058       $pdata$0$win_GetEnv        0000000180069058     win.obj
 0003:00002064       $pdata$1$win_GetEnv        0000000180069064     win.obj
 0003:00002070       $pdata$win_SetEnv          0000000180069070     win.obj
 0003:0000219c       $pdata$CheckHKey           000000018006919c     win.obj
 0003:0000207c       $pdata$win_SetRegKey       000000018006907c     win.obj
 0003:00002088       $pdata$win_GetRegKey       0000000180069088     win.obj
 0003:00002094       $pdata$win_DeleteRegKey    0000000180069094     win.obj
 0003:000020a0       $pdata$win_DeleteRegValue  00000001800690a0     win.obj
 0003:000020ac       $pdata$win_EnumRegKey      00000001800690ac     win.obj
 0003:000020b8       $pdata$win_EnumRegValue    00000001800690b8     win.obj
 0003:000020c4       $pdata$win_ExtractKey      00000001800690c4     win.obj
 0003:000020d0       $pdata$win_ExtractKeyEx    00000001800690d0     win.obj
 0003:000020dc       $pdata$win_GetFileInfo     00000001800690dc     win.obj
 0003:000020e8       $pdata$win_GetSystemTimeAsFileTime 00000001800690e8     win.obj
 0003:000020f4       $pdata$win_FileTimeToSystemTime 00000001800690f4     win.obj
 0003:00002100       $pdata$win_SystemTimeToFileTime 0000000180069100     win.obj
 0003:0000210c       $pdata$win_FileTimeToLocalFileTime 000000018006910c     win.obj
 0003:00002118       $pdata$win_CompareString   0000000180069118     win.obj
 0003:00002124       $pdata$win_wcscmp          0000000180069124     win.obj
 0003:00002130       $pdata$win_GetVirtualKeys  0000000180069130     win.obj
 0003:0000213c       $pdata$win_GetConsoleScreenBufferInfo 000000018006913c     win.obj
 0003:00002148       $pdata$win_CopyFile        0000000180069148     win.obj
 0003:00002154       $pdata$win_MoveFile        0000000180069154     win.obj
 0003:00002160       $pdata$win_DeleteFile      0000000180069160     win.obj
 0003:000021b4       $pdata$mkdir               00000001800691b4     win.obj
 0003:000021c0       $pdata$0$mkdir             00000001800691c0     win.obj
 0003:0000216c       $pdata$win_CreateDir       000000018006916c     win.obj
 0003:00002178       $pdata$win_RemoveDir       0000000180069178     win.obj
 0003:00002184       $pdata$win_ShellExecute    0000000180069184     win.obj
 0003:00002190       $pdata$win_IsProcess64bit  0000000180069190     win.obj
 0003:000021a8       $pdata$luaopen_win         00000001800691a8     win.obj
 0003:000021d8       $pdata$?dllmain_crt_process_attach@@YAHQEAUHINSTANCE__@@QEAX@Z 00000001800691d8     LIBCMT:dll_dllmain.obj
 0003:0000393c       $pdata$?fin$0@?0??dllmain_crt_process_attach@@YAHQEAUHINSTANCE__@@QEAX@Z@4HA 000000018006a93c     LIBCMT:dll_dllmain.obj
 0003:000021e4       $pdata$?dllmain_crt_process_detach@@YAH_N@Z 00000001800691e4     LIBCMT:dll_dllmain.obj
 0003:00003948       $pdata$?fin$0@?0??dllmain_crt_process_detach@@YAH_N@Z@4HA 000000018006a948     LIBCMT:dll_dllmain.obj
 0003:000021cc       $pdata$?dllmain_crt_dispatch@@YAHQEAUHINSTANCE__@@KQEAX@Z 00000001800691cc     LIBCMT:dll_dllmain.obj
 0003:000021f0       $pdata$?dllmain_dispatch@@YAHQEAUHINSTANCE__@@KQEAX@Z 00000001800691f0     LIBCMT:dll_dllmain.obj
 0003:00003954       $pdata$?filt$0@?0??dllmain_dispatch@@YAHQEAUHINSTANCE__@@KQEAX@Z@4HA 000000018006a954     LIBCMT:dll_dllmain.obj
 0003:000021fc       $pdata$_DllMainCRTStartup  00000001800691fc     LIBCMT:dll_dllmain.obj
 0003:00002208       $pdata$__security_init_cookie 0000000180069208     LIBCMT:gs_support.obj
 0003:00002214       $pdata$__scrt_initialize_default_local_stdio_options 0000000180069214     LIBCMT:default_local_stdio_options.obj
 0003:00002298       $pdata$__scrt_is_nonwritable_in_current_image 0000000180069298     LIBCMT:utility.obj
 0003:00003960       $pdata$__scrt_is_nonwritable_in_current_image$filt$0 000000018006a960     LIBCMT:utility.obj
 0003:00002220       $pdata$__scrt_acquire_startup_lock 0000000180069220     LIBCMT:utility.obj
 0003:000022a4       $pdata$__scrt_release_startup_lock 00000001800692a4     LIBCMT:utility.obj
 0003:00002280       $pdata$__scrt_initialize_crt 0000000180069280     LIBCMT:utility.obj
 0003:000022b0       $pdata$__scrt_uninitialize_crt 00000001800692b0     LIBCMT:utility.obj
 0003:0000228c       $pdata$__scrt_initialize_onexit_tables 000000018006928c     LIBCMT:utility.obj
 0003:0000225c       $pdata$__scrt_dllmain_exception_filter 000000018006925c     LIBCMT:utility.obj
 0003:00002238       $pdata$__scrt_dllmain_before_initialize_c 0000000180069238     LIBCMT:utility.obj
 0003:0000222c       $pdata$__scrt_dllmain_after_initialize_c 000000018006922c     LIBCMT:utility.obj
 0003:00002268       $pdata$__scrt_dllmain_uninitialize_c 0000000180069268     LIBCMT:utility.obj
 0003:00002274       $pdata$__scrt_dllmain_uninitialize_critical 0000000180069274     LIBCMT:utility.obj
 0003:00002244       $pdata$__scrt_dllmain_crt_thread_attach 0000000180069244     LIBCMT:utility.obj
 0003:00002250       $pdata$__scrt_dllmain_crt_thread_detach 0000000180069250     LIBCMT:utility.obj
 0003:000022bc       $pdata$__scrt_fastfail     00000001800692bc     LIBCMT:utility_desktop.obj
 0003:000022c8       $pdata$_RTC_Initialize     00000001800692c8     LIBCMT:_initsect_.obj
 0003:000022d4       $pdata$_RTC_Terminate      00000001800692d4     LIBCMT:_initsect_.obj
 0003:000022e0       $pdata$__isa_available_init 00000001800692e0     LIBCMT:_cpu_disp_.obj
 0003:00002304       $pdata$wcsstr              0000000180069304     libvcruntime:wcsstr.obj
 0003:00002310       $pdata$strchr              0000000180069310     libvcruntime:strchr.obj
 0003:0000231c       $pdata$wcschr              000000018006931c     libvcruntime:wcschr.obj
 0003:00002340       $pdata$strrchr             0000000180069340     libvcruntime:strrchr.obj
 0003:0000234c       $pdata$__C_specific_handler 000000018006934c     libvcruntime:_riscchandler_.obj
 0003:00002358       $pdata$__std_type_info_destroy_list 0000000180069358     libvcruntime:std_type_info.obj
 0003:00002364       $pdata$__vcrt_initialize   0000000180069364     libvcruntime:initialization.obj
 0003:00002388       $pdata$__vcrt_uninitialize 0000000180069388     libvcruntime:initialization.obj
 0003:00002394       $pdata$__vcrt_uninitialize_critical 0000000180069394     libvcruntime:initialization.obj
 0003:00002370       $pdata$__vcrt_thread_attach 0000000180069370     libvcruntime:initialization.obj
 0003:0000237c       $pdata$__vcrt_thread_detach 000000018006937c     libvcruntime:initialization.obj
 0003:000023f4       $pdata$__vcrt_initialize_ptd 00000001800693f4     libvcruntime:per_thread_data.obj
 0003:00002400       $pdata$__vcrt_uninitialize_ptd 0000000180069400     libvcruntime:per_thread_data.obj
 0003:000023e8       $pdata$__vcrt_getptd_noexit 00000001800693e8     libvcruntime:per_thread_data.obj
 0003:000023dc       $pdata$__vcrt_freeptd      00000001800693dc     libvcruntime:per_thread_data.obj
 0003:000023d0       $pdata$__vcrt_freefls      00000001800693d0     libvcruntime:per_thread_data.obj
 0003:0000240c       $pdata$__vcrt_initialize_locks 000000018006940c     libvcruntime:locks.obj
 0003:00002418       $pdata$__vcrt_uninitialize_locks 0000000180069418     libvcruntime:locks.obj
 0003:00002430       $pdata$__vcrt_FlsAlloc     0000000180069430     libvcruntime:winapi_downlevel.obj
 0003:0000243c       $pdata$__vcrt_FlsFree      000000018006943c     libvcruntime:winapi_downlevel.obj
 0003:00002448       $pdata$__vcrt_FlsGetValue  0000000180069448     libvcruntime:winapi_downlevel.obj
 0003:00002454       $pdata$__vcrt_FlsSetValue  0000000180069454     libvcruntime:winapi_downlevel.obj
 0003:00002460       $pdata$__vcrt_InitializeCriticalSectionEx 0000000180069460     libvcruntime:winapi_downlevel.obj
 0003:0000246c       $pdata$__vcrt_initialize_winapi_thunks 000000018006946c     libvcruntime:winapi_downlevel.obj
 0003:00002478       $pdata$__vcrt_uninitialize_winapi_thunks 0000000180069478     libvcruntime:winapi_downlevel.obj
 0003:00002424       $pdata$?try_get_function@@YAPEAXW4function_id@?A0x89697e75@@QEBDQEBW4module_id@2@2@Z 0000000180069424     libvcruntime:winapi_downlevel.obj
 0003:00002490       $pdata$__DestructExceptionObject 0000000180069490     libvcruntime:ehhelpers.obj
 0003:0000396c       $pdata$__DestructExceptionObject$filt$0 000000018006a96c     libvcruntime:ehhelpers.obj
 0003:0000252c       $pdata$??0_LocaleUpdate@@QEAA@QEAU__crt_locale_pointers@@@Z 000000018006952c     libucrt:output.obj
 0003:000026d0       $pdata$__stdio_common_vfprintf 00000001800696d0     libucrt:output.obj
 0003:0000267c       $pdata$?validate_stream_is_ansi_if_required@?$__acrt_stdio_char_traits@D@@SA_NQEAU_iobuf@@@Z 000000018006967c     libucrt:output.obj
 0003:00002544       $pdata$?force_decimal_point@__crt_stdio_output@@YAXPEADQEAU__crt_locale_pointers@@@Z 0000000180069544     libucrt:output.obj
 0003:000024a8       $pdata$??$common_vsprintf@Vstandard_base@__crt_stdio_output@@D@@YAH_KQEAD0QEBDQEAU__crt_locale_pointers@@1@Z 00000001800694a8     libucrt:output.obj
 0003:000024b4       $pdata$??$common_vsprintf@Vstandard_base@__crt_stdio_output@@_W@@YAH_KQEA_W0QEB_WQEAU__crt_locale_pointers@@QEAD@Z 00000001800694b4     libucrt:output.obj
 0003:000026c4       $pdata$?write_string_impl@?$output_adapter_common@DV?$stream_output_adapter@D@__crt_stdio_output@@@__crt_stdio_output@@IEBAXQEBDHQEAHAEAV__crt_deferred_errno_cache@@@Z 00000001800696c4     libucrt:output.obj
 0003:00002568       $pdata$?process@?$output_processor@DV?$stream_output_adapter@D@__crt_stdio_output@@V?$standard_base@DV?$stream_output_adapter@D@__crt_stdio_output@@@2@@__crt_stdio_output@@QEAAHXZ 0000000180069568     libucrt:output.obj
 0003:0000258c       $pdata$?state_case_normal@?$output_processor@DV?$stream_output_adapter@D@__crt_stdio_output@@V?$standard_base@DV?$stream_output_adapter@D@__crt_stdio_output@@@2@@__crt_stdio_output@@AEAA_NXZ 000000018006958c     libucrt:output.obj
 0003:000025a4       $pdata$?state_case_normal_tchar@?$output_processor@DV?$stream_output_adapter@D@__crt_stdio_output@@V?$standard_base@DV?$stream_output_adapter@D@__crt_stdio_output@@@2@@__crt_stdio_output@@AEAA_ND@Z 00000001800695a4     libucrt:output.obj
 0003:00002550       $pdata$?parse_int_from_format_string@?$output_processor@DV?$stream_output_adapter@D@__crt_stdio_output@@V?$standard_base@DV?$stream_output_adapter@D@__crt_stdio_output@@@2@@__crt_stdio_output@@AEAA_NQEAH@Z 0000000180069550     libucrt:output.obj
 0003:00002550       $pdata$?parse_int_from_format_string@?$output_processor@DV?$string_output_adapter@D@__crt_stdio_output@@V?$standard_base@DV?$string_output_adapter@D@__crt_stdio_output@@@2@@__crt_stdio_output@@AEAA_NQEAH@Z 0000000180069550     libucrt:output.obj
 0003:000025bc       $pdata$?state_case_size@?$output_processor@DV?$stream_output_adapter@D@__crt_stdio_output@@V?$standard_base@DV?$stream_output_adapter@D@__crt_stdio_output@@@2@@__crt_stdio_output@@AEAA_NXZ 00000001800695bc     libucrt:output.obj
 0003:000025e0       $pdata$?state_case_type@?$output_processor@DV?$stream_output_adapter@D@__crt_stdio_output@@V?$standard_base@DV?$stream_output_adapter@D@__crt_stdio_output@@@2@@__crt_stdio_output@@AEAA_NXZ 00000001800695e0     libucrt:output.obj
 0003:00002628       $pdata$?type_case_c_tchar@?$output_processor@DV?$string_output_adapter@D@__crt_stdio_output@@V?$standard_base@DV?$string_output_adapter@D@__crt_stdio_output@@@2@@__crt_stdio_output@@AEAA_ND@Z 0000000180069628     libucrt:output.obj
 0003:00002628       $pdata$?type_case_c_tchar@?$output_processor@DV?$stream_output_adapter@D@__crt_stdio_output@@V?$standard_base@DV?$stream_output_adapter@D@__crt_stdio_output@@@2@@__crt_stdio_output@@AEAA_ND@Z 0000000180069628     libucrt:output.obj
 0003:00002664       $pdata$?type_case_s@?$output_processor@DV?$string_output_adapter@D@__crt_stdio_output@@V?$standard_base@DV?$string_output_adapter@D@__crt_stdio_output@@@2@@__crt_stdio_output@@AEAA_NXZ 0000000180069664     libucrt:output.obj
 0003:00002664       $pdata$?type_case_s@?$output_processor@DV?$stream_output_adapter@D@__crt_stdio_output@@V?$standard_base@DV?$stream_output_adapter@D@__crt_stdio_output@@@2@@__crt_stdio_output@@AEAA_NXZ 0000000180069664     libucrt:output.obj
 0003:00002610       $pdata$?type_case_a@?$output_processor@DV?$string_output_adapter@D@__crt_stdio_output@@V?$standard_base@DV?$string_output_adapter@D@__crt_stdio_output@@@2@@__crt_stdio_output@@AEAA_NXZ 0000000180069610     libucrt:output.obj
 0003:00002610       $pdata$?type_case_a@?$output_processor@DV?$stream_output_adapter@D@__crt_stdio_output@@V?$standard_base@DV?$stream_output_adapter@D@__crt_stdio_output@@@2@@__crt_stdio_output@@AEAA_NXZ 0000000180069610     libucrt:output.obj
 0003:00002640       $pdata$?type_case_integer@?$output_processor@DV?$stream_output_adapter@D@__crt_stdio_output@@V?$standard_base@DV?$stream_output_adapter@D@__crt_stdio_output@@@2@@__crt_stdio_output@@AEAA_NI_N@Z 0000000180069640     libucrt:output.obj
 0003:00002640       $pdata$?type_case_integer@?$output_processor@DV?$string_output_adapter@D@__crt_stdio_output@@V?$standard_base@DV?$string_output_adapter@D@__crt_stdio_output@@@2@@__crt_stdio_output@@AEAA_NI_N@Z 0000000180069640     libucrt:output.obj
 0003:00002658       $pdata$?type_case_n@?$output_processor@_WV?$string_output_adapter@_W@__crt_stdio_output@@V?$standard_base@_WV?$string_output_adapter@_W@__crt_stdio_output@@@2@@__crt_stdio_output@@AEAA_NXZ 0000000180069658     libucrt:output.obj
 0003:00002658       $pdata$?type_case_n@?$output_processor@DV?$string_output_adapter@D@__crt_stdio_output@@V?$standard_base@DV?$string_output_adapter@D@__crt_stdio_output@@@2@@__crt_stdio_output@@AEAA_NXZ 0000000180069658     libucrt:output.obj
 0003:00002658       $pdata$?type_case_n@?$output_processor@DV?$stream_output_adapter@D@__crt_stdio_output@@V?$standard_base@DV?$stream_output_adapter@D@__crt_stdio_output@@@2@@__crt_stdio_output@@AEAA_NXZ 0000000180069658     libucrt:output.obj
 0003:00002688       $pdata$?write_stored_string_tchar@?$output_processor@DV?$stream_output_adapter@D@__crt_stdio_output@@V?$standard_base@DV?$stream_output_adapter@D@__crt_stdio_output@@@2@@__crt_stdio_output@@AEAA_ND@Z 0000000180069688     libucrt:output.obj
 0003:00002538       $pdata$??R<lambda_a31071773b9a94e445cbd5d04ef99106>@@QEBAHXZ 0000000180069538     libucrt:output.obj
 0003:000026ac       $pdata$?write_string@?$string_output_adapter@D@__crt_stdio_output@@QEBAXQEBDHQEAHAEAV__crt_deferred_errno_cache@@@Z 00000001800696ac     libucrt:output.obj
 0003:00002574       $pdata$?process@?$output_processor@DV?$string_output_adapter@D@__crt_stdio_output@@V?$standard_base@DV?$string_output_adapter@D@__crt_stdio_output@@@2@@__crt_stdio_output@@QEAAHXZ 0000000180069574     libucrt:output.obj
 0003:00002598       $pdata$?state_case_normal@?$output_processor@DV?$string_output_adapter@D@__crt_stdio_output@@V?$standard_base@DV?$string_output_adapter@D@__crt_stdio_output@@@2@@__crt_stdio_output@@AEAA_NXZ 0000000180069598     libucrt:output.obj
 0003:000025b0       $pdata$?state_case_normal_tchar@?$output_processor@DV?$string_output_adapter@D@__crt_stdio_output@@V?$standard_base@DV?$string_output_adapter@D@__crt_stdio_output@@@2@@__crt_stdio_output@@AEAA_ND@Z 00000001800695b0     libucrt:output.obj
 0003:000025c8       $pdata$?state_case_size@?$output_processor@DV?$string_output_adapter@D@__crt_stdio_output@@V?$standard_base@DV?$string_output_adapter@D@__crt_stdio_output@@@2@@__crt_stdio_output@@AEAA_NXZ 00000001800695c8     libucrt:output.obj
 0003:000025ec       $pdata$?state_case_type@?$output_processor@DV?$string_output_adapter@D@__crt_stdio_output@@V?$standard_base@DV?$string_output_adapter@D@__crt_stdio_output@@@2@@__crt_stdio_output@@AEAA_NXZ 00000001800695ec     libucrt:output.obj
 0003:00002694       $pdata$?write_stored_string_tchar@?$output_processor@DV?$string_output_adapter@D@__crt_stdio_output@@V?$standard_base@DV?$string_output_adapter@D@__crt_stdio_output@@@2@@__crt_stdio_output@@AEAA_ND@Z 0000000180069694     libucrt:output.obj
 0003:000026b8       $pdata$?write_string@?$string_output_adapter@_W@__crt_stdio_output@@QEBAXQEB_WHQEAHAEAV__crt_deferred_errno_cache@@@Z 00000001800696b8     libucrt:output.obj
 0003:00002580       $pdata$?process@?$output_processor@_WV?$string_output_adapter@_W@__crt_stdio_output@@V?$standard_base@_WV?$string_output_adapter@_W@__crt_stdio_output@@@2@@__crt_stdio_output@@QEAAHXZ 0000000180069580     libucrt:output.obj
 0003:0000255c       $pdata$?parse_int_from_format_string@?$output_processor@_WV?$string_output_adapter@_W@__crt_stdio_output@@V?$standard_base@_WV?$string_output_adapter@_W@__crt_stdio_output@@@2@@__crt_stdio_output@@AEAA_NQEAH@Z 000000018006955c     libucrt:output.obj
 0003:000025d4       $pdata$?state_case_size@?$output_processor@_WV?$string_output_adapter@_W@__crt_stdio_output@@V?$standard_base@_WV?$string_output_adapter@_W@__crt_stdio_output@@@2@@__crt_stdio_output@@AEAA_NXZ 00000001800695d4     libucrt:output.obj
 0003:000025f8       $pdata$?state_case_type@?$output_processor@_WV?$string_output_adapter@_W@__crt_stdio_output@@V?$standard_base@_WV?$string_output_adapter@_W@__crt_stdio_output@@@2@@__crt_stdio_output@@AEAA_NXZ 00000001800695f8     libucrt:output.obj
 0003:00002634       $pdata$?type_case_c_tchar@?$output_processor@_WV?$string_output_adapter@_W@__crt_stdio_output@@V?$standard_base@_WV?$string_output_adapter@_W@__crt_stdio_output@@@2@@__crt_stdio_output@@AEAA_N_W@Z 0000000180069634     libucrt:output.obj
 0003:00002604       $pdata$?type_case_Z@?$output_processor@_WV?$string_output_adapter@_W@__crt_stdio_output@@V?$standard_base@_WV?$string_output_adapter@_W@__crt_stdio_output@@@2@@__crt_stdio_output@@AEAA_NXZ 0000000180069604     libucrt:output.obj
 0003:00002670       $pdata$?type_case_s@?$output_processor@_WV?$string_output_adapter@_W@__crt_stdio_output@@V?$standard_base@_WV?$string_output_adapter@_W@__crt_stdio_output@@@2@@__crt_stdio_output@@AEAA_NXZ 0000000180069670     libucrt:output.obj
 0003:0000261c       $pdata$?type_case_a@?$output_processor@_WV?$string_output_adapter@_W@__crt_stdio_output@@V?$standard_base@_WV?$string_output_adapter@_W@__crt_stdio_output@@@2@@__crt_stdio_output@@AEAA_NXZ 000000018006961c     libucrt:output.obj
 0003:0000264c       $pdata$?type_case_integer@?$output_processor@_WV?$string_output_adapter@_W@__crt_stdio_output@@V?$standard_base@_WV?$string_output_adapter@_W@__crt_stdio_output@@@2@@__crt_stdio_output@@AEAA_NI_N@Z 000000018006964c     libucrt:output.obj
 0003:000026a0       $pdata$?write_stored_string_tchar@?$output_processor@_WV?$string_output_adapter@_W@__crt_stdio_output@@V?$standard_base@_WV?$string_output_adapter@_W@__crt_stdio_output@@@2@@__crt_stdio_output@@AEAA_N_W@Z 00000001800696a0     libucrt:output.obj
 0003:00002520       $pdata$??$write_multiple_characters@V?$string_output_adapter@_W@__crt_stdio_output@@D@__crt_stdio_output@@YAXAEBV?$string_output_adapter@_W@0@DHQEAH@Z 0000000180069520     libucrt:output.obj
 0003:00002514       $pdata$??$write_multiple_characters@V?$string_output_adapter@D@__crt_stdio_output@@D@__crt_stdio_output@@YAXAEBV?$string_output_adapter@D@0@DHQEAH@Z 0000000180069514     libucrt:output.obj
 0003:00002508       $pdata$??$write_multiple_characters@V?$stream_output_adapter@D@__crt_stdio_output@@D@__crt_stdio_output@@YAXAEBV?$stream_output_adapter@D@0@DHQEAH@Z 0000000180069508     libucrt:output.obj
 0003:000024c0       $pdata$??$ensure_buffer_is_big_enough@D@formatting_buffer@__crt_stdio_output@@QEAA_N_K@Z 00000001800694c0     libucrt:output.obj
 0003:000024cc       $pdata$??$ensure_buffer_is_big_enough@_W@formatting_buffer@__crt_stdio_output@@QEAA_N_K@Z 00000001800694cc     libucrt:output.obj
 0003:000024fc       $pdata$??$type_case_integer_parse_into_buffer@_K@?$output_processor@_WV?$string_output_adapter@_W@__crt_stdio_output@@V?$standard_base@_WV?$string_output_adapter@_W@__crt_stdio_output@@@2@@__crt_stdio_output@@AEAAX_KI_N@Z 00000001800694fc     libucrt:output.obj
 0003:000024e4       $pdata$??$type_case_integer_parse_into_buffer@I@?$output_processor@_WV?$string_output_adapter@_W@__crt_stdio_output@@V?$standard_base@_WV?$string_output_adapter@_W@__crt_stdio_output@@@2@@__crt_stdio_output@@AEAAXII_N@Z 00000001800694e4     libucrt:output.obj
 0003:000024f0       $pdata$??$type_case_integer_parse_into_buffer@_K@?$output_processor@DV?$string_output_adapter@D@__crt_stdio_output@@V?$standard_base@DV?$string_output_adapter@D@__crt_stdio_output@@@2@@__crt_stdio_output@@AEAAX_KI_N@Z 00000001800694f0     libucrt:output.obj
 0003:000024f0       $pdata$??$type_case_integer_parse_into_buffer@_K@?$output_processor@DV?$stream_output_adapter@D@__crt_stdio_output@@V?$standard_base@DV?$stream_output_adapter@D@__crt_stdio_output@@@2@@__crt_stdio_output@@AEAAX_KI_N@Z 00000001800694f0     libucrt:output.obj
 0003:000024d8       $pdata$??$type_case_integer_parse_into_buffer@I@?$output_processor@DV?$stream_output_adapter@D@__crt_stdio_output@@V?$standard_base@DV?$stream_output_adapter@D@__crt_stdio_output@@@2@@__crt_stdio_output@@AEAAXII_N@Z 00000001800694d8     libucrt:output.obj
 0003:000024d8       $pdata$??$type_case_integer_parse_into_buffer@I@?$output_processor@DV?$string_output_adapter@D@__crt_stdio_output@@V?$standard_base@DV?$string_output_adapter@D@__crt_stdio_output@@@2@@__crt_stdio_output@@AEAAXII_N@Z 00000001800694d8     libucrt:output.obj
 0003:0000249c       $pdata$??$?RV<lambda_a62c933ada0517137acf5807a1eeac1f>@@AEAV<lambda_a31071773b9a94e445cbd5d04ef99106>@@V<lambda_56065050dbf3ada7e59a83db45153de3>@@@?$__crt_seh_guarded_call@H@@QEAAH$$QEAV<lambda_a62c933ada0517137acf5807a1eeac1f>@@AEAV<lambda_a31071773b9a94e445cbd5d04ef99106>@@$$QEAV<lambda_56065050dbf3ada7e59a83db45153de3>@@@Z 000000018006949c     libucrt:output.obj
 0003:00003978       $pdata$?fin$0@?0???$?RV<lambda_842d9ff0dc9ef11c61343bbaebe7f885>@@AEAV<lambda_c5860995281e5c4ce005b3de8f5874ee>@@V<lambda_d90129c13df834fdcbf8d2b88dafcf2d>@@@?$__crt_seh_guarded_call@X@@QEAAX$$QEAV<lambda_842d9ff0dc9ef11c61343bbaebe7f885>@@AEAV<lambda_c5860995281e5c4ce005b3de8f5874ee>@@$$QEAV<lambda_d90129c13df834fdcbf8d2b88dafcf2d>@@@Z@4HA 000000018006a978     libucrt:fflush.obj
 0003:00003978       $pdata$?fin$0@?0???$?RV<lambda_c376a267cfb53b6959b3b692ec76b120>@@AEAV<lambda_9a32fed5bf61b6b509b2d3f6003082a1>@@V<lambda_572fbb9fa0ab338edf41edfd4b5fcc8d>@@@?$__crt_seh_guarded_call@H@@QEAAH$$QEAV<lambda_c376a267cfb53b6959b3b692ec76b120>@@AEAV<lambda_9a32fed5bf61b6b509b2d3f6003082a1>@@$$QEAV<lambda_572fbb9fa0ab338edf41edfd4b5fcc8d>@@@Z@4HA 000000018006a978     libucrt:fflush.obj
 0003:00003978       $pdata$?fin$0@?0???$?RV<lambda_a62c933ada0517137acf5807a1eeac1f>@@AEAV<lambda_a31071773b9a94e445cbd5d04ef99106>@@V<lambda_56065050dbf3ada7e59a83db45153de3>@@@?$__crt_seh_guarded_call@H@@QEAAH$$QEAV<lambda_a62c933ada0517137acf5807a1eeac1f>@@AEAV<lambda_a31071773b9a94e445cbd5d04ef99106>@@$$QEAV<lambda_56065050dbf3ada7e59a83db45153de3>@@@Z@4HA 000000018006a978     libucrt:output.obj
 0003:00003978       $pdata$?fin$0@?0???$?RV<lambda_bdbcead8b570fa3d5ec6d9679862a6e5>@@AEAV<lambda_96f4279ff90247a4c5c5d9824f56f8c1>@@V<lambda_4606be27f17b5e5579e09050fab91818>@@@?$__crt_seh_guarded_call@_K@@QEAA_K$$QEAV<lambda_bdbcead8b570fa3d5ec6d9679862a6e5>@@AEAV<lambda_96f4279ff90247a4c5c5d9824f56f8c1>@@$$QEAV<lambda_4606be27f17b5e5579e09050fab91818>@@@Z@4HA 000000018006a978     libucrt:fwrite.obj
 0003:00003978       $pdata$?fin$0@?0???$?RV<lambda_84ec643ea9557e2f7dc01bb0e9624395>@@AEAV<lambda_ca71763b3c0644891230e4f79ea54fa6>@@V<lambda_439a761618c59b0600e24586724d733b>@@@?$__crt_seh_guarded_call@H@@QEAAH$$QEAV<lambda_84ec643ea9557e2f7dc01bb0e9624395>@@AEAV<lambda_ca71763b3c0644891230e4f79ea54fa6>@@$$QEAV<lambda_439a761618c59b0600e24586724d733b>@@@Z@4HA 000000018006a978     libucrt:setvbuf.obj
 0003:00003978       $pdata$?fin$0@?0???$?RV<lambda_082dd7c0feb7dbdaf245f261e54a6583>@@AEAV<lambda_f3caf1ecae5fe01a9a1a6239afa44510>@@V<lambda_c640b76c0755ae85b317b35c67c61e6b>@@@?$__crt_seh_guarded_call@H@@QEAAH$$QEAV<lambda_082dd7c0feb7dbdaf245f261e54a6583>@@AEAV<lambda_f3caf1ecae5fe01a9a1a6239afa44510>@@$$QEAV<lambda_c640b76c0755ae85b317b35c67c61e6b>@@@Z@4HA 000000018006a978     libucrt:input.obj
 0003:000026dc       $pdata$_wcsdup             00000001800696dc     libucrt:wcsdup.obj
 0003:000026e8       $pdata$??$common_fsopen@_W@@YAPEAU_iobuf@@QEB_W0H@Z 00000001800696e8     libucrt:fopen.obj
 0003:00003984       $pdata$?fin$0@?0???$common_fsopen@_W@@YAPEAU_iobuf@@QEB_W0H@Z@4HA 000000018006a984     libucrt:fopen.obj
 0003:00002700       $pdata$fclose              0000000180069700     libucrt:fclose.obj
 0003:00003990       $pdata$rewind$fin$0        000000018006a990     libucrt:rewind.obj
 0003:00003990       $pdata$fclose$fin$0        000000018006a990     libucrt:fclose.obj
 0003:00003990       $pdata$?fin$0@?0???$common_ftell@J@@YAJV__crt_stdio_stream@@@Z@4HA 000000018006a990     libucrt:ftell.obj
 0003:00003990       $pdata$?fin$0@?0??common_fseek@@YAHV__crt_stdio_stream@@_JH@Z@4HA 000000018006a990     libucrt:fseek.obj
 0003:00003990       $pdata$clearerr_s$fin$0    000000018006a990     libucrt:clearerr.obj
 0003:000026f4       $pdata$_fclose_nolock      00000001800696f4     libucrt:fclose.obj
 0003:0000270c       $pdata$_clearfp            000000018006970c     libucrt:ieee.obj
 0003:00002718       $pdata$common_control87    0000000180069718     libucrt:ieee.obj
 0003:0000399c       $pdata$common_control87$filt$0 000000018006a99c     libucrt:ieee.obj
 0003:0000399c       $pdata$_ctrlfp$filt$0      000000018006a99c     libucrt:fpctrl.obj
 0003:0000273c       $pdata$_errno              000000018006973c     libucrt:errno.obj
 0003:00002730       $pdata$__doserrno          0000000180069730     libucrt:errno.obj
 0003:00002724       $pdata$__acrt_errno_map_os_error 0000000180069724     libucrt:errno.obj
 0003:00002748       $pdata$strerror            0000000180069748     libucrt:strerror.obj
 0003:00002754       $pdata$__acrt_initialize_stdio 0000000180069754     libucrt:_file.obj
 0003:00002760       $pdata$__acrt_uninitialize_stdio 0000000180069760     libucrt:_file.obj
 0003:00002778       $pdata$_wfreopen           0000000180069778     libucrt:freopen.obj
 0003:0000276c       $pdata$??$common_freopen@_W@@YAHQEAPEAU_iobuf@@QEB_W1V__crt_stdio_stream@@H@Z 000000018006976c     libucrt:freopen.obj
 0003:000039a8       $pdata$?fin$0@?0???$common_freopen@_W@@YAHQEAPEAU_iobuf@@QEB_W1V__crt_stdio_stream@@H@Z@4HA 000000018006a9a8     libucrt:freopen.obj
 0003:00002784       $pdata$feof                0000000180069784     libucrt:feoferr.obj
 0003:00002790       $pdata$ferror              0000000180069790     libucrt:feoferr.obj
 0003:000027b4       $pdata$fread_s             00000001800697b4     libucrt:fread.obj
 0003:000039b4       $pdata$fread_s$fin$0       000000018006a9b4     libucrt:fread.obj
 0003:000027a8       $pdata$fread               00000001800697a8     libucrt:fread.obj
 0003:0000279c       $pdata$_fread_nolock_s     000000018006979c     libucrt:fread.obj
 0003:000027cc       $pdata$fgetc               00000001800697cc     libucrt:fgetc.obj
 0003:000039c0       $pdata$fgetc$fin$0         000000018006a9c0     libucrt:fgetc.obj
 0003:000027c0       $pdata$_fgetc_nolock       00000001800697c0     libucrt:fgetc.obj
 0003:000027d8       $pdata$rewind              00000001800697d8     libucrt:rewind.obj
 0003:000027f0       $pdata$ungetc              00000001800697f0     libucrt:ungetc.obj
 0003:000039cc       $pdata$ungetc$fin$0        000000018006a9cc     libucrt:ungetc.obj
 0003:000027e4       $pdata$_ungetc_nolock      00000001800697e4     libucrt:ungetc.obj
 0003:00002808       $pdata$iswctype            0000000180069808     libucrt:iswctype.obj
 0003:00002814       $pdata$isdigit             0000000180069814     libucrt:_ctype.obj
 0003:00002820       $pdata$isspace             0000000180069820     libucrt:_ctype.obj
 0003:0000282c       $pdata$wcsncpy             000000018006982c     libucrt:wcsncpy.obj
 0003:00002838       $pdata$_wcsicmp            0000000180069838     libucrt:wcsicmp.obj
 0003:00002844       $pdata$_wcsicmp_l          0000000180069844     libucrt:wcsicmp.obj
 0003:00002874       $pdata$strpbrk             0000000180069874     libucrt:strpbrk.obj
 0003:00002868       $pdata$fallbackMethod      0000000180069868     libucrt:strpbrk.obj
 0003:000028b0       $pdata$_pclose             00000001800698b0     libucrt:popen.obj
 0003:000039e4       $pdata$_pclose$fin$0       000000018006a9e4     libucrt:popen.obj
 0003:000028a4       $pdata$?idtab@@YAPEAUprocess_handle_pair@?A0xe43b7539@@QEAU_iobuf@@@Z 00000001800698a4     libucrt:popen.obj
 0003:00002880       $pdata$??$common_popen@_W@@YAPEAU_iobuf@@QEB_W0@Z 0000000180069880     libucrt:popen.obj
 0003:000039d8       $pdata$?fin$0@?0???$common_popen@_W@@YAPEAU_iobuf@@QEB_W0@Z@4HA 000000018006a9d8     libucrt:popen.obj
 0003:0000288c       $pdata$??$common_popen_nolock@_W@@YAPEAU_iobuf@@QEB_W0HAEAY01H@Z 000000018006988c     libucrt:popen.obj
 0003:00002898       $pdata$??$get_executable_path@_W@@YAPEB_WQEB_W@Z 0000000180069898     libucrt:popen.obj
 0003:000028bc       $pdata$clearerr_s          00000001800698bc     libucrt:clearerr.obj
 0003:00002910       $pdata$fflush              0000000180069910     libucrt:fflush.obj
 0003:00002904       $pdata$_fflush_nolock      0000000180069904     libucrt:fflush.obj
 0003:000028f8       $pdata$__acrt_stdio_flush_nolock 00000001800698f8     libucrt:fflush.obj
 0003:000028ec       $pdata$?common_flush_all@@YAH_N@Z 00000001800698ec     libucrt:fflush.obj
 0003:000028c8       $pdata$??$?RV<lambda_842d9ff0dc9ef11c61343bbaebe7f885>@@AEAV<lambda_c5860995281e5c4ce005b3de8f5874ee>@@V<lambda_d90129c13df834fdcbf8d2b88dafcf2d>@@@?$__crt_seh_guarded_call@X@@QEAAX$$QEAV<lambda_842d9ff0dc9ef11c61343bbaebe7f885>@@AEAV<lambda_c5860995281e5c4ce005b3de8f5874ee>@@$$QEAV<lambda_d90129c13df834fdcbf8d2b88dafcf2d>@@@Z 00000001800698c8     libucrt:fflush.obj
 0003:000028d4       $pdata$??$?RV<lambda_886d6c58226a84441f68b9f2b8217b83>@@AEAV<lambda_ab61a845afdef5b7c387490eaf3616ee>@@V<lambda_f7f22ab5edc0698d5f6905b0d3f44752>@@@?$__crt_seh_guarded_call@X@@QEAAX$$QEAV<lambda_886d6c58226a84441f68b9f2b8217b83>@@AEAV<lambda_ab61a845afdef5b7c387490eaf3616ee>@@$$QEAV<lambda_f7f22ab5edc0698d5f6905b0d3f44752>@@@Z 00000001800698d4     libucrt:fflush.obj
 0003:000039f0       $pdata$?fin$0@?0???$?RV<lambda_886d6c58226a84441f68b9f2b8217b83>@@AEAV<lambda_ab61a845afdef5b7c387490eaf3616ee>@@V<lambda_f7f22ab5edc0698d5f6905b0d3f44752>@@@?$__crt_seh_guarded_call@X@@QEAAX$$QEAV<lambda_886d6c58226a84441f68b9f2b8217b83>@@AEAV<lambda_ab61a845afdef5b7c387490eaf3616ee>@@$$QEAV<lambda_f7f22ab5edc0698d5f6905b0d3f44752>@@@Z@4HA 000000018006a9f0     libucrt:fflush.obj
 0003:000028e0       $pdata$??$?RV<lambda_c376a267cfb53b6959b3b692ec76b120>@@AEAV<lambda_9a32fed5bf61b6b509b2d3f6003082a1>@@V<lambda_572fbb9fa0ab338edf41edfd4b5fcc8d>@@@?$__crt_seh_guarded_call@H@@QEAAH$$QEAV<lambda_c376a267cfb53b6959b3b692ec76b120>@@AEAV<lambda_9a32fed5bf61b6b509b2d3f6003082a1>@@$$QEAV<lambda_572fbb9fa0ab338edf41edfd4b5fcc8d>@@@Z 00000001800698e0     libucrt:fflush.obj
 0003:0000291c       $pdata$??$common_fgets@D@@YAPEADQEADHV__crt_stdio_stream@@@Z 000000018006991c     libucrt:fgets.obj
 0003:000039fc       $pdata$?fin$0@?0???$common_fgets@D@@YAPEADQEADHV__crt_stdio_stream@@@Z@4HA 000000018006a9fc     libucrt:fgets.obj
 0003:00002934       $pdata$?common_fseek_binary_mode_read_only_fast_track_nolock@@YA_NV__crt_stdio_stream@@_JH@Z 0000000180069934     libucrt:fseek.obj
 0003:00002940       $pdata$?common_fseek_nolock@@YAHV__crt_stdio_stream@@_JH@Z 0000000180069940     libucrt:fseek.obj
 0003:00002928       $pdata$?common_fseek@@YAHV__crt_stdio_stream@@_JH@Z 0000000180069928     libucrt:fseek.obj
 0003:00002970       $pdata$?common_ftell_translated_utf8_nolock@@YA_JV__crt_stdio_stream@@_J@Z 0000000180069970     libucrt:ftell.obj
 0003:00002964       $pdata$?common_ftell_read_mode_nolock@@YA_JV__crt_stdio_stream@@_J1@Z 0000000180069964     libucrt:ftell.obj
 0003:00002958       $pdata$??$common_ftell_nolock@_J@@YA_JV__crt_stdio_stream@@@Z 0000000180069958     libucrt:ftell.obj
 0003:0000294c       $pdata$??$common_ftell@J@@YAJV__crt_stdio_stream@@@Z 000000018006994c     libucrt:ftell.obj
 0003:000029a0       $pdata$fwrite              00000001800699a0     libucrt:fwrite.obj
 0003:00002994       $pdata$_fwrite_nolock      0000000180069994     libucrt:fwrite.obj
 0003:00002988       $pdata$??R<lambda_96f4279ff90247a4c5c5d9824f56f8c1>@@QEBA_KXZ 0000000180069988     libucrt:fwrite.obj
 0003:0000297c       $pdata$??$?RV<lambda_bdbcead8b570fa3d5ec6d9679862a6e5>@@AEAV<lambda_96f4279ff90247a4c5c5d9824f56f8c1>@@V<lambda_4606be27f17b5e5579e09050fab91818>@@@?$__crt_seh_guarded_call@_K@@QEAA_K$$QEAV<lambda_bdbcead8b570fa3d5ec6d9679862a6e5>@@AEAV<lambda_96f4279ff90247a4c5c5d9824f56f8c1>@@$$QEAV<lambda_4606be27f17b5e5579e09050fab91818>@@@Z 000000018006997c     libucrt:fwrite.obj
 0003:000029c4       $pdata$setvbuf             00000001800699c4     libucrt:setvbuf.obj
 0003:000029b8       $pdata$??R<lambda_ca71763b3c0644891230e4f79ea54fa6>@@QEBAHXZ 00000001800699b8     libucrt:setvbuf.obj
 0003:000029ac       $pdata$??$?RV<lambda_84ec643ea9557e2f7dc01bb0e9624395>@@AEAV<lambda_ca71763b3c0644891230e4f79ea54fa6>@@V<lambda_439a761618c59b0600e24586724d733b>@@@?$__crt_seh_guarded_call@H@@QEAAH$$QEAV<lambda_84ec643ea9557e2f7dc01bb0e9624395>@@AEAV<lambda_ca71763b3c0644891230e4f79ea54fa6>@@$$QEAV<lambda_439a761618c59b0600e24586724d733b>@@@Z 00000001800699ac     libucrt:setvbuf.obj
 0003:00002a18       $pdata$tmpfile             0000000180069a18     libucrt:tmpfile.obj
 0003:00002a0c       $pdata$__acrt_stdio_free_tmpfile_name_buffers_nolock 0000000180069a0c     libucrt:tmpfile.obj
 0003:00002a00       $pdata$?common_tmpfile_nolock@@YAHQEAPEAU_iobuf@@H@Z 0000000180069a00     libucrt:tmpfile.obj
 0003:00003a14       $pdata$?fin$0@?0??common_tmpfile_nolock@@YAHQEAPEAU_iobuf@@H@Z@4HA 000000018006aa14     libucrt:tmpfile.obj
 0003:000029dc       $pdata$??$get_tmpfile_buffer_nolock@D@@YAPEADW4buffer_id@?A0x5b9a7937@@@Z 00000001800699dc     libucrt:tmpfile.obj
 0003:000029e8       $pdata$??$initialize_tmpfile_buffer_nolock@D@@YA_NW4buffer_id@?A0x5b9a7937@@@Z 00000001800699e8     libucrt:tmpfile.obj
 0003:000029d0       $pdata$??$generate_tmpfile_file_name@D@@YA_NQEAD_K@Z 00000001800699d0     libucrt:tmpfile.obj
 0003:000029f4       $pdata$?common_tmpfile@@YAHQEAPEAU_iobuf@@H@Z 00000001800699f4     libucrt:tmpfile.obj
 0003:00003a08       $pdata$?fin$0@?0??common_tmpfile@@YAHQEAPEAU_iobuf@@H@Z@4HA 000000018006aa08     libucrt:tmpfile.obj
 0003:00002c04       $pdata$memcpy_s            0000000180069c04     libucrt:cfout.obj
 0003:00002c04       $pdata$memcpy_s            0000000180069c04     libucrt:input.obj
 0003:00002bf8       $pdata$__stdio_common_vfscanf 0000000180069bf8     libucrt:input.obj
 0003:00002b50       $pdata$?divide@__crt_strtox@@YA_KAEAUbig_integer@1@AEBU21@@Z 0000000180069b50     libucrt:input.obj
 0003:00002b5c       $pdata$5$?divide@__crt_strtox@@YA_KAEAUbig_integer@1@AEBU21@@Z 0000000180069b5c     libucrt:input.obj
 0003:00002b68       $pdata$6$?divide@__crt_strtox@@YA_KAEAUbig_integer@1@AEBU21@@Z 0000000180069b68     libucrt:input.obj
 0003:00002b08       $pdata$?as_double@floating_point_value@__crt_strtox@@QEBAAEANXZ 0000000180069b08     libucrt:input.obj
 0003:00002b14       $pdata$?as_float@floating_point_value@__crt_strtox@@QEBAAEAMXZ 0000000180069b14     libucrt:input.obj
 0003:00002b20       $pdata$?assemble_floating_point_value@__crt_strtox@@YA?AW4SLD_STATUS@@_KH_N1AEBVfloating_point_value@1@@Z 0000000180069b20     libucrt:input.obj
 0003:00002b2c       $pdata$?assemble_floating_point_value_from_big_integer@__crt_strtox@@YA?AW4SLD_STATUS@@AEBUbig_integer@1@I_N1AEBVfloating_point_value@1@@Z 0000000180069b2c     libucrt:input.obj
 0003:00002b38       $pdata$?convert_decimal_string_to_floating_type_common@__crt_strtox@@YA?AW4SLD_STATUS@@AEBUfloating_point_string@1@AEBVfloating_point_value@1@@Z 0000000180069b38     libucrt:input.obj
 0003:00002b44       $pdata$?convert_hexadecimal_string_to_floating_type_common@__crt_strtox@@YA?AW4SLD_STATUS@@AEBUfloating_point_string@1@AEBVfloating_point_value@1@@Z 0000000180069b44     libucrt:input.obj
 0003:00002b74       $pdata$?process@?$input_processor@DV?$stream_input_adapter@D@__crt_stdio_input@@@__crt_stdio_input@@QEAAHXZ 0000000180069b74     libucrt:input.obj
 0003:00002bb0       $pdata$?process_state@?$input_processor@DV?$stream_input_adapter@D@__crt_stdio_input@@@__crt_stdio_input@@AEAA_NXZ 0000000180069bb0     libucrt:input.obj
 0003:00002ba4       $pdata$?process_literal_character_tchar@?$input_processor@DV?$stream_input_adapter@D@__crt_stdio_input@@@__crt_stdio_input@@AEAA_ND@Z 0000000180069ba4     libucrt:input.obj
 0003:00002b80       $pdata$?process_conversion_specifier@?$input_processor@DV?$stream_input_adapter@D@__crt_stdio_input@@@__crt_stdio_input@@AEAA_NXZ 0000000180069b80     libucrt:input.obj
 0003:00002bbc       $pdata$?process_string_specifier@?$input_processor@DV?$stream_input_adapter@D@__crt_stdio_input@@@__crt_stdio_input@@AEAA_NW4conversion_mode@2@@Z 0000000180069bbc     libucrt:input.obj
 0003:00002be0       $pdata$?write_character@?$input_processor@DV?$stream_input_adapter@D@__crt_stdio_input@@@__crt_stdio_input@@AEAA_NQEFA_W_KAEAPEFA_WAEA_KD@Z 0000000180069be0     libucrt:input.obj
 0003:00002b98       $pdata$?process_integer_specifier@?$input_processor@DV?$stream_input_adapter@D@__crt_stdio_input@@@__crt_stdio_input@@AEAA_NI_N@Z 0000000180069b98     libucrt:input.obj
 0003:00002b8c       $pdata$?process_floating_point_specifier@?$input_processor@DV?$stream_input_adapter@D@__crt_stdio_input@@@__crt_stdio_input@@AEAA_NXZ 0000000180069b8c     libucrt:input.obj
 0003:00002bec       $pdata$?write_integer@?$input_processor@DV?$stream_input_adapter@D@__crt_stdio_input@@@__crt_stdio_input@@AEAA_N_K@Z 0000000180069bec     libucrt:input.obj
 0003:00002afc       $pdata$?advance@?$format_string_parser@D@__crt_stdio_input@@QEAA_NXZ 0000000180069afc     libucrt:input.obj
 0003:00002bc8       $pdata$?scan_optional_field_width@?$format_string_parser@D@__crt_stdio_input@@AEAA_NXZ 0000000180069bc8     libucrt:input.obj
 0003:00002bd4       $pdata$?scan_scanset_range@?$format_string_parser@D@__crt_stdio_input@@AEAA_NXZ 0000000180069bd4     libucrt:input.obj
 0003:00002af0       $pdata$??R<lambda_f3caf1ecae5fe01a9a1a6239afa44510>@@QEBAHXZ 0000000180069af0     libucrt:input.obj
 0003:00002ad8       $pdata$??$skip_whitespace@Vstream_input_adapter@__crt_stdio_input@@D@__crt_stdio_input@@YAHAEAV?$stream_input_adapter@D@0@QEAU__crt_locale_pointers@@@Z 0000000180069ad8     libucrt:input.obj
 0003:00002aa8       $pdata$??$process_floating_point_specifier_t@M@?$input_processor@DV?$stream_input_adapter@D@__crt_stdio_input@@@__crt_stdio_input@@AEAA_NXZ 0000000180069aa8     libucrt:input.obj
 0003:00002ab4       $pdata$??$process_floating_point_specifier_t@N@?$input_processor@DV?$stream_input_adapter@D@__crt_stdio_input@@@__crt_stdio_input@@AEAA_NXZ 0000000180069ab4     libucrt:input.obj
 0003:00002a9c       $pdata$??$parse_integer@_KV?$input_adapter_character_source@V?$stream_input_adapter@D@__crt_stdio_input@@@__crt_strtox@@@__crt_strtox@@YA_KQEAU__crt_locale_pointers@@V?$input_adapter_character_source@V?$stream_input_adapter@D@__crt_stdio_input@@@0@H_N@Z 0000000180069a9c     libucrt:input.obj
 0003:00002ac0       $pdata$??$process_string_specifier_tchar@D@?$input_processor@DV?$stream_input_adapter@D@__crt_stdio_input@@@__crt_stdio_input@@AEAA_NW4conversion_mode@1@D@Z 0000000180069ac0     libucrt:input.obj
 0003:00002acc       $pdata$??$process_string_specifier_tchar@_W@?$input_processor@DV?$stream_input_adapter@D@__crt_stdio_input@@@__crt_stdio_input@@AEAA_NW4conversion_mode@1@_W@Z 0000000180069acc     libucrt:input.obj
 0003:00002a24       $pdata$??$?RV<lambda_082dd7c0feb7dbdaf245f261e54a6583>@@AEAV<lambda_f3caf1ecae5fe01a9a1a6239afa44510>@@V<lambda_c640b76c0755ae85b317b35c67c61e6b>@@@?$__crt_seh_guarded_call@H@@QEAAH$$QEAV<lambda_082dd7c0feb7dbdaf245f261e54a6583>@@AEAV<lambda_f3caf1ecae5fe01a9a1a6239afa44510>@@$$QEAV<lambda_c640b76c0755ae85b317b35c67c61e6b>@@@Z 0000000180069a24     libucrt:input.obj
 0003:00002a30       $pdata$??$parse_floating_point@V?$input_adapter_character_source@V?$stream_input_adapter@D@__crt_stdio_input@@@__crt_strtox@@M@__crt_strtox@@YA?AW4SLD_STATUS@@QEAU__crt_locale_pointers@@V?$input_adapter_character_source@V?$stream_input_adapter@D@__crt_stdio_input@@@0@QEAM@Z 0000000180069a30     libucrt:input.obj
 0003:00002a3c       $pdata$??$parse_floating_point@V?$input_adapter_character_source@V?$stream_input_adapter@D@__crt_stdio_input@@@__crt_strtox@@N@__crt_strtox@@YA?AW4SLD_STATUS@@QEAU__crt_locale_pointers@@V?$input_adapter_character_source@V?$stream_input_adapter@D@__crt_stdio_input@@@0@QEAN@Z 0000000180069a3c     libucrt:input.obj
 0003:00002a84       $pdata$??$parse_floating_point_write_result@M@__crt_strtox@@YA?AW4SLD_STATUS@@W4floating_point_parse_result@0@AEBUfloating_point_string@0@QEAM@Z 0000000180069a84     libucrt:input.obj
 0003:00002a90       $pdata$??$parse_floating_point_write_result@N@__crt_strtox@@YA?AW4SLD_STATUS@@W4floating_point_parse_result@0@AEBUfloating_point_string@0@QEAN@Z 0000000180069a90     libucrt:input.obj
 0003:00002a48       $pdata$??$parse_floating_point_from_source@V?$input_adapter_character_source@V?$stream_input_adapter@D@__crt_stdio_input@@@__crt_strtox@@@__crt_strtox@@YA?AW4floating_point_parse_result@0@QEAU__crt_locale_pointers@@AEAV?$input_adapter_character_source@V?$stream_input_adapter@D@__crt_stdio_input@@@0@AEAUfloating_point_string@0@@Z 0000000180069a48     libucrt:input.obj
 0003:00002a54       $pdata$??$parse_floating_point_possible_infinity@DV?$input_adapter_character_source@V?$stream_input_adapter@D@__crt_stdio_input@@@__crt_strtox@@_K@__crt_strtox@@YA?AW4floating_point_parse_result@0@AEADAEAV?$input_adapter_character_source@V?$stream_input_adapter@D@__crt_stdio_input@@@0@_K@Z 0000000180069a54     libucrt:input.obj
 0003:00002a60       $pdata$??$parse_floating_point_possible_nan@DV?$input_adapter_character_source@V?$stream_input_adapter@D@__crt_stdio_input@@@__crt_strtox@@_K@__crt_strtox@@YA?AW4floating_point_parse_result@0@AEADAEAV?$input_adapter_character_source@V?$stream_input_adapter@D@__crt_stdio_input@@@0@_K@Z 0000000180069a60     libucrt:input.obj
 0003:00002ae4       $pdata$??R<lambda_156378f40168adef48d7ddfcff3a1264>@@QEBA_NXZ 0000000180069ae4     libucrt:input.obj
 0003:00002a78       $pdata$??$parse_floating_point_possible_nan_is_snan@DV?$input_adapter_character_source@V?$stream_input_adapter@D@__crt_stdio_input@@@__crt_strtox@@@__crt_strtox@@YA_NAEADAEAV?$input_adapter_character_source@V?$stream_input_adapter@D@__crt_stdio_input@@@0@@Z 0000000180069a78     libucrt:input.obj
 0003:00002a6c       $pdata$??$parse_floating_point_possible_nan_is_ind@DV?$input_adapter_character_source@V?$stream_input_adapter@D@__crt_stdio_input@@@__crt_strtox@@@__crt_strtox@@YA_NAEADAEAV?$input_adapter_character_source@V?$stream_input_adapter@D@__crt_stdio_input@@@0@@Z 0000000180069a6c     libucrt:input.obj
 0003:00002c34       $pdata$_wdupenv_s          0000000180069c34     libucrt:getenv.obj
 0003:00002c1c       $pdata$??$common_getenv@_W@@YAPEA_WQEB_W@Z 0000000180069c1c     libucrt:getenv.obj
 0003:00003a2c       $pdata$?fin$0@?0???$common_getenv@_W@@YAPEA_WQEB_W@Z@4HA 000000018006aa2c     libucrt:getenv.obj
 0003:00002c10       $pdata$??$common_dupenv_s@_W@@YAHQEAPEA_WQEA_KQEB_WHQEBDH@Z 0000000180069c10     libucrt:getenv.obj
 0003:00003a20       $pdata$?fin$0@?0???$common_dupenv_s@_W@@YAHQEAPEA_WQEA_KQEB_WHQEBDH@Z@4HA 000000018006aa20     libucrt:getenv.obj
 0003:00002c28       $pdata$??$common_getenv_nolock@_W@@YAPEA_WQEB_W@Z 0000000180069c28     libucrt:getenv.obj
 0003:00002c40       $pdata$_wsystem            0000000180069c40     libucrt:system.obj
 0003:00002c4c       $pdata$_initterm           0000000180069c4c     libucrt:initterm.obj
 0003:00002c58       $pdata$_initterm_e         0000000180069c58     libucrt:initterm.obj
 0003:00002c64       $pdata$_seh_filter_exe     0000000180069c64     libucrt:exception_filter.obj
 0003:00002ca0       $pdata$?try_cor_exit_process@@YAXI@Z 0000000180069ca0     libucrt:exit.obj
 0003:00002c94       $pdata$?exit_or_terminate_process@@YAXI@Z 0000000180069c94     libucrt:exit.obj
 0003:00002c88       $pdata$?common_exit@@YAXHW4_crt_exit_cleanup_mode@@W4_crt_exit_return_mode@@@Z 0000000180069c88     libucrt:exit.obj
 0003:00002c7c       $pdata$??R<lambda_6e4b09c48022b2350581041d5f6b0c4c>@@QEBA@XZ 0000000180069c7c     libucrt:exit.obj
 0003:00003a44       $pdata$?filt$0@?0???R<lambda_6e4b09c48022b2350581041d5f6b0c4c>@@QEBA@XZ@4HA 000000018006aa44     libucrt:exit.obj
 0003:00002c70       $pdata$??$?RV<lambda_d80eeec6fff315bfe5c115232f3240e3>@@AEAV<lambda_6e4b09c48022b2350581041d5f6b0c4c>@@V<lambda_2358e3775559c9db80273638284d5e45>@@@?$__crt_seh_guarded_call@X@@QEAAX$$QEAV<lambda_d80eeec6fff315bfe5c115232f3240e3>@@AEAV<lambda_6e4b09c48022b2350581041d5f6b0c4c>@@$$QEAV<lambda_2358e3775559c9db80273638284d5e45>@@@Z 0000000180069c70     libucrt:exit.obj
 0003:00003a38       $pdata$?fin$0@?0???$?RV<lambda_450d765d439847d4c735a33c368b5fc0>@@AEAV<lambda_44731a7d0e6d81c3e6aa82d741081786>@@V<lambda_601a2a7da3b7a96e9554ac7215c4b07c>@@@?$__crt_seh_guarded_call@P6AXH@Z@@QEAAP6AXH@Z$$QEAV<lambda_450d765d439847d4c735a33c368b5fc0>@@AEAV<lambda_44731a7d0e6d81c3e6aa82d741081786>@@$$QEAV<lambda_601a2a7da3b7a96e9554ac7215c4b07c>@@@Z@4HA 000000018006aa38     libucrt:signal.obj
 0003:00003a38       $pdata$?fin$0@?0???$?RV<lambda_7777bce6b2f8c936911f934f8298dc43>@@AEAV<lambda_f03950bc5685219e0bcd2087efbe011e>@@V<lambda_3883c3dff614d5e0c5f61bb1ac94921c>@@@?$__crt_seh_guarded_call@H@@QEAAH$$QEAV<lambda_7777bce6b2f8c936911f934f8298dc43>@@AEAV<lambda_f03950bc5685219e0bcd2087efbe011e>@@$$QEAV<lambda_3883c3dff614d5e0c5f61bb1ac94921c>@@@Z@4HA 000000018006aa38     libucrt:onexit.obj
 0003:00003a38       $pdata$?fin$0@?0???$?RV<lambda_2d41944a1d46af3157314b8a01080d33>@@AEAV<lambda_8f455de75cd7d7f24b4096f044d8b9e6>@@V<lambda_aa500f224e6afead328df44964fe2772>@@@?$__crt_seh_guarded_call@X@@QEAAX$$QEAV<lambda_2d41944a1d46af3157314b8a01080d33>@@AEAV<lambda_8f455de75cd7d7f24b4096f044d8b9e6>@@$$QEAV<lambda_aa500f224e6afead328df44964fe2772>@@@Z@4HA 000000018006aa38     libucrt:per_thread_data.obj
 0003:00003a38       $pdata$?fin$0@?0???$?RV<lambda_aa87e3671a710a21b5dc78c0bdf72e11>@@AEAV<lambda_92619d2358a28f41a33ba319515a20b9>@@V<lambda_6992ecaafeb10aed2b74cb1fae11a551>@@@?$__crt_seh_guarded_call@X@@QEAAX$$QEAV<lambda_aa87e3671a710a21b5dc78c0bdf72e11>@@AEAV<lambda_92619d2358a28f41a33ba319515a20b9>@@$$QEAV<lambda_6992ecaafeb10aed2b74cb1fae11a551>@@@Z@4HA 000000018006aa38     libucrt:per_thread_data.obj
 0003:00003a38       $pdata$?fin$0@?0???$?RV<lambda_efdfa57d1f175319df784efa44bb7b81>@@AEAV<lambda_5f0a4c1567f8adc6734073e5d1e1b35c>@@V<lambda_2e8a7d3640ea6ccb4c2413664c2db6fd>@@@?$__crt_seh_guarded_call@X@@QEAAX$$QEAV<lambda_efdfa57d1f175319df784efa44bb7b81>@@AEAV<lambda_5f0a4c1567f8adc6734073e5d1e1b35c>@@$$QEAV<lambda_2e8a7d3640ea6ccb4c2413664c2db6fd>@@@Z@4HA 000000018006aa38     libucrt:mbctype.obj
 0003:00003a38       $pdata$?fin$0@?0???$?RV<lambda_f2e299630e499de9f9a165e60fcd3db5>@@AEAV<lambda_2ae9d31cdba2644fcbeaf08da7c24588>@@V<lambda_40d01ff24d0e7b3814fdbdcee8eab3c7>@@@?$__crt_seh_guarded_call@X@@QEAAX$$QEAV<lambda_f2e299630e499de9f9a165e60fcd3db5>@@AEAV<lambda_2ae9d31cdba2644fcbeaf08da7c24588>@@$$QEAV<lambda_40d01ff24d0e7b3814fdbdcee8eab3c7>@@@Z@4HA 000000018006aa38     libucrt:per_thread_data.obj
 0003:00003a38       $pdata$?fin$0@?0???$?RV<lambda_d80eeec6fff315bfe5c115232f3240e3>@@AEAV<lambda_6e4b09c48022b2350581041d5f6b0c4c>@@V<lambda_2358e3775559c9db80273638284d5e45>@@@?$__crt_seh_guarded_call@X@@QEAAX$$QEAV<lambda_d80eeec6fff315bfe5c115232f3240e3>@@AEAV<lambda_6e4b09c48022b2350581041d5f6b0c4c>@@$$QEAV<lambda_2358e3775559c9db80273638284d5e45>@@@Z@4HA 000000018006aa38     libucrt:exit.obj
 0003:00003a38       $pdata$?fin$0@?0???$?RV<lambda_0ae27a3a962d80f24befdcbee591983d>@@AEAV<lambda_8d0ee55de4b1038c4002e0adecdf1839>@@V<lambda_dc504788e8f1664fe9b84e20bfb512f2>@@@?$__crt_seh_guarded_call@X@@QEAAX$$QEAV<lambda_0ae27a3a962d80f24befdcbee591983d>@@AEAV<lambda_8d0ee55de4b1038c4002e0adecdf1839>@@$$QEAV<lambda_dc504788e8f1664fe9b84e20bfb512f2>@@@Z@4HA 000000018006aa38     libucrt:per_thread_data.obj
 0003:00003a38       $pdata$?fin$0@?0???$?RV<lambda_a22f0c497e5168315e06dae667770027>@@AEAV<lambda_a094494068278ba5130ab06e1292f60a>@@V<lambda_24dc10c13f43218c635520766e23e324>@@@?$__crt_seh_guarded_call@_N@@QEAA_N$$QEAV<lambda_a22f0c497e5168315e06dae667770027>@@AEAV<lambda_a094494068278ba5130ab06e1292f60a>@@$$QEAV<lambda_24dc10c13f43218c635520766e23e324>@@@Z@4HA 000000018006aa38     libucrt:spawnv.obj
 0003:00002cc4       $pdata$_configure_narrow_argv 0000000180069cc4     libucrt:argv_parsing.obj
 0003:00002cb8       $pdata$__acrt_allocate_buffer_for_argv 0000000180069cb8     libucrt:argv_parsing.obj
 0003:00002cac       $pdata$??$parse_command_line@D@@YAXPEADPEAPEAD0PEA_K2@Z 0000000180069cac     libucrt:argv_parsing.obj
 0003:00002d30       $pdata$__dcrt_get_or_create_wide_environment_nolock 0000000180069d30     libucrt:environment_initialization.obj
 0003:00002d3c       $pdata$__dcrt_uninitialize_environments_nolock 0000000180069d3c     libucrt:environment_initialization.obj
 0003:00002cd0       $pdata$??$common_initialize_environment_nolock@D@@YAHXZ 0000000180069cd0     libucrt:environment_initialization.obj
 0003:00002cdc       $pdata$??$common_initialize_environment_nolock@_W@@YAHXZ 0000000180069cdc     libucrt:environment_initialization.obj
 0003:00002d18       $pdata$??$uninitialize_environment_internal@D@@YAXAEAPEAPEAD@Z 0000000180069d18     libucrt:environment_initialization.obj
 0003:00002d24       $pdata$??$uninitialize_environment_internal@_W@@YAXAEAPEAPEA_W@Z 0000000180069d24     libucrt:environment_initialization.obj
 0003:00002d00       $pdata$??$free_environment@D@@YAXQEAPEAD@Z 0000000180069d00     libucrt:environment_initialization.obj
 0003:00002d00       $pdata$??$free_environment@_W@@YAXQEAPEA_W@Z 0000000180069d00     libucrt:environment_initialization.obj
 0003:00002ce8       $pdata$??$create_environment@D@@YAQEAPEADQEAD@Z 0000000180069ce8     libucrt:environment_initialization.obj
 0003:00002cf4       $pdata$??$create_environment@_W@@YAQEAPEA_WQEA_W@Z 0000000180069cf4     libucrt:environment_initialization.obj
 0003:00002d0c       $pdata$??$initialize_environment_by_cloning_nolock@_W@@YAHXZ 0000000180069d0c     libucrt:environment_initialization.obj
 0003:00002d60       $pdata$_execute_onexit_table 0000000180069d60     libucrt:onexit.obj
 0003:00002d54       $pdata$??R<lambda_f03950bc5685219e0bcd2087efbe011e>@@QEBAHXZ 0000000180069d54     libucrt:onexit.obj
 0003:00002d48       $pdata$??$?RV<lambda_7777bce6b2f8c936911f934f8298dc43>@@AEAV<lambda_f03950bc5685219e0bcd2087efbe011e>@@V<lambda_3883c3dff614d5e0c5f61bb1ac94921c>@@@?$__crt_seh_guarded_call@H@@QEAAH$$QEAV<lambda_7777bce6b2f8c936911f934f8298dc43>@@AEAV<lambda_f03950bc5685219e0bcd2087efbe011e>@@$$QEAV<lambda_3883c3dff614d5e0c5f61bb1ac94921c>@@@Z 0000000180069d48     libucrt:onexit.obj
 0003:00002dc0       $pdata$__acrt_uninitialize 0000000180069dc0     libucrt:initialization.obj
 0003:00002dcc       $pdata$__acrt_uninitialize_critical 0000000180069dcc     libucrt:initialization.obj
 0003:00002da8       $pdata$__acrt_thread_attach 0000000180069da8     libucrt:initialization.obj
 0003:00002db4       $pdata$__acrt_thread_detach 0000000180069db4     libucrt:initialization.obj
 0003:00002d6c       $pdata$initialize_c        0000000180069d6c     libucrt:initialization.obj
 0003:00002d78       $pdata$uninitialize_environment 0000000180069d78     libucrt:initialization.obj
 0003:00002d84       $pdata$initialize_pointers 0000000180069d84     libucrt:initialization.obj
 0003:00002d90       $pdata$uninitialize_allocated_memory 0000000180069d90     libucrt:initialization.obj
 0003:00002d9c       $pdata$uninitialize_allocated_io_buffers 0000000180069d9c     libucrt:initialization.obj
 0003:00002dd8       $pdata$terminate           0000000180069dd8     libucrt:terminate.obj
 0003:00002df0       $pdata$_strupr             0000000180069df0     libucrt:strupr.obj
 0003:00002dfc       $pdata$_strupr_s_l         0000000180069dfc     libucrt:strupr.obj
 0003:00002de4       $pdata$?_strupr_s_l_stat@@YAHQEAD_KQEAU__crt_locale_pointers@@@Z 0000000180069de4     libucrt:strupr.obj
 0003:00002e08       $pdata$strcpy_s            0000000180069e08     libucrt:strcpy_s.obj
 0003:00002e14       $pdata$??$parse_integer@KV?$c_string_character_source@D@__crt_strtox@@@__crt_strtox@@YAKQEAU__crt_locale_pointers@@V?$c_string_character_source@D@0@H_N@Z 0000000180069e14     libucrt:atox.obj
 0003:00002e2c       $pdata$??$parse_integer@_KV?$c_string_character_source@D@__crt_strtox@@@__crt_strtox@@YA_KQEAU__crt_locale_pointers@@V?$c_string_character_source@D@0@H_N@Z 0000000180069e2c     libucrt:atox.obj
 0003:00002e20       $pdata$??$parse_integer@KV?$c_string_character_source@_W@__crt_strtox@@@__crt_strtox@@YAKQEAU__crt_locale_pointers@@V?$c_string_character_source@_W@0@H_N@Z 0000000180069e20     libucrt:atox.obj
 0003:00002e38       $pdata$abort               0000000180069e38     libucrt:abort.obj
 0003:00002e5c       $pdata$_invalid_parameter_noinfo 0000000180069e5c     libucrt:invalid_parameter.obj
 0003:00002e68       $pdata$_invoke_watson      0000000180069e68     libucrt:invalid_parameter.obj
 0003:00002e44       $pdata$__acrt_call_reportfault 0000000180069e44     libucrt:invalid_parameter.obj
 0003:00002e50       $pdata$_invalid_parameter  0000000180069e50     libucrt:invalid_parameter.obj
 0003:00002e8c       $pdata$tolower             0000000180069e8c     libucrt:tolower_toupper.obj
 0003:00002e80       $pdata$_tolower_l          0000000180069e80     libucrt:tolower_toupper.obj
 0003:00002e74       $pdata$?internal_isupper_l@@YA_NHQEAU__crt_locale_pointers@@@Z 0000000180069e74     libucrt:tolower_toupper.obj
 0003:00002e98       $pdata$_free_base          0000000180069e98     libucrt:free_base.obj
 0003:00002ea4       $pdata$_malloc_base        0000000180069ea4     libucrt:malloc_base.obj
 0003:00002ec8       $pdata$wcstol              0000000180069ec8     libucrt:strtox.obj
 0003:00002eb0       $pdata$strtol              0000000180069eb0     libucrt:strtox.obj
 0003:00002ebc       $pdata$strtoull            0000000180069ebc     libucrt:strtox.obj
 0003:00002ed4       $pdata$_mbtowc_l           0000000180069ed4     libucrt:mbtowc.obj
 0003:00002eec       $pdata$wctomb_s            0000000180069eec     libucrt:wctomb.obj
 0003:00002ee0       $pdata$_wctomb_s_l         0000000180069ee0     libucrt:wctomb.obj
 0003:00002f88       $pdata$__acrt_initialize_ptd 0000000180069f88     libucrt:per_thread_data.obj
 0003:00002f94       $pdata$__acrt_uninitialize_ptd 0000000180069f94     libucrt:per_thread_data.obj
 0003:00002f64       $pdata$__acrt_getptd       0000000180069f64     libucrt:per_thread_data.obj
 0003:00002f70       $pdata$__acrt_getptd_head  0000000180069f70     libucrt:per_thread_data.obj
 0003:00002f7c       $pdata$__acrt_getptd_noexit 0000000180069f7c     libucrt:per_thread_data.obj
 0003:00002f58       $pdata$__acrt_freeptd      0000000180069f58     libucrt:per_thread_data.obj
 0003:00002f34       $pdata$?destroy_fls@@YAXPEAX@Z 0000000180069f34     libucrt:per_thread_data.obj
 0003:00002f4c       $pdata$?replace_current_thread_locale_nolock@@YAXQEAU__acrt_ptd@@QEAU__crt_locale_data@@@Z 0000000180069f4c     libucrt:per_thread_data.obj
 0003:00002f28       $pdata$?construct_ptd_array@@YAXQEAU__acrt_ptd@@@Z 0000000180069f28     libucrt:per_thread_data.obj
 0003:00002f40       $pdata$?destroy_ptd_array@@YAXQEAU__acrt_ptd@@@Z 0000000180069f40     libucrt:per_thread_data.obj
 0003:00002ef8       $pdata$??$?RV<lambda_0ae27a3a962d80f24befdcbee591983d>@@AEAV<lambda_8d0ee55de4b1038c4002e0adecdf1839>@@V<lambda_dc504788e8f1664fe9b84e20bfb512f2>@@@?$__crt_seh_guarded_call@X@@QEAAX$$QEAV<lambda_0ae27a3a962d80f24befdcbee591983d>@@AEAV<lambda_8d0ee55de4b1038c4002e0adecdf1839>@@$$QEAV<lambda_dc504788e8f1664fe9b84e20bfb512f2>@@@Z 0000000180069ef8     libucrt:per_thread_data.obj
 0003:00002f10       $pdata$??$?RV<lambda_aa87e3671a710a21b5dc78c0bdf72e11>@@AEAV<lambda_92619d2358a28f41a33ba319515a20b9>@@V<lambda_6992ecaafeb10aed2b74cb1fae11a551>@@@?$__crt_seh_guarded_call@X@@QEAAX$$QEAV<lambda_aa87e3671a710a21b5dc78c0bdf72e11>@@AEAV<lambda_92619d2358a28f41a33ba319515a20b9>@@$$QEAV<lambda_6992ecaafeb10aed2b74cb1fae11a551>@@@Z 0000000180069f10     libucrt:per_thread_data.obj
 0003:00002f1c       $pdata$??$?RV<lambda_f2e299630e499de9f9a165e60fcd3db5>@@AEAV<lambda_2ae9d31cdba2644fcbeaf08da7c24588>@@V<lambda_40d01ff24d0e7b3814fdbdcee8eab3c7>@@@?$__crt_seh_guarded_call@X@@QEAAX$$QEAV<lambda_f2e299630e499de9f9a165e60fcd3db5>@@AEAV<lambda_2ae9d31cdba2644fcbeaf08da7c24588>@@$$QEAV<lambda_40d01ff24d0e7b3814fdbdcee8eab3c7>@@@Z 0000000180069f1c     libucrt:per_thread_data.obj
 0003:00002f04       $pdata$??$?RV<lambda_2d41944a1d46af3157314b8a01080d33>@@AEAV<lambda_8f455de75cd7d7f24b4096f044d8b9e6>@@V<lambda_aa500f224e6afead328df44964fe2772>@@@?$__crt_seh_guarded_call@X@@QEAAX$$QEAV<lambda_2d41944a1d46af3157314b8a01080d33>@@AEAV<lambda_8f455de75cd7d7f24b4096f044d8b9e6>@@$$QEAV<lambda_aa500f224e6afead328df44964fe2772>@@@Z 0000000180069f04     libucrt:per_thread_data.obj
 0003:00002fa0       $pdata$__acrt_update_locale_info 0000000180069fa0     libucrt:locale_update.obj
 0003:00002fac       $pdata$__acrt_update_multibyte_info 0000000180069fac     libucrt:locale_update.obj
 0003:00003000       $pdata$__acrt_fp_format    000000018006a000     libucrt:cvt.obj
 0003:00002ff4       $pdata$?fp_format_nan_or_infinity@@YAHW4__acrt_fp_class@@_NPEAD_K1@Z 0000000180069ff4     libucrt:cvt.obj
 0003:00002fd0       $pdata$?fp_format_e_internal@@YAHQEAD_KH_NIQEAU_strflt@@2QEAU__crt_locale_pointers@@@Z 0000000180069fd0     libucrt:cvt.obj
 0003:00002fc4       $pdata$?fp_format_e@@YAHQEBNQEAD_K12H_NIQEAU__crt_locale_pointers@@@Z 0000000180069fc4     libucrt:cvt.obj
 0003:00002fb8       $pdata$?fp_format_a@@YAHQEBNPEAD_KQEAD2H_NIQEAU__crt_locale_pointers@@@Z 0000000180069fb8     libucrt:cvt.obj
 0003:00002fdc       $pdata$?fp_format_f_internal@@YAHQEAD_KHQEAU_strflt@@_NQEAU__crt_locale_pointers@@@Z 0000000180069fdc     libucrt:cvt.obj
 0003:00002fe8       $pdata$?fp_format_g@@YAHQEBNQEAD_K12H_NIQEAU__crt_locale_pointers@@@Z 0000000180069fe8     libucrt:cvt.obj
 0003:0000300c       $pdata$_fileno             000000018006a00c     libucrt:fileno.obj
 0003:00003018       $pdata$__acrt_stdio_begin_temporary_buffering_nolock 000000018006a018     libucrt:_sftbuf.obj
 0003:00003024       $pdata$__acrt_stdio_end_temporary_buffering_nolock 000000018006a024     libucrt:_sftbuf.obj
 0003:0000303c       $pdata$__acrt_uninitialize_locale 000000018006a03c     libucrt:wsetlocale.obj
 0003:00003030       $pdata$??$?RV<lambda_410d79af7f07d98d83a3f525b3859a53>@@AEAV<lambda_3e16ef9562a7dcce91392c22ab16ea36>@@V<lambda_38119f0e861e05405d8a144b9b982f0a>@@@?$__crt_seh_guarded_call@X@@QEAAX$$QEAV<lambda_410d79af7f07d98d83a3f525b3859a53>@@AEAV<lambda_3e16ef9562a7dcce91392c22ab16ea36>@@$$QEAV<lambda_38119f0e861e05405d8a144b9b982f0a>@@@Z 000000018006a030     libucrt:wsetlocale.obj
 0003:00003a50       $pdata$?fin$0@?0???$?RV<lambda_410d79af7f07d98d83a3f525b3859a53>@@AEAV<lambda_3e16ef9562a7dcce91392c22ab16ea36>@@V<lambda_38119f0e861e05405d8a144b9b982f0a>@@@?$__crt_seh_guarded_call@X@@QEAAX$$QEAV<lambda_410d79af7f07d98d83a3f525b3859a53>@@AEAV<lambda_3e16ef9562a7dcce91392c22ab16ea36>@@$$QEAV<lambda_38119f0e861e05405d8a144b9b982f0a>@@@Z@4HA 000000018006aa50     libucrt:wsetlocale.obj
 0003:00003060       $pdata$__acrt_initialize_lowio 000000018006a060     libucrt:ioinit.obj
 0003:00003a5c       $pdata$__acrt_lowio_ensure_fh_exists$fin$0 000000018006aa5c     libucrt:osfinfo.obj
 0003:00003a5c       $pdata$__acrt_initialize_lowio$fin$0 000000018006aa5c     libucrt:ioinit.obj
 0003:00003a5c       $pdata$_alloc_osfhnd$fin$0 000000018006aa5c     libucrt:osfinfo.obj
 0003:0000306c       $pdata$__acrt_uninitialize_lowio 000000018006a06c     libucrt:ioinit.obj
 0003:00003048       $pdata$?initialize_inherited_file_handles_nolock@@YAXXZ 000000018006a048     libucrt:ioinit.obj
 0003:00003054       $pdata$?initialize_stdio_handles_nolock@@YAXXZ 000000018006a054     libucrt:ioinit.obj
 0003:00003078       $pdata$wcscpy_s            000000018006a078     libucrt:wcscpy_s.obj
 0003:00003084       $pdata$?__acrt_stdio_allocate_stream@@YA?AV__crt_stdio_stream@@XZ 000000018006a084     libucrt:stream.obj
 0003:00003a68       $pdata$?fin$0@?0??__acrt_stdio_allocate_stream@@YA?AV__crt_stdio_stream@@XZ@4HA 000000018006aa68     libucrt:stream.obj
 0003:00003a68       $pdata$_fcloseall$fin$0    000000018006aa68     libucrt:closeall.obj
 0003:00003090       $pdata$?find_or_allocate_unused_stream_nolock@@YA?AV__crt_stdio_stream@@XZ 000000018006a090     libucrt:stream.obj
 0003:000030a8       $pdata$_wopenfile          000000018006a0a8     libucrt:openfile.obj
 0003:0000309c       $pdata$??$__acrt_stdio_parse_mode@_W@@YA?AU__acrt_stdio_stream_mode@@QEB_W@Z 000000018006a09c     libucrt:openfile.obj
 0003:000030c0       $pdata$_close              000000018006a0c0     libucrt:close.obj
 0003:000030cc       $pdata$_close_nolock       000000018006a0cc     libucrt:close.obj
 0003:000030b4       $pdata$??$?RV<lambda_751a882b2c74d4b022dec766aa51a29a>@@AEAV<lambda_628dfdc04ba53c8bfc02c9951375f3f5>@@V<lambda_f6c7be5f7998530c34de24c7437d6b54>@@@?$__crt_seh_guarded_call@H@@QEAAH$$QEAV<lambda_751a882b2c74d4b022dec766aa51a29a>@@AEAV<lambda_628dfdc04ba53c8bfc02c9951375f3f5>@@$$QEAV<lambda_f6c7be5f7998530c34de24c7437d6b54>@@@Z 000000018006a0b4     libucrt:close.obj
 0003:00003a74       $pdata$?fin$0@?0???$?RV<lambda_751a882b2c74d4b022dec766aa51a29a>@@AEAV<lambda_628dfdc04ba53c8bfc02c9951375f3f5>@@V<lambda_f6c7be5f7998530c34de24c7437d6b54>@@@?$__crt_seh_guarded_call@H@@QEAAH$$QEAV<lambda_751a882b2c74d4b022dec766aa51a29a>@@AEAV<lambda_628dfdc04ba53c8bfc02c9951375f3f5>@@$$QEAV<lambda_f6c7be5f7998530c34de24c7437d6b54>@@@Z@4HA 000000018006aa74     libucrt:close.obj
 0003:00003a74       $pdata$?fin$0@?0???$?RV<lambda_a37b2b86f63e897a80ea819b0eb08c01>@@AEAV<lambda_38ce7e780aa69e748d6df282ebc68efe>@@V<lambda_99fb1378e971ab6e7edea83e3a7a83a2>@@@?$__crt_seh_guarded_call@H@@QEAAH$$QEAV<lambda_a37b2b86f63e897a80ea819b0eb08c01>@@AEAV<lambda_38ce7e780aa69e748d6df282ebc68efe>@@$$QEAV<lambda_99fb1378e971ab6e7edea83e3a7a83a2>@@@Z@4HA 000000018006aa74     libucrt:commit.obj
 0003:000030d8       $pdata$__acrt_stdio_free_buffer_nolock 000000018006a0d8     libucrt:_freebuf.obj
 0003:000030f0       $pdata$_calloc_base        000000018006a0f0     libucrt:calloc_base.obj
 0003:000030fc       $pdata$strncpy_s           000000018006a0fc     libucrt:strncpy_s.obj
 0003:0000318c       $pdata$__acrt_initialize_winapi_thunks 000000018006a18c     libucrt:winapi_thunks.obj
 0003:00003198       $pdata$__acrt_uninitialize_winapi_thunks 000000018006a198     libucrt:winapi_thunks.obj
 0003:00003120       $pdata$__acrt_AreFileApisANSI 000000018006a120     libucrt:winapi_thunks.obj
 0003:0000312c       $pdata$__acrt_CompareStringEx 000000018006a12c     libucrt:winapi_thunks.obj
 0003:00003138       $pdata$__acrt_FlsAlloc     000000018006a138     libucrt:winapi_thunks.obj
 0003:00003144       $pdata$__acrt_FlsFree      000000018006a144     libucrt:winapi_thunks.obj
 0003:00003150       $pdata$__acrt_FlsGetValue  000000018006a150     libucrt:winapi_thunks.obj
 0003:0000315c       $pdata$__acrt_FlsSetValue  000000018006a15c     libucrt:winapi_thunks.obj
 0003:00003168       $pdata$__acrt_InitializeCriticalSectionEx 000000018006a168     libucrt:winapi_thunks.obj
 0003:00003174       $pdata$__acrt_LCMapStringEx 000000018006a174     libucrt:winapi_thunks.obj
 0003:00003180       $pdata$__acrt_LocaleNameToLCID 000000018006a180     libucrt:winapi_thunks.obj
 0003:00003114       $pdata$__acrt_AppPolicyGetProcessTerminationMethodInternal 000000018006a114     libucrt:winapi_thunks.obj
 0003:00003108       $pdata$?try_get_function@@YAPEAXW4function_id@?A0x391cf84c@@QEBDQEBW4module_id@2@2@Z 000000018006a108     libucrt:winapi_thunks.obj
 0003:000031a4       $pdata$_fcloseall          000000018006a1a4     libucrt:closeall.obj
 0003:000031d4       $pdata$_read               000000018006a1d4     libucrt:read.obj
 0003:00003a80       $pdata$_read$fin$0         000000018006aa80     libucrt:read.obj
 0003:000031e0       $pdata$_read_nolock        000000018006a1e0     libucrt:read.obj
 0003:000031c8       $pdata$?translate_ansi_or_utf8_nolock@@YAHHQEAD_KQEA_W1@Z 000000018006a1c8     libucrt:read.obj
 0003:000031b0       $pdata$??$translate_text_mode_nolock@D@@YAHHQEAD_K@Z 000000018006a1b0     libucrt:read.obj
 0003:000031bc       $pdata$??$translate_text_mode_nolock@_W@@YAHHQEA_W_K@Z 000000018006a1bc     libucrt:read.obj
 0003:000031ec       $pdata$__acrt_stdio_refill_and_read_narrow_nolock 000000018006a1ec     libucrt:_filbuf.obj
 0003:000031f8       $pdata$??$common_lseek@J@@YAJHJH@Z 000000018006a1f8     libucrt:lseek.obj
 0003:00003a8c       $pdata$?fin$0@?0???$common_lseek@_J@@YA_JH_JH@Z@4HA 000000018006aa8c     libucrt:lseek.obj
 0003:00003a8c       $pdata$_write$fin$0        000000018006aa8c     libucrt:write.obj
 0003:00003a8c       $pdata$?fin$0@?0???$common_lseek@J@@YAJHJH@Z@4HA 000000018006aa8c     libucrt:lseek.obj
 0003:00003204       $pdata$??$common_lseek@_J@@YA_JH_JH@Z 000000018006a204     libucrt:lseek.obj
 0003:00003210       $pdata$??$common_lseek_nolock@J@@YAJHJH@Z 000000018006a210     libucrt:lseek.obj
 0003:0000321c       $pdata$??$common_lseek_nolock@_J@@YA_JH_JH@Z 000000018006a21c     libucrt:lseek.obj
 0003:00003228       $pdata$__acrt_stdio_allocate_buffer_nolock 000000018006a228     libucrt:_getbuf.obj
 0003:00003234       $pdata$__pctype_func       000000018006a234     libucrt:ctype.obj
 0003:00003240       $pdata$_isctype_l          000000018006a240     libucrt:isctype.obj
 0003:0000324c       $pdata$_towlower_l         000000018006a24c     libucrt:towlower.obj
 0003:00003258       $pdata$_recalloc_base      000000018006a258     libucrt:recalloc.obj
 0003:00003264       $pdata$wcscat_s            000000018006a264     libucrt:wcscat_s.obj
 0003:00003270       $pdata$_cwait              000000018006a270     libucrt:wait.obj
 0003:0000327c       $pdata$__acrt_wgetpath     000000018006a27c     libucrt:getpath.obj
 0003:00003288       $pdata$__acrt_initialize_locks 000000018006a288     libucrt:locks.obj
 0003:00003294       $pdata$__acrt_uninitialize_locks 000000018006a294     libucrt:locks.obj
 0003:000032a0       $pdata$_waccess_s          000000018006a2a0     libucrt:waccess.obj
 0003:000032ac       $pdata$_pipe               000000018006a2ac     libucrt:pipe.obj
 0003:00003a98       $pdata$_pipe$fin$1         000000018006aa98     libucrt:pipe.obj
 0003:00003aa4       $pdata$_pipe$fin$0         000000018006aaa4     libucrt:pipe.obj
 0003:000032b8       $pdata$??$common_fdopen@_W@@YAPEAU_iobuf@@HQEB_W@Z 000000018006a2b8     libucrt:fdopen.obj
 0003:00003ab0       $pdata$?fin$0@?0???$common_fdopen@_W@@YAPEAU_iobuf@@HQEB_W@Z@4HA 000000018006aab0     libucrt:fdopen.obj
 0003:000032d0       $pdata$_commit             000000018006a2d0     libucrt:commit.obj
 0003:000032c4       $pdata$??$?RV<lambda_a37b2b86f63e897a80ea819b0eb08c01>@@AEAV<lambda_38ce7e780aa69e748d6df282ebc68efe>@@V<lambda_99fb1378e971ab6e7edea83e3a7a83a2>@@@?$__crt_seh_guarded_call@H@@QEAAH$$QEAV<lambda_a37b2b86f63e897a80ea819b0eb08c01>@@AEAV<lambda_38ce7e780aa69e748d6df282ebc68efe>@@$$QEAV<lambda_99fb1378e971ab6e7edea83e3a7a83a2>@@@Z 000000018006a2c4     libucrt:commit.obj
 0003:0000330c       $pdata$_write              000000018006a30c     libucrt:write.obj
 0003:00003318       $pdata$_write_nolock       000000018006a318     libucrt:write.obj
 0003:000032dc       $pdata$?write_double_translated_ansi_nolock@@YA?AUwrite_result@?A0x17268360@@HQEBDI@Z 000000018006a2dc     libucrt:write.obj
 0003:000032e8       $pdata$?write_text_ansi_nolock@@YA?AUwrite_result@?A0x17268360@@HQEBDI@Z 000000018006a2e8     libucrt:write.obj
 0003:000032f4       $pdata$?write_text_utf16le_nolock@@YA?AUwrite_result@?A0x17268360@@HQEBDI@Z 000000018006a2f4     libucrt:write.obj
 0003:00003300       $pdata$?write_text_utf8_nolock@@YA?AUwrite_result@?A0x17268360@@HQEBDI@Z 000000018006a300     libucrt:write.obj
 0003:00003330       $pdata$__acrt_stdio_flush_and_write_narrow_nolock 000000018006a330     libucrt:_flsbuf.obj
 0003:00003324       $pdata$??$write_buffer_nolock@D@@YA_NDV__crt_stdio_stream@@@Z 000000018006a324     libucrt:_flsbuf.obj
 0003:00003354       $pdata$_ui64toa_s          000000018006a354     libucrt:xtoa.obj
 0003:00003348       $pdata$??$common_xtox_s@_KD@@YAH_KQEAD0I_N@Z 000000018006a348     libucrt:xtoa.obj
 0003:0000333c       $pdata$??$common_xtox@_KD@@YAH_KQEAD0I_N@Z 000000018006a33c     libucrt:xtoa.obj
 0003:00003360       $pdata$_strdup             000000018006a360     libucrt:strdup.obj
 0003:0000336c       $pdata$__acrt_GetTempPathA 000000018006a36c     libucrt:gettemppath.obj
 0003:000033d8       $pdata$_wsopen_s           000000018006a3d8     libucrt:open.obj
 0003:000033c0       $pdata$_sopen_s            000000018006a3c0     libucrt:open.obj
 0003:000033b4       $pdata$_sopen_nolock       000000018006a3b4     libucrt:open.obj
 0003:000033cc       $pdata$_wsopen_nolock      000000018006a3cc     libucrt:open.obj
 0003:00003378       $pdata$??$common_sopen_dispatch@D@@YAHQEBDHHHQEAHH@Z 000000018006a378     libucrt:open.obj
 0003:00003abc       $pdata$?fin$0@?0???$common_sopen_dispatch@_W@@YAHQEB_WHHHQEAHH@Z@4HA 000000018006aabc     libucrt:open.obj
 0003:00003abc       $pdata$?fin$0@?0???$common_sopen_dispatch@D@@YAHQEBDHHHQEAHH@Z@4HA 000000018006aabc     libucrt:open.obj
 0003:00003384       $pdata$??$common_sopen_dispatch@_W@@YAHQEB_WHHHQEAHH@Z 000000018006a384     libucrt:open.obj
 0003:0000339c       $pdata$?decode_options@@YA?AUfile_options@?A0xa9d50aae@@HHH@Z 000000018006a39c     libucrt:open.obj
 0003:000033a8       $pdata$?truncate_ctrl_z_if_present@@YAHH@Z 000000018006a3a8     libucrt:open.obj
 0003:00003390       $pdata$?configure_text_mode@@YAHHUfile_options@?A0xa9d50aae@@HAEAW4__crt_lowio_text_mode@@@Z 000000018006a390     libucrt:open.obj
 0003:000033f0       $pdata$_rmtmp              000000018006a3f0     libucrt:rmtmp.obj
 0003:00003ac8       $pdata$_rmtmp$fin$0        000000018006aac8     libucrt:rmtmp.obj
 0003:00003ad4       $pdata$_rmtmp$fin$1        000000018006aad4     libucrt:rmtmp.obj
 0003:000033e4       $pdata$__acrt_uninitialize_tmpfile 000000018006a3e4     libucrt:rmtmp.obj
 0003:000033fc       $pdata$fegetround          000000018006a3fc     libucrt:fegetround.obj
 0003:00003408       $pdata$_wcsnicoll          000000018006a408     libucrt:wcsnicol.obj
 0003:00003414       $pdata$_wcsnicoll_l        000000018006a414     libucrt:wcsnicol.obj
 0003:00003450       $pdata$?accumulate_inheritable_handles@@YA_NQEAPEAEQEA_K_N@Z 000000018006a450     libucrt:spawnv.obj
 0003:00003444       $pdata$??R<lambda_a094494068278ba5130ab06e1292f60a>@@QEBA_NXZ 000000018006a444     libucrt:spawnv.obj
 0003:0000342c       $pdata$??$common_spawnv@_W@@YA_JHQEB_WQEBQEB_W1@Z 000000018006a42c     libucrt:spawnv.obj
 0003:00003420       $pdata$??$?RV<lambda_a22f0c497e5168315e06dae667770027>@@AEAV<lambda_a094494068278ba5130ab06e1292f60a>@@V<lambda_24dc10c13f43218c635520766e23e324>@@@?$__crt_seh_guarded_call@_N@@QEAA_N$$QEAV<lambda_a22f0c497e5168315e06dae667770027>@@AEAV<lambda_a094494068278ba5130ab06e1292f60a>@@$$QEAV<lambda_24dc10c13f43218c635520766e23e324>@@@Z 000000018006a420     libucrt:spawnv.obj
 0003:00003438       $pdata$??$execute_command@_W@@YA_JHQEB_WQEBQEB_W1@Z 000000018006a438     libucrt:spawnv.obj
 0003:0000345c       $pdata$??$common_spawnvp@_W@@YA_JHQEB_WQEBQEB_W1@Z 000000018006a45c     libucrt:spawnvp.obj
 0003:00003468       $pdata$__acrt_get_process_end_policy 000000018006a468     libucrt:win_policies.obj
 0003:00003474       $pdata$??$common_expand_argv_wildcards@D@@YAHQEAPEADQEAPEAPEAD@Z 000000018006a474     libucrt:argv_wildcards.obj
 0003:00003480       $pdata$??$copy_and_add_argument_to_buffer@D@@YAHQEBD0_KAEAV?$argument_list@D@?A0x5f5c8891@@@Z 000000018006a480     libucrt:argv_wildcards.obj
 0003:0000348c       $pdata$??$expand_argument_wildcards@D@@YAHQEAD0AEAV?$argument_list@D@?A0x5f5c8891@@@Z 000000018006a48c     libucrt:argv_wildcards.obj
 0003:000034ec       $pdata$__acrt_update_thread_multibyte_data 000000018006a4ec     libucrt:mbctype.obj
 0003:000034e0       $pdata$__acrt_initialize_multibyte 000000018006a4e0     libucrt:mbctype.obj
 0003:000034f8       $pdata$_setmbcp_nolock     000000018006a4f8     libucrt:mbctype.obj
 0003:000034a4       $pdata$?getSystemCP@@YAHH@Z 000000018006a4a4     libucrt:mbctype.obj
 0003:000034b0       $pdata$?setSBCS@@YAXPEAU__crt_multibyte_data@@@Z 000000018006a4b0     libucrt:mbctype.obj
 0003:000034d4       $pdata$?update_thread_multibyte_data_internal@@YAPEAU__crt_multibyte_data@@QEAU__acrt_ptd@@QEAPEAU1@@Z 000000018006a4d4     libucrt:mbctype.obj
 0003:00003ae0       $pdata$?fin$0@?0??update_thread_multibyte_data_internal@@YAPEAU__crt_multibyte_data@@QEAU__acrt_ptd@@QEAPEAU1@@Z@4HA 000000018006aae0     libucrt:mbctype.obj
 0003:000034c8       $pdata$?setmbcp_internal@@YAHH_NQEAU__acrt_ptd@@QEAPEAU__crt_multibyte_data@@@Z 000000018006a4c8     libucrt:mbctype.obj
 0003:000034bc       $pdata$?setSBUpLow@@YAXPEAU__crt_multibyte_data@@@Z 000000018006a4bc     libucrt:mbctype.obj
 0003:00003498       $pdata$??$?RV<lambda_efdfa57d1f175319df784efa44bb7b81>@@AEAV<lambda_5f0a4c1567f8adc6734073e5d1e1b35c>@@V<lambda_2e8a7d3640ea6ccb4c2413664c2db6fd>@@@?$__crt_seh_guarded_call@X@@QEAAX$$QEAV<lambda_efdfa57d1f175319df784efa44bb7b81>@@AEAV<lambda_5f0a4c1567f8adc6734073e5d1e1b35c>@@$$QEAV<lambda_2e8a7d3640ea6ccb4c2413664c2db6fd>@@@Z 000000018006a498     libucrt:mbctype.obj
 0003:00003504       $pdata$?x_ismbbtype_l@@YAHPEAU__crt_locale_pointers@@IHH@Z 000000018006a504     libucrt:ismbbyte.obj
 0003:00003510       $pdata$__acrt_initialize_command_line 000000018006a510     libucrt:argv_data.obj
 0003:0000351c       $pdata$__dcrt_get_narrow_environment_from_os 000000018006a51c     libucrt:get_environment_from_os.obj
 0003:00003528       $pdata$__dcrt_get_wide_environment_from_os 000000018006a528     libucrt:get_environment_from_os.obj
 0003:00003534       $pdata$??$common_set_variable_in_environment_nolock@_W@@YAHQEA_WH@Z 000000018006a534     libucrt:setenv.obj
 0003:00003540       $pdata$??$copy_environment@_W@@YAPEAPEA_WQEAPEA_W@Z 000000018006a540     libucrt:setenv.obj
 0003:0000354c       $pdata$__acrt_initialize_heap 000000018006a54c     libucrt:heap_handle.obj
 0003:00003558       $pdata$__acrt_execute_initializers 000000018006a558     libucrt:shared_initialization.obj
 0003:00003564       $pdata$__acrt_execute_uninitializers 000000018006a564     libucrt:shared_initialization.obj
 0003:00003570       $pdata$_callnewh           000000018006a570     libucrt:new_handler.obj
 0003:0000357c       $pdata$_query_new_handler  000000018006a57c     libucrt:new_handler.obj
 0003:00003aec       $pdata$_query_new_handler$fin$0 000000018006aaec     libucrt:new_handler.obj
 0003:00003594       $pdata$__acrt_get_sigabrt_handler 000000018006a594     libucrt:signal.obj
 0003:000035a0       $pdata$raise               000000018006a5a0     libucrt:signal.obj
 0003:00003af8       $pdata$raise$fin$0         000000018006aaf8     libucrt:signal.obj
 0003:00003588       $pdata$??$?RV<lambda_450d765d439847d4c735a33c368b5fc0>@@AEAV<lambda_44731a7d0e6d81c3e6aa82d741081786>@@V<lambda_601a2a7da3b7a96e9554ac7215c4b07c>@@@?$__crt_seh_guarded_call@P6AXH@Z@@QEAAP6AXH@Z$$QEAV<lambda_450d765d439847d4c735a33c368b5fc0>@@AEAV<lambda_44731a7d0e6d81c3e6aa82d741081786>@@$$QEAV<lambda_601a2a7da3b7a96e9554ac7215c4b07c>@@@Z 000000018006a588     libucrt:signal.obj
 0003:000035b8       $pdata$__acrt_LCMapStringA 000000018006a5b8     libucrt:lcmapstringa.obj
 0003:000035ac       $pdata$?__acrt_LCMapStringA_stat@@YAHPEAU__crt_locale_pointers@@PEB_WKPEBDHPEADHHH@Z 000000018006a5ac     libucrt:lcmapstringa.obj
 0003:000035c4       $pdata$_isleadbyte_l       000000018006a5c4     libucrt:_wctype.obj
 0003:000035e8       $pdata$__acrt_release_locale_ref 000000018006a5e8     libucrt:locale_refcounting.obj
 0003:000035d0       $pdata$__acrt_free_locale  000000018006a5d0     libucrt:locale_refcounting.obj
 0003:000035dc       $pdata$__acrt_locale_free_lc_time_if_unreferenced 000000018006a5dc     libucrt:locale_refcounting.obj
 0003:000035f4       $pdata$__acrt_update_thread_locale_data 000000018006a5f4     libucrt:locale_refcounting.obj
 0003:00003b04       $pdata$__acrt_update_thread_locale_data$fin$0 000000018006ab04     libucrt:locale_refcounting.obj
 0003:00003600       $pdata$_updatetlocinfoEx_nolock 000000018006a600     libucrt:locale_refcounting.obj
 0003:0000360c       $pdata$__acrt_fp_strflt_to_string 000000018006a60c     libucrt:_fptostr.obj
 0003:00003618       $pdata$__acrt_fltout       000000018006a618     libucrt:cfout.obj
 0003:00003624       $pdata$_isatty             000000018006a624     libucrt:isatty.obj
 0003:00003630       $pdata$__acrt_locale_free_monetary 000000018006a630     libucrt:initmon.obj
 0003:0000363c       $pdata$__acrt_locale_free_numeric 000000018006a63c     libucrt:initnum.obj
 0003:00003654       $pdata$__acrt_locale_free_time 000000018006a654     libucrt:inittime.obj
 0003:00003648       $pdata$?free_crt_array_internal@@YAXQEAPEBX_K@Z 000000018006a648     libucrt:inittime.obj
 0003:00003660       $pdata$__acrt_GetStringTypeA 000000018006a660     libucrt:getstringtypea.obj
 0003:000036b4       $pdata$_get_osfhandle      000000018006a6b4     libucrt:osfinfo.obj
 0003:0000369c       $pdata$_alloc_osfhnd       000000018006a69c     libucrt:osfinfo.obj
 0003:000036a8       $pdata$_free_osfhnd        000000018006a6a8     libucrt:osfinfo.obj
 0003:00003690       $pdata$__acrt_lowio_set_os_handle 000000018006a690     libucrt:osfinfo.obj
 0003:0000366c       $pdata$__acrt_lowio_create_handle_array 000000018006a66c     libucrt:osfinfo.obj
 0003:00003678       $pdata$__acrt_lowio_destroy_handle_array 000000018006a678     libucrt:osfinfo.obj
 0003:00003684       $pdata$__acrt_lowio_ensure_fh_exists 000000018006a684     libucrt:osfinfo.obj
 0003:000036c0       $pdata$_wcsnicmp           000000018006a6c0     libucrt:wcsnicmp.obj
 0003:000036cc       $pdata$_wcsnicmp_l         000000018006a6cc     libucrt:wcsnicmp.obj
 0003:000036e4       $pdata$__acrt_DownlevelLocaleNameToLCID 000000018006a6e4     libucrt:lcidtoname_downlevel.obj
 0003:000036d8       $pdata$?GetTableIndexFromLocaleName@@YAHPEB_W@Z 000000018006a6d8     libucrt:lcidtoname_downlevel.obj
 0003:000036f0       $pdata$__acrt_LCMapStringW 000000018006a6f0     libucrt:lcmapstringw.obj
 0003:000036fc       $pdata$_msize_base         000000018006a6fc     libucrt:msize.obj
 0003:00003708       $pdata$_realloc_base       000000018006a708     libucrt:realloc_base.obj
 0003:00003714       $pdata$__acrt_copy_path_to_wide_string 000000018006a714     libucrt:string_utilities.obj
 0003:00003720       $pdata$_get_fmode          000000018006a720     libucrt:setmode.obj
 0003:0000372c       $pdata$_setmode_nolock     000000018006a72c     libucrt:setmode.obj
 0003:00003738       $pdata$_putwch_nolock      000000018006a738     libucrt:putwch.obj
 0003:00003744       $pdata$_chsize_nolock      000000018006a744     libucrt:chsize.obj
 0003:00003750       $pdata$__acrt_fenv_set_control 000000018006a750     libucrt:_fenvutils.obj
 0003:0000375c       $pdata$__acrt_CompareStringW 000000018006a75c     libucrt:comparestringw.obj
 0003:00003774       $pdata$__acrt_pack_wide_command_line_and_environment 000000018006a774     libucrt:cenvarg.obj
 0003:00003768       $pdata$??$construct_environment_block@_W@@YAHQEBQEB_WQEAPEA_W@Z 000000018006a768     libucrt:cenvarg.obj
 0003:00003780       $pdata$qsort               000000018006a780     libucrt:qsort.obj
 0003:0000378c       $pdata$4$qsort             000000018006a78c     libucrt:qsort.obj
 0003:00003798       $pdata$5$qsort             000000018006a798     libucrt:qsort.obj
 0003:000037a4       $pdata$_mbsdec_l           000000018006a7a4     libucrt:mbsdec.obj
 0003:000037b0       $pdata$?initialize_multibyte@@YAHXZ 000000018006a7b0     libucrt:multibyte_initializer.obj
 0003:000037bc       $pdata$fegetenv            000000018006a7bc     libucrt:fegetenv.obj
 0003:000037c8       $pdata$fesetenv            000000018006a7c8     libucrt:fesetenv.obj
 0003:000037d4       $pdata$feholdexcept        000000018006a7d4     libucrt:feholdexcept.obj
 0003:000037ec       $pdata$__dcrt_lowio_ensure_console_output_initialized 000000018006a7ec     libucrt:initcon.obj
 0003:00003804       $pdata$__dcrt_write_console_w 000000018006a804     libucrt:initcon.obj
 0003:000037f8       $pdata$__dcrt_terminate_console_output 000000018006a7f8     libucrt:initcon.obj
 0003:00003810       $pdata$_call_matherr       000000018006a810     libucrt:libm_error.obj
 0003:0000381c       $pdata$_exception_enabled  000000018006a81c     libucrt:libm_error.obj
 0003:00003828       $pdata$_handle_error       000000018006a828     libucrt:libm_error.obj
 0003:00003834       $pdata$__acrt_initialize_fma3 000000018006a834     libucrt:fma3_available.obj
 0003:0000384c       $pdata$_log_special_common 000000018006a84c     libucrt:log_special.obj
 0003:00003840       $pdata$_log10_special      000000018006a840     libucrt:log_special.obj
 0003:00003870       $pdata$_set_errno_from_matherr 000000018006a870     libucrt:fpexcept.obj
 0003:00003858       $pdata$_raise_exc          000000018006a858     libucrt:fpexcept.obj
 0003:00003864       $pdata$_raise_exc_ex       000000018006a864     libucrt:fpexcept.obj
 0003:0000387c       $pdata$_clrfp              000000018006a87c     libucrt:fpctrl.obj
 0003:00003888       $pdata$_ctrlfp             000000018006a888     libucrt:fpctrl.obj
 0003:000038a0       $pdata$_statfp             000000018006a8a0     libucrt:fpctrl.obj
 0003:00003894       $pdata$_set_statfp         000000018006a894     libucrt:fpctrl.obj
 0003:000038ac       $pdata$_IsNonwritableInCurrentImage 000000018006a8ac     LIBCMT:pesect.obj
 0003:00003b10       $pdata$_IsNonwritableInCurrentImage$filt$0 000000018006ab10     LIBCMT:pesect.obj
 0003:000038c4       $pdata$__GSHandlerCheckCommon 000000018006a8c4     LIBCMT:_gshandler_.obj
 0003:000038b8       $pdata$__GSHandlerCheck    000000018006a8b8     LIBCMT:_gshandler_.obj
 0003:00003900       $pdata$__report_securityfailure 000000018006a900     LIBCMT:gs_report.obj
 0003:000038f4       $pdata$__report_rangecheckfailure 000000018006a8f4     LIBCMT:gs_report.obj
 0003:000038e8       $pdata$__report_gsfailure  000000018006a8e8     LIBCMT:gs_report.obj
 0003:0000390c       $pdata$capture_current_context 000000018006a90c     LIBCMT:gs_report.obj
 0003:00003918       $pdata$capture_previous_context 000000018006a918     LIBCMT:gs_report.obj
 0003:000038dc       $pdata$__raise_securityfailure 000000018006a8dc     LIBCMT:gs_report.obj
 0003:00003924       $pdata$__GSHandlerCheck_SEH 000000018006a924     LIBCMT:_gshandlerseh_.obj
 0004:00001224       .idata$6                   000000018006c224     kernel32:KERNEL32.dll
 0004:00001240       .idata$6                   000000018006c240     user32:USER32.dll
 0004:000012e4       .idata$6                   000000018006c2e4     advapi32:ADVAPI32.dll
 0004:00001316       .idata$6                   000000018006c316     shell32:SHELL32.dll
 0004:000018ae       .idata$6                   000000018006c8ae     lua51:lua51.dll
 0004:000018fa       .idata$6                   000000018006c8fa     rpcrt4:RPCRT4.dll
 0005:00000060       $R000000                   000000018006d060     luafar3.res
